 fontmanager

 Timestamp is 98509204 (reproducible build file hash)

 Preferred load address is 0000000180000000

 Start         Length     Name                   Class
 0001:00000000 00089c70H .text$mn                CODE
 0001:00089c70 00000036H .text$mn$00             CODE
 0001:00089ca6 00000092H .text$x                 CODE
 0002:00000000 00000460H .idata$5                DATA
 0002:00000460 00000038H .00cfg                  DATA
 0002:00000498 00000008H .CRT$XCA                DATA
 0002:000004a0 00000008H .CRT$XCZ                DATA
 0002:000004a8 00000008H .CRT$XIA                DATA
 0002:000004b0 00000008H .CRT$XIZ                DATA
 0002:000004b8 00000008H .CRT$XPA                DATA
 0002:000004c0 00000008H .CRT$XPZ                DATA
 0002:000004c8 00000008H .CRT$XTA                DATA
 0002:000004d0 00000010H .CRT$XTZ                DATA
 0002:000004d8 00000000H .gehcont$y              DATA
 0002:000004d8 00000000H .gfids$y                DATA
 0002:000004e0 0002f520H .rdata                  DATA
 0002:0002fa00 00000000H .rdata$CastGuardVftablesA DATA
 0002:0002fa00 00000000H .rdata$CastGuardVftablesC DATA
 0002:0002fa00 00000980H .rdata$voltmd           DATA
 0002:00030380 000002c8H .rdata$zzzdbg           DATA
 0002:00030648 00000008H .rtc$IAA                DATA
 0002:00030650 00000008H .rtc$IZZ                DATA
 0002:00030658 00000008H .rtc$TAA                DATA
 0002:00030660 00000008H .rtc$TZZ                DATA
 0002:00030668 000083d8H .xdata                  DATA
 0002:00038a40 000008ccH .edata                  DATA
 0002:0003930c 0000012cH .idata$2                DATA
 0002:00039438 00000018H .idata$3                DATA
 0002:00039450 00000460H .idata$4                DATA
 0002:000398b0 00000a60H .idata$6                DATA
 0003:00000000 00000b60H .data                   DATA
 0003:00000b60 00001720H .bss                    DATA
 0004:00000000 0000675cH .pdata                  DATA
 0005:00000000 00000030H _RDATA                  DATA
 0006:00000000 00000060H .rsrc$01                DATA
 0006:00000060 00000338H .rsrc$02                DATA

  Address         Publics by Value              Rva+Base               Lib:Object

 0000:00000000       __AbsoluteZero             0000000000000000     <absolute>
 0000:00000000       ___safe_se_handler_count   0000000000000000     <absolute>
 0000:00000000       ___safe_se_handler_table   0000000000000000     <absolute>
 0000:00000000       __arm64x_extra_rfe_table   0000000000000000     <absolute>
 0000:00000000       __arm64x_extra_rfe_table_size 0000000000000000     <absolute>
 0000:00000000       __arm64x_native_entrypoint 0000000000000000     <absolute>
 0000:00000000       __arm64x_redirection_metadata 0000000000000000     <absolute>
 0000:00000000       __arm64x_redirection_metadata_count 0000000000000000     <absolute>
 0000:00000000       __dynamic_value_reloc_table 0000000000000000     <absolute>
 0000:00000000       __enclave_config           0000000000000000     <absolute>
 0000:00000000       __guard_check_icall_a64n_fptr 0000000000000000     <absolute>
 0000:00000000       __guard_eh_cont_count      0000000000000000     <absolute>
 0000:00000000       __guard_eh_cont_table      0000000000000000     <absolute>
 0000:00000000       __guard_fids_count         0000000000000000     <absolute>
 0000:00000000       __guard_fids_table         0000000000000000     <absolute>
 0000:00000000       __guard_iat_count          0000000000000000     <absolute>
 0000:00000000       __guard_iat_table          0000000000000000     <absolute>
 0000:00000000       __guard_longjmp_count      0000000000000000     <absolute>
 0000:00000000       __guard_longjmp_table      0000000000000000     <absolute>
 0000:00000000       __hybrid_auxiliary_delayload_iat 0000000000000000     <absolute>
 0000:00000000       __hybrid_auxiliary_delayload_iat_copy 0000000000000000     <absolute>
 0000:00000000       __hybrid_auxiliary_iat     0000000000000000     <absolute>
 0000:00000000       __hybrid_auxiliary_iat_copy 0000000000000000     <absolute>
 0000:00000000       __hybrid_code_map          0000000000000000     <absolute>
 0000:00000000       __hybrid_code_map_count    0000000000000000     <absolute>
 0000:00000000       __hybrid_image_info_bitfield 0000000000000000     <absolute>
 0000:00000000       __x64_code_ranges_to_entry_points 0000000000000000     <absolute>
 0000:00000000       __x64_code_ranges_to_entry_points_count 0000000000000000     <absolute>
 0000:00000100       __guard_flags              0000000000000100     <absolute>
 0000:00000000       __ImageBase                0000000180000000     <linker-defined>
 0001:000000b0       Java_sun_font_ColorGlyphSurfaceData_initOps 00000001800010b0 f   ColorGlyphSurfaceData.obj
 0001:00000100       Java_sun_font_ColorGlyphSurfaceData_setCurrentGlyph 0000000180001100 f   ColorGlyphSurfaceData.obj
 0001:00000120       Java_sun_java2d_loops_DrawGlyphListAA_DrawGlyphListAA 0000000180001120 f   DrawGlyphList.obj
 0001:00000120       Java_sun_java2d_loops_DrawGlyphList_DrawGlyphList 0000000180001120 f   DrawGlyphList.obj
 0001:00000200       Java_sun_java2d_loops_DrawGlyphListLCD_DrawGlyphListLCD 0000000180001200 f   DrawGlyphList.obj
 0001:00000320       RefineBounds               0000000180001320 f   DrawGlyphList.obj
 0001:000008c0       initLCDGammaTables         00000001800018c0 f   DrawGlyphList.obj
 0001:00000910       initLUT                    0000000180001910 f   DrawGlyphList.obj
 0001:00000ab0       setupBlitVector            0000000180001ab0 f   DrawGlyphList.obj
 0001:00000ed0       setupLCDBlitVector         0000000180001ed0 f   DrawGlyphList.obj
 0001:00001510       Java_sun_font_SunLayoutEngine_shape 0000000180002510 f   HBShaper.obj
 0001:00001970       storeGVData                0000000180002970 f   HBShaper.obj
 0001:00002790       Java_sun_awt_Win32FontManager_getFontPath 0000000180003790 f   fontpath.obj
 0001:00002ac0       Java_sun_awt_Win32FontManager_populateFontFileNameMap0 0000000180003ac0 f   fontpath.obj
 0001:00003750       Java_sun_font_FreetypeFontScaler_createScalerContextNative 0000000180004750 f   freetypeScaler.obj
 0001:00003960       Java_sun_font_FreetypeFontScaler_disposeNativeScaler 0000000180004960 f   freetypeScaler.obj
 0001:000039d0       Java_sun_font_FreetypeFontScaler_getFontMetricsNative 00000001800049d0 f   freetypeScaler.obj
 0001:00003dc0       Java_sun_font_FreetypeFontScaler_getGlyphAdvanceNative 0000000180004dc0 f   freetypeScaler.obj
 0001:00003e20       Java_sun_font_FreetypeFontScaler_getGlyphCodeNative 0000000180004e20 f   freetypeScaler.obj
 0001:00003ed0       Java_sun_font_FreetypeFontScaler_getGlyphImageNative 0000000180004ed0 f   freetypeScaler.obj
 0001:00003f00       Java_sun_font_FreetypeFontScaler_getGlyphMetricsNative 0000000180004f00 f   freetypeScaler.obj
 0001:00003fc0       Java_sun_font_FreetypeFontScaler_getGlyphOutlineBoundsNative 0000000180004fc0 f   freetypeScaler.obj
 0001:00004120       Java_sun_font_FreetypeFontScaler_getGlyphOutlineNative 0000000180005120 f   freetypeScaler.obj
 0001:00004190       Java_sun_font_FreetypeFontScaler_getGlyphPointNative 0000000180005190 f   freetypeScaler.obj
 0001:00004260       Java_sun_font_FreetypeFontScaler_getGlyphVectorOutlineNative 0000000180005260 f   freetypeScaler.obj
 0001:00004560       Java_sun_font_FreetypeFontScaler_getMissingGlyphCodeNative 0000000180005560 f   freetypeScaler.obj
 0001:00004560       __scrt_stub_for_is_c_termination_complete 0000000180005560 f   MSVCRT:ucrt_stubs.obj
 0001:00004560       _is_c_termination_complete 0000000180005560 f   MSVCRT:ucrt_stubs.obj
 0001:00004570       Java_sun_font_FreetypeFontScaler_getNumGlyphsNative 0000000180005570 f   freetypeScaler.obj
 0001:00004620       Java_sun_font_FreetypeFontScaler_getUnitsPerEMNative 0000000180005620 f   freetypeScaler.obj
 0001:00004640       Java_sun_font_FreetypeFontScaler_initIDs 0000000180005640 f   freetypeScaler.obj
 0001:000046a0       Java_sun_font_FreetypeFontScaler_initNativeScaler 00000001800056a0 f   freetypeScaler.obj
 0001:00005550       ?fini@hb_user_data_array_t@@QEAAXXZ 0000000180006550 f i gsubgpos-context.obj
 0001:00005660       ?hb_ot_layout_position_finish_advances@@YAXPEAUhb_font_t@@PEAUhb_buffer_t@@@Z 0000000180006660 f   hb-ot-layout.obj
 0001:00005660       _guard_check_icall_nop     0000000180006660 f   MSVCRT:guard_support.obj
 0001:00005660       _hb_fallback_shaper_face_data_destroy 0000000180006660 f   hb-fallback-shape.obj
 0001:00005660       _hb_fallback_shaper_font_data_destroy 0000000180006660 f   hb-fallback-shape.obj
 0001:00005660       _hb_ot_shaper_face_data_destroy 0000000180006660 f   hb-ot-shape.obj
 0001:00005660       _hb_ot_shaper_font_data_destroy 0000000180006660 f   hb-ot-shape.obj
 0001:00005670       ??$check_range@U?$IntType@E$00@OT@@@hb_sanitize_context_t@@QEBA_NPEBU?$IntType@E$00@OT@@II@Z 0000000180006670 f i hb-aat-layout.obj
 0001:000056b0       ??$dispatch@UCoverage@Common@Layout@OT@@$$V@hb_sanitize_context_t@@QEAA_NAEBUCoverage@Common@Layout@OT@@@Z 00000001800066b0 f i hb-aat-layout.obj
 0001:00005770       ??$dispatch@Uhb_aat_apply_context_t@AAT@@$$V@?$ChainSubtable@UExtendedTypes@AAT@@@AAT@@QEBA_NPEAUhb_aat_apply_context_t@1@@Z 0000000180006770 f i hb-aat-layout.obj
 0001:00005a80       ??$dispatch@Uhb_aat_apply_context_t@AAT@@$$V@?$ChainSubtable@UObsoleteTypes@AAT@@@AAT@@QEBA_NPEAUhb_aat_apply_context_t@1@@Z 0000000180006a80 f i hb-aat-layout.obj
 0001:00005d10       ??$dispatch@Uhb_aat_apply_context_t@AAT@@$$V@KerxSubTable@AAT@@QEBA_NPEAUhb_aat_apply_context_t@1@@Z 0000000180006d10 f i hb-aat-layout.obj
 0001:00005fc0       ??$dispatch@Uhb_sanitize_context_t@@$$V@?$ChainSubtable@UExtendedTypes@AAT@@@AAT@@QEBA_NPEAUhb_sanitize_context_t@@@Z 0000000180006fc0 f i hb-aat-layout.obj
 0001:00006260       ??$dispatch@Uhb_sanitize_context_t@@$$V@?$ChainSubtable@UObsoleteTypes@AAT@@@AAT@@QEBA_NPEAUhb_sanitize_context_t@@@Z 0000000180007260 f i hb-aat-layout.obj
 0001:00006410       ??$dispatch@Uhb_sanitize_context_t@@$$V@KerxSubTable@AAT@@QEBA_NPEAUhb_sanitize_context_t@@@Z 0000000180007410 f i hb-aat-layout.obj
 0001:00006590       ??$drive@Udriver_context_t@?$ContextualSubtable@UExtendedTypes@AAT@@@AAT@@@?$StateTableDriver@UExtendedTypes@AAT@@UEntryData@?$ContextualSubtable@UExtendedTypes@AAT@@@2@@AAT@@QEAAXPEAUdriver_context_t@?$ContextualSubtable@UExtendedTypes@AAT@@@1@PEAUhb_aat_apply_context_t@1@@Z 0000000180007590 f i hb-aat-layout.obj
 0001:00006a70       ??$drive@Udriver_context_t@?$ContextualSubtable@UObsoleteTypes@AAT@@@AAT@@@?$StateTableDriver@UObsoleteTypes@AAT@@UEntryData@?$ContextualSubtable@UObsoleteTypes@AAT@@@2@@AAT@@QEAAXPEAUdriver_context_t@?$ContextualSubtable@UObsoleteTypes@AAT@@@1@PEAUhb_aat_apply_context_t@1@@Z 0000000180007a70 f i hb-aat-layout.obj
 0001:00007100       ??$drive@Udriver_context_t@?$InsertionSubtable@UExtendedTypes@AAT@@@AAT@@@?$StateTableDriver@UExtendedTypes@AAT@@UEntryData@?$InsertionSubtable@UExtendedTypes@AAT@@@2@@AAT@@QEAAXPEAUdriver_context_t@?$InsertionSubtable@UExtendedTypes@AAT@@@1@PEAUhb_aat_apply_context_t@1@@Z 0000000180008100 f i hb-aat-layout.obj
 0001:000075f0       ??$drive@Udriver_context_t@?$InsertionSubtable@UObsoleteTypes@AAT@@@AAT@@@?$StateTableDriver@UObsoleteTypes@AAT@@UEntryData@?$InsertionSubtable@UObsoleteTypes@AAT@@@2@@AAT@@QEAAXPEAUdriver_context_t@?$InsertionSubtable@UObsoleteTypes@AAT@@@1@PEAUhb_aat_apply_context_t@1@@Z 00000001800085f0 f i hb-aat-layout.obj
 0001:00007ab0       ??$drive@Udriver_context_t@?$KerxSubTableFormat1@UKerxSubTableHeader@AAT@@@AAT@@@?$StateTableDriver@UExtendedTypes@AAT@@UEntryData@?$Format1Entry@$00@2@@AAT@@QEAAXPEAUdriver_context_t@?$KerxSubTableFormat1@UKerxSubTableHeader@AAT@@@1@PEAUhb_aat_apply_context_t@1@@Z 0000000180008ab0 f i hb-aat-layout.obj
 0001:00007ef0       ??$drive@Udriver_context_t@?$KerxSubTableFormat4@UKerxSubTableHeader@AAT@@@AAT@@@?$StateTableDriver@UExtendedTypes@AAT@@UEntryData@?$KerxSubTableFormat4@UKerxSubTableHeader@AAT@@@2@@AAT@@QEAAXPEAUdriver_context_t@?$KerxSubTableFormat4@UKerxSubTableHeader@AAT@@@1@PEAUhb_aat_apply_context_t@1@@Z 0000000180008ef0 f i hb-aat-layout.obj
 0001:00008330       ??$drive@Udriver_context_t@?$LigatureSubtable@UExtendedTypes@AAT@@@AAT@@@?$StateTableDriver@UExtendedTypes@AAT@@UEntryData@?$LigatureEntry@$00@2@@AAT@@QEAAXPEAUdriver_context_t@?$LigatureSubtable@UExtendedTypes@AAT@@@1@PEAUhb_aat_apply_context_t@1@@Z 0000000180009330 f i hb-aat-layout.obj
 0001:00008750       ??$drive@Udriver_context_t@?$LigatureSubtable@UObsoleteTypes@AAT@@@AAT@@@?$StateTableDriver@UObsoleteTypes@AAT@@X@AAT@@QEAAXPEAUdriver_context_t@?$LigatureSubtable@UObsoleteTypes@AAT@@@1@PEAUhb_aat_apply_context_t@1@@Z 0000000180009750 f i hb-aat-layout.obj
 0001:00008b40       ??$drive@Udriver_context_t@?$RearrangementSubtable@UExtendedTypes@AAT@@@AAT@@@?$StateTableDriver@UExtendedTypes@AAT@@X@AAT@@QEAAXPEAUdriver_context_t@?$RearrangementSubtable@UExtendedTypes@AAT@@@1@PEAUhb_aat_apply_context_t@1@@Z 0000000180009b40 f i hb-aat-layout.obj
 0001:00008f40       ??$drive@Udriver_context_t@?$RearrangementSubtable@UObsoleteTypes@AAT@@@AAT@@@?$StateTableDriver@UObsoleteTypes@AAT@@X@AAT@@QEAAXPEAUdriver_context_t@?$RearrangementSubtable@UObsoleteTypes@AAT@@@1@PEAUhb_aat_apply_context_t@1@@Z 0000000180009f40 f i hb-aat-layout.obj
 0001:000092e0       ??$replace_glyphs@UHBGlyphID16@OT@@@hb_buffer_t@@QEAA_NIIPEBUHBGlyphID16@OT@@@Z 000000018000a2e0 f i hb-aat-layout.obj
 0001:000093c0       ??$sanitize@$$V@?$ArrayOf@U?$IntType@G$01@OT@@U12@@OT@@QEBA_NPEAUhb_sanitize_context_t@@@Z 000000018000a3c0 f i hb-aat-layout.obj
 0001:000093c0       ??$sanitize@$$V@?$ArrayOf@UHBGlyphID16@OT@@U?$IntType@G$01@2@@OT@@QEBA_NPEAUhb_sanitize_context_t@@@Z 000000018000a3c0 f i hb-aat-layout.obj
 0001:000093c0       ??$sanitize@$$V@?$ArrayOf@UIndex@OT@@U?$IntType@G$01@2@@OT@@QEBA_NPEAUhb_sanitize_context_t@@@Z 000000018000a3c0 f i hb-ot-layout.obj
 0001:00009430       ??$sanitize@$$V@?$OffsetTo@U?$ArrayOf@UAnchor@AAT@@U?$IntType@I$03@OT@@@OT@@U?$IntType@G$01@2@$0A@@OT@@QEBA_NPEAUhb_sanitize_context_t@@PEBX@Z 000000018000a430 f i hb-aat-layout.obj
 0001:000094f0       ??$sanitize@$$V@?$OffsetTo@U?$ClassTable@U?$IntType@E$00@OT@@@AAT@@U?$IntType@G$01@OT@@$0A@@OT@@QEBA_NPEAUhb_sanitize_context_t@@PEBX@Z 000000018000a4f0 f i hb-aat-layout.obj
 0001:000095b0       ??$sanitize@$$V@?$OffsetTo@U?$Lookup@U?$IntType@G$01@OT@@@AAT@@U?$IntType@I$03@OT@@$0A@@OT@@QEBA_NPEAUhb_sanitize_context_t@@PEBX@Z 000000018000a5b0 f i hb-aat-layout.obj
 0001:00009640       ??$sanitize@$$V@?$OffsetTo@U?$Lookup@U?$IntType@I$03@OT@@@AAT@@U?$IntType@I$03@OT@@$0A@@OT@@QEBA_NPEAUhb_sanitize_context_t@@PEBX@Z 000000018000a640 f i hb-aat-layout.obj
 0001:000096d0       ??$sanitize@$$V@?$OffsetTo@UAttachList@OT@@U?$IntType@G$01@2@$00@OT@@QEBA_NPEAUhb_sanitize_context_t@@PEBX@Z 000000018000a6d0 f i hb-aat-layout.obj
 0001:000098c0       ??$sanitize@$$V@?$OffsetTo@UClassDef@OT@@U?$IntType@G$01@2@$00@OT@@QEBA_NPEAUhb_sanitize_context_t@@PEBX@Z 000000018000a8c0 f i hb-aat-layout.obj
 0001:00009a00       ??$sanitize@$$V@?$OffsetTo@UCoverage@Common@Layout@OT@@U?$IntType@G$01@4@$00@OT@@QEBA_NPEAUhb_sanitize_context_t@@PEBX@Z 000000018000aa00 f i hb-aat-layout.obj
 0001:00009ab0       ??$sanitize@$$V@?$OffsetTo@UDevice@OT@@U?$IntType@G$01@2@$00@OT@@QEBA_NPEAUhb_sanitize_context_t@@PEBX@Z 000000018000aab0 f i hb-aat-layout.obj
 0001:00009be0       ??$sanitize@$$V@?$OffsetTo@ULigCaretList@OT@@U?$IntType@G$01@2@$00@OT@@QEBA_NPEAUhb_sanitize_context_t@@PEBX@Z 000000018000abe0 f i hb-aat-layout.obj
 0001:00009da0       ??$sanitize@$$V@?$OffsetTo@UVarData@OT@@U?$IntType@I$03@2@$00@OT@@QEBA_NPEAUhb_sanitize_context_t@@PEBX@Z 000000018000ada0 f i hb-aat-layout.obj
 0001:00009f10       ??$sanitize@$$V@?$OffsetTo@UVariationStore@OT@@U?$IntType@I$03@2@$00@OT@@QEBA_NPEAUhb_sanitize_context_t@@PEBX@Z 000000018000af10 f i hb-aat-layout.obj
 0001:00009fc0       ??$sanitize@$$V@?$UnsizedListOfOffset16To@U?$Lookup@UHBGlyphID16@OT@@@AAT@@U?$IntType@G$01@OT@@$0A@@OT@@QEBA_NPEAUhb_sanitize_context_t@@I@Z 000000018000afc0 f i hb-aat-layout.obj
 0001:0000a090       ??$sanitize@$$V@?$UnsizedListOfOffset16To@U?$Lookup@UHBGlyphID16@OT@@@AAT@@U?$IntType@I$03@OT@@$0A@@OT@@QEBA_NPEAUhb_sanitize_context_t@@I@Z 000000018000b090 f i hb-aat-layout.obj
 0001:0000a170       ??$sanitize@AEAPEBX@?$UnsizedArrayOf@U?$OffsetTo@U?$ArrayOf@UAnchor@AAT@@U?$IntType@I$03@OT@@@OT@@U?$IntType@G$01@2@$0A@@OT@@@OT@@QEBA_NPEAUhb_sanitize_context_t@@IAEAPEBX@Z 000000018000b170 f i hb-aat-layout.obj
 0001:0000a200       ??$sanitize@PEBU?$LookupFormat4@U?$IntType@G$01@OT@@@AAT@@@?$VarSizedBinSearchArrayOf@U?$LookupSegmentArray@U?$IntType@G$01@OT@@@AAT@@@OT@@QEBA_NPEAUhb_sanitize_context_t@@$$QEAPEBU?$LookupFormat4@U?$IntType@G$01@OT@@@AAT@@@Z 000000018000b200 f i hb-aat-layout.obj
 0001:0000a200       ??$sanitize@PEBU?$LookupFormat4@UHBGlyphID16@OT@@@AAT@@@?$VarSizedBinSearchArrayOf@U?$LookupSegmentArray@UHBGlyphID16@OT@@@AAT@@@OT@@QEBA_NPEAUhb_sanitize_context_t@@$$QEAPEBU?$LookupFormat4@UHBGlyphID16@OT@@@AAT@@@Z 000000018000b200 f i hb-aat-layout.obj
 0001:0000a3c0       ??$sanitize@PEBU?$LookupFormat4@U?$IntType@I$03@OT@@@AAT@@@?$VarSizedBinSearchArrayOf@U?$LookupSegmentArray@U?$IntType@I$03@OT@@@AAT@@@OT@@QEBA_NPEAUhb_sanitize_context_t@@$$QEAPEBU?$LookupFormat4@U?$IntType@I$03@OT@@@AAT@@@Z 000000018000b3c0 f i hb-aat-layout.obj
 0001:0000a580       ??$sanitize@PEBU?$LookupFormat4@U?$OffsetTo@U?$ArrayOf@UAnchor@AAT@@U?$IntType@I$03@OT@@@OT@@U?$IntType@G$01@2@$0A@@OT@@@AAT@@AEAPEBX@?$VarSizedBinSearchArrayOf@U?$LookupSegmentArray@U?$OffsetTo@U?$ArrayOf@UAnchor@AAT@@U?$IntType@I$03@OT@@@OT@@U?$IntType@G$01@2@$0A@@OT@@@AAT@@@OT@@QEBA_NPEAUhb_sanitize_context_t@@$$QEAPEBU?$LookupFormat4@U?$OffsetTo@U?$ArrayOf@UAnchor@AAT@@U?$IntType@I$03@OT@@@OT@@U?$IntType@G$01@2@$0A@@OT@@@AAT@@AEAPEBX@Z 000000018000b580 f i hb-aat-layout.obj
 0001:0000a770       ??$sanitize@PEBULigGlyph@OT@@@?$ArrayOf@U?$OffsetTo@UCaretValue@OT@@U?$IntType@G$01@2@$00@OT@@U?$IntType@G$01@2@@OT@@QEBA_NPEAUhb_sanitize_context_t@@$$QEAPEBULigGlyph@1@@Z 000000018000b770 f i hb-aat-layout.obj
 0001:0000a920       ??$sanitize_blob@UGDEF@OT@@@hb_sanitize_context_t@@QEAAPEAUhb_blob_t@@PEAU1@@Z 000000018000b920 f i hb-aat-layout.obj
 0001:0000ac30       ??$sanitize_blob@Uankr@AAT@@@hb_sanitize_context_t@@QEAAPEAUhb_blob_t@@PEAU1@@Z 000000018000bc30 f i hb-aat-layout.obj
 0001:0000b060       ??$sanitize_blob@Ufeat@AAT@@@hb_sanitize_context_t@@QEAAPEAUhb_blob_t@@PEAU1@@Z 000000018000c060 f i hb-aat-layout.obj
 0001:0000b3e0       ??$sanitize_blob@Ukerx@AAT@@@hb_sanitize_context_t@@QEAAPEAUhb_blob_t@@PEAU1@@Z 000000018000c3e0 f i hb-aat-layout.obj
 0001:0000b570       ??$sanitize_blob@Ultag@AAT@@@hb_sanitize_context_t@@QEAAPEAUhb_blob_t@@PEAU1@@Z 000000018000c570 f i hb-aat-layout.obj
 0001:0000b9a0       ??$sanitize_blob@Umort@AAT@@@hb_sanitize_context_t@@QEAAPEAUhb_blob_t@@PEAU1@@Z 000000018000c9a0 f i hb-aat-layout.obj
 0001:0000bb30       ??$sanitize_blob@Umorx@AAT@@@hb_sanitize_context_t@@QEAAPEAUhb_blob_t@@PEAU1@@Z 000000018000cb30 f i hb-aat-layout.obj
 0001:0000be80       ??$sanitize_blob@Utrak@AAT@@@hb_sanitize_context_t@@QEAAPEAUhb_blob_t@@PEAU1@@Z 000000018000ce80 f i hb-aat-layout.obj
 0001:0000c3b0       ??0hb_aat_apply_context_t@AAT@@QEAA@PEBUhb_ot_shape_plan_t@@PEAUhb_font_t@@PEAUhb_buffer_t@@PEAUhb_blob_t@@@Z 000000018000d3b0 f   hb-aat-layout.obj
 0001:0000c4a0       ??0hb_ot_apply_context_t@OT@@QEAA@IPEAUhb_font_t@@PEAUhb_buffer_t@@@Z 000000018000d4a0 f i hb-aat-layout.obj
 0001:0000c780       ??1hb_aat_apply_context_t@AAT@@QEAA@XZ 000000018000d780 f   hb-aat-layout.obj
 0001:0000c790       ??C?$hb_lazy_loader_t@UGDEF_accelerator_t@OT@@U?$hb_face_lazy_loader_t@UGDEF_accelerator_t@OT@@$0BI@@@Uhb_face_t@@$0BI@U12@@@QEBAPEBUGDEF_accelerator_t@OT@@XZ 000000018000d790 f i hb-aat-layout.obj
 0001:0000c8e0       ??C?$hb_lazy_loader_t@Ufeat@AAT@@U?$hb_table_lazy_loader_t@Ufeat@AAT@@$0CC@$0A@@@Uhb_face_t@@$0CC@Uhb_blob_t@@@@QEBAPEBUfeat@AAT@@XZ 000000018000d8e0 f i hb-aat-layout.obj
 0001:0000c9e0       ??C?$hb_lazy_loader_t@Ultag@AAT@@U?$hb_table_lazy_loader_t@Ultag@AAT@@$0CB@$0A@@@Uhb_face_t@@$0CB@Uhb_blob_t@@@@QEBAPEBUltag@AAT@@XZ 000000018000d9e0 f i hb-aat-layout.obj
 0001:0000cae0       ?_infos_find_min_cluster@hb_buffer_t@@QEAAIPEBUhb_glyph_info_t@@III@Z 000000018000dae0 f i hb-aat-layout.obj
 0001:0000cb70       ?_infos_set_glyph_flags@hb_buffer_t@@QEAAXPEAUhb_glyph_info_t@@IIII@Z 000000018000db70 f i hb-aat-layout.obj
 0001:0000cc60       ?alloc@?$hb_vector_t@U?$hb_vector_t@Urange_flags_t@hb_aat_map_t@@$00@@$0A@@@QEAA_NI_N@Z 000000018000dc60 f i hb-aat-layout.obj
 0001:0000cdd0       ?apply@?$Chain@UExtendedTypes@AAT@@@AAT@@QEBAXPEAUhb_aat_apply_context_t@2@@Z 000000018000ddd0 f i hb-aat-layout.obj
 0001:0000d130       ?apply@?$Chain@UObsoleteTypes@AAT@@@AAT@@QEBAXPEAUhb_aat_apply_context_t@2@@Z 000000018000e130 f i hb-aat-layout.obj
 0001:0000d450       ?apply@?$KerxTable@Ukerx@AAT@@@AAT@@QEBA_NPEAUhb_aat_apply_context_t@2@@Z 000000018000e450 f i hb-aat-layout.obj
 0001:0000d6d0       ?apply@?$NoncontextualSubtable@UExtendedTypes@AAT@@@AAT@@QEBA_NPEAUhb_aat_apply_context_t@2@@Z 000000018000e6d0 f i hb-aat-layout.obj
 0001:0000d6d0       ?apply@?$NoncontextualSubtable@UObsoleteTypes@AAT@@@AAT@@QEBA_NPEAUhb_aat_apply_context_t@2@@Z 000000018000e6d0 f i hb-aat-layout.obj
 0001:0000d840       ?apply@trak@AAT@@QEBA_NPEAUhb_aat_apply_context_t@2@@Z 000000018000e840 f i hb-aat-layout.obj
 0001:0000dac0       ?backtrack_len@hb_buffer_t@@QEBAIXZ 000000018000eac0 f i hb-aat-layout.obj
 0001:0000dad0       ?check_range@hb_sanitize_context_t@@QEBA_NPEBXI@Z 000000018000ead0 f i hb-aat-layout.obj
 0001:0000db90       ?compile_flags@?$Chain@UExtendedTypes@AAT@@@AAT@@QEBAIPEBUhb_aat_map_builder_t@@@Z 000000018000eb90 f i hb-aat-layout.obj
 0001:0000dde0       ?compile_flags@?$Chain@UObsoleteTypes@AAT@@@AAT@@QEBAIPEBUhb_aat_map_builder_t@@@Z 000000018000ede0 f i hb-aat-layout.obj
 0001:0000e020       ?compile_flags@?$mortmorx@UExtendedTypes@AAT@@$0GNGPHCHI@@AAT@@QEBAXPEBUhb_aat_map_builder_t@@PEAUhb_aat_map_t@@@Z 000000018000f020 f i hb-aat-layout.obj
 0001:0000e210       ?compile_flags@?$mortmorx@UObsoleteTypes@AAT@@$0GNGPHCHE@@AAT@@QEBAXPEBUhb_aat_map_builder_t@@PEAUhb_aat_map_t@@@Z 000000018000f210 f i hb-aat-layout.obj
 0001:0000e400       ?copy_glyph@hb_buffer_t@@QEAA_NXZ 000000018000f400 f i hb-aat-layout.obj
 0001:0000e470       ?create_cache@VariationStore@OT@@QEBAPEAMXZ 000000018000f470 f i hb-aat-layout.obj
 0001:0000e500       ?end_processing@hb_sanitize_context_t@@QEAAXXZ 000000018000f500 f i hb-aat-layout.obj
 0001:0000e580       ?get@?$hb_lazy_loader_t@Utrak@AAT@@U?$hb_table_lazy_loader_t@Utrak@AAT@@$0CA@$0A@@@Uhb_face_t@@$0CA@Uhb_blob_t@@@@QEBAPEBUtrak@AAT@@XZ 000000018000f580 f i hb-aat-layout.obj
 0001:0000e680       ?get_anchor@ankr@AAT@@QEBAAEBUAnchor@2@III@Z 000000018000f680 f i hb-aat-layout.obj
 0001:0000e750       ?get_class@ClassDef@OT@@QEBAII@Z 000000018000f750 f i hb-aat-layout.obj
 0001:0000e860       ?get_coverage@?$CoverageFormat1_3@USmallTypes@Layout@OT@@@Common@Layout@OT@@AEBAII@Z 000000018000f860 f i hb-aat-layout.obj
 0001:0000e8d0       ?get_coverage@?$CoverageFormat2_4@USmallTypes@Layout@OT@@@Common@Layout@OT@@AEBAII@Z 000000018000f8d0 f i hb-aat-layout.obj
 0001:0000e9c0       ?get_feature@feat@AAT@@QEBAAEBUFeatureName@2@W4hb_aat_layout_feature_type_t@@@Z 000000018000f9c0 f i hb-aat-layout.obj
 0001:0000ea40       ?get_glyph_contour_point_for_origin@hb_font_t@@QEAAHIIW4hb_direction_t@@PEAH1@Z 000000018000fa40 f i hb-aat-layout.obj
 0001:0000eb10       ?get_glyph_h_origin_with_fallback@hb_font_t@@QEAAXIPEAH0@Z 000000018000fb10 f i hb-aat-layout.obj
 0001:0000ec70       ?get_glyph_origin_for_direction@hb_font_t@@QEAAXIW4hb_direction_t@@PEAH1@Z 000000018000fc70 f i hb-aat-layout.obj
 0001:0000eef0       ?get_glyph_props@GDEF@OT@@QEBAII@Z 000000018000fef0 f i hb-aat-layout.obj
 0001:0000efe0       ?get_glyph_v_origin_with_fallback@hb_font_t@@QEAAXIPEAH0@Z 000000018000ffe0 f i hb-aat-layout.obj
 0001:0000f140       ?get_kerning@?$KerxSubTableFormat0@UKerxSubTableHeader@AAT@@@AAT@@QEBAHIIPEAUhb_aat_apply_context_t@2@@Z 0000000180010140 f i hb-aat-layout.obj
 0001:0000f2a0       ?get_kerning@?$KerxSubTableFormat2@UKerxSubTableHeader@AAT@@@AAT@@QEBAHIIPEAUhb_aat_apply_context_t@2@@Z 00000001800102a0 f i hb-aat-layout.obj
 0001:0000f450       ?get_kerning@?$KerxSubTableFormat6@UKerxSubTableHeader@AAT@@@AAT@@QEBAHIIPEAUhb_aat_apply_context_t@2@@Z 0000000180010450 f i hb-aat-layout.obj
 0001:0000f7b0       ?get_length@?$VarSizedBinSearchArrayOf@U?$LookupSegmentArray@U?$IntType@G$01@OT@@@AAT@@@OT@@QEBAIXZ 00000001800107b0 f i hb-aat-layout.obj
 0001:0000f7b0       ?get_length@?$VarSizedBinSearchArrayOf@U?$LookupSegmentArray@U?$IntType@I$03@OT@@@AAT@@@OT@@QEBAIXZ 00000001800107b0 f i hb-aat-layout.obj
 0001:0000f7b0       ?get_length@?$VarSizedBinSearchArrayOf@U?$LookupSegmentArray@U?$OffsetTo@U?$ArrayOf@UAnchor@AAT@@U?$IntType@I$03@OT@@@OT@@U?$IntType@G$01@2@$0A@@OT@@@AAT@@@OT@@QEBAIXZ 00000001800107b0 f i hb-aat-layout.obj
 0001:0000f7b0       ?get_length@?$VarSizedBinSearchArrayOf@U?$LookupSegmentArray@UHBGlyphID16@OT@@@AAT@@@OT@@QEBAIXZ 00000001800107b0 f i hb-aat-layout.obj
 0001:0000f7b0       ?get_length@?$VarSizedBinSearchArrayOf@U?$LookupSegmentSingle@U?$OffsetTo@U?$ArrayOf@UAnchor@AAT@@U?$IntType@I$03@OT@@@OT@@U?$IntType@G$01@2@$0A@@OT@@@AAT@@@OT@@QEBAIXZ 00000001800107b0 f i hb-aat-layout.obj
 0001:0000f850       ?get_length@?$VarSizedBinSearchArrayOf@U?$LookupSingle@U?$OffsetTo@U?$ArrayOf@UAnchor@AAT@@U?$IntType@I$03@OT@@@OT@@U?$IntType@G$01@2@$0A@@OT@@@AAT@@@OT@@QEBAIXZ 0000000180010850 f i hb-aat-layout.obj
 0001:0000f8f0       ?get_size@HintingDevice@OT@@QEBAIXZ 00000001800108f0 f i hb-aat-layout.obj
 0001:0000f960       ?get_stored@?$hb_lazy_loader_t@Ukerx@AAT@@U?$hb_table_lazy_loader_t@Ukerx@AAT@@$0BO@$0A@@@Uhb_face_t@@$0BO@Uhb_blob_t@@@@QEBAPEAUhb_blob_t@@XZ 0000000180010960 f i hb-aat-layout.obj
 0001:0000fa60       ?get_stored@?$hb_lazy_loader_t@Umort@AAT@@U?$hb_table_lazy_loader_t@Umort@AAT@@$0BN@$0A@@@Uhb_face_t@@$0BN@Uhb_blob_t@@@@QEBAPEAUhb_blob_t@@XZ 0000000180010a60 f i hb-aat-layout.obj
 0001:0000fb60       ?get_stored@?$hb_lazy_loader_t@Umorx@AAT@@U?$hb_table_lazy_loader_t@Umorx@AAT@@$0BM@$0A@@@Uhb_face_t@@$0BM@Uhb_blob_t@@@@QEBAPEAUhb_blob_t@@XZ 0000000180010b60 f i hb-aat-layout.obj
 0001:0000fc60       ?get_tracking@TrackData@AAT@@QEBAHPEBXM@Z 0000000180010c60 f i hb-aat-layout.obj
 0001:0000ff80       ?get_value@?$Lookup@U?$IntType@G$01@OT@@@AAT@@QEBAPEBU?$IntType@G$01@OT@@II@Z 0000000180010f80 f i hb-aat-layout.obj
 0001:0000ff80       ?get_value@?$Lookup@U?$OffsetTo@U?$ArrayOf@UAnchor@AAT@@U?$IntType@I$03@OT@@@OT@@U?$IntType@G$01@2@$0A@@OT@@@AAT@@QEBAPEBU?$OffsetTo@U?$ArrayOf@UAnchor@AAT@@U?$IntType@I$03@OT@@@OT@@U?$IntType@G$01@2@$0A@@OT@@II@Z 0000000180010f80 f i hb-aat-layout.obj
 0001:0000ff80       ?get_value@?$Lookup@UHBGlyphID16@OT@@@AAT@@QEBAPEBUHBGlyphID16@OT@@II@Z 0000000180010f80 f i hb-aat-layout.obj
 0001:00010190       ?get_value@?$Lookup@U?$IntType@I$03@OT@@@AAT@@QEBAPEBU?$IntType@I$03@OT@@II@Z 0000000180011190 f i hb-aat-layout.obj
 0001:000103a0       ?get_value@?$LookupFormat2@U?$IntType@G$01@OT@@@AAT@@AEBAPEBU?$IntType@G$01@OT@@I@Z 00000001800113a0 f i hb-aat-layout.obj
 0001:000103a0       ?get_value@?$LookupFormat2@U?$IntType@I$03@OT@@@AAT@@AEBAPEBU?$IntType@I$03@OT@@I@Z 00000001800113a0 f i hb-aat-layout.obj
 0001:000103a0       ?get_value@?$LookupFormat2@U?$OffsetTo@U?$ArrayOf@UAnchor@AAT@@U?$IntType@I$03@OT@@@OT@@U?$IntType@G$01@2@$0A@@OT@@@AAT@@AEBAPEBU?$OffsetTo@U?$ArrayOf@UAnchor@AAT@@U?$IntType@I$03@OT@@@OT@@U?$IntType@G$01@2@$0A@@OT@@I@Z 00000001800113a0 f i hb-aat-layout.obj
 0001:000103a0       ?get_value@?$LookupFormat2@UHBGlyphID16@OT@@@AAT@@AEBAPEBUHBGlyphID16@OT@@I@Z 00000001800113a0 f i hb-aat-layout.obj
 0001:000104e0       ?get_value@?$LookupFormat4@U?$IntType@G$01@OT@@@AAT@@AEBAPEBU?$IntType@G$01@OT@@I@Z 00000001800114e0 f i hb-aat-layout.obj
 0001:000104e0       ?get_value@?$LookupFormat4@U?$OffsetTo@U?$ArrayOf@UAnchor@AAT@@U?$IntType@I$03@OT@@@OT@@U?$IntType@G$01@2@$0A@@OT@@@AAT@@AEBAPEBU?$OffsetTo@U?$ArrayOf@UAnchor@AAT@@U?$IntType@I$03@OT@@@OT@@U?$IntType@G$01@2@$0A@@OT@@I@Z 00000001800114e0 f i hb-aat-layout.obj
 0001:000104e0       ?get_value@?$LookupFormat4@UHBGlyphID16@OT@@@AAT@@AEBAPEBUHBGlyphID16@OT@@I@Z 00000001800114e0 f i hb-aat-layout.obj
 0001:00010670       ?get_value@?$LookupFormat4@U?$IntType@I$03@OT@@@AAT@@AEBAPEBU?$IntType@I$03@OT@@I@Z 0000000180011670 f i hb-aat-layout.obj
 0001:00010800       ?get_value_or_null@?$Lookup@U?$IntType@G$01@OT@@@AAT@@QEBA?BGII@Z 0000000180011800 f i hb-aat-layout.obj
 0001:00010900       ?get_value_or_null@?$Lookup@U?$IntType@I$03@OT@@@AAT@@QEBA?BIII@Z 0000000180011900 f i hb-aat-layout.obj
 0001:00010a20       ?hb_aat_layout_compile_map@@YAXPEBUhb_aat_map_builder_t@@PEAUhb_aat_map_t@@@Z 0000000180011a20 f   hb-aat-layout.obj
 0001:00010ad0       ?hb_aat_layout_find_feature_mapping@@YAPEBUhb_aat_feature_mapping_t@@I@Z 0000000180011ad0 f   hb-aat-layout.obj
 0001:00010b30       ?hb_aat_layout_position@@YAXPEBUhb_ot_shape_plan_t@@PEAUhb_font_t@@PEAUhb_buffer_t@@@Z 0000000180011b30 f   hb-aat-layout.obj
 0001:00010ce0       ?hb_aat_layout_remove_deleted_glyphs@@YAXPEAUhb_buffer_t@@@Z 0000000180011ce0 f   hb-aat-layout.obj
 0001:00010cf0       ?hb_aat_layout_substitute@@YAXPEBUhb_ot_shape_plan_t@@PEAUhb_font_t@@PEAUhb_buffer_t@@PEBUhb_feature_t@@I@Z 0000000180011cf0 f   hb-aat-layout.obj
 0001:000110c0       ?hb_aat_layout_track@@YAXPEBUhb_ot_shape_plan_t@@PEAUhb_font_t@@PEAUhb_buffer_t@@@Z 00000001800120c0 f   hb-aat-layout.obj
 0001:00011150       ?hb_aat_layout_zero_width_deleted_glyphs@@YAXPEAUhb_buffer_t@@@Z 0000000180012150 f   hb-aat-layout.obj
 0001:00011190       ?init_iters@hb_ot_apply_context_t@OT@@QEAAXXZ 0000000180012190 f i hb-aat-layout.obj
 0001:00011250       ?interpolate_at@TrackData@AAT@@QEBAMIMAEBUTrackTableEntry@2@PEBX@Z 0000000180012250 f i hb-aat-layout.obj
 0001:000113f0       ?kern@?$hb_kern_machine_t@Uaccelerator_t@?$KerxSubTableFormat0@UKerxSubTableHeader@AAT@@@AAT@@@OT@@QEBAXPEAUhb_font_t@@PEAUhb_buffer_t@@I_N@Z 00000001800123f0 f i hb-aat-layout.obj
 0001:00011770       ?kern@?$hb_kern_machine_t@Uaccelerator_t@?$KerxSubTableFormat2@UKerxSubTableHeader@AAT@@@AAT@@@OT@@QEBAXPEAUhb_font_t@@PEAUhb_buffer_t@@I_N@Z 0000000180012770 f i hb-aat-layout.obj
 0001:00011af0       ?kern@?$hb_kern_machine_t@Uaccelerator_t@?$KerxSubTableFormat6@UKerxSubTableHeader@AAT@@@AAT@@@OT@@QEBAXPEAUhb_font_t@@PEAUhb_buffer_t@@I_N@Z 0000000180012af0 f i hb-aat-layout.obj
 0001:00011e70       ?mark_set_covers@GDEF@OT@@QEBA_NII@Z 0000000180012e70 f i hb-aat-layout.obj
 0001:00011fe0       ?may_edit@hb_sanitize_context_t@@QEAA_NPEBXI@Z 0000000180012fe0 f i hb-aat-layout.obj
 0001:00012090       ?may_skip@matcher_t@hb_ot_apply_context_t@OT@@QEBA?AW4may_skip_t@123@PEBU23@AEBUhb_glyph_info_t@@@Z 0000000180013090 f i hb-aat-layout.obj
 0001:00012170       ?message@hb_buffer_t@@QEAA_NPEAUhb_font_t@@PEBDZZ 0000000180013170 f i hb-aat-layout.obj
 0001:000121a0       ?next@skipping_iterator_t@hb_ot_apply_context_t@OT@@QEAA_NPEAI@Z 00000001800131a0 f i hb-aat-layout.obj
 0001:000122b0       ?next_glyph@hb_buffer_t@@QEAA_NXZ 00000001800132b0 f i hb-aat-layout.obj
 0001:00012350       ?replace_glyph@hb_buffer_t@@QEAA_NI@Z 0000000180013350 f i hb-aat-layout.obj
 0001:000123e0       ?reverse_range@hb_buffer_t@@QEAAXII@Z 00000001800133e0 f i hb-aat-layout.obj
 0001:000124f0       ?sanitize@?$Chain@UExtendedTypes@AAT@@@AAT@@QEBA_NPEAUhb_sanitize_context_t@@I@Z 00000001800134f0 f i hb-aat-layout.obj
 0001:00012760       ?sanitize@?$ChainSubtable@UObsoleteTypes@AAT@@@AAT@@QEBA_NPEAUhb_sanitize_context_t@@@Z 0000000180013760 f i hb-aat-layout.obj
 0001:00012840       ?sanitize@?$GDEFVersion1_2@USmallTypes@Layout@OT@@@OT@@QEBA_NPEAUhb_sanitize_context_t@@@Z 0000000180013840 f i hb-aat-layout.obj
 0001:00012a30       ?sanitize@?$KerxSubTableFormat6@UKerxSubTableHeader@AAT@@@AAT@@QEBA_NPEAUhb_sanitize_context_t@@@Z 0000000180013a30 f i hb-aat-layout.obj
 0001:00012c30       ?sanitize@?$KerxTable@Ukerx@AAT@@@AAT@@QEBA_NPEAUhb_sanitize_context_t@@@Z 0000000180013c30 f i hb-aat-layout.obj
 0001:00012e50       ?sanitize@?$Lookup@U?$IntType@G$01@OT@@@AAT@@QEBA_NPEAUhb_sanitize_context_t@@@Z 0000000180013e50 f i hb-aat-layout.obj
 0001:00012e50       ?sanitize@?$Lookup@UHBGlyphID16@OT@@@AAT@@QEBA_NPEAUhb_sanitize_context_t@@@Z 0000000180013e50 f i hb-aat-layout.obj
 0001:00013070       ?sanitize@?$Lookup@U?$IntType@I$03@OT@@@AAT@@QEBA_NPEAUhb_sanitize_context_t@@@Z 0000000180014070 f i hb-aat-layout.obj
 0001:000132a0       ?sanitize@?$Lookup@U?$OffsetTo@U?$ArrayOf@UAnchor@AAT@@U?$IntType@I$03@OT@@@OT@@U?$IntType@G$01@2@$0A@@OT@@@AAT@@QEBA_NPEAUhb_sanitize_context_t@@PEBX@Z 00000001800142a0 f i hb-aat-layout.obj
 0001:00013610       ?sanitize@?$StateTable@UExtendedTypes@AAT@@UEntryData@?$ContextualSubtable@UExtendedTypes@AAT@@@2@@AAT@@QEBA_NPEAUhb_sanitize_context_t@@PEAI@Z 0000000180014610 f i hb-aat-layout.obj
 0001:00013610       ?sanitize@?$StateTable@UExtendedTypes@AAT@@UEntryData@?$InsertionSubtable@UExtendedTypes@AAT@@@2@@AAT@@QEBA_NPEAUhb_sanitize_context_t@@PEAI@Z 0000000180014610 f i hb-aat-layout.obj
 0001:00013970       ?sanitize@?$StateTable@UExtendedTypes@AAT@@UEntryData@?$Format1Entry@$00@2@@AAT@@QEBA_NPEAUhb_sanitize_context_t@@PEAI@Z 0000000180014970 f i hb-aat-layout.obj
 0001:00013970       ?sanitize@?$StateTable@UExtendedTypes@AAT@@UEntryData@?$KerxSubTableFormat4@UKerxSubTableHeader@AAT@@@2@@AAT@@QEBA_NPEAUhb_sanitize_context_t@@PEAI@Z 0000000180014970 f i hb-aat-layout.obj
 0001:00013970       ?sanitize@?$StateTable@UExtendedTypes@AAT@@UEntryData@?$LigatureEntry@$00@2@@AAT@@QEBA_NPEAUhb_sanitize_context_t@@PEAI@Z 0000000180014970 f i hb-aat-layout.obj
 0001:00013ce0       ?sanitize@?$StateTable@UExtendedTypes@AAT@@X@AAT@@QEBA_NPEAUhb_sanitize_context_t@@PEAI@Z 0000000180014ce0 f i hb-aat-layout.obj
 0001:00014040       ?sanitize@?$StateTable@UObsoleteTypes@AAT@@UEntryData@?$ContextualSubtable@UObsoleteTypes@AAT@@@2@@AAT@@QEBA_NPEAUhb_sanitize_context_t@@PEAI@Z 0000000180015040 f i hb-aat-layout.obj
 0001:00014040       ?sanitize@?$StateTable@UObsoleteTypes@AAT@@UEntryData@?$InsertionSubtable@UObsoleteTypes@AAT@@@2@@AAT@@QEBA_NPEAUhb_sanitize_context_t@@PEAI@Z 0000000180015040 f i hb-aat-layout.obj
 0001:00014350       ?sanitize@?$StateTable@UObsoleteTypes@AAT@@X@AAT@@QEBA_NPEAUhb_sanitize_context_t@@PEAI@Z 0000000180015350 f i hb-aat-layout.obj
 0001:00014660       ?sanitize@?$mortmorx@UExtendedTypes@AAT@@$0GNGPHCHI@@AAT@@QEBA_NPEAUhb_sanitize_context_t@@@Z 0000000180015660 f i hb-aat-layout.obj
 0001:00014770       ?sanitize@?$mortmorx@UObsoleteTypes@AAT@@$0GNGPHCHE@@AAT@@QEBA_NPEAUhb_sanitize_context_t@@@Z 0000000180015770 f i hb-aat-layout.obj
 0001:00014970       ?sanitize@MarkGlyphSets@OT@@QEBA_NPEAUhb_sanitize_context_t@@@Z 0000000180015970 f i hb-aat-layout.obj
 0001:00014ad0       ?sanitize@TrackData@AAT@@QEBA_NPEAUhb_sanitize_context_t@@PEBX@Z 0000000180015ad0 f i hb-aat-layout.obj
 0001:00014c50       ?sanitize@VariationStore@OT@@QEBA_NPEAUhb_sanitize_context_t@@@Z 0000000180015c50 f i hb-aat-layout.obj
 0001:00014e00       ?sanitize@ankr@AAT@@QEBA_NPEAUhb_sanitize_context_t@@@Z 0000000180015e00 f i hb-aat-layout.obj
 0001:00014f50       ?sanitize@feat@AAT@@QEBA_NPEAUhb_sanitize_context_t@@@Z 0000000180015f50 f i hb-aat-layout.obj
 0001:00015070       ?sanitize@ltag@AAT@@QEBA_NPEAUhb_sanitize_context_t@@@Z 0000000180016070 f i hb-aat-layout.obj
 0001:000151d0       ?sanitize@trak@AAT@@QEBA_NPEAUhb_sanitize_context_t@@@Z 00000001800161d0 f i hb-aat-layout.obj
 0001:00015320       ?sanitize_shallow@?$OffsetTo@U?$UnsizedListOfOffset16To@U?$Lookup@UHBGlyphID16@OT@@@AAT@@U?$IntType@I$03@OT@@$0A@@OT@@U?$IntType@I$03@2@$0A@@OT@@QEBA_NPEAUhb_sanitize_context_t@@PEBX@Z 0000000180016320 f i hb-aat-layout.obj
 0001:00015390       ?shrink_vector@?$hb_vector_t@U?$hb_vector_t@Urange_flags_t@hb_aat_map_t@@$00@@$0A@@@QEAAXI@Z 0000000180016390 f i hb-aat-layout.obj
 0001:00015410       ?start_processing@hb_sanitize_context_t@@QEAAXXZ 0000000180016410 f i hb-aat-layout.obj
 0001:000154e0       ?transition@driver_context_t@?$ContextualSubtable@UExtendedTypes@AAT@@@AAT@@QEAAXPEAU?$StateTableDriver@UExtendedTypes@AAT@@UEntryData@?$ContextualSubtable@UExtendedTypes@AAT@@@2@@3@AEBU?$Entry@UEntryData@?$ContextualSubtable@UExtendedTypes@AAT@@@AAT@@@3@@Z 00000001800164e0 f i hb-aat-layout.obj
 0001:00015720       ?transition@driver_context_t@?$InsertionSubtable@UExtendedTypes@AAT@@@AAT@@QEAAXPEAU?$StateTableDriver@UExtendedTypes@AAT@@UEntryData@?$InsertionSubtable@UExtendedTypes@AAT@@@2@@3@AEBU?$Entry@UEntryData@?$InsertionSubtable@UExtendedTypes@AAT@@@AAT@@@3@@Z 0000000180016720 f i hb-aat-layout.obj
 0001:00015720       ?transition@driver_context_t@?$InsertionSubtable@UObsoleteTypes@AAT@@@AAT@@QEAAXPEAU?$StateTableDriver@UObsoleteTypes@AAT@@UEntryData@?$InsertionSubtable@UObsoleteTypes@AAT@@@2@@3@AEBU?$Entry@UEntryData@?$InsertionSubtable@UObsoleteTypes@AAT@@@AAT@@@3@@Z 0000000180016720 f i hb-aat-layout.obj
 0001:00015980       ?transition@driver_context_t@?$KerxSubTableFormat1@UKerxSubTableHeader@AAT@@@AAT@@QEAAXPEAU?$StateTableDriver@UExtendedTypes@AAT@@UEntryData@?$Format1Entry@$00@2@@3@AEBU?$Entry@UEntryData@?$Format1Entry@$00@AAT@@@3@@Z 0000000180016980 f i hb-aat-layout.obj
 0001:00015d50       ?transition@driver_context_t@?$KerxSubTableFormat4@UKerxSubTableHeader@AAT@@@AAT@@QEAAXPEAU?$StateTableDriver@UExtendedTypes@AAT@@UEntryData@?$KerxSubTableFormat4@UKerxSubTableHeader@AAT@@@2@@3@AEBU?$Entry@UEntryData@?$KerxSubTableFormat4@UKerxSubTableHeader@AAT@@@AAT@@@3@@Z 0000000180016d50 f i hb-aat-layout.obj
 0001:000161a0       ?transition@driver_context_t@?$LigatureSubtable@UExtendedTypes@AAT@@@AAT@@QEAAXPEAU?$StateTableDriver@UExtendedTypes@AAT@@UEntryData@?$LigatureEntry@$00@2@@3@AEBU?$Entry@UEntryData@?$LigatureEntry@$00@AAT@@@3@@Z 00000001800171a0 f i hb-aat-layout.obj
 0001:000164d0       ?transition@driver_context_t@?$LigatureSubtable@UObsoleteTypes@AAT@@@AAT@@QEAAXPEAU?$StateTableDriver@UObsoleteTypes@AAT@@X@3@AEBU?$Entry@X@3@@Z 00000001800174d0 f i hb-aat-layout.obj
 0001:00016850       ?transition@driver_context_t@?$RearrangementSubtable@UExtendedTypes@AAT@@@AAT@@QEAAXPEAU?$StateTableDriver@UExtendedTypes@AAT@@X@3@AEBU?$Entry@X@3@@Z 0000000180017850 f i hb-aat-layout.obj
 0001:00016850       ?transition@driver_context_t@?$RearrangementSubtable@UObsoleteTypes@AAT@@@AAT@@QEAAXPEAU?$StateTableDriver@UObsoleteTypes@AAT@@X@3@AEBU?$Entry@X@3@@Z 0000000180017850 f i hb-aat-layout.obj
 0001:00016b60       ?unsafe_to_break@hb_buffer_t@@QEAAXII@Z 0000000180017b60 f i hb-aat-layout.obj
 0001:00016be0       ?unsafe_to_break_from_outbuffer@hb_buffer_t@@QEAAXII@Z 0000000180017be0 f i hb-aat-layout.obj
 0001:00016cd0       ?unsafe_to_concat@hb_buffer_t@@QEAAXII@Z 0000000180017cd0 f i hb-aat-layout.obj
 0001:00016d50       hb_aat_layout_has_positioning 0000000180017d50 f   hb-aat-layout.obj
 0001:00016da0       hb_aat_layout_has_substitution 0000000180017da0 f   hb-aat-layout.obj
 0001:00016e40       hb_aat_layout_has_tracking 0000000180017e40 f   hb-aat-layout.obj
 0001:000171f0       ?add_feature@hb_aat_map_builder_t@@QEAAXAEBUhb_feature_t@@@Z 00000001800181f0 f   hb-aat-map.obj
 0001:000173b0       ?alloc@?$hb_vector_t@Ufeature_info_t@hb_aat_map_builder_t@@$00@@QEAA_NI_N@Z 00000001800183b0 f i hb-aat-map.obj
 0001:00017460       ?cmp@feature_event_t@hb_aat_map_builder_t@@SAHPEBX0@Z 0000000180018460 f i hb-aat-map.obj
 0001:00017490       ?cmp@feature_info_t@hb_aat_map_builder_t@@SAHPEBX0@Z 0000000180018490 f i hb-aat-map.obj
 0001:000174f0       ?compile@hb_aat_map_builder_t@@QEAAXAEAUhb_aat_map_t@@@Z 00000001800184f0 f   hb-aat-map.obj
 0001:00018210       ?push@?$hb_vector_t@Ufeature_event_t@hb_aat_map_builder_t@@$0A@@@QEAAPEAUfeature_event_t@hb_aat_map_builder_t@@XZ 0000000180019210 f i hb-aat-map.obj
 0001:00018210       ?push@?$hb_vector_t@Ufeature_range_t@hb_aat_map_builder_t@@$00@@QEAAPEAUfeature_range_t@hb_aat_map_builder_t@@XZ 0000000180019210 f i hb-aat-map.obj
 0001:00018320       ??$replace_or_insert@Uhb_user_data_item_t@hb_user_data_array_t@@@?$hb_lockable_set_t@Uhb_user_data_item_t@hb_user_data_array_t@@Uhb_mutex_t@@@@QEAAPEAUhb_user_data_item_t@hb_user_data_array_t@@U12@AEAUhb_mutex_t@@_N@Z 0000000180019320 f i hb-blob.obj
 0001:00018570       ?try_make_writable@hb_blob_t@@QEAA_NXZ 0000000180019570 f   hb-blob.obj
 0001:000186a0       hb_blob_create             00000001800196a0 f   hb-blob.obj
 0001:000186f0       hb_blob_create_or_fail     00000001800196f0 f   hb-blob.obj
 0001:000187c0       hb_blob_create_sub_blob    00000001800197c0 f   hb-blob.obj
 0001:00018930       hb_blob_destroy            0000000180019930 f   hb-blob.obj
 0001:000189c0       hb_blob_get_data_writable  00000001800199c0 f   hb-blob.obj
 0001:00018a20       hb_blob_get_empty          0000000180019a20 f   hb-blob.obj
 0001:00018a30       hb_blob_make_immutable     0000000180019a30 f   hb-blob.obj
 0001:00018a30       hb_draw_funcs_make_immutable 0000000180019a30 f   hb-draw.obj
 0001:00018a30       hb_face_make_immutable     0000000180019a30 f   hb-face.obj
 0001:00018a30       hb_font_funcs_make_immutable 0000000180019a30 f   hb-font.obj
 0001:00018a30       hb_paint_funcs_make_immutable 0000000180019a30 f   hb-paint.obj
 0001:00018a30       hb_unicode_funcs_make_immutable 0000000180019a30 f   hb-unicode.obj
 0001:00018a40       hb_blob_reference          0000000180019a40 f   hb-blob.obj
 0001:00018a40       hb_face_reference          0000000180019a40 f   hb-face.obj
 0001:00018a40       hb_unicode_funcs_reference 0000000180019a40 f   hb-unicode.obj
 0001:00018a60       __local_stdio_printf_options 0000000180019a60 f i hb-buffer-serialize.obj
 0001:00018a70       hb_buffer_serialize_unicode 0000000180019a70 f   hb-buffer-serialize.obj
 0001:00018db0       snprintf                   0000000180019db0 f i hb-buffer-serialize.obj
 0001:00019610       ?verify@hb_buffer_t@@QEAA_NPEAU1@PEAUhb_font_t@@PEBUhb_feature_t@@IPEBQEBD@Z 000000018001a610 f   hb-buffer-verify.obj
 0001:00019820       fprintf                    000000018001a820 f i hb-buffer-verify.obj
 0001:00019b10       ??$reverse_groups@$$A6A_NAEBUhb_glyph_info_t@@0@Z@hb_buffer_t@@QEAAXA6A_NAEBUhb_glyph_info_t@@0@Z_N@Z 000000018001ab10 f i hb-buffer.obj
 0001:00019cd0       ?clear_output@hb_buffer_t@@QEAAXXZ 000000018001acd0 f   hb-buffer.obj
 0001:00019cf0       ?clear_positions@hb_buffer_t@@QEAAXXZ 000000018001acf0 f   hb-buffer.obj
 0001:00019d30       ?delete_glyph@hb_buffer_t@@QEAAXXZ 000000018001ad30 f   hb-buffer.obj
 0001:00019e00       ?delete_glyphs_inplace@hb_buffer_t@@QEAAXP6A_NPEBUhb_glyph_info_t@@@Z@Z 000000018001ae00 f   hb-buffer.obj
 0001:00019f60       ?enlarge@hb_buffer_t@@QEAA_NI@Z 000000018001af60 f   hb-buffer.obj
 0001:0001a070       ?ensure@hb_buffer_t@@QEAA_NI@Z 000000018001b070 f i hb-buffer.obj
 0001:0001a190       ?enter@hb_buffer_t@@QEAAXXZ 000000018001b190 f   hb-buffer.obj
 0001:0001a1f0       ?leave@hb_buffer_t@@QEAAXXZ 000000018001b1f0 f   hb-buffer.obj
 0001:0001a210       ?make_room_for@hb_buffer_t@@QEAA_NII@Z 000000018001b210 f   hb-buffer.obj
 0001:0001a290       ?merge_clusters_impl@hb_buffer_t@@QEAAXII@Z 000000018001b290 f   hb-buffer.obj
 0001:0001a490       ?merge_out_clusters@hb_buffer_t@@QEAAXII@Z 000000018001b490 f   hb-buffer.obj
 0001:0001a610       ?message_impl@hb_buffer_t@@QEAA_NPEAUhb_font_t@@PEBDPEAD@Z 000000018001b610 f   hb-buffer.obj
 0001:0001a6b0       ?move_to@hb_buffer_t@@QEAA_NI@Z 000000018001b6b0 f   hb-buffer.obj
 0001:0001a830       ?reset@hb_buffer_t@@QEAAXXZ 000000018001b830 f   hb-buffer.obj
 0001:0001a8c0       ?set_masks@hb_buffer_t@@QEAAXIIII@Z 000000018001b8c0 f   hb-buffer.obj
 0001:0001a930       ?sort@hb_buffer_t@@QEAAXIIP6AHPEBUhb_glyph_info_t@@0@Z@Z 000000018001b930 f   hb-buffer.obj
 0001:0001aa90       ?sync@hb_buffer_t@@QEAA_NXZ 000000018001ba90 f   hb-buffer.obj
 0001:0001ab60       ?sync_so_far@hb_buffer_t@@QEAAHXZ 000000018001bb60 f   hb-buffer.obj
 0001:0001ac70       hb_buffer_add_utf16        000000018001bc70 f   hb-buffer.obj
 0001:0001ac80       hb_buffer_append           000000018001bc80 f   hb-buffer.obj
 0001:0001b0d0       hb_buffer_clear_contents   000000018001c0d0 f   hb-buffer.obj
 0001:0001b140       hb_buffer_create           000000018001c140 f   hb-buffer.obj
 0001:0001b1c0       hb_buffer_create_similar   000000018001c1c0 f   hb-buffer.obj
 0001:0001b280       hb_buffer_destroy          000000018001c280 f   hb-buffer.obj
 0001:0001b320       hb_buffer_diff             000000018001c320 f   hb-buffer.obj
 0001:0001b4d0       hb_buffer_get_direction    000000018001c4d0 f   hb-buffer.obj
 0001:0001b4e0       hb_buffer_get_flags        000000018001c4e0 f   hb-buffer.obj
 0001:0001b4f0       hb_buffer_get_glyph_infos  000000018001c4f0 f   hb-buffer.obj
 0001:0001b500       hb_buffer_get_glyph_positions 000000018001c500 f   hb-buffer.obj
 0001:0001b570       hb_buffer_get_length       000000018001c570 f   hb-buffer.obj
 0001:0001b580       hb_buffer_get_segment_properties 000000018001c580 f   hb-buffer.obj
 0001:0001b590       hb_buffer_reverse          000000018001c590 f   hb-buffer.obj
 0001:0001b5a0       hb_buffer_set_cluster_level 000000018001c5a0 f   hb-buffer.obj
 0001:0001b5b0       hb_buffer_set_direction    000000018001c5b0 f   hb-buffer.obj
 0001:0001b5c0       hb_buffer_set_flags        000000018001c5c0 f   hb-buffer.obj
 0001:0001b5d0       hb_buffer_set_language     000000018001c5d0 f   hb-buffer.obj
 0001:0001b5e0       hb_buffer_set_length       000000018001c5e0 f   hb-buffer.obj
 0001:0001b6a0       hb_buffer_set_script       000000018001c6a0 f   hb-buffer.obj
 0001:0001b6b0       hb_buffer_set_segment_properties 000000018001c6b0 f   hb-buffer.obj
 0001:0001b6d0       hb_segment_properties_equal 000000018001c6d0 f   hb-buffer.obj
 0001:0001b710       ??$get_points@Uglyf_accelerator_t@OT@@@Glyph@glyf_impl@OT@@QEBA_NPEAUhb_font_t@@AEBUglyf_accelerator_t@2@AEAUcontour_point_vector_t@2@PEAU52@PEAUhead_maxp_info_t@@PEAI_N66U?$hb_array_t@H@@I5@Z 000000018001c710 f i hb-common.obj
 0001:0001c6c0       ??$get_points@Upoints_aggregator_t@glyf_accelerator_t@OT@@@glyf_accelerator_t@OT@@IEBA_NPEAUhb_font_t@@IUpoints_aggregator_t@01@@Z 000000018001d6c0 f i hb-common.obj
 0001:0001cce0       ??$sanitize@$$V@?$OffsetTo@UDeltaSetIndexMap@OT@@U?$IntType@I$03@2@$00@OT@@QEBA_NPEAUhb_sanitize_context_t@@PEBX@Z 000000018001dce0 f i hb-common.obj
 0001:0001ce80       ??$sanitize_blob@UHVAR@OT@@@hb_sanitize_context_t@@QEAAPEAUhb_blob_t@@PEAU1@@Z 000000018001de80 f i hb-common.obj
 0001:0001d110       ??$sanitize_blob@UVVAR@OT@@@hb_sanitize_context_t@@QEAAPEAUhb_blob_t@@PEAU1@@Z 000000018001e110 f i hb-common.obj
 0001:0001d2e0       ??$sanitize_blob@Ugvar@OT@@@hb_sanitize_context_t@@QEAAPEAUhb_blob_t@@PEAU1@@Z 000000018001e2e0 f i hb-common.obj
 0001:0001d660       ??$sanitize_blob@Uhead@OT@@@hb_sanitize_context_t@@QEAAPEAUhb_blob_t@@PEAU1@@Z 000000018001e660 f i hb-common.obj
 0001:0001d9a0       ??$sanitize_blob@Uhhea@OT@@@hb_sanitize_context_t@@QEAAPEAUhb_blob_t@@PEAU1@@Z 000000018001e9a0 f i hb-common.obj
 0001:0001d9a0       ??$sanitize_blob@Uvhea@OT@@@hb_sanitize_context_t@@QEAAPEAUhb_blob_t@@PEAU1@@Z 000000018001e9a0 f i hb-common.obj
 0001:0001dc90       ??$sanitize_blob@Umaxp@OT@@@hb_sanitize_context_t@@QEAAPEAUhb_blob_t@@PEAU1@@Z 000000018001ec90 f i hb-common.obj
 0001:0001df90       ??0accelerator_t@?$hmtxvmtx@Uhmtx@OT@@Uhhea@2@UHVAR@2@@OT@@QEAA@PEAUhb_face_t@@@Z 000000018001ef90 f i hb-common.obj
 0001:0001e200       ??0accelerator_t@?$hmtxvmtx@Uvmtx@OT@@Uvhea@2@UVVAR@2@@OT@@QEAA@PEAUhb_face_t@@@Z 000000018001f200 f i hb-common.obj
 0001:0001e470       ??0accelerator_t@gvar@OT@@QEAA@PEAUhb_face_t@@@Z 000000018001f470 f i hb-common.obj
 0001:0001e740       ??0glyf_accelerator_t@OT@@QEAA@PEAUhb_face_t@@@Z 000000018001f740 f i hb-common.obj
 0001:0001ec60       ??C?$hb_lazy_loader_t@Uglyf_accelerator_t@OT@@U?$hb_face_lazy_loader_t@Uglyf_accelerator_t@OT@@$0P@@@Uhb_face_t@@$0P@U12@@@QEBAPEBUglyf_accelerator_t@OT@@XZ 000000018001fc60 f i hb-common.obj
 0001:0001ed10       ??C?$hb_lazy_loader_t@Uhhea@OT@@U?$hb_table_lazy_loader_t@Uhhea@OT@@$03$00@@Uhb_face_t@@$03Uhb_blob_t@@@@QEBAPEBUhhea@OT@@XZ 000000018001fd10 f i hb-common.obj
 0001:0001edf0       ??C?$hb_lazy_loader_t@Umaxp@OT@@U?$hb_table_lazy_loader_t@Umaxp@OT@@$01$00@@Uhb_face_t@@$01Uhb_blob_t@@@@QEBAPEBUmaxp@OT@@XZ 000000018001fdf0 f i hb-common.obj
 0001:0001eed0       ??C?$hb_lazy_loader_t@Uvhea@OT@@U?$hb_table_lazy_loader_t@Uvhea@OT@@$0L@$00@@Uhb_face_t@@$0L@Uhb_blob_t@@@@QEBAPEBUvhea@OT@@XZ 000000018001fed0 f i hb-common.obj
 0001:0001efb0       ?_glyf_get_advance_with_var_unscaled@@YAIPEAUhb_font_t@@I_N@Z 000000018001ffb0 f   hb-common.obj
 0001:0001f160       ?_glyf_get_leading_bearing_with_var_unscaled@@YA_NPEAUhb_font_t@@I_NPEAH@Z 0000000180020160 f   hb-common.obj
 0001:0001f2a0       ?_hb_options_init@@YAXXZ   00000001800202a0 f   hb-common.obj
 0001:0001f390       ?alloc@?$hb_vector_t@Ucontour_point_t@OT@@$0A@@@QEAA_NI_N@Z 0000000180020390 f i hb-common.obj
 0001:0001f390       ?alloc@?$hb_vector_t@Ulookup_map_t@hb_ot_map_t@@$0A@@@QEAA_NI_N@Z 0000000180020390 f i hb-ot-map.obj
 0001:0001f450       ?apply_deltas_to_points@accelerator_t@gvar@OT@@QEBA_NIU?$hb_array_t@H@@U?$hb_array_t@Ucontour_point_t@OT@@@@@Z 0000000180020450 f i hb-common.obj
 0001:00020920       ?calculate_scalar@TupleVariationHeader@OT@@QEBAMU?$hb_array_t@H@@IU?$hb_array_t@$$CBU?$HBFixed@U?$IntType@F$01@OT@@$0O@@OT@@@@PEBU?$hb_vector_t@H$0A@@@@Z 0000000180021920 f i hb-common.obj
 0001:00020ba0       ?extend@contour_point_vector_t@OT@@QEAAXAEBU?$hb_array_t@Ucontour_point_t@OT@@@@@Z 0000000180021ba0 f i hb-common.obj
 0001:00020c90       ?get@?$hb_lazy_loader_t@Uhead@OT@@U?$hb_table_lazy_loader_t@Uhead@OT@@$00$00@@Uhb_face_t@@$00Uhb_blob_t@@@@QEBAPEBUhead@OT@@XZ 0000000180021c90 f i hb-common.obj
 0001:00020d70       ?get@?$hb_lazy_loader_t@Uhmtx_accelerator_t@OT@@U?$hb_face_lazy_loader_t@Uhmtx_accelerator_t@OT@@$04@@Uhb_face_t@@$04U12@@@QEBAPEBUhmtx_accelerator_t@OT@@XZ 0000000180021d70 f i hb-common.obj
 0001:00020e30       ?get@?$hb_lazy_loader_t@Uvmtx_accelerator_t@OT@@U?$hb_face_lazy_loader_t@Uvmtx_accelerator_t@OT@@$0M@@@Uhb_face_t@@$0M@U12@@@QEBAPEBUvmtx_accelerator_t@OT@@XZ 0000000180021e30 f i hb-common.obj
 0001:00020ef0       ?get_advance_without_var_unscaled@accelerator_t@?$hmtxvmtx@Uhmtx@OT@@Uhhea@2@UHVAR@2@@OT@@QEBAII@Z 0000000180021ef0 f i hb-common.obj
 0001:00020ef0       ?get_advance_without_var_unscaled@accelerator_t@?$hmtxvmtx@Uvmtx@OT@@Uvhea@2@UVVAR@2@@OT@@QEBAII@Z 0000000180021ef0 f i hb-common.obj
 0001:00020f70       ?get_contour_points@SimpleGlyph@glyf_impl@OT@@QEBA_NAEAUcontour_point_vector_t@3@_N@Z 0000000180021f70 f i hb-common.obj
 0001:000212f0       ?get_glyph_var_data_bytes@gvar@OT@@IEBA?BU?$hb_array_t@$$CBD@@PEAUhb_blob_t@@II@Z 00000001800222f0 f i hb-common.obj
 0001:00021480       ?get_leading_bearing_without_var_unscaled@accelerator_t@?$hmtxvmtx@Uhmtx@OT@@Uhhea@2@UHVAR@2@@OT@@QEBA_NIPEAH@Z 0000000180022480 f i hb-common.obj
 0001:00021480       ?get_leading_bearing_without_var_unscaled@accelerator_t@?$hmtxvmtx@Uvmtx@OT@@Uvhea@2@UVVAR@2@@OT@@QEBA_NIPEAH@Z 0000000180022480 f i hb-common.obj
 0001:00021540       ?get_transformation@CompositeGlyphRecord@glyf_impl@OT@@QEBA_NAEAY03MAEAUcontour_point_t@3@@Z 0000000180022540 f i hb-common.obj
 0001:00021780       ?glyph_for_gid@glyf_accelerator_t@OT@@QEBA?BUGlyph@glyf_impl@2@I_N@Z 0000000180022780 f i hb-common.obj
 0001:00021b80       ?load_num_glyphs@hb_face_t@@AEBAIXZ 0000000180022b80 f   hb-common.obj
 0001:00021bb0       ?load_upem@hb_face_t@@AEBAIXZ 0000000180022bb0 f   hb-common.obj
 0001:00022140       ?read_points@SimpleGlyph@glyf_impl@OT@@SA_NAEAPEBU?$IntType@E$00@3@AEAUcontour_point_vector_t@3@PEBU43@PEQcontour_point_t@3@MW4simple_glyph_flag_t@123@4@Z 0000000180023140 f i hb-common.obj
 0001:00022270       ?resize@?$hb_vector_t@Ucontour_point_t@OT@@$0A@@@QEAA_NH_N0@Z 0000000180023270 f i hb-common.obj
 0001:000222f0       ?sanitize@HVARVVAR@OT@@QEBA_NPEAUhb_sanitize_context_t@@@Z 00000001800232f0 f i hb-common.obj
 0001:000223a0       ?sanitize@gvar@OT@@QEBA_NPEAUhb_sanitize_context_t@@@Z 00000001800233a0 f i hb-common.obj
 0001:000224c0       ?sanitize@maxp@OT@@QEBA_NPEAUhb_sanitize_context_t@@@Z 00000001800234c0 f i hb-common.obj
 0001:00022560       ?scale_glyph_extents@hb_font_t@@QEAAXPEAUhb_glyph_extents_t@@@Z 0000000180023560 f i hb-common.obj
 0001:000226e0       ?transform@contour_point_vector_t@OT@@QEAAXAEAY03$$CBM@Z 00000001800236e0 f i hb-common.obj
 0001:00022890       ?translate@contour_point_vector_t@OT@@QEAAXAEBUcontour_point_t@2@@Z 0000000180023890 f i hb-common.obj
 0001:000229c0       ?trim_padding@SimpleGlyph@glyf_impl@OT@@QEBA?BU?$hb_array_t@$$CBD@@XZ 00000001800239c0 f i hb-common.obj
 0001:00022b20       ?unpack_deltas@TupleVariationData@OT@@SA_NAEAPEBU?$IntType@E$00@2@AEAU?$hb_vector_t@H$0A@@@PEBU32@@Z 0000000180023b20 f i hb-common.obj
 0001:00022d00       ?unpack_points@TupleVariationData@OT@@SA_NAEAPEBU?$IntType@E$00@2@AEAU?$hb_vector_t@I$0A@@@PEBU32@@Z 0000000180023d00 f i hb-common.obj
 0001:00022ee0       hb_feature_from_string     0000000180023ee0 f   hb-common.obj
 0001:00022f50       hb_language_from_string    0000000180023f50 f   hb-common.obj
 0001:00022ff0       hb_language_matches        0000000180023ff0 f   hb-common.obj
 0001:00023090       hb_language_to_string      0000000180024090 f   hb-common.obj
 0001:000230a0       hb_script_get_horizontal_direction 00000001800240a0 f   hb-common.obj
 0001:00023250       hb_tag_from_string         0000000180024250 f   hb-common.obj
 0001:00023300       hb_tag_to_string           0000000180024300 f   hb-common.obj
 0001:000233c0       ?close_path@hb_draw_funcs_t@@QEAAXPEAXAEAUhb_draw_state_t@@@Z 00000001800243c0 f i hb-draw.obj
 0001:00023480       ?cubic_to@hb_draw_funcs_t@@QEAAXPEAXAEAUhb_draw_state_t@@MMMMMM@Z 0000000180024480 f i hb-draw.obj
 0001:000235a0       ?line_to@hb_draw_funcs_t@@QEAAXPEAXAEAUhb_draw_state_t@@MM@Z 00000001800245a0 f i hb-draw.obj
 0001:00023670       ?quadratic_to@hb_draw_funcs_t@@QEAAXPEAXAEAUhb_draw_state_t@@MMMM@Z 0000000180024670 f i hb-draw.obj
 0001:00023770       hb_draw_funcs_create       0000000180024770 f   hb-draw.obj
 0001:000237e0       hb_draw_funcs_destroy      00000001800247e0 f   hb-draw.obj
 0001:00023910       hb_draw_funcs_get_empty    0000000180024910 f   hb-draw.obj
 0001:00023920       hb_draw_funcs_set_close_path_func 0000000180024920 f   hb-draw.obj
 0001:00023a40       hb_draw_funcs_set_cubic_to_func 0000000180024a40 f   hb-draw.obj
 0001:00023b60       hb_draw_funcs_set_line_to_func 0000000180024b60 f   hb-draw.obj
 0001:00023c80       hb_draw_funcs_set_move_to_func 0000000180024c80 f   hb-draw.obj
 0001:00023d90       hb_draw_funcs_set_quadratic_to_func 0000000180024d90 f   hb-draw.obj
 0001:00023eb0       ??0hb_serialize_context_t@@QEAA@PEAXI@Z 0000000180024eb0 f i hb-face-builder.obj
 0001:00023ff0       ??1?$hb_pool_t@Uobject_t@hb_serialize_context_t@@$0CA@@@QEAA@XZ 0000000180024ff0 f i hb-face-builder.obj
 0001:000240e0       ??8item_t@?$hb_hashmap_t@PEBUobject_t@hb_serialize_context_t@@I$0A@@@QEBA_NAEBQEBUobject_t@hb_serialize_context_t@@@Z 00000001800250e0 f i hb-face-builder.obj
 0001:00024180       ?alloc@?$hb_pool_t@Uobject_t@hb_serialize_context_t@@$0CA@@@QEAAPEAUobject_t@hb_serialize_context_t@@XZ 0000000180025180 f i hb-face-builder.obj
 0001:00024420       ?end_serialize@hb_serialize_context_t@@QEAAXXZ 0000000180025420 f i hb-face-builder.obj
 0001:00024510       ?fini@?$hb_hashmap_t@PEBUobject_t@hb_serialize_context_t@@I$0A@@@QEAAXXZ 0000000180025510 f i hb-face-builder.obj
 0001:00024580       ?fini@hb_serialize_context_t@@QEAAXXZ 0000000180025580 f i hb-face-builder.obj
 0001:000246c0       ?fini@object_t@hb_serialize_context_t@@QEAAXXZ 00000001800256c0 f i hb-face-builder.obj
 0001:00024720       ?hash@object_t@hb_serialize_context_t@@QEBAIXZ 0000000180025720 f i hb-face-builder.obj
 0001:000247b0       ?item_for_hash@?$hb_hashmap_t@PEBUobject_t@hb_serialize_context_t@@I$0A@@@QEBAAEAUitem_t@1@AEBQEBUobject_t@hb_serialize_context_t@@I@Z 00000001800257b0 f i hb-face-builder.obj
 0001:00024930       ?pop_pack@hb_serialize_context_t@@QEAAI_N@Z 0000000180025930 f i hb-face-builder.obj
 0001:00024d00       ?resize@?$hb_hashmap_t@PEBUobject_t@hb_serialize_context_t@@I$0A@@@QEAA_NI@Z 0000000180025d00 f i hb-face-builder.obj
 0001:00025030       ?resolve_links@hb_serialize_context_t@@QEAAXXZ 0000000180026030 f i hb-face-builder.obj
 0001:00025300       ??$bsearch@I@?$SortedArrayOf@UCmapSubtableLongGroup@OT@@U?$IntType@I$03@2@@OT@@QEBAAEBUCmapSubtableLongGroup@1@AEBIAEBU21@@Z 0000000180026300 f i hb-face.obj
 0001:000253c0       ??$get_glyph_from@UCmapSubtable@OT@@@accelerator_t@cmap@OT@@KA_NPEBXIPEAI@Z 00000001800263c0 f i hb-face.obj
 0001:000253d0       ??$get_glyph_from@UCmapSubtableFormat12@OT@@@accelerator_t@cmap@OT@@KA_NPEBXIPEAI@Z 00000001800263d0 f i hb-face.obj
 0001:000259c0       ??$sanitize@$$V@?$ArrayOf@UCmapSubtableLongGroup@OT@@U?$IntType@I$03@2@@OT@@QEBA_NPEAUhb_sanitize_context_t@@@Z 00000001800269c0 f i hb-face.obj
 0001:00025a40       ??$sanitize_blob@UOS2@OT@@@hb_sanitize_context_t@@QEAAPEAUhb_blob_t@@PEAU1@@Z 0000000180026a40 f i hb-face.obj
 0001:00025e80       ??$sanitize_blob@Ucmap@OT@@@hb_sanitize_context_t@@QEAAPEAUhb_blob_t@@PEAU1@@Z 0000000180026e80 f i hb-face.obj
 0001:000263d0       ??0accelerator_t@cmap@OT@@QEAA@PEAUhb_face_t@@@Z 00000001800273d0 f i hb-face.obj
 0001:000267e0       ??C?$hb_lazy_loader_t@UOS2@OT@@U?$hb_table_lazy_loader_t@UOS2@OT@@$05$00@@Uhb_face_t@@$05Uhb_blob_t@@@@QEBAPEBUOS2@OT@@XZ 00000001800277e0 f i hb-face.obj
 0001:000268e0       ??C?$hb_lazy_loader_t@Ucmap_accelerator_t@OT@@U?$hb_face_lazy_loader_t@Ucmap_accelerator_t@OT@@$02@@Uhb_face_t@@$02U12@@@QEBAPEBUcmap_accelerator_t@OT@@XZ 00000001800278e0 f i hb-face.obj
 0001:00026ad0       ?find_subtable@cmap@OT@@IEBAPEBUCmapSubtable@2@II@Z 0000000180027ad0 f i hb-face.obj
 0001:00026c20       ?get_glyph@?$CmapSubtableLongSegmented@UCmapSubtableFormat12@OT@@@OT@@QEBA_NIPEAI@Z 0000000180027c20 f i hb-face.obj
 0001:00026c70       ?get_glyph@CmapSubtable@OT@@QEBA_NIPEAI@Z 0000000180027c70 f i hb-face.obj
 0001:00026ec0       ?get_glyph@accelerator_t@CmapSubtableFormat4@OT@@QEBA_NIPEAI@Z 0000000180027ec0 f i hb-face.obj
 0001:00027010       ?get_glyph_func@accelerator_t@CmapSubtableFormat4@OT@@SA_NPEBXIPEAI@Z 0000000180028010 f i hb-face.obj
 0001:00027020       ?group_get_glyph@CmapSubtableFormat12@OT@@SAIAEBUCmapSubtableLongGroup@2@I@Z 0000000180028020 f i hb-face.obj
 0001:000270d0       ?sanitize@CmapSubtable@OT@@QEBA_NPEAUhb_sanitize_context_t@@@Z 00000001800280d0 f i hb-face.obj
 0001:00027420       ?sanitize@OS2@OT@@QEBA_NPEAUhb_sanitize_context_t@@@Z 0000000180028420 f i hb-face.obj
 0001:00027510       ?sanitize@VariationSelectorRecord@OT@@QEBA_NPEAUhb_sanitize_context_t@@PEBX@Z 0000000180028510 f i hb-face.obj
 0001:00027700       ?sanitize@cmap@OT@@QEBA_NPEAUhb_sanitize_context_t@@@Z 0000000180028700 f i hb-face.obj
 0001:00027870       hb_face_create_for_tables  0000000180028870 f   hb-face.obj
 0001:000278f0       hb_face_destroy            00000001800288f0 f   hb-face.obj
 0001:000279e0       hb_face_get_empty          00000001800289e0 f   hb-face.obj
 0001:000279f0       hb_face_get_glyph_count    00000001800289f0 f   hb-face.obj
 0001:00027a00       hb_face_get_upem           0000000180028a00 f   hb-face.obj
 0001:00027a10       hb_face_get_user_data      0000000180028a10 f   hb-face.obj
 0001:00027ae0       hb_face_reference_table    0000000180028ae0 f   hb-face.obj
 0001:00027b10       hb_face_set_user_data      0000000180028b10 f   hb-face.obj
 0001:00027b30       _hb_fallback_shape         0000000180028b30 f   hb-fallback-shape.obj
 0001:00027e40       _get_startup_argv_mode     0000000180028e40 f   MSVCRT:argv_mode.obj
 0001:00027e40       _hb_fallback_shaper_face_data_create 0000000180028e40 f   hb-fallback-shape.obj
 0001:00027e40       _hb_fallback_shaper_font_data_create 0000000180028e40 f   hb-fallback-shape.obj
 0001:00027e40       _hb_ot_shaper_face_data_create 0000000180028e40 f   hb-ot-shape.obj
 0001:00027e40       _hb_ot_shaper_font_data_create 0000000180028e40 f   hb-ot-shape.obj
 0001:00029180       ??$sanitize_blob@Uavar@OT@@@hb_sanitize_context_t@@QEAAPEAUhb_blob_t@@PEAU1@@Z 000000018002a180 f i hb-font.obj
 0001:00029700       ??$sanitize_blob@Ufvar@OT@@@hb_sanitize_context_t@@QEAAPEAUhb_blob_t@@PEAU1@@Z 000000018002a700 f i hb-font.obj
 0001:00029af0       ??C?$hb_lazy_loader_t@Uavar@OT@@U?$hb_table_lazy_loader_t@Uavar@OT@@$0BD@$00@@Uhb_face_t@@$0BD@Uhb_blob_t@@@@QEBAPEBUavar@OT@@XZ 000000018002aaf0 f i hb-font.obj
 0001:00029ce0       ?get@?$hb_lazy_loader_t@Ufvar@OT@@U?$hb_table_lazy_loader_t@Ufvar@OT@@$0BC@$00@@Uhb_face_t@@$0BC@Uhb_blob_t@@@@QEBAPEBUfvar@OT@@XZ 000000018002ace0 f i hb-font.obj
 0001:00029dd0       ?get_delta@VarData@OT@@QEBAMIPEBHIAEBUVarRegionList@2@PEAM@Z 000000018002add0 f i hb-font.obj
 0001:0002a530       ?get_delta@VariationStore@OT@@QEBAMIPEBHIPEAM@Z 000000018002b530 f i hb-font.obj
 0001:0002a600       ?get_instance@fvar@OT@@QEBAPEBUInstanceRecord@2@I@Z 000000018002b600 f i hb-font.obj
 0001:0002a680       ?has_func@hb_font_t@@QEAA_NI@Z 000000018002b680 f   hb-font.obj
 0001:0002a6d0       ?map@DeltaSetIndexMap@OT@@QEBAII@Z 000000018002b6d0 f i hb-font.obj
 0001:0002a7e0       ?map@SegmentMaps@OT@@QEBAHHII@Z 000000018002b7e0 f i hb-font.obj
 0001:0002aa20       ?map_coords@avar@OT@@QEBAXPEAHI@Z 000000018002ba20 f i hb-font.obj
 0001:0002afc0       ?mults_changed@hb_font_t@@QEAAXXZ 000000018002bfc0 f i hb-font.obj
 0001:0002b130       ?sanitize@avar@OT@@QEBA_NPEAUhb_sanitize_context_t@@@Z 000000018002c130 f i hb-font.obj
 0001:0002b2e0       ?sanitize@fvar@OT@@QEBA_NPEAUhb_sanitize_context_t@@@Z 000000018002c2e0 f i hb-font.obj
 0001:0002b480       hb_font_create             000000018002c480 f   hb-font.obj
 0001:0002b4e0       hb_font_destroy            000000018002c4e0 f   hb-font.obj
 0001:0002b5e0       hb_font_draw_glyph         000000018002c5e0 f   hb-font.obj
 0001:0002b620       hb_font_funcs_create       000000018002c620 f   hb-font.obj
 0001:0002b6f0       hb_font_funcs_destroy      000000018002c6f0 f   hb-font.obj
 0001:0002b9f0       hb_font_funcs_get_empty    000000018002c9f0 f   hb-font.obj
 0001:0002ba00       hb_font_funcs_set_draw_glyph_func 000000018002ca00 f   hb-font.obj
 0001:0002bb30       hb_font_funcs_set_font_h_extents_func 000000018002cb30 f   hb-font.obj
 0001:0002bc50       hb_font_funcs_set_font_v_extents_func 000000018002cc50 f   hb-font.obj
 0001:0002bd70       hb_font_funcs_set_glyph_contour_point_func 000000018002cd70 f   hb-font.obj
 0001:0002be90       hb_font_funcs_set_glyph_extents_func 000000018002ce90 f   hb-font.obj
 0001:0002bfb0       hb_font_funcs_set_glyph_from_name_func 000000018002cfb0 f   hb-font.obj
 0001:0002c0e0       hb_font_funcs_set_glyph_h_advance_func 000000018002d0e0 f   hb-font.obj
 0001:0002c200       hb_font_funcs_set_glyph_h_advances_func 000000018002d200 f   hb-font.obj
 0001:0002c320       hb_font_funcs_set_glyph_h_kerning_func 000000018002d320 f   hb-font.obj
 0001:0002c440       hb_font_funcs_set_glyph_h_origin_func 000000018002d440 f   hb-font.obj
 0001:0002c560       hb_font_funcs_set_glyph_name_func 000000018002d560 f   hb-font.obj
 0001:0002c680       hb_font_funcs_set_glyph_v_advance_func 000000018002d680 f   hb-font.obj
 0001:0002c7a0       hb_font_funcs_set_glyph_v_advances_func 000000018002d7a0 f   hb-font.obj
 0001:0002c8c0       hb_font_funcs_set_glyph_v_kerning_func 000000018002d8c0 f   hb-font.obj
 0001:0002c9e0       hb_font_funcs_set_glyph_v_origin_func 000000018002d9e0 f   hb-font.obj
 0001:0002cb00       hb_font_funcs_set_nominal_glyph_func 000000018002db00 f   hb-font.obj
 0001:0002cc20       hb_font_funcs_set_nominal_glyphs_func 000000018002dc20 f   hb-font.obj
 0001:0002cd40       hb_font_funcs_set_paint_glyph_func 000000018002dd40 f   hb-font.obj
 0001:0002ce70       hb_font_funcs_set_variation_glyph_func 000000018002de70 f   hb-font.obj
 0001:0002cf90       hb_font_get_face           000000018002df90 f   hb-font.obj
 0001:0002cfa0       hb_font_get_glyph          000000018002dfa0 f   hb-font.obj
 0001:0002d020       hb_font_get_glyph_extents  000000018002e020 f   hb-font.obj
 0001:0002d060       hb_font_get_glyph_h_advance 000000018002e060 f   hb-font.obj
 0001:0002d0a0       hb_font_get_nominal_glyph  000000018002e0a0 f   hb-font.obj
 0001:0002d0e0       hb_font_set_funcs          000000018002e0e0 f   hb-font.obj
 0001:0002d1a0       hb_font_set_scale          000000018002e1a0 f   hb-font.obj
 0001:0002d1d0       hb_font_set_var_coords_normalized 000000018002e1d0 f   hb-font.obj
 0001:0002d550       hb_font_set_variations     000000018002e550 f   hb-font.obj
 0001:0002d970       ?CallIntMethod@JNIEnv_@@QEAAJPEAV_jobject@@PEAU_jmethodID@@ZZ 000000018002e970 f i hb-jdk-font.obj
 0001:0002d9a0       ?CallObjectMethod@JNIEnv_@@QEAAPEAV_jobject@@PEAV2@PEAU_jmethodID@@ZZ 000000018002e9a0 f i hb-jdk-font.obj
 0001:0002de00       Java_sun_font_SunLayoutEngine_createFace 000000018002ee00 f   hb-jdk-font.obj
 0001:0002dea0       Java_sun_font_SunLayoutEngine_disposeFace 000000018002eea0 f   hb-jdk-font.obj
 0001:0002deb0       hb_jdk_font_create         000000018002eeb0 f   hb-jdk-font.obj
 0001:0002e040       ?hb_parse_double@@YA_NPEAPEBDPEBDPEAN_N@Z 000000018002f040 f   hb-number.obj
 0001:0002e0b0       ?hb_parse_int@@YA_NPEAPEBDPEBDPEAH_N@Z 000000018002f0b0 f   hb-number.obj
 0001:0002e480       ??$?0$$CBUaccelerator_t@cff1@OT@@@cff1_cs_interp_env_t@CFF@@QEAA@AEBU?$hb_array_t@$$CBE@@AEBUaccelerator_t@cff1@OT@@IPEBHI@Z 000000018002f480 f i hb-ot-cff1-table.obj
 0001:0002e680       ??0?$cff_stack_t@Ucall_context_t@CFF@@$09@CFF@@QEAA@XZ 000000018002f680 f i hb-ot-cff1-table.obj
 0001:0002e740       ??A?$CFFIndex@U?$IntType@G$01@OT@@@CFF@@QEBA?AU?$hb_array_t@$$CBE@@I@Z 000000018002f740 f i hb-ot-cff1-table.obj
 0001:0002eb70       ?call_subr@?$cs_interp_env_t@Unumber_t@CFF@@U?$Subrs@U?$IntType@G$01@OT@@@2@@CFF@@QEAAXAEBU?$biased_subrs_t@U?$Subrs@U?$IntType@G$01@OT@@@CFF@@@2@W4cs_type_t@2@@Z 000000018002fb70 f i hb-ot-cff1-table.obj
 0001:0002ed00       ?check_width@?$cff1_cs_opset_t@Ucff1_cs_opset_extents_t@@Ucff1_extents_param_t@@Ucff1_path_procs_extents_t@@@CFF@@SAXIAEAUcff1_cs_interp_env_t@2@AEAUcff1_extents_param_t@@@Z 000000018002fd00 f i hb-ot-cff1-table.obj
 0001:0002ed00       ?check_width@?$cff1_cs_opset_t@Ucff1_cs_opset_path_t@@Ucff1_path_param_t@@Ucff1_path_procs_path_t@@@CFF@@SAXIAEAUcff1_cs_interp_env_t@2@AEAUcff1_path_param_t@@@Z 000000018002fd00 f i hb-ot-cff1-table.obj
 0001:0002edd0       ?cubic_to@hb_draw_session_t@@QEAAXMMMMMM@Z 000000018002fdd0 f i hb-ot-cff1-table.obj
 0001:0002ee80       ?curve@cff1_path_procs_extents_t@@SAXAEAUcff1_cs_interp_env_t@CFF@@AEAUcff1_extents_param_t@@AEBUpoint_t@3@22@Z 000000018002fe80 f i hb-ot-cff1-table.obj
 0001:0002f040       ?curve@cff1_path_procs_path_t@@SAXAEAUcff1_cs_interp_env_t@CFF@@AEAUcff1_path_param_t@@AEBUpoint_t@3@22@Z 0000000180030040 f i hb-ot-cff1-table.obj
 0001:0002f1a0       ?flex1@?$path_procs_t@Ucff1_path_procs_extents_t@@Ucff1_cs_interp_env_t@CFF@@Ucff1_extents_param_t@@@CFF@@SAXAEAUcff1_cs_interp_env_t@2@AEAUcff1_extents_param_t@@@Z 00000001800301a0 f i hb-ot-cff1-table.obj
 0001:0002f4f0       ?flex1@?$path_procs_t@Ucff1_path_procs_path_t@@Ucff1_cs_interp_env_t@CFF@@Ucff1_path_param_t@@@CFF@@SAXAEAUcff1_cs_interp_env_t@2@AEAUcff1_path_param_t@@@Z 00000001800304f0 f i hb-ot-cff1-table.obj
 0001:0002f840       ?flex@?$path_procs_t@Ucff1_path_procs_extents_t@@Ucff1_cs_interp_env_t@CFF@@Ucff1_extents_param_t@@@CFF@@SAXAEAUcff1_cs_interp_env_t@2@AEAUcff1_extents_param_t@@@Z 0000000180030840 f i hb-ot-cff1-table.obj
 0001:0002faf0       ?flex@?$path_procs_t@Ucff1_path_procs_path_t@@Ucff1_cs_interp_env_t@CFF@@Ucff1_path_param_t@@@CFF@@SAXAEAUcff1_cs_interp_env_t@2@AEAUcff1_path_param_t@@@Z 0000000180030af0 f i hb-ot-cff1-table.obj
 0001:0002fda0       ?get_extents@accelerator_t@cff1@OT@@QEBA_NPEAUhb_font_t@@IPEAUhb_glyph_extents_t@@@Z 0000000180030da0 f   hb-ot-cff1-table.obj
 0001:00030010       ?get_fd@FDSelect@CFF@@QEBAII@Z 0000000180031010 f i hb-ot-cff1-table.obj
 0001:00030140       ?get_glyph@Charset@CFF@@QEBAIII@Z 0000000180031140 f i hb-ot-cff1-table.obj
 0001:000302e0       ?get_path@accelerator_t@cff1@OT@@QEBA_NPEAUhb_font_t@@IAEAUhb_draw_session_t@@@Z 00000001800312e0 f   hb-ot-cff1-table.obj
 0001:00030300       ?hflex1@?$path_procs_t@Ucff1_path_procs_extents_t@@Ucff1_cs_interp_env_t@CFF@@Ucff1_extents_param_t@@@CFF@@SAXAEAUcff1_cs_interp_env_t@2@AEAUcff1_extents_param_t@@@Z 0000000180031300 f i hb-ot-cff1-table.obj
 0001:00030550       ?hflex1@?$path_procs_t@Ucff1_path_procs_path_t@@Ucff1_cs_interp_env_t@CFF@@Ucff1_path_param_t@@@CFF@@SAXAEAUcff1_cs_interp_env_t@2@AEAUcff1_path_param_t@@@Z 0000000180031550 f i hb-ot-cff1-table.obj
 0001:000307a0       ?hflex@?$path_procs_t@Ucff1_path_procs_extents_t@@Ucff1_cs_interp_env_t@CFF@@Ucff1_extents_param_t@@@CFF@@SAXAEAUcff1_cs_interp_env_t@2@AEAUcff1_extents_param_t@@@Z 00000001800317a0 f i hb-ot-cff1-table.obj
 0001:000309a0       ?hflex@?$path_procs_t@Ucff1_path_procs_path_t@@Ucff1_cs_interp_env_t@CFF@@Ucff1_path_param_t@@@CFF@@SAXAEAUcff1_cs_interp_env_t@2@AEAUcff1_path_param_t@@@Z 00000001800319a0 f i hb-ot-cff1-table.obj
 0001:00030ba0       ?hhcurveto@?$path_procs_t@Ucff1_path_procs_extents_t@@Ucff1_cs_interp_env_t@CFF@@Ucff1_extents_param_t@@@CFF@@SAXAEAUcff1_cs_interp_env_t@2@AEAUcff1_extents_param_t@@@Z 0000000180031ba0 f i hb-ot-cff1-table.obj
 0001:00030eb0       ?hhcurveto@?$path_procs_t@Ucff1_path_procs_path_t@@Ucff1_cs_interp_env_t@CFF@@Ucff1_path_param_t@@@CFF@@SAXAEAUcff1_cs_interp_env_t@2@AEAUcff1_path_param_t@@@Z 0000000180031eb0 f i hb-ot-cff1-table.obj
 0001:00031130       ?hlineto@?$path_procs_t@Ucff1_path_procs_extents_t@@Ucff1_cs_interp_env_t@CFF@@Ucff1_extents_param_t@@@CFF@@SAXAEAUcff1_cs_interp_env_t@2@AEAUcff1_extents_param_t@@@Z 0000000180032130 f i hb-ot-cff1-table.obj
 0001:000314b0       ?hlineto@?$path_procs_t@Ucff1_path_procs_path_t@@Ucff1_cs_interp_env_t@CFF@@Ucff1_path_param_t@@@CFF@@SAXAEAUcff1_cs_interp_env_t@2@AEAUcff1_path_param_t@@@Z 00000001800324b0 f i hb-ot-cff1-table.obj
 0001:00031710       ?hvcurveto@?$path_procs_t@Ucff1_path_procs_extents_t@@Ucff1_cs_interp_env_t@CFF@@Ucff1_extents_param_t@@@CFF@@SAXAEAUcff1_cs_interp_env_t@2@AEAUcff1_extents_param_t@@@Z 0000000180032710 f i hb-ot-cff1-table.obj
 0001:00032470       ?hvcurveto@?$path_procs_t@Ucff1_path_procs_path_t@@Ucff1_cs_interp_env_t@CFF@@Ucff1_path_param_t@@@CFF@@SAXAEAUcff1_cs_interp_env_t@2@AEAUcff1_path_param_t@@@Z 0000000180033470 f i hb-ot-cff1-table.obj
 0001:00032db0       ?in_error@?$interp_env_t@Unumber_t@CFF@@@CFF@@QEBA_NXZ 0000000180033db0 f i hb-ot-cff1-table.obj
 0001:00032dd0       ?interpret@?$cs_interpreter_t@Ucff1_cs_interp_env_t@CFF@@Ucff1_cs_opset_extents_t@@Ucff1_extents_param_t@@@CFF@@QEAA_NAEAUcff1_extents_param_t@@@Z 0000000180033dd0 f i hb-ot-cff1-table.obj
 0001:00032f40       ?interpret@?$cs_interpreter_t@Ucff1_cs_interp_env_t@CFF@@Ucff1_cs_opset_path_t@@Ucff1_path_param_t@@@CFF@@QEAA_NAEAUcff1_path_param_t@@@Z 0000000180033f40 f i hb-ot-cff1-table.obj
 0001:000330b0       ?lookup_expert_charset_for_glyph@cff1@OT@@KAII@Z 00000001800340b0 f   hb-ot-cff1-table.obj
 0001:000330f0       ?lookup_expert_charset_for_sid@cff1@OT@@KAII@Z 00000001800340f0 f   hb-ot-cff1-table.obj
 0001:00033110       ?lookup_expert_subset_charset_for_glyph@cff1@OT@@KAII@Z 0000000180034110 f   hb-ot-cff1-table.obj
 0001:00033150       ?lookup_expert_subset_charset_for_sid@cff1@OT@@KAII@Z 0000000180034150 f   hb-ot-cff1-table.obj
 0001:00033170       ?merge@bounds_t@@QEAAXAEBU1@@Z 0000000180034170 f i hb-ot-cff1-table.obj
 0001:00033210       ?move_to@hb_draw_session_t@@QEAAXMM@Z 0000000180034210 f i hb-ot-cff1-table.obj
 0001:00033270       ?moveto@cff1_path_procs_path_t@@SAXAEAUcff1_cs_interp_env_t@CFF@@AEAUcff1_path_param_t@@AEBUpoint_t@3@@Z 0000000180034270 f i hb-ot-cff1-table.obj
 0001:00033330       ?offset_at@?$CFFIndex@U?$IntType@G$01@OT@@@CFF@@AEBAII@Z 0000000180034330 f i hb-ot-cff1-table.obj
 0001:000333b0       ?process_op@?$cs_opset_t@Unumber_t@CFF@@Ucff1_cs_opset_extents_t@@Ucff1_cs_interp_env_t@2@Ucff1_extents_param_t@@Ucff1_path_procs_extents_t@@@CFF@@SAXIAEAUcff1_cs_interp_env_t@2@AEAUcff1_extents_param_t@@@Z 00000001800343b0 f i hb-ot-cff1-table.obj
 0001:00033990       ?process_op@?$cs_opset_t@Unumber_t@CFF@@Ucff1_cs_opset_path_t@@Ucff1_cs_interp_env_t@2@Ucff1_path_param_t@@Ucff1_path_procs_path_t@@@CFF@@SAXIAEAUcff1_cs_interp_env_t@2@AEAUcff1_path_param_t@@@Z 0000000180034990 f i hb-ot-cff1-table.obj
 0001:00034030       ?process_op@?$opset_t@Unumber_t@CFF@@@CFF@@SAXIAEAU?$interp_env_t@Unumber_t@CFF@@@2@@Z 0000000180035030 f i hb-ot-cff1-table.obj
 0001:00034320       ?process_post_move@?$cs_opset_t@Unumber_t@CFF@@Ucff1_cs_opset_extents_t@@Ucff1_cs_interp_env_t@2@Ucff1_extents_param_t@@Ucff1_path_procs_extents_t@@@CFF@@SAXIAEAUcff1_cs_interp_env_t@2@AEAUcff1_extents_param_t@@@Z 0000000180035320 f i hb-ot-cff1-table.obj
 0001:00034320       ?process_post_move@?$cs_opset_t@Unumber_t@CFF@@Ucff1_cs_opset_path_t@@Ucff1_cs_interp_env_t@2@Ucff1_path_param_t@@Ucff1_path_procs_path_t@@@CFF@@SAXIAEAUcff1_cs_interp_env_t@2@AEAUcff1_path_param_t@@@Z 0000000180035320 f i hb-ot-cff1-table.obj
 0001:000343b0       ?process_seac@cff1_cs_opset_extents_t@@SAXAEAUcff1_cs_interp_env_t@CFF@@AEAUcff1_extents_param_t@@@Z 00000001800353b0 f i hb-ot-cff1-table.obj
 0001:00034660       ?process_seac@cff1_cs_opset_path_t@@SAXAEAUcff1_cs_interp_env_t@CFF@@AEAUcff1_path_param_t@@@Z 0000000180035660 f i hb-ot-cff1-table.obj
 0001:00034880       ?push_fixed_from_substr@?$arg_stack_t@Unumber_t@CFF@@@CFF@@QEAA_NAEAUbyte_str_ref_t@2@@Z 0000000180035880 f i hb-ot-cff1-table.obj
 0001:00034920       ?push_int@?$arg_stack_t@Unumber_t@CFF@@@CFF@@QEAAXH@Z 0000000180035920 f i hb-ot-cff1-table.obj
 0001:00034950       ?rcurveline@?$path_procs_t@Ucff1_path_procs_extents_t@@Ucff1_cs_interp_env_t@CFF@@Ucff1_extents_param_t@@@CFF@@SAXAEAUcff1_cs_interp_env_t@2@AEAUcff1_extents_param_t@@@Z 0000000180035950 f i hb-ot-cff1-table.obj
 0001:00034df0       ?rcurveline@?$path_procs_t@Ucff1_path_procs_path_t@@Ucff1_cs_interp_env_t@CFF@@Ucff1_path_param_t@@@CFF@@SAXAEAUcff1_cs_interp_env_t@2@AEAUcff1_path_param_t@@@Z 0000000180035df0 f i hb-ot-cff1-table.obj
 0001:000351b0       ?return_from_subr@?$cs_interp_env_t@Unumber_t@CFF@@U?$Subrs@U?$IntType@G$01@OT@@@2@@CFF@@QEAAXXZ 00000001800361b0 f i hb-ot-cff1-table.obj
 0001:000351b0       ?return_from_subr@?$cs_interp_env_t@Unumber_t@CFF@@U?$Subrs@U?$IntType@I$03@OT@@@2@@CFF@@QEAAXXZ 00000001800361b0 f i hb-ot-cff2-table.obj
 0001:00035230       ?rlinecurve@?$path_procs_t@Ucff1_path_procs_extents_t@@Ucff1_cs_interp_env_t@CFF@@Ucff1_extents_param_t@@@CFF@@SAXAEAUcff1_cs_interp_env_t@2@AEAUcff1_extents_param_t@@@Z 0000000180036230 f i hb-ot-cff1-table.obj
 0001:000356e0       ?rlinecurve@?$path_procs_t@Ucff1_path_procs_path_t@@Ucff1_cs_interp_env_t@CFF@@Ucff1_path_param_t@@@CFF@@SAXAEAUcff1_cs_interp_env_t@2@AEAUcff1_path_param_t@@@Z 00000001800366e0 f i hb-ot-cff1-table.obj
 0001:000359c0       ?rlineto@?$path_procs_t@Ucff1_path_procs_extents_t@@Ucff1_cs_interp_env_t@CFF@@Ucff1_extents_param_t@@@CFF@@SAXAEAUcff1_cs_interp_env_t@2@AEAUcff1_extents_param_t@@@Z 00000001800369c0 f i hb-ot-cff1-table.obj
 0001:00035b50       ?rrcurveto@?$path_procs_t@Ucff1_path_procs_extents_t@@Ucff1_cs_interp_env_t@CFF@@Ucff1_extents_param_t@@@CFF@@SAXAEAUcff1_cs_interp_env_t@2@AEAUcff1_extents_param_t@@@Z 0000000180036b50 f i hb-ot-cff1-table.obj
 0001:00035e80       ?rrcurveto@?$path_procs_t@Ucff1_path_procs_path_t@@Ucff1_cs_interp_env_t@CFF@@Ucff1_path_param_t@@@CFF@@SAXAEAUcff1_cs_interp_env_t@2@AEAUcff1_path_param_t@@@Z 0000000180036e80 f i hb-ot-cff1-table.obj
 0001:00036150       ?vhcurveto@?$path_procs_t@Ucff1_path_procs_extents_t@@Ucff1_cs_interp_env_t@CFF@@Ucff1_extents_param_t@@@CFF@@SAXAEAUcff1_cs_interp_env_t@2@AEAUcff1_extents_param_t@@@Z 0000000180037150 f i hb-ot-cff1-table.obj
 0001:00036ea0       ?vhcurveto@?$path_procs_t@Ucff1_path_procs_path_t@@Ucff1_cs_interp_env_t@CFF@@Ucff1_path_param_t@@@CFF@@SAXAEAUcff1_cs_interp_env_t@2@AEAUcff1_path_param_t@@@Z 0000000180037ea0 f i hb-ot-cff1-table.obj
 0001:000377f0       ?vlineto@?$path_procs_t@Ucff1_path_procs_extents_t@@Ucff1_cs_interp_env_t@CFF@@Ucff1_extents_param_t@@@CFF@@SAXAEAUcff1_cs_interp_env_t@2@AEAUcff1_extents_param_t@@@Z 00000001800387f0 f i hb-ot-cff1-table.obj
 0001:00037b70       ?vlineto@?$path_procs_t@Ucff1_path_procs_path_t@@Ucff1_cs_interp_env_t@CFF@@Ucff1_path_param_t@@@CFF@@SAXAEAUcff1_cs_interp_env_t@2@AEAUcff1_path_param_t@@@Z 0000000180038b70 f i hb-ot-cff1-table.obj
 0001:00037dd0       ?vvcurveto@?$path_procs_t@Ucff1_path_procs_extents_t@@Ucff1_cs_interp_env_t@CFF@@Ucff1_extents_param_t@@@CFF@@SAXAEAUcff1_cs_interp_env_t@2@AEAUcff1_extents_param_t@@@Z 0000000180038dd0 f i hb-ot-cff1-table.obj
 0001:000380e0       ?vvcurveto@?$path_procs_t@Ucff1_path_procs_path_t@@Ucff1_cs_interp_env_t@CFF@@Ucff1_path_param_t@@@CFF@@SAXAEAUcff1_cs_interp_env_t@2@AEAUcff1_path_param_t@@@Z 00000001800390e0 f i hb-ot-cff1-table.obj
 0001:00038390       ??$?0$$CBUaccelerator_t@cff2@OT@@@?$cff2_cs_interp_env_t@Unumber_t@CFF@@@CFF@@QEAA@AEBU?$hb_array_t@$$CBE@@AEBUaccelerator_t@cff2@OT@@IPEBHI@Z 0000000180039390 f i hb-ot-cff2-table.obj
 0001:00038650       ??A?$CFFIndex@U?$IntType@I$03@OT@@@CFF@@QEBA?AU?$hb_array_t@$$CBE@@I@Z 0000000180039650 f i hb-ot-cff2-table.obj
 0001:00038820       ?blend_deltas@?$cff2_cs_interp_env_t@Unumber_t@CFF@@@CFF@@QEBANU?$hb_array_t@$$CBUnumber_t@CFF@@@@@Z 0000000180039820 f i hb-ot-cff2-table.obj
 0001:00038960       ?call_subr@?$cs_interp_env_t@Unumber_t@CFF@@U?$Subrs@U?$IntType@I$03@OT@@@2@@CFF@@QEAAXAEBU?$biased_subrs_t@U?$Subrs@U?$IntType@I$03@OT@@@CFF@@@2@W4cs_type_t@2@@Z 0000000180039960 f i hb-ot-cff2-table.obj
 0001:00038b10       ?curve@cff2_path_procs_extents_t@@SAXAEAU?$cff2_cs_interp_env_t@Unumber_t@CFF@@@CFF@@AEAUcff2_extents_param_t@@AEBUpoint_t@3@22@Z 0000000180039b10 f i hb-ot-cff2-table.obj
 0001:00038cc0       ?flex1@?$path_procs_t@Ucff2_path_procs_extents_t@@U?$cff2_cs_interp_env_t@Unumber_t@CFF@@@CFF@@Ucff2_extents_param_t@@@CFF@@SAXAEAU?$cff2_cs_interp_env_t@Unumber_t@CFF@@@2@AEAUcff2_extents_param_t@@@Z 0000000180039cc0 f i hb-ot-cff2-table.obj
 0001:00039020       ?flex1@?$path_procs_t@Ucff2_path_procs_path_t@@U?$cff2_cs_interp_env_t@Unumber_t@CFF@@@CFF@@Ucff2_path_param_t@@@CFF@@SAXAEAU?$cff2_cs_interp_env_t@Unumber_t@CFF@@@2@AEAUcff2_path_param_t@@@Z 000000018003a020 f i hb-ot-cff2-table.obj
 0001:00039560       ?flex@?$path_procs_t@Ucff2_path_procs_extents_t@@U?$cff2_cs_interp_env_t@Unumber_t@CFF@@@CFF@@Ucff2_extents_param_t@@@CFF@@SAXAEAU?$cff2_cs_interp_env_t@Unumber_t@CFF@@@2@AEAUcff2_extents_param_t@@@Z 000000018003a560 f i hb-ot-cff2-table.obj
 0001:00039810       ?flex@?$path_procs_t@Ucff2_path_procs_path_t@@U?$cff2_cs_interp_env_t@Unumber_t@CFF@@@CFF@@Ucff2_path_param_t@@@CFF@@SAXAEAU?$cff2_cs_interp_env_t@Unumber_t@CFF@@@2@AEAUcff2_path_param_t@@@Z 000000018003a810 f i hb-ot-cff2-table.obj
 0001:00039ca0       ?get_extents@accelerator_t@cff2@OT@@QEBA_NPEAUhb_font_t@@IPEAUhb_glyph_extents_t@@@Z 000000018003aca0 f   hb-ot-cff2-table.obj
 0001:0003a230       ?get_fd@CFF2FDSelect@CFF@@QEBAII@Z 000000018003b230 f i hb-ot-cff2-table.obj
 0001:0003a490       ?get_path@accelerator_t@cff2@OT@@QEBA_NPEAUhb_font_t@@IAEAUhb_draw_session_t@@@Z 000000018003b490 f   hb-ot-cff2-table.obj
 0001:0003a7f0       ?get_region_scalars@VarData@OT@@QEBAXPEBHIAEBUVarRegionList@2@PEAMI@Z 000000018003b7f0 f i hb-ot-cff2-table.obj
 0001:0003aa50       ?hflex1@?$path_procs_t@Ucff2_path_procs_extents_t@@U?$cff2_cs_interp_env_t@Unumber_t@CFF@@@CFF@@Ucff2_extents_param_t@@@CFF@@SAXAEAU?$cff2_cs_interp_env_t@Unumber_t@CFF@@@2@AEAUcff2_extents_param_t@@@Z 000000018003ba50 f i hb-ot-cff2-table.obj
 0001:0003aca0       ?hflex1@?$path_procs_t@Ucff2_path_procs_path_t@@U?$cff2_cs_interp_env_t@Unumber_t@CFF@@@CFF@@Ucff2_path_param_t@@@CFF@@SAXAEAU?$cff2_cs_interp_env_t@Unumber_t@CFF@@@2@AEAUcff2_path_param_t@@@Z 000000018003bca0 f i hb-ot-cff2-table.obj
 0001:0003b060       ?hflex@?$path_procs_t@Ucff2_path_procs_extents_t@@U?$cff2_cs_interp_env_t@Unumber_t@CFF@@@CFF@@Ucff2_extents_param_t@@@CFF@@SAXAEAU?$cff2_cs_interp_env_t@Unumber_t@CFF@@@2@AEAUcff2_extents_param_t@@@Z 000000018003c060 f i hb-ot-cff2-table.obj
 0001:0003b260       ?hflex@?$path_procs_t@Ucff2_path_procs_path_t@@U?$cff2_cs_interp_env_t@Unumber_t@CFF@@@CFF@@Ucff2_path_param_t@@@CFF@@SAXAEAU?$cff2_cs_interp_env_t@Unumber_t@CFF@@@2@AEAUcff2_path_param_t@@@Z 000000018003c260 f i hb-ot-cff2-table.obj
 0001:0003b5c0       ?hhcurveto@?$path_procs_t@Ucff2_path_procs_extents_t@@U?$cff2_cs_interp_env_t@Unumber_t@CFF@@@CFF@@Ucff2_extents_param_t@@@CFF@@SAXAEAU?$cff2_cs_interp_env_t@Unumber_t@CFF@@@2@AEAUcff2_extents_param_t@@@Z 000000018003c5c0 f i hb-ot-cff2-table.obj
 0001:0003b8e0       ?hhcurveto@?$path_procs_t@Ucff2_path_procs_path_t@@U?$cff2_cs_interp_env_t@Unumber_t@CFF@@@CFF@@Ucff2_path_param_t@@@CFF@@SAXAEAU?$cff2_cs_interp_env_t@Unumber_t@CFF@@@2@AEAUcff2_path_param_t@@@Z 000000018003c8e0 f i hb-ot-cff2-table.obj
 0001:0003bb30       ?hlineto@?$path_procs_t@Ucff2_path_procs_extents_t@@U?$cff2_cs_interp_env_t@Unumber_t@CFF@@@CFF@@Ucff2_extents_param_t@@@CFF@@SAXAEAU?$cff2_cs_interp_env_t@Unumber_t@CFF@@@2@AEAUcff2_extents_param_t@@@Z 000000018003cb30 f i hb-ot-cff2-table.obj
 0001:0003beb0       ?hlineto@?$path_procs_t@Ucff2_path_procs_path_t@@U?$cff2_cs_interp_env_t@Unumber_t@CFF@@@CFF@@Ucff2_path_param_t@@@CFF@@SAXAEAU?$cff2_cs_interp_env_t@Unumber_t@CFF@@@2@AEAUcff2_path_param_t@@@Z 000000018003ceb0 f i hb-ot-cff2-table.obj
 0001:0003c0e0       ?hvcurveto@?$path_procs_t@Ucff2_path_procs_extents_t@@U?$cff2_cs_interp_env_t@Unumber_t@CFF@@@CFF@@Ucff2_extents_param_t@@@CFF@@SAXAEAU?$cff2_cs_interp_env_t@Unumber_t@CFF@@@2@AEAUcff2_extents_param_t@@@Z 000000018003d0e0 f i hb-ot-cff2-table.obj
 0001:0003ce30       ?hvcurveto@?$path_procs_t@Ucff2_path_procs_path_t@@U?$cff2_cs_interp_env_t@Unumber_t@CFF@@@CFF@@Ucff2_path_param_t@@@CFF@@SAXAEAU?$cff2_cs_interp_env_t@Unumber_t@CFF@@@2@AEAUcff2_path_param_t@@@Z 000000018003de30 f i hb-ot-cff2-table.obj
 0001:0003d720       ?in_error@?$cs_interp_env_t@Unumber_t@CFF@@U?$Subrs@U?$IntType@I$03@OT@@@2@@CFF@@QEBA_NXZ 000000018003e720 f i hb-ot-cff2-table.obj
 0001:0003d740       ?offset_at@?$CFFIndex@U?$IntType@I$03@OT@@@CFF@@AEBAII@Z 000000018003e740 f i hb-ot-cff2-table.obj
 0001:0003d7c0       ?pop_uint@?$arg_stack_t@Unumber_t@CFF@@@CFF@@QEAAIXZ 000000018003e7c0 f i hb-ot-cff2-table.obj
 0001:0003d800       ?process_blend@?$cff2_cs_interp_env_t@Unumber_t@CFF@@@CFF@@QEAAXXZ 000000018003e800 f i hb-ot-cff2-table.obj
 0001:0003dae0       ?process_op@?$cs_opset_t@Unumber_t@CFF@@Ucff2_cs_opset_extents_t@@U?$cff2_cs_interp_env_t@Unumber_t@CFF@@@2@Ucff2_extents_param_t@@Ucff2_path_procs_extents_t@@@CFF@@SAXIAEAU?$cff2_cs_interp_env_t@Unumber_t@CFF@@@2@AEAUcff2_extents_param_t@@@Z 000000018003eae0 f i hb-ot-cff2-table.obj
 0001:0003e250       ?process_op@?$cs_opset_t@Unumber_t@CFF@@Ucff2_cs_opset_path_t@@U?$cff2_cs_interp_env_t@Unumber_t@CFF@@@2@Ucff2_path_param_t@@Ucff2_path_procs_path_t@@@CFF@@SAXIAEAU?$cff2_cs_interp_env_t@Unumber_t@CFF@@@2@AEAUcff2_path_param_t@@@Z 000000018003f250 f i hb-ot-cff2-table.obj
 0001:0003e940       ?process_vsindex@?$cff2_cs_interp_env_t@Unumber_t@CFF@@@CFF@@QEAAXXZ 000000018003f940 f i hb-ot-cff2-table.obj
 0001:0003e9b0       ?rcurveline@?$path_procs_t@Ucff2_path_procs_extents_t@@U?$cff2_cs_interp_env_t@Unumber_t@CFF@@@CFF@@Ucff2_extents_param_t@@@CFF@@SAXAEAU?$cff2_cs_interp_env_t@Unumber_t@CFF@@@2@AEAUcff2_extents_param_t@@@Z 000000018003f9b0 f i hb-ot-cff2-table.obj
 0001:0003ee70       ?rcurveline@?$path_procs_t@Ucff2_path_procs_path_t@@U?$cff2_cs_interp_env_t@Unumber_t@CFF@@@CFF@@Ucff2_path_param_t@@@CFF@@SAXAEAU?$cff2_cs_interp_env_t@Unumber_t@CFF@@@2@AEAUcff2_path_param_t@@@Z 000000018003fe70 f i hb-ot-cff2-table.obj
 0001:0003f1d0       ?rlinecurve@?$path_procs_t@Ucff2_path_procs_extents_t@@U?$cff2_cs_interp_env_t@Unumber_t@CFF@@@CFF@@Ucff2_extents_param_t@@@CFF@@SAXAEAU?$cff2_cs_interp_env_t@Unumber_t@CFF@@@2@AEAUcff2_extents_param_t@@@Z 00000001800401d0 f i hb-ot-cff2-table.obj
 0001:0003f690       ?rlinecurve@?$path_procs_t@Ucff2_path_procs_path_t@@U?$cff2_cs_interp_env_t@Unumber_t@CFF@@@CFF@@Ucff2_path_param_t@@@CFF@@SAXAEAU?$cff2_cs_interp_env_t@Unumber_t@CFF@@@2@AEAUcff2_path_param_t@@@Z 0000000180040690 f i hb-ot-cff2-table.obj
 0001:0003fa00       ?rrcurveto@?$path_procs_t@Ucff2_path_procs_extents_t@@U?$cff2_cs_interp_env_t@Unumber_t@CFF@@@CFF@@Ucff2_extents_param_t@@@CFF@@SAXAEAU?$cff2_cs_interp_env_t@Unumber_t@CFF@@@2@AEAUcff2_extents_param_t@@@Z 0000000180040a00 f i hb-ot-cff2-table.obj
 0001:0003fd40       ?rrcurveto@?$path_procs_t@Ucff2_path_procs_path_t@@U?$cff2_cs_interp_env_t@Unumber_t@CFF@@@CFF@@Ucff2_path_param_t@@@CFF@@SAXAEAU?$cff2_cs_interp_env_t@Unumber_t@CFF@@@2@AEAUcff2_path_param_t@@@Z 0000000180040d40 f i hb-ot-cff2-table.obj
 0001:0003ffd0       ?vhcurveto@?$path_procs_t@Ucff2_path_procs_extents_t@@U?$cff2_cs_interp_env_t@Unumber_t@CFF@@@CFF@@Ucff2_extents_param_t@@@CFF@@SAXAEAU?$cff2_cs_interp_env_t@Unumber_t@CFF@@@2@AEAUcff2_extents_param_t@@@Z 0000000180040fd0 f i hb-ot-cff2-table.obj
 0001:00040d10       ?vhcurveto@?$path_procs_t@Ucff2_path_procs_path_t@@U?$cff2_cs_interp_env_t@Unumber_t@CFF@@@CFF@@Ucff2_path_param_t@@@CFF@@SAXAEAU?$cff2_cs_interp_env_t@Unumber_t@CFF@@@2@AEAUcff2_path_param_t@@@Z 0000000180041d10 f i hb-ot-cff2-table.obj
 0001:00041600       ?vlineto@?$path_procs_t@Ucff2_path_procs_extents_t@@U?$cff2_cs_interp_env_t@Unumber_t@CFF@@@CFF@@Ucff2_extents_param_t@@@CFF@@SAXAEAU?$cff2_cs_interp_env_t@Unumber_t@CFF@@@2@AEAUcff2_extents_param_t@@@Z 0000000180042600 f i hb-ot-cff2-table.obj
 0001:00041980       ?vlineto@?$path_procs_t@Ucff2_path_procs_path_t@@U?$cff2_cs_interp_env_t@Unumber_t@CFF@@@CFF@@Ucff2_path_param_t@@@CFF@@SAXAEAU?$cff2_cs_interp_env_t@Unumber_t@CFF@@@2@AEAUcff2_path_param_t@@@Z 0000000180042980 f i hb-ot-cff2-table.obj
 0001:00041bb0       ?vvcurveto@?$path_procs_t@Ucff2_path_procs_extents_t@@U?$cff2_cs_interp_env_t@Unumber_t@CFF@@@CFF@@Ucff2_extents_param_t@@@CFF@@SAXAEAU?$cff2_cs_interp_env_t@Unumber_t@CFF@@@2@AEAUcff2_extents_param_t@@@Z 0000000180042bb0 f i hb-ot-cff2-table.obj
 0001:00041ed0       ?vvcurveto@?$path_procs_t@Ucff2_path_procs_path_t@@U?$cff2_cs_interp_env_t@Unumber_t@CFF@@@CFF@@Ucff2_path_param_t@@@CFF@@SAXAEAU?$cff2_cs_interp_env_t@Unumber_t@CFF@@@2@AEAUcff2_path_param_t@@@Z 0000000180042ed0 f i hb-ot-cff2-table.obj
 0001:00042130       ??$dispatch@Uhb_sanitize_context_t@@$$V@Paint@OT@@QEBA_NPEAUhb_sanitize_context_t@@@Z 0000000180043130 f i hb-ot-color.obj
 0001:000425d0       ??$sanitize@$$V@?$OffsetTo@U?$ColorLine@UNoVariable@OT@@@OT@@U?$IntType@I$02@2@$00@OT@@QEBA_NPEAUhb_sanitize_context_t@@PEBX@Z 00000001800435d0 f i hb-ot-color.obj
 0001:000426c0       ??$sanitize@$$V@?$OffsetTo@U?$ColorLine@UVariable@OT@@@OT@@U?$IntType@I$02@2@$00@OT@@QEBA_NPEAUhb_sanitize_context_t@@PEBX@Z 00000001800436c0 f i hb-ot-color.obj
 0001:000427b0       ??$sanitize@$$V@?$OffsetTo@UBaseGlyphList@OT@@U?$IntType@I$03@2@$00@OT@@QEBA_NPEAUhb_sanitize_context_t@@PEBX@Z 00000001800437b0 f i hb-ot-color.obj
 0001:00042920       ??$sanitize@$$V@?$OffsetTo@ULayerList@OT@@U?$IntType@I$03@2@$00@OT@@QEBA_NPEAUhb_sanitize_context_t@@PEBX@Z 0000000180043920 f i hb-ot-color.obj
 0001:00042a70       ??$sanitize@$$V@?$OffsetTo@UPaint@OT@@U?$IntType@I$02@2@$00@OT@@QEBA_NPEAUhb_sanitize_context_t@@PEBX@Z 0000000180043a70 f i hb-ot-color.obj
 0001:00042b10       ??$sanitize@$$V@?$OffsetTo@UPaint@OT@@U?$IntType@I$03@2@$00@OT@@QEBA_NPEAUhb_sanitize_context_t@@PEBX@Z 0000000180043b10 f i hb-ot-color.obj
 0001:00042be0       ??$sanitize@$$V@Paint@OT@@QEBA_NPEAUhb_sanitize_context_t@@@Z 0000000180043be0 f i hb-ot-color.obj
 0001:00042c10       ??$sanitize@I@?$OffsetTo@UIndexSubtable@OT@@U?$IntType@I$03@2@$00@OT@@QEBA_NPEAUhb_sanitize_context_t@@PEBX$$QEAI@Z 0000000180043c10 f i hb-ot-color.obj
 0001:00042d60       ??$sanitize@PEBUClipList@OT@@@?$ArrayOf@UClipRecord@OT@@U?$IntType@I$03@2@@OT@@QEBA_NPEAUhb_sanitize_context_t@@$$QEAPEBUClipList@1@@Z 0000000180043d60 f i hb-ot-color.obj
 0001:00042f40       ??$sanitize@PEBUsbix@OT@@@?$ArrayOf@U?$OffsetTo@USBIXStrike@OT@@U?$IntType@I$03@2@$00@OT@@U?$IntType@I$03@2@@OT@@QEBA_NPEAUhb_sanitize_context_t@@$$QEAPEBUsbix@1@@Z 0000000180043f40 f i hb-ot-color.obj
 0001:000430d0       ??$sanitize_blob@UCBDT@OT@@@hb_sanitize_context_t@@QEAAPEAUhb_blob_t@@PEAU1@@Z 00000001800440d0 f i hb-ot-color.obj
 0001:000433c0       ??$sanitize_blob@UCBLC@OT@@@hb_sanitize_context_t@@QEAAPEAUhb_blob_t@@PEAU1@@Z 00000001800443c0 f i hb-ot-color.obj
 0001:00043730       ??$sanitize_blob@UCOLR@OT@@@hb_sanitize_context_t@@QEAAPEAUhb_blob_t@@PEAU1@@Z 0000000180044730 f i hb-ot-color.obj
 0001:000438c0       ??$sanitize_blob@UCPAL@OT@@@hb_sanitize_context_t@@QEAAPEAUhb_blob_t@@PEAU1@@Z 00000001800448c0 f i hb-ot-color.obj
 0001:00043cf0       ??$sanitize_blob@USVG@OT@@@hb_sanitize_context_t@@QEAAPEAUhb_blob_t@@PEAU1@@Z 0000000180044cf0 f i hb-ot-color.obj
 0001:00044000       ??$sanitize_blob@Usbix@OT@@@hb_sanitize_context_t@@QEAAPEAUhb_blob_t@@PEAU1@@Z 0000000180045000 f i hb-ot-color.obj
 0001:00044330       ??C?$hb_lazy_loader_t@UCOLR@OT@@U?$hb_table_lazy_loader_t@UCOLR@OT@@$0CD@$00@@Uhb_face_t@@$0CD@Uhb_blob_t@@@@QEBAPEBUCOLR@OT@@XZ 0000000180045330 f i hb-ot-color.obj
 0001:00044420       ??C?$hb_lazy_loader_t@UCPAL@OT@@U?$hb_table_lazy_loader_t@UCPAL@OT@@$0CE@$00@@Uhb_face_t@@$0CE@Uhb_blob_t@@@@QEBAPEBUCPAL@OT@@XZ 0000000180045420 f i hb-ot-color.obj
 0001:00044510       ??C?$hb_lazy_loader_t@Usbix_accelerator_t@OT@@U?$hb_face_lazy_loader_t@Usbix_accelerator_t@OT@@$0CG@@@Uhb_face_t@@$0CG@U12@@@QEBAPEBUsbix_accelerator_t@OT@@XZ 0000000180045510 f i hb-ot-color.obj
 0001:00044630       ?choose_strike@CBLC@OT@@IEBAAEBUBitmapSizeTable@2@PEAUhb_font_t@@@Z 0000000180045630 f i hb-ot-color.obj
 0001:00044730       ?choose_strike@accelerator_t@sbix@OT@@AEBAAEBUSBIXStrike@3@PEAUhb_font_t@@@Z 0000000180045730 f i hb-ot-color.obj
 0001:00044910       ?find_table@IndexSubtableArray@OT@@QEBAPEBUIndexSubtableRecord@2@II@Z 0000000180045910 f i hb-ot-color.obj
 0001:000449c0       ?get_base_glyph_paint@COLR@OT@@QEBAPEBUPaint@2@I@Z 00000001800459c0 f i hb-ot-color.obj
 0001:00044af0       ?get_glyph_blob@SBIXStrike@OT@@QEBAPEAUhb_blob_t@@IPEAU3@IPEAH1IPEAI@Z 0000000180045af0 f i hb-ot-color.obj
 0001:00044e40       ?get_image_data@IndexSubtable@OT@@QEBA_NIPEAI00@Z 0000000180045e40 f i hb-ot-color.obj
 0001:000450d0       ?get_palette_colors@CPAL@OT@@QEBAIIIPEAI0@Z 00000001800460d0 f i hb-ot-color.obj
 0001:000452e0       ?get_stored@?$hb_lazy_loader_t@UCBDT_accelerator_t@OT@@U?$hb_face_lazy_loader_t@UCBDT_accelerator_t@OT@@$0CF@@@Uhb_face_t@@$0CF@U12@@@QEBAPEAUCBDT_accelerator_t@OT@@XZ 00000001800462e0 f i hb-ot-color.obj
 0001:00045470       ?get_strike@sbix@OT@@QEBAAEBUSBIXStrike@2@I@Z 0000000180046470 f i hb-ot-color.obj
 0001:00045520       ?reference_blob_for_glyph@accelerator_t@SVG@OT@@QEBAPEAUhb_blob_t@@I@Z 0000000180046520 f i hb-ot-color.obj
 0001:00045680       ?reference_png@accelerator_t@CBDT@OT@@QEBAPEAUhb_blob_t@@PEAUhb_font_t@@I@Z 0000000180046680 f i hb-ot-color.obj
 0001:00045930       ?sanitize@BitmapSizeTable@OT@@QEBA_NPEAUhb_sanitize_context_t@@PEBX@Z 0000000180046930 f i hb-ot-color.obj
 0001:00045af0       ?sanitize@CBLC@OT@@QEBA_NPEAUhb_sanitize_context_t@@@Z 0000000180046af0 f i hb-ot-color.obj
 0001:00045c20       ?sanitize@COLR@OT@@QEBA_NPEAUhb_sanitize_context_t@@@Z 0000000180046c20 f i hb-ot-color.obj
 0001:00045e90       ?sanitize@CPAL@OT@@QEBA_NPEAUhb_sanitize_context_t@@@Z 0000000180046e90 f i hb-ot-color.obj
 0001:00046060       ?sanitize@SVG@OT@@QEBA_NPEAUhb_sanitize_context_t@@@Z 0000000180047060 f i hb-ot-color.obj
 0001:00046120       hb_ot_color_palette_get_colors 0000000180047120 f   hb-ot-color.obj
 0001:00046170       ??1?$accelerator_templ_t@Ucff1_private_dict_opset_t@CFF@@U?$cff1_private_dict_values_base_t@Udict_val_t@CFF@@@2@@cff1@OT@@QEAA@XZ 0000000180047170 f i hb-ot-face.obj
 0001:00046220       ??1?$accelerator_templ_t@Ucff2_private_dict_opset_t@CFF@@U?$cff2_private_dict_values_base_t@Udict_val_t@CFF@@@2@@cff2@OT@@QEAA@XZ 0000000180047220 f i hb-ot-face.obj
 0001:000462c0       ?_fini@?$accelerator_templ_t@Ucff2_private_dict_opset_t@CFF@@U?$cff2_private_dict_values_base_t@Udict_val_t@CFF@@@2@@cff2@OT@@QEAAXXZ 00000001800472c0 f i hb-ot-face.obj
 0001:00046370       ?fini@?$accelerator_templ_t@Ucff1_private_dict_opset_t@CFF@@U?$cff1_private_dict_values_base_t@Udict_val_t@CFF@@@2@@cff1@OT@@QEAAXXZ 0000000180047370 f i hb-ot-face.obj
 0001:00046430       ?fini@hb_ot_face_t@@QEAAXXZ 0000000180047430 f   hb-ot-face.obj
 0001:00046bb0       ?init0@hb_ot_face_t@@QEAAXPEAUhb_face_t@@@Z 0000000180047bb0 f   hb-ot-face.obj
 0001:00046bc0       ?shrink_vector@?$hb_vector_t@U?$cff1_private_dict_values_base_t@Udict_val_t@CFF@@@CFF@@$0A@@@QEAAXI@Z 0000000180047bc0 f i hb-ot-face.obj
 0001:00046bc0       ?shrink_vector@?$hb_vector_t@Ucff1_font_dict_values_t@CFF@@$0A@@@QEAAXI@Z 0000000180047bc0 f i hb-ot-face.obj
 0001:00046bc0       ?shrink_vector@?$hb_vector_t@Ucff2_font_dict_values_t@CFF@@$0A@@@QEAAXI@Z 0000000180047bc0 f i hb-ot-face.obj
 0001:00046c50       ?shrink_vector@?$hb_vector_t@U?$cff2_private_dict_values_base_t@Udict_val_t@CFF@@@CFF@@$0A@@@QEAAXI@Z 0000000180047c50 f i hb-ot-face.obj
 0001:00046ce0       ??$check_array@U?$IntType@E$00@OT@@@hb_sanitize_context_t@@QEBA_NPEBU?$IntType@E$00@OT@@II@Z 0000000180047ce0 f i hb-ot-font.obj
 0001:00046d30       ??$dispatch@Uhb_paint_context_t@OT@@$$V@Paint@OT@@QEBA?AUhb_empty_t@@PEAUhb_paint_context_t@1@@Z 0000000180047d30 f i hb-ot-font.obj
 0001:00047390       ??$get_extents_without_var_scaled@Uglyf_accelerator_t@OT@@@GlyphHeader@glyf_impl@OT@@QEBA_NPEAUhb_font_t@@AEBUglyf_accelerator_t@2@IPEAUhb_glyph_extents_t@@@Z 0000000180048390 f i hb-ot-font.obj
 0001:00047610       ??$push@Uhb_bounds_t@@U1@$0A@@?$hb_vector_t@Uhb_bounds_t@@$0A@@@QEAAPEAUhb_bounds_t@@$$QEAU1@@Z 0000000180048610 f i hb-ot-font.obj
 0001:000476f0       ??$realloc_vector@U?$cff2_private_dict_values_base_t@Udict_val_t@CFF@@@CFF@@$0A@@?$hb_vector_t@U?$cff2_private_dict_values_base_t@Udict_val_t@CFF@@@CFF@@$0A@@@QEAAPEAU?$cff2_private_dict_values_base_t@Udict_val_t@CFF@@@CFF@@I@Z 00000001800486f0 f i hb-ot-font.obj
 0001:00047830       ??$sanitize_blob@UVORG@OT@@@hb_sanitize_context_t@@QEAAPEAUhb_blob_t@@PEAU1@@Z 0000000180048830 f i hb-ot-font.obj
 0001:00047b30       ??$sanitize_blob@Ucff1@OT@@@hb_sanitize_context_t@@QEAAPEAUhb_blob_t@@PEAU1@@Z 0000000180048b30 f i hb-ot-font.obj
 0001:00047df0       ??$sanitize_blob@Ucff2@OT@@@hb_sanitize_context_t@@QEAAPEAUhb_blob_t@@PEAU1@@Z 0000000180048df0 f i hb-ot-font.obj
 0001:000480b0       ??$sanitize_blob@Upost@OT@@@hb_sanitize_context_t@@QEAAPEAUhb_blob_t@@PEAU1@@Z 00000001800490b0 f i hb-ot-font.obj
 0001:00048790       ??0?$accelerator_templ_t@Ucff2_private_dict_opset_t@CFF@@U?$cff2_private_dict_values_base_t@Udict_val_t@CFF@@@2@@cff2@OT@@QEAA@PEAUhb_face_t@@@Z 0000000180049790 f i hb-ot-font.obj
 0001:00049350       ??0accelerator_t@post@OT@@QEAA@PEAUhb_face_t@@@Z 000000018004a350 f i hb-ot-font.obj
 0001:00049610       ??0hb_paint_extents_context_t@@QEAA@XZ 000000018004a610 f i hb-ot-font.obj
 0001:00049890       ??1hb_paint_extents_context_t@@QEAA@XZ 000000018004a890 f i hb-ot-font.obj
 0001:00049910       ??C?$hb_lazy_loader_t@Ucff2_accelerator_t@OT@@U?$hb_face_lazy_loader_t@Ucff2_accelerator_t@OT@@$0BB@@@Uhb_face_t@@$0BB@U12@@@QEBAPEBUcff2_accelerator_t@OT@@XZ 000000018004a910 f i hb-ot-font.obj
 0001:000499c0       ??C?$hb_lazy_loader_t@Upost_accelerator_t@OT@@U?$hb_face_lazy_loader_t@Upost_accelerator_t@OT@@$06@@Uhb_face_t@@$06U12@@@QEBAPEBUpost_accelerator_t@OT@@XZ 000000018004a9c0 f i hb-ot-font.obj
 0001:00049ad0       ?add_op@?$parsed_values_t@Udict_val_t@CFF@@@CFF@@QEAAXIAEBUbyte_str_ref_t@2@AEBUdict_val_t@2@@Z 000000018004aad0 f i hb-ot-font.obj
 0001:00049ad0       ?add_op@?$parsed_values_t@Uop_str_t@CFF@@@CFF@@QEAAXIAEBUbyte_str_ref_t@2@AEBUop_str_t@2@@Z 000000018004aad0 f i hb-ot-font.obj
 0001:00049bf0       ?alloc@?$hb_vector_t@U?$cff1_private_dict_values_base_t@Udict_val_t@CFF@@@CFF@@$0A@@@QEAA_NI_N@Z 000000018004abf0 f i hb-ot-font.obj
 0001:00049db0       ?alloc@?$hb_vector_t@Ucff1_font_dict_values_t@CFF@@$0A@@@QEAA_NI_N@Z 000000018004adb0 f i hb-ot-font.obj
 0001:00049f80       ?alloc@?$hb_vector_t@Ucff2_font_dict_values_t@CFF@@$0A@@@QEAA_NI_N@Z 000000018004af80 f i hb-ot-font.obj
 0001:0004a140       ?cmp@gname_t@accelerator_t@cff1@OT@@SAHPEBX0@Z 000000018004b140 f i hb-ot-font.obj
 0001:0004a180       ?cmp_gids@accelerator_t@post@OT@@KAHPEBX0PEAX@Z 000000018004b180 f i hb-ot-font.obj
 0001:0004a210       ?consume_point@path_builder_t@glyf_impl@OT@@QEAAXAEBUcontour_point_t@3@@Z 000000018004b210 f i hb-ot-font.obj
 0001:0004a6a0       ?find_glyph_name@accelerator_t@post@OT@@IEBA?AU?$hb_array_t@$$CBD@@I@Z 000000018004b6a0 f i hb-ot-font.obj
 0001:0004a7a0       ?get_advance_delta_unscaled@HVARVVAR@OT@@QEBAMIPEBHIPEAM@Z 000000018004b7a0 f i hb-ot-font.obj
 0001:0004a850       ?get_base_glyph_record@COLR@OT@@QEBAPEBUBaseGlyphRecord@2@I@Z 000000018004b850 f i hb-ot-font.obj
 0001:0004a900       ?get_clip_box@ClipBoxFormat2@OT@@QEBAXAEAUClipBoxData@2@AEBUVarStoreInstancer@2@@Z 000000018004b900 f i hb-ot-font.obj
 0001:0004aba0       ?get_color@hb_paint_context_t@OT@@QEAAIIMPEAH@Z 000000018004bba0 f i hb-ot-font.obj
 0001:0004ac80       ?get_color_stop@ColorStop@OT@@QEBAXPEAUhb_paint_context_t@2@PEAUhb_color_stop_t@@IAEBUVarStoreInstancer@2@@Z 000000018004bc80 f i hb-ot-font.obj
 0001:0004adc0       ?get_extents@COLR@OT@@QEBA_NPEAUhb_font_t@@IPEAUhb_glyph_extents_t@@@Z 000000018004bdc0 f i hb-ot-font.obj
 0001:0004b050       ?get_extents@ClipList@OT@@QEBA_NIPEAUhb_glyph_extents_t@@AEBUVarStoreInstancer@2@@Z 000000018004c050 f i hb-ot-font.obj
 0001:0004b1e0       ?get_extents@accelerator_t@CBDT@OT@@QEBA_NPEAUhb_font_t@@IPEAUhb_glyph_extents_t@@_N@Z 000000018004c1e0 f i hb-ot-font.obj
 0001:0004b4e0       ?get_extents@glyf_accelerator_t@OT@@QEBA_NPEAUhb_font_t@@IPEAUhb_glyph_extents_t@@@Z 000000018004c4e0 f i hb-ot-font.obj
 0001:0004b5c0       ?get_glyph@VariationSelectorRecord@OT@@QEBA?AW4glyph_variant_t@2@IPEAIPEBX@Z 000000018004c5c0 f i hb-ot-font.obj
 0001:0004b760       ?get_glyph_from_name@accelerator_t@cff1@OT@@QEBA_NPEBDHPEAI@Z 000000018004c760 f i hb-ot-font.obj
 0001:0004bb70       ?get_glyph_from_name@accelerator_t@post@OT@@QEBA_NPEBDHPEAI@Z 000000018004cb70 f i hb-ot-font.obj
 0001:0004bcf0       ?get_nominal_glyph@accelerator_t@cmap@OT@@QEBA_NIPEAIPEAU?$hb_cache_t@$0BF@$0BA@$07$00@@@Z 000000018004ccf0 f i hb-ot-font.obj
 0001:0004bda0       ?get_png_extents@accelerator_t@sbix@OT@@AEBA_NPEAUhb_font_t@@IPEAUhb_glyph_extents_t@@_N@Z 000000018004cda0 f i hb-ot-font.obj
 0001:0004bfd0       ?get_sid@Charset@CFF@@QEBAIII@Z 000000018004cfd0 f i hb-ot-font.obj
 0001:0004c100       ?get_size@?$CFFIndex@U?$IntType@G$01@OT@@@CFF@@QEBAIXZ 000000018004d100 f i hb-ot-font.obj
 0001:0004c1e0       ?get_stored@?$hb_lazy_loader_t@Ucff1_accelerator_t@OT@@U?$hb_face_lazy_loader_t@Ucff1_accelerator_t@OT@@$0BA@@@Uhb_face_t@@$0BA@U12@@@QEBAPEAUcff1_accelerator_t@OT@@XZ 000000018004d1e0 f i hb-ot-font.obj
 0001:0004c370       ?glyph_to_sid@?$accelerator_templ_t@Ucff1_private_dict_opset_t@CFF@@U?$cff1_private_dict_values_base_t@Udict_val_t@CFF@@@2@@cff1@OT@@QEBAII@Z 000000018004d370 f i hb-ot-font.obj
 0001:0004dfe0       ?init@?$accelerator_templ_t@Ucff1_private_dict_opset_t@CFF@@U?$cff1_private_dict_values_base_t@Udict_val_t@CFF@@@2@@cff1@OT@@QEAAXPEAUhb_face_t@@@Z 000000018004efe0 f i hb-ot-font.obj
 0001:0004eb30       ?interpret@?$dict_interpreter_t@Ucff1_font_dict_opset_t@CFF@@Ucff1_font_dict_values_t@2@U?$interp_env_t@Unumber_t@CFF@@@2@@CFF@@QEAA_NAEAUcff1_font_dict_values_t@2@@Z 000000018004fb30 f i hb-ot-font.obj
 0001:0004ed40       ?interpret@?$dict_interpreter_t@Ucff1_private_dict_opset_t@CFF@@U?$cff1_private_dict_values_base_t@Udict_val_t@CFF@@@2@U?$interp_env_t@Unumber_t@CFF@@@2@@CFF@@QEAA_NAEAU?$cff1_private_dict_values_base_t@Udict_val_t@CFF@@@2@@Z 000000018004fd40 f i hb-ot-font.obj
 0001:0004ef40       ?interpret@?$dict_interpreter_t@Ucff2_font_dict_opset_t@CFF@@Ucff2_font_dict_values_t@2@U?$interp_env_t@Unumber_t@CFF@@@2@@CFF@@QEAA_NAEAUcff2_font_dict_values_t@2@@Z 000000018004ff40 f i hb-ot-font.obj
 0001:0004f100       ?interpret@?$dict_interpreter_t@Ucff2_private_dict_opset_t@CFF@@U?$cff2_private_dict_values_base_t@Udict_val_t@CFF@@@2@Ucff2_priv_dict_interp_env_t@2@@CFF@@QEAA_NAEAU?$cff2_private_dict_values_base_t@Udict_val_t@CFF@@@2@@Z 0000000180050100 f i hb-ot-font.obj
 0001:0004f390       ?paint_glyph@?$PaintLinearGradient@UNoVariable@OT@@@OT@@QEBAXPEAUhb_paint_context_t@2@I@Z 0000000180050390 f i hb-ot-font.obj
 0001:0004f750       ?paint_glyph@?$PaintLinearGradient@UVariable@OT@@@OT@@QEBAXPEAUhb_paint_context_t@2@I@Z 0000000180050750 f i hb-ot-font.obj
 0001:0004fb10       ?paint_glyph@?$PaintRadialGradient@UNoVariable@OT@@@OT@@QEBAXPEAUhb_paint_context_t@2@I@Z 0000000180050b10 f i hb-ot-font.obj
 0001:0004fee0       ?paint_glyph@?$PaintRadialGradient@UVariable@OT@@@OT@@QEBAXPEAUhb_paint_context_t@2@I@Z 0000000180050ee0 f i hb-ot-font.obj
 0001:000502b0       ?paint_glyph@?$PaintSweepGradient@UNoVariable@OT@@@OT@@QEBAXPEAUhb_paint_context_t@2@I@Z 00000001800512b0 f i hb-ot-font.obj
 0001:00050580       ?paint_glyph@?$PaintSweepGradient@UVariable@OT@@@OT@@QEBAXPEAUhb_paint_context_t@2@I@Z 0000000180051580 f i hb-ot-font.obj
 0001:00050850       ?paint_glyph@Affine2x3@OT@@QEBAXPEAUhb_paint_context_t@2@I@Z 0000000180051850 f i hb-ot-font.obj
 0001:00050bc0       ?paint_glyph@COLR@OT@@QEBA_NPEAUhb_font_t@@IPEAUhb_paint_funcs_t@@PEAXII_N@Z 0000000180051bc0 f i hb-ot-font.obj
 0001:000511f0       ?paint_glyph@PaintColrGlyph@OT@@QEBAXPEAUhb_paint_context_t@2@@Z 00000001800521f0 f i hb-ot-font.obj
 0001:00051360       ?paint_glyph@PaintColrLayers@OT@@QEBAXPEAUhb_paint_context_t@2@@Z 0000000180052360 f i hb-ot-font.obj
 0001:00051530       ?paint_glyph@PaintGlyph@OT@@QEBAXPEAUhb_paint_context_t@2@@Z 0000000180052530 f i hb-ot-font.obj
 0001:00051700       ?paint_glyph@PaintRotate@OT@@QEBAXPEAUhb_paint_context_t@2@I@Z 0000000180052700 f i hb-ot-font.obj
 0001:00051800       ?paint_glyph@PaintRotateAroundCenter@OT@@QEBAXPEAUhb_paint_context_t@2@I@Z 0000000180052800 f i hb-ot-font.obj
 0001:00051b40       ?paint_glyph@PaintScale@OT@@QEBAXPEAUhb_paint_context_t@2@I@Z 0000000180052b40 f i hb-ot-font.obj
 0001:00051d10       ?paint_glyph@PaintScaleAroundCenter@OT@@QEBAXPEAUhb_paint_context_t@2@I@Z 0000000180052d10 f i hb-ot-font.obj
 0001:00052110       ?paint_glyph@PaintScaleUniform@OT@@QEBAXPEAUhb_paint_context_t@2@I@Z 0000000180053110 f i hb-ot-font.obj
 0001:00052260       ?paint_glyph@PaintScaleUniformAroundCenter@OT@@QEBAXPEAUhb_paint_context_t@2@I@Z 0000000180053260 f i hb-ot-font.obj
 0001:000525e0       ?paint_glyph@PaintSkew@OT@@QEBAXPEAUhb_paint_context_t@2@I@Z 00000001800535e0 f i hb-ot-font.obj
 0001:00052760       ?paint_glyph@PaintSkewAroundCenter@OT@@QEBAXPEAUhb_paint_context_t@2@I@Z 0000000180053760 f i hb-ot-font.obj
 0001:00052b10       ?paint_glyph@PaintSolid@OT@@QEBAXPEAUhb_paint_context_t@2@I@Z 0000000180053b10 f i hb-ot-font.obj
 0001:00052bf0       ?paint_glyph@PaintTranslate@OT@@QEBAXPEAUhb_paint_context_t@2@I@Z 0000000180053bf0 f i hb-ot-font.obj
 0001:00052dc0       ?parse_bcd@dict_opset_t@CFF@@SANAEAUbyte_str_ref_t@2@@Z 0000000180053dc0 f i hb-ot-font.obj
 0001:00052ef0       ?process_op@cff1_top_dict_opset_t@CFF@@SAXIAEAUcff1_top_dict_interp_env_t@2@AEAUcff1_top_dict_values_t@2@@Z 0000000180053ef0 f i hb-ot-font.obj
 0001:00053410       ?process_op@cff2_top_dict_opset_t@CFF@@SAXIAEAU?$interp_env_t@Unumber_t@CFF@@@2@AEAUcff2_top_dict_values_t@2@@Z 0000000180054410 f i hb-ot-font.obj
 0001:00053630       ?process_op@dict_opset_t@CFF@@SAXIAEAU?$interp_env_t@Unumber_t@CFF@@@2@@Z 0000000180054630 f i hb-ot-font.obj
 0001:00053760       ?push_root_transform@hb_paint_funcs_t@@QEAAXPEAXPEBUhb_font_t@@@Z 0000000180054760 f i hb-ot-font.obj
 0001:00053800       ?push_rotate@hb_paint_funcs_t@@QEAA_NPEAXM@Z 0000000180054800 f i hb-ot-font.obj
 0001:000538c0       ?push_skew@hb_paint_funcs_t@@QEAA_NPEAXMM@Z 00000001800548c0 f i hb-ot-font.obj
 0001:00053990       ?quadratic_to@hb_draw_session_t@@QEAAXMMMM@Z 0000000180054990 f i hb-ot-font.obj
 0001:000539f0       ?recurse@hb_paint_context_t@OT@@QEAAXAEBUPaint@2@@Z 00000001800549f0 f i hb-ot-font.obj
 0001:00053a30       ?sanitize@?$CFFIndex@U?$IntType@G$01@OT@@@CFF@@QEBA_NPEAUhb_sanitize_context_t@@@Z 0000000180054a30 f i hb-ot-font.obj
 0001:00053b40       ?sanitize@?$CFFIndex@U?$IntType@I$03@OT@@@CFF@@QEBA_NPEAUhb_sanitize_context_t@@@Z 0000000180054b40 f i hb-ot-font.obj
 0001:00053c70       ?sanitize@?$FDSelect3_4@U?$IntType@G$01@OT@@U?$IntType@E$00@2@@CFF@@QEBA_NPEAUhb_sanitize_context_t@@I@Z 0000000180054c70 f i hb-ot-font.obj
 0001:00053ec0       ?sanitize@?$FDSelect3_4@U?$IntType@I$03@OT@@U?$IntType@G$01@2@@CFF@@QEBA_NPEAUhb_sanitize_context_t@@I@Z 0000000180054ec0 f i hb-ot-font.obj
 0001:000541c0       ?sanitize@Charset@CFF@@QEBA_NPEAUhb_sanitize_context_t@@@Z 00000001800551c0 f i hb-ot-font.obj
 0001:00054450       ?sanitize@Encoding@CFF@@QEBA_NPEAUhb_sanitize_context_t@@@Z 0000000180055450 f i hb-ot-font.obj
 0001:00054590       ?sanitize@FDSelect0@CFF@@QEBA_NPEAUhb_sanitize_context_t@@I@Z 0000000180055590 f i hb-ot-font.obj
 0001:00054620       ?sanitize@VORG@OT@@QEBA_NPEAUhb_sanitize_context_t@@@Z 0000000180055620 f i hb-ot-font.obj
 0001:000546c0       ?sanitize@post@OT@@QEBA_NPEAUhb_sanitize_context_t@@@Z 00000001800556c0 f i hb-ot-font.obj
 0001:000547a0       ?static_get_color_stops@?$ColorLine@UNoVariable@OT@@@OT@@SAIPEAUhb_color_line_t@@PEAXIPEAIPEAUhb_color_stop_t@@1@Z 00000001800557a0 f i hb-ot-font.obj
 0001:000548a0       ?static_get_color_stops@?$ColorLine@UVariable@OT@@@OT@@SAIPEAUhb_color_line_t@@PEAXIPEAIPEAUhb_color_stop_t@@1@Z 00000001800558a0 f i hb-ot-font.obj
 0001:000549b0       ?static_get_extend@?$ColorLine@UNoVariable@OT@@@OT@@SA?AW4hb_paint_extend_t@@PEAUhb_color_line_t@@PEAX1@Z 00000001800559b0 f i hb-ot-font.obj
 0001:000549b0       ?static_get_extend@?$ColorLine@UVariable@OT@@@OT@@SA?AW4hb_paint_extend_t@@PEAUhb_color_line_t@@PEAX1@Z 00000001800559b0 f i hb-ot-font.obj
 0001:000549c0       hb_ot_font_set_funcs       00000001800559c0 f   hb-ot-font.obj
 0001:00054c10       ??$_dispatch@U?$ChainRule@USmallTypes@Layout@OT@@@OT@@$$V@hb_sanitize_context_t@@AEAA_NAEBU?$ChainRule@USmallTypes@Layout@OT@@@OT@@U?$hb_priority@$00@@@Z 0000000180055c10 f i hb-ot-layout.obj
 0001:00054d40       ??$apply@UGPOSProxy@@@hb_ot_map_t@@QEBAXAEBUGPOSProxy@@PEBUhb_ot_shape_plan_t@@PEAUhb_font_t@@PEAUhb_buffer_t@@@Z 0000000180055d40 f i hb-ot-layout.obj
 0001:000553c0       ??$apply@UGSUBProxy@@@hb_ot_map_t@@QEBAXAEBUGSUBProxy@@PEBUhb_ot_shape_plan_t@@PEAUhb_font_t@@PEAUhb_buffer_t@@@Z 00000001800563c0 f i hb-ot-layout.obj
 0001:00055af0       ??$apply_cached_to@U?$AlternateSubstFormat1_2@USmallTypes@Layout@OT@@@GSUB_impl@Layout@OT@@@hb_accelerate_subtables_context_t@OT@@SA_NPEBXPEAUhb_ot_apply_context_t@1@@Z 0000000180056af0 f i hb-ot-layout.obj
 0001:00055af0       ??$apply_to@U?$AlternateSubstFormat1_2@USmallTypes@Layout@OT@@@GSUB_impl@Layout@OT@@@hb_accelerate_subtables_context_t@OT@@SA_NPEBXPEAUhb_ot_apply_context_t@1@@Z 0000000180056af0 f i hb-ot-layout.obj
 0001:00055b00       ??$apply_cached_to@U?$ChainContextFormat1_4@USmallTypes@Layout@OT@@@OT@@@hb_accelerate_subtables_context_t@OT@@SA_NPEBXPEAUhb_ot_apply_context_t@1@@Z 0000000180056b00 f i hb-ot-layout.obj
 0001:00055b00       ??$apply_to@U?$ChainContextFormat1_4@USmallTypes@Layout@OT@@@OT@@@hb_accelerate_subtables_context_t@OT@@SA_NPEBXPEAUhb_ot_apply_context_t@1@@Z 0000000180056b00 f i hb-ot-layout.obj
 0001:00055b10       ??$apply_cached_to@U?$ChainContextFormat2_5@USmallTypes@Layout@OT@@@OT@@@hb_accelerate_subtables_context_t@OT@@SA_NPEBXPEAUhb_ot_apply_context_t@1@@Z 0000000180056b10 f i hb-ot-layout.obj
 0001:00055b20       ??$apply_cached_to@U?$ContextFormat1_4@USmallTypes@Layout@OT@@@OT@@@hb_accelerate_subtables_context_t@OT@@SA_NPEBXPEAUhb_ot_apply_context_t@1@@Z 0000000180056b20 f i hb-ot-layout.obj
 0001:00055b20       ??$apply_to@U?$ContextFormat1_4@USmallTypes@Layout@OT@@@OT@@@hb_accelerate_subtables_context_t@OT@@SA_NPEBXPEAUhb_ot_apply_context_t@1@@Z 0000000180056b20 f i hb-ot-layout.obj
 0001:00055b30       ??$apply_cached_to@U?$ContextFormat2_5@USmallTypes@Layout@OT@@@OT@@@hb_accelerate_subtables_context_t@OT@@SA_NPEBXPEAUhb_ot_apply_context_t@1@@Z 0000000180056b30 f i hb-ot-layout.obj
 0001:00055b40       ??$apply_cached_to@U?$LigatureSubstFormat1_2@USmallTypes@Layout@OT@@@GSUB_impl@Layout@OT@@@hb_accelerate_subtables_context_t@OT@@SA_NPEBXPEAUhb_ot_apply_context_t@1@@Z 0000000180056b40 f i hb-ot-layout.obj
 0001:00055b40       ??$apply_to@U?$LigatureSubstFormat1_2@USmallTypes@Layout@OT@@@GSUB_impl@Layout@OT@@@hb_accelerate_subtables_context_t@OT@@SA_NPEBXPEAUhb_ot_apply_context_t@1@@Z 0000000180056b40 f i hb-ot-layout.obj
 0001:00055b50       ??$apply_cached_to@U?$MarkBasePosFormat1_2@USmallTypes@Layout@OT@@@GPOS_impl@Layout@OT@@@hb_accelerate_subtables_context_t@OT@@SA_NPEBXPEAUhb_ot_apply_context_t@1@@Z 0000000180056b50 f i hb-ot-layout.obj
 0001:00055b50       ??$apply_to@U?$MarkBasePosFormat1_2@USmallTypes@Layout@OT@@@GPOS_impl@Layout@OT@@@hb_accelerate_subtables_context_t@OT@@SA_NPEBXPEAUhb_ot_apply_context_t@1@@Z 0000000180056b50 f i hb-ot-layout.obj
 0001:00055b60       ??$apply_cached_to@U?$MarkLigPosFormat1_2@USmallTypes@Layout@OT@@@GPOS_impl@Layout@OT@@@hb_accelerate_subtables_context_t@OT@@SA_NPEBXPEAUhb_ot_apply_context_t@1@@Z 0000000180056b60 f i hb-ot-layout.obj
 0001:00055b60       ??$apply_to@U?$MarkLigPosFormat1_2@USmallTypes@Layout@OT@@@GPOS_impl@Layout@OT@@@hb_accelerate_subtables_context_t@OT@@SA_NPEBXPEAUhb_ot_apply_context_t@1@@Z 0000000180056b60 f i hb-ot-layout.obj
 0001:00055b70       ??$apply_cached_to@U?$MarkMarkPosFormat1_2@USmallTypes@Layout@OT@@@GPOS_impl@Layout@OT@@@hb_accelerate_subtables_context_t@OT@@SA_NPEBXPEAUhb_ot_apply_context_t@1@@Z 0000000180056b70 f i hb-ot-layout.obj
 0001:00055b70       ??$apply_to@U?$MarkMarkPosFormat1_2@USmallTypes@Layout@OT@@@GPOS_impl@Layout@OT@@@hb_accelerate_subtables_context_t@OT@@SA_NPEBXPEAUhb_ot_apply_context_t@1@@Z 0000000180056b70 f i hb-ot-layout.obj
 0001:00055b80       ??$apply_cached_to@U?$MultipleSubstFormat1_2@USmallTypes@Layout@OT@@@GSUB_impl@Layout@OT@@@hb_accelerate_subtables_context_t@OT@@SA_NPEBXPEAUhb_ot_apply_context_t@1@@Z 0000000180056b80 f i hb-ot-layout.obj
 0001:00055b80       ??$apply_to@U?$MultipleSubstFormat1_2@USmallTypes@Layout@OT@@@GSUB_impl@Layout@OT@@@hb_accelerate_subtables_context_t@OT@@SA_NPEBXPEAUhb_ot_apply_context_t@1@@Z 0000000180056b80 f i hb-ot-layout.obj
 0001:00055b90       ??$apply_cached_to@U?$PairPosFormat1_3@USmallTypes@Layout@OT@@@GPOS_impl@Layout@OT@@@hb_accelerate_subtables_context_t@OT@@SA_NPEBXPEAUhb_ot_apply_context_t@1@@Z 0000000180056b90 f i hb-ot-layout.obj
 0001:00055b90       ??$apply_to@U?$PairPosFormat1_3@USmallTypes@Layout@OT@@@GPOS_impl@Layout@OT@@@hb_accelerate_subtables_context_t@OT@@SA_NPEBXPEAUhb_ot_apply_context_t@1@@Z 0000000180056b90 f i hb-ot-layout.obj
 0001:00055ba0       ??$apply_cached_to@U?$PairPosFormat2_4@USmallTypes@Layout@OT@@@GPOS_impl@Layout@OT@@@hb_accelerate_subtables_context_t@OT@@SA_NPEBXPEAUhb_ot_apply_context_t@1@@Z 0000000180056ba0 f i hb-ot-layout.obj
 0001:00055ba0       ??$apply_to@U?$PairPosFormat2_4@USmallTypes@Layout@OT@@@GPOS_impl@Layout@OT@@@hb_accelerate_subtables_context_t@OT@@SA_NPEBXPEAUhb_ot_apply_context_t@1@@Z 0000000180056ba0 f i hb-ot-layout.obj
 0001:00055bb0       ??$apply_cached_to@U?$SingleSubstFormat1_3@USmallTypes@Layout@OT@@@GSUB_impl@Layout@OT@@@hb_accelerate_subtables_context_t@OT@@SA_NPEBXPEAUhb_ot_apply_context_t@1@@Z 0000000180056bb0 f i hb-ot-layout.obj
 0001:00055bb0       ??$apply_to@U?$SingleSubstFormat1_3@USmallTypes@Layout@OT@@@GSUB_impl@Layout@OT@@@hb_accelerate_subtables_context_t@OT@@SA_NPEBXPEAUhb_ot_apply_context_t@1@@Z 0000000180056bb0 f i hb-ot-layout.obj
 0001:00055bc0       ??$apply_cached_to@U?$SingleSubstFormat2_4@USmallTypes@Layout@OT@@@GSUB_impl@Layout@OT@@@hb_accelerate_subtables_context_t@OT@@SA_NPEBXPEAUhb_ot_apply_context_t@1@@Z 0000000180056bc0 f i hb-ot-layout.obj
 0001:00055bc0       ??$apply_to@U?$SingleSubstFormat2_4@USmallTypes@Layout@OT@@@GSUB_impl@Layout@OT@@@hb_accelerate_subtables_context_t@OT@@SA_NPEBXPEAUhb_ot_apply_context_t@1@@Z 0000000180056bc0 f i hb-ot-layout.obj
 0001:00055bd0       ??$apply_cached_to@UChainContextFormat3@OT@@@hb_accelerate_subtables_context_t@OT@@SA_NPEBXPEAUhb_ot_apply_context_t@1@@Z 0000000180056bd0 f i hb-ot-layout.obj
 0001:00055bd0       ??$apply_to@UChainContextFormat3@OT@@@hb_accelerate_subtables_context_t@OT@@SA_NPEBXPEAUhb_ot_apply_context_t@1@@Z 0000000180056bd0 f i hb-ot-layout.obj
 0001:00055be0       ??$apply_cached_to@UContextFormat3@OT@@@hb_accelerate_subtables_context_t@OT@@SA_NPEBXPEAUhb_ot_apply_context_t@1@@Z 0000000180056be0 f i hb-ot-layout.obj
 0001:00055be0       ??$apply_to@UContextFormat3@OT@@@hb_accelerate_subtables_context_t@OT@@SA_NPEBXPEAUhb_ot_apply_context_t@1@@Z 0000000180056be0 f i hb-ot-layout.obj
 0001:00055bf0       ??$apply_cached_to@UCursivePosFormat1@GPOS_impl@Layout@OT@@@hb_accelerate_subtables_context_t@OT@@SA_NPEBXPEAUhb_ot_apply_context_t@1@@Z 0000000180056bf0 f i hb-ot-layout.obj
 0001:00055bf0       ??$apply_to@UCursivePosFormat1@GPOS_impl@Layout@OT@@@hb_accelerate_subtables_context_t@OT@@SA_NPEBXPEAUhb_ot_apply_context_t@1@@Z 0000000180056bf0 f i hb-ot-layout.obj
 0001:00055c00       ??$apply_cached_to@UReverseChainSingleSubstFormat1@GSUB_impl@Layout@OT@@@hb_accelerate_subtables_context_t@OT@@SA_NPEBXPEAUhb_ot_apply_context_t@1@@Z 0000000180056c00 f i hb-ot-layout.obj
 0001:00055c00       ??$apply_to@UReverseChainSingleSubstFormat1@GSUB_impl@Layout@OT@@@hb_accelerate_subtables_context_t@OT@@SA_NPEBXPEAUhb_ot_apply_context_t@1@@Z 0000000180056c00 f i hb-ot-layout.obj
 0001:00055c10       ??$apply_cached_to@USinglePosFormat1@GPOS_impl@Layout@OT@@@hb_accelerate_subtables_context_t@OT@@SA_NPEBXPEAUhb_ot_apply_context_t@1@@Z 0000000180056c10 f i hb-ot-layout.obj
 0001:00055c10       ??$apply_to@USinglePosFormat1@GPOS_impl@Layout@OT@@@hb_accelerate_subtables_context_t@OT@@SA_NPEBXPEAUhb_ot_apply_context_t@1@@Z 0000000180056c10 f i hb-ot-layout.obj
 0001:00055c20       ??$apply_cached_to@USinglePosFormat2@GPOS_impl@Layout@OT@@@hb_accelerate_subtables_context_t@OT@@SA_NPEBXPEAUhb_ot_apply_context_t@1@@Z 0000000180056c20 f i hb-ot-layout.obj
 0001:00055c20       ??$apply_to@USinglePosFormat2@GPOS_impl@Layout@OT@@@hb_accelerate_subtables_context_t@OT@@SA_NPEBXPEAUhb_ot_apply_context_t@1@@Z 0000000180056c20 f i hb-ot-layout.obj
 0001:00055db0       ??$apply_to@U?$ChainContextFormat2_5@USmallTypes@Layout@OT@@@OT@@@hb_accelerate_subtables_context_t@OT@@SA_NPEBXPEAUhb_ot_apply_context_t@1@@Z 0000000180056db0 f i hb-ot-layout.obj
 0001:00055dc0       ??$apply_to@U?$ContextFormat2_5@USmallTypes@Layout@OT@@@OT@@@hb_accelerate_subtables_context_t@OT@@SA_NPEBXPEAUhb_ot_apply_context_t@1@@Z 0000000180056dc0 f i hb-ot-layout.obj
 0001:00055dd0       ??$cache_func_to@U?$AlternateSubstFormat1_2@USmallTypes@Layout@OT@@@GSUB_impl@Layout@OT@@@hb_accelerate_subtables_context_t@OT@@SA_NPEBXPEAUhb_ot_apply_context_t@1@_N@Z 0000000180056dd0 f i hb-ot-layout.obj
 0001:00055dd0       ??$cache_func_to@U?$ChainContextFormat1_4@USmallTypes@Layout@OT@@@OT@@@hb_accelerate_subtables_context_t@OT@@SA_NPEBXPEAUhb_ot_apply_context_t@1@_N@Z 0000000180056dd0 f i hb-ot-layout.obj
 0001:00055dd0       ??$cache_func_to@U?$ContextFormat1_4@USmallTypes@Layout@OT@@@OT@@@hb_accelerate_subtables_context_t@OT@@SA_NPEBXPEAUhb_ot_apply_context_t@1@_N@Z 0000000180056dd0 f i hb-ot-layout.obj
 0001:00055dd0       ??$cache_func_to@U?$LigatureSubstFormat1_2@USmallTypes@Layout@OT@@@GSUB_impl@Layout@OT@@@hb_accelerate_subtables_context_t@OT@@SA_NPEBXPEAUhb_ot_apply_context_t@1@_N@Z 0000000180056dd0 f i hb-ot-layout.obj
 0001:00055dd0       ??$cache_func_to@U?$MarkBasePosFormat1_2@USmallTypes@Layout@OT@@@GPOS_impl@Layout@OT@@@hb_accelerate_subtables_context_t@OT@@SA_NPEBXPEAUhb_ot_apply_context_t@1@_N@Z 0000000180056dd0 f i hb-ot-layout.obj
 0001:00055dd0       ??$cache_func_to@U?$MarkLigPosFormat1_2@USmallTypes@Layout@OT@@@GPOS_impl@Layout@OT@@@hb_accelerate_subtables_context_t@OT@@SA_NPEBXPEAUhb_ot_apply_context_t@1@_N@Z 0000000180056dd0 f i hb-ot-layout.obj
 0001:00055dd0       ??$cache_func_to@U?$MarkMarkPosFormat1_2@USmallTypes@Layout@OT@@@GPOS_impl@Layout@OT@@@hb_accelerate_subtables_context_t@OT@@SA_NPEBXPEAUhb_ot_apply_context_t@1@_N@Z 0000000180056dd0 f i hb-ot-layout.obj
 0001:00055dd0       ??$cache_func_to@U?$MultipleSubstFormat1_2@USmallTypes@Layout@OT@@@GSUB_impl@Layout@OT@@@hb_accelerate_subtables_context_t@OT@@SA_NPEBXPEAUhb_ot_apply_context_t@1@_N@Z 0000000180056dd0 f i hb-ot-layout.obj
 0001:00055dd0       ??$cache_func_to@U?$PairPosFormat1_3@USmallTypes@Layout@OT@@@GPOS_impl@Layout@OT@@@hb_accelerate_subtables_context_t@OT@@SA_NPEBXPEAUhb_ot_apply_context_t@1@_N@Z 0000000180056dd0 f i hb-ot-layout.obj
 0001:00055dd0       ??$cache_func_to@U?$PairPosFormat2_4@USmallTypes@Layout@OT@@@GPOS_impl@Layout@OT@@@hb_accelerate_subtables_context_t@OT@@SA_NPEBXPEAUhb_ot_apply_context_t@1@_N@Z 0000000180056dd0 f i hb-ot-layout.obj
 0001:00055dd0       ??$cache_func_to@U?$SingleSubstFormat1_3@USmallTypes@Layout@OT@@@GSUB_impl@Layout@OT@@@hb_accelerate_subtables_context_t@OT@@SA_NPEBXPEAUhb_ot_apply_context_t@1@_N@Z 0000000180056dd0 f i hb-ot-layout.obj
 0001:00055dd0       ??$cache_func_to@U?$SingleSubstFormat2_4@USmallTypes@Layout@OT@@@GSUB_impl@Layout@OT@@@hb_accelerate_subtables_context_t@OT@@SA_NPEBXPEAUhb_ot_apply_context_t@1@_N@Z 0000000180056dd0 f i hb-ot-layout.obj
 0001:00055dd0       ??$cache_func_to@UChainContextFormat3@OT@@@hb_accelerate_subtables_context_t@OT@@SA_NPEBXPEAUhb_ot_apply_context_t@1@_N@Z 0000000180056dd0 f i hb-ot-layout.obj
 0001:00055dd0       ??$cache_func_to@UContextFormat3@OT@@@hb_accelerate_subtables_context_t@OT@@SA_NPEBXPEAUhb_ot_apply_context_t@1@_N@Z 0000000180056dd0 f i hb-ot-layout.obj
 0001:00055dd0       ??$cache_func_to@UCursivePosFormat1@GPOS_impl@Layout@OT@@@hb_accelerate_subtables_context_t@OT@@SA_NPEBXPEAUhb_ot_apply_context_t@1@_N@Z 0000000180056dd0 f i hb-ot-layout.obj
 0001:00055dd0       ??$cache_func_to@UReverseChainSingleSubstFormat1@GSUB_impl@Layout@OT@@@hb_accelerate_subtables_context_t@OT@@SA_NPEBXPEAUhb_ot_apply_context_t@1@_N@Z 0000000180056dd0 f i hb-ot-layout.obj
 0001:00055dd0       ??$cache_func_to@USinglePosFormat1@GPOS_impl@Layout@OT@@@hb_accelerate_subtables_context_t@OT@@SA_NPEBXPEAUhb_ot_apply_context_t@1@_N@Z 0000000180056dd0 f i hb-ot-layout.obj
 0001:00055dd0       ??$cache_func_to@USinglePosFormat2@GPOS_impl@Layout@OT@@@hb_accelerate_subtables_context_t@OT@@SA_NPEBXPEAUhb_ot_apply_context_t@1@_N@Z 0000000180056dd0 f i hb-ot-layout.obj
 0001:00055de0       ??$cache_func_to@U?$ChainContextFormat2_5@USmallTypes@Layout@OT@@@OT@@@hb_accelerate_subtables_context_t@OT@@SA_NPEBXPEAUhb_ot_apply_context_t@1@_N@Z 0000000180056de0 f i hb-ot-layout.obj
 0001:00055de0       ??$cache_func_to@U?$ContextFormat2_5@USmallTypes@Layout@OT@@@OT@@@hb_accelerate_subtables_context_t@OT@@SA_NPEBXPEAUhb_ot_apply_context_t@1@_N@Z 0000000180056de0 f i hb-ot-layout.obj
 0001:00055ff0       ??$collect_coverage@U?$hb_set_digest_combiner_t@U?$hb_set_digest_bits_pattern_t@K$03@@U?$hb_set_digest_combiner_t@U?$hb_set_digest_bits_pattern_t@K$0A@@@U?$hb_set_digest_bits_pattern_t@K$08@@@@@@@Coverage@Common@Layout@OT@@QEBA_NPEAU?$hb_set_digest_combiner_t@U?$hb_set_digest_bits_pattern_t@K$03@@U?$hb_set_digest_combiner_t@U?$hb_set_digest_bits_pattern_t@K$0A@@@U?$hb_set_digest_bits_pattern_t@K$08@@@@@@@Z 0000000180056ff0 f i hb-ot-layout.obj
 0001:00056320       ??$create@USubstLookup@GSUB_impl@Layout@OT@@@hb_ot_layout_lookup_accelerator_t@OT@@SAPEAU01@AEBUSubstLookup@GSUB_impl@Layout@1@@Z 0000000180057320 f i hb-ot-layout.obj
 0001:000564f0       ??$dispatch@U?$ChainContextFormat2_5@USmallTypes@Layout@OT@@@OT@@@hb_accelerate_subtables_context_t@OT@@QEAA?AUhb_empty_t@@AEBU?$ChainContextFormat2_5@USmallTypes@Layout@OT@@@1@@Z 00000001800574f0 f i hb-ot-layout.obj
 0001:00056630       ??$dispatch@U?$ContextFormat2_5@USmallTypes@Layout@OT@@@OT@@@hb_accelerate_subtables_context_t@OT@@QEAA?AUhb_empty_t@@AEBU?$ContextFormat2_5@USmallTypes@Layout@OT@@@1@@Z 0000000180057630 f i hb-ot-layout.obj
 0001:00056770       ??$dispatch@Uhb_accelerate_subtables_context_t@OT@@$$V@ChainContext@OT@@QEBA?AUhb_empty_t@@PEAUhb_accelerate_subtables_context_t@1@@Z 0000000180057770 f i hb-ot-layout.obj
 0001:000568c0       ??$dispatch@Uhb_accelerate_subtables_context_t@OT@@$$V@Context@OT@@QEBA?AUhb_empty_t@@PEAUhb_accelerate_subtables_context_t@1@@Z 00000001800578c0 f i hb-ot-layout.obj
 0001:00056a30       ??$dispatch@Uhb_accelerate_subtables_context_t@OT@@$$V@PosLookupSubTable@GPOS_impl@Layout@OT@@QEBA?AUhb_empty_t@@PEAUhb_accelerate_subtables_context_t@3@I@Z 0000000180057a30 f i hb-ot-layout.obj
 0001:00056e00       ??$dispatch@Uhb_accelerate_subtables_context_t@OT@@$$V@SubstLookupSubTable@GSUB_impl@Layout@OT@@QEBA?AUhb_empty_t@@PEAUhb_accelerate_subtables_context_t@3@I@Z 0000000180057e00 f i hb-ot-layout.obj
 0001:00057150       ??$dispatch@Uhb_sanitize_context_t@@$$V@?$KernSubTable@UKernAATSubTableHeader@OT@@@OT@@QEBA_NPEAUhb_sanitize_context_t@@@Z 0000000180058150 f i hb-ot-layout.obj
 0001:000572a0       ??$dispatch@Uhb_sanitize_context_t@@$$V@AlternateSubst@GSUB_impl@Layout@OT@@QEBA_NPEAUhb_sanitize_context_t@@@Z 00000001800582a0 f i hb-ot-layout.obj
 0001:000572a0       ??$dispatch@Uhb_sanitize_context_t@@$$V@MultipleSubst@GSUB_impl@Layout@OT@@QEBA_NPEAUhb_sanitize_context_t@@@Z 00000001800582a0 f i hb-ot-layout.obj
 0001:00057460       ??$dispatch@Uhb_sanitize_context_t@@$$V@ChainContext@OT@@QEBA_NPEAUhb_sanitize_context_t@@@Z 0000000180058460 f i hb-ot-layout.obj
 0001:00057700       ??$dispatch@Uhb_sanitize_context_t@@$$V@Context@OT@@QEBA_NPEAUhb_sanitize_context_t@@@Z 0000000180058700 f i hb-ot-layout.obj
 0001:00057990       ??$dispatch@Uhb_sanitize_context_t@@$$V@PosLookupSubTable@GPOS_impl@Layout@OT@@QEBA_NPEAUhb_sanitize_context_t@@I@Z 0000000180058990 f i hb-ot-layout.obj
 0001:00057da0       ??$dispatch@Uhb_sanitize_context_t@@$$V@SubstLookupSubTable@GSUB_impl@Layout@OT@@QEBA_NPEAUhb_sanitize_context_t@@I@Z 0000000180058da0 f i hb-ot-layout.obj
 0001:00058590       ??$dispatch@Uhb_would_apply_context_t@OT@@$$V@ChainContext@OT@@QEBA_NPEAUhb_would_apply_context_t@1@@Z 0000000180059590 f i hb-ot-layout.obj
 0001:00058890       ??$dispatch@Uhb_would_apply_context_t@OT@@$$V@Context@OT@@QEBA_NPEAUhb_would_apply_context_t@1@@Z 0000000180059890 f i hb-ot-layout.obj
 0001:00058aa0       ??$dispatch@Uhb_would_apply_context_t@OT@@$$V@SubstLookupSubTable@GSUB_impl@Layout@OT@@QEBA_NPEAUhb_would_apply_context_t@3@I@Z 0000000180059aa0 f i hb-ot-layout.obj
 0001:00058cd0       ??$dispatch_recurse_func@Uhb_ot_apply_context_t@OT@@@PosLookup@GPOS_impl@Layout@OT@@SA_NPEAUhb_ot_apply_context_t@3@I@Z 0000000180059cd0 f i hb-ot-layout.obj
 0001:00058df0       ??$dispatch_recurse_func@Uhb_ot_apply_context_t@OT@@@SubstLookup@GSUB_impl@Layout@OT@@SA_NPEAUhb_ot_apply_context_t@3@I@Z 0000000180059df0 f i hb-ot-layout.obj
 0001:00058f10       ??$drive@Udriver_context_t@?$KerxSubTableFormat1@UKernAATSubTableHeader@OT@@@AAT@@@?$StateTableDriver@UObsoleteTypes@AAT@@X@AAT@@QEAAXPEAUdriver_context_t@?$KerxSubTableFormat1@UKernAATSubTableHeader@OT@@@1@PEAUhb_aat_apply_context_t@1@@Z 0000000180059f10 f i hb-ot-layout.obj
 0001:000592f0       ??$get_subtable@UPosLookupSubTable@GPOS_impl@Layout@OT@@@Lookup@OT@@QEBAAEBUPosLookupSubTable@GPOS_impl@Layout@1@I@Z 000000018005a2f0 f i hb-ot-layout.obj
 0001:000592f0       ??$get_subtable@USubstLookupSubTable@GSUB_impl@Layout@OT@@@Lookup@OT@@QEBAAEBUSubstLookupSubTable@GSUB_impl@Layout@1@I@Z 000000018005a2f0 f i hb-ot-layout.obj
 0001:00059aa0       ??$sanitize@$$V@?$ArrayOf@ULookupRecord@OT@@U?$IntType@G$01@2@@OT@@QEBA_NPEAUhb_sanitize_context_t@@@Z 000000018005aaa0 f i hb-ot-layout.obj
 0001:00059b10       ??$sanitize@$$V@?$OffsetTo@U?$ChainRuleSet@USmallTypes@Layout@OT@@@OT@@U?$IntType@G$01@2@$00@OT@@QEBA_NPEAUhb_sanitize_context_t@@PEBX@Z 000000018005ab10 f i hb-ot-layout.obj
 0001:00059cb0       ??$sanitize@$$V@?$OffsetTo@U?$ClassTable@U?$IntType@G$01@OT@@@AAT@@U?$IntType@G$01@OT@@$0A@@OT@@QEBA_NPEAUhb_sanitize_context_t@@PEBX@Z 000000018005acb0 f i hb-ot-layout.obj
 0001:00059d40       ??$sanitize@$$V@?$OffsetTo@U?$List16OfOffsetTo@UPosLookup@GPOS_impl@Layout@OT@@U?$IntType@G$01@4@@OT@@U?$IntType@G$01@2@$00@OT@@QEBA_NPEAUhb_sanitize_context_t@@PEBX@Z 000000018005ad40 f i hb-ot-layout.obj
 0001:00059ed0       ??$sanitize@$$V@?$OffsetTo@U?$List16OfOffsetTo@USubstLookup@GSUB_impl@Layout@OT@@U?$IntType@G$01@4@@OT@@U?$IntType@G$01@2@$00@OT@@QEBA_NPEAUhb_sanitize_context_t@@PEBX@Z 000000018005aed0 f i hb-ot-layout.obj
 0001:0005a060       ??$sanitize@$$V@?$OffsetTo@U?$RecordListOf@UFeature@OT@@@OT@@U?$IntType@G$01@2@$00@OT@@QEBA_NPEAUhb_sanitize_context_t@@PEBX@Z 000000018005b060 f i hb-ot-layout.obj
 0001:0005a110       ??$sanitize@$$V@?$OffsetTo@U?$RuleSet@USmallTypes@Layout@OT@@@OT@@U?$IntType@G$01@2@$00@OT@@QEBA_NPEAUhb_sanitize_context_t@@PEBX@Z 000000018005b110 f i hb-ot-layout.obj
 0001:0005a1d0       ??$sanitize@$$V@?$OffsetTo@UAnchor@GPOS_impl@Layout@OT@@U?$IntType@G$01@4@$00@OT@@QEBA_NPEAUhb_sanitize_context_t@@PEBX@Z 000000018005b1d0 f i hb-ot-layout.obj
 0001:0005a310       ??$sanitize@$$V@?$OffsetTo@UConditionSet@OT@@U?$IntType@I$03@2@$00@OT@@QEBA_NPEAUhb_sanitize_context_t@@PEBX@Z 000000018005b310 f i hb-ot-layout.obj
 0001:0005a4f0       ??$sanitize@$$V@?$OffsetTo@UFeatureVariations@OT@@U?$IntType@I$03@2@$00@OT@@QEBA_NPEAUhb_sanitize_context_t@@PEBX@Z 000000018005b4f0 f i hb-ot-layout.obj
 0001:0005a5e0       ??$sanitize@$$V@?$OffsetTo@UMarkArray@GPOS_impl@Layout@OT@@U?$IntType@G$01@4@$00@OT@@QEBA_NPEAUhb_sanitize_context_t@@PEBX@Z 000000018005b5e0 f i hb-ot-layout.obj
 0001:0005a720       ??$sanitize@$$V@?$OffsetTo@URecordListOfScript@OT@@U?$IntType@G$01@2@$00@OT@@QEBA_NPEAUhb_sanitize_context_t@@PEBX@Z 000000018005b720 f i hb-ot-layout.obj
 0001:0005a8e0       ??$sanitize@I@?$OffsetTo@UAnchorMatrix@GPOS_impl@Layout@OT@@U?$IntType@G$01@4@$00@OT@@QEBA_NPEAUhb_sanitize_context_t@@PEBX$$QEAI@Z 000000018005b8e0 f i hb-ot-layout.obj
 0001:0005aa50       ??$sanitize@I@?$OffsetTo@UFeatureParams@OT@@U?$IntType@G$01@2@$00@OT@@QEBA_NPEAUhb_sanitize_context_t@@PEBX$$QEAI@Z 000000018005ba50 f i hb-ot-layout.obj
 0001:0005ab00       ??$sanitize@PEAUsanitize_closure_t@?$PairSet@USmallTypes@Layout@OT@@@GPOS_impl@Layout@OT@@@?$OffsetTo@U?$PairSet@USmallTypes@Layout@OT@@@GPOS_impl@Layout@OT@@U?$IntType@G$01@4@$00@OT@@QEBA_NPEAUhb_sanitize_context_t@@PEBX$$QEAPEAUsanitize_closure_t@?$PairSet@USmallTypes@Layout@OT@@@GPOS_impl@Layout@1@@Z 000000018005bb00 f i hb-ot-layout.obj
 0001:0005ac80       ??$sanitize@PEBU?$LigatureSet@USmallTypes@Layout@OT@@@GSUB_impl@Layout@OT@@@?$ArrayOf@U?$OffsetTo@U?$Ligature@USmallTypes@Layout@OT@@@GSUB_impl@Layout@OT@@U?$IntType@G$01@4@$00@OT@@U?$IntType@G$01@2@@OT@@QEBA_NPEAUhb_sanitize_context_t@@$$QEAPEBU?$LigatureSet@USmallTypes@Layout@OT@@@GSUB_impl@Layout@1@@Z 000000018005bc80 f i hb-ot-layout.obj
 0001:0005ae10       ??$sanitize@PEBU?$RuleSet@USmallTypes@Layout@OT@@@OT@@@?$ArrayOf@U?$OffsetTo@U?$Rule@USmallTypes@Layout@OT@@@OT@@U?$IntType@G$01@2@$00@OT@@U?$IntType@G$01@2@@OT@@QEBA_NPEAUhb_sanitize_context_t@@$$QEAPEBU?$RuleSet@USmallTypes@Layout@OT@@@1@@Z 000000018005be10 f i hb-ot-layout.obj
 0001:0005afc0       ??$sanitize@PEBUChainContextFormat3@OT@@@?$ArrayOf@U?$OffsetTo@UCoverage@Common@Layout@OT@@U?$IntType@G$01@4@$00@OT@@U?$IntType@G$01@2@@OT@@QEBA_NPEAUhb_sanitize_context_t@@$$QEAPEBUChainContextFormat3@1@@Z 000000018005bfc0 f i hb-ot-layout.obj
 0001:0005afc0       ??$sanitize@PEBUReverseChainSingleSubstFormat1@GSUB_impl@Layout@OT@@@?$ArrayOf@U?$OffsetTo@UCoverage@Common@Layout@OT@@U?$IntType@G$01@4@$00@OT@@U?$IntType@G$01@2@@OT@@QEBA_NPEAUhb_sanitize_context_t@@$$QEAPEBUReverseChainSingleSubstFormat1@GSUB_impl@Layout@1@@Z 000000018005bfc0 f i hb-ot-layout.obj
 0001:0005b070       ??$sanitize@PEBUFeatureVariations@OT@@@?$ArrayOf@UFeatureVariationRecord@OT@@U?$IntType@I$03@2@@OT@@QEBA_NPEAUhb_sanitize_context_t@@$$QEAPEBUFeatureVariations@1@@Z 000000018005c070 f i hb-ot-layout.obj
 0001:0005b1e0       ??$sanitize@UPosLookupSubTable@GPOS_impl@Layout@OT@@@Lookup@OT@@QEBA_NPEAUhb_sanitize_context_t@@@Z 000000018005c1e0 f i hb-ot-layout.obj
 0001:0005b470       ??$sanitize@USubstLookupSubTable@GSUB_impl@Layout@OT@@@Lookup@OT@@QEBA_NPEAUhb_sanitize_context_t@@@Z 000000018005c470 f i hb-ot-layout.obj
 0001:0005b700       ??$sanitize_blob@UGPOS@Layout@OT@@@hb_sanitize_context_t@@QEAAPEAUhb_blob_t@@PEAU1@@Z 000000018005c700 f i hb-ot-layout.obj
 0001:0005b9c0       ??$sanitize_blob@UGSUB@Layout@OT@@@hb_sanitize_context_t@@QEAAPEAUhb_blob_t@@PEAU1@@Z 000000018005c9c0 f i hb-ot-layout.obj
 0001:0005bc80       ??$sanitize_blob@Ukern@OT@@@hb_sanitize_context_t@@QEAAPEAUhb_blob_t@@PEAU1@@Z 000000018005cc80 f i hb-ot-layout.obj
 0001:0005bfc0       ?_set_glyph_class@hb_ot_apply_context_t@OT@@QEAAXII_N0@Z 000000018005cfc0 f i hb-ot-layout.obj
 0001:0005c0e0       ?apply@?$AlternateSet@USmallTypes@Layout@OT@@@GSUB_impl@Layout@OT@@QEBA_NPEAUhb_ot_apply_context_t@4@@Z 000000018005d0e0 f i hb-ot-layout.obj
 0001:0005c270       ?apply@?$AlternateSubstFormat1_2@USmallTypes@Layout@OT@@@GSUB_impl@Layout@OT@@QEBA_NPEAUhb_ot_apply_context_t@4@@Z 000000018005d270 f i hb-ot-layout.obj
 0001:0005c380       ?apply@?$ChainContextFormat1_4@USmallTypes@Layout@OT@@@OT@@QEBA_NPEAUhb_ot_apply_context_t@2@@Z 000000018005d380 f i hb-ot-layout.obj
 0001:0005c4b0       ?apply@?$ChainContextFormat2_5@USmallTypes@Layout@OT@@@OT@@QEBA_NPEAUhb_ot_apply_context_t@2@_N@Z 000000018005d4b0 f i hb-ot-layout.obj
 0001:0005c6a0       ?apply@?$ChainRuleSet@USmallTypes@Layout@OT@@@OT@@QEBA_NPEAUhb_ot_apply_context_t@2@AEBUChainContextApplyLookupContext@2@@Z 000000018005d6a0 f i hb-ot-layout.obj
 0001:0005c8b0       ?apply@?$ContextFormat1_4@USmallTypes@Layout@OT@@@OT@@QEBA_NPEAUhb_ot_apply_context_t@2@@Z 000000018005d8b0 f i hb-ot-layout.obj
 0001:0005c9d0       ?apply@?$ContextFormat2_5@USmallTypes@Layout@OT@@@OT@@QEBA_NPEAUhb_ot_apply_context_t@2@_N@Z 000000018005d9d0 f i hb-ot-layout.obj
 0001:0005cb90       ?apply@?$KerxTable@UKernAAT@OT@@@AAT@@QEBA_NPEAUhb_aat_apply_context_t@2@@Z 000000018005db90 f i hb-ot-layout.obj
 0001:0005cfc0       ?apply@?$KerxTable@UKernOT@OT@@@AAT@@QEBA_NPEAUhb_aat_apply_context_t@2@@Z 000000018005dfc0 f i hb-ot-layout.obj
 0001:0005d2a0       ?apply@?$Ligature@USmallTypes@Layout@OT@@@GSUB_impl@Layout@OT@@QEBA_NPEAUhb_ot_apply_context_t@4@@Z 000000018005e2a0 f i hb-ot-layout.obj
 0001:0005d590       ?apply@?$LigatureSubstFormat1_2@USmallTypes@Layout@OT@@@GSUB_impl@Layout@OT@@QEBA_NPEAUhb_ot_apply_context_t@4@@Z 000000018005e590 f i hb-ot-layout.obj
 0001:0005d720       ?apply@?$MarkBasePosFormat1_2@USmallTypes@Layout@OT@@@GPOS_impl@Layout@OT@@QEBA_NPEAUhb_ot_apply_context_t@4@@Z 000000018005e720 f i hb-ot-layout.obj
 0001:0005db10       ?apply@?$MarkLigPosFormat1_2@USmallTypes@Layout@OT@@@GPOS_impl@Layout@OT@@QEBA_NPEAUhb_ot_apply_context_t@4@@Z 000000018005eb10 f i hb-ot-layout.obj
 0001:0005dea0       ?apply@?$MarkMarkPosFormat1_2@USmallTypes@Layout@OT@@@GPOS_impl@Layout@OT@@QEBA_NPEAUhb_ot_apply_context_t@4@@Z 000000018005eea0 f i hb-ot-layout.obj
 0001:0005e160       ?apply@?$MultipleSubstFormat1_2@USmallTypes@Layout@OT@@@GSUB_impl@Layout@OT@@QEBA_NPEAUhb_ot_apply_context_t@4@@Z 000000018005f160 f i hb-ot-layout.obj
 0001:0005e270       ?apply@?$PairPosFormat1_3@USmallTypes@Layout@OT@@@GPOS_impl@Layout@OT@@QEBA_NPEAUhb_ot_apply_context_t@4@@Z 000000018005f270 f i hb-ot-layout.obj
 0001:0005e410       ?apply@?$PairPosFormat2_4@USmallTypes@Layout@OT@@@GPOS_impl@Layout@OT@@QEBA_NPEAUhb_ot_apply_context_t@4@@Z 000000018005f410 f i hb-ot-layout.obj
 0001:0005e810       ?apply@?$PairSet@USmallTypes@Layout@OT@@@GPOS_impl@Layout@OT@@QEBA_NPEAUhb_ot_apply_context_t@4@PEBUValueFormat@234@I@Z 000000018005f810 f i hb-ot-layout.obj
 0001:0005eac0       ?apply@?$RuleSet@USmallTypes@Layout@OT@@@OT@@QEBA_NPEAUhb_ot_apply_context_t@2@AEBUContextApplyLookupContext@2@@Z 000000018005fac0 f i hb-ot-layout.obj
 0001:0005ec50       ?apply@?$Sequence@USmallTypes@Layout@OT@@@GSUB_impl@Layout@OT@@QEBA_NPEAUhb_ot_apply_context_t@4@@Z 000000018005fc50 f i hb-ot-layout.obj
 0001:0005efe0       ?apply@?$SingleSubstFormat1_3@USmallTypes@Layout@OT@@@GSUB_impl@Layout@OT@@QEBA_NPEAUhb_ot_apply_context_t@4@@Z 000000018005ffe0 f i hb-ot-layout.obj
 0001:0005f120       ?apply@?$SingleSubstFormat2_4@USmallTypes@Layout@OT@@@GSUB_impl@Layout@OT@@QEBA_NPEAUhb_ot_apply_context_t@4@@Z 0000000180060120 f i hb-ot-layout.obj
 0001:0005f290       ?apply@ChainContextFormat3@OT@@QEBA_NPEAUhb_ot_apply_context_t@2@@Z 0000000180060290 f i hb-ot-layout.obj
 0001:0005f450       ?apply@ContextFormat3@OT@@QEBA_NPEAUhb_ot_apply_context_t@2@@Z 0000000180060450 f i hb-ot-layout.obj
 0001:0005f550       ?apply@CursivePosFormat1@GPOS_impl@Layout@OT@@QEBA_NPEAUhb_ot_apply_context_t@4@@Z 0000000180060550 f i hb-ot-layout.obj
 0001:0005fb40       ?apply@MarkArray@GPOS_impl@Layout@OT@@QEBA_NPEAUhb_ot_apply_context_t@4@IIAEBUAnchorMatrix@234@II@Z 0000000180060b40 f i hb-ot-layout.obj
 0001:0005fda0       ?apply@ReverseChainSingleSubstFormat1@GSUB_impl@Layout@OT@@QEBA_NPEAUhb_ot_apply_context_t@4@@Z 0000000180060da0 f i hb-ot-layout.obj
 0001:00060010       ?apply@SinglePosFormat1@GPOS_impl@Layout@OT@@QEBA_NPEAUhb_ot_apply_context_t@4@@Z 0000000180061010 f i hb-ot-layout.obj
 0001:00060140       ?apply@SinglePosFormat2@GPOS_impl@Layout@OT@@QEBA_NPEAUhb_ot_apply_context_t@4@@Z 0000000180061140 f i hb-ot-layout.obj
 0001:000602f0       ?apply@hb_ot_layout_lookup_accelerator_t@OT@@QEBA_NPEAUhb_ot_apply_context_t@2@I_N@Z 00000001800612f0 f i hb-ot-layout.obj
 0001:00060ed0       ?apply_value@ValueFormat@GPOS_impl@Layout@OT@@QEBA_NPEAUhb_ot_apply_context_t@4@PEBXPEBU?$IntType@G$01@4@AEAUhb_glyph_position_t@@@Z 0000000180061ed0 f i hb-ot-layout.obj
 0001:00061230       ?find_index@FeatureVariations@OT@@QEBA_NPEBHIPEAI@Z 0000000180062230 f i hb-ot-layout.obj
 0001:00061410       ?find_script_index@GSUBGPOS@OT@@QEBA_NIPEAI@Z 0000000180062410 f i hb-ot-layout.obj
 0001:00061500       ?get_accel@?$accelerator_t@UGPOS@Layout@OT@@@GSUBGPOS@OT@@QEBAPEAUhb_ot_layout_lookup_accelerator_t@3@I@Z 0000000180062500 f i hb-ot-layout.obj
 0001:00061760       ?get_accel@?$accelerator_t@UGSUB@Layout@OT@@@GSUBGPOS@OT@@QEBAPEAUhb_ot_layout_lookup_accelerator_t@3@I@Z 0000000180062760 f i hb-ot-layout.obj
 0001:000619c0       ?get_anchor@Anchor@GPOS_impl@Layout@OT@@QEBAXPEAUhb_ot_apply_context_t@4@IPEAM1@Z 00000001800629c0 f i hb-ot-layout.obj
 0001:00061c10       ?get_anchor@AnchorFormat3@GPOS_impl@Layout@OT@@QEBAXPEAUhb_ot_apply_context_t@4@IPEAM1@Z 0000000180062c10 f i hb-ot-layout.obj
 0001:00061d70       ?get_coverage@ChainContextFormat3@OT@@QEBAAEBUCoverage@Common@Layout@2@XZ 0000000180062d70 f i hb-ot-layout.obj
 0001:00061de0       ?get_delta@HintingDevice@OT@@AEBAHIH@Z 0000000180062de0 f i hb-ot-layout.obj
 0001:00061f00       ?get_feature@GSUBGPOS@OT@@QEBAAEBUFeature@2@I@Z 0000000180062f00 f i hb-ot-layout.obj
 0001:00061fb0       ?get_feature_tag@GSUBGPOS@OT@@QEBAII@Z 0000000180062fb0 f i hb-ot-layout.obj
 0001:00062050       ?get_feature_variation@GSUBGPOS@OT@@QEBAAEBUFeature@2@II@Z 0000000180063050 f i hb-ot-layout.obj
 0001:00062260       ?get_indexes@IndexArray@OT@@QEBAIIPEAI0@Z 0000000180063260 f i hb-ot-layout.obj
 0001:000623c0       ?get_kerning@?$KerxSubTableFormat0@UKernAATSubTableHeader@OT@@@AAT@@QEBAHIIPEAUhb_aat_apply_context_t@2@@Z 00000001800633c0 f i hb-ot-layout.obj
 0001:000624a0       ?get_kerning@?$KerxSubTableFormat0@UKernOTSubTableHeader@OT@@@AAT@@QEBAHIIPEAUhb_aat_apply_context_t@2@@Z 00000001800634a0 f i hb-ot-layout.obj
 0001:00062580       ?get_kerning@?$KerxSubTableFormat2@UKernAATSubTableHeader@OT@@@AAT@@QEBAHIIPEAUhb_aat_apply_context_t@2@@Z 0000000180063580 f i hb-ot-layout.obj
 0001:000626b0       ?get_kerning@?$KerxSubTableFormat2@UKernOTSubTableHeader@OT@@@AAT@@QEBAHIIPEAUhb_aat_apply_context_t@2@@Z 00000001800636b0 f i hb-ot-layout.obj
 0001:000627e0       ?get_lang_sys@Script@OT@@QEBAAEBULangSys@2@I@Z 00000001800637e0 f i hb-ot-layout.obj
 0001:00062870       ?get_lookup@GSUBGPOS@OT@@QEBAAEBULookup@2@I@Z 0000000180063870 f i hb-ot-layout.obj
 0001:00062920       ?get_population@Coverage@Common@Layout@OT@@QEBAIXZ 0000000180063920 f i hb-ot-layout.obj
 0001:000629f0       ?get_script@GSUBGPOS@OT@@QEBAAEBUScript@2@I@Z 00000001800639f0 f i hb-ot-layout.obj
 0001:00062aa0       ?get_stored@?$hb_lazy_loader_t@UGPOS_accelerator_t@OT@@U?$hb_face_lazy_loader_t@UGPOS_accelerator_t@OT@@$0BK@@@Uhb_face_t@@$0BK@U12@@@QEBAPEAUGPOS_accelerator_t@OT@@XZ 0000000180063aa0 f i hb-ot-layout.obj
 0001:00062c80       ?get_stored@?$hb_lazy_loader_t@UGSUB_accelerator_t@OT@@U?$hb_face_lazy_loader_t@UGSUB_accelerator_t@OT@@$0BJ@@@Uhb_face_t@@$0BJ@U12@@@QEBAPEAUGSUB_accelerator_t@OT@@XZ 0000000180063c80 f i hb-ot-layout.obj
 0001:00062e60       ?get_stored@?$hb_lazy_loader_t@Ukern@OT@@U?$hb_table_lazy_loader_t@Ukern@OT@@$0BH@$00@@Uhb_face_t@@$0BH@Uhb_blob_t@@@@QEBAPEAUhb_blob_t@@XZ 0000000180063e60 f i hb-ot-layout.obj
 0001:00062f50       ?get_x_delta@Device@OT@@QEBAHPEAUhb_font_t@@AEBUVariationStore@2@PEAM@Z 0000000180063f50 f i hb-ot-layout.obj
 0001:00063000       ?get_y_delta@Device@OT@@QEBAHPEAUhb_font_t@@AEBUVariationStore@2@PEAM@Z 0000000180064000 f i hb-ot-layout.obj
 0001:000630b0       ?hb_ot_layout_has_cross_kerning@@YA_NPEAUhb_face_t@@@Z 00000001800640b0 f   hb-ot-layout.obj
 0001:000631a0       ?hb_ot_layout_has_kerning@@YA_NPEAUhb_face_t@@@Z 00000001800641a0 f   hb-ot-layout.obj
 0001:000631f0       ?hb_ot_layout_has_machine_kerning@@YA_NPEAUhb_face_t@@@Z 00000001800641f0 f   hb-ot-layout.obj
 0001:000632e0       ?hb_ot_layout_kern@@YAXPEBUhb_ot_shape_plan_t@@PEAUhb_font_t@@PEAUhb_buffer_t@@@Z 00000001800642e0 f   hb-ot-layout.obj
 0001:000633c0       ?hb_ot_layout_position_finish_offsets@@YAXPEAUhb_font_t@@PEAUhb_buffer_t@@@Z 00000001800643c0 f   hb-ot-layout.obj
 0001:000633d0       ?hb_ot_layout_position_start@@YAXPEAUhb_font_t@@PEAUhb_buffer_t@@@Z 00000001800643d0 f   hb-ot-layout.obj
 0001:00063400       ?hb_ot_layout_substitute_lookup@@YAXPEAUhb_ot_apply_context_t@OT@@AEBUSubstLookup@GSUB_impl@Layout@2@AEBUhb_ot_layout_lookup_accelerator_t@2@@Z 0000000180064400 f   hb-ot-layout.obj
 0001:00063410       ?hb_ot_layout_substitute_start@@YAXPEAUhb_font_t@@PEAUhb_buffer_t@@@Z 0000000180064410 f   hb-ot-layout.obj
 0001:00063590       ?hb_ot_layout_table_find_feature@@YA_NPEAUhb_face_t@@IIPEAI@Z 0000000180064590 f   hb-ot-layout.obj
 0001:000636f0       ?is_blocklisted@GDEF@OT@@QEBA_NPEAUhb_blob_t@@PEAUhb_face_t@@@Z 00000001800646f0 f   hb-ot-layout.obj
 0001:000639e0       ?kern@?$hb_kern_machine_t@U?$KernSubTableFormat3@UKernAATSubTableHeader@OT@@@OT@@@OT@@QEBAXPEAUhb_font_t@@PEAUhb_buffer_t@@I_N@Z 00000001800649e0 f i hb-ot-layout.obj
 0001:00063e90       ?kern@?$hb_kern_machine_t@Uaccelerator_t@?$KerxSubTableFormat0@UKernAATSubTableHeader@OT@@@AAT@@@OT@@QEBAXPEAUhb_font_t@@PEAUhb_buffer_t@@I_N@Z 0000000180064e90 f i hb-ot-layout.obj
 0001:00064210       ?kern@?$hb_kern_machine_t@Uaccelerator_t@?$KerxSubTableFormat0@UKernOTSubTableHeader@OT@@@AAT@@@OT@@QEBAXPEAUhb_font_t@@PEAUhb_buffer_t@@I_N@Z 0000000180065210 f i hb-ot-layout.obj
 0001:00064590       ?kern@?$hb_kern_machine_t@Uaccelerator_t@?$KerxSubTableFormat2@UKernAATSubTableHeader@OT@@@AAT@@@OT@@QEBAXPEAUhb_font_t@@PEAUhb_buffer_t@@I_N@Z 0000000180065590 f i hb-ot-layout.obj
 0001:00064910       ?kern@?$hb_kern_machine_t@Uaccelerator_t@?$KerxSubTableFormat2@UKernOTSubTableHeader@OT@@@AAT@@@OT@@QEBAXPEAUhb_font_t@@PEAUhb_buffer_t@@I_N@Z 0000000180065910 f i hb-ot-layout.obj
 0001:00065150       ?position@hb_ot_map_t@@QEBAXPEBUhb_ot_shape_plan_t@@PEAUhb_font_t@@PEAUhb_buffer_t@@@Z 0000000180066150 f   hb-ot-layout.obj
 0001:000651f0       ?position_finish_offsets@GPOS@Layout@OT@@SAXPEAUhb_font_t@@PEAUhb_buffer_t@@@Z 00000001800661f0 f i hb-ot-layout.obj
 0001:00065400       ?prev@skipping_iterator_t@hb_ot_apply_context_t@OT@@QEAA_NPEAI@Z 0000000180066400 f i hb-ot-layout.obj
 0001:000656f0       ?sanitize@?$KerxTable@UKernAAT@OT@@@AAT@@QEBA_NPEAUhb_sanitize_context_t@@@Z 00000001800666f0 f i hb-ot-layout.obj
 0001:00065910       ?sanitize@?$KerxTable@UKernOT@OT@@@AAT@@QEBA_NPEAUhb_sanitize_context_t@@@Z 0000000180066910 f i hb-ot-layout.obj
 0001:00065b70       ?sanitize@?$MarkLigPosFormat1_2@USmallTypes@Layout@OT@@@GPOS_impl@Layout@OT@@QEBA_NPEAUhb_sanitize_context_t@@@Z 0000000180066b70 f i hb-ot-layout.obj
 0001:00065d00       ?sanitize@?$PairPosFormat1_3@USmallTypes@Layout@OT@@@GPOS_impl@Layout@OT@@QEBA_NPEAUhb_sanitize_context_t@@@Z 0000000180066d00 f i hb-ot-layout.obj
 0001:00065eb0       ?sanitize@?$PairPosFormat2_4@USmallTypes@Layout@OT@@@GPOS_impl@Layout@OT@@QEBA_NPEAUhb_sanitize_context_t@@@Z 0000000180066eb0 f i hb-ot-layout.obj
 0001:000660b0       ?sanitize@?$RecordListOf@UFeature@OT@@@OT@@QEBA_NPEAUhb_sanitize_context_t@@@Z 00000001800670b0 f i hb-ot-layout.obj
 0001:00066230       ?sanitize@Feature@OT@@QEBA_NPEAUhb_sanitize_context_t@@PEBURecord_sanitize_closure_t@2@@Z 0000000180067230 f i hb-ot-layout.obj
 0001:00066430       ?sanitize@FeatureParams@OT@@QEBA_NPEAUhb_sanitize_context_t@@I@Z 0000000180067430 f i hb-ot-layout.obj
 0001:000665c0       ?sanitize@FeatureTableSubstitution@OT@@QEBA_NPEAUhb_sanitize_context_t@@@Z 00000001800675c0 f i hb-ot-layout.obj
 0001:00066740       ?sanitize@GPOS@Layout@OT@@QEBA_NPEAUhb_sanitize_context_t@@@Z 0000000180067740 f i hb-ot-layout.obj
 0001:00066810       ?sanitize@GSUB@Layout@OT@@QEBA_NPEAUhb_sanitize_context_t@@@Z 0000000180067810 f i hb-ot-layout.obj
 0001:000668e0       ?sanitize@Script@OT@@QEBA_NPEAUhb_sanitize_context_t@@PEBURecord_sanitize_closure_t@2@@Z 00000001800678e0 f i hb-ot-layout.obj
 0001:00066ab0       ?sanitize@SinglePosFormat1@GPOS_impl@Layout@OT@@QEBA_NPEAUhb_sanitize_context_t@@@Z 0000000180067ab0 f i hb-ot-layout.obj
 0001:00066bf0       ?sanitize@kern@OT@@QEBA_NPEAUhb_sanitize_context_t@@@Z 0000000180067bf0 f i hb-ot-layout.obj
 0001:00066c70       ?sanitize_shallow@?$OffsetTo@ULangSys@OT@@U?$IntType@G$01@2@$00@OT@@QEBA_NPEAUhb_sanitize_context_t@@PEBX@Z 0000000180067c70 f i hb-ot-layout.obj
 0001:00066cf0       ?sanitize_value_devices@ValueFormat@GPOS_impl@Layout@OT@@AEBA_NPEAUhb_sanitize_context_t@@PEBXPEBU?$IntType@G$01@4@@Z 0000000180067cf0 f i hb-ot-layout.obj
 0001:00066dd0       ?sanitize_values@ValueFormat@GPOS_impl@Layout@OT@@QEBA_NPEAUhb_sanitize_context_t@@PEBXPEBU?$IntType@G$01@4@I@Z 0000000180067dd0 f i hb-ot-layout.obj
 0001:00066f90       ?sanitize_values_stride_unsafe@ValueFormat@GPOS_impl@Layout@OT@@QEBA_NPEAUhb_sanitize_context_t@@PEBXPEBU?$IntType@G$01@4@II@Z 0000000180067f90 f i hb-ot-layout.obj
 0001:000670c0       ?substitute@hb_ot_map_t@@QEBAXPEBUhb_ot_shape_plan_t@@PEAUhb_font_t@@PEAUhb_buffer_t@@@Z 00000001800680c0 f   hb-ot-layout.obj
 0001:00067160       ?transition@driver_context_t@?$KerxSubTableFormat1@UKernAATSubTableHeader@OT@@@AAT@@QEAAXPEAU?$StateTableDriver@UObsoleteTypes@AAT@@X@3@AEBU?$Entry@X@3@@Z 0000000180068160 f i hb-ot-layout.obj
 0001:000674f0       ?unsafe_to_concat_from_outbuffer@hb_buffer_t@@QEAAXII@Z 00000001800684f0 f i hb-ot-layout.obj
 0001:000675a0       ?would_apply@?$ChainRuleSet@USmallTypes@Layout@OT@@@OT@@QEBA_NPEAUhb_would_apply_context_t@2@AEBUChainContextApplyLookupContext@2@@Z 00000001800685a0 f i hb-ot-layout.obj
 0001:00067780       ?would_apply@?$LigatureSubstFormat1_2@USmallTypes@Layout@OT@@@GSUB_impl@Layout@OT@@QEBA_NPEAUhb_would_apply_context_t@4@@Z 0000000180068780 f i hb-ot-layout.obj
 0001:000679e0       ?would_apply@?$RuleSet@USmallTypes@Layout@OT@@@OT@@QEBA_NPEAUhb_would_apply_context_t@2@AEBUContextApplyLookupContext@2@@Z 00000001800689e0 f i hb-ot-layout.obj
 0001:00067b40       hb_ot_layout_feature_with_variations_get_lookups 0000000180068b40 f   hb-ot-layout.obj
 0001:00067b90       hb_ot_layout_has_glyph_classes 0000000180068b90 f   hb-ot-layout.obj
 0001:00067c00       hb_ot_layout_has_positioning 0000000180068c00 f   hb-ot-layout.obj
 0001:00067c60       hb_ot_layout_has_substitution 0000000180068c60 f   hb-ot-layout.obj
 0001:00067cc0       hb_ot_layout_language_find_feature 0000000180068cc0 f   hb-ot-layout.obj
 0001:00067e50       hb_ot_layout_language_get_required_feature 0000000180068e50 f   hb-ot-layout.obj
 0001:00067f10       hb_ot_layout_lookup_would_substitute 0000000180068f10 f   hb-ot-layout.obj
 0001:000680e0       hb_ot_layout_script_select_language 00000001800690e0 f   hb-ot-layout.obj
 0001:00068270       hb_ot_layout_table_find_feature_variations 0000000180069270 f   hb-ot-layout.obj
 0001:00068310       hb_ot_layout_table_get_lookup_count 0000000180069310 f   hb-ot-layout.obj
 0001:00068380       hb_ot_layout_table_select_script 0000000180069380 f   hb-ot-layout.obj
 0001:00068570       ??0hb_ot_map_builder_t@@QEAA@PEAUhb_face_t@@AEBUhb_segment_properties_t@@@Z 0000000180069570 f   hb-ot-map.obj
 0001:000686e0       ??1hb_ot_map_builder_t@@QEAA@XZ 00000001800696e0 f   hb-ot-map.obj
 0001:000687e0       ?add_feature@hb_ot_map_builder_t@@QEAAXIW4hb_ot_map_feature_flags_t@@I@Z 00000001800697e0 f   hb-ot-map.obj
 0001:00068940       ?add_lookups@hb_ot_map_builder_t@@AEAAXAEAUhb_ot_map_t@@IIII_N111I@Z 0000000180069940 f   hb-ot-map.obj
 0001:00068bd0       ?add_pause@hb_ot_map_builder_t@@AEAAXIP6A_NPEBUhb_ot_shape_plan_t@@PEAUhb_font_t@@PEAUhb_buffer_t@@@Z@Z 0000000180069bd0 f   hb-ot-map.obj
 0001:00068ce0       ?alloc@?$hb_vector_t@Ufeature_info_t@hb_ot_map_builder_t@@$0A@@@QEAA_NI_N@Z 0000000180069ce0 f i hb-ot-map.obj
 0001:00068d90       ?cmp@feature_info_t@hb_ot_map_builder_t@@SAHPEBX0@Z 0000000180069d90 f i hb-ot-map.obj
 0001:00068dc0       ?cmp@lookup_map_t@hb_ot_map_t@@SAHPEBX0@Z 0000000180069dc0 f i hb-ot-map.obj
 0001:00068de0       ?compile@hb_ot_map_builder_t@@QEAAXAEAUhb_ot_map_t@@AEBUhb_ot_shape_plan_key_t@@@Z 0000000180069de0 f   hb-ot-map.obj
 0001:00069830       ?has_feature@hb_ot_map_builder_t@@QEAA_NI@Z 000000018006a830 f   hb-ot-map.obj
 0001:000698b0       ??$sanitize_blob@UMVAR@OT@@@hb_sanitize_context_t@@QEAAPEAUhb_blob_t@@PEAU1@@Z 000000018006a8b0 f i hb-ot-metrics.obj
 0001:00069d90       ?_hb_ot_metrics_get_position_common@@YA_NPEAUhb_font_t@@W4hb_ot_metrics_tag_t@@PEAH@Z 000000018006ad90 f   hb-ot-metrics.obj
 0001:0006a1f0       ?get@?$hb_lazy_loader_t@UMVAR@OT@@U?$hb_table_lazy_loader_t@UMVAR@OT@@$0BG@$00@@Uhb_face_t@@$0BG@Uhb_blob_t@@@@QEBAPEBUMVAR@OT@@XZ 000000018006b1f0 f i hb-ot-metrics.obj
 0001:0006a2e0       ?get_var@MVAR@OT@@QEBAMIPEBHI@Z 000000018006b2e0 f i hb-ot-metrics.obj
 0001:0006a410       ?has_data@OS2@OT@@QEBA_NXZ 000000018006b410 f i hb-ot-metrics.obj
 0001:0006a470       ?sanitize@MVAR@OT@@QEBA_NPEAUhb_sanitize_context_t@@@Z 000000018006b470 f i hb-ot-metrics.obj
 0001:0006a5b0       ?_hb_ot_shape_fallback_kern@@YAXPEBUhb_ot_shape_plan_t@@PEAUhb_font_t@@PEAUhb_buffer_t@@@Z 000000018006b5b0 f   hb-ot-shape-fallback.obj
 0001:0006a690       ?_hb_ot_shape_fallback_mark_position@@YAXPEBUhb_ot_shape_plan_t@@PEAUhb_font_t@@PEAUhb_buffer_t@@_N@Z 000000018006b690 f   hb-ot-shape-fallback.obj
 0001:0006a800       ?_hb_ot_shape_fallback_mark_position_recategorize_marks@@YAXPEBUhb_ot_shape_plan_t@@PEAUhb_font_t@@PEAUhb_buffer_t@@@Z 000000018006b800 f   hb-ot-shape-fallback.obj
 0001:0006aa90       ?_hb_ot_shape_fallback_spaces@@YAXPEBUhb_ot_shape_plan_t@@PEAUhb_font_t@@PEAUhb_buffer_t@@@Z 000000018006ba90 f   hb-ot-shape-fallback.obj
 0001:0006add0       ?kern@?$hb_kern_machine_t@Uhb_ot_shape_fallback_kern_driver_t@@@OT@@QEBAXPEAUhb_font_t@@PEAUhb_buffer_t@@I_N@Z 000000018006bdd0 f i hb-ot-shape-fallback.obj
 0001:0006bb90       ?_hb_ot_shape_normalize@@YAXPEBUhb_ot_shape_plan_t@@PEAUhb_buffer_t@@PEAUhb_font_t@@@Z 000000018006cb90 f   hb-ot-shape-normalize.obj
 0001:0006d0c0       ?compile@hb_ot_shape_planner_t@@QEAAXAEAUhb_ot_shape_plan_t@@AEBUhb_ot_shape_plan_key_t@@@Z 000000018006e0c0 f   hb-ot-shape.obj
 0001:0006d650       ?fini@hb_ot_map_t@@QEAAXXZ 000000018006e650 f i hb-ot-shape.obj
 0001:0006d720       ?fini@hb_ot_shape_plan_t@@QEAAXXZ 000000018006e720 f   hb-ot-shape.obj
 0001:0006d750       ?has_glyph@hb_font_t@@QEAA_NI@Z 000000018006e750 f i hb-ot-shape.obj
 0001:0006f500       ?init0@hb_ot_shape_plan_t@@QEAA_NPEAUhb_face_t@@PEBUhb_shape_plan_key_t@@@Z 0000000180070500 f   hb-ot-shape.obj
 0001:0006f720       _hb_ot_shape               0000000180070720 f   hb-ot-shape.obj
 0001:0006faa0       ?data_create_arabic@@YAPEAXPEBUhb_ot_shape_plan_t@@@Z 0000000180070aa0 f   hb-ot-shaper-arabic.obj
 0001:0006fc60       ?data_destroy_arabic@@YAXPEAX@Z 0000000180070c60 f   hb-ot-shaper-arabic.obj
 0001:0006ff90       ??$add_link@U?$OffsetTo@U?$Ligature@USmallTypes@Layout@OT@@@GSUB_impl@Layout@OT@@U?$IntType@G$01@4@$00@OT@@@hb_serialize_context_t@@QEAAXAEAU?$OffsetTo@U?$Ligature@USmallTypes@Layout@OT@@@GSUB_impl@Layout@OT@@U?$IntType@G$01@4@$00@OT@@IW4whence_t@0@I@Z 0000000180070f90 f i hb-ot-shaper-arabic.obj
 0001:0006ff90       ??$add_link@U?$OffsetTo@U?$LigatureSet@USmallTypes@Layout@OT@@@GSUB_impl@Layout@OT@@U?$IntType@G$01@4@$00@OT@@@hb_serialize_context_t@@QEAAXAEAU?$OffsetTo@U?$LigatureSet@USmallTypes@Layout@OT@@@GSUB_impl@Layout@OT@@U?$IntType@G$01@4@$00@OT@@IW4whence_t@0@I@Z 0000000180070f90 f i hb-ot-shaper-arabic.obj
 0001:0006ff90       ??$add_link@U?$OffsetTo@UCoverage@Common@Layout@OT@@U?$IntType@G$01@4@$00@OT@@@hb_serialize_context_t@@QEAAXAEAU?$OffsetTo@UCoverage@Common@Layout@OT@@U?$IntType@G$01@4@$00@OT@@IW4whence_t@0@I@Z 0000000180070f90 f i hb-ot-shaper-arabic.obj
 0001:000715d0       ??$extend@ULookup@OT@@$$V@hb_serialize_context_t@@QEAAPEAULookup@OT@@PEAU12@@Z 00000001800725d0 f i hb-ot-shaper-arabic.obj
 0001:00071690       ??$extend_min@U?$CoverageFormat2_4@USmallTypes@Layout@OT@@@Common@Layout@OT@@@hb_serialize_context_t@@QEAAPEAU?$CoverageFormat2_4@USmallTypes@Layout@OT@@@Common@Layout@OT@@PEAU1234@@Z 0000000180072690 f i hb-ot-shaper-arabic.obj
 0001:00071690       ??$extend_min@U?$Ligature@USmallTypes@Layout@OT@@@GSUB_impl@Layout@OT@@@hb_serialize_context_t@@QEAAPEAU?$Ligature@USmallTypes@Layout@OT@@@GSUB_impl@Layout@OT@@PEAU1234@@Z 0000000180072690 f i hb-ot-shaper-arabic.obj
 0001:00071740       ??$extend_min@U?$IntType@G$01@OT@@@hb_serialize_context_t@@QEAAPEAU?$IntType@G$01@OT@@AEAU12@@Z 0000000180072740 f i hb-ot-shaper-arabic.obj
 0001:00071740       ??$extend_min@U?$LigatureSet@USmallTypes@Layout@OT@@@GSUB_impl@Layout@OT@@@hb_serialize_context_t@@QEAAPEAU?$LigatureSet@USmallTypes@Layout@OT@@@GSUB_impl@Layout@OT@@PEAU1234@@Z 0000000180072740 f i hb-ot-shaper-arabic.obj
 0001:00071740       ??$extend_min@UCoverage@Common@Layout@OT@@@hb_serialize_context_t@@QEAAPEAUCoverage@Common@Layout@OT@@PEAU1234@@Z 0000000180072740 f i hb-ot-shaper-arabic.obj
 0001:000717f0       ??$extend_min@U?$LigatureSubstFormat1_2@USmallTypes@Layout@OT@@@GSUB_impl@Layout@OT@@@hb_serialize_context_t@@QEAAPEAU?$LigatureSubstFormat1_2@USmallTypes@Layout@OT@@@GSUB_impl@Layout@OT@@PEAU1234@@Z 00000001800727f0 f i hb-ot-shaper-arabic.obj
 0001:000717f0       ??$extend_min@U?$SingleSubstFormat1_3@USmallTypes@Layout@OT@@@GSUB_impl@Layout@OT@@@hb_serialize_context_t@@QEAAPEAU?$SingleSubstFormat1_3@USmallTypes@Layout@OT@@@GSUB_impl@Layout@OT@@PEAU1234@@Z 00000001800727f0 f i hb-ot-shaper-arabic.obj
 0001:000717f0       ??$extend_min@U?$SingleSubstFormat2_4@USmallTypes@Layout@OT@@@GSUB_impl@Layout@OT@@@hb_serialize_context_t@@QEAAPEAU?$SingleSubstFormat2_4@USmallTypes@Layout@OT@@@GSUB_impl@Layout@OT@@PEAU1234@@Z 00000001800727f0 f i hb-ot-shaper-arabic.obj
 0001:000717f0       ??$extend_min@ULookup@OT@@@hb_serialize_context_t@@QEAAPEAULookup@OT@@PEAU12@@Z 00000001800727f0 f i hb-ot-shaper-arabic.obj
 0001:000718a0       ??$extend_size@U?$ArrayOf@UHBGlyphID16@OT@@U?$IntType@G$01@2@@OT@@@hb_serialize_context_t@@QEAAPEAU?$ArrayOf@UHBGlyphID16@OT@@U?$IntType@G$01@2@@OT@@PEAU12@_K_N@Z 00000001800728a0 f i hb-ot-shaper-arabic.obj
 0001:000718a0       ??$extend_size@U?$HeadlessArrayOf@UHBGlyphID16@OT@@U?$IntType@G$01@2@@OT@@@hb_serialize_context_t@@QEAAPEAU?$HeadlessArrayOf@UHBGlyphID16@OT@@U?$IntType@G$01@2@@OT@@PEAU12@_K_N@Z 00000001800728a0 f i hb-ot-shaper-arabic.obj
 0001:00071a70       ??$push@UCoverage@Common@Layout@OT@@@hb_serialize_context_t@@QEAAPEAUCoverage@Common@Layout@OT@@XZ 0000000180072a70 f i hb-ot-shaper-arabic.obj
 0001:00071ae0       ??$serialize@U?$hb_map_iter_t@U?$hb_zip_iter_t@U?$hb_sorted_array_t@UHBGlyphID16@OT@@@@U?$hb_array_t@UHBGlyphID16@OT@@@@@@AEBU<unnamed-type-hb_first>@@$00$0A@@@$0A@@?$CoverageFormat2_4@USmallTypes@Layout@OT@@@Common@Layout@OT@@AEAA_NPEAUhb_serialize_context_t@@U?$hb_map_iter_t@U?$hb_zip_iter_t@U?$hb_sorted_array_t@UHBGlyphID16@OT@@@@U?$hb_array_t@UHBGlyphID16@OT@@@@@@AEBU<unnamed-type-hb_first>@@$00$0A@@@@Z 0000000180072ae0 f i hb-ot-shaper-arabic.obj
 0001:00071e30       ??$serialize@U?$hb_map_iter_t@U?$hb_zip_iter_t@U?$hb_sorted_array_t@UHBGlyphID16@OT@@@@U?$hb_array_t@UHBGlyphID16@OT@@@@@@AEBU<unnamed-type-hb_first>@@$00$0A@@@$0A@@Coverage@Common@Layout@OT@@QEAA_NPEAUhb_serialize_context_t@@U?$hb_map_iter_t@U?$hb_zip_iter_t@U?$hb_sorted_array_t@UHBGlyphID16@OT@@@@U?$hb_array_t@UHBGlyphID16@OT@@@@@@AEBU<unnamed-type-hb_first>@@$00$0A@@@@Z 0000000180072e30 f i hb-ot-shaper-arabic.obj
 0001:00072120       ??$serialize@U?$hb_sorted_array_t@$$CBUHBGlyphID16@OT@@@@$0A@@?$CoverageFormat2_4@USmallTypes@Layout@OT@@@Common@Layout@OT@@AEAA_NPEAUhb_serialize_context_t@@U?$hb_sorted_array_t@$$CBUHBGlyphID16@OT@@@@@Z 0000000180073120 f i hb-ot-shaper-arabic.obj
 0001:00072340       ??$serialize@U?$hb_zip_iter_t@U?$hb_sorted_array_t@UHBGlyphID16@OT@@@@U?$hb_array_t@UHBGlyphID16@OT@@@@@@$0A@@SingleSubst@GSUB_impl@Layout@OT@@QEAA_NPEAUhb_serialize_context_t@@U?$hb_zip_iter_t@U?$hb_sorted_array_t@UHBGlyphID16@OT@@@@U?$hb_array_t@UHBGlyphID16@OT@@@@@@@Z 0000000180073340 f i hb-ot-shaper-arabic.obj
 0001:000727e0       ??$serialize_serialize@AEAU?$hb_map_iter_t@U?$hb_zip_iter_t@U?$hb_sorted_array_t@UHBGlyphID16@OT@@@@U?$hb_array_t@UHBGlyphID16@OT@@@@@@AEBU<unnamed-type-hb_first>@@$00$0A@@@@?$OffsetTo@UCoverage@Common@Layout@OT@@U?$IntType@G$01@4@$00@OT@@QEAA_NPEAUhb_serialize_context_t@@AEAU?$hb_map_iter_t@U?$hb_zip_iter_t@U?$hb_sorted_array_t@UHBGlyphID16@OT@@@@U?$hb_array_t@UHBGlyphID16@OT@@@@@@AEBU<unnamed-type-hb_first>@@$00$0A@@@@Z 00000001800737e0 f i hb-ot-shaper-arabic.obj
 0001:00072890       ??$serialize_serialize@AEAU?$hb_sorted_array_t@$$CBUHBGlyphID16@OT@@@@@?$OffsetTo@UCoverage@Common@Layout@OT@@U?$IntType@G$01@4@$00@OT@@QEAA_NPEAUhb_serialize_context_t@@AEAU?$hb_sorted_array_t@$$CBUHBGlyphID16@OT@@@@@Z 0000000180073890 f i hb-ot-shaper-arabic.obj
 0001:00072ac0       ??$start_serialize@USubstLookup@GSUB_impl@Layout@OT@@@hb_serialize_context_t@@QEAAPEAUSubstLookup@GSUB_impl@Layout@OT@@XZ 0000000180073ac0 f i hb-ot-shaper-arabic.obj
 0001:00074060       ?cmp@?$IntType@G$01@OT@@SAHPEBU12@0@Z 0000000180075060 f i hb-ot-shaper-arabic.obj
 0001:000740c0       ?discard_stale_objects@hb_serialize_context_t@@QEAAXXZ 00000001800750c0 f i hb-ot-shaper-arabic.obj
 0001:000742b0       ?end@?$hb_iter_t@U?$hb_map_iter_t@U?$hb_zip_iter_t@U?$hb_sorted_array_t@UHBGlyphID16@OT@@@@U?$hb_array_t@UHBGlyphID16@OT@@@@@@AEBU<unnamed-type-hb_first>@@$00$0A@@@AEAUHBGlyphID16@OT@@@@QEBA?AU?$hb_map_iter_t@U?$hb_zip_iter_t@U?$hb_sorted_array_t@UHBGlyphID16@OT@@@@U?$hb_array_t@UHBGlyphID16@OT@@@@@@AEBU<unnamed-type-hb_first>@@$00$0A@@@XZ 00000001800752b0 f i hb-ot-shaper-arabic.obj
 0001:00074520       ?pop_discard@hb_serialize_context_t@@QEAAXXZ 0000000180075520 f i hb-ot-shaper-arabic.obj
 0001:000745a0       ?push@?$hb_vector_t@Ulink_t@object_t@hb_serialize_context_t@@$0A@@@QEAAPEAUlink_t@object_t@hb_serialize_context_t@@XZ 00000001800755a0 f i hb-ot-shaper-arabic.obj
 0001:00074710       ?safe_to_insert_tatweel@hb_buffer_t@@QEAAXII@Z 0000000180075710 f i hb-ot-shaper-arabic.obj
 0001:000747a0       ?serialize@?$ArrayOf@UHBGlyphID16@OT@@U?$IntType@G$01@2@@OT@@QEAA_NPEAUhb_serialize_context_t@@I_N@Z 00000001800757a0 f i hb-ot-shaper-arabic.obj
 0001:000748b0       ?serialize@?$HeadlessArrayOf@UHBGlyphID16@OT@@U?$IntType@G$01@2@@OT@@QEAA_NPEAUhb_serialize_context_t@@I_N@Z 00000001800758b0 f i hb-ot-shaper-arabic.obj
 0001:000749d0       ?serialize@?$LigatureSet@USmallTypes@Layout@OT@@@GSUB_impl@Layout@OT@@QEAA_NPEAUhb_serialize_context_t@@U?$hb_array_t@$$CBUHBGlyphID16@OT@@@@U?$hb_array_t@$$CBI@@AEAU6@@Z 00000001800759d0 f i hb-ot-shaper-arabic.obj
 0001:00074dc0       ?serialize@?$LigatureSubstFormat1_2@USmallTypes@Layout@OT@@@GSUB_impl@Layout@OT@@QEAA_NPEAUhb_serialize_context_t@@U?$hb_sorted_array_t@$$CBUHBGlyphID16@OT@@@@U?$hb_array_t@$$CBI@@U?$hb_array_t@$$CBUHBGlyphID16@OT@@@@23@Z 0000000180075dc0 f i hb-ot-shaper-arabic.obj
 0001:00075150       ?serialize@?$SortedArrayOf@U?$RangeRecord@USmallTypes@Layout@OT@@@Common@Layout@OT@@U?$IntType@G$01@4@@OT@@QEAA_NPEAUhb_serialize_context_t@@I@Z 0000000180076150 f i hb-ot-shaper-arabic.obj
 0001:000752a0       ?serialize@Lookup@OT@@QEAA_NPEAUhb_serialize_context_t@@III@Z 00000001800762a0 f i hb-ot-shaper-arabic.obj
 0001:000754a0       ?setup_masks_arabic_plan@@YAXPEBUarabic_shape_plan_t@@PEAUhb_buffer_t@@W4hb_script_t@@@Z 00000001800764a0 f   hb-ot-shaper-arabic.obj
 0001:00076980       ?hb_indic_get_categories@@YAGI@Z 0000000180077980 f   hb-ot-shaper-indic-table.obj
 0001:00077ec0       ?find_syllables_indic@@YAXPEAUhb_buffer_t@@@Z 0000000180078ec0 f i hb-ot-shaper-indic.obj
 0001:00078570       ?init@hb_indic_would_substitute_feature_t@@QEAAXPEBUhb_ot_map_t@@I_N@Z 0000000180079570 f i hb-ot-shaper-indic.obj
 0001:00079760       ?would_substitute@hb_indic_would_substitute_feature_t@@QEBA_NPEBIIPEAUhb_face_t@@@Z 000000018007a760 f i hb-ot-shaper-indic.obj
 0001:00079c60       ?find_syllables_khmer@@YAXPEAUhb_buffer_t@@@Z 000000018007ac60 f i hb-ot-shaper-khmer.obj
 0001:0007a6d0       ?find_syllables_myanmar@@YAXPEAUhb_buffer_t@@@Z 000000018007b6d0 f i hb-ot-shaper-myanmar.obj
 0001:0007afa0       ?hb_syllabic_clear_var@@YA_NPEBUhb_ot_shape_plan_t@@PEAUhb_font_t@@PEAUhb_buffer_t@@@Z 000000018007bfa0 f   hb-ot-shaper-syllabic.obj
 0001:0007afb0       ?hb_syllabic_insert_dotted_circles@@YA_NPEAUhb_font_t@@PEAUhb_buffer_t@@IIHH@Z 000000018007bfb0 f   hb-ot-shaper-syllabic.obj
 0001:0007c050       ?__item__@?$hb_zip_iter_t@U?$hb_iota_iter_t@II@@U?$hb_array_t@Uhb_glyph_info_t@@@@@@QEBA?AU?$hb_pair_t@IAEAUhb_glyph_info_t@@@@XZ 000000018007d050 f i hb-ot-shaper-use.obj
 0001:0007e190       ?_hb_preprocess_text_vowel_constraints@@YAXPEBUhb_ot_shape_plan_t@@PEAUhb_buffer_t@@PEAUhb_font_t@@@Z 000000018007f190 f   hb-ot-shaper-vowel-constraints.obj
 0001:00081b70       hb_ot_tag_to_language      0000000180082b70 f   hb-ot-tag.obj
 0001:00081cf0       hb_ot_tags_from_script_and_language 0000000180082cf0 f   hb-ot-tag.obj
 0001:00082320       hb_ot_var_named_instance_get_design_coords 0000000180083320 f   hb-ot-var.obj
 0001:00082420       hb_ot_var_normalize_coords 0000000180083420 f   hb-ot-var.obj
 0001:00082670       ??$push@Uhb_outline_point_t@@U1@$0A@@?$hb_vector_t@Uhb_outline_point_t@@$0A@@@QEAAPEAUhb_outline_point_t@@$$QEAU1@@Z 0000000180083670 f i hb-outline.obj
 0001:00082750       ?control_area@hb_outline_t@@QEBAMXZ 0000000180083750 f   hb-outline.obj
 0001:000829d0       ?embolden@hb_outline_t@@QEAAXMMMM@Z 00000001800839d0 f   hb-outline.obj
 0001:00083060       ?hb_outline_recording_pen_get_funcs@@YAPEAUhb_draw_funcs_t@@XZ 0000000180084060 f   hb-outline.obj
 0001:00083230       ?replay@hb_outline_t@@QEBAXPEAUhb_draw_funcs_t@@PEAX@Z 0000000180084230 f   hb-outline.obj
 0001:000837e0       ?add_point@hb_extents_t@@QEAAXMM@Z 00000001800847e0 f i hb-paint-extents.obj
 0001:00083910       ?hb_paint_extents_get_funcs@@YAPEAUhb_paint_funcs_t@@XZ 0000000180084910 f   hb-paint-extents.obj
 0001:00083ed0       ?paint@hb_paint_extents_context_t@@QEAAXXZ 0000000180084ed0 f i hb-paint-extents.obj
 0001:00083f50       ?pop_group@hb_paint_extents_context_t@@QEAAXW4hb_paint_composite_mode_t@@@Z 0000000180084f50 f i hb-paint-extents.obj
 0001:000841a0       ?push_transform@hb_paint_extents_context_t@@QEAAXAEBUhb_transform_t@@@Z 00000001800851a0 f i hb-paint-extents.obj
 0001:00084410       ?transform_extents@hb_transform_t@@QEBAXAEAUhb_extents_t@@@Z 0000000180085410 f i hb-paint-extents.obj
 0001:00084650       ?union_@hb_bounds_t@@QEAAXAEBU1@@Z 0000000180085650 f i hb-paint-extents.obj
 0001:000846e0       hb_paint_funcs_create      00000001800856e0 f   hb-paint.obj
 0001:00084780       hb_paint_funcs_destroy     0000000180085780 f   hb-paint.obj
 0001:000849e0       hb_paint_funcs_get_empty   00000001800859e0 f   hb-paint.obj
 0001:000849f0       hb_paint_funcs_set_color_func 00000001800859f0 f   hb-paint.obj
 0001:00084b10       hb_paint_funcs_set_image_func 0000000180085b10 f   hb-paint.obj
 0001:00084c30       hb_paint_funcs_set_linear_gradient_func 0000000180085c30 f   hb-paint.obj
 0001:00084d50       hb_paint_funcs_set_pop_clip_func 0000000180085d50 f   hb-paint.obj
 0001:00084e70       hb_paint_funcs_set_pop_group_func 0000000180085e70 f   hb-paint.obj
 0001:00084f90       hb_paint_funcs_set_pop_transform_func 0000000180085f90 f   hb-paint.obj
 0001:000850b0       hb_paint_funcs_set_push_clip_glyph_func 00000001800860b0 f   hb-paint.obj
 0001:000851d0       hb_paint_funcs_set_push_clip_rectangle_func 00000001800861d0 f   hb-paint.obj
 0001:000852f0       hb_paint_funcs_set_push_group_func 00000001800862f0 f   hb-paint.obj
 0001:00085410       hb_paint_funcs_set_push_transform_func 0000000180086410 f   hb-paint.obj
 0001:00085530       hb_paint_funcs_set_radial_gradient_func 0000000180086530 f   hb-paint.obj
 0001:00085650       hb_paint_funcs_set_sweep_gradient_func 0000000180086650 f   hb-paint.obj
 0001:00085770       ??1hb_ot_map_t@@QEAA@XZ    0000000180086770 f i hb-shape-plan.obj
 0001:000859e0       ?init@hb_shape_plan_key_t@@QEAA_N_NPEAUhb_face_t@@PEBUhb_segment_properties_t@@PEBUhb_feature_t@@IPEBHIPEBQEBD@Z 00000001800869e0 f   hb-shape-plan.obj
 0001:00085d40       hb_shape_plan_create2      0000000180086d40 f   hb-shape-plan.obj
 0001:00085f00       hb_shape_plan_create_cached2 0000000180086f00 f   hb-shape-plan.obj
 0001:000864c0       hb_shape_plan_destroy      00000001800874c0 f   hb-shape-plan.obj
 0001:00086550       hb_shape_plan_execute      0000000180087550 f   hb-shape-plan.obj
 0001:00086580       hb_shape_full              0000000180087580 f   hb-shape.obj
 0001:000866d0       ?_hb_shapers_get@@YAPEBUhb_shaper_entry_t@@XZ 00000001800876d0 f   hb-shaper.obj
 0001:000866e0       ?get_stored@?$hb_lazy_loader_t@Uhb_shaper_entry_t@@Uhb_shapers_lazy_loader_t@@X$0A@U1@@@QEBAPEAUhb_shaper_entry_t@@XZ 00000001800876e0 f i hb-shaper.obj
 0001:00086ec0       hb_ucd_get_unicode_funcs   0000000180087ec0 f   hb-ucd.obj
 0001:00087000       ?_hb_unicode_is_emoji_Extended_Pictographic@@YA_NI@Z 0000000180088000 f   hb-unicode.obj
 0001:00087080       hb_unicode_funcs_create    0000000180088080 f   hb-unicode.obj
 0001:00087160       hb_unicode_funcs_destroy   0000000180088160 f   hb-unicode.obj
 0001:00087280       hb_unicode_funcs_get_default 0000000180088280 f   hb-unicode.obj
 0001:00087290       hb_unicode_funcs_get_empty 0000000180088290 f   hb-unicode.obj
 0001:000872a0       hb_unicode_funcs_set_combining_class_func 00000001800882a0 f   hb-unicode.obj
 0001:00087330       hb_unicode_funcs_set_compose_func 0000000180088330 f   hb-unicode.obj
 0001:000873d0       hb_unicode_funcs_set_decompose_func 00000001800883d0 f   hb-unicode.obj
 0001:00087470       hb_unicode_funcs_set_general_category_func 0000000180088470 f   hb-unicode.obj
 0001:00087500       hb_unicode_funcs_set_mirroring_func 0000000180088500 f   hb-unicode.obj
 0001:00087590       hb_unicode_funcs_set_script_func 0000000180088590 f   hb-unicode.obj
 0001:00087620       Java_sun_font_FileFontStrike__1getGlyphImageFromWindows 0000000180088620 f   lcdglyph.obj
 0001:00087fc0       Java_sun_font_FileFontStrike_initNative 0000000180088fc0 f   lcdglyph.obj
 0001:00087fe0       getHBScriptCode            0000000180088fe0 f   scriptMapping.obj
 0001:00088000       Java_sun_font_NullFontScaler_getGlyphImage 0000000180089000 f   sunFont.obj
 0001:00088010       Java_sun_font_NullFontScaler_getNullScalerContext 0000000180089010 f   sunFont.obj
 0001:00088040       Java_sun_font_StrikeCache_freeIntMemory 0000000180089040 f   sunFont.obj
 0001:00088130       Java_sun_font_StrikeCache_freeIntPointer 0000000180089130 f   sunFont.obj
 0001:00088140       Java_sun_font_StrikeCache_freeLongMemory 0000000180089140 f   sunFont.obj
 0001:00088230       Java_sun_font_StrikeCache_freeLongPointer 0000000180089230 f   sunFont.obj
 0001:00088240       Java_sun_font_StrikeCache_getGlyphCacheDescription 0000000180089240 f   sunFont.obj
 0001:00088340       Java_sun_font_SunFontManager_initIDs 0000000180089340 f   sunFont.obj
 0001:00088350       getSunFontIDs              0000000180089350 f   sunFont.obj
 0001:00088b80       isNullScalerContext        0000000180089b80 f   sunFont.obj
 0001:00088b8d       FT_Init_FreeType           0000000180089b8d f   freetype:freetype.dll
 0001:00088b93       FT_Done_FreeType           0000000180089b93 f   freetype:freetype.dll
 0001:00088b99       FT_New_Memory_Face         0000000180089b99 f   freetype:freetype.dll
 0001:00088b9f       FT_Open_Face               0000000180089b9f f   freetype:freetype.dll
 0001:00088ba5       FT_Done_Face               0000000180089ba5 f   freetype:freetype.dll
 0001:00088bab       FT_Set_Char_Size           0000000180089bab f   freetype:freetype.dll
 0001:00088bb1       FT_Load_Glyph              0000000180089bb1 f   freetype:freetype.dll
 0001:00088bb7       FT_Set_Transform           0000000180089bb7 f   freetype:freetype.dll
 0001:00088bbd       FT_Render_Glyph            0000000180089bbd f   freetype:freetype.dll
 0001:00088bc3       FT_Get_Char_Index          0000000180089bc3 f   freetype:freetype.dll
 0001:00088bc9       FT_MulFix                  0000000180089bc9 f   freetype:freetype.dll
 0001:00088bcf       FT_Matrix_Multiply         0000000180089bcf f   freetype:freetype.dll
 0001:00088bd5       FT_Outline_Get_BBox        0000000180089bd5 f   freetype:freetype.dll
 0001:00088bdb       FT_Activate_Size           0000000180089bdb f   freetype:freetype.dll
 0001:00088be1       FT_Outline_Decompose       0000000180089be1 f   freetype:freetype.dll
 0001:00088be7       FT_Outline_Get_CBox        0000000180089be7 f   freetype:freetype.dll
 0001:00088bed       FT_Outline_Translate       0000000180089bed f   freetype:freetype.dll
 0001:00088bf3       FT_Outline_Embolden        0000000180089bf3 f   freetype:freetype.dll
 0001:00088bf9       FT_Library_SetLcdFilter    0000000180089bf9 f   freetype:freetype.dll
 0001:00088bff       FT_Property_Set            0000000180089bff f   freetype:freetype.dll
 0001:00088c05       JNU_ThrowOutOfMemoryError  0000000180089c05 f   java:java.dll
 0001:00088c0b       JNU_ThrowInternalError     0000000180089c0b f   java:java.dll
 0001:00088c11       JNU_ThrowArrayIndexOutOfBoundsException 0000000180089c11 f   java:java.dll
 0001:00088c17       JNU_NewStringPlatform      0000000180089c17 f   java:java.dll
 0001:00088c1d       JNU_CallStaticMethodByName 0000000180089c1d f   java:java.dll
 0001:00088c23       SurfaceData_GetOps         0000000180089c23 f   awt:awt.dll
 0001:00088c29       SurfaceData_IntersectBounds 0000000180089c29 f   awt:awt.dll
 0001:00088c2f       SurfaceData_InitOps        0000000180089c2f f   awt:awt.dll
 0001:00088c35       GetNativePrim              0000000180089c35 f   awt:awt.dll
 0001:00088c3b       GrPrim_Sg2dGetCompInfo     0000000180089c3b f   awt:awt.dll
 0001:00088c41       GrPrim_Sg2dGetClip         0000000180089c41 f   awt:awt.dll
 0001:00088c47       GrPrim_Sg2dGetPixel        0000000180089c47 f   awt:awt.dll
 0001:00088c4d       GrPrim_Sg2dGetEaRGB        0000000180089c4d f   awt:awt.dll
 0001:00088c53       GrPrim_Sg2dGetLCDTextContrast 0000000180089c53 f   awt:awt.dll
 0001:00088c59       AccelGlyphCache_RemoveAllCellInfos 0000000180089c59 f   awt:awt.dll
 0001:00088c60       __GSHandlerCheck           0000000180089c60 f   MSVCRT:gshandler.obj
 0001:00088c80       __GSHandlerCheckCommon     0000000180089c80 f   MSVCRT:gshandler.obj
 0001:00088cf0       __security_check_cookie    0000000180089cf0 f   MSVCRT:amdsecgs.obj
 0001:00088d10       __raise_securityfailure    0000000180089d10 f   MSVCRT:gs_report.obj
 0001:00088d44       __report_gsfailure         0000000180089d44 f   MSVCRT:gs_report.obj
 0001:00088e18       __report_rangecheckfailure 0000000180089e18 f   MSVCRT:gs_report.obj
 0001:00088e2c       __report_securityfailure   0000000180089e2c f   MSVCRT:gs_report.obj
 0001:00088fc0       __chkstk                   0000000180089fc0 f   MSVCRT:chkstk.obj
 0001:00088fc0       _alloca_probe              0000000180089fc0 f   MSVCRT:chkstk.obj
 0001:00089010       __vdecl_floorf4            000000018008a010 f   MSVCRT:svml_sfloorf4_dispatch.obj
 0001:00089344       _DllMainCRTStartup         000000018008a344 f   MSVCRT:dll_dllmain.obj
 0001:00089384       __isa_available_init       000000018008a384 f   MSVCRT:cpu_disp.obj
 0001:00089530       __sse2_floorf4@@16         000000018008a530 f   MSVCRT:svml_sfloorf4_sse2.obj
 0001:00089580       __sse4_floorf4@@16         000000018008a580 f   MSVCRT:svml_sfloorf4_sse4.obj
 0001:00089588       __security_init_cookie     000000018008a588 f   MSVCRT:gs_support.obj
 0001:00089634       DllMain                    000000018008a634 f   MSVCRT:dll_dllmain_stub.obj
 0001:00089658       ?__scrt_initialize_type_info@@YAXXZ 000000018008a658 f   MSVCRT:tncleanup.obj
 0001:00089668       ?__scrt_uninitialize_type_info@@YAXXZ 000000018008a668 f   MSVCRT:tncleanup.obj
 0001:00089674       __local_stdio_scanf_options 000000018008a674 f i MSVCRT:default_local_stdio_options.obj
 0001:0008967c       __scrt_initialize_default_local_stdio_options 000000018008a67c f   MSVCRT:default_local_stdio_options.obj
 0001:00089698       __scrt_acquire_startup_lock 000000018008a698 f   MSVCRT:utility.obj
 0001:000896d4       __scrt_dllmain_after_initialize_c 000000018008a6d4 f   MSVCRT:utility.obj
 0001:00089708       __scrt_dllmain_before_initialize_c 000000018008a708 f   MSVCRT:utility.obj
 0001:00089720       __scrt_dllmain_crt_thread_attach 000000018008a720 f   MSVCRT:utility.obj
 0001:00089748       __scrt_dllmain_crt_thread_detach 000000018008a748 f   MSVCRT:utility.obj
 0001:00089760       __scrt_dllmain_exception_filter 000000018008a760 f   MSVCRT:utility.obj
 0001:000897c0       __scrt_dllmain_uninitialize_c 000000018008a7c0 f   MSVCRT:utility.obj
 0001:000897f0       __scrt_dllmain_uninitialize_critical 000000018008a7f0 f   MSVCRT:utility.obj
 0001:00089804       __scrt_initialize_crt      000000018008a804 f   MSVCRT:utility.obj
 0001:00089850       __scrt_initialize_onexit_tables 000000018008a850 f   MSVCRT:utility.obj
 0001:000898dc       __scrt_is_nonwritable_in_current_image 000000018008a8dc f   MSVCRT:utility.obj
 0001:00089974       __scrt_release_startup_lock 000000018008a974 f   MSVCRT:utility.obj
 0001:00089998       __scrt_uninitialize_crt    000000018008a998 f   MSVCRT:utility.obj
 0001:000899c4       __scrt_get_dyn_tls_init_callback 000000018008a9c4 f   MSVCRT:dyn_tls_init.obj
 0001:000899cc       __crt_debugger_hook        000000018008a9cc f   MSVCRT:utility_desktop.obj
 0001:000899d4       __scrt_fastfail            000000018008a9d4 f   MSVCRT:utility_desktop.obj
 0001:00089b20       _RTC_Initialize            000000018008ab20 f   MSVCRT:initsect.obj
 0001:00089b5c       _RTC_Terminate             000000018008ab5c f   MSVCRT:initsect.obj
 0001:00089b98       __scrt_is_ucrt_dll_in_use  000000018008ab98 f   MSVCRT:ucrt_detection.obj
 0001:00089bb0       memset                     000000018008abb0 f   vcruntime:VCRUNTIME140.dll
 0001:00089bb6       strrchr                    000000018008abb6 f   vcruntime:VCRUNTIME140.dll
 0001:00089bbc       wcsrchr                    000000018008abbc f   vcruntime:VCRUNTIME140.dll
 0001:00089bc2       wcsstr                     000000018008abc2 f   vcruntime:VCRUNTIME140.dll
 0001:00089bc8       strstr                     000000018008abc8 f   vcruntime:VCRUNTIME140.dll
 0001:00089bce       memcpy                     000000018008abce f   vcruntime:VCRUNTIME140.dll
 0001:00089bd4       memmove                    000000018008abd4 f   vcruntime:VCRUNTIME140.dll
 0001:00089bda       strchr                     000000018008abda f   vcruntime:VCRUNTIME140.dll
 0001:00089be0       memcmp                     000000018008abe0 f   vcruntime:VCRUNTIME140.dll
 0001:00089be6       __C_specific_handler       000000018008abe6 f   vcruntime:VCRUNTIME140.dll
 0001:00089bec       __std_type_info_destroy_list 000000018008abec f   vcruntime:VCRUNTIME140.dll
 0001:00089bf2       floor                      000000018008abf2 f   ucrt:api-ms-win-crt-math-l1-1-0.dll
 0001:00089bf8       pow                        000000018008abf8 f   ucrt:api-ms-win-crt-math-l1-1-0.dll
 0001:00089bfe       sqrt                       000000018008abfe f   ucrt:api-ms-win-crt-math-l1-1-0.dll
 0001:00089c04       floorf                     000000018008ac04 f   ucrt:api-ms-win-crt-math-l1-1-0.dll
 0001:00089c0a       ceilf                      000000018008ac0a f   ucrt:api-ms-win-crt-math-l1-1-0.dll
 0001:00089c10       cosf                       000000018008ac10 f   ucrt:api-ms-win-crt-math-l1-1-0.dll
 0001:00089c16       sinf                       000000018008ac16 f   ucrt:api-ms-win-crt-math-l1-1-0.dll
 0001:00089c1c       tanf                       000000018008ac1c f   ucrt:api-ms-win-crt-math-l1-1-0.dll
 0001:00089c22       strcmp                     000000018008ac22 f   ucrt:api-ms-win-crt-string-l1-1-0.dll
 0001:00089c28       _hypotf                    000000018008ac28 f   ucrt:api-ms-win-crt-math-l1-1-0.dll
 0001:00089c2e       _initterm                  000000018008ac2e f   ucrt:api-ms-win-crt-runtime-l1-1-0.dll
 0001:00089c34       _initterm_e                000000018008ac34 f   ucrt:api-ms-win-crt-runtime-l1-1-0.dll
 0001:00089c3a       _seh_filter_dll            000000018008ac3a f   ucrt:api-ms-win-crt-runtime-l1-1-0.dll
 0001:00089c40       _configure_narrow_argv     000000018008ac40 f   ucrt:api-ms-win-crt-runtime-l1-1-0.dll
 0001:00089c46       _initialize_narrow_environment 000000018008ac46 f   ucrt:api-ms-win-crt-runtime-l1-1-0.dll
 0001:00089c4c       _initialize_onexit_table   000000018008ac4c f   ucrt:api-ms-win-crt-runtime-l1-1-0.dll
 0001:00089c52       _execute_onexit_table      000000018008ac52 f   ucrt:api-ms-win-crt-runtime-l1-1-0.dll
 0001:00089c58       _cexit                     000000018008ac58 f   ucrt:api-ms-win-crt-runtime-l1-1-0.dll
 0001:00089c60       __acrt_initialize          000000018008ac60 f   MSVCRT:ucrt_stubs.obj
 0001:00089c60       __acrt_thread_attach       000000018008ac60 f   MSVCRT:ucrt_stubs.obj
 0001:00089c60       __acrt_thread_detach       000000018008ac60 f   MSVCRT:ucrt_stubs.obj
 0001:00089c60       __acrt_uninitialize        000000018008ac60 f   MSVCRT:ucrt_stubs.obj
 0001:00089c60       __acrt_uninitialize_critical 000000018008ac60 f   MSVCRT:ucrt_stubs.obj
 0001:00089c60       __scrt_stub_for_acrt_initialize 000000018008ac60 f   MSVCRT:ucrt_stubs.obj
 0001:00089c60       __scrt_stub_for_acrt_thread_attach 000000018008ac60 f   MSVCRT:ucrt_stubs.obj
 0001:00089c60       __scrt_stub_for_acrt_thread_detach 000000018008ac60 f   MSVCRT:ucrt_stubs.obj
 0001:00089c60       __scrt_stub_for_acrt_uninitialize 000000018008ac60 f   MSVCRT:ucrt_stubs.obj
 0001:00089c60       __scrt_stub_for_acrt_uninitialize_critical 000000018008ac60 f   MSVCRT:ucrt_stubs.obj
 0001:00089c60       __vcrt_initialize          000000018008ac60 f   MSVCRT:ucrt_stubs.obj
 0001:00089c60       __vcrt_thread_attach       000000018008ac60 f   MSVCRT:ucrt_stubs.obj
 0001:00089c60       __vcrt_thread_detach       000000018008ac60 f   MSVCRT:ucrt_stubs.obj
 0001:00089c60       __vcrt_uninitialize        000000018008ac60 f   MSVCRT:ucrt_stubs.obj
 0001:00089c60       __vcrt_uninitialize_critical 000000018008ac60 f   MSVCRT:ucrt_stubs.obj
 0001:00089c80       _guard_dispatch_icall_nop  000000018008ac80 f   MSVCRT:guard_dispatch.obj
 0001:00089ca0       _guard_xfg_dispatch_icall_nop 000000018008aca0 f   MSVCRT:guard_xfg_dispatch.obj
 0002:00000000       __imp_RegCloseKey          000000018008b000     advapi32:ADVAPI32.dll
 0002:00000008       __imp_RegOpenKeyExA        000000018008b008     advapi32:ADVAPI32.dll
 0002:00000010       __imp_RegQueryInfoKeyW     000000018008b010     advapi32:ADVAPI32.dll
 0002:00000018       __imp_RegEnumValueW        000000018008b018     advapi32:ADVAPI32.dll
 0002:00000020       \177ADVAPI32_NULL_THUNK_DATA 000000018008b020     advapi32:ADVAPI32.dll
 0002:00000028       __imp_GetDIBits            000000018008b028     gdi32:GDI32.dll
 0002:00000030       __imp_GetDeviceCaps        000000018008b030     gdi32:GDI32.dll
 0002:00000038       __imp_DeleteObject         000000018008b038     gdi32:GDI32.dll
 0002:00000040       __imp_CreateFontIndirectW  000000018008b040     gdi32:GDI32.dll
 0002:00000048       __imp_CreateCompatibleDC   000000018008b048     gdi32:GDI32.dll
 0002:00000050       __imp_GetGlyphOutlineA     000000018008b050     gdi32:GDI32.dll
 0002:00000058       __imp_EnumFontFamiliesExW  000000018008b058     gdi32:GDI32.dll
 0002:00000060       __imp_SetMapMode           000000018008b060     gdi32:GDI32.dll
 0002:00000068       __imp_SetTextColor         000000018008b068     gdi32:GDI32.dll
 0002:00000070       __imp_GetTextMetricsA      000000018008b070     gdi32:GDI32.dll
 0002:00000078       __imp_ExtTextOutW          000000018008b078     gdi32:GDI32.dll
 0002:00000080       __imp_GetFontData          000000018008b080     gdi32:GDI32.dll
 0002:00000088       __imp_GetStockObject       000000018008b088     gdi32:GDI32.dll
 0002:00000090       __imp_SelectObject         000000018008b090     gdi32:GDI32.dll
 0002:00000098       __imp_CreateCompatibleBitmap 000000018008b098     gdi32:GDI32.dll
 0002:000000a0       __imp_SetBkColor           000000018008b0a0     gdi32:GDI32.dll
 0002:000000a8       \177GDI32_NULL_THUNK_DATA  000000018008b0a8     gdi32:GDI32.dll
 0002:000000b0       __imp_DeleteCriticalSection 000000018008b0b0     kernel32:KERNEL32.dll
 0002:000000b8       __imp_EnterCriticalSection 000000018008b0b8     kernel32:KERNEL32.dll
 0002:000000c0       __imp_InitializeCriticalSection 000000018008b0c0     kernel32:KERNEL32.dll
 0002:000000c8       __imp_RtlCaptureContext    000000018008b0c8     kernel32:KERNEL32.dll
 0002:000000d0       __imp_GetWindowsDirectoryA 000000018008b0d0     kernel32:KERNEL32.dll
 0002:000000d8       __imp_GetSystemDirectoryA  000000018008b0d8     kernel32:KERNEL32.dll
 0002:000000e0       __imp_RtlVirtualUnwind     000000018008b0e0     kernel32:KERNEL32.dll
 0002:000000e8       __imp_RtlLookupFunctionEntry 000000018008b0e8     kernel32:KERNEL32.dll
 0002:000000f0       __imp_UnhandledExceptionFilter 000000018008b0f0     kernel32:KERNEL32.dll
 0002:000000f8       __imp_SetUnhandledExceptionFilter 000000018008b0f8     kernel32:KERNEL32.dll
 0002:00000100       __imp_GetCurrentProcess    000000018008b100     kernel32:KERNEL32.dll
 0002:00000108       __imp_TerminateProcess     000000018008b108     kernel32:KERNEL32.dll
 0002:00000110       __imp_IsProcessorFeaturePresent 000000018008b110     kernel32:KERNEL32.dll
 0002:00000118       __imp_QueryPerformanceCounter 000000018008b118     kernel32:KERNEL32.dll
 0002:00000120       __imp_GetCurrentProcessId  000000018008b120     kernel32:KERNEL32.dll
 0002:00000128       __imp_GetCurrentThreadId   000000018008b128     kernel32:KERNEL32.dll
 0002:00000130       __imp_GetSystemTimeAsFileTime 000000018008b130     kernel32:KERNEL32.dll
 0002:00000138       __imp_DisableThreadLibraryCalls 000000018008b138     kernel32:KERNEL32.dll
 0002:00000140       __imp_InitializeSListHead  000000018008b140     kernel32:KERNEL32.dll
 0002:00000148       __imp_IsDebuggerPresent    000000018008b148     kernel32:KERNEL32.dll
 0002:00000150       __imp_LeaveCriticalSection 000000018008b150     kernel32:KERNEL32.dll
 0002:00000158       \177KERNEL32_NULL_THUNK_DATA 000000018008b158     kernel32:KERNEL32.dll
 0002:00000160       __imp_GetDesktopWindow     000000018008b160     user32:USER32.dll
 0002:00000168       __imp_FillRect             000000018008b168     user32:USER32.dll
 0002:00000170       __imp_GetWindowDC          000000018008b170     user32:USER32.dll
 0002:00000178       __imp_GetDC                000000018008b178     user32:USER32.dll
 0002:00000180       __imp_ReleaseDC            000000018008b180     user32:USER32.dll
 0002:00000188       __imp_SystemParametersInfoA 000000018008b188     user32:USER32.dll
 0002:00000190       \177USER32_NULL_THUNK_DATA 000000018008b190     user32:USER32.dll
 0002:00000198       __imp_memcmp               000000018008b198     vcruntime:VCRUNTIME140.dll
 0002:000001a0       __imp_strchr               000000018008b1a0     vcruntime:VCRUNTIME140.dll
 0002:000001a8       __imp___C_specific_handler 000000018008b1a8     vcruntime:VCRUNTIME140.dll
 0002:000001b0       __imp_memcpy               000000018008b1b0     vcruntime:VCRUNTIME140.dll
 0002:000001b8       __imp_strstr               000000018008b1b8     vcruntime:VCRUNTIME140.dll
 0002:000001c0       __imp_wcsstr               000000018008b1c0     vcruntime:VCRUNTIME140.dll
 0002:000001c8       __imp_wcsrchr              000000018008b1c8     vcruntime:VCRUNTIME140.dll
 0002:000001d0       __imp_strrchr              000000018008b1d0     vcruntime:VCRUNTIME140.dll
 0002:000001d8       __imp___std_type_info_destroy_list 000000018008b1d8     vcruntime:VCRUNTIME140.dll
 0002:000001e0       __imp_memset               000000018008b1e0     vcruntime:VCRUNTIME140.dll
 0002:000001e8       __imp_memmove              000000018008b1e8     vcruntime:VCRUNTIME140.dll
 0002:000001f0       \177VCRUNTIME140_NULL_THUNK_DATA 000000018008b1f0     vcruntime:VCRUNTIME140.dll
 0002:000001f8       __imp_strtol               000000018008b1f8     ucrt:api-ms-win-crt-convert-l1-1-0.dll
 0002:00000200       \177api-ms-win-crt-convert-l1-1-0_NULL_THUNK_DATA 000000018008b200     ucrt:api-ms-win-crt-convert-l1-1-0.dll
 0002:00000208       __imp_getenv               000000018008b208     ucrt:api-ms-win-crt-environment-l1-1-0.dll
 0002:00000210       \177api-ms-win-crt-environment-l1-1-0_NULL_THUNK_DATA 000000018008b210     ucrt:api-ms-win-crt-environment-l1-1-0.dll
 0002:00000218       __imp_malloc               000000018008b218     ucrt:api-ms-win-crt-heap-l1-1-0.dll
 0002:00000220       __imp_calloc               000000018008b220     ucrt:api-ms-win-crt-heap-l1-1-0.dll
 0002:00000228       __imp_realloc              000000018008b228     ucrt:api-ms-win-crt-heap-l1-1-0.dll
 0002:00000230       __imp_free                 000000018008b230     ucrt:api-ms-win-crt-heap-l1-1-0.dll
 0002:00000238       \177api-ms-win-crt-heap-l1-1-0_NULL_THUNK_DATA 000000018008b238     ucrt:api-ms-win-crt-heap-l1-1-0.dll
 0002:00000240       __imp_tanf                 000000018008b240     ucrt:api-ms-win-crt-math-l1-1-0.dll
 0002:00000248       __imp__hypotf              000000018008b248     ucrt:api-ms-win-crt-math-l1-1-0.dll
 0002:00000250       __imp_floor                000000018008b250     ucrt:api-ms-win-crt-math-l1-1-0.dll
 0002:00000258       __imp_sqrt                 000000018008b258     ucrt:api-ms-win-crt-math-l1-1-0.dll
 0002:00000260       __imp_sinf                 000000018008b260     ucrt:api-ms-win-crt-math-l1-1-0.dll
 0002:00000268       __imp_floorf               000000018008b268     ucrt:api-ms-win-crt-math-l1-1-0.dll
 0002:00000270       __imp_ceilf                000000018008b270     ucrt:api-ms-win-crt-math-l1-1-0.dll
 0002:00000278       __imp_pow                  000000018008b278     ucrt:api-ms-win-crt-math-l1-1-0.dll
 0002:00000280       __imp_cosf                 000000018008b280     ucrt:api-ms-win-crt-math-l1-1-0.dll
 0002:00000288       \177api-ms-win-crt-math-l1-1-0_NULL_THUNK_DATA 000000018008b288     ucrt:api-ms-win-crt-math-l1-1-0.dll
 0002:00000290       __imp__errno               000000018008b290     ucrt:api-ms-win-crt-runtime-l1-1-0.dll
 0002:00000298       __imp__execute_onexit_table 000000018008b298     ucrt:api-ms-win-crt-runtime-l1-1-0.dll
 0002:000002a0       __imp__initialize_onexit_table 000000018008b2a0     ucrt:api-ms-win-crt-runtime-l1-1-0.dll
 0002:000002a8       __imp__initialize_narrow_environment 000000018008b2a8     ucrt:api-ms-win-crt-runtime-l1-1-0.dll
 0002:000002b0       __imp__configure_narrow_argv 000000018008b2b0     ucrt:api-ms-win-crt-runtime-l1-1-0.dll
 0002:000002b8       __imp__seh_filter_dll      000000018008b2b8     ucrt:api-ms-win-crt-runtime-l1-1-0.dll
 0002:000002c0       __imp__initterm            000000018008b2c0     ucrt:api-ms-win-crt-runtime-l1-1-0.dll
 0002:000002c8       __imp__cexit               000000018008b2c8     ucrt:api-ms-win-crt-runtime-l1-1-0.dll
 0002:000002d0       __imp__initterm_e          000000018008b2d0     ucrt:api-ms-win-crt-runtime-l1-1-0.dll
 0002:000002d8       \177api-ms-win-crt-runtime-l1-1-0_NULL_THUNK_DATA 000000018008b2d8     ucrt:api-ms-win-crt-runtime-l1-1-0.dll
 0002:000002e0       __imp___stdio_common_vsprintf 000000018008b2e0     ucrt:api-ms-win-crt-stdio-l1-1-0.dll
 0002:000002e8       __imp___stdio_common_vfprintf 000000018008b2e8     ucrt:api-ms-win-crt-stdio-l1-1-0.dll
 0002:000002f0       __imp___acrt_iob_func      000000018008b2f0     ucrt:api-ms-win-crt-stdio-l1-1-0.dll
 0002:000002f8       \177api-ms-win-crt-stdio-l1-1-0_NULL_THUNK_DATA 000000018008b2f8     ucrt:api-ms-win-crt-stdio-l1-1-0.dll
 0002:00000300       __imp__stricmp             000000018008b300     ucrt:api-ms-win-crt-string-l1-1-0.dll
 0002:00000300       __imp_stricmp              000000018008b300     ucrt:api-ms-win-crt-string-l1-1-0.dll
 0002:00000308       __imp_strncpy              000000018008b308     ucrt:api-ms-win-crt-string-l1-1-0.dll
 0002:00000310       __imp__wcsicmp             000000018008b310     ucrt:api-ms-win-crt-string-l1-1-0.dll
 0002:00000310       __imp_wcsicmp              000000018008b310     ucrt:api-ms-win-crt-string-l1-1-0.dll
 0002:00000318       __imp_strncmp              000000018008b318     ucrt:api-ms-win-crt-string-l1-1-0.dll
 0002:00000320       __imp_strcmp               000000018008b320     ucrt:api-ms-win-crt-string-l1-1-0.dll
 0002:00000328       \177api-ms-win-crt-string-l1-1-0_NULL_THUNK_DATA 000000018008b328     ucrt:api-ms-win-crt-string-l1-1-0.dll
 0002:00000330       __imp_GetNativePrim        000000018008b330     awt:awt.dll
 0002:00000338       __imp_GrPrim_Sg2dGetCompInfo 000000018008b338     awt:awt.dll
 0002:00000340       __imp_GrPrim_Sg2dGetClip   000000018008b340     awt:awt.dll
 0002:00000348       __imp_GrPrim_Sg2dGetPixel  000000018008b348     awt:awt.dll
 0002:00000350       __imp_SurfaceData_InitOps  000000018008b350     awt:awt.dll
 0002:00000358       __imp_SurfaceData_IntersectBounds 000000018008b358     awt:awt.dll
 0002:00000360       __imp_GrPrim_Sg2dGetEaRGB  000000018008b360     awt:awt.dll
 0002:00000368       __imp_GrPrim_Sg2dGetLCDTextContrast 000000018008b368     awt:awt.dll
 0002:00000370       __imp_AccelGlyphCache_RemoveAllCellInfos 000000018008b370     awt:awt.dll
 0002:00000378       __imp_SurfaceData_GetOps   000000018008b378     awt:awt.dll
 0002:00000380       \177awt_NULL_THUNK_DATA    000000018008b380     awt:awt.dll
 0002:00000388       __imp_FT_Init_FreeType     000000018008b388     freetype:freetype.dll
 0002:00000390       __imp_FT_Done_Face         000000018008b390     freetype:freetype.dll
 0002:00000398       __imp_FT_Open_Face         000000018008b398     freetype:freetype.dll
 0002:000003a0       __imp_FT_Property_Set      000000018008b3a0     freetype:freetype.dll
 0002:000003a8       __imp_FT_Library_SetLcdFilter 000000018008b3a8     freetype:freetype.dll
 0002:000003b0       __imp_FT_Outline_Embolden  000000018008b3b0     freetype:freetype.dll
 0002:000003b8       __imp_FT_Outline_Translate 000000018008b3b8     freetype:freetype.dll
 0002:000003c0       __imp_FT_Outline_Get_CBox  000000018008b3c0     freetype:freetype.dll
 0002:000003c8       __imp_FT_Outline_Decompose 000000018008b3c8     freetype:freetype.dll
 0002:000003d0       __imp_FT_Activate_Size     000000018008b3d0     freetype:freetype.dll
 0002:000003d8       __imp_FT_Outline_Get_BBox  000000018008b3d8     freetype:freetype.dll
 0002:000003e0       __imp_FT_Matrix_Multiply   000000018008b3e0     freetype:freetype.dll
 0002:000003e8       __imp_FT_MulFix            000000018008b3e8     freetype:freetype.dll
 0002:000003f0       __imp_FT_Get_Char_Index    000000018008b3f0     freetype:freetype.dll
 0002:000003f8       __imp_FT_Render_Glyph      000000018008b3f8     freetype:freetype.dll
 0002:00000400       __imp_FT_Set_Transform     000000018008b400     freetype:freetype.dll
 0002:00000408       __imp_FT_Load_Glyph        000000018008b408     freetype:freetype.dll
 0002:00000410       __imp_FT_Set_Char_Size     000000018008b410     freetype:freetype.dll
 0002:00000418       __imp_FT_Done_FreeType     000000018008b418     freetype:freetype.dll
 0002:00000420       __imp_FT_New_Memory_Face   000000018008b420     freetype:freetype.dll
 0002:00000428       \177freetype_NULL_THUNK_DATA 000000018008b428     freetype:freetype.dll
 0002:00000430       __imp_JNU_ThrowArrayIndexOutOfBoundsException 000000018008b430     java:java.dll
 0002:00000438       __imp_JNU_NewStringPlatform 000000018008b438     java:java.dll
 0002:00000440       __imp_JNU_CallStaticMethodByName 000000018008b440     java:java.dll
 0002:00000448       __imp_JNU_ThrowOutOfMemoryError 000000018008b448     java:java.dll
 0002:00000450       __imp_JNU_ThrowInternalError 000000018008b450     java:java.dll
 0002:00000458       \177java_NULL_THUNK_DATA   000000018008b458     java:java.dll
 0002:00000460       __guard_check_icall_fptr   000000018008b460     MSVCRT:guard_support.obj
 0002:00000468       __guard_xfg_check_icall_fptr 000000018008b468     MSVCRT:guard_support.obj
 0002:00000470       __guard_dispatch_icall_fptr 000000018008b470     MSVCRT:guard_support.obj
 0002:00000478       __guard_xfg_dispatch_icall_fptr 000000018008b478     MSVCRT:guard_support.obj
 0002:00000480       __guard_xfg_table_dispatch_icall_fptr 000000018008b480     MSVCRT:guard_support.obj
 0002:00000488       __castguard_check_failure_os_handled_fptr 000000018008b488     MSVCRT:guard_support.obj
 0002:00000490       __guard_memcpy_fptr        000000018008b490     vcruntime:softmemtag.obj
 0002:00000498       __xc_a                     000000018008b498     MSVCRT:initializers.obj
 0002:000004a0       __xc_z                     000000018008b4a0     MSVCRT:initializers.obj
 0002:000004a8       __xi_a                     000000018008b4a8     MSVCRT:initializers.obj
 0002:000004b0       __xi_z                     000000018008b4b0     MSVCRT:initializers.obj
 0002:000004b8       __xp_a                     000000018008b4b8     MSVCRT:initializers.obj
 0002:000004c0       __xp_z                     000000018008b4c0     MSVCRT:initializers.obj
 0002:000004c8       __xt_a                     000000018008b4c8     MSVCRT:initializers.obj
 0002:000004d0       __xt_z                     000000018008b4d0     MSVCRT:initializers.obj
 0002:000004e0       ??_C@_0CJ@PGKOGMIO@Unsupported?5mode?5for?5glyph?5imag@ 000000018008b4e0     ColorGlyphSurfaceData.obj
 0002:00000510       ??_C@_0CP@FKLHLEEM@Initialization?5of?5ColorGlyphSur@ 000000018008b510     ColorGlyphSurfaceData.obj
 0002:00000540       __real@3eaaaaaa            000000018008b540     DrawGlyphList.obj
 0002:00000548       __real@3ff0000000000000    000000018008b548     DrawGlyphList.obj
 0002:00000550       __real@40400000            000000018008b550     DrawGlyphList.obj
 0002:00000558       __real@4059000000000000    000000018008b558     DrawGlyphList.obj
 0002:00000560       __real@406fe00000000000    000000018008b560     DrawGlyphList.obj
 0002:00000568       __real@beaaaaaa            000000018008b568     DrawGlyphList.obj
 0002:00000570       ??_C@_0BM@DODCGPJL@sun?1font?1GlyphLayout$GVData@ 000000018008b570     HBShaper.obj
 0002:0000058c       ??_C@_01JPJNBJEM@I@        000000018008b58c     HBShaper.obj
 0002:00000590       ??_C@_06HHPHCOMB@_count@   000000018008b590     HBShaper.obj
 0002:00000598       ??_C@_06PPHBKICC@_flags@   000000018008b598     HBShaper.obj
 0002:000005a0       ??_C@_02EBOMBDPA@?$FLI@    000000018008b5a0     HBShaper.obj
 0002:000005a8       ??_C@_07PKNHOODJ@_glyphs@  000000018008b5a8     HBShaper.obj
 0002:000005b0       ??_C@_02MGHEAPDP@?$FLF@    000000018008b5b0     HBShaper.obj
 0002:000005b8       ??_C@_0L@BHNDECPI@_positions@ 000000018008b5b8     HBShaper.obj
 0002:000005c8       ??_C@_08MEOKMKLN@_indices@ 000000018008b5c8     HBShaper.obj
 0002:000005d4       ??_C@_03GAEACAIP@?$CI?$CJV@ 000000018008b5d4     HBShaper.obj
 0002:000005d8       ??_C@_04PAAMKIIE@grow@     000000018008b5d8     HBShaper.obj
 0002:000005dd       ??_C@_00CNPNBAHC@@         000000018008b5dd     HBShaper.obj
 0002:000005e0       ??_C@_0L@LCGIKEMB@HB_NODEVTX@ 000000018008b5e0     HBShaper.obj
 0002:000005ec       ??_C@_04HHMMLDJI@kern@     000000018008b5ec     HBShaper.obj
 0002:000005f4       ??_C@_05LLBOPDMO@?9kern@   000000018008b5f4     HBShaper.obj
 0002:000005fc       ??_C@_04BCEPKNGE@liga@     000000018008b5fc     HBShaper.obj
 0002:00000604       ??_C@_05NOJNONDC@?9liga@   000000018008b604     HBShaper.obj
 0002:0000060c       __real@37800000            000000018008b60c     HBShaper.obj
 0002:00000610       __real@3f000000            000000018008b610     HBShaper.obj
 0002:00000614       __real@3f800000            000000018008b614     HBShaper.obj
 0002:00000620       __xmm@80000000800000008000000080000000 000000018008b620     HBShaper.obj
 0002:00000698       ??_C@_11LOCGONAA@@         000000018008b698     fontpath.obj
 0002:000006a0       ??_C@_07GCCENIMJ@?2System@ 000000018008b6a0     fontpath.obj
 0002:000006a8       ??_C@_09FJGNFLHN@?2System32@ 000000018008b6a8     fontpath.obj
 0002:000006b4       ??_C@_06MIJGMACG@?2Fonts@  000000018008b6b4     fontpath.obj
 0002:000006bc       ??_C@_01ICJEACDI@?$DL@     000000018008b6bc     fontpath.obj
 0002:000006c0       ??_C@_17BCGMALNF@?$AA?5?$AA?$CG?$AA?5@ 000000018008b6c0     fontpath.obj
 0002:000006c8       ??_C@_19OLAFNMII@?$AA?4?$AAt?$AAt?$AAf@ 000000018008b6c8     fontpath.obj
 0002:000006d8       ??_C@_19MKNEPBPF@?$AA?4?$AAo?$AAt?$AAf@ 000000018008b6d8     fontpath.obj
 0002:000006e8       ??_C@_0BC@LEKPNIDO@java?1util?1HashMap@ 000000018008b6e8     fontpath.obj
 0002:00000700       ??_C@_0DJ@FLFJBGBN@?$CILjava?1lang?1Object?$DLLjava?1lang?1O@ 000000018008b700     fontpath.obj
 0002:0000073c       ??_C@_03KMONJGDG@put@      000000018008b73c     fontpath.obj
 0002:00000740       ??_C@_0BG@DHOOFEJE@?$CILjava?1lang?1Object?$DL?$CJZ@ 000000018008b740     fontpath.obj
 0002:00000758       ??_C@_0M@ILMAKOC@containsKey@ 000000018008b758     fontpath.obj
 0002:00000768       ??_C@_0BE@GPOIDJOH@java?1util?1ArrayList@ 000000018008b768     fontpath.obj
 0002:0000077c       ??_C@_04PFANPMCN@?$CII?$CJV@ 000000018008b77c     fontpath.obj
 0002:00000784       ??_C@_06FALKBLGB@?$DMinit?$DO@ 000000018008b784     fontpath.obj
 0002:0000078c       ??_C@_03BDGOHNNK@add@      000000018008b78c     fontpath.obj
 0002:00000790       ??_C@_0BB@FLFAIHG@java?1lang?1String@ 000000018008b790     fontpath.obj
 0002:000007a8       ??_C@_0CH@BHMNPKMP@?$CILjava?1util?1Locale?$DL?$CJLjava?1lang?1@ 000000018008b7a8     fontpath.obj
 0002:000007d0       ??_C@_0M@IMBDOEKL@toLowerCase@ 000000018008b7d0     fontpath.obj
 0002:00000808       ??_C@_0BB@NIMAMPFF@invalidateScaler@ 000000018008b808     freetypeScaler.obj
 0002:0000081c       ??_C@_03MMPFGPID@?$CI?$CJZ@ 000000018008b81c     freetypeScaler.obj
 0002:00000820       ??_C@_0L@NFPPEDEE@debugFonts@ 000000018008b820     freetypeScaler.obj
 0002:00000830       ??_C@_0BH@MINLIFDD@sun?1font?1FontUtilities@ 000000018008b830     freetypeScaler.obj
 0002:00000848       ??_C@_0BE@LLDKDDBI@FREETYPE_PROPERTIES@ 000000018008b848     freetypeScaler.obj
 0002:00000860       ??_C@_08OKLLNAKL@truetype@ 000000018008b860     freetypeScaler.obj
 0002:00000870       ??_C@_0BE@OJJAFABD@interpreter?9version@ 000000018008b870     freetypeScaler.obj
 0002:00000884       __real@3c800000            000000018008b884     freetypeScaler.obj
 0002:00000888       __real@3ef0000000000000    000000018008b888     freetypeScaler.obj
 0002:00000890       __real@3f90000000000000    000000018008b890     freetypeScaler.obj
 0002:00000898       __real@4050000000000000    000000018008b898     freetypeScaler.obj
 0002:000008a0       __real@42800000            000000018008b8a0     freetypeScaler.obj
 0002:000008a4       __real@47800000            000000018008b8a4     freetypeScaler.obj
 0002:000008a8       __real@c7800000            000000018008b8a8     freetypeScaler.obj
 0002:000008b0       __xmm@00010000000000000000366a00010000 000000018008b8b0     freetypeScaler.obj
 0002:000008c0       __xmm@80000000000000008000000000000000 000000018008b8c0     freetypeScaler.obj
 0002:00000dd0       ??_C@_08EMNHGPIL@SANITIZE@ 000000018008bdd0     hb-aat-layout.obj
 0002:00000de0       ??_C@_0BL@LJCAAAA@start?5?$FL?$CFp?4?4?$CFp?$FN?5?$CI?$CFlu?5bytes?$CJ@ 000000018008bde0     hb-aat-layout.obj
 0002:00000e00       ??_C@_0BO@NFKLCDNJ@end?5?$FL?$CFp?4?4?$CFp?$FN?5?$CFu?5edit?5requests@ 000000018008be00     hb-aat-layout.obj
 0002:00000e20       ??_C@_02GIPFHKNO@OK@       000000018008be20     hb-aat-layout.obj
 0002:00000e28       ??_C@_0N@FLBMHONH@OUT?9OF?9RANGE@ 000000018008be28     hb-aat-layout.obj
 0002:00000e38       ??_C@_0DC@DHOCDOGD@check_range?5?$FL?$CFp?4?4?$CFp?$FN?5?$CI?$CFu?5bytes?$CJ@ 000000018008be38     hb-aat-layout.obj
 0002:00000e70       ??_C@_07IICDHBMC@GRANTED@  000000018008be70     hb-aat-layout.obj
 0002:00000e78       ??_C@_06GONJNOIB@DENIED@   000000018008be78     hb-aat-layout.obj
 0002:00000e80       ??_C@_0DD@ENACFAKI@may_edit?$CI?$CFu?$CJ?5?$FL?$CFp?4?4?$CFp?$FN?5?$CI?$CFu?5bytes@ 000000018008be80     hb-aat-layout.obj
 0002:00000eb8       ??_C@_0BB@HBIIGPNG@start?5table?5morx@ 000000018008beb8     hb-aat-layout.obj
 0002:00000ed0       ??_C@_0P@CBPBJJBN@end?5table?5morx@ 000000018008bed0     hb-aat-layout.obj
 0002:00000ee0       ??_C@_0BB@NNDNCANK@start?5table?5mort@ 000000018008bee0     hb-aat-layout.obj
 0002:00000ef8       ??_C@_0P@INEENGBB@end?5table?5mort@ 000000018008bef8     hb-aat-layout.obj
 0002:00000f08       ??_C@_0BB@JBHFHKBC@start?5table?5kerx@ 000000018008bf08     hb-aat-layout.obj
 0002:00000f20       ??_C@_0P@MBAMIMNJ@end?5table?5kerx@ 000000018008bf20     hb-aat-layout.obj
 0002:00000f30       ??_C@_0BC@JDHEBHPG@start?5subtable?5?$CFu@ 000000018008bf30     hb-aat-layout.obj
 0002:00000f48       ??_C@_0BA@JPJCHFDI@end?5subtable?5?$CFu@ 000000018008bf48     hb-aat-layout.obj
 0002:00000f58       ??_C@_0BH@HOIFGKFM@start?5chainsubtable?5?$CFu@ 000000018008bf58     hb-aat-layout.obj
 0002:00000f70       ??_C@_0BF@LIFFOAHA@end?5chainsubtable?5?$CFu@ 000000018008bf70     hb-aat-layout.obj
 0002:00000f88       ??_C@_0L@PIONBGHN@start?5kern@ 000000018008bf88     hb-aat-layout.obj
 0002:00000f98       ??_C@_08PMCHELIJ@end?5kern@ 000000018008bf98     hb-aat-layout.obj
 0002:00000fa8       __real@3fe999999999999a    000000018008bfa8     hb-aat-layout.obj
 0002:00000fb8       ??_C@_04HDKFADDE@BLOB@     000000018008bfb8     hb-blob.obj
 0002:00000fc0       ??_C@_0BH@NNGJHJOL@current?5data?5is?5?9?$DO?5?$CFp?6@ 000000018008bfc0     hb-blob.obj
 0002:00000fd8       ??_C@_0DA@EJAJOMDI@bool?5__cdecl?5hb_blob_t?3?3try_mak@ 000000018008bfd8     hb-blob.obj
 0002:00001008       ??_C@_0BL@NAAIMIGO@dupped?5successfully?5?9?$DO?5?$CFp?6@ 000000018008c008     hb-blob.obj
 0002:00001024       ??_C@_04CIMGMMMG@text@     000000018008c024     hb-buffer-serialize.obj
 0002:0000102c       ??_C@_04CLCAKCEI@json@     000000018008c02c     hb-buffer-serialize.obj
 0002:00002ac4       ??_C@_02GMHACPFF@?$CFu@    000000018008dac4     hb-buffer-serialize.obj
 0002:00002ac8       ??_C@_08ELFBALIN@?0?$CCcl?$CC?3?$CFu@ 000000018008dac8     hb-buffer-serialize.obj
 0002:00002ad4       ??_C@_04MAFNGINP@?$CCu?$CC?3@ 000000018008dad4     hb-buffer-serialize.obj
 0002:00002adc       ??_C@_03LADEAJCH@?$DN?$CFu@ 000000018008dadc     hb-buffer-serialize.obj
 0002:00002ae0       ??_C@_06NGBPNBKB@U?$CL?$CF04X@ 000000018008dae0     hb-buffer-serialize.obj
 0002:00002ae8       ??_C@_09CPCAOBOK@harfbuzz?5@ 000000018008dae8     hb-buffer-verify.obj
 0002:00002af4       ??_C@_01EEMJAFIK@?6@       000000018008daf4     hb-buffer-verify.obj
 0002:00002af8       ??_C@_0DA@OHKIDNHD@buffer?5verify?5error?3?5clusters?5a@ 000000018008daf8     hb-buffer-verify.obj
 0002:00002b28       ??_C@_0DM@MPDBGHGJ@buffer?5verify?5error?3?5shaping?5fa@ 000000018008db28     hb-buffer-verify.obj
 0002:00002b68       ??_C@_0DC@KJMJOHEC@buffer?5verify?5error?3?5unsafe?9to?9@ 000000018008db68     hb-buffer-verify.obj
 0002:00002ba0       ??_C@_0DD@CKNGEJOG@buffer?5verify?5error?3?5unsafe?9to?9@ 000000018008dba0     hb-buffer-verify.obj
 0002:00002bd8       ??_C@_0CD@DIKIFAKO@buffer?5verify?5error?3?5text?5was?3?5@ 000000018008dbd8     hb-buffer-verify.obj
 0002:00002c10       ?minus_1@@3IB              000000018008dc10     hb-common.obj
 0002:00002c14       ?_hb_Null_OT_Index@@3QBEB  000000018008dc14     hb-common.obj
 0002:00002c28       ?_hb_Null_AAT_Lookup@@3QBEB 000000018008dc28     hb-common.obj
 0002:00002d30       ?_hb_Null_OT_LangSys@@3QBEB 000000018008dd30     hb-common.obj
 0002:00002d38       ?_hb_Null_OT_RangeRecord@@3QBEB 000000018008dd38     hb-common.obj
 0002:00003880       ?_hb_NullPool@@3QB_KB      000000018008e880     hb-common.obj
 0002:00003a40       ?_hb_Null_OT_VarIdx@@3QBEB 000000018008ea40     hb-common.obj
 0002:0000423c       ?_hb_Null_OT_ClipRecord@@3QBEB 000000018008f23c     hb-common.obj
 0002:00004244       ?_hb_Null_AAT_SettingName@@3QBEB 000000018008f244     hb-common.obj
 0002:000049c0       ?_hb_Null_OT_CmapSubtableLongGroup@@3QBEB 000000018008f9c0     hb-common.obj
 0002:000049d0       ??_C@_0L@PGCGEAJK@HB_OPTIONS@ 000000018008f9d0     hb-common.obj
 0002:000049e0       ??_C@_0BJ@EELCEACD@uniscribe?9bug?9compatible@ 000000018008f9e0     hb-common.obj
 0002:000049fc       __real@38800000            000000018008f9fc     hb-common.obj
 0002:00004a00       __real@4f000000            000000018008fa00     hb-common.obj
 0002:00004a10       __xmm@ff7fffffff7fffff7f7fffff7f7fffff 000000018008fa10     hb-common.obj
 0002:00004a20       __real@3eaaaaab            000000018008fa20     hb-draw.obj
 0002:00004a38       ??_C@_0L@LHCHIOPJ@successful@ 000000018008fa38     hb-face-builder.obj
 0002:00004a48       ??_C@_0N@KIEOCLDL@UNSUCCESSFUL@ 000000018008fa48     hb-face-builder.obj
 0002:00004a58       ??_C@_0CF@PIDDOBFK@end?5?$FL?$CFp?4?4?$CFp?$FN?5serialized?5?$CFu?5byte@ 000000018008fa58     hb-face-builder.obj
 0002:00004a80       ??_C@_09EPPNEDIL@SERIALIZE@ 000000018008fa80     hb-face-builder.obj
 0002:00005a10       __real@40000000            0000000180090a10     hb-font.obj
 0002:00005a20       __xmm@7fffffff7fffffff7fffffff7fffffff 0000000180090a20     hb-font.obj
 0002:00005ba8       __real@0010000000000000    0000000180090ba8     hb-number.obj
 0002:00005bb0       __real@4024000000000000    0000000180090bb0     hb-number.obj
 0002:00005bb8       __real@42f9999999999990    0000000180090bb8     hb-number.obj
 0002:00005bc0       __real@7fefffffffffffff    0000000180090bc0     hb-number.obj
 0002:00005bc8       __real@8010000000000000    0000000180090bc8     hb-number.obj
 0002:00005bd0       __real@bff0000000000000    0000000180090bd0     hb-number.obj
 0002:00005bd8       __real@ffefffffffffffff    0000000180090bd8     hb-number.obj
 0002:000078b0       __xmm@41dfffffffc0000041dfffffffc00000 00000001800928b0     hb-ot-cff1-table.obj
 0002:000078c0       __xmm@7fffffffffffffff7fffffffffffffff 00000001800928c0     hb-ot-cff1-table.obj
 0002:000078d0       __xmm@c1e0000000000000c1e0000000000000 00000001800928d0     hb-ot-cff1-table.obj
 0002:0000d5b0       ??_C@_0BB@HNNCONOI@0123456789?4EE?$DP?9?$DP@ 00000001800985b0     hb-ot-font.obj
 0002:0000d5c4       __real@40490fdb            00000001800985c4     hb-ot-font.obj
 0002:0000d5d0       __xmm@3f0000003f0000003f0000003f000000 00000001800985d0     hb-ot-font.obj
 0002:0000d5e0       __xmm@3f80000000000000000000003f800000 00000001800985e0     hb-ot-font.obj
 0002:0000d5f0       __xmm@bf800000bf8000000000000000000000 00000001800985f0     hb-ot-font.obj
 0002:0000de00       ??_C@_0BN@IMAOBAG@recursing?5to?5lookup?5?$CFu?5at?5?$CFu@ 0000000180098e00     hb-ot-layout.obj
 0002:0000de20       ??_C@_0BG@HECNAHM@recursed?5to?5lookup?5?$CFu@ 0000000180098e20     hb-ot-layout.obj
 0002:0000de38       ??_C@_0BI@LEONKCCB@positioning?5glyph?5at?5?$CFu@ 0000000180098e38     hb-ot-layout.obj
 0002:0000de50       ??_C@_0BH@NHBAIFPO@positioned?5glyph?5at?5?$CFu@ 0000000180098e50     hb-ot-layout.obj
 0002:0000de68       ??_C@_0CN@LEDGNLBP@cursive?5attaching?5glyph?5at?5?$CFu?5t@ 0000000180098e68     hb-ot-layout.obj
 0002:0000de98       ??_C@_0CM@NPOIGCBF@cursive?5attached?5glyph?5at?5?$CFu?5to@ 0000000180098e98     hb-ot-layout.obj
 0002:0000dec8       ??_C@_0CK@HCENOEA@attaching?5mark?5glyph?5at?5?$CFu?5to?5g@ 0000000180098ec8     hb-ot-layout.obj
 0002:0000def8       ??_C@_0CJ@IBLNDIDG@attached?5mark?5glyph?5at?5?$CFu?5to?5gl@ 0000000180098ef8     hb-ot-layout.obj
 0002:0000df28       ??_C@_0DG@CFBMBHJC@replacing?5glyph?5at?5?$CFu?5?$CIreverse?5@ 0000000180098f28     hb-ot-layout.obj
 0002:0000df60       ??_C@_0DF@HANPKIIM@replaced?5glyph?5at?5?$CFu?5?$CIreverse?5c@ 0000000180098f60     hb-ot-layout.obj
 0002:0000df98       ??_C@_0BB@INONMPMF@start?5table?5kern@ 0000000180098f98     hb-ot-layout.obj
 0002:0000dfb0       ??_C@_0P@NNJEDJAO@end?5table?5kern@ 0000000180098fb0     hb-ot-layout.obj
 0002:0000dfc0       ??_C@_0BB@FIKPJBHG@start?5table?5GSUB@ 0000000180098fc0     hb-ot-layout.obj
 0002:0000dfd8       ??_C@_0P@INGGHLN@end?5table?5GSUB@ 0000000180098fd8     hb-ot-layout.obj
 0002:0000dfe8       ??_C@_0BB@IHCDLCO@start?5table?5GPOS@ 0000000180098fe8     hb-ot-layout.obj
 0002:0000e000       ??_C@_0P@FIALMNOF@end?5table?5GPOS@ 0000000180099000     hb-ot-layout.obj
 0002:0000e010       ??_C@_0CD@BOMDBIAK@start?5lookup?5?$CFu?5feature?5?8?$CFc?$CFc?$CFc@ 0000000180099010     hb-ot-layout.obj
 0002:0000e038       ??_C@_0DO@IEOLAPEI@skipped?5lookup?5?$CFu?5feature?5?8?$CFc?$CFc@ 0000000180099038     hb-ot-layout.obj
 0002:0000e078       ??_C@_0CB@CHKBGOD@end?5lookup?5?$CFu?5feature?5?8?$CFc?$CFc?$CFc?$CFc@ 0000000180099078     hb-ot-layout.obj
 0002:0000e0a0       ??_C@_0CM@MBFHEMDL@replacing?5glyph?5at?5?$CFu?5?$CIsingle?5s@ 00000001800990a0     hb-ot-layout.obj
 0002:0000e0d0       ??_C@_0CL@HNJEFGAB@replaced?5glyph?5at?5?$CFu?5?$CIsingle?5su@ 00000001800990d0     hb-ot-layout.obj
 0002:0000e100       ??_C@_0BM@ILJLMNPF@try?5kerning?5glyphs?5at?5?$CFu?0?$CFu@ 0000000180099100     hb-ot-layout.obj
 0002:0000e120       ??_C@_0BH@OPPMFNJB@kerned?5glyphs?5at?5?$CFu?0?$CFu@ 0000000180099120     hb-ot-layout.obj
 0002:0000e138       ??_C@_0BO@DMMODMBI@tried?5kerning?5glyphs?5at?5?$CFu?0?$CFu@ 0000000180099138     hb-ot-layout.obj
 0002:0000e158       ??_C@_0CP@EIOKABLL@replacing?5glyph?5at?5?$CFu?5?$CIalternat@ 0000000180099158     hb-ot-layout.obj
 0002:0000e188       ??_C@_0CO@NDFGAIJA@replaced?5glyph?5at?5?$CFu?5?$CIalternate@ 0000000180099188     hb-ot-layout.obj
 0002:0000e1b8       ??_C@_0CO@BKNPNBH@replacing?5glyph?5at?5?$CFu?5?$CImultiple@ 00000001800991b8     hb-ot-layout.obj
 0002:0000e1e8       ??_C@_0CM@MEKJGOCL@replaced?5glyph?5at?5?$CFu?5?$CImultiple?5@ 00000001800991e8     hb-ot-layout.obj
 0002:0000e218       ??_C@_0CN@NDMMJMPC@deleting?5glyph?5at?5?$CFu?5?$CImultiple?5@ 0000000180099218     hb-ot-layout.obj
 0002:0000e248       ??_C@_0CM@LFICHOPB@deleted?5glyph?5at?5?$CFu?5?$CImultiple?5s@ 0000000180099248     hb-ot-layout.obj
 0002:0000e278       ??_C@_0BI@MNHOPBOM@multiplying?5glyph?5at?5?$CFu@ 0000000180099278     hb-ot-layout.obj
 0002:0000e290       ??_C@_0BI@MMDNIBFC@multiplied?5glyphs?5at?5?$CFs@ 0000000180099290     hb-ot-layout.obj
 0002:0000e2a8       ??_C@_0CO@NFINLDBE@replacing?5glyph?5at?5?$CFu?5?$CIligature@ 00000001800992a8     hb-ot-layout.obj
 0002:0000e2d8       ??_C@_0CN@NEGCINE@replaced?5glyph?5at?5?$CFu?5?$CIligature?5@ 00000001800992d8     hb-ot-layout.obj
 0002:0000e308       ??_C@_0BG@PELKDOGC@ligating?5glyphs?5at?5?$CFs@ 0000000180099308     hb-ot-layout.obj
 0002:0000e320       ??_C@_0BE@CENOONDG@ligated?5glyph?5at?5?$CFu@ 0000000180099320     hb-ot-layout.obj
 0002:0000e340       __xmm@ffffffffffffffffffffffffffffffff 0000000180099340     hb-ot-layout.obj
 0002:0000f6d0       ??_C@_0BE@JHLPALHA@start?5fallback?5mark@ 000000018009a6d0     hb-ot-shape-fallback.obj
 0002:0000f6e8       ??_C@_0BC@GBHKPNCC@end?5fallback?5mark@ 000000018009a6e8     hb-ot-shape-fallback.obj
 0002:0000f700       ??_C@_0BE@OKOKJNMC@start?5fallback?5kern@ 000000018009a700     hb-ot-shape-fallback.obj
 0002:0000f718       ??_C@_0BC@BMCPGLJA@end?5fallback?5kern@ 000000018009a718     hb-ot-shape-fallback.obj
 0002:0000f738       ??_C@_0O@PHODME@start?5reorder@ 000000018009a738     hb-ot-shape-normalize.obj
 0002:0000f748       ??_C@_0M@MGJODAHL@end?5reorder@ 000000018009a748     hb-ot-shape-normalize.obj
 0002:0000f7d0       ??_C@_0BJ@JCPBKLAK@start?5postprocess?9glyphs@ 000000018009a7d0     hb-ot-shape.obj
 0002:0000f7f0       ??_C@_0BH@KGKNGMEK@end?5postprocess?9glyphs@ 000000018009a7f0     hb-ot-shape.obj
 0002:0000f808       ??_C@_0BG@KEPPLGKM@start?5preprocess?9text@ 000000018009a808     hb-ot-shape.obj
 0002:0000f820       ??_C@_0BE@HIKMCIJG@end?5preprocess?9text@ 000000018009a820     hb-ot-shape.obj
 0002:0000f834       ??_C@_02IGGBGAC@ot@        000000018009a834     hb-ot-shape.obj
 0002:0000f840       __xmm@00000007000000070000000700000007 000000018009a840     hb-ot-shape.obj
 0002:0000fa10       ?_hb_ot_shaper_arabic@@3Uhb_ot_shaper_t@@B 000000018009aa10     hb-ot-shaper-arabic.obj
 0002:00010ad0       ??_C@_09BJHPDKCP@measuring@ 000000018009bad0     hb-ot-shaper-arabic.obj
 0002:00010ae0       ??_C@_07MINDNCFJ@cutting@  000000018009bae0     hb-ot-shaper-arabic.obj
 0002:00010ae8       ??_C@_0BJ@CMFJBMOA@?$CFs?5stretch?5at?5?$CI?$CFu?0?$CFu?0?$CFu?$CJ@ 000000018009bae8     hb-ot-shaper-arabic.obj
 0002:00010b04       ??_C@_06DBDILMHG@ARABIC@   000000018009bb04     hb-ot-shaper-arabic.obj
 0002:00010b20       ?_hb_ot_shaper_default@@3Uhb_ot_shaper_t@@B 000000018009bb20     hb-ot-shaper-default.obj
 0002:00010b80       ?_hb_ot_shaper_dumber@@3Uhb_ot_shaper_t@@B 000000018009bb80     hb-ot-shaper-default.obj
 0002:00010bf0       ?_hb_ot_shaper_hangul@@3Uhb_ot_shaper_t@@B 000000018009bbf0     hb-ot-shaper-hangul.obj
 0002:00010c70       ?_hb_ot_shaper_hebrew@@3Uhb_ot_shaper_t@@B 000000018009bc70     hb-ot-shaper-hebrew.obj
 0002:00013700       ?_hb_ot_shaper_indic@@3Uhb_ot_shaper_t@@B 000000018009e700     hb-ot-shaper-indic.obj
 0002:000144c8       ??_C@_0BP@PFJNIBAL@start?5reordering?5indic?5initial@ 000000018009f4c8     hb-ot-shaper-indic.obj
 0002:000144e8       ??_C@_0BN@DEJECPK@end?5reordering?5indic?5initial@ 000000018009f4e8     hb-ot-shaper-indic.obj
 0002:00014508       ??_C@_0BN@BEFMFOMM@start?5reordering?5indic?5final@ 000000018009f508     hb-ot-shaper-indic.obj
 0002:00014528       ??_C@_0BL@CMBCGANJ@end?5reordering?5indic?5final@ 000000018009f528     hb-ot-shaper-indic.obj
 0002:00014560       ?_hb_ot_shaper_khmer@@3Uhb_ot_shaper_t@@B 000000018009f560     hb-ot-shaper-khmer.obj
 0002:00014be8       ??_C@_0BH@LEEFGPFH@start?5reordering?5khmer@ 000000018009fbe8     hb-ot-shaper-khmer.obj
 0002:00014c00       ??_C@_0BF@HCJFOFHL@end?5reordering?5khmer@ 000000018009fc00     hb-ot-shaper-khmer.obj
 0002:00014c30       ?_hb_ot_shaper_myanmar@@3Uhb_ot_shaper_t@@B 000000018009fc30     hb-ot-shaper-myanmar.obj
 0002:00014c90       ?_hb_ot_shaper_myanmar_zawgyi@@3Uhb_ot_shaper_t@@B 000000018009fc90     hb-ot-shaper-myanmar.obj
 0002:00015760       ??_C@_0BJ@HDEFJBCC@start?5reordering?5myanmar@ 00000001800a0760     hb-ot-shaper-myanmar.obj
 0002:00015780       ??_C@_0BH@EHBJFGGC@end?5reordering?5myanmar@ 00000001800a0780     hb-ot-shaper-myanmar.obj
 0002:000157b0       ?_hb_ot_shaper_thai@@3Uhb_ot_shaper_t@@B 00000001800a07b0     hb-ot-shaper-thai.obj
 0002:00016c50       ?_hb_ot_shaper_use@@3Uhb_ot_shaper_t@@B 00000001800a1c50     hb-ot-shaper-use.obj
 0002:000183e0       ??_C@_0BF@INKMBGAO@start?5reordering?5USE@ 00000001800a33e0     hb-ot-shaper-use.obj
 0002:000183f8       ??_C@_0BD@IDPODCA@end?5reordering?5USE@ 00000001800a33f8     hb-ot-shaper-use.obj
 0002:0001b048       ??_C@_08LOEDBOED@?9fonnapa@ 00000001800a6048     hb-ot-tag.obj
 0002:0001b058       ??_C@_08GMLKJDFJ@?9polyton@ 00000001800a6058     hb-ot-tag.obj
 0002:0001b068       ??_C@_08NJCBHCMA@?9arevmda@ 00000001800a6068     hb-ot-tag.obj
 0002:0001b078       ??_C@_08DCLOKPKI@?9provenc@ 00000001800a6078     hb-ot-tag.obj
 0002:0001b088       ??_C@_07KBFBNAFC@?9fonipa@ 00000001800a6088     hb-ot-tag.obj
 0002:0001b090       ??_C@_05BHGHNKKJ@?9geok@   00000001800a6090     hb-ot-tag.obj
 0002:0001b098       ??_C@_05BCLFBOGB@?9syre@   00000001800a6098     hb-ot-tag.obj
 0002:0001b0a0       ??_C@_05JFCNACKO@?9syrj@   00000001800a60a0     hb-ot-tag.obj
 0002:0001b0a8       ??_C@_05PBEBMHKK@?9syrn@   00000001800a60a8     hb-ot-tag.obj
 0002:0001b0b0       ??_C@_09GEIHALDG@rt?9lojban@ 00000001800a60b0     hb-ot-tag.obj
 0002:0001b0c0       ??_C@_0L@KFNBBKMN@do?9hant?9hk@ 00000001800a60c0     hb-ot-tag.obj
 0002:0001b0d0       ??_C@_0L@MHHGBNCC@do?9hant?9mo@ 00000001800a60d0     hb-ot-tag.obj
 0002:0001b0e0       ??_C@_0L@NNBHMAGE@jy?9hant?9hk@ 00000001800a60e0     hb-ot-tag.obj
 0002:0001b0f0       ??_C@_0L@LPLAMHIL@jy?9hant?9mo@ 00000001800a60f0     hb-ot-tag.obj
 0002:0001b100       ??_C@_0L@DBFOEPHG@mn?9hant?9hk@ 00000001800a6100     hb-ot-tag.obj
 0002:0001b110       ??_C@_0L@FDPJEIJJ@mn?9hant?9mo@ 00000001800a6110     hb-ot-tag.obj
 0002:0001b120       ??_C@_0L@JBNLJICM@np?9hant?9hk@ 00000001800a6120     hb-ot-tag.obj
 0002:0001b130       ??_C@_0L@PDHMJPMD@np?9hant?9mo@ 00000001800a6130     hb-ot-tag.obj
 0002:0001b140       ??_C@_0L@HOIMDHBF@px?9hant?9hk@ 00000001800a6140     hb-ot-tag.obj
 0002:0001b150       ??_C@_0L@BMCLDAPK@px?9hant?9mo@ 00000001800a6150     hb-ot-tag.obj
 0002:0001b160       ??_C@_0L@PELJBBOA@sp?9hant?9hk@ 00000001800a6160     hb-ot-tag.obj
 0002:0001b170       ??_C@_0L@JGBOBGAP@sp?9hant?9mo@ 00000001800a6170     hb-ot-tag.obj
 0002:0001b180       ??_C@_0L@LLINOOHJ@zh?9hant?9hk@ 00000001800a6180     hb-ot-tag.obj
 0002:0001b190       ??_C@_0L@NJCKOJJG@zh?9hant?9mo@ 00000001800a6190     hb-ot-tag.obj
 0002:0001b1a0       ??_C@_0L@FJFBPFAA@zo?9hant?9hk@ 00000001800a61a0     hb-ot-tag.obj
 0002:0001b1b0       ??_C@_0L@DLPGPCOP@zo?9hant?9mo@ 00000001800a61b0     hb-ot-tag.obj
 0002:0001b1c0       ??_C@_07GEDDMEMG@do?9hans@ 00000001800a61c0     hb-ot-tag.obj
 0002:0001b1c8       ??_C@_07CLHCFCAB@do?9hant@ 00000001800a61c8     hb-ot-tag.obj
 0002:0001b1d0       ??_C@_07HFLHHPAA@jy?9hans@ 00000001800a61d0     hb-ot-tag.obj
 0002:0001b1d8       ??_C@_07DKPGOJMH@jy?9hant@ 00000001800a61d8     hb-ot-tag.obj
 0002:0001b1e0       ??_C@_07NNALNEFJ@mn?9hans@ 00000001800a61e0     hb-ot-tag.obj
 0002:0001b1e8       ??_C@_07JCEKECJO@mn?9hant@ 00000001800a61e8     hb-ot-tag.obj
 0002:0001b1f0       ??_C@_07GEGFDECJ@np?9hans@ 00000001800a61f0     hb-ot-tag.obj
 0002:0001b1f8       ??_C@_07CLCEKCOO@np?9hant@ 00000001800a61f8     hb-ot-tag.obj
 0002:0001b200       ??_C@_07DOLLFJFH@px?9hans@ 00000001800a6200     hb-ot-tag.obj
 0002:0001b208       ??_C@_07HBPKMPJA@px?9hant@ 00000001800a6208     hb-ot-tag.obj
 0002:0001b210       ??_C@_07IDNLBAND@sp?9hans@ 00000001800a6210     hb-ot-tag.obj
 0002:0001b218       ??_C@_07MMJKIGBE@sp?9hant@ 00000001800a6218     hb-ot-tag.obj
 0002:0001b220       ??_C@_07MIKFNJFB@zh?9hans@ 00000001800a6220     hb-ot-tag.obj
 0002:0001b228       ??_C@_07IHOEEPJG@zh?9hant@ 00000001800a6228     hb-ot-tag.obj
 0002:0001b230       ??_C@_07NACOHNP@zo?9hans@  00000001800a6230     hb-ot-tag.obj
 0002:0001b238       ??_C@_07ECEDHBBI@zo?9hant@ 00000001800a6238     hb-ot-tag.obj
 0002:0001b240       ??_C@_03JFOJGEF@do?9@      00000001800a6240     hb-ot-tag.obj
 0002:0001b244       ??_C@_03EMCOHPPE@?9hk@     00000001800a6244     hb-ot-tag.obj
 0002:0001b248       ??_C@_03COIJHIBL@?9mo@     00000001800a6248     hb-ot-tag.obj
 0002:0001b24c       ??_C@_03LPGFHILN@?9tw@     00000001800a624c     hb-ot-tag.obj
 0002:0001b250       ??_C@_03PBCKDOLE@jy?9@     00000001800a6250     hb-ot-tag.obj
 0002:0001b254       ??_C@_03HFJELDPI@mn?9@     00000001800a6254     hb-ot-tag.obj
 0002:0001b258       ??_C@_03HBJJJCGM@np?9@     00000001800a6258     hb-ot-tag.obj
 0002:0001b25c       ??_C@_03MPEMODHI@px?9@     00000001800a625c     hb-ot-tag.obj
 0002:0001b260       ??_C@_03NDOKBNCO@sp?9@     00000001800a6260     hb-ot-tag.obj
 0002:0001b264       ??_C@_03LMNHKAGM@zh?9@     00000001800a6264     hb-ot-tag.obj
 0002:0001b268       ??_C@_03LJJILGOJ@zo?9@     00000001800a6268     hb-ot-tag.obj
 0002:0001b270       ??_C@_0L@DLEENNLB@an?9hant?9hk@ 00000001800a6270     hb-ot-tag.obj
 0002:0001b280       ??_C@_0L@FJODNKFO@an?9hant?9mo@ 00000001800a6280     hb-ot-tag.obj
 0002:0001b290       ??_C@_07IKKEMBBG@an?9hans@ 00000001800a6290     hb-ot-tag.obj
 0002:0001b298       ??_C@_07MFOFFHNB@an?9hant@ 00000001800a6298     hb-ot-tag.obj
 0002:0001b2a0       ??_C@_06FCHMEGPO@a?9latg@  00000001800a62a0     hb-ot-tag.obj
 0002:0001b2a8       ??_C@_03DPECAMEA@an?9@     00000001800a62a8     hb-ot-tag.obj
 0002:0001b2b0       ??_C@_0L@NNGNBGPF@ak?9hant?9hk@ 00000001800a62b0     hb-ot-tag.obj
 0002:0001b2c0       ??_C@_0L@LPMKBBBK@ak?9hant?9mo@ 00000001800a62c0     hb-ot-tag.obj
 0002:0001b2d0       ??_C@_0L@MNNOKALL@sn?9hant?9hk@ 00000001800a62d0     hb-ot-tag.obj
 0002:0001b2e0       ??_C@_0L@KPHJKHFE@sn?9hant?9mo@ 00000001800a62e0     hb-ot-tag.obj
 0002:0001b2f0       ??_C@_07NIJMOOLB@ak?9hans@ 00000001800a62f0     hb-ot-tag.obj
 0002:0001b2f8       ??_C@_07JHNNHIHG@ak?9hant@ 00000001800a62f8     hb-ot-tag.obj
 0002:0001b300       ??_C@_07LEDKPHEA@sn?9hans@ 00000001800a6300     hb-ot-tag.obj
 0002:0001b308       ??_C@_07PLHLGBIH@sn?9hant@ 00000001800a6308     hb-ot-tag.obj
 0002:0001b310       ??_C@_03DJIJMOKL@ak?9@     00000001800a6310     hb-ot-tag.obj
 0002:0001b314       ??_C@_03MFFCJDFE@sn?9@     00000001800a6314     hb-ot-tag.obj
 0002:0001b318       ??_C@_07LCKCAAMB@?9navajo@ 00000001800a6318     hb-ot-tag.obj
 0002:0001b320       ??_C@_04DBACCPMA@?9hak@    00000001800a6320     hb-ot-tag.obj
 0002:0001b328       ??_C@_04MEKAPCKJ@?9lux@    00000001800a6328     hb-ot-tag.obj
 0002:0001b330       ??_C@_03HENGIEOJ@nw?9@     00000001800a6330     hb-ot-tag.obj
 0002:0001b334       ??_C@_03HCDPHGCD@?9th@     00000001800a6334     hb-ot-tag.obj
 0002:0001b338       ??_C@_05NKGDAJJP@o?9bok@   00000001800a6338     hb-ot-tag.obj
 0002:0001b340       ??_C@_05PFGJJNKA@o?9nyn@   00000001800a6340     hb-ot-tag.obj
 0002:0001b348       ??_C@_02GDBPPABP@o?9@      00000001800a6348     hb-ot-tag.obj
 0002:0001b34c       ??_C@_03MNHNKBNA@?9md@     00000001800a634c     hb-ot-tag.obj
 0002:0001b350       ??_C@_0L@PKCFBAOH@uu?9hant?9hk@ 00000001800a6350     hb-ot-tag.obj
 0002:0001b360       ??_C@_0L@JIICBHAI@uu?9hant?9mo@ 00000001800a6360     hb-ot-tag.obj
 0002:0001b370       ??_C@_07BHIMDGPD@uu?9hans@ 00000001800a6370     hb-ot-tag.obj
 0002:0001b378       ??_C@_07FIMNKADE@uu?9hant@ 00000001800a6378     hb-ot-tag.obj
 0002:0001b380       ??_C@_03PAEKIABJ@uu?9@     00000001800a6380     hb-ot-tag.obj
 0002:0001b388       ??_C@_07HAFCKKDN@ue?9hans@ 00000001800a6388     hb-ot-tag.obj
 0002:0001b390       ??_C@_09CPANDNJE@h?9hant?9hk@ 00000001800a6390     hb-ot-tag.obj
 0002:0001b3a0       ??_C@_09ENKKDKHL@h?9hant?9mo@ 00000001800a63a0     hb-ot-tag.obj
 0002:0001b3b0       ??_C@_09JKAGOIDE@h?9min?9nan@ 00000001800a63b0     hb-ot-tag.obj
 0002:0001b3bc       ??_C@_06NHLFEBO@h?9hans@   00000001800a63bc     hb-ot-tag.obj
 0002:0001b3c4       ??_C@_06ECDKMCNJ@h?9hant@  00000001800a63c4     hb-ot-tag.obj
 0002:0001b3cc       ??_C@_05OGPPKBIG@h?9min@   00000001800a63cc     hb-ot-tag.obj
 0002:0001b3d4       ??_C@_02GGFAOGJK@h?9@      00000001800a63d4     hb-ot-tag.obj
 0002:0001b3d8       ??_C@_03FHLPDODD@alt@      00000001800a63d8     hb-ot-tag.obj
 0002:0001b3e0       ??_C@_0M@EFNICDFC@und?9fonnapa@ 00000001800a63e0     hb-ot-tag.obj
 0002:0001b3ec       ??_C@_02FEKCJMIO@ar@       00000001800a63ec     hb-ot-tag.obj
 0002:0001b3f0       ??_C@_03OPDALMNL@rki@      00000001800a63f0     hb-ot-tag.obj
 0002:0001b3f4       ??_C@_03KDPNJBKG@ath@      00000001800a63f4     hb-ot-tag.obj
 0002:0001b3f8       ??_C@_03BMIBANNE@ber@      00000001800a63f8     hb-ot-tag.obj
 0002:0001b3fc       ??_C@_03IOJLFNKI@bik@      00000001800a63fc     hb-ot-tag.obj
 0002:0001b400       ??_C@_03JKGFGNIL@btk@      00000001800a6400     hb-ot-tag.obj
 0002:0001b404       ??_C@_03IPGCLNMG@crp@      00000001800a6404     hb-ot-tag.obj
 0002:0001b408       ??_C@_03EHLLDHMO@crx@      00000001800a6408     hb-ot-tag.obj
 0002:0001b40c       ??_C@_03JNELBMEE@doi@      00000001800a640c     hb-ot-tag.obj
 0002:0001b410       ??_C@_03NGIHPGDB@din@      00000001800a6410     hb-ot-tag.obj
 0002:0001b414       ??_C@_03OGODBGHE@prs@      00000001800a6414     hb-ot-tag.obj
 0002:0001b418       ??_C@_02JKLANEGN@dz@       00000001800a6418     hb-ot-tag.obj
 0002:0001b41c       ??_C@_02FPBJDNE@et@        00000001800a641c     hb-ot-tag.obj
 0002:0001b420       ??_C@_02DAACMLJJ@fa@       00000001800a6420     hb-ot-tag.obj
 0002:0001b424       ??_C@_03MALPCFGN@gon@      00000001800a6424     hb-ot-tag.obj
 0002:0001b428       ??_C@_03NPJADACO@mrj@      00000001800a6428     hb-ot-tag.obj
 0002:0001b42c       ??_C@_03JLFIOBFF@hmn@      00000001800a642c     hb-ot-tag.obj
 0002:0001b430       ??_C@_03GDPBLHIG@hnd@      00000001800a6430     hb-ot-tag.obj
 0002:0001b434       ??_C@_03BLHHEDOB@hyw@      00000001800a6434     hb-ot-tag.obj
 0002:0001b438       ??_C@_03KPCANNMC@iba@      00000001800a6438     hb-ot-tag.obj
 0002:0001b43c       ??_C@_03DPLAKBPE@ijo@      00000001800a643c     hb-ot-tag.obj
 0002:0001b440       ??_C@_02BFPAFLPB@iu@       00000001800a6440     hb-ot-tag.obj
 0002:0001b444       ??_C@_02MBLBGECO@ik@       00000001800a6444     hb-ot-tag.obj
 0002:0001b448       ??_C@_0L@OOCAKEAN@und?9fonipa@ 00000001800a6448     hb-ot-tag.obj
 0002:0001b458       ??_C@_07LBNNMAEP@ga?9Latg@ 00000001800a6458     hb-ot-tag.obj
 0002:0001b460       ??_C@_02OPKBKFNM@yi@       00000001800a6460     hb-ot-tag.obj
 0002:0001b464       ??_C@_03IICPCEIM@kln@      00000001800a6464     hb-ot-tag.obj
 0002:0001b468       ??_C@_08IBMBBMEF@und?9Geok@ 00000001800a6468     hb-ot-tag.obj
 0002:0001b474       ??_C@_02FJDFBJFI@kr@       00000001800a6474     hb-ot-tag.obj
 0002:0001b478       ??_C@_03CJCPPGJN@okm@      00000001800a6478     hb-ot-tag.obj
 0002:0001b47c       ??_C@_03PHBOGOJA@kok@      00000001800a647c     hb-ot-tag.obj
 0002:0001b480       ??_C@_02DNFJNMFM@kv@       00000001800a6480     hb-ot-tag.obj
 0002:0001b484       ??_C@_03HOOHKHFD@kpe@      00000001800a6484     hb-ot-tag.obj
 0002:0001b488       ??_C@_03GGIAOKIC@kar@      00000001800a6488     hb-ot-tag.obj
 0002:0001b48c       ??_C@_03HCOHIEGC@uki@      00000001800a648c     hb-ot-tag.obj
 0002:0001b490       ??_C@_02BGHEIPJP@ku@       00000001800a6490     hb-ot-tag.obj
 0002:0001b494       ??_C@_03EMDKIONB@mhr@      00000001800a6494     hb-ot-tag.obj
 0002:0001b498       ??_C@_03DIMAAFM@luy@       00000001800a6498     hb-ot-tag.obj
 0002:0001b49c       ??_C@_02DIBGMKNJ@lv@       00000001800a649c     hb-ot-tag.obj
 0002:0001b4a0       ??_C@_03FLEAGKJM@mwr@      00000001800a64a0     hb-ot-tag.obj
 0002:0001b4a4       ??_C@_02GKANIDPO@mg@       00000001800a64a4     hb-ot-tag.obj
 0002:0001b4a8       ??_C@_02EEKDFEKL@ms@       00000001800a64a8     hb-ot-tag.obj
 0002:0001b4ac       ??_C@_02LLMPDILH@mn@       00000001800a64ac     hb-ot-tag.obj
 0002:0001b4b0       ??_C@_03KFJMOIAD@man@      00000001800a64b0     hb-ot-tag.obj
 0002:0001b4b4       ??_C@_05KNLKPBHL@ro?9MD@   00000001800a64b4     hb-ot-tag.obj
 0002:0001b4bc       ??_C@_06PALDGLND@mnw?9TH@  00000001800a64bc     hb-ot-tag.obj
 0002:0001b4c4       ??_C@_03LHKJBKML@myn@      00000001800a64c4     hb-ot-tag.obj
 0002:0001b4c8       ??_C@_03OBHDOAGL@nah@      00000001800a64c8     hb-ot-tag.obj
 0002:0001b4cc       ??_C@_02FKHNFPCF@ne@       00000001800a64cc     hb-ot-tag.obj
 0002:0001b4d0       ??_C@_03JFNCHPFJ@njz@      00000001800a64d0     hb-ot-tag.obj
 0002:0001b4d4       ??_C@_02KAJCLHKP@no@       00000001800a64d4     hb-ot-tag.obj
 0002:0001b4d8       ??_C@_02NMCHCJNN@oj@       00000001800a64d8     hb-ot-tag.obj
 0002:0001b4dc       ??_C@_02JDGGLPBK@om@       00000001800a64dc     hb-ot-tag.obj
 0002:0001b4e0       ??_C@_02FAFNGEII@ps@       00000001800a64e0     hb-ot-tag.obj
 0002:0001b4e8       ??_C@_0L@LGMOIJP@el?9polyton@ 00000001800a64e8     hb-ot-tag.obj
 0002:0001b4f4       ??_C@_03JEELCJ@pro@        00000001800a64f4     hb-ot-tag.obj
 0002:0001b4f8       ??_C@_03PCCGKMAO@quh@      00000001800a64f8     hb-ot-tag.obj
 0002:0001b4fc       ??_C@_02HMFKJDJ@qu@        00000001800a64fc     hb-ot-tag.obj
 0002:0001b500       ??_C@_03OJHLCDBG@qvi@      00000001800a6500     hb-ot-tag.obj
 0002:0001b504       ??_C@_03PBKCHIGA@qwh@      00000001800a6504     hb-ot-tag.obj
 0002:0001b508       ??_C@_03MJIKGKMO@raj@      00000001800a6508     hb-ot-tag.obj
 0002:0001b50c       ??_C@_02LFKOONLL@ro@       00000001800a650c     hb-ot-tag.obj
 0002:0001b510       ??_C@_03IMFFNBAD@rom@      00000001800a6510     hb-ot-tag.obj
 0002:0001b514       ??_C@_02GACNLIFD@sq@       00000001800a6514     hb-ot-tag.obj
 0002:0001b518       ??_C@_02ELAAOLJA@sr@       00000001800a6518     hb-ot-tag.obj
 0002:0001b51c       ??_C@_03KNGLMNJH@xnj@      00000001800a651c     hb-ot-tag.obj
 0002:0001b520       ??_C@_03OBBIGHDK@syr@      00000001800a6520     hb-ot-tag.obj
 0002:0001b528       ??_C@_08IEBDNIIN@und?9Syre@ 00000001800a6528     hb-ot-tag.obj
 0002:0001b538       ??_C@_08DILMEEC@und?9Syrj@ 00000001800a6538     hb-ot-tag.obj
 0002:0001b548       ??_C@_08GHOHABEG@und?9Syrn@ 00000001800a6548     hb-ot-tag.obj
 0002:0001b554       ??_C@_03NHMNKOPE@tmh@      00000001800a6554     hb-ot-tag.obj
 0002:0001b558       ??_C@_03MDOLKBCN@xwo@      00000001800a6558     hb-ot-tag.obj
 0002:0001b55c       ??_C@_05HCJKHBCC@zh?9HK@   00000001800a655c     hb-ot-tag.obj
 0002:0001b568       ??_C@_07JGEPGFF@zh?9Hans@  00000001800a6568     hb-ot-tag.obj
 0002:0001b570       ??_C@_07EGCFGAJC@zh?9Hant@ 00000001800a6570     hb-ot-tag.obj
 0002:0001b578       ??_C@_05BADNHGMN@zh?9MO@   00000001800a6578     hb-ot-tag.obj
 0002:0001b580       ??_C@_03PPLJNHHL@zza@      00000001800a6580     hb-ot-tag.obj
 0002:0001b584       ??_C@_05NFAFKFNN@?9hbsc@   00000001800a6584     hb-ot-tag.obj
 0002:0001b58c       ??_C@_05MFLKHLFP@?9hbot@   00000001800a658c     hb-ot-tag.obj
 0002:0001b598       ??_C@_0M@MFILKOCI@x?9hbot?9?$CF08x@ 00000001800a6598     hb-ot-tag.obj
 0002:0001b5b0       __real@46800000            00000001800a65b0     hb-ot-var.obj
 0002:0001b5b4       __real@bf700000            00000001800a65b4     hb-outline.obj
 0002:0001b5c8       ??_C@_08LFBOCJLE@fallback@ 00000001800a65c8     hb-shape-plan.obj
 0002:0001b5d8       ??_C@_0DF@MPFFHONM@face?$DN?$CFp?5num_features?$DN?$CFu?5num_coo@ 00000001800a65d8     hb-shape-plan.obj
 0002:0001b610       ??_C@_0MH@MMALGGGN@struct?5hb_shape_plan_t?5?$CK__cdecl@ 00000001800a6610     hb-shape-plan.obj
 0002:0001b6d8       ??_C@_0L@HJBOBLCO@SHAPE_PLAN@ 00000001800a66d8     hb-shape-plan.obj
 0002:0001b6e8       ??_C@_0CP@GAFDBLDO@num_features?$DN?$CFu?5shaper_func?$DN?$CFp?0@ 00000001800a66e8     hb-shape-plan.obj
 0002:0001b720       ??_C@_0JI@JOJJJOPA@bool?5__cdecl?5_hb_shape_plan_exe@ 00000001800a6720     hb-shape-plan.obj
 0002:0001b7b8       ??_C@_0CH@EAKAEIJM@face?$DN?$CFp?5num_features?$DN?$CFu?5shaper_@ 00000001800a67b8     hb-shape-plan.obj
 0002:0001b7e0       ??_C@_0MO@MGHFPDJG@struct?5hb_shape_plan_t?5?$CK__cdecl@ 00000001800a67e0     hb-shape-plan.obj
 0002:0001b8f0       ??_C@_0P@GEOKODDH@HB_SHAPER_LIST@ 00000001800a68f0     hb-shaper.obj
 0002:0002f180       ?_hb_modified_combining_class@@3QBEB 00000001800ba180     hb-unicode.obj
 0002:0002f450       ??_C@_0BG@NKHBBPH@sun?1font?1TrueTypeFont@ 00000001800ba450     sunFont.obj
 0002:0002f468       ??_C@_0BL@GAAGJDLL@?$CILjava?1nio?1ByteBuffer?$DLII?$CJI@ 00000001800ba468     sunFont.obj
 0002:0002f488       ??_C@_09CKAKNPHP@readBlock@ 00000001800ba488     sunFont.obj
 0002:0002f494       ??_C@_06JMOJDKIE@?$CIII?$CJ?$FLB@ 00000001800ba494     sunFont.obj
 0002:0002f4a0       ??_C@_09IDIEPDPI@readBytes@ 00000001800ba4a0     sunFont.obj
 0002:0002f4b0       ??_C@_0BD@OPLCIPMH@sun?1font?1Type1Font@ 00000001800ba4b0     sunFont.obj
 0002:0002f4c8       ??_C@_0BJ@LMHMPPKE@?$CILjava?1nio?1ByteBuffer?$DL?$CJV@ 00000001800ba4c8     sunFont.obj
 0002:0002f4e8       ??_C@_08CJNGBMAG@readFile@ 00000001800ba4e8     sunFont.obj
 0002:0002f4f8       ??_C@_0BM@DGICEJAA@java?1awt?1geom?1Point2D$Float@ 00000001800ba4f8     sunFont.obj
 0002:0002f514       ??_C@_05BHHDPELC@?$CIFF?$CJV@ 00000001800ba514     sunFont.obj
 0002:0002f51c       ??_C@_01BIAFAFID@F@        00000001800ba51c     sunFont.obj
 0002:0002f520       ??_C@_01FJMABOPO@x@        00000001800ba520     sunFont.obj
 0002:0002f524       ??_C@_01EANLCPLP@y@        00000001800ba524     sunFont.obj
 0002:0002f528       ??_C@_0BH@ENELCGL@sun?1font?1StrikeMetrics@ 00000001800ba528     sunFont.obj
 0002:0002f540       ??_C@_0O@LBAHCNJL@?$CIFFFFFFFFFF?$CJV@ 00000001800ba540     sunFont.obj
 0002:0002f550       ??_C@_0CA@PDMBNICK@java?1awt?1geom?1Rectangle2D$Float@ 00000001800ba550     sunFont.obj
 0002:0002f570       ??_C@_07PMCFNNPC@?$CIFFFF?$CJV@ 00000001800ba570     sunFont.obj
 0002:0002f578       ??_C@_05IGKADHGO@width@    00000001800ba578     sunFont.obj
 0002:0002f580       ??_C@_06LNLHEAAG@height@   00000001800ba580     sunFont.obj
 0002:0002f588       ??_C@_0BK@COJNCHEM@java?1awt?1geom?1GeneralPath@ 00000001800ba588     sunFont.obj
 0002:0002f5a8       ??_C@_0L@MDPODKN@?$CII?$FLBI?$FLFI?$CJV@ 00000001800ba5a8     sunFont.obj
 0002:0002f5b8       ??_C@_0BA@OKNBFGCN@sun?1font?1Font2D@ 00000001800ba5b8     sunFont.obj
 0002:0002f5c8       ??_C@_04DIFHPCLD@?$CII?$CJI@ 00000001800ba5c8     sunFont.obj
 0002:0002f5d0       ??_C@_0M@NMGOHDEJ@charToGlyph@ 00000001800ba5d0     sunFont.obj
 0002:0002f5dc       ??_C@_05BKHNKL@?$CIII?$CJI@ 00000001800ba5dc     sunFont.obj
 0002:0002f5e8       ??_C@_0BF@NFJAPLLH@charToVariationGlyph@ 00000001800ba5e8     sunFont.obj
 0002:0002f600       ??_C@_0BP@CBNLOFNN@?$CI?$CJLsun?1font?1CharToGlyphMapper?$DL@ 00000001800ba600     sunFont.obj
 0002:0002f620       ??_C@_09DGCMEJKL@getMapper@ 00000001800ba620     sunFont.obj
 0002:0002f62c       ??_C@_05IPLNOPFN@?$CII?$CJ?$FLB@ 00000001800ba62c     sunFont.obj
 0002:0002f638       ??_C@_0O@DBNIPDIH@getTableBytes@ 00000001800ba638     sunFont.obj
 0002:0002f648       ??_C@_04DGAFFDEF@?$CIC?$CJZ@ 00000001800ba648     sunFont.obj
 0002:0002f650       ??_C@_0L@PGEPPKMA@canDisplay@ 00000001800ba650     sunFont.obj
 0002:0002f660       ??_C@_0BL@GAPGNAAC@sun?1font?1CharToGlyphMapper@ 00000001800ba660     sunFont.obj
 0002:0002f680       ??_C@_0BI@GDBHNKM@sun?1font?1PhysicalStrike@ 00000001800ba680     sunFont.obj
 0002:0002f698       ??_C@_0CB@IBGFEOCM@?$CII?$CJLjava?1awt?1geom?1Point2D$Float@ 00000001800ba698     sunFont.obj
 0002:0002f6c0       ??_C@_0BA@FMKHNFIF@getGlyphMetrics@ 00000001800ba6c0     sunFont.obj
 0002:0002f6d0       ??_C@_0CC@IBLMDHKA@?$CIII?$CJLjava?1awt?1geom?1Point2D$Floa@ 00000001800ba6d0     sunFont.obj
 0002:0002f6f8       ??_C@_0O@NHLNHECD@getGlyphPoint@ 00000001800ba6f8     sunFont.obj
 0002:0002f708       ??_C@_0CB@CONGGNHA@?$CILjava?1awt?1geom?1Point2D$Float?$DL?$CJ@ 00000001800ba708     sunFont.obj
 0002:0002f730       ??_C@_0M@MJABIGBP@adjustPoint@ 00000001800ba730     sunFont.obj
 0002:0002f73c       ??_C@_01LELAEKIP@J@        00000001800ba73c     sunFont.obj
 0002:0002f740       ??_C@_0P@DPIICNJB@pScalerContext@ 00000001800ba740     sunFont.obj
 0002:0002f750       ??_C@_0BD@LPHBDEDB@sun?1font?1GlyphList@ 00000001800ba750     sunFont.obj
 0002:0002f764       ??_C@_05HAAKEDND@gposx@    00000001800ba764     sunFont.obj
 0002:0002f76c       ??_C@_05GJBBHCJC@gposy@    00000001800ba76c     sunFont.obj
 0002:0002f774       ??_C@_03BKCJCHLK@len@      00000001800ba774     sunFont.obj
 0002:0002f778       ??_C@_02GKMBEADD@?$FLJ@    00000001800ba778     sunFont.obj
 0002:0002f77c       ??_C@_06IAHKIHIK@images@   00000001800ba77c     sunFont.obj
 0002:0002f784       ??_C@_01POHCFINO@Z@        00000001800ba784     sunFont.obj
 0002:0002f788       ??_C@_0N@CLHDJEN@usePositions@ 00000001800ba788     sunFont.obj
 0002:0002f798       ??_C@_09HEJILCIA@positions@ 00000001800ba798     sunFont.obj
 0002:0002f7a8       ??_C@_0M@IOGNPDID@lcdRGBOrder@ 00000001800ba7a8     sunFont.obj
 0002:0002f7b8       ??_C@_0N@OIMCCICM@lcdSubPixPos@ 00000001800ba7b8     sunFont.obj
 0002:0002f7d8       _pDefaultRawDllMain        00000001800ba7d8     MSVCRT:dll_dllmain.obj
 0002:0002f7d8       _pRawDllMain               00000001800ba7d8     MSVCRT:dll_dllmain.obj
 0002:0002f7e0       _load_config_used          00000001800ba7e0     MSVCRT:loadcfg.obj
 0002:0002fa00       __volatile_metadata        00000001800baa00     <linker-defined>
 0002:00030648       __rtc_iaa                  00000001800bb648     MSVCRT:initsect.obj
 0002:00030650       __rtc_izz                  00000001800bb650     MSVCRT:initsect.obj
 0002:00030658       __rtc_taa                  00000001800bb658     MSVCRT:initsect.obj
 0002:00030660       __rtc_tzz                  00000001800bb660     MSVCRT:initsect.obj
 0002:0003930c       __IMPORT_DESCRIPTOR_freetype 00000001800c430c     freetype:freetype.dll
 0002:00039320       __IMPORT_DESCRIPTOR_java   00000001800c4320     java:java.dll
 0002:00039334       __IMPORT_DESCRIPTOR_ADVAPI32 00000001800c4334     advapi32:ADVAPI32.dll
 0002:00039348       __IMPORT_DESCRIPTOR_USER32 00000001800c4348     user32:USER32.dll
 0002:0003935c       __IMPORT_DESCRIPTOR_GDI32  00000001800c435c     gdi32:GDI32.dll
 0002:00039370       __IMPORT_DESCRIPTOR_awt    00000001800c4370     awt:awt.dll
 0002:00039384       __IMPORT_DESCRIPTOR_KERNEL32 00000001800c4384     kernel32:KERNEL32.dll
 0002:00039398       __IMPORT_DESCRIPTOR_VCRUNTIME140 00000001800c4398     vcruntime:VCRUNTIME140.dll
 0002:000393ac       __IMPORT_DESCRIPTOR_api-ms-win-crt-heap-l1-1-0 00000001800c43ac     ucrt:api-ms-win-crt-heap-l1-1-0.dll
 0002:000393c0       __IMPORT_DESCRIPTOR_api-ms-win-crt-math-l1-1-0 00000001800c43c0     ucrt:api-ms-win-crt-math-l1-1-0.dll
 0002:000393d4       __IMPORT_DESCRIPTOR_api-ms-win-crt-environment-l1-1-0 00000001800c43d4     ucrt:api-ms-win-crt-environment-l1-1-0.dll
 0002:000393e8       __IMPORT_DESCRIPTOR_api-ms-win-crt-convert-l1-1-0 00000001800c43e8     ucrt:api-ms-win-crt-convert-l1-1-0.dll
 0002:000393fc       __IMPORT_DESCRIPTOR_api-ms-win-crt-stdio-l1-1-0 00000001800c43fc     ucrt:api-ms-win-crt-stdio-l1-1-0.dll
 0002:00039410       __IMPORT_DESCRIPTOR_api-ms-win-crt-string-l1-1-0 00000001800c4410     ucrt:api-ms-win-crt-string-l1-1-0.dll
 0002:00039424       __IMPORT_DESCRIPTOR_api-ms-win-crt-runtime-l1-1-0 00000001800c4424     ucrt:api-ms-win-crt-runtime-l1-1-0.dll
 0002:00039438       __NULL_IMPORT_DESCRIPTOR   00000001800c4438     freetype:freetype.dll
 0003:00000000       defaultGammaLUT            00000001800c6000     DrawGlyphList.obj
 0003:00000100       defaultInvGammaLUT         00000001800c6100     DrawGlyphList.obj
 0003:00000230       ?_hb_Null_hb_buffer_t@@3Uhb_buffer_t@@B 00000001800c6230     hb-buffer.obj
 0003:00000310       ?_hb_Null_hb_draw_funcs_t@@3Uhb_draw_funcs_t@@B 00000001800c6310     hb-draw.obj
 0003:00000360       ?_hb_Null_hb_face_t@@3Uhb_face_t@@B 00000001800c6360     hb-face.obj
 0003:00000500       ?_hb_Null_hb_font_funcs_t@@3Uhb_font_funcs_t@@B 00000001800c6500     hb-font.obj
 0003:000005c0       ?_hb_Null_hb_font_t@@3Uhb_font_t@@B 00000001800c65c0     hb-font.obj
 0003:000007f0       ?_hb_Null_hb_paint_funcs_t@@3Uhb_paint_funcs_t@@B 00000001800c67f0     hb-paint.obj
 0003:00000950       ?_hb_Null_hb_unicode_funcs_t@@3Uhb_unicode_funcs_t@@B 00000001800c6950     hb-unicode.obj
 0003:00000a30       MAX_ICU_SCRIPTCODE         00000001800c6a30     scriptMapping.obj
 0003:00000a40       ICU_to_Harfbuzz_ScriptCode 00000001800c6a40     scriptMapping.obj
 0003:00000b00       __security_cookie_complement 00000001800c6b00     MSVCRT:gs_cookie.obj
 0003:00000b08       __security_cookie          00000001800c6b08     MSVCRT:gs_cookie.obj
 0003:00000b10       _fltused                   00000001800c6b10     MSVCRT:fltused.obj
 0003:00000b20       __isa_available            00000001800c6b20     MSVCRT:cpu_disp.obj
 0003:00000b24       __isa_enabled              00000001800c6b24     MSVCRT:cpu_disp.obj
 0003:00000b28       __memset_fast_string_threshold 00000001800c6b28     MSVCRT:cpu_disp.obj
 0003:00000b30       __memset_nt_threshold      00000001800c6b30     MSVCRT:cpu_disp.obj
 0003:00000b40       __scrt_native_dllmain_reason 00000001800c6b40     MSVCRT:utility.obj
 0003:00000b50       __scrt_ucrt_dll_is_in_use  00000001800c6b50     MSVCRT:ucrt_stubs.obj
 0003:00000bb8       ?_OptionsStorage@?1??__local_stdio_printf_options@@9@4_KA 00000001800c6bb8     hb-buffer-serialize.obj
 0003:00000bc0       ?_hb_CrapPool@@3PA_KA      00000001800c6bc0     hb-common.obj
 0003:00000d80       ?_hb_options@@3Uhb_atomic_int_t@@A 00000001800c6d80     hb-common.obj
 0003:00000dd8       ?_hb_subset_accelerator_user_data_key@@3Uhb_user_data_key_t@@A 00000001800c6dd8     hb-subset.obj
 0003:00001744       __favor                    00000001800c7744     MSVCRT:cpu_disp.obj
 0003:00001750       ?__type_info_root_node@@3U__type_info_node@@A 00000001800c7750     MSVCRT:tncleanup.obj
 0003:00001760       ?_OptionsStorage@?1??__local_stdio_scanf_options@@9@4_KA 00000001800c7760     MSVCRT:default_local_stdio_options.obj
 0003:00001768       __scrt_current_native_startup_state 00000001800c7768     MSVCRT:utility.obj
 0003:00001770       __scrt_native_startup_lock 00000001800c7770     MSVCRT:utility.obj
 0003:000017b0       __scrt_debugger_hook_flag  00000001800c77b0     MSVCRT:utility_desktop.obj
 0003:000017c0       sunFontIDs                 00000001800c77c0     <common>
 0003:00001900       lcdInvGammaLUT             00000001800c7900     <common>
 0003:00001dc0       lcdGammaLUT                00000001800c7dc0     <common>
 0003:00002278       __dyn_tls_init_callback    00000001800c8278     <common>

 entry point at        0001:00089344

 Static symbols

 0000:fff2d000       .debug$S                   0000000180000000     fontmanager.exp
 0000:fff2d000       .debug$S                   0000000180000000     vcruntime:VCRUNTIME140.dll
 0000:fff2d000       .debug$S                   0000000180000000     vcruntime:VCRUNTIME140.dll
 0000:fff2d000       .debug$S                   0000000180000000     vcruntime:VCRUNTIME140.dll
 0000:fff2d000       .debug$S                   0000000180000000     vcruntime:VCRUNTIME140.dll
 0000:fff2d000       .debug$S                   0000000180000000     vcruntime:VCRUNTIME140.dll
 0000:fff2d000       .debug$S                   0000000180000000     vcruntime:VCRUNTIME140.dll
 0000:fff2d000       .debug$S                   0000000180000000     vcruntime:VCRUNTIME140.dll
 0000:fff2d000       .debug$S                   0000000180000000     vcruntime:VCRUNTIME140.dll
 0000:fff2d000       .debug$S                   0000000180000000     vcruntime:VCRUNTIME140.dll
 0000:fff2d000       .debug$S                   0000000180000000     vcruntime:VCRUNTIME140.dll
 0000:fff2d000       .debug$S                   0000000180000000     vcruntime:VCRUNTIME140.dll
 0000:fff2d000       .debug$S                   0000000180000000     vcruntime:VCRUNTIME140.dll
 0000:fff2d000       .debug$S                   0000000180000000     vcruntime:VCRUNTIME140.dll
 0000:fff2d000       .debug$S                   0000000180000000     ucrt:api-ms-win-crt-convert-l1-1-0.dll
 0000:fff2d000       .debug$S                   0000000180000000     ucrt:api-ms-win-crt-convert-l1-1-0.dll
 0000:fff2d000       .debug$S                   0000000180000000     ucrt:api-ms-win-crt-convert-l1-1-0.dll
 0000:fff2d000       .debug$S                   0000000180000000     ucrt:api-ms-win-crt-environment-l1-1-0.dll
 0000:fff2d000       .debug$S                   0000000180000000     ucrt:api-ms-win-crt-heap-l1-1-0.dll
 0000:fff2d000       .debug$S                   0000000180000000     ucrt:api-ms-win-crt-heap-l1-1-0.dll
 0000:fff2d000       .debug$S                   0000000180000000     ucrt:api-ms-win-crt-heap-l1-1-0.dll
 0000:fff2d000       .debug$S                   0000000180000000     ucrt:api-ms-win-crt-heap-l1-1-0.dll
 0000:fff2d000       .debug$S                   0000000180000000     ucrt:api-ms-win-crt-math-l1-1-0.dll
 0000:fff2d000       .debug$S                   0000000180000000     ucrt:api-ms-win-crt-math-l1-1-0.dll
 0000:fff2d000       .debug$S                   0000000180000000     ucrt:api-ms-win-crt-math-l1-1-0.dll
 0000:fff2d000       .debug$S                   0000000180000000     ucrt:api-ms-win-crt-math-l1-1-0.dll
 0000:fff2d000       .debug$S                   0000000180000000     ucrt:api-ms-win-crt-math-l1-1-0.dll
 0000:fff2d000       .debug$S                   0000000180000000     ucrt:api-ms-win-crt-math-l1-1-0.dll
 0000:fff2d000       .debug$S                   0000000180000000     ucrt:api-ms-win-crt-math-l1-1-0.dll
 0000:fff2d000       .debug$S                   0000000180000000     ucrt:api-ms-win-crt-math-l1-1-0.dll
 0000:fff2d000       .debug$S                   0000000180000000     ucrt:api-ms-win-crt-math-l1-1-0.dll
 0000:fff2d000       .debug$S                   0000000180000000     ucrt:api-ms-win-crt-math-l1-1-0.dll
 0000:fff2d000       .debug$S                   0000000180000000     ucrt:api-ms-win-crt-math-l1-1-0.dll
 0000:fff2d000       .debug$S                   0000000180000000     ucrt:api-ms-win-crt-runtime-l1-1-0.dll
 0000:fff2d000       .debug$S                   0000000180000000     ucrt:api-ms-win-crt-runtime-l1-1-0.dll
 0000:fff2d000       .debug$S                   0000000180000000     ucrt:api-ms-win-crt-runtime-l1-1-0.dll
 0000:fff2d000       .debug$S                   0000000180000000     ucrt:api-ms-win-crt-runtime-l1-1-0.dll
 0000:fff2d000       .debug$S                   0000000180000000     ucrt:api-ms-win-crt-runtime-l1-1-0.dll
 0000:fff2d000       .debug$S                   0000000180000000     ucrt:api-ms-win-crt-runtime-l1-1-0.dll
 0000:fff2d000       .debug$S                   0000000180000000     ucrt:api-ms-win-crt-runtime-l1-1-0.dll
 0000:fff2d000       .debug$S                   0000000180000000     ucrt:api-ms-win-crt-runtime-l1-1-0.dll
 0000:fff2d000       .debug$S                   0000000180000000     ucrt:api-ms-win-crt-runtime-l1-1-0.dll
 0000:fff2d000       .debug$S                   0000000180000000     ucrt:api-ms-win-crt-runtime-l1-1-0.dll
 0000:fff2d000       .debug$S                   0000000180000000     ucrt:api-ms-win-crt-runtime-l1-1-0.dll
 0000:fff2d000       .debug$S                   0000000180000000     ucrt:api-ms-win-crt-runtime-l1-1-0.dll
 0000:fff2d000       .debug$S                   0000000180000000     ucrt:api-ms-win-crt-runtime-l1-1-0.dll
 0000:fff2d000       .debug$S                   0000000180000000     ucrt:api-ms-win-crt-stdio-l1-1-0.dll
 0000:fff2d000       .debug$S                   0000000180000000     ucrt:api-ms-win-crt-stdio-l1-1-0.dll
 0000:fff2d000       .debug$S                   0000000180000000     ucrt:api-ms-win-crt-stdio-l1-1-0.dll
 0000:fff2d000       .debug$S                   0000000180000000     ucrt:api-ms-win-crt-stdio-l1-1-0.dll
 0000:fff2d000       .debug$S                   0000000180000000     ucrt:api-ms-win-crt-stdio-l1-1-0.dll
 0000:fff2d000       .debug$S                   0000000180000000     ucrt:api-ms-win-crt-stdio-l1-1-0.dll
 0000:fff2d000       .debug$S                   0000000180000000     ucrt:api-ms-win-crt-stdio-l1-1-0.dll
 0000:fff2d000       .debug$S                   0000000180000000     ucrt:api-ms-win-crt-stdio-l1-1-0.dll
 0000:fff2d000       .debug$S                   0000000180000000     ucrt:api-ms-win-crt-string-l1-1-0.dll
 0000:fff2d000       .debug$S                   0000000180000000     ucrt:api-ms-win-crt-string-l1-1-0.dll
 0000:fff2d000       .debug$S                   0000000180000000     ucrt:api-ms-win-crt-string-l1-1-0.dll
 0000:fff2d000       .debug$S                   0000000180000000     ucrt:api-ms-win-crt-string-l1-1-0.dll
 0000:fff2d000       .debug$S                   0000000180000000     ucrt:api-ms-win-crt-string-l1-1-0.dll
 0000:fff2d000       .debug$S                   0000000180000000     advapi32:ADVAPI32.dll
 0000:fff2d000       .debug$S                   0000000180000000     advapi32:ADVAPI32.dll
 0000:fff2d000       .debug$S                   0000000180000000     advapi32:ADVAPI32.dll
 0000:fff2d000       .debug$S                   0000000180000000     advapi32:ADVAPI32.dll
 0000:fff2d000       .debug$S                   0000000180000000     gdi32:GDI32.dll
 0000:fff2d000       .debug$S                   0000000180000000     gdi32:GDI32.dll
 0000:fff2d000       .debug$S                   0000000180000000     gdi32:GDI32.dll
 0000:fff2d000       .debug$S                   0000000180000000     gdi32:GDI32.dll
 0000:fff2d000       .debug$S                   0000000180000000     gdi32:GDI32.dll
 0000:fff2d000       .debug$S                   0000000180000000     gdi32:GDI32.dll
 0000:fff2d000       .debug$S                   0000000180000000     gdi32:GDI32.dll
 0000:fff2d000       .debug$S                   0000000180000000     gdi32:GDI32.dll
 0000:fff2d000       .debug$S                   0000000180000000     gdi32:GDI32.dll
 0000:fff2d000       .debug$S                   0000000180000000     gdi32:GDI32.dll
 0000:fff2d000       .debug$S                   0000000180000000     gdi32:GDI32.dll
 0000:fff2d000       .debug$S                   0000000180000000     gdi32:GDI32.dll
 0000:fff2d000       .debug$S                   0000000180000000     gdi32:GDI32.dll
 0000:fff2d000       .debug$S                   0000000180000000     gdi32:GDI32.dll
 0000:fff2d000       .debug$S                   0000000180000000     gdi32:GDI32.dll
 0000:fff2d000       .debug$S                   0000000180000000     gdi32:GDI32.dll
 0000:fff2d000       .debug$S                   0000000180000000     kernel32:KERNEL32.dll
 0000:fff2d000       .debug$S                   0000000180000000     kernel32:KERNEL32.dll
 0000:fff2d000       .debug$S                   0000000180000000     kernel32:KERNEL32.dll
 0000:fff2d000       .debug$S                   0000000180000000     kernel32:KERNEL32.dll
 0000:fff2d000       .debug$S                   0000000180000000     kernel32:KERNEL32.dll
 0000:fff2d000       .debug$S                   0000000180000000     kernel32:KERNEL32.dll
 0000:fff2d000       .debug$S                   0000000180000000     kernel32:KERNEL32.dll
 0000:fff2d000       .debug$S                   0000000180000000     kernel32:KERNEL32.dll
 0000:fff2d000       .debug$S                   0000000180000000     kernel32:KERNEL32.dll
 0000:fff2d000       .debug$S                   0000000180000000     kernel32:KERNEL32.dll
 0000:fff2d000       .debug$S                   0000000180000000     kernel32:KERNEL32.dll
 0000:fff2d000       .debug$S                   0000000180000000     kernel32:KERNEL32.dll
 0000:fff2d000       .debug$S                   0000000180000000     kernel32:KERNEL32.dll
 0000:fff2d000       .debug$S                   0000000180000000     kernel32:KERNEL32.dll
 0000:fff2d000       .debug$S                   0000000180000000     kernel32:KERNEL32.dll
 0000:fff2d000       .debug$S                   0000000180000000     kernel32:KERNEL32.dll
 0000:fff2d000       .debug$S                   0000000180000000     kernel32:KERNEL32.dll
 0000:fff2d000       .debug$S                   0000000180000000     kernel32:KERNEL32.dll
 0000:fff2d000       .debug$S                   0000000180000000     kernel32:KERNEL32.dll
 0000:fff2d000       .debug$S                   0000000180000000     kernel32:KERNEL32.dll
 0000:fff2d000       .debug$S                   0000000180000000     kernel32:KERNEL32.dll
 0000:fff2d000       .debug$S                   0000000180000000     kernel32:KERNEL32.dll
 0000:fff2d000       .debug$S                   0000000180000000     kernel32:KERNEL32.dll
 0000:fff2d000       .debug$S                   0000000180000000     kernel32:KERNEL32.dll
 0000:fff2d000       .debug$S                   0000000180000000     kernel32:KERNEL32.dll
 0000:fff2d000       .debug$S                   0000000180000000     kernel32:KERNEL32.dll
 0000:fff2d000       .debug$S                   0000000180000000     kernel32:KERNEL32.dll
 0000:fff2d000       .debug$S                   0000000180000000     kernel32:KERNEL32.dll
 0000:fff2d000       .debug$S                   0000000180000000     kernel32:KERNEL32.dll
 0000:fff2d000       .debug$S                   0000000180000000     user32:USER32.dll
 0000:fff2d000       .debug$S                   0000000180000000     user32:USER32.dll
 0000:fff2d000       .debug$S                   0000000180000000     user32:USER32.dll
 0000:fff2d000       .debug$S                   0000000180000000     user32:USER32.dll
 0000:fff2d000       .debug$S                   0000000180000000     user32:USER32.dll
 0000:fff2d000       .debug$S                   0000000180000000     user32:USER32.dll
 0000:fff2d000       .debug$S                   0000000180000000     java:java.dll
 0000:fff2d000       .debug$S                   0000000180000000     java:java.dll
 0000:fff2d000       .debug$S                   0000000180000000     java:java.dll
 0000:fff2d000       .debug$S                   0000000180000000     java:java.dll
 0000:fff2d000       .debug$S                   0000000180000000     java:java.dll
 0000:fff2d000       .debug$S                   0000000180000000     awt:awt.dll
 0000:fff2d000       .debug$S                   0000000180000000     awt:awt.dll
 0000:fff2d000       .debug$S                   0000000180000000     awt:awt.dll
 0000:fff2d000       .debug$S                   0000000180000000     awt:awt.dll
 0000:fff2d000       .debug$S                   0000000180000000     awt:awt.dll
 0000:fff2d000       .debug$S                   0000000180000000     awt:awt.dll
 0000:fff2d000       .debug$S                   0000000180000000     awt:awt.dll
 0000:fff2d000       .debug$S                   0000000180000000     awt:awt.dll
 0000:fff2d000       .debug$S                   0000000180000000     awt:awt.dll
 0000:fff2d000       .debug$S                   0000000180000000     awt:awt.dll
 0000:fff2d000       .debug$S                   0000000180000000     freetype:freetype.dll
 0000:fff2d000       .debug$S                   0000000180000000     freetype:freetype.dll
 0000:fff2d000       .debug$S                   0000000180000000     freetype:freetype.dll
 0000:fff2d000       .debug$S                   0000000180000000     freetype:freetype.dll
 0000:fff2d000       .debug$S                   0000000180000000     freetype:freetype.dll
 0000:fff2d000       .debug$S                   0000000180000000     freetype:freetype.dll
 0000:fff2d000       .debug$S                   0000000180000000     freetype:freetype.dll
 0000:fff2d000       .debug$S                   0000000180000000     freetype:freetype.dll
 0000:fff2d000       .debug$S                   0000000180000000     freetype:freetype.dll
 0000:fff2d000       .debug$S                   0000000180000000     freetype:freetype.dll
 0000:fff2d000       .debug$S                   0000000180000000     freetype:freetype.dll
 0000:fff2d000       .debug$S                   0000000180000000     freetype:freetype.dll
 0000:fff2d000       .debug$S                   0000000180000000     freetype:freetype.dll
 0000:fff2d000       .debug$S                   0000000180000000     freetype:freetype.dll
 0000:fff2d000       .debug$S                   0000000180000000     freetype:freetype.dll
 0000:fff2d000       .debug$S                   0000000180000000     freetype:freetype.dll
 0000:fff2d000       .debug$S                   0000000180000000     freetype:freetype.dll
 0000:fff2d000       .debug$S                   0000000180000000     freetype:freetype.dll
 0000:fff2d000       .debug$S                   0000000180000000     freetype:freetype.dll
 0000:fff2d000       .debug$S                   0000000180000000     freetype:freetype.dll
 0001:00000000       Glyph_GetRasInfo           0000000180001000 f   ColorGlyphSurfaceData.obj
 0001:00000030       Glyph_Lock                 0000000180001030 f   ColorGlyphSurfaceData.obj
 0001:00000450       drawGlyphList              0000000180001450 f   DrawGlyphList.obj
 0001:00000600       drawGlyphListLCD           0000000180001600 f   DrawGlyphList.obj
 0001:00001880       euclidianDistance          0000000180002880 f   HBShaper.obj
 0001:000021e0       CheckFontFamilyProcW       00000001800031e0 f   fontpath.obj
 0001:00002220       EnumFamilyNamesW           0000000180003220 f   fontpath.obj
 0001:00002550       EnumFontFacesInFamilyProcW 0000000180003550 f   fontpath.obj
 0001:00002d70       populateFontFileNameFromRegistryKey 0000000180003d70 f   fontpath.obj
 0001:00003020       registerFontW              0000000180004020 f   fontpath.obj
 0001:000032d0       moveTo                     00000001800042d0 f   freetypeScaler.obj
 0001:00003350       lineTo                     0000000180004350 f   freetypeScaler.obj
 0001:000033b0       conicTo                    00000001800043b0 f   freetypeScaler.obj
 0001:00003460       cubicTo                    0000000180004460 f   freetypeScaler.obj
 0001:00003560       CopyBW2Grey8               0000000180004560 f   freetypeScaler.obj
 0001:00003690       GlyphSlot_Embolden         0000000180004690 f   freetypeScaler.obj
 0001:00004560       ?hb_font_get_glyph_h_kerning_nil@@YAHPEAUhb_font_t@@PEAXII1@Z 0000000180005560 f   hb-font.obj
 0001:00004560       ?hb_font_get_glyph_v_kerning_nil@@YAHPEAUhb_font_t@@PEAXII1@Z 0000000180005560 f   hb-font.obj
 0001:00004560       ?hb_jdk_get_glyph_extents@@YAHPEAUhb_font_t@@PEAXIPEAUhb_glyph_extents_t@@1@Z 0000000180005560 f   hb-jdk-font.obj
 0001:00004560       ?hb_jdk_get_glyph_from_name@@YAHPEAUhb_font_t@@PEAXPEBDHPEAI1@Z 0000000180005560 f   hb-jdk-font.obj
 0001:00004560       ?hb_jdk_get_glyph_h_kerning@@YAHPEAUhb_font_t@@PEAXII1@Z 0000000180005560 f   hb-jdk-font.obj
 0001:00004560       ?hb_jdk_get_glyph_name@@YAHPEAUhb_font_t@@PEAXIPEADI1@Z 0000000180005560 f   hb-jdk-font.obj
 0001:00004560       ?hb_jdk_get_glyph_v_kerning@@YAHPEAUhb_font_t@@PEAXII1@Z 0000000180005560 f   hb-jdk-font.obj
 0001:00004560       ?hb_jdk_get_glyph_v_origin@@YAHPEAUhb_font_t@@PEAXIPEAH21@Z 0000000180005560 f   hb-jdk-font.obj
 0001:00004560       ?hb_paint_custom_palette_color_nil@@YAHPEAUhb_paint_funcs_t@@PEAXIPEAI1@Z 0000000180005560 f   hb-paint.obj
 0001:00004560       ?hb_paint_image_nil@@YAHPEAUhb_paint_funcs_t@@PEAXPEAUhb_blob_t@@IIIMPEAUhb_glyph_extents_t@@1@Z 0000000180005560 f   hb-paint.obj
 0001:00004560       ?hb_unicode_combining_class_nil@@YA?AW4hb_unicode_combining_class_t@@PEAUhb_unicode_funcs_t@@IPEAX@Z 0000000180005560 f   hb-unicode.obj
 0001:00004560       ?hb_unicode_compose_nil@@YAHPEAUhb_unicode_funcs_t@@IIPEAIPEAX@Z 0000000180005560 f   hb-unicode.obj
 0001:00004560       ?hb_unicode_decompose_compatibility_nil@@YAIPEAUhb_unicode_funcs_t@@IPEAIPEAX@Z 0000000180005560 f   hb-unicode.obj
 0001:00004560       ?hb_unicode_decompose_nil@@YAHPEAUhb_unicode_funcs_t@@IPEAI1PEAX@Z 0000000180005560 f   hb-unicode.obj
 0001:00004950       ReadTTFontFileFunc         0000000180005950 f   freetypeScaler.obj
 0001:00004ba0       getFTOutline               0000000180005ba0 f   freetypeScaler.obj
 0001:00004c90       getGlyphGeneralPath        0000000180005c90 f   freetypeScaler.obj
 0001:00004e90       getGlyphImageNativeInternal 0000000180005e90 f   freetypeScaler.obj
 0001:000053c0       invalidateJavaScaler       00000001800063c0 f   freetypeScaler.obj
 0001:00005460       setupFTContext             0000000180006460 f   freetypeScaler.obj
 0001:00005660       ??$_hb_debug_msg@$0A@@@YAXPEBDPEBX0_NIH0ZZ 0000000180006660 f   hb-aat-layout.obj
 0001:00005660       ??$_hb_debug_msg@$0A@@@YAXPEBDPEBX0_NIH0ZZ 0000000180006660 f   hb-blob.obj
 0001:00005660       ??$_hb_debug_msg@$0A@@@YAXPEBDPEBX0_NIH0ZZ 0000000180006660 f   hb-common.obj
 0001:00005660       ?hb_draw_close_path_nil@@YAXPEAUhb_draw_funcs_t@@PEAXPEAUhb_draw_state_t@@1@Z 0000000180006660 f   hb-draw.obj
 0001:00005660       ?hb_draw_cubic_to_nil@@YAXPEAUhb_draw_funcs_t@@PEAXPEAUhb_draw_state_t@@MMMMMM1@Z 0000000180006660 f   hb-draw.obj
 0001:00005660       ?hb_draw_line_to_nil@@YAXPEAUhb_draw_funcs_t@@PEAXPEAUhb_draw_state_t@@MM1@Z 0000000180006660 f   hb-draw.obj
 0001:00005660       ?hb_draw_move_to_nil@@YAXPEAUhb_draw_funcs_t@@PEAXPEAUhb_draw_state_t@@MM1@Z 0000000180006660 f   hb-draw.obj
 0001:00005660       ??$_hb_debug_msg@$0A@@@YAXPEBDPEBX0_NIH0ZZ 0000000180006660 f   hb-face-builder.obj
 0001:00005660       ??$_hb_debug_msg@$0A@@@YAXPEBDPEBX0_NIH0ZZ 0000000180006660 f   hb-face.obj
 0001:00005660       ??$_hb_debug_msg@$0A@@@YAXPEBDPEBX0_NIH0ZZ 0000000180006660 f   hb-font.obj
 0001:00005660       ?hb_font_draw_glyph_nil@@YAXPEAUhb_font_t@@PEAXIPEAUhb_draw_funcs_t@@11@Z 0000000180006660 f   hb-font.obj
 0001:00005660       ?hb_font_paint_glyph_nil@@YAXPEAUhb_font_t@@PEAXIPEAUhb_paint_funcs_t@@1II1@Z 0000000180006660 f   hb-font.obj
 0001:00005660       ?_do_nothing@@YAXXZ        0000000180006660 f   hb-jdk-font.obj
 0001:00005660       ??$_hb_debug_msg@$0A@@@YAXPEBDPEBX0_NIH0ZZ 0000000180006660 f   hb-ot-color.obj
 0001:00005660       ??$_hb_debug_msg@$0A@@@YAXPEBDPEBX0_NIH0ZZ 0000000180006660 f   hb-ot-font.obj
 0001:00005660       ??$_hb_debug_msg@$0A@@@YAXPEBDPEBX0_NIH0ZZ 0000000180006660 f   hb-ot-layout.obj
 0001:00005660       ??$_hb_debug_msg@$0A@@@YAXPEBDPEBX0_NIH0ZZ 0000000180006660 f   hb-ot-metrics.obj
 0001:00005660       ??$_hb_debug_msg@$0A@@@YAXPEBDPEBX0_NIH0ZZ 0000000180006660 f   hb-ot-shaper-arabic.obj
 0001:00005660       ?hb_paint_color_nil@@YAXPEAUhb_paint_funcs_t@@PEAXHI1@Z 0000000180006660 f   hb-paint.obj
 0001:00005660       ?hb_paint_linear_gradient_nil@@YAXPEAUhb_paint_funcs_t@@PEAXPEAUhb_color_line_t@@MMMMMM1@Z 0000000180006660 f   hb-paint.obj
 0001:00005660       ?hb_paint_pop_clip_nil@@YAXPEAUhb_paint_funcs_t@@PEAX1@Z 0000000180006660 f   hb-paint.obj
 0001:00005660       ?hb_paint_pop_group_nil@@YAXPEAUhb_paint_funcs_t@@PEAXW4hb_paint_composite_mode_t@@1@Z 0000000180006660 f   hb-paint.obj
 0001:00005660       ?hb_paint_pop_transform_nil@@YAXPEAUhb_paint_funcs_t@@PEAX1@Z 0000000180006660 f   hb-paint.obj
 0001:00005660       ?hb_paint_push_clip_glyph_nil@@YAXPEAUhb_paint_funcs_t@@PEAXIPEAUhb_font_t@@1@Z 0000000180006660 f   hb-paint.obj
 0001:00005660       ?hb_paint_push_clip_rectangle_nil@@YAXPEAUhb_paint_funcs_t@@PEAXMMMM1@Z 0000000180006660 f   hb-paint.obj
 0001:00005660       ?hb_paint_push_group_nil@@YAXPEAUhb_paint_funcs_t@@PEAX1@Z 0000000180006660 f   hb-paint.obj
 0001:00005660       ?hb_paint_push_transform_nil@@YAXPEAUhb_paint_funcs_t@@PEAXMMMMMM1@Z 0000000180006660 f   hb-paint.obj
 0001:00005660       ?hb_paint_radial_gradient_nil@@YAXPEAUhb_paint_funcs_t@@PEAXPEAUhb_color_line_t@@MMMMMM1@Z 0000000180006660 f   hb-paint.obj
 0001:00005660       ?hb_paint_sweep_gradient_nil@@YAXPEAUhb_paint_funcs_t@@PEAXPEAUhb_color_line_t@@MMMM1@Z 0000000180006660 f   hb-paint.obj
 0001:00005660       ??$_hb_debug_msg@$0A@@@YAXPEBDPEBX0_NIH0ZZ 0000000180006660 f   hb-shape-plan.obj
 0001:000113e0       ?is_deleted_glyph@@YA_NPEBUhb_glyph_info_t@@@Z 00000001800123e0 f   hb-aat-layout.obj
 0001:00013040       $LN270                     0000000180014040     hb-aat-layout.obj
 0001:00013040       $LN270                     0000000180014040     hb-aat-layout.obj
 0001:00013268       $LN270                     0000000180014268     hb-aat-layout.obj
 0001:000135d8       $LN201                     00000001800145d8     hb-aat-layout.obj
 0001:00016e80       ??$sort_r_simple@$$V@@YAXPEAX_K1P6AHPEBX2@Z@Z 0000000180017e80 f   hb-aat-map.obj
 0001:00016e80       ??$sort_r_simple@$$V@@YAXPEAX_K1P6AHPEBX2@Z@Z 0000000180017e80 f   hb-ot-font.obj
 0001:00016e80       ??$sort_r_simple@$$V@@YAXPEAX_K1P6AHPEBX2@Z@Z 0000000180017e80 f   hb-ot-map.obj
 0001:000184e0       ?_hb_blob_destroy@@YAXPEAX@Z 00000001800194e0 f   hb-blob.obj
 0001:00018e10       ?buffer_verify_error@@YAXPEAUhb_buffer_t@@PEAUhb_font_t@@PEBDZZ 0000000180019e10 f   hb-buffer-verify.obj
 0001:00018ec0       ?buffer_verify_unsafe_to_break@@YA_NPEAUhb_buffer_t@@0PEAUhb_font_t@@PEBUhb_feature_t@@IPEBQEBD@Z 0000000180019ec0 f   hb-buffer-verify.obj
 0001:000191f0       ?buffer_verify_unsafe_to_concat@@YA_NPEAUhb_buffer_t@@0PEAUhb_font_t@@PEBUhb_feature_t@@IPEBQEBD@Z 000000018001a1f0 f   hb-buffer-verify.obj
 0001:00019870       ??$hb_buffer_add_utf@U?$hb_utf16_xe_t@G@@@@YAXPEAUhb_buffer_t@@PEBGHIH@Z 000000018001a870 f   hb-buffer.obj
 0001:00021a10       ?lang_find_or_insert@@YAPEAUhb_language_item_t@@PEBD@Z 0000000180022a10 f   hb-common.obj
 0001:00021bf0       ?parse_bool@@YA_NPEAPEBDPEBDPEAI@Z 0000000180022bf0 f   hb-common.obj
 0001:00021d20       ?parse_feature_indices@@YA_NPEAPEBDPEBDPEAUhb_feature_t@@@Z 0000000180022d20 f   hb-common.obj
 0001:00021ec0       ?parse_one_feature@@YA_NPEAPEBDPEBDPEAUhb_feature_t@@@Z 0000000180022ec0 f   hb-common.obj
 0001:00022040       ?parse_tag@@YA_NPEAPEBDPEBDPEAI@Z 0000000180023040 f   hb-common.obj
 0001:00023320       ?hb_draw_quadratic_to_nil@@YAXPEAUhb_draw_funcs_t@@PEAXPEAUhb_draw_state_t@@MMMM1@Z 0000000180024320 f   hb-draw.obj
 0001:00025420       ??$get_glyph_from_symbol@UCmapSubtable@OT@@$1?_hb_arabic_pua_simp_map@@YAII@Z@accelerator_t@cmap@OT@@KA_NPEBXIPEAI@Z 0000000180026420 f   hb-face.obj
 0001:00025490       ??$get_glyph_from_symbol@UCmapSubtable@OT@@$1?_hb_arabic_pua_trad_map@@YAII@Z@accelerator_t@cmap@OT@@KA_NPEBXIPEAI@Z 0000000180026490 f   hb-face.obj
 0001:00025500       ??$get_glyph_from_symbol@UCmapSubtable@OT@@$1?_hb_symbol_pua_map@2@YAII@Z@accelerator_t@cmap@OT@@KA_NPEBXIPEAI@Z 0000000180026500 f   hb-face.obj
 0001:00025570       ??$hb_object_create@Uhb_face_t@@$$V@@YAPEAUhb_face_t@@XZ 0000000180026570 f   hb-face.obj
 0001:000256e0       ??$hb_object_set_user_data@Uhb_face_t@@@@YA_NPEAUhb_face_t@@PEAUhb_user_data_key_t@@PEAXP6AX2@ZH@Z 00000001800266e0 f   hb-face.obj
 0001:00026990       ?_hb_arabic_pua_simp_map@@YAII@Z 0000000180027990 f   hb-face.obj
 0001:00026a30       ?_hb_arabic_pua_trad_map@@YAII@Z 0000000180027a30 f   hb-face.obj
 0001:00026e80       $LN92                      0000000180027e80     hb-face.obj
 0001:000273e4       $LN181                     00000001800283e4     hb-face.obj
 0001:00027e40       ?hb_jdk_get_glyph_h_origin@@YAHPEAUhb_font_t@@PEAXIPEAH21@Z 0000000180028e40 f   hb-jdk-font.obj
 0001:00027e40       ?hb_unicode_eastasian_width_nil@@YAIPEAUhb_unicode_funcs_t@@IPEAX@Z 0000000180028e40 f   hb-unicode.obj
 0001:00027e50       ?hb_font_get_font_h_extents_nil@@YAHPEAUhb_font_t@@PEAXPEAUhb_font_extents_t@@1@Z 0000000180028e50 f   hb-font.obj
 0001:00027e50       ?hb_font_get_font_v_extents_nil@@YAHPEAUhb_font_t@@PEAXPEAUhb_font_extents_t@@1@Z 0000000180028e50 f   hb-font.obj
 0001:00027e70       ?hb_font_get_font_h_extents_default@@YAHPEAUhb_font_t@@PEAXPEAUhb_font_extents_t@@1@Z 0000000180028e70 f   hb-font.obj
 0001:00027f60       ?hb_font_get_font_v_extents_default@@YAHPEAUhb_font_t@@PEAXPEAUhb_font_extents_t@@1@Z 0000000180028f60 f   hb-font.obj
 0001:00028050       ?hb_font_get_nominal_glyph_nil@@YAHPEAUhb_font_t@@PEAXIPEAI1@Z 0000000180029050 f   hb-font.obj
 0001:00028060       ?hb_font_get_nominal_glyph_default@@YAHPEAUhb_font_t@@PEAXIPEAI1@Z 0000000180029060 f   hb-font.obj
 0001:000280f0       ?hb_font_get_nominal_glyphs_default@@YAIPEAUhb_font_t@@PEAXIPEBIIPEAII1@Z 00000001800290f0 f   hb-font.obj
 0001:00028200       ?hb_font_get_glyph_from_name_nil@@YAHPEAUhb_font_t@@PEAXPEBDHPEAI1@Z 0000000180029200 f   hb-font.obj
 0001:00028200       ?hb_font_get_variation_glyph_nil@@YAHPEAUhb_font_t@@PEAXIIPEAI1@Z 0000000180029200 f   hb-font.obj
 0001:00028210       ?hb_font_get_variation_glyph_default@@YAHPEAUhb_font_t@@PEAXIIPEAI1@Z 0000000180029210 f   hb-font.obj
 0001:00028250       ?hb_font_get_glyph_h_advance_nil@@YAHPEAUhb_font_t@@PEAXI1@Z 0000000180029250 f   hb-font.obj
 0001:00028260       ?hb_font_get_glyph_h_advance_default@@YAHPEAUhb_font_t@@PEAXI1@Z 0000000180029260 f   hb-font.obj
 0001:00028330       ?hb_font_get_glyph_v_advance_nil@@YAHPEAUhb_font_t@@PEAXI1@Z 0000000180029330 f   hb-font.obj
 0001:00028340       ?hb_font_get_glyph_v_advance_default@@YAHPEAUhb_font_t@@PEAXI1@Z 0000000180029340 f   hb-font.obj
 0001:00028410       ?hb_font_get_glyph_h_advances_default@@YAXPEAUhb_font_t@@PEAXIPEBIIPEAHI1@Z 0000000180029410 f   hb-font.obj
 0001:00028560       ?hb_font_get_glyph_v_advances_default@@YAXPEAUhb_font_t@@PEAXIPEBIIPEAHI1@Z 0000000180029560 f   hb-font.obj
 0001:000286b0       ?hb_font_get_glyph_h_origin_nil@@YAHPEAUhb_font_t@@PEAXIPEAH21@Z 00000001800296b0 f   hb-font.obj
 0001:000286c0       ?hb_font_get_glyph_h_origin_default@@YAHPEAUhb_font_t@@PEAXIPEAH21@Z 00000001800296c0 f   hb-font.obj
 0001:00028780       ?hb_font_get_glyph_v_origin_nil@@YAHPEAUhb_font_t@@PEAXIPEAH21@Z 0000000180029780 f   hb-font.obj
 0001:00028790       ?hb_font_get_glyph_v_origin_default@@YAHPEAUhb_font_t@@PEAXIPEAH21@Z 0000000180029790 f   hb-font.obj
 0001:00028850       ?hb_font_get_glyph_h_kerning_default@@YAHPEAUhb_font_t@@PEAXII1@Z 0000000180029850 f   hb-font.obj
 0001:000288c0       ?hb_font_get_glyph_v_kerning_default@@YAHPEAUhb_font_t@@PEAXII1@Z 00000001800298c0 f   hb-font.obj
 0001:00028930       ?hb_font_get_glyph_extents_nil@@YAHPEAUhb_font_t@@PEAXIPEAUhb_glyph_extents_t@@1@Z 0000000180029930 f   hb-font.obj
 0001:00028940       ?hb_font_get_glyph_extents_default@@YAHPEAUhb_font_t@@PEAXIPEAUhb_glyph_extents_t@@1@Z 0000000180029940 f   hb-font.obj
 0001:00028a60       ?hb_font_get_glyph_contour_point_nil@@YAHPEAUhb_font_t@@PEAXIIPEAH21@Z 0000000180029a60 f   hb-font.obj
 0001:00028a80       ?hb_font_get_glyph_contour_point_default@@YAHPEAUhb_font_t@@PEAXIIPEAH21@Z 0000000180029a80 f   hb-font.obj
 0001:00028b50       ?hb_font_get_glyph_name_nil@@YAHPEAUhb_font_t@@PEAXIPEADI1@Z 0000000180029b50 f   hb-font.obj
 0001:00028b60       ?hb_font_get_glyph_name_default@@YAHPEAUhb_font_t@@PEAXIPEADI1@Z 0000000180029b60 f   hb-font.obj
 0001:00028ba0       ?hb_font_get_glyph_from_name_default@@YAHPEAUhb_font_t@@PEAXPEBDHPEAI1@Z 0000000180029ba0 f   hb-font.obj
 0001:00028c00       ?hb_draw_move_to_default@@YAXPEAUhb_draw_funcs_t@@PEAXPEAUhb_draw_state_t@@MM1@Z 0000000180029c00 f   hb-font.obj
 0001:00028c50       ?hb_draw_line_to_default@@YAXPEAUhb_draw_funcs_t@@PEAXPEAUhb_draw_state_t@@MM1@Z 0000000180029c50 f   hb-font.obj
 0001:00028ce0       ?hb_draw_quadratic_to_default@@YAXPEAUhb_draw_funcs_t@@PEAXPEAUhb_draw_state_t@@MMMM1@Z 0000000180029ce0 f   hb-font.obj
 0001:00028dc0       ?hb_draw_cubic_to_default@@YAXPEAUhb_draw_funcs_t@@PEAXPEAUhb_draw_state_t@@MMMMMM1@Z 0000000180029dc0 f   hb-font.obj
 0001:00028f00       ?hb_draw_close_path_default@@YAXPEAUhb_draw_funcs_t@@PEAXPEAUhb_draw_state_t@@1@Z 0000000180029f00 f   hb-font.obj
 0001:00028f30       ?hb_font_draw_glyph_default@@YAXPEAUhb_font_t@@PEAXIPEAUhb_draw_funcs_t@@11@Z 0000000180029f30 f   hb-font.obj
 0001:00029020       ?hb_font_paint_glyph_default@@YAXPEAUhb_font_t@@PEAXIPEAUhb_paint_funcs_t@@1II1@Z 000000018002a020 f   hb-font.obj
 0001:00029be0       ?_hb_font_create@@YAPEAUhb_font_t@@PEAUhb_face_t@@@Z 000000018002abe0 f   hb-font.obj
 0001:0002d9d0       ?cleanupFontInfo@@YAXPEAX@Z 000000018002e9d0 f   hb-jdk-font.obj
 0001:0002da10       ?hb_jdk_get_glyph_contour_point@@YAHPEAUhb_font_t@@PEAXIIPEAH21@Z 000000018002ea10 f   hb-jdk-font.obj
 0001:0002daf0       ?hb_jdk_get_glyph_h_advance@@YAHPEAUhb_font_t@@PEAXI1@Z 000000018002eaf0 f   hb-jdk-font.obj
 0001:0002dba0       ?hb_jdk_get_glyph_v_advance@@YAHPEAUhb_font_t@@PEAXI1@Z 000000018002eba0 f   hb-jdk-font.obj
 0001:0002dc40       ?hb_jdk_get_nominal_glyph@@YAHPEAUhb_font_t@@PEAXIPEAI1@Z 000000018002ec40 f   hb-jdk-font.obj
 0001:0002dca0       ?hb_jdk_get_variation_glyph@@YAHPEAUhb_font_t@@PEAXIIPEAI1@Z 000000018002eca0 f   hb-jdk-font.obj
 0001:0002dd10       ?reference_table@@YAPEAUhb_blob_t@@PEAUhb_face_t@@IPEAX@Z 000000018002ed10 f   hb-jdk-font.obj
 0001:0002e1a0       ?strtod_rl@@YANPEBDPEAPEBD@Z 000000018002f1a0 f   hb-number.obj
 0001:0002e900       ?_get_bounds@@YA_NPEBUaccelerator_t@cff1@OT@@IAEAUbounds_t@@_N@Z 000000018002f900 f   hb-ot-cff1-table.obj
 0001:0002ea40       ?_get_path@@YA_NPEBUaccelerator_t@cff1@OT@@PEAUhb_font_t@@IAEAUhb_draw_session_t@@_NPEAUpoint_t@CFF@@@Z 000000018002fa40 f   hb-ot-cff1-table.obj
 0001:0002eda0       $LN30                      000000018002fda0     hb-ot-cff1-table.obj
 0001:0002eda0       $LN30                      000000018002fda0     hb-ot-cff1-table.obj
 0001:0002edb0       $LN29                      000000018002fdb0     hb-ot-cff1-table.obj
 0001:0002edb0       $LN29                      000000018002fdb0     hb-ot-cff1-table.obj
 0001:00033834       $LN578                     0000000180034834     hb-ot-cff1-table.obj
 0001:0003388c       $LN577                     000000018003488c     hb-ot-cff1-table.obj
 0001:00033ed4       $LN661                     0000000180034ed4     hb-ot-cff1-table.obj
 0001:00033f2c       $LN660                     0000000180034f2c     hb-ot-cff1-table.obj
 0001:0003422c       $LN93                      000000018003522c     hb-ot-cff1-table.obj
 0001:0003423c       $LN92                      000000018003523c     hb-ot-cff1-table.obj
 0001:0003e0f0       $LN529                     000000018003f0f0     hb-ot-cff2-table.obj
 0001:0003e148       $LN528                     000000018003f148     hb-ot-cff2-table.obj
 0001:0003e7e8       $LN566                     000000018003f7e8     hb-ot-cff2-table.obj
 0001:0003e840       $LN565                     000000018003f840     hb-ot-cff2-table.obj
 0001:0004254c       $LN675                     000000018004354c     hb-ot-color.obj
 0001:0004730c       $LN369                     000000018004830c     hb-ot-font.obj
 0001:000483e0       ??$sort_r_simple@PEAX@@YAXPEAX_K1P6AHPEBX20@Z0@Z 00000001800493e0 f   hb-ot-font.obj
 0001:00049aa0       ?_hb_ot_font_destroy@@YAXPEAX@Z 000000018004aaa0 f   hb-ot-font.obj
 0001:0004c3d0       ?hb_ot_draw_glyph@@YAXPEAUhb_font_t@@PEAXIPEAUhb_draw_funcs_t@@11@Z 000000018004d3d0 f   hb-ot-font.obj
 0001:0004c820       ?hb_ot_get_font_h_extents@@YAHPEAUhb_font_t@@PEAXPEAUhb_font_extents_t@@1@Z 000000018004d820 f   hb-ot-font.obj
 0001:0004c890       ?hb_ot_get_font_v_extents@@YAHPEAUhb_font_t@@PEAXPEAUhb_font_extents_t@@1@Z 000000018004d890 f   hb-ot-font.obj
 0001:0004c900       ?hb_ot_get_glyph_extents@@YAHPEAUhb_font_t@@PEAXIPEAUhb_glyph_extents_t@@1@Z 000000018004d900 f   hb-ot-font.obj
 0001:0004ca20       ?hb_ot_get_glyph_from_name@@YAHPEAUhb_font_t@@PEAXPEBDHPEAI1@Z 000000018004da20 f   hb-ot-font.obj
 0001:0004cab0       ?hb_ot_get_glyph_h_advances@@YAXPEAUhb_font_t@@PEAXIPEBIIPEAHI1@Z 000000018004dab0 f   hb-ot-font.obj
 0001:0004cef0       ?hb_ot_get_glyph_name@@YAHPEAUhb_font_t@@PEAXIPEADI1@Z 000000018004def0 f   hb-ot-font.obj
 0001:0004d020       ?hb_ot_get_glyph_v_advances@@YAXPEAUhb_font_t@@PEAXIPEBIIPEAHI1@Z 000000018004e020 f   hb-ot-font.obj
 0001:0004d310       ?hb_ot_get_glyph_v_origin@@YAHPEAUhb_font_t@@PEAXIPEAH21@Z 000000018004e310 f   hb-ot-font.obj
 0001:0004d830       ?hb_ot_get_nominal_glyph@@YAHPEAUhb_font_t@@PEAXIPEAI1@Z 000000018004e830 f   hb-ot-font.obj
 0001:0004d900       ?hb_ot_get_nominal_glyphs@@YAIPEAUhb_font_t@@PEAXIPEBIIPEAII1@Z 000000018004e900 f   hb-ot-font.obj
 0001:0004da00       ?hb_ot_get_variation_glyph@@YAHPEAUhb_font_t@@PEAXIIPEAI1@Z 000000018004ea00 f   hb-ot-font.obj
 0001:0004db10       ?hb_ot_paint_glyph@@YAXPEAUhb_font_t@@PEAXIPEAUhb_paint_funcs_t@@1II1@Z 000000018004eb10 f   hb-ot-font.obj
 0001:0004eecc       $LN98                      000000018004fecc     hb-ot-font.obj
 0001:0004ef0c       $LN97                      000000018004ff0c     hb-ot-font.obj
 0001:0004f31c       $LN124                     000000018005031c     hb-ot-font.obj
 0001:0004f364       $LN123                     0000000180050364     hb-ot-font.obj
 0001:00053378       $LN279                     0000000180054378     hb-ot-font.obj
 0001:000533c4       $LN278                     00000001800543c4     hb-ot-font.obj
 0001:000533dc       $LN277                     00000001800543dc     hb-ot-font.obj
 0001:00055c30       ??$apply_string@UGSUBProxy@@@@YA_NPEAUhb_ot_apply_context_t@OT@@AEBUSubstLookup@GSUB_impl@Layout@1@AEBUhb_ot_layout_lookup_accelerator_t@1@@Z 0000000180056c30 f   hb-ot-layout.obj
 0001:00055e60       ??$chain_context_apply_lookup@U?$IntType@G$01@OT@@@OT@@YA_NPEAUhb_ot_apply_context_t@0@IQEBU?$IntType@G$01@0@I1I1IQEBULookupRecord@0@AEBUChainContextApplyLookupContext@0@@Z 0000000180056e60 f   hb-ot-layout.obj
 0001:00056230       ??$context_apply_lookup@U?$IntType@G$01@OT@@@OT@@YA_NPEAUhb_ot_apply_context_t@0@IQEBU?$IntType@G$01@0@IQEBULookupRecord@0@AEBUContextApplyLookupContext@0@@Z 0000000180057230 f   hb-ot-layout.obj
 0001:00056dd8       $LN412                     0000000180057dd8     hb-ot-layout.obj
 0001:00057128       $LN333                     0000000180058128     hb-ot-layout.obj
 0001:00057d70       $LN300                     0000000180058d70     hb-ot-layout.obj
 0001:0005856c       $LN345                     000000018005956c     hb-ot-layout.obj
 0001:00058cb0       $LN293                     0000000180059cb0     hb-ot-layout.obj
 0001:00059360       ??$match_backtrack@U?$IntType@G$01@OT@@@OT@@YA_NPEAUhb_ot_apply_context_t@0@IQEBU?$IntType@G$01@0@P6A_NAEAUhb_glyph_info_t@@IPEBX@Z3PEAI@Z 000000018005a360 f   hb-ot-layout.obj
 0001:00059540       ??$match_input@U?$IntType@G$01@OT@@@OT@@YA_NPEAUhb_ot_apply_context_t@0@IQEBU?$IntType@G$01@0@P6A_NAEAUhb_glyph_info_t@@IPEBX@Z3PEAIQEAI5@Z 000000018005a540 f   hb-ot-layout.obj
 0001:00059540       ??$match_input@UHBGlyphID16@OT@@@OT@@YA_NPEAUhb_ot_apply_context_t@0@IQEBUHBGlyphID16@0@P6A_NAEAUhb_glyph_info_t@@IPEBX@Z3PEAIQEAI5@Z 000000018005a540 f   hb-ot-layout.obj
 0001:000598c0       ??$match_lookahead@U?$IntType@G$01@OT@@@OT@@YA_NPEAUhb_ot_apply_context_t@0@IQEBU?$IntType@G$01@0@P6A_NAEAUhb_glyph_info_t@@IPEBX@Z3IPEAI@Z 000000018005a8c0 f   hb-ot-layout.obj
 0001:0005bee0       ??$would_match_input@U?$IntType@G$01@OT@@@OT@@YA_NPEAUhb_would_apply_context_t@0@IQEBU?$IntType@G$01@0@P6A_NAEAUhb_glyph_info_t@@IPEBX@Z3@Z 000000018005cee0 f   hb-ot-layout.obj
 0001:0005bf90       ?_hb_allocate_lig_id@@YAEPEAUhb_buffer_t@@@Z 000000018005cf90 f   hb-ot-layout.obj
 0001:000604b0       ?apply_backward@@YA_NPEAUhb_ot_apply_context_t@OT@@AEBUhb_ot_layout_lookup_accelerator_t@2@I@Z 00000001800614b0 f   hb-ot-layout.obj
 0001:000606c0       ?apply_forward@@YA_NPEAUhb_ot_apply_context_t@OT@@AEBUhb_ot_layout_lookup_accelerator_t@2@I@Z 00000001800616c0 f   hb-ot-layout.obj
 0001:00060a50       ?apply_lookup@OT@@YAXPEAUhb_ot_apply_context_t@1@IQEAIIQEBULookupRecord@1@I@Z 0000000180061a50 f   hb-ot-layout.obj
 0001:000621d0       ?get_gsubgpos_table@@YAAEBUGSUBGPOS@OT@@PEAUhb_face_t@@I@Z 00000001800631d0 f   hb-ot-layout.obj
 0001:00064c90       ?ligate_input@OT@@YA_NPEAUhb_ot_apply_context_t@1@IQEBIIII@Z 0000000180065c90 f   hb-ot-layout.obj
 0001:00065040       ?match_class@OT@@YA_NAEAUhb_glyph_info_t@@IPEBX@Z 0000000180066040 f   hb-ot-layout.obj
 0001:00065060       ?match_class_cached@OT@@YA_NAEAUhb_glyph_info_t@@IPEBX@Z 0000000180066060 f   hb-ot-layout.obj
 0001:000650a0       ?match_coverage@OT@@YA_NAEAUhb_glyph_info_t@@IPEBX@Z 00000001800660a0 f   hb-ot-layout.obj
 0001:00065140       ?match_glyph@OT@@YA_NAEAUhb_glyph_info_t@@IPEBX@Z 0000000180066140 f   hb-ot-layout.obj
 0001:00065520       ?propagate_attachment_offsets@Layout@OT@@YAXPEAUhb_glyph_position_t@@IIW4hb_direction_t@@I@Z 0000000180066520 f   hb-ot-layout.obj
 0001:00065650       ?reverse_cursive_minor_offset@GPOS_impl@Layout@OT@@YAXPEAUhb_glyph_position_t@@IW4hb_direction_t@@I@Z 0000000180066650 f   hb-ot-layout.obj
 0001:00069d50       ?_fix_ascender_descender@@YAMMW4hb_ot_metrics_tag_t@@@Z 000000018006ad50 f   hb-ot-metrics.obj
 0001:0006a93c       $LN94                      000000018006b93c     hb-ot-shape-fallback.obj
 0001:0006a94c       $LN93                      000000018006b94c     hb-ot-shape-fallback.obj
 0001:0006a9ec       $LN92                      000000018006b9ec     hb-ot-shape-fallback.obj
 0001:0006aa08       $LN91                      000000018006ba08     hb-ot-shape-fallback.obj
 0001:0006ada0       $LN93                      000000018006bda0     hb-ot-shape-fallback.obj
 0001:0006adb8       $LN92                      000000018006bdb8     hb-ot-shape-fallback.obj
 0001:0006b1b0       ?position_around_base@@YAXPEBUhb_ot_shape_plan_t@@PEAUhb_font_t@@PEAUhb_buffer_t@@II_N@Z 000000018006c1b0 f   hb-ot-shape-fallback.obj
 0001:0006b5f0       ?position_cluster@@YAXPEBUhb_ot_shape_plan_t@@PEAUhb_font_t@@PEAUhb_buffer_t@@II_N@Z 000000018006c5f0 f   hb-ot-shape-fallback.obj
 0001:0006b6d0       ?position_mark@@YAXPEBUhb_ot_shape_plan_t@@PEAUhb_font_t@@PEAUhb_buffer_t@@AEAUhb_glyph_extents_t@@II@Z 000000018006c6d0 f   hb-ot-shape-fallback.obj
 0001:0006b8c0       $LN59                      000000018006c8c0     hb-ot-shape-fallback.obj
 0001:0006b8d4       $LN58                      000000018006c8d4     hb-ot-shape-fallback.obj
 0001:0006b8f8       $LN57                      000000018006c8f8     hb-ot-shape-fallback.obj
 0001:0006b90c       $LN56                      000000018006c90c     hb-ot-shape-fallback.obj
 0001:0006b930       ?_hb_glyph_info_set_unicode_props@@YAXPEAUhb_glyph_info_t@@PEAUhb_buffer_t@@@Z 000000018006c930 f   hb-ot-shape-normalize.obj
 0001:0006b930       ?_hb_glyph_info_set_unicode_props@@YAXPEAUhb_glyph_info_t@@PEAUhb_buffer_t@@@Z 000000018006c930 f   hb-ot-shape.obj
 0001:0006c590       $LN379                     000000018006d590     hb-ot-shape-normalize.obj
 0001:0006c5c0       $LN378                     000000018006d5c0     hb-ot-shape-normalize.obj
 0001:0006c620       ?compare_combining_class@@YAHPEBUhb_glyph_info_t@@0@Z 000000018006d620 f   hb-ot-shape-normalize.obj
 0001:0006c670       ?compose_unicode@@YA_NPEBUhb_ot_shape_normalize_context_t@@IIPEAI@Z 000000018006d670 f   hb-ot-shape-normalize.obj
 0001:0006c6b0       ?decompose@@YAIPEBUhb_ot_shape_normalize_context_t@@_NI@Z 000000018006d6b0 f   hb-ot-shape-normalize.obj
 0001:0006c830       ?decompose_current_character@@YAXPEBUhb_ot_shape_normalize_context_t@@_N@Z 000000018006d830 f   hb-ot-shape-normalize.obj
 0001:0006cb10       $LN98                      000000018006db10     hb-ot-shape-normalize.obj
 0001:0006cb40       $LN97                      000000018006db40     hb-ot-shape-normalize.obj
 0001:0006cba0       ?decompose_unicode@@YA_NPEBUhb_ot_shape_normalize_context_t@@IPEAI1@Z 000000018006dba0 f   hb-ot-shape-normalize.obj
 0001:0006cbd0       ?handle_variation_selector_cluster@@YAXPEBUhb_ot_shape_normalize_context_t@@I_N@Z 000000018006dbd0 f   hb-ot-shape-normalize.obj
 0001:0006cfe0       ?output_char@@YAXPEAUhb_buffer_t@@II@Z 000000018006dfe0 f   hb-ot-shape-normalize.obj
 0001:0006d090       ?_hb_glyph_info_is_default_ignorable@@YA_NPEBUhb_glyph_info_t@@@Z 000000018006e090 f   hb-ot-shape.obj
 0001:0006d0b0       ?_hb_grapheme_group_func@@YA_NAEBUhb_glyph_info_t@@0@Z 000000018006e0b0 f   hb-ot-shape.obj
 0001:0006d790       ?hb_form_clusters@@YAXPEAUhb_buffer_t@@@Z 000000018006e790 f   hb-ot-shape.obj
 0001:0006d910       ?hb_ot_position_default@@YAXPEBUhb_ot_shape_context_t@@@Z 000000018006e910 f   hb-ot-shape.obj
 0001:0006dac0       ?hb_ot_position_plan@@YAXPEBUhb_ot_shape_context_t@@@Z 000000018006eac0 f   hb-ot-shape.obj
 0001:0006dd70       ?hb_ot_rotate_chars@@YAXPEBUhb_ot_shape_context_t@@@Z 000000018006ed70 f   hb-ot-shape.obj
 0001:0006e06c       $LN90                      000000018006f06c     hb-ot-shape.obj
 0001:0006e0a0       $LN89                      000000018006f0a0     hb-ot-shape.obj
 0001:0006e100       $LN88                      000000018006f100     hb-ot-shape.obj
 0001:0006e160       ?hb_ot_shape_collect_features@@YAXPEAUhb_ot_shape_planner_t@@PEBUhb_feature_t@@I@Z 000000018006f160 f   hb-ot-shape.obj
 0001:0006e400       ?hb_ot_shape_internal@@YAXPEAUhb_ot_shape_context_t@@@Z 000000018006f400 f   hb-ot-shape.obj
 0001:0006e7a0       ?hb_ot_shape_setup_masks_fraction@@YAXPEBUhb_ot_shape_context_t@@@Z 000000018006f7a0 f   hb-ot-shape.obj
 0001:0006e970       ?hb_ot_shaper_categorize@@YAPEBUhb_ot_shaper_t@@PEBUhb_ot_shape_planner_t@@@Z 000000018006f970 f   hb-ot-shape.obj
 0001:0006ee60       ?hb_ot_substitute_default@@YAXPEBUhb_ot_shape_context_t@@@Z 000000018006fe60 f   hb-ot-shape.obj
 0001:0006efe0       ?hb_ot_substitute_post@@YAXPEBUhb_ot_shape_context_t@@@Z 000000018006ffe0 f   hb-ot-shape.obj
 0001:0006f130       ?hb_propagate_flags@@YAXPEAUhb_buffer_t@@@Z 0000000180070130 f   hb-ot-shape.obj
 0001:0006f3c0       ?hb_set_unicode_props@@YAXPEAUhb_buffer_t@@@Z 00000001800703c0 f   hb-ot-shape.obj
 0001:0006f690       ?zero_mark_widths_by_gdef@@YAXPEAUhb_buffer_t@@_N@Z 0000000180070690 f   hb-ot-shape.obj
 0001:0006f770       ?setup_masks_arabic@@YAXPEBUhb_ot_shape_plan_t@@PEAUhb_buffer_t@@PEAUhb_font_t@@@Z 0000000180070770 f   hb-ot-shaper-arabic.obj
 0001:0006f840       ?postprocess_glyphs_arabic@@YAXPEBUhb_ot_shape_plan_t@@PEAUhb_buffer_t@@PEAUhb_font_t@@@Z 0000000180070840 f   hb-ot-shaper-arabic.obj
 0001:0006f850       ?reorder_marks_arabic@@YAXPEBUhb_ot_shape_plan_t@@PEAUhb_buffer_t@@II@Z 0000000180070850 f   hb-ot-shaper-arabic.obj
 0001:0006fcf0       ?collect_features_arabic@@YAXPEAUhb_ot_shape_planner_t@@@Z 0000000180070cf0 f   hb-ot-shaper-arabic.obj
 0001:00070020       ??$arabic_fallback_synthesize_lookup_ligature@$$BY00Uligature_3_set_t@@@@YAPEAUSubstLookup@GSUB_impl@Layout@OT@@PEBUhb_ot_shape_plan_t@@PEAUhb_font_t@@AEAY00$$CBUligature_3_set_t@@I@Z 0000000180071020 f   hb-ot-shaper-arabic.obj
 0001:00070730       ??$arabic_fallback_synthesize_lookup_ligature@$$BY00Uligature_mark_set_t@@@@YAPEAUSubstLookup@GSUB_impl@Layout@OT@@PEBUhb_ot_shape_plan_t@@PEAUhb_font_t@@AEAY00$$CBUligature_mark_set_t@@I@Z 0000000180071730 f   hb-ot-shaper-arabic.obj
 0001:00070fb0       ??$arabic_fallback_synthesize_lookup_ligature@$$BY0BC@Uligature_set_t@@@@YAPEAUSubstLookup@GSUB_impl@Layout@OT@@PEBUhb_ot_shape_plan_t@@PEAUhb_font_t@@AEAY0BC@$$CBUligature_set_t@@I@Z 0000000180071fb0 f   hb-ot-shaper-arabic.obj
 0001:00071940       ??$hb_stable_sort@UHBGlyphID16@OT@@U?$IntType@G$01@2@I@@YAXPEAUHBGlyphID16@OT@@IP6AHPEBU?$IntType@G$01@1@1@ZPEAI@Z 0000000180072940 f   hb-ot-shaper-arabic.obj
 0001:00072b70       ?apply_stch@@YAXPEBUhb_ot_shape_plan_t@@PEAUhb_buffer_t@@PEAUhb_font_t@@@Z 0000000180073b70 f   hb-ot-shaper-arabic.obj
 0001:00073070       ?arabic_fallback_plan_init_unicode@@YA_NPEAUarabic_fallback_plan_t@@PEBUhb_ot_shape_plan_t@@PEAUhb_font_t@@@Z 0000000180074070 f   hb-ot-shaper-arabic.obj
 0001:000733b0       ?arabic_fallback_plan_init_win1256@@YA_NPEAUarabic_fallback_plan_t@@PEBUhb_ot_shape_plan_t@@PEAUhb_font_t@@@Z 00000001800743b0 f   hb-ot-shaper-arabic.obj
 0001:00073600       ?arabic_fallback_shape@@YA_NPEBUhb_ot_shape_plan_t@@PEAUhb_font_t@@PEAUhb_buffer_t@@@Z 0000000180074600 f   hb-ot-shaper-arabic.obj
 0001:000737e0       ?arabic_fallback_synthesize_lookup_single@@YAPEAUSubstLookup@GSUB_impl@Layout@OT@@PEBUhb_ot_shape_plan_t@@PEAUhb_font_t@@I@Z 00000001800747e0 f   hb-ot-shaper-arabic.obj
 0001:00073cb0       ?arabic_joining@@YAXPEAUhb_buffer_t@@@Z 0000000180074cb0 f   hb-ot-shaper-arabic.obj
 0001:000740b0       ?deallocate_buffer_var@@YA_NPEBUhb_ot_shape_plan_t@@PEAUhb_font_t@@PEAUhb_buffer_t@@@Z 00000001800750b0 f   hb-ot-shaper-arabic.obj
 0001:000743a0       ?get_joining_type@@YAIIW4hb_unicode_general_category_t@@@Z 00000001800753a0 f   hb-ot-shaper-arabic.obj
 0001:000744dc       $LN49                      00000001800754dc     hb-ot-shaper-arabic.obj
 0001:000744fc       $LN48                      00000001800754fc     hb-ot-shaper-arabic.obj
 0001:000746b0       ?record_stch@@YA_NPEBUhb_ot_shape_plan_t@@PEAUhb_font_t@@PEAUhb_buffer_t@@@Z 00000001800756b0 f   hb-ot-shaper-arabic.obj
 0001:00075570       ?collect_features_hangul@@YAXPEAUhb_ot_shape_planner_t@@@Z 0000000180076570 f   hb-ot-shaper-hangul.obj
 0001:000755c0       ?override_features_hangul@@YAXPEAUhb_ot_shape_planner_t@@@Z 00000001800765c0 f   hb-ot-shaper-hangul.obj
 0001:000755e0       ?data_create_hangul@@YAPEAXPEBUhb_ot_shape_plan_t@@@Z 00000001800765e0 f   hb-ot-shaper-hangul.obj
 0001:00075770       ?data_destroy_hangul@@YAXPEAX@Z 0000000180076770 f   hb-ot-shaper-hangul.obj
 0001:00075770       ?data_destroy_indic@@YAXPEAX@Z 0000000180076770 f   hb-ot-shaper-indic.obj
 0001:00075770       ?data_destroy_khmer@@YAXPEAX@Z 0000000180076770 f   hb-ot-shaper-khmer.obj
 0001:00075780       ?preprocess_text_hangul@@YAXPEBUhb_ot_shape_plan_t@@PEAUhb_buffer_t@@PEAUhb_font_t@@@Z 0000000180076780 f   hb-ot-shaper-hangul.obj
 0001:00076630       ?setup_masks_hangul@@YAXPEBUhb_ot_shape_plan_t@@PEAUhb_buffer_t@@PEAUhb_font_t@@@Z 0000000180077630 f   hb-ot-shaper-hangul.obj
 0001:00076670       ?compose_hebrew@@YA_NPEBUhb_ot_shape_normalize_context_t@@IIPEAI@Z 0000000180077670 f   hb-ot-shaper-hebrew.obj
 0001:00076818       $LN41                      0000000180077818     hb-ot-shaper-hebrew.obj
 0001:00076860       ?reorder_marks_hebrew@@YAXPEBUhb_ot_shape_plan_t@@PEAUhb_buffer_t@@II@Z 0000000180077860 f   hb-ot-shaper-hebrew.obj
 0001:00076b48       $LN59                      0000000180077b48     hb-ot-shaper-indic-table.obj
 0001:00076b90       ?collect_features_indic@@YAXPEAUhb_ot_shape_planner_t@@@Z 0000000180077b90 f   hb-ot-shaper-indic.obj
 0001:00076c80       ?override_features_indic@@YAXPEAUhb_ot_shape_planner_t@@@Z 0000000180077c80 f   hb-ot-shaper-indic.obj
 0001:00076cc0       ?data_create_indic@@YAPEAXPEBUhb_ot_shape_plan_t@@@Z 0000000180077cc0 f   hb-ot-shaper-indic.obj
 0001:00076ea0       ?setup_masks_indic@@YAXPEBUhb_ot_shape_plan_t@@PEAUhb_buffer_t@@PEAUhb_font_t@@@Z 0000000180077ea0 f   hb-ot-shaper-indic.obj
 0001:00076ef0       ?preprocess_text_indic@@YAXPEBUhb_ot_shape_plan_t@@PEAUhb_buffer_t@@PEAUhb_font_t@@@Z 0000000180077ef0 f   hb-ot-shaper-indic.obj
 0001:00076f10       ?decompose_indic@@YA_NPEBUhb_ot_shape_normalize_context_t@@IPEAI1@Z 0000000180077f10 f   hb-ot-shaper-indic.obj
 0001:00076f70       ?compose_indic@@YA_NPEBUhb_ot_shape_normalize_context_t@@IIPEAI@Z 0000000180077f70 f   hb-ot-shaper-indic.obj
 0001:00077020       ?consonant_position_from_face@@YA?AW4ot_position_t@@PEBUindic_shape_plan_t@@IIPEAUhb_face_t@@@Z 0000000180078020 f   hb-ot-shaper-indic.obj
 0001:00077270       ?final_reordering_indic@@YA_NPEBUhb_ot_shape_plan_t@@PEAUhb_font_t@@PEAUhb_buffer_t@@@Z 0000000180078270 f   hb-ot-shaper-indic.obj
 0001:00077370       ?final_reordering_syllable_indic@@YAXPEBUhb_ot_shape_plan_t@@PEAUhb_buffer_t@@II@Z 0000000180078370 f   hb-ot-shaper-indic.obj
 0001:00078518       $LN241                     0000000180079518     hb-ot-shaper-indic.obj
 0001:00078690       ?initial_reordering_consonant_syllable@@YAXPEBUhb_ot_shape_plan_t@@PEAUhb_face_t@@PEAUhb_buffer_t@@II@Z 0000000180079690 f   hb-ot-shaper-indic.obj
 0001:00079410       ?initial_reordering_indic@@YA_NPEBUhb_ot_shape_plan_t@@PEAUhb_font_t@@PEAUhb_buffer_t@@@Z 000000018007a410 f   hb-ot-shaper-indic.obj
 0001:00079640       ?setup_syllables_indic@@YA_NPEBUhb_ot_shape_plan_t@@PEAUhb_font_t@@PEAUhb_buffer_t@@@Z 000000018007a640 f   hb-ot-shaper-indic.obj
 0001:000797f0       ?collect_features_khmer@@YAXPEAUhb_ot_shape_planner_t@@@Z 000000018007a7f0 f   hb-ot-shaper-khmer.obj
 0001:000798d0       ?override_features_khmer@@YAXPEAUhb_ot_shape_planner_t@@@Z 000000018007a8d0 f   hb-ot-shaper-khmer.obj
 0001:00079940       ?data_create_khmer@@YAPEAXPEBUhb_ot_shape_plan_t@@@Z 000000018007a940 f   hb-ot-shaper-khmer.obj
 0001:00079ac0       ?setup_masks_khmer@@YAXPEBUhb_ot_shape_plan_t@@PEAUhb_buffer_t@@PEAUhb_font_t@@@Z 000000018007aac0 f   hb-ot-shaper-khmer.obj
 0001:00079b00       ?decompose_khmer@@YA_NPEBUhb_ot_shape_normalize_context_t@@IPEAI1@Z 000000018007ab00 f   hb-ot-shaper-khmer.obj
 0001:00079bc0       ?compose_khmer@@YA_NPEBUhb_ot_shape_normalize_context_t@@IIPEAI@Z 000000018007abc0 f   hb-ot-shaper-khmer.obj
 0001:00079bc0       ?compose_use@@YA_NPEBUhb_ot_shape_normalize_context_t@@IIPEAI@Z 000000018007abc0 f   hb-ot-shaper-use.obj
 0001:0007a034       $LN151                     000000018007b034     hb-ot-shaper-khmer.obj
 0001:0007a070       ?reorder_consonant_syllable@@YAXPEBUhb_ot_shape_plan_t@@PEAUhb_face_t@@PEAUhb_buffer_t@@II@Z 000000018007b070 f   hb-ot-shaper-khmer.obj
 0001:0007a320       ?reorder_khmer@@YA_NPEBUhb_ot_shape_plan_t@@PEAUhb_font_t@@PEAUhb_buffer_t@@@Z 000000018007b320 f   hb-ot-shaper-khmer.obj
 0001:0007a450       ?setup_syllables_khmer@@YA_NPEBUhb_ot_shape_plan_t@@PEAUhb_font_t@@PEAUhb_buffer_t@@@Z 000000018007b450 f   hb-ot-shaper-khmer.obj
 0001:0007a570       ?collect_features_myanmar@@YAXPEAUhb_ot_shape_planner_t@@@Z 000000018007b570 f   hb-ot-shaper-myanmar.obj
 0001:0007a680       ?setup_masks_myanmar@@YAXPEBUhb_ot_shape_plan_t@@PEAUhb_buffer_t@@PEAUhb_font_t@@@Z 000000018007b680 f   hb-ot-shaper-myanmar.obj
 0001:0007a6c0       ?compare_myanmar_order@@YAHPEBUhb_glyph_info_t@@0@Z 000000018007b6c0 f   hb-ot-shaper-myanmar.obj
 0001:0007a9e8       $LN128                     000000018007b9e8     hb-ot-shaper-myanmar.obj
 0001:0007aa10       ?initial_reordering_consonant_syllable@@YAXPEAUhb_buffer_t@@II@Z 000000018007ba10 f   hb-ot-shaper-myanmar.obj
 0001:0007ad50       ?reorder_myanmar@@YA_NPEBUhb_ot_shape_plan_t@@PEAUhb_font_t@@PEAUhb_buffer_t@@@Z 000000018007bd50 f   hb-ot-shaper-myanmar.obj
 0001:0007ae80       ?setup_syllables_myanmar@@YA_NPEBUhb_ot_shape_plan_t@@PEAUhb_font_t@@PEAUhb_buffer_t@@@Z 000000018007be80 f   hb-ot-shaper-myanmar.obj
 0001:0007b230       ?preprocess_text_thai@@YAXPEBUhb_ot_shape_plan_t@@PEAUhb_buffer_t@@PEAUhb_font_t@@@Z 000000018007c230 f   hb-ot-shaper-thai.obj
 0001:0007b560       ?do_thai_pua_shaping@@YAXPEBUhb_ot_shape_plan_t@@PEAUhb_buffer_t@@PEAUhb_font_t@@@Z 000000018007c560 f   hb-ot-shaper-thai.obj
 0001:0007b800       ?thai_pua_shape@@YAIIW4thai_action_t@@PEAUhb_font_t@@@Z 000000018007c800 f   hb-ot-shaper-thai.obj
 0001:0007b8e0       ?collect_features_use@@YAXPEAUhb_ot_shape_planner_t@@@Z 000000018007c8e0 f   hb-ot-shaper-use.obj
 0001:0007baa0       ?data_create_use@@YAPEAXPEBUhb_ot_shape_plan_t@@@Z 000000018007caa0 f   hb-ot-shaper-use.obj
 0001:0007bbb0       ?data_destroy_use@@YAXPEAX@Z 000000018007cbb0 f   hb-ot-shaper-use.obj
 0001:0007bbe0       ?setup_masks_use@@YAXPEBUhb_ot_shape_plan_t@@PEAUhb_buffer_t@@PEAUhb_font_t@@@Z 000000018007cbe0 f   hb-ot-shaper-use.obj
 0001:0007bcf0       ?preprocess_text_use@@YAXPEBUhb_ot_shape_plan_t@@PEAUhb_buffer_t@@PEAUhb_font_t@@@Z 000000018007ccf0 f   hb-ot-shaper-use.obj
 0001:0007bd00       ??0?$hb_filter_iter_t@U?$hb_filter_iter_t@U?$hb_zip_iter_t@U?$hb_iota_iter_t@II@@U?$hb_array_t@Uhb_glyph_info_t@@@@@@V<lambda_e52748becc06432fe81365edeb8c4003>@@AEBU<unnamed-type-hb_second>@@$0A@@@V<lambda_a2885d5959499a7c5bcf896c0de144bb>@@AEBU<unnamed-type-hb_identity>@@$0A@@@QEAA@AEBU?$hb_filter_iter_t@U?$hb_zip_iter_t@U?$hb_iota_iter_t@II@@U?$hb_array_t@Uhb_glyph_info_t@@@@@@V<lambda_e52748becc06432fe81365edeb8c4003>@@AEBU<unnamed-type-hb_second>@@$0A@@@V<lambda_a2885d5959499a7c5bcf896c0de144bb>@@AEBU<unnamed-type-hb_identity>@@@Z 000000018007cd00 f   hb-ot-shaper-use.obj
 0001:0007bea0       ??4?$machine_index_t@U?$hb_zip_iter_t@U?$hb_iota_iter_t@II@@U?$hb_filter_iter_t@U?$hb_filter_iter_t@U?$hb_zip_iter_t@U?$hb_iota_iter_t@II@@U?$hb_array_t@Uhb_glyph_info_t@@@@@@V<lambda_e52748becc06432fe81365edeb8c4003>@@AEBU<unnamed-type-hb_second>@@$0A@@@V<lambda_a2885d5959499a7c5bcf896c0de144bb>@@AEBU<unnamed-type-hb_identity>@@$0A@@@@@@@QEAAXAEBU0@@Z 000000018007cea0 f   hb-ot-shaper-use.obj
 0001:0007bfb0       ??Y?$hb_iter_t@U?$hb_zip_iter_t@U?$hb_iota_iter_t@II@@U?$hb_filter_iter_t@U?$hb_filter_iter_t@U?$hb_zip_iter_t@U?$hb_iota_iter_t@II@@U?$hb_array_t@Uhb_glyph_info_t@@@@@@V<lambda_e52748becc06432fe81365edeb8c4003>@@AEBU<unnamed-type-hb_second>@@$0A@@@V<lambda_a2885d5959499a7c5bcf896c0de144bb>@@AEBU<unnamed-type-hb_identity>@@$0A@@@@@U?$hb_pair_t@IU?$hb_pair_t@IAEAUhb_glyph_info_t@@@@@@@@QEGAAAEAU?$hb_zip_iter_t@U?$hb_iota_iter_t@II@@U?$hb_filter_iter_t@U?$hb_filter_iter_t@U?$hb_zip_iter_t@U?$hb_iota_iter_t@II@@U?$hb_array_t@Uhb_glyph_info_t@@@@@@V<lambda_e52748becc06432fe81365edeb8c4003>@@AEBU<unnamed-type-hb_second>@@$0A@@@V<lambda_a2885d5959499a7c5bcf896c0de144bb>@@AEBU<unnamed-type-hb_identity>@@$0A@@@@@I@Z 000000018007cfb0 f   hb-ot-shaper-use.obj
 0001:0007c0c0       ?__item__@?$hb_zip_iter_t@U?$hb_iota_iter_t@II@@U?$hb_filter_iter_t@U?$hb_filter_iter_t@U?$hb_zip_iter_t@U?$hb_iota_iter_t@II@@U?$hb_array_t@Uhb_glyph_info_t@@@@@@V<lambda_e52748becc06432fe81365edeb8c4003>@@AEBU<unnamed-type-hb_second>@@$0A@@@V<lambda_a2885d5959499a7c5bcf896c0de144bb>@@AEBU<unnamed-type-hb_identity>@@$0A@@@@@QEBA?AU?$hb_pair_t@IU?$hb_pair_t@IAEAUhb_glyph_info_t@@@@@@XZ 000000018007d0c0 f   hb-ot-shaper-use.obj
 0001:0007c140       ?__next__@?$hb_filter_iter_t@U?$hb_filter_iter_t@U?$hb_zip_iter_t@U?$hb_iota_iter_t@II@@U?$hb_array_t@Uhb_glyph_info_t@@@@@@V<lambda_e52748becc06432fe81365edeb8c4003>@@AEBU<unnamed-type-hb_second>@@$0A@@@V<lambda_a2885d5959499a7c5bcf896c0de144bb>@@AEBU<unnamed-type-hb_identity>@@$0A@@@QEAAXXZ 000000018007d140 f   hb-ot-shaper-use.obj
 0001:0007c2c0       ?__prev__@?$hb_filter_iter_t@U?$hb_filter_iter_t@U?$hb_zip_iter_t@U?$hb_iota_iter_t@II@@U?$hb_array_t@Uhb_glyph_info_t@@@@@@V<lambda_e52748becc06432fe81365edeb8c4003>@@AEBU<unnamed-type-hb_second>@@$0A@@@V<lambda_a2885d5959499a7c5bcf896c0de144bb>@@AEBU<unnamed-type-hb_identity>@@$0A@@@QEAAXXZ 000000018007d2c0 f   hb-ot-shaper-use.obj
 0001:0007c440       ?_hb_clear_substitution_flags@@YA_NPEBUhb_ot_shape_plan_t@@PEAUhb_font_t@@PEAUhb_buffer_t@@@Z 000000018007d440 f   hb-ot-shaper-use.obj
 0001:0007c470       ?find_syllables_use@@YAXPEAUhb_buffer_t@@@Z 000000018007d470 f   hb-ot-shaper-use.obj
 0001:0007d6d8       $LN1772                    000000018007e6d8     hb-ot-shaper-use.obj
 0001:0007d720       ?record_pref_use@@YA_NPEBUhb_ot_shape_plan_t@@PEAUhb_font_t@@PEAUhb_buffer_t@@@Z 000000018007e720 f   hb-ot-shaper-use.obj
 0001:0007d7f0       ?record_rphf_use@@YA_NPEBUhb_ot_shape_plan_t@@PEAUhb_font_t@@PEAUhb_buffer_t@@@Z 000000018007e7f0 f   hb-ot-shaper-use.obj
 0001:0007d8e0       ?reorder_syllable_use@@YAXPEAUhb_buffer_t@@II@Z 000000018007e8e0 f   hb-ot-shaper-use.obj
 0001:0007db10       ?reorder_use@@YA_NPEBUhb_ot_shape_plan_t@@PEAUhb_font_t@@PEAUhb_buffer_t@@@Z 000000018007eb10 f   hb-ot-shaper-use.obj
 0001:0007dc20       ?setup_syllables_use@@YA_NPEBUhb_ot_shape_plan_t@@PEAUhb_font_t@@PEAUhb_buffer_t@@@Z 000000018007ec20 f   hb-ot-shaper-use.obj
 0001:0007de00       ?setup_topographical_masks@@YAXPEBUhb_ot_shape_plan_t@@PEAUhb_buffer_t@@@Z 000000018007ee00 f   hb-ot-shaper-use.obj
 0001:0007e168       $LN184                     000000018007f168     hb-ot-shaper-use.obj
 0001:0007ed50       $LN454                     000000018007fd50     hb-ot-shaper-vowel-constraints.obj
 0001:0007ed8c       $LN453                     000000018007fd8c     hb-ot-shaper-vowel-constraints.obj
 0001:0007ed94       $LN452                     000000018007fd94     hb-ot-shaper-vowel-constraints.obj
 0001:0007edb4       $LN451                     000000018007fdb4     hb-ot-shaper-vowel-constraints.obj
 0001:0007edf4       $LN450                     000000018007fdf4     hb-ot-shaper-vowel-constraints.obj
 0001:0007edfc       $LN449                     000000018007fdfc     hb-ot-shaper-vowel-constraints.obj
 0001:0007ee20       ?_output_with_dotted_circle@@YAXPEAUhb_buffer_t@@@Z 000000018007fe20 f   hb-ot-shaper-vowel-constraints.obj
 0001:0007eec0       ?hb_ot_ambiguous_tag_to_language@@YAPEBUhb_language_impl_t@@I@Z 000000018007fec0 f   hb-ot-tag.obj
 0001:0007f710       ?hb_ot_tags_from_complex_language@@YA_NPEBD0PEAI1@Z 0000000180080710 f   hb-ot-tag.obj
 0001:00081864       $LN994                     0000000180082864     hb-ot-tag.obj
 0001:000818d0       ?hb_ot_tags_from_language@@YAXPEBD0PEAI1@Z 00000001800828d0 f   hb-ot-tag.obj
 0001:00081ae0       ?subtag_matches@@YA_NPEBD00I@Z 0000000180082ae0 f   hb-ot-tag.obj
 0001:00082f00       ?hb_outline_recording_pen_close_path@@YAXPEAUhb_draw_funcs_t@@PEAXPEAUhb_draw_state_t@@1@Z 0000000180083f00 f   hb-outline.obj
 0001:00082fc0       ?hb_outline_recording_pen_cubic_to@@YAXPEAUhb_draw_funcs_t@@PEAXPEAUhb_draw_state_t@@MMMMMM1@Z 0000000180083fc0 f   hb-outline.obj
 0001:00083160       ?hb_outline_recording_pen_line_to@@YAXPEAUhb_draw_funcs_t@@PEAXPEAUhb_draw_state_t@@MM1@Z 0000000180084160 f   hb-outline.obj
 0001:00083190       ?hb_outline_recording_pen_move_to@@YAXPEAUhb_draw_funcs_t@@PEAXPEAUhb_draw_state_t@@MM1@Z 0000000180084190 f   hb-outline.obj
 0001:000831c0       ?hb_outline_recording_pen_quadratic_to@@YAXPEAUhb_draw_funcs_t@@PEAXPEAUhb_draw_state_t@@MMMM1@Z 00000001800841c0 f   hb-outline.obj
 0001:00083860       ?hb_draw_extents_cubic_to@@YAXPEAUhb_draw_funcs_t@@PEAXPEAUhb_draw_state_t@@MMMMMM1@Z 0000000180084860 f   hb-paint-extents.obj
 0001:000838b0       ?hb_draw_extents_line_to@@YAXPEAUhb_draw_funcs_t@@PEAXPEAUhb_draw_state_t@@MM1@Z 00000001800848b0 f   hb-paint-extents.obj
 0001:000838b0       ?hb_draw_extents_move_to@@YAXPEAUhb_draw_funcs_t@@PEAXPEAUhb_draw_state_t@@MM1@Z 00000001800848b0 f   hb-paint-extents.obj
 0001:000838d0       ?hb_draw_extents_quadratic_to@@YAXPEAUhb_draw_funcs_t@@PEAXPEAUhb_draw_state_t@@MMMM1@Z 00000001800848d0 f   hb-paint-extents.obj
 0001:00083aa0       ?hb_paint_extents_paint_color@@YAXPEAUhb_paint_funcs_t@@PEAXHI1@Z 0000000180084aa0 f   hb-paint-extents.obj
 0001:00083aa0       ?hb_paint_extents_paint_linear_gradient@@YAXPEAUhb_paint_funcs_t@@PEAXPEAUhb_color_line_t@@MMMMMM1@Z 0000000180084aa0 f   hb-paint-extents.obj
 0001:00083aa0       ?hb_paint_extents_paint_radial_gradient@@YAXPEAUhb_paint_funcs_t@@PEAXPEAUhb_color_line_t@@MMMMMM1@Z 0000000180084aa0 f   hb-paint-extents.obj
 0001:00083aa0       ?hb_paint_extents_paint_sweep_gradient@@YAXPEAUhb_paint_funcs_t@@PEAXPEAUhb_color_line_t@@MMMM1@Z 0000000180084aa0 f   hb-paint-extents.obj
 0001:00083ab0       ?hb_paint_extents_paint_image@@YAHPEAUhb_paint_funcs_t@@PEAXPEAUhb_blob_t@@IIIMPEAUhb_glyph_extents_t@@1@Z 0000000180084ab0 f   hb-paint-extents.obj
 0001:00083bb0       ?hb_paint_extents_pop_clip@@YAXPEAUhb_paint_funcs_t@@PEAX1@Z 0000000180084bb0 f   hb-paint-extents.obj
 0001:00083bc0       ?hb_paint_extents_pop_group@@YAXPEAUhb_paint_funcs_t@@PEAXW4hb_paint_composite_mode_t@@1@Z 0000000180084bc0 f   hb-paint-extents.obj
 0001:00083bd0       ?hb_paint_extents_pop_transform@@YAXPEAUhb_paint_funcs_t@@PEAX1@Z 0000000180084bd0 f   hb-paint-extents.obj
 0001:00083be0       ?hb_paint_extents_push_clip_glyph@@YAXPEAUhb_paint_funcs_t@@PEAXIPEAUhb_font_t@@1@Z 0000000180084be0 f   hb-paint-extents.obj
 0001:00083d80       ?hb_paint_extents_push_clip_rectangle@@YAXPEAUhb_paint_funcs_t@@PEAXMMMM1@Z 0000000180084d80 f   hb-paint-extents.obj
 0001:00083e40       ?hb_paint_extents_push_group@@YAXPEAUhb_paint_funcs_t@@PEAX1@Z 0000000180084e40 f   hb-paint-extents.obj
 0001:00083e70       ?hb_paint_extents_push_transform@@YAXPEAUhb_paint_funcs_t@@PEAXMMMMMM1@Z 0000000180084e70 f   hb-paint-extents.obj
 0001:00084170       $LN69                      0000000180085170     hb-paint-extents.obj
 0001:00085840       ?_hb_shape_plan_execute_internal@@YA_NPEAUhb_shape_plan_t@@PEAUhb_font_t@@PEAUhb_buffer_t@@PEBUhb_feature_t@@I@Z 0000000180086840 f   hb-shape-plan.obj
 0001:00086930       ?hb_ucd_combining_class@@YA?AW4hb_unicode_combining_class_t@@PEAUhb_unicode_funcs_t@@IPEAX@Z 0000000180087930 f   hb-ucd.obj
 0001:000869b0       ?hb_ucd_compose@@YAHPEAUhb_unicode_funcs_t@@IIPEAIPEAX@Z 00000001800879b0 f   hb-ucd.obj
 0001:00086b60       ?hb_ucd_decompose@@YAHPEAUhb_unicode_funcs_t@@IPEAI1PEAX@Z 0000000180087b60 f   hb-ucd.obj
 0001:00086d10       ?hb_ucd_general_category@@YA?AW4hb_unicode_general_category_t@@PEAUhb_unicode_funcs_t@@IPEAX@Z 0000000180087d10 f   hb-ucd.obj
 0001:00086da0       ?hb_ucd_mirroring@@YAIPEAUhb_unicode_funcs_t@@IPEAX@Z 0000000180087da0 f   hb-ucd.obj
 0001:00086e30       ?hb_ucd_script@@YA?AW4hb_script_t@@PEAUhb_unicode_funcs_t@@IPEAX@Z 0000000180087e30 f   hb-ucd.obj
 0001:00086fd0       ?hb_unicode_general_category_nil@@YA?AW4hb_unicode_general_category_t@@PEAUhb_unicode_funcs_t@@IPEAX@Z 0000000180087fd0 f   hb-unicode.obj
 0001:00086fe0       ?hb_unicode_mirroring_nil@@YAIPEAUhb_unicode_funcs_t@@IPEAX@Z 0000000180087fe0 f   hb-unicode.obj
 0001:00086ff0       ?hb_unicode_script_nil@@YA?AW4hb_script_t@@PEAUhb_unicode_funcs_t@@IPEAX@Z 0000000180087ff0 f   hb-unicode.obj
 0001:000883f0       initFontIDs                00000001800893f0 f   sunFont.obj
 0001:00088ce0       $$000000                   0000000180089ce0     MSVCRT:amdsecgs.obj
 0001:00088ec8       capture_current_context    0000000180089ec8 f   MSVCRT:gs_report.obj
 0001:00088f38       capture_previous_context   0000000180089f38 f   MSVCRT:gs_report.obj
 0001:00088fb0       $$000000                   0000000180089fb0     MSVCRT:chkstk.obj
 0001:00089010       $$000000                   000000018008a010     MSVCRT:svml_sfloorf4_dispatch.obj
 0001:00089024       ?dllmain_crt_dispatch@@YAHQEAUHINSTANCE__@@KQEAX@Z 000000018008a024 f   MSVCRT:dll_dllmain.obj
 0001:00089074       ?dllmain_crt_process_attach@@YAHQEAUHINSTANCE__@@QEAX@Z 000000018008a074 f   MSVCRT:dll_dllmain.obj
 0001:0008918c       ?dllmain_crt_process_detach@@YAH_N@Z 000000018008a18c f   MSVCRT:dll_dllmain.obj
 0001:00089210       ?dllmain_dispatch@@YAHQEAUHINSTANCE__@@KQEAX@Z 000000018008a210 f   MSVCRT:dll_dllmain.obj
 0001:00089530       $$000000                   000000018008a530     MSVCRT:svml_sfloorf4_sse2.obj
 0001:00089580       $$000000                   000000018008a580     MSVCRT:svml_sfloorf4_sse4.obj
 0001:00089c70       $$000000                   000000018008ac70     MSVCRT:guard_dispatch.obj
 0001:00089c90       $$000000                   000000018008ac90     MSVCRT:guard_xfg_dispatch.obj
 0001:00089ca6       ?fin$0@?0??dllmain_crt_process_attach@@YAHQEAUHINSTANCE__@@QEAX@Z@4HA 000000018008aca6 f   MSVCRT:dll_dllmain.obj
 0001:00089cbd       ?fin$0@?0??dllmain_crt_process_detach@@YAH_N@Z@4HA 000000018008acbd f   MSVCRT:dll_dllmain.obj
 0001:00089cd6       ?fin$1@?0??dllmain_crt_process_detach@@YAH_N@Z@4HA 000000018008acd6 f   MSVCRT:dll_dllmain.obj
 0001:00089cea       ?filt$0@?0??dllmain_dispatch@@YAHQEAUHINSTANCE__@@KQEAX@Z@4HA 000000018008acea f   MSVCRT:dll_dllmain.obj
 0001:00089d20       __scrt_is_nonwritable_in_current_image$filt$0 000000018008ad20 f   MSVCRT:utility.obj
 0002:00000630       FONTKEY_NT                 000000018008b630     fontpath.obj
 0002:00000668       ?TTSUFFIX@?1??RegistryToBaseTTNameW@@9@9 000000018008b668     fontpath.obj
 0002:00000680       ?OTSUFFIX@?1??RegistryToBaseTTNameW@@9@9 000000018008b680     fontpath.obj
 0002:000007e0       ?outline_funcs@?1??addToGP@@9@9 000000018008b7e0     freetypeScaler.obj
 0002:000008d0       ?table_tags@@3QBIB         000000018008b8d0     gsubgpos-context.obj
 0002:000008d8       ?hb_identity@@3U<unnamed-type-hb_identity>@@B 000000018008b8d8     gsubgpos-context.obj
 0002:000008d9       ?hb_ridentity@@3U<unnamed-type-hb_ridentity>@@B 000000018008b8d9     gsubgpos-context.obj
 0002:000008e0       ?table_tags@@3QBIB         000000018008b8e0     hb-aat-layout.obj
 0002:000008f0       ?feature_mappings@@3QBUhb_aat_feature_mapping_t@@B 000000018008b8f0     hb-aat-layout.obj
 0002:00000fb0       ?table_tags@@3QBIB         000000018008bfb0     hb-aat-map.obj
 0002:00001040       ?_deserialize_json_trans_keys@@3QBEB 000000018008c040     hb-buffer-serialize.obj
 0002:000010b8       ?_deserialize_json_key_spans@@3QBDB 000000018008c0b8     hb-buffer-serialize.obj
 0002:00001100       ?_deserialize_json_index_offsets@@3QBFB 000000018008c100     hb-buffer-serialize.obj
 0002:00001180       ?_deserialize_json_indicies@@3QBDB 000000018008c180     hb-buffer-serialize.obj
 0002:00001eb0       ?_deserialize_json_trans_targs@@3QBDB 000000018008ceb0     hb-buffer-serialize.obj
 0002:00001f20       ?_deserialize_json_trans_actions@@3QBDB 000000018008cf20     hb-buffer-serialize.obj
 0002:00001f88       ?_deserialize_text_glyphs_trans_keys@@3QBEB 000000018008cf88     hb-buffer-serialize.obj
 0002:00001fc0       ?_deserialize_text_glyphs_key_spans@@3QBDB 000000018008cfc0     hb-buffer-serialize.obj
 0002:00001fe0       ?_deserialize_text_glyphs_index_offsets@@3QBFB 000000018008cfe0     hb-buffer-serialize.obj
 0002:00002020       ?_deserialize_text_glyphs_indicies@@3QBDB 000000018008d020     hb-buffer-serialize.obj
 0002:000026f0       ?_deserialize_text_glyphs_trans_targs@@3QBDB 000000018008d6f0     hb-buffer-serialize.obj
 0002:00002730       ?_deserialize_text_glyphs_trans_actions@@3QBDB 000000018008d730     hb-buffer-serialize.obj
 0002:00002770       ?_deserialize_text_glyphs_eof_actions@@3QBDB 000000018008d770     hb-buffer-serialize.obj
 0002:00002790       ?_deserialize_text_unicode_trans_keys@@3QBEB 000000018008d790     hb-buffer-serialize.obj
 0002:000027a8       ?_deserialize_text_unicode_key_spans@@3QBDB 000000018008d7a8     hb-buffer-serialize.obj
 0002:000027b8       ?_deserialize_text_unicode_index_offsets@@3QBFB 000000018008d7b8     hb-buffer-serialize.obj
 0002:000027d0       ?_deserialize_text_unicode_indicies@@3QBDB 000000018008d7d0     hb-buffer-serialize.obj
 0002:00002a98       ?_deserialize_text_unicode_trans_targs@@3QBDB 000000018008da98     hb-buffer-serialize.obj
 0002:00002aa8       ?_deserialize_text_unicode_trans_actions@@3QBDB 000000018008daa8     hb-buffer-serialize.obj
 0002:00002ab8       ?_deserialize_text_unicode_eof_actions@@3QBDB 000000018008dab8     hb-buffer-serialize.obj
 0002:00002c00       ?table_tags@@3QBIB         000000018008dc00     hb-buffer.obj
 0002:00002c18       ?direction_strings@@3QAY03$$CBDA 000000018008dc18     hb-common.obj
 0002:00002c30       ?canon_map@@3QBDB          000000018008dc30     hb-common.obj
 0002:00002d50       ?_hb_ms_language_map@@3QBUhb_ot_language_map_t@@B 000000018008dd50     hb-common.obj
 0002:000034d0       ?_hb_mac_language_map@@3QBUhb_ot_language_map_t@@B 000000018008e4d0     hb-common.obj
 0002:00003878       ?table_tags@@3QBIB         000000018008e878     hb-common.obj
 0002:00003a50       ?_hb_os2_unicode_ranges@OT@@3QBUOS2Range@1@B 000000018008ea50     hb-common.obj
 0002:00004250       ?_hb_arabic_u8@@3QBEB      000000018008f250     hb-common.obj
 0002:00004420       ?_hb_arabic_u16@@3QBGB     000000018008f420     hb-common.obj
 0002:00004a28       ?table_tags@@3QBIB         000000018008fa28     hb-face-builder.obj
 0002:00004a30       ?hb_identity@@3U<unnamed-type-hb_identity>@@B 000000018008fa30     hb-face-builder.obj
 0002:00004a31       ?hb_ridentity@@3U<unnamed-type-hb_ridentity>@@B 000000018008fa31     hb-face-builder.obj
 0002:00004a90       ?_hb_os2_unicode_ranges@OT@@3QBUOS2Range@1@B 000000018008fa90     hb-face.obj
 0002:00005280       ?table_tags@@3QBIB         0000000180090280     hb-face.obj
 0002:00005290       ?_hb_arabic_u8@@3QBEB      0000000180090290     hb-face.obj
 0002:00005460       ?_hb_arabic_u16@@3QBGB     0000000180090460     hb-face.obj
 0002:00005a00       ?table_tags@@3QBIB         0000000180090a00     hb-fallback-shape.obj
 0002:00005a08       ?table_tags@@3QBIB         0000000180090a08     hb-font.obj
 0002:00005a30       ?hb_identity@@3U<unnamed-type-hb_identity>@@B 0000000180090a30     hb-map.obj
 0002:00005a31       ?hb_ridentity@@3U<unnamed-type-hb_ridentity>@@B 0000000180090a31     hb-map.obj
 0002:00005a40       ?_double_parser_trans_keys@@3QBEB 0000000180090a40     hb-number.obj
 0002:00005a58       ?_double_parser_key_spans@@3QBDB 0000000180090a58     hb-number.obj
 0002:00005a68       ?_double_parser_index_offsets@@3QBEB 0000000180090a68     hb-number.obj
 0002:00005a80       ?_double_parser_indicies@@3QBDB 0000000180090a80     hb-number.obj
 0002:00005b40       ?_double_parser_trans_targs@@3QBDB 0000000180090b40     hb-number.obj
 0002:00005b50       ?_double_parser_trans_actions@@3QBDB 0000000180090b50     hb-number.obj
 0002:00005b60       ?_powers_of_10@?1??_pow10@@YANI@Z@4QBNB 0000000180090b60     hb-number.obj
 0002:00005be0       ?standard_encoding_to_code@@3QBEB 0000000180090be0     hb-ot-cff1-table.obj
 0002:00005c80       ?expert_encoding_to_code@@3QBEB 0000000180090c80     hb-ot-cff1-table.obj
 0002:00005e00       ?expert_charset_to_sid@@3QBGB 0000000180090e00     hb-ot-cff1-table.obj
 0002:00005f50       ?expert_subset_charset_to_sid@@3QBGB 0000000180090f50     hb-ot-cff1-table.obj
 0002:00006000       ?expert_charset_sid_to_gid@@3QBUsid_to_gid_t@@B 0000000180091000     hb-ot-cff1-table.obj
 0002:000062a0       ?expert_subset_charset_sid_to_gid@@3QBUsid_to_gid_t@@B 00000001800912a0     hb-ot-cff1-table.obj
 0002:00006400       ?standard_encoding_to_sid@@3QBEB 0000000180091400     hb-ot-cff1-table.obj
 0002:00006500       ?table_tags@@3QBIB         0000000180091500     hb-ot-cff1-table.obj
 0002:00006510       ?cff1_std_strings_msgstr@@3Tcff1_std_strings_msgstr_t@@B 0000000180091510     hb-ot-cff1-table.obj
 0002:00007290       ?cff1_std_strings_msgidx@@3QBIB 0000000180092290     hb-ot-cff1-table.obj
 0002:000078e0       ?table_tags@@3QBIB         00000001800928e0     hb-ot-cff2-table.obj
 0002:000078e8       ?table_tags@@3QBIB         00000001800928e8     hb-ot-color.obj
 0002:000078f0       ?format1_names_msgstr@@3Tformat1_names_msgstr_t@@B 00000001800928f0     hb-ot-face.obj
 0002:00008030       ?format1_names_msgidx@@3QBIB 0000000180093030     hb-ot-face.obj
 0002:00008440       ?cff1_std_strings_msgstr@@3Tcff1_std_strings_msgstr_t@@B 0000000180093440     hb-ot-face.obj
 0002:000091c0       ?cff1_std_strings_msgidx@@3QBIB 00000001800941c0     hb-ot-face.obj
 0002:000097e0       ?_hb_arabic_u8@@3QBEB      00000001800947e0     hb-ot-face.obj
 0002:000099b0       ?_hb_arabic_u16@@3QBGB     00000001800949b0     hb-ot-face.obj
 0002:00009f50       ?_hb_os2_unicode_ranges@OT@@3QBUOS2Range@1@B 0000000180094f50     hb-ot-face.obj
 0002:0000a740       ?table_tags@@3QBIB         0000000180095740     hb-ot-face.obj
 0002:0000a750       ?format1_names_msgstr@@3Tformat1_names_msgstr_t@@B 0000000180095750     hb-ot-font.obj
 0002:0000ae90       ?format1_names_msgidx@@3QBIB 0000000180095e90     hb-ot-font.obj
 0002:0000b2a0       ?cff1_std_strings_msgstr@@3Tcff1_std_strings_msgstr_t@@B 00000001800962a0     hb-ot-font.obj
 0002:0000c020       ?cff1_std_strings_msgidx@@3QBIB 0000000180097020     hb-ot-font.obj
 0002:0000c640       ?table_tags@@3QBIB         0000000180097640     hb-ot-font.obj
 0002:0000c650       ?_hb_arabic_u8@@3QBEB      0000000180097650     hb-ot-font.obj
 0002:0000c820       ?_hb_arabic_u16@@3QBGB     0000000180097820     hb-ot-font.obj
 0002:0000cdc0       ?_hb_os2_unicode_ranges@OT@@3QBUOS2Range@1@B 0000000180097dc0     hb-ot-font.obj
 0002:0000d600       ?_hb_os2_unicode_ranges@OT@@3QBUOS2Range@1@B 0000000180098600     hb-ot-layout.obj
 0002:0000ddf0       ?table_tags@@3QBIB         0000000180098df0     hb-ot-layout.obj
 0002:0000ddf8       ?hb_identity@@3U<unnamed-type-hb_identity>@@B 0000000180098df8     hb-ot-layout.obj
 0002:0000ddf9       ?hb_first@@3U<unnamed-type-hb_first>@@B 0000000180098df9     hb-ot-layout.obj
 0002:0000ddfa       ?hb_second@@3U<unnamed-type-hb_second>@@B 0000000180098dfa     hb-ot-layout.obj
 0002:0000ddfb       ?hb_add@@3U<unnamed-type-hb_add>@@B 0000000180098dfb     hb-ot-layout.obj
 0002:0000e350       ?table_tags@@3QBIB         0000000180099350     hb-ot-map.obj
 0002:0000e358       ?table_tags@@3QBIB         0000000180099358     hb-ot-math.obj
 0002:0000e360       ?table_tags@@3QBIB         0000000180099360     hb-ot-meta.obj
 0002:0000e370       ?_hb_os2_unicode_ranges@OT@@3QBUOS2Range@1@B 0000000180099370     hb-ot-metrics.obj
 0002:0000eb60       ?table_tags@@3QBIB         0000000180099b60     hb-ot-metrics.obj
 0002:0000eb70       ?format1_names_msgstr@@3Tformat1_names_msgstr_t@@B 0000000180099b70     hb-ot-metrics.obj
 0002:0000f2b0       ?format1_names_msgidx@@3QBIB 000000018009a2b0     hb-ot-metrics.obj
 0002:0000f6c0       ?table_tags@@3QBIB         000000018009a6c0     hb-ot-name.obj
 0002:0000f6c8       ?table_tags@@3QBIB         000000018009a6c8     hb-ot-shape-fallback.obj
 0002:0000f730       ?table_tags@@3QBIB         000000018009a730     hb-ot-shape-normalize.obj
 0002:0000f758       ?table_tags@@3QBIB         000000018009a758     hb-ot-shape.obj
 0002:0000f760       ?common_features@@3QBUhb_ot_map_feature_t@@B 000000018009a760     hb-ot-shape.obj
 0002:0000f798       ?horizontal_features@@3QBUhb_ot_map_feature_t@@B 000000018009a798     hb-ot-shape.obj
 0002:0000f850       ?arabic_fallback_features@@3QBIB 000000018009a850     hb-ot-shaper-arabic.obj
 0002:0000f870       ?arabic_win1256_gsub_lookups@@3U0@B 000000018009a870     hb-ot-shaper-arabic.obj
 0002:0000fa08       ?table_tags@@3QBIB         000000018009aa08     hb-ot-shaper-arabic.obj
 0002:0000fa70       ?joining_table@@3QBEB      000000018009aa70     hb-ot-shaper-arabic.obj
 0002:00010010       ?shaping_table@@3QAY03$$CBGA 000000018009b010     hb-ot-shaper-arabic.obj
 0002:000105b0       ?ligature_table@@3QBUligature_set_t@@B 000000018009b5b0     hb-ot-shaper-arabic.obj
 0002:000109c8       ?ligature_mark_table@@3QBUligature_mark_set_t@@B 000000018009b9c8     hb-ot-shaper-arabic.obj
 0002:000109e0       ?ligature_3_table@@3QBUligature_3_set_t@@B 000000018009b9e0     hb-ot-shaper-arabic.obj
 0002:000109f8       ?arabic_features@@3QBIB    000000018009b9f8     hb-ot-shaper-arabic.obj
 0002:00010a20       ?arabic_state_table@@3QAY05$$CBUarabic_state_table_entry@@A 000000018009ba20     hb-ot-shaper-arabic.obj
 0002:00010ac8       ?hb_first@@3U<unnamed-type-hb_first>@@B 000000018009bac8     hb-ot-shaper-arabic.obj
 0002:00010ac9       ?hb_second@@3U<unnamed-type-hb_second>@@B 000000018009bac9     hb-ot-shaper-arabic.obj
 0002:00010aca       ?hb_add@@3U<unnamed-type-hb_add>@@B 000000018009baca     hb-ot-shaper-arabic.obj
 0002:00010b10       ?table_tags@@3QBIB         000000018009bb10     hb-ot-shaper-default.obj
 0002:00010be0       ?table_tags@@3QBIB         000000018009bbe0     hb-ot-shaper-hangul.obj
 0002:00010c50       ?hangul_features@@3QBIB    000000018009bc50     hb-ot-shaper-hangul.obj
 0002:00010c60       ?table_tags@@3QBIB         000000018009bc60     hb-ot-shaper-hebrew.obj
 0002:00010cd0       ?sDageshForms@?1??compose_hebrew@@YA_NPEBUhb_ot_shape_normalize_context_t@@IIPEAI@Z@4QBIB 000000018009bcd0     hb-ot-shaper-hebrew.obj
 0002:00010d40       ?table_tags@@3QBIB         000000018009bd40     hb-ot-shaper-indic-table.obj
 0002:00010d50       ?_indic_syllable_machine_trans_keys@@3QBEB 000000018009bd50     hb-ot-shaper-indic-table.obj
 0002:00010e70       ?_indic_syllable_machine_key_spans@@3QBDB 000000018009be70     hb-ot-shaper-indic-table.obj
 0002:00010f00       ?_indic_syllable_machine_index_offsets@@3QBFB 000000018009bf00     hb-ot-shaper-indic-table.obj
 0002:00011020       ?_indic_syllable_machine_indicies@@3QBEB 000000018009c020     hb-ot-shaper-indic-table.obj
 0002:000115c0       ?_indic_syllable_machine_trans_targs@@3QBEB 000000018009c5c0     hb-ot-shaper-indic-table.obj
 0002:00011660       ?_indic_syllable_machine_trans_actions@@3QBDB 000000018009c660     hb-ot-shaper-indic-table.obj
 0002:00011700       ?_indic_syllable_machine_to_state_actions@@3QBDB 000000018009c700     hb-ot-shaper-indic-table.obj
 0002:00011790       ?_indic_syllable_machine_from_state_actions@@3QBDB 000000018009c790     hb-ot-shaper-indic-table.obj
 0002:00011820       ?_indic_syllable_machine_eof_trans@@3QBFB 000000018009c820     hb-ot-shaper-indic-table.obj
 0002:00011940       ?_khmer_syllable_machine_trans_keys@@3QBEB 000000018009c940     hb-ot-shaper-indic-table.obj
 0002:00011998       ?_khmer_syllable_machine_key_spans@@3QBDB 000000018009c998     hb-ot-shaper-indic-table.obj
 0002:000119d0       ?_khmer_syllable_machine_index_offsets@@3QBFB 000000018009c9d0     hb-ot-shaper-indic-table.obj
 0002:00011a30       ?_khmer_syllable_machine_indicies@@3QBDB 000000018009ca30     hb-ot-shaper-indic-table.obj
 0002:00011df0       ?_khmer_syllable_machine_trans_targs@@3QBDB 000000018009cdf0     hb-ot-shaper-indic-table.obj
 0002:00011e28       ?_khmer_syllable_machine_trans_actions@@3QBDB 000000018009ce28     hb-ot-shaper-indic-table.obj
 0002:00011e60       ?_khmer_syllable_machine_to_state_actions@@3QBDB 000000018009ce60     hb-ot-shaper-indic-table.obj
 0002:00011e90       ?_khmer_syllable_machine_from_state_actions@@3QBDB 000000018009ce90     hb-ot-shaper-indic-table.obj
 0002:00011ec0       ?_khmer_syllable_machine_eof_trans@@3QBFB 000000018009cec0     hb-ot-shaper-indic-table.obj
 0002:00011f20       ?_myanmar_syllable_machine_trans_keys@@3QBEB 000000018009cf20     hb-ot-shaper-indic-table.obj
 0002:00011f90       ?_myanmar_syllable_machine_key_spans@@3QBDB 000000018009cf90     hb-ot-shaper-indic-table.obj
 0002:00011fd0       ?_myanmar_syllable_machine_index_offsets@@3QBFB 000000018009cfd0     hb-ot-shaper-indic-table.obj
 0002:00012040       ?_myanmar_syllable_machine_indicies@@3QBDB 000000018009d040     hb-ot-shaper-indic-table.obj
 0002:00012810       ?_myanmar_syllable_machine_trans_targs@@3QBDB 000000018009d810     hb-ot-shaper-indic-table.obj
 0002:00012850       ?_myanmar_syllable_machine_trans_actions@@3QBDB 000000018009d850     hb-ot-shaper-indic-table.obj
 0002:00012890       ?_myanmar_syllable_machine_to_state_actions@@3QBDB 000000018009d890     hb-ot-shaper-indic-table.obj
 0002:000128c8       ?_myanmar_syllable_machine_from_state_actions@@3QBDB 000000018009d8c8     hb-ot-shaper-indic-table.obj
 0002:00012900       ?_myanmar_syllable_machine_eof_trans@@3QBFB 000000018009d900     hb-ot-shaper-indic-table.obj
 0002:00012970       ?indic_table@@3QBGB        000000018009d970     hb-ot-shaper-indic-table.obj
 0002:000136f0       ?table_tags@@3QBIB         000000018009e6f0     hb-ot-shaper-indic.obj
 0002:00013760       ?_indic_syllable_machine_trans_keys@@3QBEB 000000018009e760     hb-ot-shaper-indic.obj
 0002:00013880       ?_indic_syllable_machine_key_spans@@3QBDB 000000018009e880     hb-ot-shaper-indic.obj
 0002:00013910       ?_indic_syllable_machine_index_offsets@@3QBFB 000000018009e910     hb-ot-shaper-indic.obj
 0002:00013a30       ?_indic_syllable_machine_indicies@@3QBEB 000000018009ea30     hb-ot-shaper-indic.obj
 0002:00013fd0       ?_indic_syllable_machine_trans_targs@@3QBEB 000000018009efd0     hb-ot-shaper-indic.obj
 0002:00014070       ?_indic_syllable_machine_trans_actions@@3QBDB 000000018009f070     hb-ot-shaper-indic.obj
 0002:00014110       ?_indic_syllable_machine_to_state_actions@@3QBDB 000000018009f110     hb-ot-shaper-indic.obj
 0002:000141a0       ?_indic_syllable_machine_from_state_actions@@3QBDB 000000018009f1a0     hb-ot-shaper-indic.obj
 0002:00014230       ?_indic_syllable_machine_eof_trans@@3QBFB 000000018009f230     hb-ot-shaper-indic.obj
 0002:00014350       ?indic_configs@@3QBUindic_config_t@@B 000000018009f350     hb-ot-shaper-indic.obj
 0002:00014440       ?indic_features@@3QBUhb_ot_map_feature_t@@B 000000018009f440     hb-ot-shaper-indic.obj
 0002:00014550       ?table_tags@@3QBIB         000000018009f550     hb-ot-shaper-khmer.obj
 0002:000145c0       ?_khmer_syllable_machine_trans_keys@@3QBEB 000000018009f5c0     hb-ot-shaper-khmer.obj
 0002:00014618       ?_khmer_syllable_machine_key_spans@@3QBDB 000000018009f618     hb-ot-shaper-khmer.obj
 0002:00014650       ?_khmer_syllable_machine_index_offsets@@3QBFB 000000018009f650     hb-ot-shaper-khmer.obj
 0002:000146b0       ?_khmer_syllable_machine_indicies@@3QBDB 000000018009f6b0     hb-ot-shaper-khmer.obj
 0002:00014a70       ?_khmer_syllable_machine_trans_targs@@3QBDB 000000018009fa70     hb-ot-shaper-khmer.obj
 0002:00014aa8       ?_khmer_syllable_machine_trans_actions@@3QBDB 000000018009faa8     hb-ot-shaper-khmer.obj
 0002:00014ae0       ?_khmer_syllable_machine_to_state_actions@@3QBDB 000000018009fae0     hb-ot-shaper-khmer.obj
 0002:00014b10       ?_khmer_syllable_machine_from_state_actions@@3QBDB 000000018009fb10     hb-ot-shaper-khmer.obj
 0002:00014b40       ?_khmer_syllable_machine_eof_trans@@3QBFB 000000018009fb40     hb-ot-shaper-khmer.obj
 0002:00014ba0       ?khmer_features@@3QBUhb_ot_map_feature_t@@B 000000018009fba0     hb-ot-shaper-khmer.obj
 0002:00014c20       ?table_tags@@3QBIB         000000018009fc20     hb-ot-shaper-myanmar.obj
 0002:00014cf0       ?_myanmar_syllable_machine_trans_keys@@3QBEB 000000018009fcf0     hb-ot-shaper-myanmar.obj
 0002:00014d60       ?_myanmar_syllable_machine_key_spans@@3QBDB 000000018009fd60     hb-ot-shaper-myanmar.obj
 0002:00014da0       ?_myanmar_syllable_machine_index_offsets@@3QBFB 000000018009fda0     hb-ot-shaper-myanmar.obj
 0002:00014e10       ?_myanmar_syllable_machine_indicies@@3QBDB 000000018009fe10     hb-ot-shaper-myanmar.obj
 0002:000155e0       ?_myanmar_syllable_machine_trans_targs@@3QBDB 00000001800a05e0     hb-ot-shaper-myanmar.obj
 0002:00015620       ?_myanmar_syllable_machine_trans_actions@@3QBDB 00000001800a0620     hb-ot-shaper-myanmar.obj
 0002:00015660       ?_myanmar_syllable_machine_to_state_actions@@3QBDB 00000001800a0660     hb-ot-shaper-myanmar.obj
 0002:00015698       ?_myanmar_syllable_machine_from_state_actions@@3QBDB 00000001800a0698     hb-ot-shaper-myanmar.obj
 0002:000156d0       ?_myanmar_syllable_machine_eof_trans@@3QBFB 00000001800a06d0     hb-ot-shaper-myanmar.obj
 0002:00015740       ?myanmar_basic_features@@3QBIB 00000001800a0740     hb-ot-shaper-myanmar.obj
 0002:00015750       ?myanmar_other_features@@3QBIB 00000001800a0750     hb-ot-shaper-myanmar.obj
 0002:00015798       ?table_tags@@3QBIB         00000001800a0798     hb-ot-shaper-syllabic.obj
 0002:000157a0       ?table_tags@@3QBIB         00000001800a07a0     hb-ot-shaper-thai.obj
 0002:00015810       ?thai_above_state_machine@@3QAY02$$CBUthai_above_state_machine_edge_t@@A 00000001800a0810     hb-ot-shaper-thai.obj
 0002:00015870       ?thai_below_state_machine@@3QAY02$$CBUthai_below_state_machine_edge_t@@A 00000001800a0870     hb-ot-shaper-thai.obj
 0002:000158b8       ?SD_mappings@?1??thai_pua_shape@@YAIIW4thai_action_t@@PEAUhb_font_t@@@Z@4QBUthai_pua_mapping_t@?1??1@YAII01@Z@B 00000001800a08b8     hb-ot-shaper-thai.obj
 0002:000158f0       ?SDL_mappings@?1??thai_pua_shape@@YAIIW4thai_action_t@@PEAUhb_font_t@@@Z@4QBUthai_pua_mapping_t@?1??1@YAII01@Z@B 00000001800a08f0     hb-ot-shaper-thai.obj
 0002:00015920       ?SL_mappings@?1??thai_pua_shape@@YAIIW4thai_action_t@@PEAUhb_font_t@@@Z@4QBUthai_pua_mapping_t@?1??1@YAII01@Z@B 00000001800a0920     hb-ot-shaper-thai.obj
 0002:00015970       ?RD_mappings@?1??thai_pua_shape@@YAIIW4thai_action_t@@PEAUhb_font_t@@@Z@4QBUthai_pua_mapping_t@?1??1@YAII01@Z@B 00000001800a0970     hb-ot-shaper-thai.obj
 0002:00015990       ?hb_use_u8@@3QBEB          00000001800a0990     hb-ot-shaper-use.obj
 0002:000165e0       ?hb_use_u16@@3QBGB         00000001800a15e0     hb-ot-shaper-use.obj
 0002:00016c00       ?use_basic_features@@3QBIB 00000001800a1c00     hb-ot-shaper-use.obj
 0002:00016c20       ?use_topographical_features@@3QBIB 00000001800a1c20     hb-ot-shaper-use.obj
 0002:00016c30       ?use_other_features@@3QBIB 00000001800a1c30     hb-ot-shaper-use.obj
 0002:00016c48       ?table_tags@@3QBIB         00000001800a1c48     hb-ot-shaper-use.obj
 0002:00016cb0       ?_use_syllable_machine_trans_keys@@3QBEB 00000001800a1cb0     hb-ot-shaper-use.obj
 0002:00016db0       ?_use_syllable_machine_key_spans@@3QBDB 00000001800a1db0     hb-ot-shaper-use.obj
 0002:00016e30       ?_use_syllable_machine_index_offsets@@3QBFB 00000001800a1e30     hb-ot-shaper-use.obj
 0002:00016f30       ?_use_syllable_machine_indicies@@3QBEB 00000001800a1f30     hb-ot-shaper-use.obj
 0002:000180c0       ?_use_syllable_machine_trans_targs@@3QBDB 00000001800a30c0     hb-ot-shaper-use.obj
 0002:00018150       ?_use_syllable_machine_trans_actions@@3QBDB 00000001800a3150     hb-ot-shaper-use.obj
 0002:000181e0       ?_use_syllable_machine_to_state_actions@@3QBDB 00000001800a31e0     hb-ot-shaper-use.obj
 0002:00018260       ?_use_syllable_machine_from_state_actions@@3QBDB 00000001800a3260     hb-ot-shaper-use.obj
 0002:000182e0       ?_use_syllable_machine_eof_trans@@3QBFB 00000001800a32e0     hb-ot-shaper-use.obj
 0002:000183dc       ?hb_identity@@3U<unnamed-type-hb_identity>@@B 00000001800a33dc     hb-ot-shaper-use.obj
 0002:000183dd       ?hb_second@@3U<unnamed-type-hb_second>@@B 00000001800a33dd     hb-ot-shaper-use.obj
 0002:00018410       ?table_tags@@3QBIB         00000001800a3410     hb-ot-shaper-vowel-constraints.obj
 0002:00018420       ?ot_languages2@@3QBULangTag@@B 00000001800a3420     hb-ot-tag.obj
 0002:00018a80       ?ot_languages3@@3QBULangTag@@B 00000001800a3a80     hb-ot-tag.obj
 0002:0001b5a8       ?table_tags@@3QBIB         00000001800a65a8     hb-ot-var.obj
 0002:0001b5b8       ?table_tags@@3QBIB         00000001800a65b8     hb-paint.obj
 0002:0001b5c0       ?table_tags@@3QBIB         00000001800a65c0     hb-shape-plan.obj
 0002:0001b8b0       ?table_tags@@3QBIB         00000001800a68b0     hb-shape.obj
 0002:0001b8b8       ?nil_shaper_list@@3QBQEBDB 00000001800a68b8     hb-shape.obj
 0002:0001b8c0       ?_hb_all_shapers@@3QBUhb_shaper_entry_t@@B 00000001800a68c0     hb-shaper.obj
 0002:0001b900       ?table_tags@@3QBIB         00000001800a6900     hb-static.obj
 0002:0001b910       ?_hb_os2_unicode_ranges@OT@@3QBUOS2Range@1@B 00000001800a6910     hb-static.obj
 0002:0001c100       ?_hb_arabic_u8@@3QBEB      00000001800a7100     hb-static.obj
 0002:0001c2d0       ?_hb_arabic_u16@@3QBGB     00000001800a72d0     hb-static.obj
 0002:0001c870       ?_hb_os2_unicode_ranges@OT@@3QBUOS2Range@1@B 00000001800a7870     hb-style.obj
 0002:0001d060       ?table_tags@@3QBIB         00000001800a8060     hb-style.obj
 0002:0001d070       ?format1_names_msgstr@@3Tformat1_names_msgstr_t@@B 00000001800a8070     hb-style.obj
 0002:0001d7b0       ?format1_names_msgidx@@3QBIB 00000001800a87b0     hb-style.obj
 0002:0001dbc0       ?table_tags@@3QBIB         00000001800a8bc0     hb-subset-cff-common.obj
 0002:0001dbd0       ?table_tags@@3QBIB         00000001800a8bd0     hb-subset-cff1.obj
 0002:0001dbe0       ?cff1_std_strings_msgstr@@3Tcff1_std_strings_msgstr_t@@B 00000001800a8be0     hb-subset-cff1.obj
 0002:0001e960       ?cff1_std_strings_msgidx@@3QBIB 00000001800a9960     hb-subset-cff1.obj
 0002:0001ef80       ?hb_identity@@3U<unnamed-type-hb_identity>@@B 00000001800a9f80     hb-subset-cff1.obj
 0002:0001ef81       ?hb_iter@@3U<unnamed-type-hb_iter>@@B 00000001800a9f81     hb-subset-cff1.obj
 0002:0001ef82       ?hb_len@@3U<unnamed-type-hb_len>@@B 00000001800a9f82     hb-subset-cff1.obj
 0002:0001ef88       ?table_tags@@3QBIB         00000001800a9f88     hb-subset-cff2.obj
 0002:0001ef90       ?hb_identity@@3U<unnamed-type-hb_identity>@@B 00000001800a9f90     hb-subset-cff2.obj
 0002:0001ef91       ?hb_iter@@3U<unnamed-type-hb_iter>@@B 00000001800a9f91     hb-subset-cff2.obj
 0002:0001ef92       ?hb_len@@3U<unnamed-type-hb_len>@@B 00000001800a9f92     hb-subset-cff2.obj
 0002:0001ef98       ?table_tags@@3QBIB         00000001800a9f98     hb-subset-input.obj
 0002:0001efa0       ?table_tags@@3QBIB         00000001800a9fa0     hb-subset-plan.obj
 0002:0001efb0       ?cff1_std_strings_msgstr@@3Tcff1_std_strings_msgstr_t@@B 00000001800a9fb0     hb-subset-plan.obj
 0002:0001fd30       ?cff1_std_strings_msgidx@@3QBIB 00000001800aad30     hb-subset-plan.obj
 0002:00020350       ?_hb_arabic_u8@@3QBEB      00000001800ab350     hb-subset-plan.obj
 0002:00020520       ?_hb_arabic_u16@@3QBGB     00000001800ab520     hb-subset-plan.obj
 0002:00020ac0       ?_hb_os2_unicode_ranges@OT@@3QBUOS2Range@1@B 00000001800abac0     hb-subset-plan.obj
 0002:000212ac       ?hb_identity@@3U<unnamed-type-hb_identity>@@B 00000001800ac2ac     hb-subset-plan.obj
 0002:000212ad       ?hb_hash@@3U<unnamed-type-hb_hash>@@B 00000001800ac2ad     hb-subset-plan.obj
 0002:000212ae       ?hb_first@@3U<unnamed-type-hb_first>@@B 00000001800ac2ae     hb-subset-plan.obj
 0002:000212af       ?hb_second@@3U<unnamed-type-hb_second>@@B 00000001800ac2af     hb-subset-plan.obj
 0002:000212b0       ?hb_add@@3U<unnamed-type-hb_add>@@B 00000001800ac2b0     hb-subset-plan.obj
 0002:000212b1       ?hb_iter@@3U<unnamed-type-hb_iter>@@B 00000001800ac2b1     hb-subset-plan.obj
 0002:000212c0       ?_hb_os2_unicode_ranges@OT@@3QBUOS2Range@1@B 00000001800ac2c0     hb-subset.obj
 0002:00021ab0       ?format1_names_msgstr@@3Tformat1_names_msgstr_t@@B 00000001800acab0     hb-subset.obj
 0002:000221f0       ?format1_names_msgidx@@3QBIB 00000001800ad1f0     hb-subset.obj
 0002:00022600       ?table_tags@@3QBIB         00000001800ad600     hb-subset.obj
 0002:00022610       ?cff1_std_strings_msgstr@@3Tcff1_std_strings_msgstr_t@@B 00000001800ad610     hb-subset.obj
 0002:00023390       ?cff1_std_strings_msgidx@@3QBIB 00000001800ae390     hb-subset.obj
 0002:000239b0       ?_hb_arabic_u8@@3QBEB      00000001800ae9b0     hb-subset.obj
 0002:00023b80       ?_hb_arabic_u16@@3QBGB     00000001800aeb80     hb-subset.obj
 0002:00024120       ?hb_identity@@3U<unnamed-type-hb_identity>@@B 00000001800af120     hb-subset.obj
 0002:00024121       ?hb_ridentity@@3U<unnamed-type-hb_ridentity>@@B 00000001800af121     hb-subset.obj
 0002:00024122       ?hb_invoke@@3U<unnamed-type-hb_invoke>@@B 00000001800af122     hb-subset.obj
 0002:00024123       ?hb_first@@3U<unnamed-type-hb_first>@@B 00000001800af123     hb-subset.obj
 0002:00024124       ?hb_second@@3U<unnamed-type-hb_second>@@B 00000001800af124     hb-subset.obj
 0002:00024125       ?hb_max@@3U<unnamed-type-hb_max>@@B 00000001800af125     hb-subset.obj
 0002:00024126       ?hb_add@@3U<unnamed-type-hb_add>@@B 00000001800af126     hb-subset.obj
 0002:00024127       ?hb_iter@@3U<unnamed-type-hb_iter>@@B 00000001800af127     hb-subset.obj
 0002:00024130       ?_hb_ucd_sc_map@@3QBW4hb_script_t@@B 00000001800af130     hb-ucd.obj
 0002:000243d0       ?_hb_ucd_dm1_p0_map@@3QBGB 00000001800af3d0     hb-ucd.obj
 0002:00024a50       ?_hb_ucd_dm1_p2_map@@3QBGB 00000001800afa50     hb-ucd.obj
 0002:00024b30       ?_hb_ucd_dm2_u32_map@@3QBIB 00000001800afb30     hb-ucd.obj
 0002:00025530       ?_hb_ucd_dm2_u64_map@@3QB_KB 00000001800b0530     hb-ucd.obj
 0002:00026150       ?_hb_ucd_u8@@3QBEB         00000001800b1150     hb-ucd.obj
 0002:0002a720       ?_hb_ucd_u16@@3QBGB        00000001800b5720     hb-ucd.obj
 0002:0002eff0       ?_hb_ucd_i16@@3QBFB        00000001800b9ff0     hb-ucd.obj
 0002:0002f280       ?_hb_emoji_u8@@3QBEB       00000001800ba280     hb-unicode.obj
 0002:0002f7c8       GS_ExceptionPointers       00000001800ba7c8     MSVCRT:gs_report.obj
 0002:00030668       $unwind$Glyph_Lock         00000001800bb668     ColorGlyphSurfaceData.obj
 0002:00030678       $unwind$Java_sun_font_ColorGlyphSurfaceData_initOps 00000001800bb678     ColorGlyphSurfaceData.obj
 0002:00030678       $unwind$Java_sun_font_ColorGlyphSurfaceData_setCurrentGlyph 00000001800bb678     ColorGlyphSurfaceData.obj
 0002:00030678       $unwind$??$dispatch@Uhb_sanitize_context_t@@$$V@?$ChainSubtable@UObsoleteTypes@AAT@@@AAT@@QEBA_NPEAUhb_sanitize_context_t@@@Z 00000001800bb678     hb-aat-layout.obj
 0002:00030678       $unwind$?get_value_or_null@?$Lookup@U?$IntType@I$03@OT@@@AAT@@QEBA?BIII@Z 00000001800bb678     hb-aat-layout.obj
 0002:00030678       $unwind$?mark_set_covers@GDEF@OT@@QEBA_NII@Z 00000001800bb678     hb-aat-layout.obj
 0002:00030678       $unwind$hb_blob_create_sub_blob 00000001800bb678     hb-blob.obj
 0002:00030678       $unwind$?reset@hb_buffer_t@@QEAAXXZ 00000001800bb678     hb-buffer.obj
 0002:00030678       $unwind$hb_buffer_create   00000001800bb678     hb-buffer.obj
 0002:00030678       $unwind$hb_buffer_get_glyph_positions 00000001800bb678     hb-buffer.obj
 0002:00030678       $unwind$?load_num_glyphs@hb_face_t@@AEBAIXZ 00000001800bb678     hb-common.obj
 0002:00030678       $unwind$?load_upem@hb_face_t@@AEBAIXZ 00000001800bb678     hb-common.obj
 0002:00030678       $unwind$hb_language_matches 00000001800bb678     hb-common.obj
 0002:00030678       $unwind$??$hb_object_create@Uhb_face_t@@$$V@@YAPEAUhb_face_t@@XZ 00000001800bb678     hb-face.obj
 0002:00030678       $unwind$?cleanupFontInfo@@YAXPEAX@Z 00000001800bb678     hb-jdk-font.obj
 0002:00030678       $unwind$?process_op@?$opset_t@Unumber_t@CFF@@@CFF@@SAXIAEAU?$interp_env_t@Unumber_t@CFF@@@2@@Z 00000001800bb678     hb-ot-cff1-table.obj
 0002:00030678       $unwind$?process_op@?$cs_opset_t@Unumber_t@CFF@@Ucff2_cs_opset_extents_t@@U?$cff2_cs_interp_env_t@Unumber_t@CFF@@@2@Ucff2_extents_param_t@@Ucff2_path_procs_extents_t@@@CFF@@SAXIAEAU?$cff2_cs_interp_env_t@Unumber_t@CFF@@@2@AEAUcff2_extents_param_t@@@Z 00000001800bb678     hb-ot-cff2-table.obj
 0002:00030678       $unwind$??$sanitize@$$V@Paint@OT@@QEBA_NPEAUhb_sanitize_context_t@@@Z 00000001800bb678     hb-ot-color.obj
 0002:00030678       $unwind$?_hb_ot_font_destroy@@YAXPEAX@Z 00000001800bb678     hb-ot-font.obj
 0002:00030678       $unwind$?process_op@dict_opset_t@CFF@@SAXIAEAU?$interp_env_t@Unumber_t@CFF@@@2@@Z 00000001800bb678     hb-ot-font.obj
 0002:00030678       $unwind$?recurse@hb_paint_context_t@OT@@QEAAXAEBUPaint@2@@Z 00000001800bb678     hb-ot-font.obj
 0002:00030678       $unwind$??$dispatch@Uhb_accelerate_subtables_context_t@OT@@$$V@Context@OT@@QEBA?AUhb_empty_t@@PEAUhb_accelerate_subtables_context_t@1@@Z 00000001800bb678     hb-ot-layout.obj
 0002:00030678       $unwind$??$dispatch@Uhb_accelerate_subtables_context_t@OT@@$$V@PosLookupSubTable@GPOS_impl@Layout@OT@@QEBA?AUhb_empty_t@@PEAUhb_accelerate_subtables_context_t@3@I@Z 00000001800bb678     hb-ot-layout.obj
 0002:00030678       $unwind$??$dispatch@Uhb_accelerate_subtables_context_t@OT@@$$V@SubstLookupSubTable@GSUB_impl@Layout@OT@@QEBA?AUhb_empty_t@@PEAUhb_accelerate_subtables_context_t@3@I@Z 00000001800bb678     hb-ot-layout.obj
 0002:00030678       $unwind$?match_class@OT@@YA_NAEAUhb_glyph_info_t@@IPEBX@Z 00000001800bb678     hb-ot-layout.obj
 0002:00030678       $unwind$?fini@hb_ot_shape_plan_t@@QEAAXXZ 00000001800bb678     hb-ot-shape.obj
 0002:00030678       $unwind$??$push@UCoverage@Common@Layout@OT@@@hb_serialize_context_t@@QEAAPEAUCoverage@Common@Layout@OT@@XZ 00000001800bb678     hb-ot-shaper-arabic.obj
 0002:00030678       $unwind$?override_features_indic@@YAXPEAUhb_ot_shape_planner_t@@@Z 00000001800bb678     hb-ot-shaper-indic.obj
 0002:00030678       $unwind$?setup_masks_indic@@YAXPEBUhb_ot_shape_plan_t@@PEAUhb_buffer_t@@PEAUhb_font_t@@@Z 00000001800bb678     hb-ot-shaper-indic.obj
 0002:00030678       $unwind$?override_features_khmer@@YAXPEAUhb_ot_shape_planner_t@@@Z 00000001800bb678     hb-ot-shaper-khmer.obj
 0002:00030678       $unwind$?setup_masks_khmer@@YAXPEBUhb_ot_shape_plan_t@@PEAUhb_buffer_t@@PEAUhb_font_t@@@Z 00000001800bb678     hb-ot-shaper-khmer.obj
 0002:00030678       $unwind$?setup_masks_myanmar@@YAXPEBUhb_ot_shape_plan_t@@PEAUhb_buffer_t@@PEAUhb_font_t@@@Z 00000001800bb678     hb-ot-shaper-myanmar.obj
 0002:00030678       $unwind$?data_destroy_use@@YAXPEAX@Z 00000001800bb678     hb-ot-shaper-use.obj
 0002:00030678       $unwind$?setup_masks_use@@YAXPEBUhb_ot_shape_plan_t@@PEAUhb_buffer_t@@PEAUhb_font_t@@@Z 00000001800bb678     hb-ot-shaper-use.obj
 0002:00030678       $unwind$?_hb_preprocess_text_vowel_constraints@@YAXPEBUhb_ot_shape_plan_t@@PEAUhb_buffer_t@@PEAUhb_font_t@@@Z 00000001800bb678     hb-ot-shaper-vowel-constraints.obj
 0002:00030678       $unwind$?_output_with_dotted_circle@@YAXPEAUhb_buffer_t@@@Z 00000001800bb678     hb-ot-shaper-vowel-constraints.obj
 0002:00030678       $unwind$?hb_draw_extents_cubic_to@@YAXPEAUhb_draw_funcs_t@@PEAXPEAUhb_draw_state_t@@MMMMMM1@Z 00000001800bb678     hb-paint-extents.obj
 0002:00030678       $unwind$?hb_draw_extents_quadratic_to@@YAXPEAUhb_draw_funcs_t@@PEAXPEAUhb_draw_state_t@@MMMM1@Z 00000001800bb678     hb-paint-extents.obj
 0002:00030678       $unwind$getSunFontIDs      00000001800bb678     sunFont.obj
 0002:00030678       $unwind$initFontIDs        00000001800bb678     sunFont.obj
 0002:00030678       $unwind$__raise_securityfailure 00000001800bb678     MSVCRT:gs_report.obj
 0002:00030678       $unwind$__scrt_initialize_crt 00000001800bb678     MSVCRT:utility.obj
 0002:00030678       $unwind$__scrt_initialize_onexit_tables 00000001800bb678     MSVCRT:utility.obj
 0002:00030678       $unwind$__scrt_release_startup_lock 00000001800bb678     MSVCRT:utility.obj
 0002:00030678       $unwind$__scrt_uninitialize_crt 00000001800bb678     MSVCRT:utility.obj
 0002:00030680       $unwind$RefineBounds       00000001800bb680     DrawGlyphList.obj
 0002:00030690       $chain$0$RefineBounds      00000001800bb690     DrawGlyphList.obj
 0002:000306a4       $chain$2$RefineBounds      00000001800bb6a4     DrawGlyphList.obj
 0002:000306bc       $chain$3$RefineBounds      00000001800bb6bc     DrawGlyphList.obj
 0002:000306cc       $chain$4$RefineBounds      00000001800bb6cc     DrawGlyphList.obj
 0002:000306dc       $unwind$setupBlitVector    00000001800bb6dc     DrawGlyphList.obj
 0002:000306fc       $chain$0$setupBlitVector   00000001800bb6fc     DrawGlyphList.obj
 0002:00030710       $chain$1$setupBlitVector   00000001800bb710     DrawGlyphList.obj
 0002:00030724       $chain$2$setupBlitVector   00000001800bb724     DrawGlyphList.obj
 0002:00030734       $chain$3$setupBlitVector   00000001800bb734     DrawGlyphList.obj
 0002:00030744       $unwind$setupLCDBlitVector 00000001800bb744     DrawGlyphList.obj
 0002:00030768       $chain$5$setupLCDBlitVector 00000001800bb768     DrawGlyphList.obj
 0002:00030790       $chain$6$setupLCDBlitVector 00000001800bb790     DrawGlyphList.obj
 0002:000307a0       $unwind$Java_sun_java2d_loops_DrawGlyphListAA_DrawGlyphListAA 00000001800bb7a0     DrawGlyphList.obj
 0002:000307a0       $unwind$Java_sun_java2d_loops_DrawGlyphList_DrawGlyphList 00000001800bb7a0     DrawGlyphList.obj
 0002:000307b4       $chain$0$Java_sun_java2d_loops_DrawGlyphListAA_DrawGlyphListAA 00000001800bb7b4     DrawGlyphList.obj
 0002:000307b4       $chain$0$Java_sun_java2d_loops_DrawGlyphList_DrawGlyphList 00000001800bb7b4     DrawGlyphList.obj
 0002:000307c8       $chain$1$Java_sun_java2d_loops_DrawGlyphListAA_DrawGlyphListAA 00000001800bb7c8     DrawGlyphList.obj
 0002:000307c8       $chain$1$Java_sun_java2d_loops_DrawGlyphList_DrawGlyphList 00000001800bb7c8     DrawGlyphList.obj
 0002:000307dc       $chain$2$Java_sun_java2d_loops_DrawGlyphListAA_DrawGlyphListAA 00000001800bb7dc     DrawGlyphList.obj
 0002:000307dc       $chain$2$Java_sun_java2d_loops_DrawGlyphList_DrawGlyphList 00000001800bb7dc     DrawGlyphList.obj
 0002:000307ec       $chain$3$Java_sun_java2d_loops_DrawGlyphListAA_DrawGlyphListAA 00000001800bb7ec     DrawGlyphList.obj
 0002:000307ec       $chain$3$Java_sun_java2d_loops_DrawGlyphList_DrawGlyphList 00000001800bb7ec     DrawGlyphList.obj
 0002:000307fc       $unwind$drawGlyphList      00000001800bb7fc     DrawGlyphList.obj
 0002:0003081c       $unwind$drawGlyphListLCD   00000001800bb81c     DrawGlyphList.obj
 0002:00030838       $chain$1$drawGlyphListLCD  00000001800bb838     DrawGlyphList.obj
 0002:00030850       $chain$2$drawGlyphListLCD  00000001800bb850     DrawGlyphList.obj
 0002:00030860       $unwind$Java_sun_java2d_loops_DrawGlyphListLCD_DrawGlyphListLCD 00000001800bb860     DrawGlyphList.obj
 0002:00030870       $chain$0$Java_sun_java2d_loops_DrawGlyphListLCD_DrawGlyphListLCD 00000001800bb870     DrawGlyphList.obj
 0002:00030884       $chain$2$Java_sun_java2d_loops_DrawGlyphListLCD_DrawGlyphListLCD 00000001800bb884     DrawGlyphList.obj
 0002:0003089c       $chain$3$Java_sun_java2d_loops_DrawGlyphListLCD_DrawGlyphListLCD 00000001800bb89c     DrawGlyphList.obj
 0002:000308ac       $chain$4$Java_sun_java2d_loops_DrawGlyphListLCD_DrawGlyphListLCD 00000001800bb8ac     DrawGlyphList.obj
 0002:000308bc       $unwind$initLUT            00000001800bb8bc     DrawGlyphList.obj
 0002:000308e0       $unwind$initLCDGammaTables 00000001800bb8e0     DrawGlyphList.obj
 0002:000308e0       $unwind$??$check_range@U?$IntType@E$00@OT@@@hb_sanitize_context_t@@QEBA_NPEBU?$IntType@E$00@OT@@II@Z 00000001800bb8e0     hb-aat-layout.obj
 0002:000308e0       $unwind$hb_aat_layout_has_positioning 00000001800bb8e0     hb-aat-layout.obj
 0002:000308e0       $unwind$hb_aat_layout_has_tracking 00000001800bb8e0     hb-aat-layout.obj
 0002:000308e0       $unwind$hb_tag_from_string 00000001800bb8e0     hb-common.obj
 0002:000308e0       $unwind$hb_draw_funcs_create 00000001800bb8e0     hb-draw.obj
 0002:000308e0       $unwind$hb_face_reference_table 00000001800bb8e0     hb-face.obj
 0002:000308e0       $unwind$?has_func@hb_font_t@@QEAA_NI@Z 00000001800bb8e0     hb-font.obj
 0002:000308e0       $unwind$hb_font_funcs_create 00000001800bb8e0     hb-font.obj
 0002:000308e0       $unwind$??$check_array@U?$IntType@E$00@OT@@@hb_sanitize_context_t@@QEBA_NPEBU?$IntType@E$00@OT@@II@Z 00000001800bb8e0     hb-ot-font.obj
 0002:000308e0       $unwind$??$dispatch@Uhb_would_apply_context_t@OT@@$$V@SubstLookupSubTable@GSUB_impl@Layout@OT@@QEBA_NPEAUhb_would_apply_context_t@3@I@Z 00000001800bb8e0     hb-ot-layout.obj
 0002:000308e0       $unwind$?get_gsubgpos_table@@YAAEBUGSUBGPOS@OT@@PEAUhb_face_t@@I@Z 00000001800bb8e0     hb-ot-layout.obj
 0002:000308e0       $unwind$?hb_ot_layout_has_cross_kerning@@YA_NPEAUhb_face_t@@@Z 00000001800bb8e0     hb-ot-layout.obj
 0002:000308e0       $unwind$?hb_ot_layout_has_kerning@@YA_NPEAUhb_face_t@@@Z 00000001800bb8e0     hb-ot-layout.obj
 0002:000308e0       $unwind$?hb_ot_layout_has_machine_kerning@@YA_NPEAUhb_face_t@@@Z 00000001800bb8e0     hb-ot-layout.obj
 0002:000308e0       $unwind$?match_coverage@OT@@YA_NAEAUhb_glyph_info_t@@IPEBX@Z 00000001800bb8e0     hb-ot-layout.obj
 0002:000308e0       $unwind$hb_ot_layout_has_glyph_classes 00000001800bb8e0     hb-ot-layout.obj
 0002:000308e0       $unwind$hb_ot_layout_has_positioning 00000001800bb8e0     hb-ot-layout.obj
 0002:000308e0       $unwind$hb_ot_layout_has_substitution 00000001800bb8e0     hb-ot-layout.obj
 0002:000308e0       $unwind$hb_ot_layout_table_get_lookup_count 00000001800bb8e0     hb-ot-layout.obj
 0002:000308e0       $unwind$?hb_outline_recording_pen_get_funcs@@YAPEAUhb_draw_funcs_t@@XZ 00000001800bb8e0     hb-outline.obj
 0002:000308e0       $unwind$?hb_paint_extents_get_funcs@@YAPEAUhb_paint_funcs_t@@XZ 00000001800bb8e0     hb-paint-extents.obj
 0002:000308e0       $unwind$?pop_group@hb_paint_extents_context_t@@QEAAXW4hb_paint_composite_mode_t@@@Z 00000001800bb8e0     hb-paint-extents.obj
 0002:000308e0       $unwind$hb_paint_funcs_create 00000001800bb8e0     hb-paint.obj
 0002:000308e0       $unwind$hb_ucd_get_unicode_funcs 00000001800bb8e0     hb-ucd.obj
 0002:000308e0       $unwind$Java_sun_font_FileFontStrike_initNative 00000001800bb8e0     lcdglyph.obj
 0002:000308e0       $unwind$Java_sun_font_NullFontScaler_getNullScalerContext 00000001800bb8e0     sunFont.obj
 0002:000308e0       $unwind$__scrt_initialize_default_local_stdio_options 00000001800bb8e0     MSVCRT:default_local_stdio_options.obj
 0002:000308e0       $unwind$?dllmain_crt_dispatch@@YAHQEAUHINSTANCE__@@KQEAX@Z 00000001800bb8e0     MSVCRT:dll_dllmain.obj
 0002:000308e0       $unwind$DllMain            00000001800bb8e0     MSVCRT:dll_dllmain_stub.obj
 0002:000308e0       $unwind$__report_rangecheckfailure 00000001800bb8e0     MSVCRT:gs_report.obj
 0002:000308e0       $unwind$__GSHandlerCheck   00000001800bb8e0     MSVCRT:gshandler.obj
 0002:000308e0       $unwind$__scrt_acquire_startup_lock 00000001800bb8e0     MSVCRT:utility.obj
 0002:000308e0       $unwind$__scrt_dllmain_after_initialize_c 00000001800bb8e0     MSVCRT:utility.obj
 0002:000308e0       $unwind$__scrt_dllmain_before_initialize_c 00000001800bb8e0     MSVCRT:utility.obj
 0002:000308e0       $unwind$__scrt_dllmain_crt_thread_attach 00000001800bb8e0     MSVCRT:utility.obj
 0002:000308e0       $unwind$__scrt_dllmain_crt_thread_detach 00000001800bb8e0     MSVCRT:utility.obj
 0002:000308e0       $unwind$__scrt_dllmain_uninitialize_c 00000001800bb8e0     MSVCRT:utility.obj
 0002:000308e0       $unwind$__scrt_dllmain_uninitialize_critical 00000001800bb8e0     MSVCRT:utility.obj
 0002:000308e8       $unwind$storeGVData        00000001800bb8e8     HBShaper.obj
 0002:00030918       $unwind$euclidianDistance  00000001800bb918     HBShaper.obj
 0002:00030924       $unwind$Java_sun_font_SunLayoutEngine_shape 00000001800bb924     HBShaper.obj
 0002:0003093c       $chain$0$Java_sun_font_SunLayoutEngine_shape 00000001800bb93c     HBShaper.obj
 0002:00030950       $chain$1$Java_sun_font_SunLayoutEngine_shape 00000001800bb950     HBShaper.obj
 0002:00030950       $chain$3$Java_sun_font_SunLayoutEngine_shape 00000001800bb950     HBShaper.obj
 0002:00030960       $chain$2$Java_sun_font_SunLayoutEngine_shape 00000001800bb960     HBShaper.obj
 0002:00030974       $unwind$Java_sun_awt_Win32FontManager_populateFontFileNameMap0 00000001800bb974     fontpath.obj
 0002:00030990       $chain$0$Java_sun_awt_Win32FontManager_populateFontFileNameMap0 00000001800bb990     fontpath.obj
 0002:000309a4       $chain$1$Java_sun_awt_Win32FontManager_populateFontFileNameMap0 00000001800bb9a4     fontpath.obj
 0002:000309b4       $unwind$Java_sun_awt_Win32FontManager_getFontPath 00000001800bb9b4     fontpath.obj
 0002:000309d8       $unwind$EnumFontFacesInFamilyProcW 00000001800bb9d8     fontpath.obj
 0002:000309f8       $unwind$EnumFamilyNamesW   00000001800bb9f8     fontpath.obj
 0002:00030a18       $unwind$registerFontW      00000001800bba18     fontpath.obj
 0002:00030a34       $unwind$populateFontFileNameFromRegistryKey 00000001800bba34     fontpath.obj
 0002:00030a4c       $chain$0$populateFontFileNameFromRegistryKey 00000001800bba4c     fontpath.obj
 0002:00030a60       $chain$1$populateFontFileNameFromRegistryKey 00000001800bba60     fontpath.obj
 0002:00030a74       $chain$4$populateFontFileNameFromRegistryKey 00000001800bba74     fontpath.obj
 0002:00030a90       $chain$5$populateFontFileNameFromRegistryKey 00000001800bba90     fontpath.obj
 0002:00030aa0       $chain$6$populateFontFileNameFromRegistryKey 00000001800bbaa0     fontpath.obj
 0002:00030ab0       $chain$7$populateFontFileNameFromRegistryKey 00000001800bbab0     fontpath.obj
 0002:00030ac0       $unwind$Java_sun_font_FreetypeFontScaler_initIDs 00000001800bbac0     freetypeScaler.obj
 0002:00030ac0       $unwind$?hb_font_get_glyph_h_kerning_default@@YAHPEAUhb_font_t@@PEAXII1@Z 00000001800bbac0     hb-font.obj
 0002:00030ac0       $unwind$?hb_font_get_glyph_v_kerning_default@@YAHPEAUhb_font_t@@PEAXII1@Z 00000001800bbac0     hb-font.obj
 0002:00030ac0       $unwind$hb_font_get_glyph  00000001800bbac0     hb-font.obj
 0002:00030ac0       $unwind$?get_x_delta@Device@OT@@QEBAHPEAUhb_font_t@@AEBUVariationStore@2@PEAM@Z 00000001800bbac0     hb-ot-layout.obj
 0002:00030ac0       $unwind$?get_y_delta@Device@OT@@QEBAHPEAUhb_font_t@@AEBUVariationStore@2@PEAM@Z 00000001800bbac0     hb-ot-layout.obj
 0002:00030ac0       $unwind$?hb_ot_substitute_post@@YAXPEBUhb_ot_shape_context_t@@@Z 00000001800bbac0     hb-ot-shape.obj
 0002:00030ac0       $unwind$?hb_outline_recording_pen_cubic_to@@YAXPEAUhb_draw_funcs_t@@PEAXPEAUhb_draw_state_t@@MMMMMM1@Z 00000001800bbac0     hb-outline.obj
 0002:00030ac0       $unwind$?hb_outline_recording_pen_quadratic_to@@YAXPEAUhb_draw_funcs_t@@PEAXPEAUhb_draw_state_t@@MMMM1@Z 00000001800bbac0     hb-outline.obj
 0002:00030ac0       $unwind$hb_shape_plan_execute 00000001800bbac0     hb-shape-plan.obj
 0002:00030ac8       $unwind$Java_sun_font_FreetypeFontScaler_initNativeScaler 00000001800bbac8     freetypeScaler.obj
 0002:00030ae0       $chain$2$Java_sun_font_FreetypeFontScaler_initNativeScaler 00000001800bbae0     freetypeScaler.obj
 0002:00030af4       $chain$3$Java_sun_font_FreetypeFontScaler_initNativeScaler 00000001800bbaf4     freetypeScaler.obj
 0002:00030b04       $unwind$Java_sun_font_FreetypeFontScaler_getFontMetricsNative 00000001800bbb04     freetypeScaler.obj
 0002:00030b20       $chain$9$Java_sun_font_FreetypeFontScaler_getFontMetricsNative 00000001800bbb20     freetypeScaler.obj
 0002:00030b58       $chain$10$Java_sun_font_FreetypeFontScaler_getFontMetricsNative 00000001800bbb58     freetypeScaler.obj
 0002:00030b68       $unwind$Java_sun_font_FreetypeFontScaler_getGlyphAdvanceNative 00000001800bbb68     freetypeScaler.obj
 0002:00030b68       $unwind$?hb_font_draw_glyph_default@@YAXPEAUhb_font_t@@PEAXIPEAUhb_draw_funcs_t@@11@Z 00000001800bbb68     hb-font.obj
 0002:00030b68       $unwind$?hhcurveto@?$path_procs_t@Ucff2_path_procs_extents_t@@U?$cff2_cs_interp_env_t@Unumber_t@CFF@@@CFF@@Ucff2_extents_param_t@@@CFF@@SAXAEAU?$cff2_cs_interp_env_t@Unumber_t@CFF@@@2@AEAUcff2_extents_param_t@@@Z 00000001800bbb68     hb-ot-cff2-table.obj
 0002:00030b68       $unwind$?vvcurveto@?$path_procs_t@Ucff2_path_procs_extents_t@@U?$cff2_cs_interp_env_t@Unumber_t@CFF@@@CFF@@Ucff2_extents_param_t@@@CFF@@SAXAEAU?$cff2_cs_interp_env_t@Unumber_t@CFF@@@2@AEAUcff2_extents_param_t@@@Z 00000001800bbb68     hb-ot-cff2-table.obj
 0002:00030b68       $unwind$_hb_ot_shape       00000001800bbb68     hb-ot-shape.obj
 0002:00030b70       $chain$0$Java_sun_font_FreetypeFontScaler_getGlyphAdvanceNative 00000001800bbb70     freetypeScaler.obj
 0002:00030b84       $chain$1$Java_sun_font_FreetypeFontScaler_getGlyphAdvanceNative 00000001800bbb84     freetypeScaler.obj
 0002:00030b94       $unwind$Java_sun_font_FreetypeFontScaler_getGlyphMetricsNative 00000001800bbb94     freetypeScaler.obj
 0002:00030ba0       $unwind$Java_sun_font_FreetypeFontScaler_getGlyphImageNative 00000001800bbba0     freetypeScaler.obj
 0002:00030ba0       $unwind$?rcurveline@?$path_procs_t@Ucff1_path_procs_extents_t@@Ucff1_cs_interp_env_t@CFF@@Ucff1_extents_param_t@@@CFF@@SAXAEAUcff1_cs_interp_env_t@2@AEAUcff1_extents_param_t@@@Z 00000001800bbba0     hb-ot-cff1-table.obj
 0002:00030ba0       $unwind$?rlinecurve@?$path_procs_t@Ucff1_path_procs_extents_t@@Ucff1_cs_interp_env_t@CFF@@Ucff1_extents_param_t@@@CFF@@SAXAEAUcff1_cs_interp_env_t@2@AEAUcff1_extents_param_t@@@Z 00000001800bbba0     hb-ot-cff1-table.obj
 0002:00030ba0       $unwind$?rrcurveto@?$path_procs_t@Ucff1_path_procs_extents_t@@Ucff1_cs_interp_env_t@CFF@@Ucff1_extents_param_t@@@CFF@@SAXAEAUcff1_cs_interp_env_t@2@AEAUcff1_extents_param_t@@@Z 00000001800bbba0     hb-ot-cff1-table.obj
 0002:00030ba0       $unwind$?quadratic_to@hb_draw_session_t@@QEAAXMMMM@Z 00000001800bbba0     hb-ot-font.obj
 0002:00030ba0       $unwind$?end@?$hb_iter_t@U?$hb_map_iter_t@U?$hb_zip_iter_t@U?$hb_sorted_array_t@UHBGlyphID16@OT@@@@U?$hb_array_t@UHBGlyphID16@OT@@@@@@AEBU<unnamed-type-hb_first>@@$00$0A@@@AEAUHBGlyphID16@OT@@@@QEBA?AU?$hb_map_iter_t@U?$hb_zip_iter_t@U?$hb_sorted_array_t@UHBGlyphID16@OT@@@@U?$hb_array_t@UHBGlyphID16@OT@@@@@@AEBU<unnamed-type-hb_first>@@$00$0A@@@XZ 00000001800bbba0     hb-ot-shaper-arabic.obj
 0002:00030ba0       $unwind$?hb_paint_extents_push_group@@YAXPEAUhb_paint_funcs_t@@PEAX1@Z 00000001800bbba0     hb-paint-extents.obj
 0002:00030ba8       $unwind$Java_sun_font_FreetypeFontScaler_getGlyphOutlineBoundsNative 00000001800bbba8     freetypeScaler.obj
 0002:00030ba8       $unwind$?parse_bcd@dict_opset_t@CFF@@SANAEAUbyte_str_ref_t@2@@Z 00000001800bbba8     hb-ot-font.obj
 0002:00030bb8       $unwind$Java_sun_font_FreetypeFontScaler_getGlyphOutlineNative 00000001800bbbb8     freetypeScaler.obj
 0002:00030bc0       $unwind$Java_sun_font_FreetypeFontScaler_getGlyphVectorOutlineNative 00000001800bbbc0     freetypeScaler.obj
 0002:00030bd8       $chain$1$Java_sun_font_FreetypeFontScaler_getGlyphVectorOutlineNative 00000001800bbbd8     freetypeScaler.obj
 0002:00030bec       $chain$4$Java_sun_font_FreetypeFontScaler_getGlyphVectorOutlineNative 00000001800bbbec     freetypeScaler.obj
 0002:00030c08       $chain$5$Java_sun_font_FreetypeFontScaler_getGlyphVectorOutlineNative 00000001800bbc08     freetypeScaler.obj
 0002:00030c18       $chain$6$Java_sun_font_FreetypeFontScaler_getGlyphVectorOutlineNative 00000001800bbc18     freetypeScaler.obj
 0002:00030c28       $unwind$Java_sun_font_FreetypeFontScaler_getGlyphPointNative 00000001800bbc28     freetypeScaler.obj
 0002:00030c38       $unwind$Java_sun_font_FreetypeFontScaler_disposeNativeScaler 00000001800bbc38     freetypeScaler.obj
 0002:00030c38       $unwind$?sanitize@?$Lookup@U?$IntType@G$01@OT@@@AAT@@QEBA_NPEAUhb_sanitize_context_t@@@Z 00000001800bbc38     hb-aat-layout.obj
 0002:00030c38       $unwind$?sanitize@?$Lookup@U?$IntType@I$03@OT@@@AAT@@QEBA_NPEAUhb_sanitize_context_t@@@Z 00000001800bbc38     hb-aat-layout.obj
 0002:00030c38       $unwind$?sanitize@?$Lookup@UHBGlyphID16@OT@@@AAT@@QEBA_NPEAUhb_sanitize_context_t@@@Z 00000001800bbc38     hb-aat-layout.obj
 0002:00030c38       $unwind$?move_to@hb_buffer_t@@QEAA_NI@Z 00000001800bbc38     hb-buffer.obj
 0002:00030c38       $unwind$??$dispatch@Uhb_sanitize_context_t@@$$V@Paint@OT@@QEBA_NPEAUhb_sanitize_context_t@@@Z 00000001800bbc38     hb-ot-color.obj
 0002:00030c44       $unwind$Java_sun_font_FreetypeFontScaler_getGlyphCodeNative 00000001800bbc44     freetypeScaler.obj
 0002:00030c50       $unwind$Java_sun_font_FreetypeFontScaler_getNumGlyphsNative 00000001800bbc50     freetypeScaler.obj
 0002:00030c50       $unwind$invalidateJavaScaler 00000001800bbc50     freetypeScaler.obj
 0002:00030c50       $unwind$??$sanitize@$$V@?$OffsetTo@U?$ArrayOf@UAnchor@AAT@@U?$IntType@I$03@OT@@@OT@@U?$IntType@G$01@2@$0A@@OT@@QEBA_NPEAUhb_sanitize_context_t@@PEBX@Z 00000001800bbc50     hb-aat-layout.obj
 0002:00030c50       $unwind$??$sanitize@$$V@?$OffsetTo@U?$ClassTable@U?$IntType@E$00@OT@@@AAT@@U?$IntType@G$01@OT@@$0A@@OT@@QEBA_NPEAUhb_sanitize_context_t@@PEBX@Z 00000001800bbc50     hb-aat-layout.obj
 0002:00030c50       $unwind$??$sanitize@$$V@?$OffsetTo@U?$Lookup@U?$IntType@G$01@OT@@@AAT@@U?$IntType@I$03@OT@@$0A@@OT@@QEBA_NPEAUhb_sanitize_context_t@@PEBX@Z 00000001800bbc50     hb-aat-layout.obj
 0002:00030c50       $unwind$??$sanitize@$$V@?$OffsetTo@U?$Lookup@U?$IntType@I$03@OT@@@AAT@@U?$IntType@I$03@OT@@$0A@@OT@@QEBA_NPEAUhb_sanitize_context_t@@PEBX@Z 00000001800bbc50     hb-aat-layout.obj
 0002:00030c50       $unwind$??$sanitize@$$V@?$OffsetTo@UClassDef@OT@@U?$IntType@G$01@2@$00@OT@@QEBA_NPEAUhb_sanitize_context_t@@PEBX@Z 00000001800bbc50     hb-aat-layout.obj
 0002:00030c50       $unwind$??$sanitize@$$V@?$OffsetTo@UCoverage@Common@Layout@OT@@U?$IntType@G$01@4@$00@OT@@QEBA_NPEAUhb_sanitize_context_t@@PEBX@Z 00000001800bbc50     hb-aat-layout.obj
 0002:00030c50       $unwind$??$sanitize@$$V@?$OffsetTo@UVariationStore@OT@@U?$IntType@I$03@2@$00@OT@@QEBA_NPEAUhb_sanitize_context_t@@PEBX@Z 00000001800bbc50     hb-aat-layout.obj
 0002:00030c50       $unwind$?next_glyph@hb_buffer_t@@QEAA_NXZ 00000001800bbc50     hb-aat-layout.obj
 0002:00030c50       $unwind$?sanitize@?$KerxSubTableFormat6@UKerxSubTableHeader@AAT@@@AAT@@QEBA_NPEAUhb_sanitize_context_t@@@Z 00000001800bbc50     hb-aat-layout.obj
 0002:00030c50       $unwind$hb_aat_layout_has_substitution 00000001800bbc50     hb-aat-layout.obj
 0002:00030c50       $unwind$?make_room_for@hb_buffer_t@@QEAA_NII@Z 00000001800bbc50     hb-buffer.obj
 0002:00030c50       $unwind$??$sanitize@$$V@?$OffsetTo@UDeltaSetIndexMap@OT@@U?$IntType@I$03@2@$00@OT@@QEBA_NPEAUhb_sanitize_context_t@@PEBX@Z 00000001800bbc50     hb-common.obj
 0002:00030c50       $unwind$??0hb_serialize_context_t@@QEAA@PEAXI@Z 00000001800bbc50     hb-face-builder.obj
 0002:00030c50       $unwind$??$get_glyph_from_symbol@UCmapSubtable@OT@@$1?_hb_arabic_pua_simp_map@@YAII@Z@accelerator_t@cmap@OT@@KA_NPEBXIPEAI@Z 00000001800bbc50     hb-face.obj
 0002:00030c50       $unwind$??$get_glyph_from_symbol@UCmapSubtable@OT@@$1?_hb_arabic_pua_trad_map@@YAII@Z@accelerator_t@cmap@OT@@KA_NPEBXIPEAI@Z 00000001800bbc50     hb-face.obj
 0002:00030c50       $unwind$??$get_glyph_from_symbol@UCmapSubtable@OT@@$1?_hb_symbol_pua_map@2@YAII@Z@accelerator_t@cmap@OT@@KA_NPEBXIPEAI@Z 00000001800bbc50     hb-face.obj
 0002:00030c50       $unwind$?sanitize@OS2@OT@@QEBA_NPEAUhb_sanitize_context_t@@@Z 00000001800bbc50     hb-face.obj
 0002:00030c50       $unwind$hb_jdk_font_create 00000001800bbc50     hb-jdk-font.obj
 0002:00030c50       $unwind$?process_op@?$cs_opset_t@Unumber_t@CFF@@Ucff1_cs_opset_extents_t@@Ucff1_cs_interp_env_t@2@Ucff1_extents_param_t@@Ucff1_path_procs_extents_t@@@CFF@@SAXIAEAUcff1_cs_interp_env_t@2@AEAUcff1_extents_param_t@@@Z 00000001800bbc50     hb-ot-cff1-table.obj
 0002:00030c50       $unwind$??$sanitize@$$V@?$OffsetTo@U?$ColorLine@UNoVariable@OT@@@OT@@U?$IntType@I$02@2@$00@OT@@QEBA_NPEAUhb_sanitize_context_t@@PEBX@Z 00000001800bbc50     hb-ot-color.obj
 0002:00030c50       $unwind$??$sanitize@$$V@?$OffsetTo@U?$ColorLine@UVariable@OT@@@OT@@U?$IntType@I$02@2@$00@OT@@QEBA_NPEAUhb_sanitize_context_t@@PEBX@Z 00000001800bbc50     hb-ot-color.obj
 0002:00030c50       $unwind$??$sanitize@$$V@?$OffsetTo@UPaint@OT@@U?$IntType@I$02@2@$00@OT@@QEBA_NPEAUhb_sanitize_context_t@@PEBX@Z 00000001800bbc50     hb-ot-color.obj
 0002:00030c50       $unwind$??$sanitize@$$V@?$OffsetTo@UPaint@OT@@U?$IntType@I$03@2@$00@OT@@QEBA_NPEAUhb_sanitize_context_t@@PEBX@Z 00000001800bbc50     hb-ot-color.obj
 0002:00030c50       $unwind$?sanitize@SVG@OT@@QEBA_NPEAUhb_sanitize_context_t@@@Z 00000001800bbc50     hb-ot-color.obj
 0002:00030c50       $unwind$??1?$accelerator_templ_t@Ucff1_private_dict_opset_t@CFF@@U?$cff1_private_dict_values_base_t@Udict_val_t@CFF@@@2@@cff1@OT@@QEAA@XZ 00000001800bbc50     hb-ot-face.obj
 0002:00030c50       $unwind$??1?$accelerator_templ_t@Ucff2_private_dict_opset_t@CFF@@U?$cff2_private_dict_values_base_t@Udict_val_t@CFF@@@2@@cff2@OT@@QEAA@XZ 00000001800bbc50     hb-ot-face.obj
 0002:00030c50       $unwind$?_fini@?$accelerator_templ_t@Ucff2_private_dict_opset_t@CFF@@U?$cff2_private_dict_values_base_t@Udict_val_t@CFF@@@2@@cff2@OT@@QEAAXXZ 00000001800bbc50     hb-ot-face.obj
 0002:00030c50       $unwind$?fini@?$accelerator_templ_t@Ucff1_private_dict_opset_t@CFF@@U?$cff1_private_dict_values_base_t@Udict_val_t@CFF@@@2@@cff1@OT@@QEAAXXZ 00000001800bbc50     hb-ot-face.obj
 0002:00030c50       $unwind$?hb_ot_get_glyph_from_name@@YAHPEAUhb_font_t@@PEAXPEBDHPEAI1@Z 00000001800bbc50     hb-ot-font.obj
 0002:00030c50       $unwind$?sanitize@?$CFFIndex@U?$IntType@G$01@OT@@@CFF@@QEBA_NPEAUhb_sanitize_context_t@@@Z 00000001800bbc50     hb-ot-font.obj
 0002:00030c50       $unwind$?sanitize@?$CFFIndex@U?$IntType@I$03@OT@@@CFF@@QEBA_NPEAUhb_sanitize_context_t@@@Z 00000001800bbc50     hb-ot-font.obj
 0002:00030c50       $unwind$?sanitize@Encoding@CFF@@QEBA_NPEAUhb_sanitize_context_t@@@Z 00000001800bbc50     hb-ot-font.obj
 0002:00030c50       $unwind$?sanitize@post@OT@@QEBA_NPEAUhb_sanitize_context_t@@@Z 00000001800bbc50     hb-ot-font.obj
 0002:00030c50       $unwind$??$sanitize@$$V@?$OffsetTo@U?$ClassTable@U?$IntType@G$01@OT@@@AAT@@U?$IntType@G$01@OT@@$0A@@OT@@QEBA_NPEAUhb_sanitize_context_t@@PEBX@Z 00000001800bbc50     hb-ot-layout.obj
 0002:00030c50       $unwind$??$sanitize@$$V@?$OffsetTo@U?$RecordListOf@UFeature@OT@@@OT@@U?$IntType@G$01@2@$00@OT@@QEBA_NPEAUhb_sanitize_context_t@@PEBX@Z 00000001800bbc50     hb-ot-layout.obj
 0002:00030c50       $unwind$??$sanitize@$$V@?$OffsetTo@U?$RuleSet@USmallTypes@Layout@OT@@@OT@@U?$IntType@G$01@2@$00@OT@@QEBA_NPEAUhb_sanitize_context_t@@PEBX@Z 00000001800bbc50     hb-ot-layout.obj
 0002:00030c50       $unwind$??$sanitize@$$V@?$OffsetTo@UAnchor@GPOS_impl@Layout@OT@@U?$IntType@G$01@4@$00@OT@@QEBA_NPEAUhb_sanitize_context_t@@PEBX@Z 00000001800bbc50     hb-ot-layout.obj
 0002:00030c50       $unwind$??$sanitize@$$V@?$OffsetTo@UFeatureVariations@OT@@U?$IntType@I$03@2@$00@OT@@QEBA_NPEAUhb_sanitize_context_t@@PEBX@Z 00000001800bbc50     hb-ot-layout.obj
 0002:00030c50       $unwind$??$extend@ULookup@OT@@$$V@hb_serialize_context_t@@QEAAPEAULookup@OT@@PEAU12@@Z 00000001800bbc50     hb-ot-shaper-arabic.obj
 0002:00030c50       $unwind$??$extend_size@U?$ArrayOf@UHBGlyphID16@OT@@U?$IntType@G$01@2@@OT@@@hb_serialize_context_t@@QEAAPEAU?$ArrayOf@UHBGlyphID16@OT@@U?$IntType@G$01@2@@OT@@PEAU12@_K_N@Z 00000001800bbc50     hb-ot-shaper-arabic.obj
 0002:00030c50       $unwind$??$extend_size@U?$HeadlessArrayOf@UHBGlyphID16@OT@@U?$IntType@G$01@2@@OT@@@hb_serialize_context_t@@QEAAPEAU?$HeadlessArrayOf@UHBGlyphID16@OT@@U?$IntType@G$01@2@@OT@@PEAU12@_K_N@Z 00000001800bbc50     hb-ot-shaper-arabic.obj
 0002:00030c50       $unwind$?setup_masks_arabic@@YAXPEBUhb_ot_shape_plan_t@@PEAUhb_buffer_t@@PEAUhb_font_t@@@Z 00000001800bbc50     hb-ot-shaper-arabic.obj
 0002:00030c50       $unwind$?setup_masks_arabic_plan@@YAXPEBUarabic_shape_plan_t@@PEAUhb_buffer_t@@W4hb_script_t@@@Z 00000001800bbc50     hb-ot-shaper-arabic.obj
 0002:00030c50       $unwind$?collect_features_hangul@@YAXPEAUhb_ot_shape_planner_t@@@Z 00000001800bbc50     hb-ot-shaper-hangul.obj
 0002:00030c50       $unwind$?collect_features_indic@@YAXPEAUhb_ot_shape_planner_t@@@Z 00000001800bbc50     hb-ot-shaper-indic.obj
 0002:00030c50       $unwind$?init@hb_indic_would_substitute_feature_t@@QEAAXPEBUhb_ot_map_t@@I_N@Z 00000001800bbc50     hb-ot-shaper-indic.obj
 0002:00030c50       $unwind$?collect_features_khmer@@YAXPEAUhb_ot_shape_planner_t@@@Z 00000001800bbc50     hb-ot-shaper-khmer.obj
 0002:00030c50       $unwind$?collect_features_use@@YAXPEAUhb_ot_shape_planner_t@@@Z 00000001800bbc50     hb-ot-shaper-use.obj
 0002:00030c50       $unwind$?subtag_matches@@YA_NPEBD00I@Z 00000001800bbc50     hb-ot-tag.obj
 0002:00030c50       $unwind$?hb_outline_recording_pen_close_path@@YAXPEAUhb_draw_funcs_t@@PEAXPEAUhb_draw_state_t@@1@Z 00000001800bbc50     hb-outline.obj
 0002:00030c50       $unwind$_DllMainCRTStartup 00000001800bbc50     MSVCRT:dll_dllmain.obj
 0002:00030c60       $unwind$Java_sun_font_FreetypeFontScaler_createScalerContextNative 00000001800bbc60     freetypeScaler.obj
 0002:00030c78       $unwind$ReadTTFontFileFunc 00000001800bbc78     freetypeScaler.obj
 0002:00030c78       $unwind$?close_path@hb_draw_funcs_t@@QEAAXPEAXAEAUhb_draw_state_t@@@Z 00000001800bbc78     hb-draw.obj
 0002:00030c78       $unwind$?apply@?$ContextFormat1_4@USmallTypes@Layout@OT@@@OT@@QEBA_NPEAUhb_ot_apply_context_t@2@@Z 00000001800bbc78     hb-ot-layout.obj
 0002:00030c78       $unwind$?serialize@Lookup@OT@@QEAA_NPEAUhb_serialize_context_t@@III@Z 00000001800bbc78     hb-ot-shaper-arabic.obj
 0002:00030c90       $unwind$GlyphSlot_Embolden 00000001800bbc90     freetypeScaler.obj
 0002:00030c9c       $chain$0$GlyphSlot_Embolden 00000001800bbc9c     freetypeScaler.obj
 0002:00030cb0       $chain$1$GlyphSlot_Embolden 00000001800bbcb0     freetypeScaler.obj
 0002:00030cc0       $unwind$setupFTContext     00000001800bbcc0     freetypeScaler.obj
 0002:00030cd4       $unwind$getGlyphImageNativeInternal 00000001800bbcd4     freetypeScaler.obj
 0002:00030cf0       $chain$0$getGlyphImageNativeInternal 00000001800bbcf0     freetypeScaler.obj
 0002:00030d04       $chain$1$getGlyphImageNativeInternal 00000001800bbd04     freetypeScaler.obj
 0002:00030d14       $unwind$CopyBW2Grey8       00000001800bbd14     freetypeScaler.obj
 0002:00030d24       $chain$1$CopyBW2Grey8      00000001800bbd24     freetypeScaler.obj
 0002:00030d3c       $chain$2$CopyBW2Grey8      00000001800bbd3c     freetypeScaler.obj
 0002:00030d4c       $unwind$getFTOutline       00000001800bbd4c     freetypeScaler.obj
 0002:00030d60       $unwind$getGlyphGeneralPath 00000001800bbd60     freetypeScaler.obj
 0002:00030d74       $chain$0$getGlyphGeneralPath 00000001800bbd74     freetypeScaler.obj
 0002:00030d88       $chain$1$getGlyphGeneralPath 00000001800bbd88     freetypeScaler.obj
 0002:00030d98       $unwind$?fini@hb_user_data_array_t@@QEAAXXZ 00000001800bbd98     gsubgpos-context.obj
 0002:00030d98       $unwind$?get_glyph@CmapSubtable@OT@@QEBA_NIPEAI@Z 00000001800bbd98     hb-face.obj
 0002:00030d98       $unwind$?process_blend@?$cff2_cs_interp_env_t@Unumber_t@CFF@@@CFF@@QEAAXXZ 00000001800bbd98     hb-ot-cff2-table.obj
 0002:00030d98       $unwind$??$start_serialize@USubstLookup@GSUB_impl@Layout@OT@@@hb_serialize_context_t@@QEAAPEAUSubstLookup@GSUB_impl@Layout@OT@@XZ 00000001800bbd98     hb-ot-shaper-arabic.obj
 0002:00030d98       $unwind$?hb_paint_extents_paint_image@@YAHPEAUhb_paint_funcs_t@@PEAXPEAUhb_blob_t@@IIIMPEAUhb_glyph_extents_t@@1@Z 00000001800bbd98     hb-paint-extents.obj
 0002:00030d98       $unwind$?hb_paint_extents_push_clip_rectangle@@YAXPEAUhb_paint_funcs_t@@PEAXMMMM1@Z 00000001800bbd98     hb-paint-extents.obj
 0002:00030da0       $chain$0$?fini@hb_user_data_array_t@@QEAAXXZ 00000001800bbda0     gsubgpos-context.obj
 0002:00030db4       $chain$1$?fini@hb_user_data_array_t@@QEAAXXZ 00000001800bbdb4     gsubgpos-context.obj
 0002:00030dc4       $unwind$?start_processing@hb_sanitize_context_t@@QEAAXXZ 00000001800bbdc4     hb-aat-layout.obj
 0002:00030dc4       $unwind$?rcurveline@?$path_procs_t@Ucff2_path_procs_extents_t@@U?$cff2_cs_interp_env_t@Unumber_t@CFF@@@CFF@@Ucff2_extents_param_t@@@CFF@@SAXAEAU?$cff2_cs_interp_env_t@Unumber_t@CFF@@@2@AEAUcff2_extents_param_t@@@Z 00000001800bbdc4     hb-ot-cff2-table.obj
 0002:00030dc4       $unwind$?rlinecurve@?$path_procs_t@Ucff2_path_procs_extents_t@@U?$cff2_cs_interp_env_t@Unumber_t@CFF@@@CFF@@Ucff2_extents_param_t@@@CFF@@SAXAEAU?$cff2_cs_interp_env_t@Unumber_t@CFF@@@2@AEAUcff2_extents_param_t@@@Z 00000001800bbdc4     hb-ot-cff2-table.obj
 0002:00030dc4       $unwind$?rrcurveto@?$path_procs_t@Ucff2_path_procs_extents_t@@U?$cff2_cs_interp_env_t@Unumber_t@CFF@@@CFF@@Ucff2_extents_param_t@@@CFF@@SAXAEAU?$cff2_cs_interp_env_t@Unumber_t@CFF@@@2@AEAUcff2_extents_param_t@@@Z 00000001800bbdc4     hb-ot-cff2-table.obj
 0002:00030dcc       $unwind$?end_processing@hb_sanitize_context_t@@QEAAXXZ 00000001800bbdcc     hb-aat-layout.obj
 0002:00030dd8       $unwind$?check_range@hb_sanitize_context_t@@QEBA_NPEBXI@Z 00000001800bbdd8     hb-aat-layout.obj
 0002:00030de0       $unwind$?may_edit@hb_sanitize_context_t@@QEAA_NPEBXI@Z 00000001800bbde0     hb-aat-layout.obj
 0002:00030de8       $unwind$?interpolate_at@TrackData@AAT@@QEBAMIMAEBUTrackTableEntry@2@PEBX@Z 00000001800bbde8     hb-aat-layout.obj
 0002:00030de8       $unwind$?reverse_range@hb_buffer_t@@QEAAXII@Z 00000001800bbde8     hb-aat-layout.obj
 0002:00030de8       $unwind$?get_kerning@?$KerxSubTableFormat0@UKernAATSubTableHeader@OT@@@AAT@@QEBAHIIPEAUhb_aat_apply_context_t@2@@Z 00000001800bbde8     hb-ot-layout.obj
 0002:00030de8       $unwind$?get_kerning@?$KerxSubTableFormat0@UKernOTSubTableHeader@OT@@@AAT@@QEBAHIIPEAUhb_aat_apply_context_t@2@@Z 00000001800bbde8     hb-ot-layout.obj
 0002:00030de8       $unwind$?record_pref_use@@YA_NPEBUhb_ot_shape_plan_t@@PEAUhb_font_t@@PEAUhb_buffer_t@@@Z 00000001800bbde8     hb-ot-shaper-use.obj
 0002:00030df8       $unwind$??$dispatch@UCoverage@Common@Layout@OT@@$$V@hb_sanitize_context_t@@QEAA_NAEBUCoverage@Common@Layout@OT@@@Z 00000001800bbdf8     hb-aat-layout.obj
 0002:00030df8       $unwind$??$dispatch@Uhb_sanitize_context_t@@$$V@KerxSubTable@AAT@@QEBA_NPEAUhb_sanitize_context_t@@@Z 00000001800bbdf8     hb-aat-layout.obj
 0002:00030df8       $unwind$??$sanitize@$$V@?$ArrayOf@U?$IntType@G$01@OT@@U12@@OT@@QEBA_NPEAUhb_sanitize_context_t@@@Z 00000001800bbdf8     hb-aat-layout.obj
 0002:00030df8       $unwind$??$sanitize@$$V@?$ArrayOf@UHBGlyphID16@OT@@U?$IntType@G$01@2@@OT@@QEBA_NPEAUhb_sanitize_context_t@@@Z 00000001800bbdf8     hb-aat-layout.obj
 0002:00030df8       $unwind$?create_cache@VariationStore@OT@@QEBAPEAMXZ 00000001800bbdf8     hb-aat-layout.obj
 0002:00030df8       $unwind$?get_anchor@ankr@AAT@@QEBAAEBUAnchor@2@III@Z 00000001800bbdf8     hb-aat-layout.obj
 0002:00030df8       $unwind$?get_value_or_null@?$Lookup@U?$IntType@G$01@OT@@@AAT@@QEBA?BGII@Z 00000001800bbdf8     hb-aat-layout.obj
 0002:00030df8       $unwind$?may_skip@matcher_t@hb_ot_apply_context_t@OT@@QEBA?AW4may_skip_t@123@PEBU23@AEBUhb_glyph_info_t@@@Z 00000001800bbdf8     hb-aat-layout.obj
 0002:00030df8       $unwind$?replace_glyph@hb_buffer_t@@QEAA_NI@Z 00000001800bbdf8     hb-aat-layout.obj
 0002:00030df8       $unwind$?sanitize@?$ChainSubtable@UObsoleteTypes@AAT@@@AAT@@QEBA_NPEAUhb_sanitize_context_t@@@Z 00000001800bbdf8     hb-aat-layout.obj
 0002:00030df8       $unwind$?sanitize_shallow@?$OffsetTo@U?$UnsizedListOfOffset16To@U?$Lookup@UHBGlyphID16@OT@@@AAT@@U?$IntType@I$03@OT@@$0A@@OT@@U?$IntType@I$03@2@$0A@@OT@@QEBA_NPEAUhb_sanitize_context_t@@PEBX@Z 00000001800bbdf8     hb-aat-layout.obj
 0002:00030df8       $unwind$hb_blob_get_data_writable 00000001800bbdf8     hb-blob.obj
 0002:00030df8       $unwind$?delete_glyph@hb_buffer_t@@QEAAXXZ 00000001800bbdf8     hb-buffer.obj
 0002:00030df8       $unwind$hb_buffer_create_similar 00000001800bbdf8     hb-buffer.obj
 0002:00030df8       $unwind$hb_buffer_set_length 00000001800bbdf8     hb-buffer.obj
 0002:00030df8       $unwind$?sanitize@HVARVVAR@OT@@QEBA_NPEAUhb_sanitize_context_t@@@Z 00000001800bbdf8     hb-common.obj
 0002:00030df8       $unwind$?sanitize@maxp@OT@@QEBA_NPEAUhb_sanitize_context_t@@@Z 00000001800bbdf8     hb-common.obj
 0002:00030df8       $unwind$?fini@?$hb_hashmap_t@PEBUobject_t@hb_serialize_context_t@@I$0A@@@QEAAXXZ 00000001800bbdf8     hb-face-builder.obj
 0002:00030df8       $unwind$?fini@object_t@hb_serialize_context_t@@QEAAXXZ 00000001800bbdf8     hb-face-builder.obj
 0002:00030df8       $unwind$??$get_glyph_from@UCmapSubtableFormat12@OT@@@accelerator_t@cmap@OT@@KA_NPEBXIPEAI@Z 00000001800bbdf8     hb-face.obj
 0002:00030df8       $unwind$??$sanitize@$$V@?$ArrayOf@UCmapSubtableLongGroup@OT@@U?$IntType@I$03@2@@OT@@QEBA_NPEAUhb_sanitize_context_t@@@Z 00000001800bbdf8     hb-face.obj
 0002:00030df8       $unwind$?_hb_font_create@@YAPEAUhb_font_t@@PEAUhb_face_t@@@Z 00000001800bbdf8     hb-font.obj
 0002:00030df8       $unwind$?hb_font_get_font_h_extents_default@@YAHPEAUhb_font_t@@PEAXPEAUhb_font_extents_t@@1@Z 00000001800bbdf8     hb-font.obj
 0002:00030df8       $unwind$?hb_font_get_font_v_extents_default@@YAHPEAUhb_font_t@@PEAXPEAUhb_font_extents_t@@1@Z 00000001800bbdf8     hb-font.obj
 0002:00030df8       $unwind$hb_font_create     00000001800bbdf8     hb-font.obj
 0002:00030df8       $unwind$?hb_jdk_get_nominal_glyph@@YAHPEAUhb_font_t@@PEAXIPEAI1@Z 00000001800bbdf8     hb-jdk-font.obj
 0002:00030df8       $unwind$??1hb_paint_extents_context_t@@QEAA@XZ 00000001800bbdf8     hb-ot-font.obj
 0002:00030df8       $unwind$?cmp@gname_t@accelerator_t@cff1@OT@@SAHPEBX0@Z 00000001800bbdf8     hb-ot-font.obj
 0002:00030df8       $unwind$?hb_ot_get_font_h_extents@@YAHPEAUhb_font_t@@PEAXPEAUhb_font_extents_t@@1@Z 00000001800bbdf8     hb-ot-font.obj
 0002:00030df8       $unwind$?hb_ot_get_font_v_extents@@YAHPEAUhb_font_t@@PEAXPEAUhb_font_extents_t@@1@Z 00000001800bbdf8     hb-ot-font.obj
 0002:00030df8       $unwind$?sanitize@VORG@OT@@QEBA_NPEAUhb_sanitize_context_t@@@Z 00000001800bbdf8     hb-ot-font.obj
 0002:00030df8       $unwind$??$dispatch@Uhb_sanitize_context_t@@$$V@?$KernSubTable@UKernAATSubTableHeader@OT@@@OT@@QEBA_NPEAUhb_sanitize_context_t@@@Z 00000001800bbdf8     hb-ot-layout.obj
 0002:00030df8       $unwind$??$sanitize@$$V@?$ArrayOf@UIndex@OT@@U?$IntType@G$01@2@@OT@@QEBA_NPEAUhb_sanitize_context_t@@@Z 00000001800bbdf8     hb-ot-layout.obj
 0002:00030df8       $unwind$??$sanitize@$$V@?$ArrayOf@ULookupRecord@OT@@U?$IntType@G$01@2@@OT@@QEBA_NPEAUhb_sanitize_context_t@@@Z 00000001800bbdf8     hb-ot-layout.obj
 0002:00030df8       $unwind$?get_kerning@?$KerxSubTableFormat2@UKernAATSubTableHeader@OT@@@AAT@@QEBAHIIPEAUhb_aat_apply_context_t@2@@Z 00000001800bbdf8     hb-ot-layout.obj
 0002:00030df8       $unwind$?get_kerning@?$KerxSubTableFormat2@UKernOTSubTableHeader@OT@@@AAT@@QEBAHIIPEAUhb_aat_apply_context_t@2@@Z 00000001800bbdf8     hb-ot-layout.obj
 0002:00030df8       $unwind$?match_class_cached@OT@@YA_NAEAUhb_glyph_info_t@@IPEBX@Z 00000001800bbdf8     hb-ot-layout.obj
 0002:00030df8       $unwind$?sanitize@FeatureParams@OT@@QEBA_NPEAUhb_sanitize_context_t@@I@Z 00000001800bbdf8     hb-ot-layout.obj
 0002:00030df8       $unwind$?sanitize@GPOS@Layout@OT@@QEBA_NPEAUhb_sanitize_context_t@@@Z 00000001800bbdf8     hb-ot-layout.obj
 0002:00030df8       $unwind$?sanitize@GSUB@Layout@OT@@QEBA_NPEAUhb_sanitize_context_t@@@Z 00000001800bbdf8     hb-ot-layout.obj
 0002:00030df8       $unwind$?sanitize@kern@OT@@QEBA_NPEAUhb_sanitize_context_t@@@Z 00000001800bbdf8     hb-ot-layout.obj
 0002:00030df8       $unwind$?sanitize_shallow@?$OffsetTo@ULangSys@OT@@U?$IntType@G$01@2@$00@OT@@QEBA_NPEAUhb_sanitize_context_t@@PEBX@Z 00000001800bbdf8     hb-ot-layout.obj
 0002:00030df8       $unwind$hb_ot_layout_feature_with_variations_get_lookups 00000001800bbdf8     hb-ot-layout.obj
 0002:00030df8       $unwind$hb_ot_layout_table_find_feature_variations 00000001800bbdf8     hb-ot-layout.obj
 0002:00030df8       $unwind$?output_char@@YAXPEAUhb_buffer_t@@II@Z 00000001800bbdf8     hb-ot-shape-normalize.obj
 0002:00030df8       $unwind$?fini@hb_ot_map_t@@QEAAXXZ 00000001800bbdf8     hb-ot-shape.obj
 0002:00030df8       $unwind$?pop_discard@hb_serialize_context_t@@QEAAXXZ 00000001800bbdf8     hb-ot-shaper-arabic.obj
 0002:00030df8       $unwind$?data_create_use@@YAPEAXPEBUhb_ot_shape_plan_t@@@Z 00000001800bbdf8     hb-ot-shaper-use.obj
 0002:00030df8       $unwind$hb_unicode_funcs_create 00000001800bbdf8     hb-unicode.obj
 0002:00030df8       $unwind$_RTC_Initialize    00000001800bbdf8     MSVCRT:initsect.obj
 0002:00030df8       $unwind$_RTC_Terminate     00000001800bbdf8     MSVCRT:initsect.obj
 0002:00030e04       $unwind$?copy_glyph@hb_buffer_t@@QEAA_NXZ 00000001800bbe04     hb-aat-layout.obj
 0002:00030e04       $unwind$?hb_font_get_glyph_extents_default@@YAHPEAUhb_font_t@@PEAXIPEAUhb_glyph_extents_t@@1@Z 00000001800bbe04     hb-font.obj
 0002:00030e04       $unwind$?hb_jdk_get_glyph_contour_point@@YAHPEAUhb_font_t@@PEAXIIPEAH21@Z 00000001800bbe04     hb-jdk-font.obj
 0002:00030e04       $unwind$?hb_jdk_get_glyph_v_advance@@YAHPEAUhb_font_t@@PEAXI1@Z 00000001800bbe04     hb-jdk-font.obj
 0002:00030e04       $unwind$?hb_jdk_get_variation_glyph@@YAHPEAUhb_font_t@@PEAXIIPEAI1@Z 00000001800bbe04     hb-jdk-font.obj
 0002:00030e10       $unwind$?unsafe_to_break@hb_buffer_t@@QEAAXII@Z 00000001800bbe10     hb-aat-layout.obj
 0002:00030e20       $unwind$?unsafe_to_concat@hb_buffer_t@@QEAAXII@Z 00000001800bbe20     hb-aat-layout.obj
 0002:00030e2c       $chain$0$?unsafe_to_concat@hb_buffer_t@@QEAAXII@Z 00000001800bbe2c     hb-aat-layout.obj
 0002:00030e40       $chain$1$?unsafe_to_concat@hb_buffer_t@@QEAAXII@Z 00000001800bbe40     hb-aat-layout.obj
 0002:00030e50       $unwind$?unsafe_to_break_from_outbuffer@hb_buffer_t@@QEAAXII@Z 00000001800bbe50     hb-aat-layout.obj
 0002:00030e68       $unwind$?message@hb_buffer_t@@QEAA_NPEAUhb_font_t@@PEBDZZ 00000001800bbe68     hb-aat-layout.obj
 0002:00030e68       $unwind$?CallIntMethod@JNIEnv_@@QEAAJPEAV_jobject@@PEAU_jmethodID@@ZZ 00000001800bbe68     hb-jdk-font.obj
 0002:00030e68       $unwind$?CallObjectMethod@JNIEnv_@@QEAAPEAV_jobject@@PEAV2@PEAU_jmethodID@@ZZ 00000001800bbe68     hb-jdk-font.obj
 0002:00030e70       $unwind$?_infos_set_glyph_flags@hb_buffer_t@@QEAAXPEAUhb_glyph_info_t@@IIII@Z 00000001800bbe70     hb-aat-layout.obj
 0002:00030e70       $unwind$?merge_out_clusters@hb_buffer_t@@QEAAXII@Z 00000001800bbe70     hb-buffer.obj
 0002:00030e70       $unwind$?get_glyph@Charset@CFF@@QEBAIII@Z 00000001800bbe70     hb-ot-cff1-table.obj
 0002:00030e70       $unwind$?hb_ucd_compose@@YAHPEAUhb_unicode_funcs_t@@IIPEAIPEAX@Z 00000001800bbe70     hb-ucd.obj
 0002:00030e70       $unwind$__GSHandlerCheckCommon 00000001800bbe70     MSVCRT:gshandler.obj
 0002:00030e78       $chain$0$?_infos_set_glyph_flags@hb_buffer_t@@QEAAXPEAUhb_glyph_info_t@@IIII@Z 00000001800bbe78     hb-aat-layout.obj
 0002:00030e8c       $chain$2$?_infos_set_glyph_flags@hb_buffer_t@@QEAAXPEAUhb_glyph_info_t@@IIII@Z 00000001800bbe8c     hb-aat-layout.obj
 0002:00030e8c       $chain$4$?_infos_set_glyph_flags@hb_buffer_t@@QEAAXPEAUhb_glyph_info_t@@IIII@Z 00000001800bbe8c     hb-aat-layout.obj
 0002:00030ea0       $chain$5$?_infos_set_glyph_flags@hb_buffer_t@@QEAAXPEAUhb_glyph_info_t@@IIII@Z 00000001800bbea0     hb-aat-layout.obj
 0002:00030eb0       $unwind$?shrink_vector@?$hb_vector_t@U?$hb_vector_t@Urange_flags_t@hb_aat_map_t@@$00@@$0A@@@QEAAXI@Z 00000001800bbeb0     hb-aat-layout.obj
 0002:00030eb0       $unwind$?shrink_vector@?$hb_vector_t@U?$cff1_private_dict_values_base_t@Udict_val_t@CFF@@@CFF@@$0A@@@QEAAXI@Z 00000001800bbeb0     hb-ot-face.obj
 0002:00030eb0       $unwind$?shrink_vector@?$hb_vector_t@U?$cff2_private_dict_values_base_t@Udict_val_t@CFF@@@CFF@@$0A@@@QEAAXI@Z 00000001800bbeb0     hb-ot-face.obj
 0002:00030eb0       $unwind$?shrink_vector@?$hb_vector_t@Ucff1_font_dict_values_t@CFF@@$0A@@@QEAAXI@Z 00000001800bbeb0     hb-ot-face.obj
 0002:00030eb0       $unwind$?shrink_vector@?$hb_vector_t@Ucff2_font_dict_values_t@CFF@@$0A@@@QEAAXI@Z 00000001800bbeb0     hb-ot-face.obj
 0002:00030ebc       $chain$1$?shrink_vector@?$hb_vector_t@U?$hb_vector_t@Urange_flags_t@hb_aat_map_t@@$00@@$0A@@@QEAAXI@Z 00000001800bbebc     hb-aat-layout.obj
 0002:00030ed4       $chain$2$?shrink_vector@?$hb_vector_t@U?$hb_vector_t@Urange_flags_t@hb_aat_map_t@@$00@@$0A@@@QEAAXI@Z 00000001800bbed4     hb-aat-layout.obj
 0002:00030ee4       $unwind$?alloc@?$hb_vector_t@U?$hb_vector_t@Urange_flags_t@hb_aat_map_t@@$00@@$0A@@@QEAA_NI_N@Z 00000001800bbee4     hb-aat-layout.obj
 0002:00030ee4       $unwind$?alloc@?$hb_vector_t@U?$cff1_private_dict_values_base_t@Udict_val_t@CFF@@@CFF@@$0A@@@QEAA_NI_N@Z 00000001800bbee4     hb-ot-font.obj
 0002:00030ee4       $unwind$?alloc@?$hb_vector_t@Ucff1_font_dict_values_t@CFF@@$0A@@@QEAA_NI_N@Z 00000001800bbee4     hb-ot-font.obj
 0002:00030ee4       $unwind$?alloc@?$hb_vector_t@Ucff2_font_dict_values_t@CFF@@$0A@@@QEAA_NI_N@Z 00000001800bbee4     hb-ot-font.obj
 0002:00030eec       $chain$2$?alloc@?$hb_vector_t@U?$hb_vector_t@Urange_flags_t@hb_aat_map_t@@$00@@$0A@@@QEAA_NI_N@Z 00000001800bbeec     hb-aat-layout.obj
 0002:00030f08       $chain$4$?alloc@?$hb_vector_t@U?$hb_vector_t@Urange_flags_t@hb_aat_map_t@@$00@@$0A@@@QEAA_NI_N@Z 00000001800bbf08     hb-aat-layout.obj
 0002:00030f24       $chain$5$?alloc@?$hb_vector_t@U?$hb_vector_t@Urange_flags_t@hb_aat_map_t@@$00@@$0A@@@QEAA_NI_N@Z 00000001800bbf24     hb-aat-layout.obj
 0002:00030f38       $chain$6$?alloc@?$hb_vector_t@U?$hb_vector_t@Urange_flags_t@hb_aat_map_t@@$00@@$0A@@@QEAA_NI_N@Z 00000001800bbf38     hb-aat-layout.obj
 0002:00030f4c       $chain$7$?alloc@?$hb_vector_t@U?$hb_vector_t@Urange_flags_t@hb_aat_map_t@@$00@@$0A@@@QEAA_NI_N@Z 00000001800bbf4c     hb-aat-layout.obj
 0002:00030f5c       $chain$8$?alloc@?$hb_vector_t@U?$hb_vector_t@Urange_flags_t@hb_aat_map_t@@$00@@$0A@@@QEAA_NI_N@Z 00000001800bbf5c     hb-aat-layout.obj
 0002:00030f6c       $unwind$??C?$hb_lazy_loader_t@UGDEF_accelerator_t@OT@@U?$hb_face_lazy_loader_t@UGDEF_accelerator_t@OT@@$0BI@@@Uhb_face_t@@$0BI@U12@@@QEBAPEBUGDEF_accelerator_t@OT@@XZ 00000001800bbf6c     hb-aat-layout.obj
 0002:00030f6c       $unwind$??C?$hb_lazy_loader_t@Usbix_accelerator_t@OT@@U?$hb_face_lazy_loader_t@Usbix_accelerator_t@OT@@$0CG@@@Uhb_face_t@@$0CG@U12@@@QEBAPEBUsbix_accelerator_t@OT@@XZ 00000001800bbf6c     hb-ot-color.obj
 0002:00030f80       $unwind$?get_stored@?$hb_lazy_loader_t@Ukerx@AAT@@U?$hb_table_lazy_loader_t@Ukerx@AAT@@$0BO@$0A@@@Uhb_face_t@@$0BO@Uhb_blob_t@@@@QEBAPEAUhb_blob_t@@XZ 00000001800bbf80     hb-aat-layout.obj
 0002:00030f80       $unwind$?get_stored@?$hb_lazy_loader_t@Umort@AAT@@U?$hb_table_lazy_loader_t@Umort@AAT@@$0BN@$0A@@@Uhb_face_t@@$0BN@Uhb_blob_t@@@@QEBAPEAUhb_blob_t@@XZ 00000001800bbf80     hb-aat-layout.obj
 0002:00030f80       $unwind$?get_stored@?$hb_lazy_loader_t@Umorx@AAT@@U?$hb_table_lazy_loader_t@Umorx@AAT@@$0BM@$0A@@@Uhb_face_t@@$0BM@Uhb_blob_t@@@@QEBAPEAUhb_blob_t@@XZ 00000001800bbf80     hb-aat-layout.obj
 0002:00030f80       $unwind$?get_clip_box@ClipBoxFormat2@OT@@QEBAXAEAUClipBoxData@2@AEBUVarStoreInstancer@2@@Z 00000001800bbf80     hb-ot-font.obj
 0002:00030f80       $unwind$?get_stored@?$hb_lazy_loader_t@Ukern@OT@@U?$hb_table_lazy_loader_t@Ukern@OT@@$0BH@$00@@Uhb_face_t@@$0BH@Uhb_blob_t@@@@QEBAPEAUhb_blob_t@@XZ 00000001800bbf80     hb-ot-layout.obj
 0002:00030f90       $unwind$??C?$hb_lazy_loader_t@Ufeat@AAT@@U?$hb_table_lazy_loader_t@Ufeat@AAT@@$0CC@$0A@@@Uhb_face_t@@$0CC@Uhb_blob_t@@@@QEBAPEBUfeat@AAT@@XZ 00000001800bbf90     hb-aat-layout.obj
 0002:00030f90       $unwind$??C?$hb_lazy_loader_t@Ultag@AAT@@U?$hb_table_lazy_loader_t@Ultag@AAT@@$0CB@$0A@@@Uhb_face_t@@$0CB@Uhb_blob_t@@@@QEBAPEBUltag@AAT@@XZ 00000001800bbf90     hb-aat-layout.obj
 0002:00030f90       $unwind$?get@?$hb_lazy_loader_t@Utrak@AAT@@U?$hb_table_lazy_loader_t@Utrak@AAT@@$0CA@$0A@@@Uhb_face_t@@$0CA@Uhb_blob_t@@@@QEBAPEBUtrak@AAT@@XZ 00000001800bbf90     hb-aat-layout.obj
 0002:00030f90       $unwind$??C?$hb_lazy_loader_t@Uhhea@OT@@U?$hb_table_lazy_loader_t@Uhhea@OT@@$03$00@@Uhb_face_t@@$03Uhb_blob_t@@@@QEBAPEBUhhea@OT@@XZ 00000001800bbf90     hb-common.obj
 0002:00030f90       $unwind$??C?$hb_lazy_loader_t@Umaxp@OT@@U?$hb_table_lazy_loader_t@Umaxp@OT@@$01$00@@Uhb_face_t@@$01Uhb_blob_t@@@@QEBAPEBUmaxp@OT@@XZ 00000001800bbf90     hb-common.obj
 0002:00030f90       $unwind$??C?$hb_lazy_loader_t@Uvhea@OT@@U?$hb_table_lazy_loader_t@Uvhea@OT@@$0L@$00@@Uhb_face_t@@$0L@Uhb_blob_t@@@@QEBAPEBUvhea@OT@@XZ 00000001800bbf90     hb-common.obj
 0002:00030f90       $unwind$?get@?$hb_lazy_loader_t@Uhead@OT@@U?$hb_table_lazy_loader_t@Uhead@OT@@$00$00@@Uhb_face_t@@$00Uhb_blob_t@@@@QEBAPEBUhead@OT@@XZ 00000001800bbf90     hb-common.obj
 0002:00030f90       $unwind$??C?$hb_lazy_loader_t@UOS2@OT@@U?$hb_table_lazy_loader_t@UOS2@OT@@$05$00@@Uhb_face_t@@$05Uhb_blob_t@@@@QEBAPEBUOS2@OT@@XZ 00000001800bbf90     hb-face.obj
 0002:00030f90       $unwind$??C?$hb_lazy_loader_t@Uavar@OT@@U?$hb_table_lazy_loader_t@Uavar@OT@@$0BD@$00@@Uhb_face_t@@$0BD@Uhb_blob_t@@@@QEBAPEBUavar@OT@@XZ 00000001800bbf90     hb-font.obj
 0002:00030f90       $unwind$?get@?$hb_lazy_loader_t@Ufvar@OT@@U?$hb_table_lazy_loader_t@Ufvar@OT@@$0BC@$00@@Uhb_face_t@@$0BC@Uhb_blob_t@@@@QEBAPEBUfvar@OT@@XZ 00000001800bbf90     hb-font.obj
 0002:00030f90       $unwind$??C?$hb_lazy_loader_t@UCOLR@OT@@U?$hb_table_lazy_loader_t@UCOLR@OT@@$0CD@$00@@Uhb_face_t@@$0CD@Uhb_blob_t@@@@QEBAPEBUCOLR@OT@@XZ 00000001800bbf90     hb-ot-color.obj
 0002:00030f90       $unwind$??C?$hb_lazy_loader_t@UCPAL@OT@@U?$hb_table_lazy_loader_t@UCPAL@OT@@$0CE@$00@@Uhb_face_t@@$0CE@Uhb_blob_t@@@@QEBAPEBUCPAL@OT@@XZ 00000001800bbf90     hb-ot-color.obj
 0002:00030f90       $unwind$?get@?$hb_lazy_loader_t@UMVAR@OT@@U?$hb_table_lazy_loader_t@UMVAR@OT@@$0BG@$00@@Uhb_face_t@@$0BG@Uhb_blob_t@@@@QEBAPEBUMVAR@OT@@XZ 00000001800bbf90     hb-ot-metrics.obj
 0002:00030f9c       $chain$0$?get@?$hb_lazy_loader_t@Utrak@AAT@@U?$hb_table_lazy_loader_t@Utrak@AAT@@$0CA@$0A@@@Uhb_face_t@@$0CA@Uhb_blob_t@@@@QEBAPEBUtrak@AAT@@XZ 00000001800bbf9c     hb-aat-layout.obj
 0002:00030fb0       $chain$1$?get@?$hb_lazy_loader_t@Utrak@AAT@@U?$hb_table_lazy_loader_t@Utrak@AAT@@$0CA@$0A@@@Uhb_face_t@@$0CA@Uhb_blob_t@@@@QEBAPEBUtrak@AAT@@XZ 00000001800bbfb0     hb-aat-layout.obj
 0002:00030fc0       $chain$0$??C?$hb_lazy_loader_t@Ultag@AAT@@U?$hb_table_lazy_loader_t@Ultag@AAT@@$0CB@$0A@@@Uhb_face_t@@$0CB@Uhb_blob_t@@@@QEBAPEBUltag@AAT@@XZ 00000001800bbfc0     hb-aat-layout.obj
 0002:00030fd4       $chain$1$??C?$hb_lazy_loader_t@Ultag@AAT@@U?$hb_table_lazy_loader_t@Ultag@AAT@@$0CB@$0A@@@Uhb_face_t@@$0CB@Uhb_blob_t@@@@QEBAPEBUltag@AAT@@XZ 00000001800bbfd4     hb-aat-layout.obj
 0002:00030fe4       $chain$0$??C?$hb_lazy_loader_t@Ufeat@AAT@@U?$hb_table_lazy_loader_t@Ufeat@AAT@@$0CC@$0A@@@Uhb_face_t@@$0CC@Uhb_blob_t@@@@QEBAPEBUfeat@AAT@@XZ 00000001800bbfe4     hb-aat-layout.obj
 0002:00030ff8       $chain$1$??C?$hb_lazy_loader_t@Ufeat@AAT@@U?$hb_table_lazy_loader_t@Ufeat@AAT@@$0CC@$0A@@@Uhb_face_t@@$0CC@Uhb_blob_t@@@@QEBAPEBUfeat@AAT@@XZ 00000001800bbff8     hb-aat-layout.obj
 0002:00031008       $unwind$?get_glyph_h_origin_with_fallback@hb_font_t@@QEAAXIPEAH0@Z 00000001800bc008     hb-aat-layout.obj
 0002:00031008       $unwind$?get_glyph_origin_for_direction@hb_font_t@@QEAAXIW4hb_direction_t@@PEAH1@Z 00000001800bc008     hb-aat-layout.obj
 0002:00031008       $unwind$?get_glyph_v_origin_with_fallback@hb_font_t@@QEAAXIPEAH0@Z 00000001800bc008     hb-aat-layout.obj
 0002:00031020       $unwind$?get_glyph_contour_point_for_origin@hb_font_t@@QEAAHIIW4hb_direction_t@@PEAH1@Z 00000001800bc020     hb-aat-layout.obj
 0002:00031038       $unwind$?get_kerning@?$KerxSubTableFormat2@UKerxSubTableHeader@AAT@@@AAT@@QEBAHIIPEAUhb_aat_apply_context_t@2@@Z 00000001800bc038     hb-aat-layout.obj
 0002:00031038       $unwind$?next@skipping_iterator_t@hb_ot_apply_context_t@OT@@QEAA_NPEAI@Z 00000001800bc038     hb-aat-layout.obj
 0002:00031038       $unwind$?sanitize@ltag@AAT@@QEBA_NPEAUhb_sanitize_context_t@@@Z 00000001800bc038     hb-aat-layout.obj
 0002:00031038       $unwind$?unpack_points@TupleVariationData@OT@@SA_NAEAPEBU?$IntType@E$00@2@AEAU?$hb_vector_t@I$0A@@@PEBU32@@Z 00000001800bc038     hb-common.obj
 0002:00031038       $unwind$??$sanitize@$$V@?$OffsetTo@UBaseGlyphList@OT@@U?$IntType@I$03@2@$00@OT@@QEBA_NPEAUhb_sanitize_context_t@@PEBX@Z 00000001800bc038     hb-ot-color.obj
 0002:00031038       $unwind$?sanitize@?$FDSelect3_4@U?$IntType@I$03@OT@@U?$IntType@G$01@2@@CFF@@QEBA_NPEAUhb_sanitize_context_t@@I@Z 00000001800bc038     hb-ot-font.obj
 0002:00031038       $unwind$??$dispatch_recurse_func@Uhb_ot_apply_context_t@OT@@@PosLookup@GPOS_impl@Layout@OT@@SA_NPEAUhb_ot_apply_context_t@3@I@Z 00000001800bc038     hb-ot-layout.obj
 0002:00031038       $unwind$??$dispatch_recurse_func@Uhb_ot_apply_context_t@OT@@@SubstLookup@GSUB_impl@Layout@OT@@SA_NPEAUhb_ot_apply_context_t@3@I@Z 00000001800bc038     hb-ot-layout.obj
 0002:00031038       $unwind$??$sanitize@$$V@?$OffsetTo@UMarkArray@GPOS_impl@Layout@OT@@U?$IntType@G$01@4@$00@OT@@QEBA_NPEAUhb_sanitize_context_t@@PEBX@Z 00000001800bc038     hb-ot-layout.obj
 0002:00031038       $unwind$?prev@skipping_iterator_t@hb_ot_apply_context_t@OT@@QEAA_NPEAI@Z 00000001800bc038     hb-ot-layout.obj
 0002:00031038       $unwind$?_hb_ot_metrics_get_position_common@@YA_NPEAUhb_font_t@@W4hb_ot_metrics_tag_t@@PEAH@Z 00000001800bc038     hb-ot-metrics.obj
 0002:00031038       $unwind$?initial_reordering_consonant_syllable@@YAXPEAUhb_buffer_t@@II@Z 00000001800bc038     hb-ot-shaper-myanmar.obj
 0002:00031050       $unwind$?get_coverage@?$CoverageFormat1_3@USmallTypes@Layout@OT@@@Common@Layout@OT@@AEBAII@Z 00000001800bc050     hb-aat-layout.obj
 0002:00031050       $unwind$?get_feature@feat@AAT@@QEBAAEBUFeatureName@2@W4hb_aat_layout_feature_type_t@@@Z 00000001800bc050     hb-aat-layout.obj
 0002:00031050       $unwind$?hb_aat_layout_find_feature_mapping@@YAPEBUhb_aat_feature_mapping_t@@I@Z 00000001800bc050     hb-aat-layout.obj
 0002:00031050       $unwind$?get_leading_bearing_without_var_unscaled@accelerator_t@?$hmtxvmtx@Uhmtx@OT@@Uhhea@2@UHVAR@2@@OT@@QEBA_NIPEAH@Z 00000001800bc050     hb-common.obj
 0002:00031050       $unwind$?get_leading_bearing_without_var_unscaled@accelerator_t@?$hmtxvmtx@Uvmtx@OT@@Uvhea@2@UVVAR@2@@OT@@QEBA_NIPEAH@Z 00000001800bc050     hb-common.obj
 0002:00031050       $unwind$?parse_bool@@YA_NPEAPEBDPEBDPEAI@Z 00000001800bc050     hb-common.obj
 0002:00031050       $unwind$?get_base_glyph_record@COLR@OT@@QEBAPEBUBaseGlyphRecord@2@I@Z 00000001800bc050     hb-ot-font.obj
 0002:00031050       $unwind$?get_feature@GSUBGPOS@OT@@QEBAAEBUFeature@2@I@Z 00000001800bc050     hb-ot-layout.obj
 0002:00031050       $unwind$?get_script@GSUBGPOS@OT@@QEBAAEBUScript@2@I@Z 00000001800bc050     hb-ot-layout.obj
 0002:00031058       $unwind$??$replace_glyphs@UHBGlyphID16@OT@@@hb_buffer_t@@QEAA_NIIPEBUHBGlyphID16@OT@@@Z 00000001800bc058     hb-aat-layout.obj
 0002:00031058       $unwind$??$sanitize@$$V@?$OffsetTo@UDevice@OT@@U?$IntType@G$01@2@$00@OT@@QEBA_NPEAUhb_sanitize_context_t@@PEBX@Z 00000001800bc058     hb-aat-layout.obj
 0002:00031058       $unwind$??$sanitize@$$V@?$OffsetTo@UVarData@OT@@U?$IntType@I$03@2@$00@OT@@QEBA_NPEAUhb_sanitize_context_t@@PEBX@Z 00000001800bc058     hb-aat-layout.obj
 0002:00031058       $unwind$??0hb_aat_apply_context_t@AAT@@QEAA@PEBUhb_ot_shape_plan_t@@PEAUhb_font_t@@PEAUhb_buffer_t@@PEAUhb_blob_t@@@Z 00000001800bc058     hb-aat-layout.obj
 0002:00031058       $unwind$?get_kerning@?$KerxSubTableFormat0@UKerxSubTableHeader@AAT@@@AAT@@QEBAHIIPEAUhb_aat_apply_context_t@2@@Z 00000001800bc058     hb-aat-layout.obj
 0002:00031058       $unwind$?hb_aat_layout_compile_map@@YAXPEBUhb_aat_map_builder_t@@PEAUhb_aat_map_t@@@Z 00000001800bc058     hb-aat-layout.obj
 0002:00031058       $unwind$?resize@?$hb_vector_t@Ucontour_point_t@OT@@$0A@@@QEAA_NH_N0@Z 00000001800bc058     hb-common.obj
 0002:00031058       $unwind$?sanitize@gvar@OT@@QEBA_NPEAUhb_sanitize_context_t@@@Z 00000001800bc058     hb-common.obj
 0002:00031058       $unwind$hb_face_create_for_tables 00000001800bc058     hb-face.obj
 0002:00031058       $unwind$??$push@Uhb_bounds_t@@U1@$0A@@?$hb_vector_t@Uhb_bounds_t@@$0A@@@QEAAPEAUhb_bounds_t@@$$QEAU1@@Z 00000001800bc058     hb-ot-font.obj
 0002:00031058       $unwind$?_set_glyph_class@hb_ot_apply_context_t@OT@@QEAAXII_N0@Z 00000001800bc058     hb-ot-layout.obj
 0002:00031058       $unwind$?is_blocklisted@GDEF@OT@@QEBA_NPEAUhb_blob_t@@PEAUhb_face_t@@@Z 00000001800bc058     hb-ot-layout.obj
 0002:00031058       $unwind$?sanitize@SinglePosFormat1@GPOS_impl@Layout@OT@@QEBA_NPEAUhb_sanitize_context_t@@@Z 00000001800bc058     hb-ot-layout.obj
 0002:00031058       $unwind$?sanitize_value_devices@ValueFormat@GPOS_impl@Layout@OT@@AEBA_NPEAUhb_sanitize_context_t@@PEBXPEBU?$IntType@G$01@4@@Z 00000001800bc058     hb-ot-layout.obj
 0002:00031058       $unwind$??1hb_ot_map_builder_t@@QEAA@XZ 00000001800bc058     hb-ot-map.obj
 0002:00031058       $unwind$??$add_link@U?$OffsetTo@U?$Ligature@USmallTypes@Layout@OT@@@GSUB_impl@Layout@OT@@U?$IntType@G$01@4@$00@OT@@@hb_serialize_context_t@@QEAAXAEAU?$OffsetTo@U?$Ligature@USmallTypes@Layout@OT@@@GSUB_impl@Layout@OT@@U?$IntType@G$01@4@$00@OT@@IW4whence_t@0@I@Z 00000001800bc058     hb-ot-shaper-arabic.obj
 0002:00031058       $unwind$??$add_link@U?$OffsetTo@U?$LigatureSet@USmallTypes@Layout@OT@@@GSUB_impl@Layout@OT@@U?$IntType@G$01@4@$00@OT@@@hb_serialize_context_t@@QEAAXAEAU?$OffsetTo@U?$LigatureSet@USmallTypes@Layout@OT@@@GSUB_impl@Layout@OT@@U?$IntType@G$01@4@$00@OT@@IW4whence_t@0@I@Z 00000001800bc058     hb-ot-shaper-arabic.obj
 0002:00031058       $unwind$??$add_link@U?$OffsetTo@UCoverage@Common@Layout@OT@@U?$IntType@G$01@4@$00@OT@@@hb_serialize_context_t@@QEAAXAEAU?$OffsetTo@UCoverage@Common@Layout@OT@@U?$IntType@G$01@4@$00@OT@@IW4whence_t@0@I@Z 00000001800bc058     hb-ot-shaper-arabic.obj
 0002:00031058       $unwind$?collect_features_arabic@@YAXPEAUhb_ot_shape_planner_t@@@Z 00000001800bc058     hb-ot-shaper-arabic.obj
 0002:00031058       $unwind$?collect_features_myanmar@@YAXPEAUhb_ot_shape_planner_t@@@Z 00000001800bc058     hb-ot-shaper-myanmar.obj
 0002:00031058       $unwind$??Y?$hb_iter_t@U?$hb_zip_iter_t@U?$hb_iota_iter_t@II@@U?$hb_filter_iter_t@U?$hb_filter_iter_t@U?$hb_zip_iter_t@U?$hb_iota_iter_t@II@@U?$hb_array_t@Uhb_glyph_info_t@@@@@@V<lambda_e52748becc06432fe81365edeb8c4003>@@AEBU<unnamed-type-hb_second>@@$0A@@@V<lambda_a2885d5959499a7c5bcf896c0de144bb>@@AEBU<unnamed-type-hb_identity>@@$0A@@@@@U?$hb_pair_t@IU?$hb_pair_t@IAEAUhb_glyph_info_t@@@@@@@@QEGAAAEAU?$hb_zip_iter_t@U?$hb_iota_iter_t@II@@U?$hb_filter_iter_t@U?$hb_filter_iter_t@U?$hb_zip_iter_t@U?$hb_iota_iter_t@II@@U?$hb_array_t@Uhb_glyph_info_t@@@@@@V<lambda_e52748becc06432fe81365edeb8c4003>@@AEBU<unnamed-type-hb_second>@@$0A@@@V<lambda_a2885d5959499a7c5bcf896c0de144bb>@@AEBU<unnamed-type-hb_identity>@@$0A@@@@@I@Z 00000001800bc058     hb-ot-shaper-use.obj
 0002:00031058       $unwind$hb_ot_var_named_instance_get_design_coords 00000001800bc058     hb-ot-var.obj
 0002:00031058       $unwind$??$push@Uhb_outline_point_t@@U1@$0A@@?$hb_vector_t@Uhb_outline_point_t@@$0A@@@QEAAPEAUhb_outline_point_t@@$$QEAU1@@Z 00000001800bc058     hb-outline.obj
 0002:00031058       $unwind$hb_unicode_funcs_set_combining_class_func 00000001800bc058     hb-unicode.obj
 0002:00031058       $unwind$hb_unicode_funcs_set_compose_func 00000001800bc058     hb-unicode.obj
 0002:00031058       $unwind$hb_unicode_funcs_set_decompose_func 00000001800bc058     hb-unicode.obj
 0002:00031058       $unwind$hb_unicode_funcs_set_general_category_func 00000001800bc058     hb-unicode.obj
 0002:00031058       $unwind$hb_unicode_funcs_set_mirroring_func 00000001800bc058     hb-unicode.obj
 0002:00031058       $unwind$hb_unicode_funcs_set_script_func 00000001800bc058     hb-unicode.obj
 0002:00031058       $unwind$__scrt_dllmain_exception_filter 00000001800bc058     MSVCRT:utility.obj
 0002:0003106c       $unwind$?hb_aat_layout_substitute@@YAXPEBUhb_ot_shape_plan_t@@PEAUhb_font_t@@PEAUhb_buffer_t@@PEBUhb_feature_t@@I@Z 00000001800bc06c     hb-aat-layout.obj
 0002:0003108c       $unwind$?hb_aat_layout_position@@YAXPEBUhb_ot_shape_plan_t@@PEAUhb_font_t@@PEAUhb_buffer_t@@@Z 00000001800bc08c     hb-aat-layout.obj
 0002:000310a0       $chain$0$?hb_aat_layout_position@@YAXPEBUhb_ot_shape_plan_t@@PEAUhb_font_t@@PEAUhb_buffer_t@@@Z 00000001800bc0a0     hb-aat-layout.obj
 0002:000310b4       $chain$1$?hb_aat_layout_position@@YAXPEBUhb_ot_shape_plan_t@@PEAUhb_font_t@@PEAUhb_buffer_t@@@Z 00000001800bc0b4     hb-aat-layout.obj
 0002:000310c8       $chain$2$?hb_aat_layout_position@@YAXPEBUhb_ot_shape_plan_t@@PEAUhb_font_t@@PEAUhb_buffer_t@@@Z 00000001800bc0c8     hb-aat-layout.obj
 0002:000310d8       $chain$3$?hb_aat_layout_position@@YAXPEBUhb_ot_shape_plan_t@@PEAUhb_font_t@@PEAUhb_buffer_t@@@Z 00000001800bc0d8     hb-aat-layout.obj
 0002:000310e8       $unwind$?hb_aat_layout_track@@YAXPEBUhb_ot_shape_plan_t@@PEAUhb_font_t@@PEAUhb_buffer_t@@@Z 00000001800bc0e8     hb-aat-layout.obj
 0002:000310e8       $unwind$?hb_ot_layout_kern@@YAXPEBUhb_ot_shape_plan_t@@PEAUhb_font_t@@PEAUhb_buffer_t@@@Z 00000001800bc0e8     hb-ot-layout.obj
 0002:00031100       $unwind$?sanitize@ankr@AAT@@QEBA_NPEAUhb_sanitize_context_t@@@Z 00000001800bc100     hb-aat-layout.obj
 0002:00031100       $unwind$?sanitize@COLR@OT@@QEBA_NPEAUhb_sanitize_context_t@@@Z 00000001800bc100     hb-ot-color.obj
 0002:00031100       $unwind$?serialize@?$SortedArrayOf@U?$RangeRecord@USmallTypes@Layout@OT@@@Common@Layout@OT@@U?$IntType@G$01@4@@OT@@QEAA_NPEAUhb_serialize_context_t@@I@Z 00000001800bc100     hb-ot-shaper-arabic.obj
 0002:00031114       $unwind$?get_value@?$Lookup@U?$IntType@G$01@OT@@@AAT@@QEBAPEBU?$IntType@G$01@OT@@II@Z 00000001800bc114     hb-aat-layout.obj
 0002:00031114       $unwind$?get_value@?$Lookup@U?$IntType@I$03@OT@@@AAT@@QEBAPEBU?$IntType@I$03@OT@@II@Z 00000001800bc114     hb-aat-layout.obj
 0002:00031114       $unwind$?get_value@?$Lookup@U?$OffsetTo@U?$ArrayOf@UAnchor@AAT@@U?$IntType@I$03@OT@@@OT@@U?$IntType@G$01@2@$0A@@OT@@@AAT@@QEBAPEBU?$OffsetTo@U?$ArrayOf@UAnchor@AAT@@U?$IntType@I$03@OT@@@OT@@U?$IntType@G$01@2@$0A@@OT@@II@Z 00000001800bc114     hb-aat-layout.obj
 0002:00031114       $unwind$?get_value@?$Lookup@UHBGlyphID16@OT@@@AAT@@QEBAPEBUHBGlyphID16@OT@@II@Z 00000001800bc114     hb-aat-layout.obj
 0002:00031114       $unwind$hb_blob_create     00000001800bc114     hb-blob.obj
 0002:00031114       $unwind$?resolve_links@hb_serialize_context_t@@QEAAXXZ 00000001800bc114     hb-face-builder.obj
 0002:00031114       $unwind$hb_face_set_user_data 00000001800bc114     hb-face.obj
 0002:00031114       $unwind$hb_font_draw_glyph 00000001800bc114     hb-font.obj
 0002:00031114       $unwind$hb_font_get_glyph_extents 00000001800bc114     hb-font.obj
 0002:00031114       $unwind$hb_font_get_nominal_glyph 00000001800bc114     hb-font.obj
 0002:00031114       $unwind$?get_path@accelerator_t@cff1@OT@@QEBA_NPEAUhb_font_t@@IAEAUhb_draw_session_t@@@Z 00000001800bc114     hb-ot-cff1-table.obj
 0002:00031114       $unwind$?hhcurveto@?$path_procs_t@Ucff1_path_procs_extents_t@@Ucff1_cs_interp_env_t@CFF@@Ucff1_extents_param_t@@@CFF@@SAXAEAUcff1_cs_interp_env_t@2@AEAUcff1_extents_param_t@@@Z 00000001800bc114     hb-ot-cff1-table.obj
 0002:00031114       $unwind$?vvcurveto@?$path_procs_t@Ucff1_path_procs_extents_t@@Ucff1_cs_interp_env_t@CFF@@Ucff1_extents_param_t@@@CFF@@SAXAEAUcff1_cs_interp_env_t@2@AEAUcff1_extents_param_t@@@Z 00000001800bc114     hb-ot-cff1-table.obj
 0002:00031114       $unwind$?compose_unicode@@YA_NPEBUhb_ot_shape_normalize_context_t@@IIPEAI@Z 00000001800bc114     hb-ot-shape-normalize.obj
 0002:00031114       $unwind$?decompose_unicode@@YA_NPEBUhb_ot_shape_normalize_context_t@@IPEAI1@Z 00000001800bc114     hb-ot-shape-normalize.obj
 0002:00031114       $unwind$?has_glyph@hb_font_t@@QEAA_NI@Z 00000001800bc114     hb-ot-shape.obj
 0002:00031114       $unwind$?decompose_indic@@YA_NPEBUhb_ot_shape_normalize_context_t@@IPEAI1@Z 00000001800bc114     hb-ot-shaper-indic.obj
 0002:00031114       $unwind$?decompose_khmer@@YA_NPEBUhb_ot_shape_normalize_context_t@@IPEAI1@Z 00000001800bc114     hb-ot-shaper-khmer.obj
 0002:00031114       $unwind$?hb_outline_recording_pen_line_to@@YAXPEAUhb_draw_funcs_t@@PEAXPEAUhb_draw_state_t@@MM1@Z 00000001800bc114     hb-outline.obj
 0002:00031114       $unwind$?hb_outline_recording_pen_move_to@@YAXPEAUhb_draw_funcs_t@@PEAXPEAUhb_draw_state_t@@MM1@Z 00000001800bc114     hb-outline.obj
 0002:0003111c       $chain$3$?get_value@?$Lookup@U?$IntType@G$01@OT@@@AAT@@QEBAPEBU?$IntType@G$01@OT@@II@Z 00000001800bc11c     hb-aat-layout.obj
 0002:0003111c       $chain$3$?get_value@?$Lookup@U?$OffsetTo@U?$ArrayOf@UAnchor@AAT@@U?$IntType@I$03@OT@@@OT@@U?$IntType@G$01@2@$0A@@OT@@@AAT@@QEBAPEBU?$OffsetTo@U?$ArrayOf@UAnchor@AAT@@U?$IntType@I$03@OT@@@OT@@U?$IntType@G$01@2@$0A@@OT@@II@Z 00000001800bc11c     hb-aat-layout.obj
 0002:0003111c       $chain$3$?get_value@?$Lookup@UHBGlyphID16@OT@@@AAT@@QEBAPEBUHBGlyphID16@OT@@II@Z 00000001800bc11c     hb-aat-layout.obj
 0002:0003113c       $chain$5$?get_value@?$Lookup@U?$IntType@G$01@OT@@@AAT@@QEBAPEBU?$IntType@G$01@OT@@II@Z 00000001800bc13c     hb-aat-layout.obj
 0002:0003113c       $chain$5$?get_value@?$Lookup@U?$OffsetTo@U?$ArrayOf@UAnchor@AAT@@U?$IntType@I$03@OT@@@OT@@U?$IntType@G$01@2@$0A@@OT@@@AAT@@QEBAPEBU?$OffsetTo@U?$ArrayOf@UAnchor@AAT@@U?$IntType@I$03@OT@@@OT@@U?$IntType@G$01@2@$0A@@OT@@II@Z 00000001800bc13c     hb-aat-layout.obj
 0002:0003113c       $chain$5$?get_value@?$Lookup@UHBGlyphID16@OT@@@AAT@@QEBAPEBUHBGlyphID16@OT@@II@Z 00000001800bc13c     hb-aat-layout.obj
 0002:00031154       $chain$6$?get_value@?$Lookup@U?$IntType@G$01@OT@@@AAT@@QEBAPEBU?$IntType@G$01@OT@@II@Z 00000001800bc154     hb-aat-layout.obj
 0002:00031154       $chain$6$?get_value@?$Lookup@U?$OffsetTo@U?$ArrayOf@UAnchor@AAT@@U?$IntType@I$03@OT@@@OT@@U?$IntType@G$01@2@$0A@@OT@@@AAT@@QEBAPEBU?$OffsetTo@U?$ArrayOf@UAnchor@AAT@@U?$IntType@I$03@OT@@@OT@@U?$IntType@G$01@2@$0A@@OT@@II@Z 00000001800bc154     hb-aat-layout.obj
 0002:00031154       $chain$6$?get_value@?$Lookup@UHBGlyphID16@OT@@@AAT@@QEBAPEBUHBGlyphID16@OT@@II@Z 00000001800bc154     hb-aat-layout.obj
 0002:00031168       $chain$7$?get_value@?$Lookup@U?$IntType@G$01@OT@@@AAT@@QEBAPEBU?$IntType@G$01@OT@@II@Z 00000001800bc168     hb-aat-layout.obj
 0002:00031168       $chain$7$?get_value@?$Lookup@U?$OffsetTo@U?$ArrayOf@UAnchor@AAT@@U?$IntType@I$03@OT@@@OT@@U?$IntType@G$01@2@$0A@@OT@@@AAT@@QEBAPEBU?$OffsetTo@U?$ArrayOf@UAnchor@AAT@@U?$IntType@I$03@OT@@@OT@@U?$IntType@G$01@2@$0A@@OT@@II@Z 00000001800bc168     hb-aat-layout.obj
 0002:00031168       $chain$7$?get_value@?$Lookup@UHBGlyphID16@OT@@@AAT@@QEBAPEBUHBGlyphID16@OT@@II@Z 00000001800bc168     hb-aat-layout.obj
 0002:00031178       $chain$8$?get_value@?$Lookup@U?$IntType@G$01@OT@@@AAT@@QEBAPEBU?$IntType@G$01@OT@@II@Z 00000001800bc178     hb-aat-layout.obj
 0002:00031178       $chain$8$?get_value@?$Lookup@U?$OffsetTo@U?$ArrayOf@UAnchor@AAT@@U?$IntType@I$03@OT@@@OT@@U?$IntType@G$01@2@$0A@@OT@@@AAT@@QEBAPEBU?$OffsetTo@U?$ArrayOf@UAnchor@AAT@@U?$IntType@I$03@OT@@@OT@@U?$IntType@G$01@2@$0A@@OT@@II@Z 00000001800bc178     hb-aat-layout.obj
 0002:00031178       $chain$8$?get_value@?$Lookup@UHBGlyphID16@OT@@@AAT@@QEBAPEBUHBGlyphID16@OT@@II@Z 00000001800bc178     hb-aat-layout.obj
 0002:0003118c       $chain$10$?get_value@?$Lookup@U?$IntType@G$01@OT@@@AAT@@QEBAPEBU?$IntType@G$01@OT@@II@Z 00000001800bc18c     hb-aat-layout.obj
 0002:0003118c       $chain$10$?get_value@?$Lookup@U?$OffsetTo@U?$ArrayOf@UAnchor@AAT@@U?$IntType@I$03@OT@@@OT@@U?$IntType@G$01@2@$0A@@OT@@@AAT@@QEBAPEBU?$OffsetTo@U?$ArrayOf@UAnchor@AAT@@U?$IntType@I$03@OT@@@OT@@U?$IntType@G$01@2@$0A@@OT@@II@Z 00000001800bc18c     hb-aat-layout.obj
 0002:0003118c       $chain$10$?get_value@?$Lookup@UHBGlyphID16@OT@@@AAT@@QEBAPEBUHBGlyphID16@OT@@II@Z 00000001800bc18c     hb-aat-layout.obj
 0002:000311b0       $chain$11$?get_value@?$Lookup@U?$IntType@G$01@OT@@@AAT@@QEBAPEBU?$IntType@G$01@OT@@II@Z 00000001800bc1b0     hb-aat-layout.obj
 0002:000311b0       $chain$11$?get_value@?$Lookup@U?$OffsetTo@U?$ArrayOf@UAnchor@AAT@@U?$IntType@I$03@OT@@@OT@@U?$IntType@G$01@2@$0A@@OT@@@AAT@@QEBAPEBU?$OffsetTo@U?$ArrayOf@UAnchor@AAT@@U?$IntType@I$03@OT@@@OT@@U?$IntType@G$01@2@$0A@@OT@@II@Z 00000001800bc1b0     hb-aat-layout.obj
 0002:000311b0       $chain$11$?get_value@?$Lookup@UHBGlyphID16@OT@@@AAT@@QEBAPEBUHBGlyphID16@OT@@II@Z 00000001800bc1b0     hb-aat-layout.obj
 0002:000311c0       $unwind$?sanitize@?$Lookup@U?$OffsetTo@U?$ArrayOf@UAnchor@AAT@@U?$IntType@I$03@OT@@@OT@@U?$IntType@G$01@2@$0A@@OT@@@AAT@@QEBA_NPEAUhb_sanitize_context_t@@PEBX@Z 00000001800bc1c0     hb-aat-layout.obj
 0002:000311d8       $unwind$?get_value@?$LookupFormat2@U?$IntType@G$01@OT@@@AAT@@AEBAPEBU?$IntType@G$01@OT@@I@Z 00000001800bc1d8     hb-aat-layout.obj
 0002:000311d8       $unwind$?get_value@?$LookupFormat2@U?$IntType@I$03@OT@@@AAT@@AEBAPEBU?$IntType@I$03@OT@@I@Z 00000001800bc1d8     hb-aat-layout.obj
 0002:000311d8       $unwind$?get_value@?$LookupFormat2@U?$OffsetTo@U?$ArrayOf@UAnchor@AAT@@U?$IntType@I$03@OT@@@OT@@U?$IntType@G$01@2@$0A@@OT@@@AAT@@AEBAPEBU?$OffsetTo@U?$ArrayOf@UAnchor@AAT@@U?$IntType@I$03@OT@@@OT@@U?$IntType@G$01@2@$0A@@OT@@I@Z 00000001800bc1d8     hb-aat-layout.obj
 0002:000311d8       $unwind$?get_value@?$LookupFormat2@UHBGlyphID16@OT@@@AAT@@AEBAPEBUHBGlyphID16@OT@@I@Z 00000001800bc1d8     hb-aat-layout.obj
 0002:000311ec       $chain$0$?get_value@?$LookupFormat2@U?$IntType@G$01@OT@@@AAT@@AEBAPEBU?$IntType@G$01@OT@@I@Z 00000001800bc1ec     hb-aat-layout.obj
 0002:000311ec       $chain$0$?get_value@?$LookupFormat2@U?$IntType@I$03@OT@@@AAT@@AEBAPEBU?$IntType@I$03@OT@@I@Z 00000001800bc1ec     hb-aat-layout.obj
 0002:000311ec       $chain$0$?get_value@?$LookupFormat2@U?$OffsetTo@U?$ArrayOf@UAnchor@AAT@@U?$IntType@I$03@OT@@@OT@@U?$IntType@G$01@2@$0A@@OT@@@AAT@@AEBAPEBU?$OffsetTo@U?$ArrayOf@UAnchor@AAT@@U?$IntType@I$03@OT@@@OT@@U?$IntType@G$01@2@$0A@@OT@@I@Z 00000001800bc1ec     hb-aat-layout.obj
 0002:000311ec       $chain$0$?get_value@?$LookupFormat2@UHBGlyphID16@OT@@@AAT@@AEBAPEBUHBGlyphID16@OT@@I@Z 00000001800bc1ec     hb-aat-layout.obj
 0002:00031200       $chain$1$?get_value@?$LookupFormat2@U?$IntType@G$01@OT@@@AAT@@AEBAPEBU?$IntType@G$01@OT@@I@Z 00000001800bc200     hb-aat-layout.obj
 0002:00031200       $chain$1$?get_value@?$LookupFormat2@U?$IntType@I$03@OT@@@AAT@@AEBAPEBU?$IntType@I$03@OT@@I@Z 00000001800bc200     hb-aat-layout.obj
 0002:00031200       $chain$1$?get_value@?$LookupFormat2@U?$OffsetTo@U?$ArrayOf@UAnchor@AAT@@U?$IntType@I$03@OT@@@OT@@U?$IntType@G$01@2@$0A@@OT@@@AAT@@AEBAPEBU?$OffsetTo@U?$ArrayOf@UAnchor@AAT@@U?$IntType@I$03@OT@@@OT@@U?$IntType@G$01@2@$0A@@OT@@I@Z 00000001800bc200     hb-aat-layout.obj
 0002:00031200       $chain$1$?get_value@?$LookupFormat2@UHBGlyphID16@OT@@@AAT@@AEBAPEBUHBGlyphID16@OT@@I@Z 00000001800bc200     hb-aat-layout.obj
 0002:00031214       $chain$2$?get_value@?$LookupFormat2@U?$IntType@G$01@OT@@@AAT@@AEBAPEBU?$IntType@G$01@OT@@I@Z 00000001800bc214     hb-aat-layout.obj
 0002:00031214       $chain$2$?get_value@?$LookupFormat2@U?$IntType@I$03@OT@@@AAT@@AEBAPEBU?$IntType@I$03@OT@@I@Z 00000001800bc214     hb-aat-layout.obj
 0002:00031214       $chain$2$?get_value@?$LookupFormat2@U?$OffsetTo@U?$ArrayOf@UAnchor@AAT@@U?$IntType@I$03@OT@@@OT@@U?$IntType@G$01@2@$0A@@OT@@@AAT@@AEBAPEBU?$OffsetTo@U?$ArrayOf@UAnchor@AAT@@U?$IntType@I$03@OT@@@OT@@U?$IntType@G$01@2@$0A@@OT@@I@Z 00000001800bc214     hb-aat-layout.obj
 0002:00031214       $chain$2$?get_value@?$LookupFormat2@UHBGlyphID16@OT@@@AAT@@AEBAPEBUHBGlyphID16@OT@@I@Z 00000001800bc214     hb-aat-layout.obj
 0002:00031224       $chain$3$?get_value@?$LookupFormat2@U?$IntType@G$01@OT@@@AAT@@AEBAPEBU?$IntType@G$01@OT@@I@Z 00000001800bc224     hb-aat-layout.obj
 0002:00031224       $chain$3$?get_value@?$LookupFormat2@U?$IntType@I$03@OT@@@AAT@@AEBAPEBU?$IntType@I$03@OT@@I@Z 00000001800bc224     hb-aat-layout.obj
 0002:00031224       $chain$3$?get_value@?$LookupFormat2@U?$OffsetTo@U?$ArrayOf@UAnchor@AAT@@U?$IntType@I$03@OT@@@OT@@U?$IntType@G$01@2@$0A@@OT@@@AAT@@AEBAPEBU?$OffsetTo@U?$ArrayOf@UAnchor@AAT@@U?$IntType@I$03@OT@@@OT@@U?$IntType@G$01@2@$0A@@OT@@I@Z 00000001800bc224     hb-aat-layout.obj
 0002:00031224       $chain$3$?get_value@?$LookupFormat2@UHBGlyphID16@OT@@@AAT@@AEBAPEBUHBGlyphID16@OT@@I@Z 00000001800bc224     hb-aat-layout.obj
 0002:00031234       $unwind$?get_length@?$VarSizedBinSearchArrayOf@U?$LookupSegmentArray@U?$IntType@G$01@OT@@@AAT@@@OT@@QEBAIXZ 00000001800bc234     hb-aat-layout.obj
 0002:00031234       $unwind$?get_length@?$VarSizedBinSearchArrayOf@U?$LookupSegmentArray@U?$IntType@I$03@OT@@@AAT@@@OT@@QEBAIXZ 00000001800bc234     hb-aat-layout.obj
 0002:00031234       $unwind$?get_length@?$VarSizedBinSearchArrayOf@U?$LookupSegmentArray@U?$OffsetTo@U?$ArrayOf@UAnchor@AAT@@U?$IntType@I$03@OT@@@OT@@U?$IntType@G$01@2@$0A@@OT@@@AAT@@@OT@@QEBAIXZ 00000001800bc234     hb-aat-layout.obj
 0002:00031234       $unwind$?get_length@?$VarSizedBinSearchArrayOf@U?$LookupSegmentArray@UHBGlyphID16@OT@@@AAT@@@OT@@QEBAIXZ 00000001800bc234     hb-aat-layout.obj
 0002:00031234       $unwind$?get_length@?$VarSizedBinSearchArrayOf@U?$LookupSegmentSingle@U?$OffsetTo@U?$ArrayOf@UAnchor@AAT@@U?$IntType@I$03@OT@@@OT@@U?$IntType@G$01@2@$0A@@OT@@@AAT@@@OT@@QEBAIXZ 00000001800bc234     hb-aat-layout.obj
 0002:00031234       $unwind$?get_length@?$VarSizedBinSearchArrayOf@U?$LookupSingle@U?$OffsetTo@U?$ArrayOf@UAnchor@AAT@@U?$IntType@I$03@OT@@@OT@@U?$IntType@G$01@2@$0A@@OT@@@AAT@@@OT@@QEBAIXZ 00000001800bc234     hb-aat-layout.obj
 0002:00031240       $unwind$?get_value@?$LookupFormat4@U?$IntType@G$01@OT@@@AAT@@AEBAPEBU?$IntType@G$01@OT@@I@Z 00000001800bc240     hb-aat-layout.obj
 0002:00031240       $unwind$?get_value@?$LookupFormat4@U?$IntType@I$03@OT@@@AAT@@AEBAPEBU?$IntType@I$03@OT@@I@Z 00000001800bc240     hb-aat-layout.obj
 0002:00031240       $unwind$?get_value@?$LookupFormat4@U?$OffsetTo@U?$ArrayOf@UAnchor@AAT@@U?$IntType@I$03@OT@@@OT@@U?$IntType@G$01@2@$0A@@OT@@@AAT@@AEBAPEBU?$OffsetTo@U?$ArrayOf@UAnchor@AAT@@U?$IntType@I$03@OT@@@OT@@U?$IntType@G$01@2@$0A@@OT@@I@Z 00000001800bc240     hb-aat-layout.obj
 0002:00031240       $unwind$?get_value@?$LookupFormat4@UHBGlyphID16@OT@@@AAT@@AEBAPEBUHBGlyphID16@OT@@I@Z 00000001800bc240     hb-aat-layout.obj
 0002:00031254       $chain$0$?get_value@?$LookupFormat4@U?$IntType@G$01@OT@@@AAT@@AEBAPEBU?$IntType@G$01@OT@@I@Z 00000001800bc254     hb-aat-layout.obj
 0002:00031254       $chain$0$?get_value@?$LookupFormat4@U?$OffsetTo@U?$ArrayOf@UAnchor@AAT@@U?$IntType@I$03@OT@@@OT@@U?$IntType@G$01@2@$0A@@OT@@@AAT@@AEBAPEBU?$OffsetTo@U?$ArrayOf@UAnchor@AAT@@U?$IntType@I$03@OT@@@OT@@U?$IntType@G$01@2@$0A@@OT@@I@Z 00000001800bc254     hb-aat-layout.obj
 0002:00031254       $chain$0$?get_value@?$LookupFormat4@UHBGlyphID16@OT@@@AAT@@AEBAPEBUHBGlyphID16@OT@@I@Z 00000001800bc254     hb-aat-layout.obj
 0002:00031268       $chain$1$?get_value@?$LookupFormat4@U?$IntType@G$01@OT@@@AAT@@AEBAPEBU?$IntType@G$01@OT@@I@Z 00000001800bc268     hb-aat-layout.obj
 0002:00031268       $chain$1$?get_value@?$LookupFormat4@U?$OffsetTo@U?$ArrayOf@UAnchor@AAT@@U?$IntType@I$03@OT@@@OT@@U?$IntType@G$01@2@$0A@@OT@@@AAT@@AEBAPEBU?$OffsetTo@U?$ArrayOf@UAnchor@AAT@@U?$IntType@I$03@OT@@@OT@@U?$IntType@G$01@2@$0A@@OT@@I@Z 00000001800bc268     hb-aat-layout.obj
 0002:00031268       $chain$1$?get_value@?$LookupFormat4@UHBGlyphID16@OT@@@AAT@@AEBAPEBUHBGlyphID16@OT@@I@Z 00000001800bc268     hb-aat-layout.obj
 0002:0003127c       $chain$2$?get_value@?$LookupFormat4@U?$IntType@G$01@OT@@@AAT@@AEBAPEBU?$IntType@G$01@OT@@I@Z 00000001800bc27c     hb-aat-layout.obj
 0002:0003127c       $chain$2$?get_value@?$LookupFormat4@U?$OffsetTo@U?$ArrayOf@UAnchor@AAT@@U?$IntType@I$03@OT@@@OT@@U?$IntType@G$01@2@$0A@@OT@@@AAT@@AEBAPEBU?$OffsetTo@U?$ArrayOf@UAnchor@AAT@@U?$IntType@I$03@OT@@@OT@@U?$IntType@G$01@2@$0A@@OT@@I@Z 00000001800bc27c     hb-aat-layout.obj
 0002:0003127c       $chain$2$?get_value@?$LookupFormat4@UHBGlyphID16@OT@@@AAT@@AEBAPEBUHBGlyphID16@OT@@I@Z 00000001800bc27c     hb-aat-layout.obj
 0002:0003128c       $chain$3$?get_value@?$LookupFormat4@U?$IntType@G$01@OT@@@AAT@@AEBAPEBU?$IntType@G$01@OT@@I@Z 00000001800bc28c     hb-aat-layout.obj
 0002:0003128c       $chain$3$?get_value@?$LookupFormat4@U?$OffsetTo@U?$ArrayOf@UAnchor@AAT@@U?$IntType@I$03@OT@@@OT@@U?$IntType@G$01@2@$0A@@OT@@@AAT@@AEBAPEBU?$OffsetTo@U?$ArrayOf@UAnchor@AAT@@U?$IntType@I$03@OT@@@OT@@U?$IntType@G$01@2@$0A@@OT@@I@Z 00000001800bc28c     hb-aat-layout.obj
 0002:0003128c       $chain$3$?get_value@?$LookupFormat4@UHBGlyphID16@OT@@@AAT@@AEBAPEBUHBGlyphID16@OT@@I@Z 00000001800bc28c     hb-aat-layout.obj
 0002:0003129c       $unwind$?get_glyph_props@GDEF@OT@@QEBAII@Z 00000001800bc29c     hb-aat-layout.obj
 0002:0003129c       $unwind$?sanitize@?$Chain@UExtendedTypes@AAT@@@AAT@@QEBA_NPEAUhb_sanitize_context_t@@I@Z 00000001800bc29c     hb-aat-layout.obj
 0002:0003129c       $unwind$?sanitize@?$KerxTable@Ukerx@AAT@@@AAT@@QEBA_NPEAUhb_sanitize_context_t@@@Z 00000001800bc29c     hb-aat-layout.obj
 0002:0003129c       $unwind$?sanitize@?$mortmorx@UExtendedTypes@AAT@@$0GNGPHCHI@@AAT@@QEBA_NPEAUhb_sanitize_context_t@@@Z 00000001800bc29c     hb-aat-layout.obj
 0002:0003129c       $unwind$?sanitize@feat@AAT@@QEBA_NPEAUhb_sanitize_context_t@@@Z 00000001800bc29c     hb-aat-layout.obj
 0002:0003129c       $unwind$?push@?$hb_vector_t@Ufeature_event_t@hb_aat_map_builder_t@@$0A@@@QEAAPEAUfeature_event_t@hb_aat_map_builder_t@@XZ 00000001800bc29c     hb-aat-map.obj
 0002:0003129c       $unwind$?push@?$hb_vector_t@Ufeature_range_t@hb_aat_map_builder_t@@$00@@QEAAPEAUfeature_range_t@hb_aat_map_builder_t@@XZ 00000001800bc29c     hb-aat-map.obj
 0002:0003129c       $unwind$hb_blob_create_or_fail 00000001800bc29c     hb-blob.obj
 0002:0003129c       $unwind$?fini@hb_serialize_context_t@@QEAAXXZ 00000001800bc29c     hb-face-builder.obj
 0002:0003129c       $unwind$?sanitize@fvar@OT@@QEBA_NPEAUhb_sanitize_context_t@@@Z 00000001800bc29c     hb-font.obj
 0002:0003129c       $unwind$?sanitize@CBLC@OT@@QEBA_NPEAUhb_sanitize_context_t@@@Z 00000001800bc29c     hb-ot-color.obj
 0002:0003129c       $unwind$?fini@hb_ot_face_t@@QEAAXXZ 00000001800bc29c     hb-ot-face.obj
 0002:0003129c       $unwind$??$dispatch@Uhb_paint_context_t@OT@@$$V@Paint@OT@@QEBA?AUhb_empty_t@@PEAUhb_paint_context_t@1@@Z 00000001800bc29c     hb-ot-font.obj
 0002:0003129c       $unwind$?hb_ot_get_variation_glyph@@YAHPEAUhb_font_t@@PEAXIIPEAI1@Z 00000001800bc29c     hb-ot-font.obj
 0002:0003129c       $unwind$??$sanitize@PEBUChainContextFormat3@OT@@@?$ArrayOf@U?$OffsetTo@UCoverage@Common@Layout@OT@@U?$IntType@G$01@4@$00@OT@@U?$IntType@G$01@2@@OT@@QEBA_NPEAUhb_sanitize_context_t@@$$QEAPEBUChainContextFormat3@1@@Z 00000001800bc29c     hb-ot-layout.obj
 0002:0003129c       $unwind$??$sanitize@PEBUReverseChainSingleSubstFormat1@GSUB_impl@Layout@OT@@@?$ArrayOf@U?$OffsetTo@UCoverage@Common@Layout@OT@@U?$IntType@G$01@4@$00@OT@@U?$IntType@G$01@2@@OT@@QEBA_NPEAUhb_sanitize_context_t@@$$QEAPEBUReverseChainSingleSubstFormat1@GSUB_impl@Layout@1@@Z 00000001800bc29c     hb-ot-layout.obj
 0002:0003129c       $unwind$?apply@?$AlternateSubstFormat1_2@USmallTypes@Layout@OT@@@GSUB_impl@Layout@OT@@QEBA_NPEAUhb_ot_apply_context_t@4@@Z 00000001800bc29c     hb-ot-layout.obj
 0002:0003129c       $unwind$?apply@?$MultipleSubstFormat1_2@USmallTypes@Layout@OT@@@GSUB_impl@Layout@OT@@QEBA_NPEAUhb_ot_apply_context_t@4@@Z 00000001800bc29c     hb-ot-layout.obj
 0002:0003129c       $unwind$?hb_ot_layout_table_find_feature@@YA_NPEAUhb_face_t@@IIPEAI@Z 00000001800bc29c     hb-ot-layout.obj
 0002:0003129c       $unwind$?sanitize@?$KerxTable@UKernAAT@OT@@@AAT@@QEBA_NPEAUhb_sanitize_context_t@@@Z 00000001800bc29c     hb-ot-layout.obj
 0002:0003129c       $unwind$hb_ot_layout_language_get_required_feature 00000001800bc29c     hb-ot-layout.obj
 0002:0003129c       $unwind$hb_ot_layout_script_select_language 00000001800bc29c     hb-ot-layout.obj
 0002:0003129c       $unwind$?_hb_glyph_info_set_unicode_props@@YAXPEAUhb_glyph_info_t@@PEAUhb_buffer_t@@@Z 00000001800bc29c     hb-ot-shape-normalize.obj
 0002:0003129c       $unwind$?_hb_glyph_info_set_unicode_props@@YAXPEAUhb_glyph_info_t@@PEAUhb_buffer_t@@@Z 00000001800bc29c     hb-ot-shape.obj
 0002:0003129c       $unwind$?push@?$hb_vector_t@Ulink_t@object_t@hb_serialize_context_t@@$0A@@@QEAAPEAUlink_t@object_t@hb_serialize_context_t@@XZ 00000001800bc29c     hb-ot-shaper-arabic.obj
 0002:0003129c       $unwind$??1hb_ot_map_t@@QEAA@XZ 00000001800bc29c     hb-shape-plan.obj
 0002:000312b4       $unwind$?get_coverage@?$CoverageFormat2_4@USmallTypes@Layout@OT@@@Common@Layout@OT@@AEBAII@Z 00000001800bc2b4     hb-aat-layout.obj
 0002:000312b4       $unwind$??$bsearch@I@?$SortedArrayOf@UCmapSubtableLongGroup@OT@@U?$IntType@I$03@2@@OT@@QEBAAEBUCmapSubtableLongGroup@1@AEBIAEBU21@@Z 00000001800bc2b4     hb-face.obj
 0002:000312b4       $unwind$?group_get_glyph@CmapSubtableFormat12@OT@@SAIAEBUCmapSubtableLongGroup@2@I@Z 00000001800bc2b4     hb-face.obj
 0002:000312b4       $unwind$?hlineto@?$path_procs_t@Ucff1_path_procs_extents_t@@Ucff1_cs_interp_env_t@CFF@@Ucff1_extents_param_t@@@CFF@@SAXAEAUcff1_cs_interp_env_t@2@AEAUcff1_extents_param_t@@@Z 00000001800bc2b4     hb-ot-cff1-table.obj
 0002:000312b4       $unwind$?vlineto@?$path_procs_t@Ucff1_path_procs_extents_t@@Ucff1_cs_interp_env_t@CFF@@Ucff1_extents_param_t@@@CFF@@SAXAEAUcff1_cs_interp_env_t@2@AEAUcff1_extents_param_t@@@Z 00000001800bc2b4     hb-ot-cff1-table.obj
 0002:000312b4       $unwind$?find_script_index@GSUBGPOS@OT@@QEBA_NIPEAI@Z 00000001800bc2b4     hb-ot-layout.obj
 0002:000312c0       $unwind$?get_class@ClassDef@OT@@QEBAII@Z 00000001800bc2c0     hb-aat-layout.obj
 0002:000312c0       $unwind$?translate@contour_point_vector_t@OT@@QEAAXAEBUcontour_point_t@2@@Z 00000001800bc2c0     hb-common.obj
 0002:000312c0       $unwind$?blend_deltas@?$cff2_cs_interp_env_t@Unumber_t@CFF@@@CFF@@QEBANU?$hb_array_t@$$CBUnumber_t@CFF@@@@@Z 00000001800bc2c0     hb-ot-cff2-table.obj
 0002:000312c0       $unwind$??$collect_coverage@U?$hb_set_digest_combiner_t@U?$hb_set_digest_bits_pattern_t@K$03@@U?$hb_set_digest_combiner_t@U?$hb_set_digest_bits_pattern_t@K$0A@@@U?$hb_set_digest_bits_pattern_t@K$08@@@@@@@Coverage@Common@Layout@OT@@QEBA_NPEAU?$hb_set_digest_combiner_t@U?$hb_set_digest_bits_pattern_t@K$03@@U?$hb_set_digest_combiner_t@U?$hb_set_digest_bits_pattern_t@K$0A@@@U?$hb_set_digest_bits_pattern_t@K$08@@@@@@@Z 00000001800bc2c0     hb-ot-layout.obj
 0002:000312c0       $unwind$?get_population@Coverage@Common@Layout@OT@@QEBAIXZ 00000001800bc2c0     hb-ot-layout.obj
 0002:000312c0       $unwind$?_hb_ot_shape_fallback_mark_position_recategorize_marks@@YAXPEBUhb_ot_shape_plan_t@@PEAUhb_font_t@@PEAUhb_buffer_t@@@Z 00000001800bc2c0     hb-ot-shape-fallback.obj
 0002:000312c8       $chain$0$?get_class@ClassDef@OT@@QEBAII@Z 00000001800bc2c8     hb-aat-layout.obj
 0002:000312dc       $chain$1$?get_class@ClassDef@OT@@QEBAII@Z 00000001800bc2dc     hb-aat-layout.obj
 0002:000312ec       $unwind$?sanitize@VariationStore@OT@@QEBA_NPEAUhb_sanitize_context_t@@@Z 00000001800bc2ec     hb-aat-layout.obj
 0002:000312ec       $unwind$?sanitize@trak@AAT@@QEBA_NPEAUhb_sanitize_context_t@@@Z 00000001800bc2ec     hb-aat-layout.obj
 0002:000312ec       $unwind$?sanitize@VariationSelectorRecord@OT@@QEBA_NPEAUhb_sanitize_context_t@@PEBX@Z 00000001800bc2ec     hb-face.obj
 0002:000312ec       $unwind$??$sanitize@$$V@?$OffsetTo@ULayerList@OT@@U?$IntType@I$03@2@$00@OT@@QEBA_NPEAUhb_sanitize_context_t@@PEBX@Z 00000001800bc2ec     hb-ot-color.obj
 0002:000312ec       $unwind$?sanitize@?$MarkLigPosFormat1_2@USmallTypes@Layout@OT@@@GPOS_impl@Layout@OT@@QEBA_NPEAUhb_sanitize_context_t@@@Z 00000001800bc2ec     hb-ot-layout.obj
 0002:00031300       $unwind$??$sanitize@PEBULigGlyph@OT@@@?$ArrayOf@U?$OffsetTo@UCaretValue@OT@@U?$IntType@G$01@2@$00@OT@@U?$IntType@G$01@2@@OT@@QEBA_NPEAUhb_sanitize_context_t@@$$QEAPEBULigGlyph@1@@Z 00000001800bc300     hb-aat-layout.obj
 0002:00031300       $unwind$??$sanitize@PEBU?$LigatureSet@USmallTypes@Layout@OT@@@GSUB_impl@Layout@OT@@@?$ArrayOf@U?$OffsetTo@U?$Ligature@USmallTypes@Layout@OT@@@GSUB_impl@Layout@OT@@U?$IntType@G$01@4@$00@OT@@U?$IntType@G$01@2@@OT@@QEBA_NPEAUhb_sanitize_context_t@@$$QEAPEBU?$LigatureSet@USmallTypes@Layout@OT@@@GSUB_impl@Layout@1@@Z 00000001800bc300     hb-ot-layout.obj
 0002:00031300       $unwind$??$sanitize@PEBU?$RuleSet@USmallTypes@Layout@OT@@@OT@@@?$ArrayOf@U?$OffsetTo@U?$Rule@USmallTypes@Layout@OT@@@OT@@U?$IntType@G$01@2@$00@OT@@U?$IntType@G$01@2@@OT@@QEBA_NPEAUhb_sanitize_context_t@@$$QEAPEBU?$RuleSet@USmallTypes@Layout@OT@@@1@@Z 00000001800bc300     hb-ot-layout.obj
 0002:00031300       $unwind$?sanitize@Script@OT@@QEBA_NPEAUhb_sanitize_context_t@@PEBURecord_sanitize_closure_t@2@@Z 00000001800bc300     hb-ot-layout.obj
 0002:0003131c       $unwind$?sanitize@MarkGlyphSets@OT@@QEBA_NPEAUhb_sanitize_context_t@@@Z 00000001800bc31c     hb-aat-layout.obj
 0002:00031338       $unwind$?sanitize@?$GDEFVersion1_2@USmallTypes@Layout@OT@@@OT@@QEBA_NPEAUhb_sanitize_context_t@@@Z 00000001800bc338     hb-aat-layout.obj
 0002:00031338       $unwind$?parse_feature_indices@@YA_NPEAPEBDPEBDPEAUhb_feature_t@@@Z 00000001800bc338     hb-common.obj
 0002:00031338       $unwind$?alloc@?$hb_pool_t@Uobject_t@hb_serialize_context_t@@$0CA@@@QEAAPEAUobject_t@hb_serialize_context_t@@XZ 00000001800bc338     hb-face-builder.obj
 0002:00031338       $unwind$??$_dispatch@U?$ChainRule@USmallTypes@Layout@OT@@@OT@@$$V@hb_sanitize_context_t@@AEAA_NAEBU?$ChainRule@USmallTypes@Layout@OT@@@OT@@U?$hb_priority@$00@@@Z 00000001800bc338     hb-ot-layout.obj
 0002:00031348       $unwind$?compile_flags@?$mortmorx@UExtendedTypes@AAT@@$0GNGPHCHI@@AAT@@QEBAXPEBUhb_aat_map_builder_t@@PEAUhb_aat_map_t@@@Z 00000001800bc348     hb-aat-layout.obj
 0002:00031348       $unwind$?compile_flags@?$mortmorx@UObsoleteTypes@AAT@@$0GNGPHCHE@@AAT@@QEBAXPEBUhb_aat_map_builder_t@@PEAUhb_aat_map_t@@@Z 00000001800bc348     hb-aat-layout.obj
 0002:0003135c       $chain$0$?compile_flags@?$mortmorx@UExtendedTypes@AAT@@$0GNGPHCHI@@AAT@@QEBAXPEBUhb_aat_map_builder_t@@PEAUhb_aat_map_t@@@Z 00000001800bc35c     hb-aat-layout.obj
 0002:00031370       $chain$1$?compile_flags@?$mortmorx@UExtendedTypes@AAT@@$0GNGPHCHI@@AAT@@QEBAXPEBUhb_aat_map_builder_t@@PEAUhb_aat_map_t@@@Z 00000001800bc370     hb-aat-layout.obj
 0002:00031384       $chain$2$?compile_flags@?$mortmorx@UExtendedTypes@AAT@@$0GNGPHCHI@@AAT@@QEBAXPEBUhb_aat_map_builder_t@@PEAUhb_aat_map_t@@@Z 00000001800bc384     hb-aat-layout.obj
 0002:00031394       $chain$3$?compile_flags@?$mortmorx@UExtendedTypes@AAT@@$0GNGPHCHI@@AAT@@QEBAXPEBUhb_aat_map_builder_t@@PEAUhb_aat_map_t@@@Z 00000001800bc394     hb-aat-layout.obj
 0002:000313a4       $unwind$?compile_flags@?$Chain@UExtendedTypes@AAT@@@AAT@@QEBAIPEBUhb_aat_map_builder_t@@@Z 00000001800bc3a4     hb-aat-layout.obj
 0002:000313a4       $unwind$?compile_flags@?$Chain@UObsoleteTypes@AAT@@@AAT@@QEBAIPEBUhb_aat_map_builder_t@@@Z 00000001800bc3a4     hb-aat-layout.obj
 0002:000313b0       $chain$5$?compile_flags@?$Chain@UExtendedTypes@AAT@@@AAT@@QEBAIPEBUhb_aat_map_builder_t@@@Z 00000001800bc3b0     hb-aat-layout.obj
 0002:000313d8       $chain$6$?compile_flags@?$Chain@UExtendedTypes@AAT@@@AAT@@QEBAIPEBUhb_aat_map_builder_t@@@Z 00000001800bc3d8     hb-aat-layout.obj
 0002:000313e8       $unwind$?apply@?$Chain@UExtendedTypes@AAT@@@AAT@@QEBAXPEAUhb_aat_apply_context_t@2@@Z 00000001800bc3e8     hb-aat-layout.obj
 0002:000313e8       $unwind$?apply@?$Chain@UObsoleteTypes@AAT@@@AAT@@QEBAXPEAUhb_aat_apply_context_t@2@@Z 00000001800bc3e8     hb-aat-layout.obj
 0002:000313f8       $chain$2$?apply@?$Chain@UExtendedTypes@AAT@@@AAT@@QEBAXPEAUhb_aat_apply_context_t@2@@Z 00000001800bc3f8     hb-aat-layout.obj
 0002:00031414       $chain$3$?apply@?$Chain@UExtendedTypes@AAT@@@AAT@@QEBAXPEAUhb_aat_apply_context_t@2@@Z 00000001800bc414     hb-aat-layout.obj
 0002:00031424       $chain$0$?compile_flags@?$mortmorx@UObsoleteTypes@AAT@@$0GNGPHCHE@@AAT@@QEBAXPEBUhb_aat_map_builder_t@@PEAUhb_aat_map_t@@@Z 00000001800bc424     hb-aat-layout.obj
 0002:00031438       $chain$1$?compile_flags@?$mortmorx@UObsoleteTypes@AAT@@$0GNGPHCHE@@AAT@@QEBAXPEBUhb_aat_map_builder_t@@PEAUhb_aat_map_t@@@Z 00000001800bc438     hb-aat-layout.obj
 0002:0003144c       $chain$2$?compile_flags@?$mortmorx@UObsoleteTypes@AAT@@$0GNGPHCHE@@AAT@@QEBAXPEBUhb_aat_map_builder_t@@PEAUhb_aat_map_t@@@Z 00000001800bc44c     hb-aat-layout.obj
 0002:0003145c       $chain$3$?compile_flags@?$mortmorx@UObsoleteTypes@AAT@@$0GNGPHCHE@@AAT@@QEBAXPEBUhb_aat_map_builder_t@@PEAUhb_aat_map_t@@@Z 00000001800bc45c     hb-aat-layout.obj
 0002:0003146c       $unwind$??$sanitize@$$V@?$OffsetTo@UAttachList@OT@@U?$IntType@G$01@2@$00@OT@@QEBA_NPEAUhb_sanitize_context_t@@PEBX@Z 00000001800bc46c     hb-aat-layout.obj
 0002:0003146c       $unwind$??$sanitize@PEBU?$LookupFormat4@U?$IntType@G$01@OT@@@AAT@@@?$VarSizedBinSearchArrayOf@U?$LookupSegmentArray@U?$IntType@G$01@OT@@@AAT@@@OT@@QEBA_NPEAUhb_sanitize_context_t@@$$QEAPEBU?$LookupFormat4@U?$IntType@G$01@OT@@@AAT@@@Z 00000001800bc46c     hb-aat-layout.obj
 0002:0003146c       $unwind$??$sanitize@PEBU?$LookupFormat4@U?$IntType@I$03@OT@@@AAT@@@?$VarSizedBinSearchArrayOf@U?$LookupSegmentArray@U?$IntType@I$03@OT@@@AAT@@@OT@@QEBA_NPEAUhb_sanitize_context_t@@$$QEAPEBU?$LookupFormat4@U?$IntType@I$03@OT@@@AAT@@@Z 00000001800bc46c     hb-aat-layout.obj
 0002:0003146c       $unwind$??$sanitize@PEBU?$LookupFormat4@UHBGlyphID16@OT@@@AAT@@@?$VarSizedBinSearchArrayOf@U?$LookupSegmentArray@UHBGlyphID16@OT@@@AAT@@@OT@@QEBA_NPEAUhb_sanitize_context_t@@$$QEAPEBU?$LookupFormat4@UHBGlyphID16@OT@@@AAT@@@Z 00000001800bc46c     hb-aat-layout.obj
 0002:0003146c       $unwind$?sanitize@?$mortmorx@UObsoleteTypes@AAT@@$0GNGPHCHE@@AAT@@QEBA_NPEAUhb_sanitize_context_t@@@Z 00000001800bc46c     hb-aat-layout.obj
 0002:0003146c       $unwind$?unpack_deltas@TupleVariationData@OT@@SA_NAEAPEBU?$IntType@E$00@2@AEAU?$hb_vector_t@H$0A@@@PEBU32@@Z 00000001800bc46c     hb-common.obj
 0002:0003146c       $unwind$?sanitize@BitmapSizeTable@OT@@QEBA_NPEAUhb_sanitize_context_t@@PEBX@Z 00000001800bc46c     hb-ot-color.obj
 0002:0003146c       $unwind$?sanitize@?$FDSelect3_4@U?$IntType@G$01@OT@@U?$IntType@E$00@2@@CFF@@QEBA_NPEAUhb_sanitize_context_t@@I@Z 00000001800bc46c     hb-ot-font.obj
 0002:0003146c       $unwind$??$sanitize@$$V@?$OffsetTo@U?$ChainRuleSet@USmallTypes@Layout@OT@@@OT@@U?$IntType@G$01@2@$00@OT@@QEBA_NPEAUhb_sanitize_context_t@@PEBX@Z 00000001800bc46c     hb-ot-layout.obj
 0002:0003146c       $unwind$??$sanitize@$$V@?$OffsetTo@U?$List16OfOffsetTo@UPosLookup@GPOS_impl@Layout@OT@@U?$IntType@G$01@4@@OT@@U?$IntType@G$01@2@$00@OT@@QEBA_NPEAUhb_sanitize_context_t@@PEBX@Z 00000001800bc46c     hb-ot-layout.obj
 0002:0003146c       $unwind$??$sanitize@$$V@?$OffsetTo@U?$List16OfOffsetTo@USubstLookup@GSUB_impl@Layout@OT@@U?$IntType@G$01@4@@OT@@U?$IntType@G$01@2@$00@OT@@QEBA_NPEAUhb_sanitize_context_t@@PEBX@Z 00000001800bc46c     hb-ot-layout.obj
 0002:0003146c       $unwind$??$sanitize@$$V@?$OffsetTo@UConditionSet@OT@@U?$IntType@I$03@2@$00@OT@@QEBA_NPEAUhb_sanitize_context_t@@PEBX@Z 00000001800bc46c     hb-ot-layout.obj
 0002:0003146c       $unwind$hb_ot_layout_language_find_feature 00000001800bc46c     hb-ot-layout.obj
 0002:0003146c       $unwind$hb_ot_layout_table_select_script 00000001800bc46c     hb-ot-layout.obj
 0002:0003146c       $unwind$?add_pause@hb_ot_map_builder_t@@AEAAXIP6A_NPEBUhb_ot_shape_plan_t@@PEAUhb_font_t@@PEAUhb_buffer_t@@@Z@Z 00000001800bc46c     hb-ot-map.obj
 0002:0003146c       $unwind$??$serialize@U?$hb_sorted_array_t@$$CBUHBGlyphID16@OT@@@@$0A@@?$CoverageFormat2_4@USmallTypes@Layout@OT@@@Common@Layout@OT@@AEAA_NPEAUhb_serialize_context_t@@U?$hb_sorted_array_t@$$CBUHBGlyphID16@OT@@@@@Z 00000001800bc46c     hb-ot-shaper-arabic.obj
 0002:00031488       $chain$5$?compile_flags@?$Chain@UObsoleteTypes@AAT@@@AAT@@QEBAIPEBUhb_aat_map_builder_t@@@Z 00000001800bc488     hb-aat-layout.obj
 0002:000314b0       $chain$6$?compile_flags@?$Chain@UObsoleteTypes@AAT@@@AAT@@QEBAIPEBUhb_aat_map_builder_t@@@Z 00000001800bc4b0     hb-aat-layout.obj
 0002:000314c0       $chain$3$?apply@?$Chain@UObsoleteTypes@AAT@@@AAT@@QEBAXPEAUhb_aat_apply_context_t@2@@Z 00000001800bc4c0     hb-aat-layout.obj
 0002:000314e0       $chain$4$?apply@?$Chain@UObsoleteTypes@AAT@@@AAT@@QEBAXPEAUhb_aat_apply_context_t@2@@Z 00000001800bc4e0     hb-aat-layout.obj
 0002:000314f0       $unwind$?sanitize@?$StateTable@UObsoleteTypes@AAT@@UEntryData@?$ContextualSubtable@UObsoleteTypes@AAT@@@2@@AAT@@QEBA_NPEAUhb_sanitize_context_t@@PEAI@Z 00000001800bc4f0     hb-aat-layout.obj
 0002:000314f0       $unwind$?sanitize@?$StateTable@UObsoleteTypes@AAT@@UEntryData@?$InsertionSubtable@UObsoleteTypes@AAT@@@2@@AAT@@QEBA_NPEAUhb_sanitize_context_t@@PEAI@Z 00000001800bc4f0     hb-aat-layout.obj
 0002:000314f0       $unwind$?sanitize@?$StateTable@UObsoleteTypes@AAT@@X@AAT@@QEBA_NPEAUhb_sanitize_context_t@@PEAI@Z 00000001800bc4f0     hb-aat-layout.obj
 0002:00031508       $unwind$?apply@?$NoncontextualSubtable@UExtendedTypes@AAT@@@AAT@@QEBA_NPEAUhb_aat_apply_context_t@2@@Z 00000001800bc508     hb-aat-layout.obj
 0002:00031508       $unwind$?apply@?$NoncontextualSubtable@UObsoleteTypes@AAT@@@AAT@@QEBA_NPEAUhb_aat_apply_context_t@2@@Z 00000001800bc508     hb-aat-layout.obj
 0002:0003151c       $chain$1$?apply@?$NoncontextualSubtable@UExtendedTypes@AAT@@@AAT@@QEBA_NPEAUhb_aat_apply_context_t@2@@Z 00000001800bc51c     hb-aat-layout.obj
 0002:0003151c       $chain$1$?apply@?$NoncontextualSubtable@UObsoleteTypes@AAT@@@AAT@@QEBA_NPEAUhb_aat_apply_context_t@2@@Z 00000001800bc51c     hb-aat-layout.obj
 0002:00031534       $chain$2$?apply@?$NoncontextualSubtable@UExtendedTypes@AAT@@@AAT@@QEBA_NPEAUhb_aat_apply_context_t@2@@Z 00000001800bc534     hb-aat-layout.obj
 0002:00031534       $chain$2$?apply@?$NoncontextualSubtable@UObsoleteTypes@AAT@@@AAT@@QEBA_NPEAUhb_aat_apply_context_t@2@@Z 00000001800bc534     hb-aat-layout.obj
 0002:00031544       $unwind$??0hb_ot_apply_context_t@OT@@QEAA@IPEAUhb_font_t@@PEAUhb_buffer_t@@@Z 00000001800bc544     hb-aat-layout.obj
 0002:00031550       $chain$0$??0hb_ot_apply_context_t@OT@@QEAA@IPEAUhb_font_t@@PEAUhb_buffer_t@@@Z 00000001800bc550     hb-aat-layout.obj
 0002:00031564       $chain$2$??0hb_ot_apply_context_t@OT@@QEAA@IPEAUhb_font_t@@PEAUhb_buffer_t@@@Z 00000001800bc564     hb-aat-layout.obj
 0002:0003157c       $chain$3$??0hb_ot_apply_context_t@OT@@QEAA@IPEAUhb_font_t@@PEAUhb_buffer_t@@@Z 00000001800bc57c     hb-aat-layout.obj
 0002:0003158c       $chain$4$??0hb_ot_apply_context_t@OT@@QEAA@IPEAUhb_font_t@@PEAUhb_buffer_t@@@Z 00000001800bc58c     hb-aat-layout.obj
 0002:0003159c       $chain$3$?get_value@?$Lookup@U?$IntType@I$03@OT@@@AAT@@QEBAPEBU?$IntType@I$03@OT@@II@Z 00000001800bc59c     hb-aat-layout.obj
 0002:000315bc       $chain$5$?get_value@?$Lookup@U?$IntType@I$03@OT@@@AAT@@QEBAPEBU?$IntType@I$03@OT@@II@Z 00000001800bc5bc     hb-aat-layout.obj
 0002:000315d4       $chain$6$?get_value@?$Lookup@U?$IntType@I$03@OT@@@AAT@@QEBAPEBU?$IntType@I$03@OT@@II@Z 00000001800bc5d4     hb-aat-layout.obj
 0002:000315e8       $chain$7$?get_value@?$Lookup@U?$IntType@I$03@OT@@@AAT@@QEBAPEBU?$IntType@I$03@OT@@II@Z 00000001800bc5e8     hb-aat-layout.obj
 0002:000315f8       $chain$8$?get_value@?$Lookup@U?$IntType@I$03@OT@@@AAT@@QEBAPEBU?$IntType@I$03@OT@@II@Z 00000001800bc5f8     hb-aat-layout.obj
 0002:0003160c       $chain$10$?get_value@?$Lookup@U?$IntType@I$03@OT@@@AAT@@QEBAPEBU?$IntType@I$03@OT@@II@Z 00000001800bc60c     hb-aat-layout.obj
 0002:00031630       $chain$11$?get_value@?$Lookup@U?$IntType@I$03@OT@@@AAT@@QEBAPEBU?$IntType@I$03@OT@@II@Z 00000001800bc630     hb-aat-layout.obj
 0002:00031640       $chain$0$?get_value@?$LookupFormat4@U?$IntType@I$03@OT@@@AAT@@AEBAPEBU?$IntType@I$03@OT@@I@Z 00000001800bc640     hb-aat-layout.obj
 0002:00031654       $chain$1$?get_value@?$LookupFormat4@U?$IntType@I$03@OT@@@AAT@@AEBAPEBU?$IntType@I$03@OT@@I@Z 00000001800bc654     hb-aat-layout.obj
 0002:00031668       $chain$2$?get_value@?$LookupFormat4@U?$IntType@I$03@OT@@@AAT@@AEBAPEBU?$IntType@I$03@OT@@I@Z 00000001800bc668     hb-aat-layout.obj
 0002:00031678       $chain$3$?get_value@?$LookupFormat4@U?$IntType@I$03@OT@@@AAT@@AEBAPEBU?$IntType@I$03@OT@@I@Z 00000001800bc678     hb-aat-layout.obj
 0002:00031688       $unwind$?sanitize@?$StateTable@UExtendedTypes@AAT@@UEntryData@?$ContextualSubtable@UExtendedTypes@AAT@@@2@@AAT@@QEBA_NPEAUhb_sanitize_context_t@@PEAI@Z 00000001800bc688     hb-aat-layout.obj
 0002:00031688       $unwind$?sanitize@?$StateTable@UExtendedTypes@AAT@@UEntryData@?$Format1Entry@$00@2@@AAT@@QEBA_NPEAUhb_sanitize_context_t@@PEAI@Z 00000001800bc688     hb-aat-layout.obj
 0002:00031688       $unwind$?sanitize@?$StateTable@UExtendedTypes@AAT@@UEntryData@?$InsertionSubtable@UExtendedTypes@AAT@@@2@@AAT@@QEBA_NPEAUhb_sanitize_context_t@@PEAI@Z 00000001800bc688     hb-aat-layout.obj
 0002:00031688       $unwind$?sanitize@?$StateTable@UExtendedTypes@AAT@@UEntryData@?$KerxSubTableFormat4@UKerxSubTableHeader@AAT@@@2@@AAT@@QEBA_NPEAUhb_sanitize_context_t@@PEAI@Z 00000001800bc688     hb-aat-layout.obj
 0002:00031688       $unwind$?sanitize@?$StateTable@UExtendedTypes@AAT@@UEntryData@?$LigatureEntry@$00@2@@AAT@@QEBA_NPEAUhb_sanitize_context_t@@PEAI@Z 00000001800bc688     hb-aat-layout.obj
 0002:00031688       $unwind$?sanitize@?$StateTable@UExtendedTypes@AAT@@X@AAT@@QEBA_NPEAUhb_sanitize_context_t@@PEAI@Z 00000001800bc688     hb-aat-layout.obj
 0002:000316a0       $unwind$?get_kerning@?$KerxSubTableFormat6@UKerxSubTableHeader@AAT@@@AAT@@QEBAHIIPEAUhb_aat_apply_context_t@2@@Z 00000001800bc6a0     hb-aat-layout.obj
 0002:000316b8       $chain$0$?get_kerning@?$KerxSubTableFormat6@UKerxSubTableHeader@AAT@@@AAT@@QEBAHIIPEAUhb_aat_apply_context_t@2@@Z 00000001800bc6b8     hb-aat-layout.obj
 0002:000316cc       $chain$1$?get_kerning@?$KerxSubTableFormat6@UKerxSubTableHeader@AAT@@@AAT@@QEBAHIIPEAUhb_aat_apply_context_t@2@@Z 00000001800bc6cc     hb-aat-layout.obj
 0002:000316dc       $unwind$?apply@?$KerxTable@Ukerx@AAT@@@AAT@@QEBA_NPEAUhb_aat_apply_context_t@2@@Z 00000001800bc6dc     hb-aat-layout.obj
 0002:000316f4       $chain$0$?apply@?$KerxTable@Ukerx@AAT@@@AAT@@QEBA_NPEAUhb_aat_apply_context_t@2@@Z 00000001800bc6f4     hb-aat-layout.obj
 0002:00031708       $chain$1$?apply@?$KerxTable@Ukerx@AAT@@@AAT@@QEBA_NPEAUhb_aat_apply_context_t@2@@Z 00000001800bc708     hb-aat-layout.obj
 0002:00031718       $unwind$?get_tracking@TrackData@AAT@@QEBAHPEBXM@Z 00000001800bc718     hb-aat-layout.obj
 0002:0003172c       $chain$0$?get_tracking@TrackData@AAT@@QEBAHPEBXM@Z 00000001800bc72c     hb-aat-layout.obj
 0002:00031740       $unwind$?sanitize@TrackData@AAT@@QEBA_NPEAUhb_sanitize_context_t@@PEBX@Z 00000001800bc740     hb-aat-layout.obj
 0002:00031740       $unwind$??$sanitize@PEBUClipList@OT@@@?$ArrayOf@UClipRecord@OT@@U?$IntType@I$03@2@@OT@@QEBA_NPEAUhb_sanitize_context_t@@$$QEAPEBUClipList@1@@Z 00000001800bc740     hb-ot-color.obj
 0002:00031740       $unwind$??$get_extents_without_var_scaled@Uglyf_accelerator_t@OT@@@GlyphHeader@glyf_impl@OT@@QEBA_NPEAUhb_font_t@@AEBUglyf_accelerator_t@2@IPEAUhb_glyph_extents_t@@@Z 00000001800bc740     hb-ot-font.obj
 0002:00031740       $unwind$?add_op@?$parsed_values_t@Udict_val_t@CFF@@@CFF@@QEAAXIAEBUbyte_str_ref_t@2@AEBUdict_val_t@2@@Z 00000001800bc740     hb-ot-font.obj
 0002:00031740       $unwind$?add_op@?$parsed_values_t@Uop_str_t@CFF@@@CFF@@QEAAXIAEBUbyte_str_ref_t@2@AEBUop_str_t@2@@Z 00000001800bc740     hb-ot-font.obj
 0002:00031740       $unwind$?sanitize@?$KerxTable@UKernOT@OT@@@AAT@@QEBA_NPEAUhb_sanitize_context_t@@@Z 00000001800bc740     hb-ot-layout.obj
 0002:0003175c       $unwind$?apply@trak@AAT@@QEBA_NPEAUhb_aat_apply_context_t@2@@Z 00000001800bc75c     hb-aat-layout.obj
 0002:00031774       $unwind$??$dispatch@Uhb_aat_apply_context_t@AAT@@$$V@KerxSubTable@AAT@@QEBA_NPEAUhb_aat_apply_context_t@1@@Z 00000001800bc774     hb-aat-layout.obj
 0002:0003178c       $chain$0$??$dispatch@Uhb_sanitize_context_t@@$$V@?$ChainSubtable@UObsoleteTypes@AAT@@@AAT@@QEBA_NPEAUhb_sanitize_context_t@@@Z 00000001800bc78c     hb-aat-layout.obj
 0002:000317a0       $chain$2$??$dispatch@Uhb_sanitize_context_t@@$$V@?$ChainSubtable@UObsoleteTypes@AAT@@@AAT@@QEBA_NPEAUhb_sanitize_context_t@@@Z 00000001800bc7a0     hb-aat-layout.obj
 0002:000317a0       $chain$4$??$dispatch@Uhb_sanitize_context_t@@$$V@?$ChainSubtable@UObsoleteTypes@AAT@@@AAT@@QEBA_NPEAUhb_sanitize_context_t@@@Z 00000001800bc7a0     hb-aat-layout.obj
 0002:000317b4       $chain$7$??$dispatch@Uhb_sanitize_context_t@@$$V@?$ChainSubtable@UObsoleteTypes@AAT@@@AAT@@QEBA_NPEAUhb_sanitize_context_t@@@Z 00000001800bc7b4     hb-aat-layout.obj
 0002:000317cc       $chain$9$??$dispatch@Uhb_sanitize_context_t@@$$V@?$ChainSubtable@UObsoleteTypes@AAT@@@AAT@@QEBA_NPEAUhb_sanitize_context_t@@@Z 00000001800bc7cc     hb-aat-layout.obj
 0002:000317e4       $chain$10$??$dispatch@Uhb_sanitize_context_t@@$$V@?$ChainSubtable@UObsoleteTypes@AAT@@@AAT@@QEBA_NPEAUhb_sanitize_context_t@@@Z 00000001800bc7e4     hb-aat-layout.obj
 0002:000317f4       $unwind$??$sanitize@$$V@?$OffsetTo@ULigCaretList@OT@@U?$IntType@G$01@2@$00@OT@@QEBA_NPEAUhb_sanitize_context_t@@PEBX@Z 00000001800bc7f4     hb-aat-layout.obj
 0002:000317f4       $unwind$??$sanitize@$$V@?$OffsetTo@URecordListOfScript@OT@@U?$IntType@G$01@2@$00@OT@@QEBA_NPEAUhb_sanitize_context_t@@PEBX@Z 00000001800bc7f4     hb-ot-layout.obj
 0002:00031810       $unwind$??$dispatch@Uhb_aat_apply_context_t@AAT@@$$V@?$ChainSubtable@UExtendedTypes@AAT@@@AAT@@QEBA_NPEAUhb_aat_apply_context_t@1@@Z 00000001800bc810     hb-aat-layout.obj
 0002:00031810       $unwind$??$dispatch@Uhb_aat_apply_context_t@AAT@@$$V@?$ChainSubtable@UObsoleteTypes@AAT@@@AAT@@QEBA_NPEAUhb_aat_apply_context_t@1@@Z 00000001800bc810     hb-aat-layout.obj
 0002:00031828       $unwind$??$sanitize_blob@UGDEF@OT@@@hb_sanitize_context_t@@QEAAPEAUhb_blob_t@@PEAU1@@Z 00000001800bc828     hb-aat-layout.obj
 0002:00031844       $unwind$??$sanitize_blob@Ufeat@AAT@@@hb_sanitize_context_t@@QEAAPEAUhb_blob_t@@PEAU1@@Z 00000001800bc844     hb-aat-layout.obj
 0002:00031844       $unwind$??$sanitize_blob@Ultag@AAT@@@hb_sanitize_context_t@@QEAAPEAUhb_blob_t@@PEAU1@@Z 00000001800bc844     hb-aat-layout.obj
 0002:00031844       $unwind$??$sanitize_blob@Umorx@AAT@@@hb_sanitize_context_t@@QEAAPEAUhb_blob_t@@PEAU1@@Z 00000001800bc844     hb-aat-layout.obj
 0002:00031844       $unwind$??$sanitize_blob@UCBLC@OT@@@hb_sanitize_context_t@@QEAAPEAUhb_blob_t@@PEAU1@@Z 00000001800bc844     hb-ot-color.obj
 0002:00031860       $unwind$??$sanitize_blob@Utrak@AAT@@@hb_sanitize_context_t@@QEAAPEAUhb_blob_t@@PEAU1@@Z 00000001800bc860     hb-aat-layout.obj
 0002:0003187c       $unwind$??$sanitize_blob@Uankr@AAT@@@hb_sanitize_context_t@@QEAAPEAUhb_blob_t@@PEAU1@@Z 00000001800bc87c     hb-aat-layout.obj
 0002:00031898       $unwind$??$sanitize_blob@Ukerx@AAT@@@hb_sanitize_context_t@@QEAAPEAUhb_blob_t@@PEAU1@@Z 00000001800bc898     hb-aat-layout.obj
 0002:00031898       $unwind$??$sanitize_blob@Umort@AAT@@@hb_sanitize_context_t@@QEAAPEAUhb_blob_t@@PEAU1@@Z 00000001800bc898     hb-aat-layout.obj
 0002:00031898       $unwind$??$sanitize_blob@UCOLR@OT@@@hb_sanitize_context_t@@QEAAPEAUhb_blob_t@@PEAU1@@Z 00000001800bc898     hb-ot-color.obj
 0002:000318b0       $unwind$?transition@driver_context_t@?$InsertionSubtable@UExtendedTypes@AAT@@@AAT@@QEAAXPEAU?$StateTableDriver@UExtendedTypes@AAT@@UEntryData@?$InsertionSubtable@UExtendedTypes@AAT@@@2@@3@AEBU?$Entry@UEntryData@?$InsertionSubtable@UExtendedTypes@AAT@@@AAT@@@3@@Z 00000001800bc8b0     hb-aat-layout.obj
 0002:000318b0       $unwind$?transition@driver_context_t@?$InsertionSubtable@UObsoleteTypes@AAT@@@AAT@@QEAAXPEAU?$StateTableDriver@UObsoleteTypes@AAT@@UEntryData@?$InsertionSubtable@UObsoleteTypes@AAT@@@2@@3@AEBU?$Entry@UEntryData@?$InsertionSubtable@UObsoleteTypes@AAT@@@AAT@@@3@@Z 00000001800bc8b0     hb-aat-layout.obj
 0002:000318c8       $unwind$??$drive@Udriver_context_t@?$InsertionSubtable@UExtendedTypes@AAT@@@AAT@@@?$StateTableDriver@UExtendedTypes@AAT@@UEntryData@?$InsertionSubtable@UExtendedTypes@AAT@@@2@@AAT@@QEAAXPEAUdriver_context_t@?$InsertionSubtable@UExtendedTypes@AAT@@@1@PEAUhb_aat_apply_context_t@1@@Z 00000001800bc8c8     hb-aat-layout.obj
 0002:000318d8       $chain$3$??$drive@Udriver_context_t@?$InsertionSubtable@UExtendedTypes@AAT@@@AAT@@@?$StateTableDriver@UExtendedTypes@AAT@@UEntryData@?$InsertionSubtable@UExtendedTypes@AAT@@@2@@AAT@@QEAAXPEAUdriver_context_t@?$InsertionSubtable@UExtendedTypes@AAT@@@1@PEAUhb_aat_apply_context_t@1@@Z 00000001800bc8d8     hb-aat-layout.obj
 0002:000318f8       $chain$4$??$drive@Udriver_context_t@?$InsertionSubtable@UExtendedTypes@AAT@@@AAT@@@?$StateTableDriver@UExtendedTypes@AAT@@UEntryData@?$InsertionSubtable@UExtendedTypes@AAT@@@2@@AAT@@QEAAXPEAUdriver_context_t@?$InsertionSubtable@UExtendedTypes@AAT@@@1@PEAUhb_aat_apply_context_t@1@@Z 00000001800bc8f8     hb-aat-layout.obj
 0002:00031908       $unwind$?transition@driver_context_t@?$LigatureSubtable@UExtendedTypes@AAT@@@AAT@@QEAAXPEAU?$StateTableDriver@UExtendedTypes@AAT@@UEntryData@?$LigatureEntry@$00@2@@3@AEBU?$Entry@UEntryData@?$LigatureEntry@$00@AAT@@@3@@Z 00000001800bc908     hb-aat-layout.obj
 0002:00031908       $unwind$?transition@driver_context_t@?$LigatureSubtable@UObsoleteTypes@AAT@@@AAT@@QEAAXPEAU?$StateTableDriver@UObsoleteTypes@AAT@@X@3@AEBU?$Entry@X@3@@Z 00000001800bc908     hb-aat-layout.obj
 0002:00031908       $unwind$capture_previous_context 00000001800bc908     MSVCRT:gs_report.obj
 0002:00031914       $chain$0$?transition@driver_context_t@?$LigatureSubtable@UExtendedTypes@AAT@@@AAT@@QEAAXPEAU?$StateTableDriver@UExtendedTypes@AAT@@UEntryData@?$LigatureEntry@$00@2@@3@AEBU?$Entry@UEntryData@?$LigatureEntry@$00@AAT@@@3@@Z 00000001800bc914     hb-aat-layout.obj
 0002:00031928       $chain$4$?transition@driver_context_t@?$LigatureSubtable@UExtendedTypes@AAT@@@AAT@@QEAAXPEAU?$StateTableDriver@UExtendedTypes@AAT@@UEntryData@?$LigatureEntry@$00@2@@3@AEBU?$Entry@UEntryData@?$LigatureEntry@$00@AAT@@@3@@Z 00000001800bc928     hb-aat-layout.obj
 0002:00031948       $chain$5$?transition@driver_context_t@?$LigatureSubtable@UExtendedTypes@AAT@@@AAT@@QEAAXPEAU?$StateTableDriver@UExtendedTypes@AAT@@UEntryData@?$LigatureEntry@$00@2@@3@AEBU?$Entry@UEntryData@?$LigatureEntry@$00@AAT@@@3@@Z 00000001800bc948     hb-aat-layout.obj
 0002:00031958       $chain$6$?transition@driver_context_t@?$LigatureSubtable@UExtendedTypes@AAT@@@AAT@@QEAAXPEAU?$StateTableDriver@UExtendedTypes@AAT@@UEntryData@?$LigatureEntry@$00@2@@3@AEBU?$Entry@UEntryData@?$LigatureEntry@$00@AAT@@@3@@Z 00000001800bc958     hb-aat-layout.obj
 0002:00031968       $unwind$??$drive@Udriver_context_t@?$LigatureSubtable@UExtendedTypes@AAT@@@AAT@@@?$StateTableDriver@UExtendedTypes@AAT@@UEntryData@?$LigatureEntry@$00@2@@AAT@@QEAAXPEAUdriver_context_t@?$LigatureSubtable@UExtendedTypes@AAT@@@1@PEAUhb_aat_apply_context_t@1@@Z 00000001800bc968     hb-aat-layout.obj
 0002:00031978       $chain$3$??$drive@Udriver_context_t@?$LigatureSubtable@UExtendedTypes@AAT@@@AAT@@@?$StateTableDriver@UExtendedTypes@AAT@@UEntryData@?$LigatureEntry@$00@2@@AAT@@QEAAXPEAUdriver_context_t@?$LigatureSubtable@UExtendedTypes@AAT@@@1@PEAUhb_aat_apply_context_t@1@@Z 00000001800bc978     hb-aat-layout.obj
 0002:00031998       $chain$4$??$drive@Udriver_context_t@?$LigatureSubtable@UExtendedTypes@AAT@@@AAT@@@?$StateTableDriver@UExtendedTypes@AAT@@UEntryData@?$LigatureEntry@$00@2@@AAT@@QEAAXPEAUdriver_context_t@?$LigatureSubtable@UExtendedTypes@AAT@@@1@PEAUhb_aat_apply_context_t@1@@Z 00000001800bc998     hb-aat-layout.obj
 0002:000319a8       $unwind$?transition@driver_context_t@?$ContextualSubtable@UExtendedTypes@AAT@@@AAT@@QEAAXPEAU?$StateTableDriver@UExtendedTypes@AAT@@UEntryData@?$ContextualSubtable@UExtendedTypes@AAT@@@2@@3@AEBU?$Entry@UEntryData@?$ContextualSubtable@UExtendedTypes@AAT@@@AAT@@@3@@Z 00000001800bc9a8     hb-aat-layout.obj
 0002:000319bc       $chain$1$?transition@driver_context_t@?$ContextualSubtable@UExtendedTypes@AAT@@@AAT@@QEAAXPEAU?$StateTableDriver@UExtendedTypes@AAT@@UEntryData@?$ContextualSubtable@UExtendedTypes@AAT@@@2@@3@AEBU?$Entry@UEntryData@?$ContextualSubtable@UExtendedTypes@AAT@@@AAT@@@3@@Z 00000001800bc9bc     hb-aat-layout.obj
 0002:000319d4       $chain$2$?transition@driver_context_t@?$ContextualSubtable@UExtendedTypes@AAT@@@AAT@@QEAAXPEAU?$StateTableDriver@UExtendedTypes@AAT@@UEntryData@?$ContextualSubtable@UExtendedTypes@AAT@@@2@@3@AEBU?$Entry@UEntryData@?$ContextualSubtable@UExtendedTypes@AAT@@@AAT@@@3@@Z 00000001800bc9d4     hb-aat-layout.obj
 0002:000319e4       $unwind$??$drive@Udriver_context_t@?$ContextualSubtable@UExtendedTypes@AAT@@@AAT@@@?$StateTableDriver@UExtendedTypes@AAT@@UEntryData@?$ContextualSubtable@UExtendedTypes@AAT@@@2@@AAT@@QEAAXPEAUdriver_context_t@?$ContextualSubtable@UExtendedTypes@AAT@@@1@PEAUhb_aat_apply_context_t@1@@Z 00000001800bc9e4     hb-aat-layout.obj
 0002:000319f4       $chain$3$??$drive@Udriver_context_t@?$ContextualSubtable@UExtendedTypes@AAT@@@AAT@@@?$StateTableDriver@UExtendedTypes@AAT@@UEntryData@?$ContextualSubtable@UExtendedTypes@AAT@@@2@@AAT@@QEAAXPEAUdriver_context_t@?$ContextualSubtable@UExtendedTypes@AAT@@@1@PEAUhb_aat_apply_context_t@1@@Z 00000001800bc9f4     hb-aat-layout.obj
 0002:00031a14       $chain$4$??$drive@Udriver_context_t@?$ContextualSubtable@UExtendedTypes@AAT@@@AAT@@@?$StateTableDriver@UExtendedTypes@AAT@@UEntryData@?$ContextualSubtable@UExtendedTypes@AAT@@@2@@AAT@@QEAAXPEAUdriver_context_t@?$ContextualSubtable@UExtendedTypes@AAT@@@1@PEAUhb_aat_apply_context_t@1@@Z 00000001800bca14     hb-aat-layout.obj
 0002:00031a24       $unwind$?transition@driver_context_t@?$RearrangementSubtable@UExtendedTypes@AAT@@@AAT@@QEAAXPEAU?$StateTableDriver@UExtendedTypes@AAT@@X@3@AEBU?$Entry@X@3@@Z 00000001800bca24     hb-aat-layout.obj
 0002:00031a24       $unwind$?transition@driver_context_t@?$RearrangementSubtable@UObsoleteTypes@AAT@@@AAT@@QEAAXPEAU?$StateTableDriver@UObsoleteTypes@AAT@@X@3@AEBU?$Entry@X@3@@Z 00000001800bca24     hb-aat-layout.obj
 0002:00031a3c       $chain$1$?transition@driver_context_t@?$RearrangementSubtable@UExtendedTypes@AAT@@@AAT@@QEAAXPEAU?$StateTableDriver@UExtendedTypes@AAT@@X@3@AEBU?$Entry@X@3@@Z 00000001800bca3c     hb-aat-layout.obj
 0002:00031a3c       $chain$1$?transition@driver_context_t@?$RearrangementSubtable@UObsoleteTypes@AAT@@@AAT@@QEAAXPEAU?$StateTableDriver@UObsoleteTypes@AAT@@X@3@AEBU?$Entry@X@3@@Z 00000001800bca3c     hb-aat-layout.obj
 0002:00031a54       $chain$4$?transition@driver_context_t@?$RearrangementSubtable@UExtendedTypes@AAT@@@AAT@@QEAAXPEAU?$StateTableDriver@UExtendedTypes@AAT@@X@3@AEBU?$Entry@X@3@@Z 00000001800bca54     hb-aat-layout.obj
 0002:00031a54       $chain$4$?transition@driver_context_t@?$RearrangementSubtable@UObsoleteTypes@AAT@@@AAT@@QEAAXPEAU?$StateTableDriver@UObsoleteTypes@AAT@@X@3@AEBU?$Entry@X@3@@Z 00000001800bca54     hb-aat-layout.obj
 0002:00031a70       $chain$5$?transition@driver_context_t@?$RearrangementSubtable@UExtendedTypes@AAT@@@AAT@@QEAAXPEAU?$StateTableDriver@UExtendedTypes@AAT@@X@3@AEBU?$Entry@X@3@@Z 00000001800bca70     hb-aat-layout.obj
 0002:00031a70       $chain$5$?transition@driver_context_t@?$RearrangementSubtable@UObsoleteTypes@AAT@@@AAT@@QEAAXPEAU?$StateTableDriver@UObsoleteTypes@AAT@@X@3@AEBU?$Entry@X@3@@Z 00000001800bca70     hb-aat-layout.obj
 0002:00031a88       $chain$6$?transition@driver_context_t@?$RearrangementSubtable@UExtendedTypes@AAT@@@AAT@@QEAAXPEAU?$StateTableDriver@UExtendedTypes@AAT@@X@3@AEBU?$Entry@X@3@@Z 00000001800bca88     hb-aat-layout.obj
 0002:00031a88       $chain$6$?transition@driver_context_t@?$RearrangementSubtable@UObsoleteTypes@AAT@@@AAT@@QEAAXPEAU?$StateTableDriver@UObsoleteTypes@AAT@@X@3@AEBU?$Entry@X@3@@Z 00000001800bca88     hb-aat-layout.obj
 0002:00031a98       $chain$7$?transition@driver_context_t@?$RearrangementSubtable@UExtendedTypes@AAT@@@AAT@@QEAAXPEAU?$StateTableDriver@UExtendedTypes@AAT@@X@3@AEBU?$Entry@X@3@@Z 00000001800bca98     hb-aat-layout.obj
 0002:00031a98       $chain$7$?transition@driver_context_t@?$RearrangementSubtable@UObsoleteTypes@AAT@@@AAT@@QEAAXPEAU?$StateTableDriver@UObsoleteTypes@AAT@@X@3@AEBU?$Entry@X@3@@Z 00000001800bca98     hb-aat-layout.obj
 0002:00031aa8       $unwind$??$drive@Udriver_context_t@?$RearrangementSubtable@UExtendedTypes@AAT@@@AAT@@@?$StateTableDriver@UExtendedTypes@AAT@@X@AAT@@QEAAXPEAUdriver_context_t@?$RearrangementSubtable@UExtendedTypes@AAT@@@1@PEAUhb_aat_apply_context_t@1@@Z 00000001800bcaa8     hb-aat-layout.obj
 0002:00031ab8       $chain$2$??$drive@Udriver_context_t@?$RearrangementSubtable@UExtendedTypes@AAT@@@AAT@@@?$StateTableDriver@UExtendedTypes@AAT@@X@AAT@@QEAAXPEAUdriver_context_t@?$RearrangementSubtable@UExtendedTypes@AAT@@@1@PEAUhb_aat_apply_context_t@1@@Z 00000001800bcab8     hb-aat-layout.obj
 0002:00031ad4       $chain$3$??$drive@Udriver_context_t@?$RearrangementSubtable@UExtendedTypes@AAT@@@AAT@@@?$StateTableDriver@UExtendedTypes@AAT@@X@AAT@@QEAAXPEAUdriver_context_t@?$RearrangementSubtable@UExtendedTypes@AAT@@@1@PEAUhb_aat_apply_context_t@1@@Z 00000001800bcad4     hb-aat-layout.obj
 0002:00031ae4       $unwind$?kern@?$hb_kern_machine_t@Uaccelerator_t@?$KerxSubTableFormat0@UKerxSubTableHeader@AAT@@@AAT@@@OT@@QEBAXPEAUhb_font_t@@PEAUhb_buffer_t@@I_N@Z 00000001800bcae4     hb-aat-layout.obj
 0002:00031ae4       $unwind$?kern@?$hb_kern_machine_t@Uaccelerator_t@?$KerxSubTableFormat2@UKerxSubTableHeader@AAT@@@AAT@@@OT@@QEBAXPEAUhb_font_t@@PEAUhb_buffer_t@@I_N@Z 00000001800bcae4     hb-aat-layout.obj
 0002:00031ae4       $unwind$?kern@?$hb_kern_machine_t@Uaccelerator_t@?$KerxSubTableFormat6@UKerxSubTableHeader@AAT@@@AAT@@@OT@@QEBAXPEAUhb_font_t@@PEAUhb_buffer_t@@I_N@Z 00000001800bcae4     hb-aat-layout.obj
 0002:00031ae4       $unwind$?kern@?$hb_kern_machine_t@Uaccelerator_t@?$KerxSubTableFormat0@UKernAATSubTableHeader@OT@@@AAT@@@OT@@QEBAXPEAUhb_font_t@@PEAUhb_buffer_t@@I_N@Z 00000001800bcae4     hb-ot-layout.obj
 0002:00031ae4       $unwind$?kern@?$hb_kern_machine_t@Uaccelerator_t@?$KerxSubTableFormat0@UKernOTSubTableHeader@OT@@@AAT@@@OT@@QEBAXPEAUhb_font_t@@PEAUhb_buffer_t@@I_N@Z 00000001800bcae4     hb-ot-layout.obj
 0002:00031ae4       $unwind$?kern@?$hb_kern_machine_t@Uaccelerator_t@?$KerxSubTableFormat2@UKernAATSubTableHeader@OT@@@AAT@@@OT@@QEBAXPEAUhb_font_t@@PEAUhb_buffer_t@@I_N@Z 00000001800bcae4     hb-ot-layout.obj
 0002:00031ae4       $unwind$?kern@?$hb_kern_machine_t@Uaccelerator_t@?$KerxSubTableFormat2@UKernOTSubTableHeader@OT@@@AAT@@@OT@@QEBAXPEAUhb_font_t@@PEAUhb_buffer_t@@I_N@Z 00000001800bcae4     hb-ot-layout.obj
 0002:00031af4       $chain$1$?kern@?$hb_kern_machine_t@Uaccelerator_t@?$KerxSubTableFormat6@UKerxSubTableHeader@AAT@@@AAT@@@OT@@QEBAXPEAUhb_font_t@@PEAUhb_buffer_t@@I_N@Z 00000001800bcaf4     hb-aat-layout.obj
 0002:00031b0c       $chain$3$?kern@?$hb_kern_machine_t@Uaccelerator_t@?$KerxSubTableFormat6@UKerxSubTableHeader@AAT@@@AAT@@@OT@@QEBAXPEAUhb_font_t@@PEAUhb_buffer_t@@I_N@Z 00000001800bcb0c     hb-aat-layout.obj
 0002:00031b24       $chain$4$?kern@?$hb_kern_machine_t@Uaccelerator_t@?$KerxSubTableFormat6@UKerxSubTableHeader@AAT@@@AAT@@@OT@@QEBAXPEAUhb_font_t@@PEAUhb_buffer_t@@I_N@Z 00000001800bcb24     hb-aat-layout.obj
 0002:00031b34       $chain$5$?kern@?$hb_kern_machine_t@Uaccelerator_t@?$KerxSubTableFormat6@UKerxSubTableHeader@AAT@@@AAT@@@OT@@QEBAXPEAUhb_font_t@@PEAUhb_buffer_t@@I_N@Z 00000001800bcb34     hb-aat-layout.obj
 0002:00031b44       $unwind$?transition@driver_context_t@?$KerxSubTableFormat4@UKerxSubTableHeader@AAT@@@AAT@@QEAAXPEAU?$StateTableDriver@UExtendedTypes@AAT@@UEntryData@?$KerxSubTableFormat4@UKerxSubTableHeader@AAT@@@2@@3@AEBU?$Entry@UEntryData@?$KerxSubTableFormat4@UKerxSubTableHeader@AAT@@@AAT@@@3@@Z 00000001800bcb44     hb-aat-layout.obj
 0002:00031b5c       $unwind$??$drive@Udriver_context_t@?$KerxSubTableFormat1@UKerxSubTableHeader@AAT@@@AAT@@@?$StateTableDriver@UExtendedTypes@AAT@@UEntryData@?$Format1Entry@$00@2@@AAT@@QEAAXPEAUdriver_context_t@?$KerxSubTableFormat1@UKerxSubTableHeader@AAT@@@1@PEAUhb_aat_apply_context_t@1@@Z 00000001800bcb5c     hb-aat-layout.obj
 0002:00031b5c       $unwind$??$drive@Udriver_context_t@?$KerxSubTableFormat4@UKerxSubTableHeader@AAT@@@AAT@@@?$StateTableDriver@UExtendedTypes@AAT@@UEntryData@?$KerxSubTableFormat4@UKerxSubTableHeader@AAT@@@2@@AAT@@QEAAXPEAUdriver_context_t@?$KerxSubTableFormat4@UKerxSubTableHeader@AAT@@@1@PEAUhb_aat_apply_context_t@1@@Z 00000001800bcb5c     hb-aat-layout.obj
 0002:00031b6c       $chain$3$??$drive@Udriver_context_t@?$KerxSubTableFormat4@UKerxSubTableHeader@AAT@@@AAT@@@?$StateTableDriver@UExtendedTypes@AAT@@UEntryData@?$KerxSubTableFormat4@UKerxSubTableHeader@AAT@@@2@@AAT@@QEAAXPEAUdriver_context_t@?$KerxSubTableFormat4@UKerxSubTableHeader@AAT@@@1@PEAUhb_aat_apply_context_t@1@@Z 00000001800bcb6c     hb-aat-layout.obj
 0002:00031b8c       $chain$4$??$drive@Udriver_context_t@?$KerxSubTableFormat4@UKerxSubTableHeader@AAT@@@AAT@@@?$StateTableDriver@UExtendedTypes@AAT@@UEntryData@?$KerxSubTableFormat4@UKerxSubTableHeader@AAT@@@2@@AAT@@QEAAXPEAUdriver_context_t@?$KerxSubTableFormat4@UKerxSubTableHeader@AAT@@@1@PEAUhb_aat_apply_context_t@1@@Z 00000001800bcb8c     hb-aat-layout.obj
 0002:00031b9c       $chain$1$?kern@?$hb_kern_machine_t@Uaccelerator_t@?$KerxSubTableFormat2@UKerxSubTableHeader@AAT@@@AAT@@@OT@@QEBAXPEAUhb_font_t@@PEAUhb_buffer_t@@I_N@Z 00000001800bcb9c     hb-aat-layout.obj
 0002:00031bb4       $chain$3$?kern@?$hb_kern_machine_t@Uaccelerator_t@?$KerxSubTableFormat2@UKerxSubTableHeader@AAT@@@AAT@@@OT@@QEBAXPEAUhb_font_t@@PEAUhb_buffer_t@@I_N@Z 00000001800bcbb4     hb-aat-layout.obj
 0002:00031bcc       $chain$4$?kern@?$hb_kern_machine_t@Uaccelerator_t@?$KerxSubTableFormat2@UKerxSubTableHeader@AAT@@@AAT@@@OT@@QEBAXPEAUhb_font_t@@PEAUhb_buffer_t@@I_N@Z 00000001800bcbcc     hb-aat-layout.obj
 0002:00031bdc       $chain$5$?kern@?$hb_kern_machine_t@Uaccelerator_t@?$KerxSubTableFormat2@UKerxSubTableHeader@AAT@@@AAT@@@OT@@QEBAXPEAUhb_font_t@@PEAUhb_buffer_t@@I_N@Z 00000001800bcbdc     hb-aat-layout.obj
 0002:00031bec       $unwind$?transition@driver_context_t@?$KerxSubTableFormat1@UKerxSubTableHeader@AAT@@@AAT@@QEAAXPEAU?$StateTableDriver@UExtendedTypes@AAT@@UEntryData@?$Format1Entry@$00@2@@3@AEBU?$Entry@UEntryData@?$Format1Entry@$00@AAT@@@3@@Z 00000001800bcbec     hb-aat-layout.obj
 0002:00031bfc       $chain$3$?transition@driver_context_t@?$KerxSubTableFormat1@UKerxSubTableHeader@AAT@@@AAT@@QEAAXPEAU?$StateTableDriver@UExtendedTypes@AAT@@UEntryData@?$Format1Entry@$00@2@@3@AEBU?$Entry@UEntryData@?$Format1Entry@$00@AAT@@@3@@Z 00000001800bcbfc     hb-aat-layout.obj
 0002:00031c1c       $chain$4$?transition@driver_context_t@?$KerxSubTableFormat1@UKerxSubTableHeader@AAT@@@AAT@@QEAAXPEAU?$StateTableDriver@UExtendedTypes@AAT@@UEntryData@?$Format1Entry@$00@2@@3@AEBU?$Entry@UEntryData@?$Format1Entry@$00@AAT@@@3@@Z 00000001800bcc1c     hb-aat-layout.obj
 0002:00031c2c       $chain$3$??$drive@Udriver_context_t@?$KerxSubTableFormat1@UKerxSubTableHeader@AAT@@@AAT@@@?$StateTableDriver@UExtendedTypes@AAT@@UEntryData@?$Format1Entry@$00@2@@AAT@@QEAAXPEAUdriver_context_t@?$KerxSubTableFormat1@UKerxSubTableHeader@AAT@@@1@PEAUhb_aat_apply_context_t@1@@Z 00000001800bcc2c     hb-aat-layout.obj
 0002:00031c4c       $chain$4$??$drive@Udriver_context_t@?$KerxSubTableFormat1@UKerxSubTableHeader@AAT@@@AAT@@@?$StateTableDriver@UExtendedTypes@AAT@@UEntryData@?$Format1Entry@$00@2@@AAT@@QEAAXPEAUdriver_context_t@?$KerxSubTableFormat1@UKerxSubTableHeader@AAT@@@1@PEAUhb_aat_apply_context_t@1@@Z 00000001800bcc4c     hb-aat-layout.obj
 0002:00031c5c       $chain$1$?kern@?$hb_kern_machine_t@Uaccelerator_t@?$KerxSubTableFormat0@UKerxSubTableHeader@AAT@@@AAT@@@OT@@QEBAXPEAUhb_font_t@@PEAUhb_buffer_t@@I_N@Z 00000001800bcc5c     hb-aat-layout.obj
 0002:00031c74       $chain$3$?kern@?$hb_kern_machine_t@Uaccelerator_t@?$KerxSubTableFormat0@UKerxSubTableHeader@AAT@@@AAT@@@OT@@QEBAXPEAUhb_font_t@@PEAUhb_buffer_t@@I_N@Z 00000001800bcc74     hb-aat-layout.obj
 0002:00031c8c       $chain$4$?kern@?$hb_kern_machine_t@Uaccelerator_t@?$KerxSubTableFormat0@UKerxSubTableHeader@AAT@@@AAT@@@OT@@QEBAXPEAUhb_font_t@@PEAUhb_buffer_t@@I_N@Z 00000001800bcc8c     hb-aat-layout.obj
 0002:00031c9c       $chain$5$?kern@?$hb_kern_machine_t@Uaccelerator_t@?$KerxSubTableFormat0@UKerxSubTableHeader@AAT@@@AAT@@@OT@@QEBAXPEAUhb_font_t@@PEAUhb_buffer_t@@I_N@Z 00000001800bcc9c     hb-aat-layout.obj
 0002:00031cac       $unwind$??$drive@Udriver_context_t@?$InsertionSubtable@UObsoleteTypes@AAT@@@AAT@@@?$StateTableDriver@UObsoleteTypes@AAT@@UEntryData@?$InsertionSubtable@UObsoleteTypes@AAT@@@2@@AAT@@QEAAXPEAUdriver_context_t@?$InsertionSubtable@UObsoleteTypes@AAT@@@1@PEAUhb_aat_apply_context_t@1@@Z 00000001800bccac     hb-aat-layout.obj
 0002:00031cbc       $chain$3$??$drive@Udriver_context_t@?$InsertionSubtable@UObsoleteTypes@AAT@@@AAT@@@?$StateTableDriver@UObsoleteTypes@AAT@@UEntryData@?$InsertionSubtable@UObsoleteTypes@AAT@@@2@@AAT@@QEAAXPEAUdriver_context_t@?$InsertionSubtable@UObsoleteTypes@AAT@@@1@PEAUhb_aat_apply_context_t@1@@Z 00000001800bccbc     hb-aat-layout.obj
 0002:00031cdc       $chain$4$??$drive@Udriver_context_t@?$InsertionSubtable@UObsoleteTypes@AAT@@@AAT@@@?$StateTableDriver@UObsoleteTypes@AAT@@UEntryData@?$InsertionSubtable@UObsoleteTypes@AAT@@@2@@AAT@@QEAAXPEAUdriver_context_t@?$InsertionSubtable@UObsoleteTypes@AAT@@@1@PEAUhb_aat_apply_context_t@1@@Z 00000001800bccdc     hb-aat-layout.obj
 0002:00031cec       $chain$0$?transition@driver_context_t@?$LigatureSubtable@UObsoleteTypes@AAT@@@AAT@@QEAAXPEAU?$StateTableDriver@UObsoleteTypes@AAT@@X@3@AEBU?$Entry@X@3@@Z 00000001800bccec     hb-aat-layout.obj
 0002:00031d00       $chain$4$?transition@driver_context_t@?$LigatureSubtable@UObsoleteTypes@AAT@@@AAT@@QEAAXPEAU?$StateTableDriver@UObsoleteTypes@AAT@@X@3@AEBU?$Entry@X@3@@Z 00000001800bcd00     hb-aat-layout.obj
 0002:00031d20       $chain$5$?transition@driver_context_t@?$LigatureSubtable@UObsoleteTypes@AAT@@@AAT@@QEAAXPEAU?$StateTableDriver@UObsoleteTypes@AAT@@X@3@AEBU?$Entry@X@3@@Z 00000001800bcd20     hb-aat-layout.obj
 0002:00031d30       $chain$6$?transition@driver_context_t@?$LigatureSubtable@UObsoleteTypes@AAT@@@AAT@@QEAAXPEAU?$StateTableDriver@UObsoleteTypes@AAT@@X@3@AEBU?$Entry@X@3@@Z 00000001800bcd30     hb-aat-layout.obj
 0002:00031d40       $unwind$??$drive@Udriver_context_t@?$LigatureSubtable@UObsoleteTypes@AAT@@@AAT@@@?$StateTableDriver@UObsoleteTypes@AAT@@X@AAT@@QEAAXPEAUdriver_context_t@?$LigatureSubtable@UObsoleteTypes@AAT@@@1@PEAUhb_aat_apply_context_t@1@@Z 00000001800bcd40     hb-aat-layout.obj
 0002:00031d40       $unwind$??$drive@Udriver_context_t@?$KerxSubTableFormat1@UKernAATSubTableHeader@OT@@@AAT@@@?$StateTableDriver@UObsoleteTypes@AAT@@X@AAT@@QEAAXPEAUdriver_context_t@?$KerxSubTableFormat1@UKernAATSubTableHeader@OT@@@1@PEAUhb_aat_apply_context_t@1@@Z 00000001800bcd40     hb-ot-layout.obj
 0002:00031d50       $chain$3$??$drive@Udriver_context_t@?$LigatureSubtable@UObsoleteTypes@AAT@@@AAT@@@?$StateTableDriver@UObsoleteTypes@AAT@@X@AAT@@QEAAXPEAUdriver_context_t@?$LigatureSubtable@UObsoleteTypes@AAT@@@1@PEAUhb_aat_apply_context_t@1@@Z 00000001800bcd50     hb-aat-layout.obj
 0002:00031d70       $chain$4$??$drive@Udriver_context_t@?$LigatureSubtable@UObsoleteTypes@AAT@@@AAT@@@?$StateTableDriver@UObsoleteTypes@AAT@@X@AAT@@QEAAXPEAUdriver_context_t@?$LigatureSubtable@UObsoleteTypes@AAT@@@1@PEAUhb_aat_apply_context_t@1@@Z 00000001800bcd70     hb-aat-layout.obj
 0002:00031d80       $unwind$??$drive@Udriver_context_t@?$ContextualSubtable@UObsoleteTypes@AAT@@@AAT@@@?$StateTableDriver@UObsoleteTypes@AAT@@UEntryData@?$ContextualSubtable@UObsoleteTypes@AAT@@@2@@AAT@@QEAAXPEAUdriver_context_t@?$ContextualSubtable@UObsoleteTypes@AAT@@@1@PEAUhb_aat_apply_context_t@1@@Z 00000001800bcd80     hb-aat-layout.obj
 0002:00031d90       $chain$2$??$drive@Udriver_context_t@?$ContextualSubtable@UObsoleteTypes@AAT@@@AAT@@@?$StateTableDriver@UObsoleteTypes@AAT@@UEntryData@?$ContextualSubtable@UObsoleteTypes@AAT@@@2@@AAT@@QEAAXPEAUdriver_context_t@?$ContextualSubtable@UObsoleteTypes@AAT@@@1@PEAUhb_aat_apply_context_t@1@@Z 00000001800bcd90     hb-aat-layout.obj
 0002:00031dac       $chain$3$??$drive@Udriver_context_t@?$ContextualSubtable@UObsoleteTypes@AAT@@@AAT@@@?$StateTableDriver@UObsoleteTypes@AAT@@UEntryData@?$ContextualSubtable@UObsoleteTypes@AAT@@@2@@AAT@@QEAAXPEAUdriver_context_t@?$ContextualSubtable@UObsoleteTypes@AAT@@@1@PEAUhb_aat_apply_context_t@1@@Z 00000001800bcdac     hb-aat-layout.obj
 0002:00031dbc       $unwind$??$drive@Udriver_context_t@?$RearrangementSubtable@UObsoleteTypes@AAT@@@AAT@@@?$StateTableDriver@UObsoleteTypes@AAT@@X@AAT@@QEAAXPEAUdriver_context_t@?$RearrangementSubtable@UObsoleteTypes@AAT@@@1@PEAUhb_aat_apply_context_t@1@@Z 00000001800bcdbc     hb-aat-layout.obj
 0002:00031dcc       $chain$2$??$drive@Udriver_context_t@?$RearrangementSubtable@UObsoleteTypes@AAT@@@AAT@@@?$StateTableDriver@UObsoleteTypes@AAT@@X@AAT@@QEAAXPEAUdriver_context_t@?$RearrangementSubtable@UObsoleteTypes@AAT@@@1@PEAUhb_aat_apply_context_t@1@@Z 00000001800bcdcc     hb-aat-layout.obj
 0002:00031de8       $chain$3$??$drive@Udriver_context_t@?$RearrangementSubtable@UObsoleteTypes@AAT@@@AAT@@@?$StateTableDriver@UObsoleteTypes@AAT@@X@AAT@@QEAAXPEAUdriver_context_t@?$RearrangementSubtable@UObsoleteTypes@AAT@@@1@PEAUhb_aat_apply_context_t@1@@Z 00000001800bcde8     hb-aat-layout.obj
 0002:00031df8       $unwind$??$sanitize@AEAPEBX@?$UnsizedArrayOf@U?$OffsetTo@U?$ArrayOf@UAnchor@AAT@@U?$IntType@I$03@OT@@@OT@@U?$IntType@G$01@2@$0A@@OT@@@OT@@QEBA_NPEAUhb_sanitize_context_t@@IAEAPEBX@Z 00000001800bcdf8     hb-aat-layout.obj
 0002:00031df8       $unwind$?sanitize@CPAL@OT@@QEBA_NPEAUhb_sanitize_context_t@@@Z 00000001800bcdf8     hb-ot-color.obj
 0002:00031e10       $unwind$??$sanitize@PEBU?$LookupFormat4@U?$OffsetTo@U?$ArrayOf@UAnchor@AAT@@U?$IntType@I$03@OT@@@OT@@U?$IntType@G$01@2@$0A@@OT@@@AAT@@AEAPEBX@?$VarSizedBinSearchArrayOf@U?$LookupSegmentArray@U?$OffsetTo@U?$ArrayOf@UAnchor@AAT@@U?$IntType@I$03@OT@@@OT@@U?$IntType@G$01@2@$0A@@OT@@@AAT@@@OT@@QEBA_NPEAUhb_sanitize_context_t@@$$QEAPEBU?$LookupFormat4@U?$OffsetTo@U?$ArrayOf@UAnchor@AAT@@U?$IntType@I$03@OT@@@OT@@U?$IntType@G$01@2@$0A@@OT@@@AAT@@AEAPEBX@Z 00000001800bce10     hb-aat-layout.obj
 0002:00031e28       $unwind$??$dispatch@Uhb_sanitize_context_t@@$$V@?$ChainSubtable@UExtendedTypes@AAT@@@AAT@@QEBA_NPEAUhb_sanitize_context_t@@@Z 00000001800bce28     hb-aat-layout.obj
 0002:00031e28       $unwind$?alloc@?$hb_vector_t@Ufeature_info_t@hb_aat_map_builder_t@@$00@@QEAA_NI_N@Z 00000001800bce28     hb-aat-map.obj
 0002:00031e28       $unwind$?alloc@?$hb_vector_t@Ucontour_point_t@OT@@$0A@@@QEAA_NI_N@Z 00000001800bce28     hb-common.obj
 0002:00031e28       $unwind$??$dispatch@Uhb_accelerate_subtables_context_t@OT@@$$V@ChainContext@OT@@QEBA?AUhb_empty_t@@PEAUhb_accelerate_subtables_context_t@1@@Z 00000001800bce28     hb-ot-layout.obj
 0002:00031e28       $unwind$?alloc@?$hb_vector_t@Ufeature_info_t@hb_ot_map_builder_t@@$0A@@@QEAA_NI_N@Z 00000001800bce28     hb-ot-map.obj
 0002:00031e28       $unwind$?alloc@?$hb_vector_t@Ulookup_map_t@hb_ot_map_t@@$0A@@@QEAA_NI_N@Z 00000001800bce28     hb-ot-map.obj
 0002:00031e30       $chain$0$??$dispatch@Uhb_sanitize_context_t@@$$V@?$ChainSubtable@UExtendedTypes@AAT@@@AAT@@QEBA_NPEAUhb_sanitize_context_t@@@Z 00000001800bce30     hb-aat-layout.obj
 0002:00031e44       $chain$2$??$dispatch@Uhb_sanitize_context_t@@$$V@?$ChainSubtable@UExtendedTypes@AAT@@@AAT@@QEBA_NPEAUhb_sanitize_context_t@@@Z 00000001800bce44     hb-aat-layout.obj
 0002:00031e44       $chain$4$??$dispatch@Uhb_sanitize_context_t@@$$V@?$ChainSubtable@UExtendedTypes@AAT@@@AAT@@QEBA_NPEAUhb_sanitize_context_t@@@Z 00000001800bce44     hb-aat-layout.obj
 0002:00031e58       $chain$7$??$dispatch@Uhb_sanitize_context_t@@$$V@?$ChainSubtable@UExtendedTypes@AAT@@@AAT@@QEBA_NPEAUhb_sanitize_context_t@@@Z 00000001800bce58     hb-aat-layout.obj
 0002:00031e70       $chain$10$??$dispatch@Uhb_sanitize_context_t@@$$V@?$ChainSubtable@UExtendedTypes@AAT@@@AAT@@QEBA_NPEAUhb_sanitize_context_t@@@Z 00000001800bce70     hb-aat-layout.obj
 0002:00031e8c       $chain$12$??$dispatch@Uhb_sanitize_context_t@@$$V@?$ChainSubtable@UExtendedTypes@AAT@@@AAT@@QEBA_NPEAUhb_sanitize_context_t@@@Z 00000001800bce8c     hb-aat-layout.obj
 0002:00031ea8       $chain$13$??$dispatch@Uhb_sanitize_context_t@@$$V@?$ChainSubtable@UExtendedTypes@AAT@@@AAT@@QEBA_NPEAUhb_sanitize_context_t@@@Z 00000001800bcea8     hb-aat-layout.obj
 0002:00031eb8       $unwind$??$sanitize@$$V@?$UnsizedListOfOffset16To@U?$Lookup@UHBGlyphID16@OT@@@AAT@@U?$IntType@G$01@OT@@$0A@@OT@@QEBA_NPEAUhb_sanitize_context_t@@I@Z 00000001800bceb8     hb-aat-layout.obj
 0002:00031ec8       $chain$1$??$sanitize@$$V@?$UnsizedListOfOffset16To@U?$Lookup@UHBGlyphID16@OT@@@AAT@@U?$IntType@G$01@OT@@$0A@@OT@@QEBA_NPEAUhb_sanitize_context_t@@I@Z 00000001800bcec8     hb-aat-layout.obj
 0002:00031ee0       $chain$3$??$sanitize@$$V@?$UnsizedListOfOffset16To@U?$Lookup@UHBGlyphID16@OT@@@AAT@@U?$IntType@G$01@OT@@$0A@@OT@@QEBA_NPEAUhb_sanitize_context_t@@I@Z 00000001800bcee0     hb-aat-layout.obj
 0002:00031ef8       $chain$4$??$sanitize@$$V@?$UnsizedListOfOffset16To@U?$Lookup@UHBGlyphID16@OT@@@AAT@@U?$IntType@G$01@OT@@$0A@@OT@@QEBA_NPEAUhb_sanitize_context_t@@I@Z 00000001800bcef8     hb-aat-layout.obj
 0002:00031f08       $unwind$??$sanitize@$$V@?$UnsizedListOfOffset16To@U?$Lookup@UHBGlyphID16@OT@@@AAT@@U?$IntType@I$03@OT@@$0A@@OT@@QEBA_NPEAUhb_sanitize_context_t@@I@Z 00000001800bcf08     hb-aat-layout.obj
 0002:00031f14       $chain$2$??$sanitize@$$V@?$UnsizedListOfOffset16To@U?$Lookup@UHBGlyphID16@OT@@@AAT@@U?$IntType@I$03@OT@@$0A@@OT@@QEBA_NPEAUhb_sanitize_context_t@@I@Z 00000001800bcf14     hb-aat-layout.obj
 0002:00031f30       $chain$4$??$sanitize@$$V@?$UnsizedListOfOffset16To@U?$Lookup@UHBGlyphID16@OT@@@AAT@@U?$IntType@I$03@OT@@$0A@@OT@@QEBA_NPEAUhb_sanitize_context_t@@I@Z 00000001800bcf30     hb-aat-layout.obj
 0002:00031f4c       $chain$5$??$sanitize@$$V@?$UnsizedListOfOffset16To@U?$Lookup@UHBGlyphID16@OT@@@AAT@@U?$IntType@I$03@OT@@$0A@@OT@@QEBA_NPEAUhb_sanitize_context_t@@I@Z 00000001800bcf4c     hb-aat-layout.obj
 0002:00031f5c       $unwind$??$sort_r_simple@$$V@@YAXPEAX_K1P6AHPEBX2@Z@Z 00000001800bcf5c     hb-aat-map.obj
 0002:00031f5c       $unwind$??$sort_r_simple@$$V@@YAXPEAX_K1P6AHPEBX2@Z@Z 00000001800bcf5c     hb-ot-font.obj
 0002:00031f5c       $unwind$??$sort_r_simple@$$V@@YAXPEAX_K1P6AHPEBX2@Z@Z 00000001800bcf5c     hb-ot-map.obj
 0002:00031f70       $chain$0$??$sort_r_simple@$$V@@YAXPEAX_K1P6AHPEBX2@Z@Z 00000001800bcf70     hb-aat-map.obj
 0002:00031f70       $chain$0$??$sort_r_simple@$$V@@YAXPEAX_K1P6AHPEBX2@Z@Z 00000001800bcf70     hb-ot-font.obj
 0002:00031f70       $chain$0$??$sort_r_simple@$$V@@YAXPEAX_K1P6AHPEBX2@Z@Z 00000001800bcf70     hb-ot-map.obj
 0002:00031f84       $chain$1$??$sort_r_simple@$$V@@YAXPEAX_K1P6AHPEBX2@Z@Z 00000001800bcf84     hb-aat-map.obj
 0002:00031f84       $chain$1$??$sort_r_simple@$$V@@YAXPEAX_K1P6AHPEBX2@Z@Z 00000001800bcf84     hb-ot-font.obj
 0002:00031f84       $chain$1$??$sort_r_simple@$$V@@YAXPEAX_K1P6AHPEBX2@Z@Z 00000001800bcf84     hb-ot-map.obj
 0002:00031f94       $unwind$?add_feature@hb_aat_map_builder_t@@QEAAXAEBUhb_feature_t@@@Z 00000001800bcf94     hb-aat-map.obj
 0002:00031f94       $unwind$?_hb_options_init@@YAXXZ 00000001800bcf94     hb-common.obj
 0002:00031fa0       $chain$0$?add_feature@hb_aat_map_builder_t@@QEAAXAEBUhb_feature_t@@@Z 00000001800bcfa0     hb-aat-map.obj
 0002:00031fb4       $chain$3$?add_feature@hb_aat_map_builder_t@@QEAAXAEBUhb_feature_t@@@Z 00000001800bcfb4     hb-aat-map.obj
 0002:00031fc8       $chain$4$?add_feature@hb_aat_map_builder_t@@QEAAXAEBUhb_feature_t@@@Z 00000001800bcfc8     hb-aat-map.obj
 0002:00031fdc       $chain$5$?add_feature@hb_aat_map_builder_t@@QEAAXAEBUhb_feature_t@@@Z 00000001800bcfdc     hb-aat-map.obj
 0002:00031fec       $chain$2$?add_feature@hb_aat_map_builder_t@@QEAAXAEBUhb_feature_t@@@Z 00000001800bcfec     hb-aat-map.obj
 0002:00032000       $chain$6$?add_feature@hb_aat_map_builder_t@@QEAAXAEBUhb_feature_t@@@Z 00000001800bd000     hb-aat-map.obj
 0002:00032010       $unwind$?compile@hb_aat_map_builder_t@@QEAAXAEAUhb_aat_map_t@@@Z 00000001800bd010     hb-aat-map.obj
 0002:00032018       $chain$6$?compile@hb_aat_map_builder_t@@QEAAXAEAUhb_aat_map_t@@@Z 00000001800bd018     hb-aat-map.obj
 0002:00032044       $chain$7$?compile@hb_aat_map_builder_t@@QEAAXAEAUhb_aat_map_t@@@Z 00000001800bd044     hb-aat-map.obj
 0002:00032054       $chain$0$?alloc@?$hb_vector_t@Ufeature_info_t@hb_aat_map_builder_t@@$00@@QEAA_NI_N@Z 00000001800bd054     hb-aat-map.obj
 0002:00032068       $chain$2$?alloc@?$hb_vector_t@Ufeature_info_t@hb_aat_map_builder_t@@$00@@QEAA_NI_N@Z 00000001800bd068     hb-aat-map.obj
 0002:00032068       $chain$4$?alloc@?$hb_vector_t@Ufeature_info_t@hb_aat_map_builder_t@@$00@@QEAA_NI_N@Z 00000001800bd068     hb-aat-map.obj
 0002:0003207c       $chain$2$hb_blob_create_sub_blob 00000001800bd07c     hb-blob.obj
 0002:00032098       $chain$3$hb_blob_create_sub_blob 00000001800bd098     hb-blob.obj
 0002:000320a8       $unwind$?_hb_blob_destroy@@YAXPEAX@Z 00000001800bd0a8     hb-blob.obj
 0002:000320a8       $unwind$hb_blob_destroy    00000001800bd0a8     hb-blob.obj
 0002:000320b0       $chain$0$hb_blob_destroy   00000001800bd0b0     hb-blob.obj
 0002:000320c4       $chain$1$hb_blob_destroy   00000001800bd0c4     hb-blob.obj
 0002:000320d4       $unwind$??$replace_or_insert@Uhb_user_data_item_t@hb_user_data_array_t@@@?$hb_lockable_set_t@Uhb_user_data_item_t@hb_user_data_array_t@@Uhb_mutex_t@@@@QEAAPEAUhb_user_data_item_t@hb_user_data_array_t@@U12@AEAUhb_mutex_t@@_N@Z 00000001800bd0d4     hb-blob.obj
 0002:000320d4       $unwind$?apply@?$ChainContextFormat2_5@USmallTypes@Layout@OT@@@OT@@QEBA_NPEAUhb_ot_apply_context_t@2@_N@Z 00000001800bd0d4     hb-ot-layout.obj
 0002:000320ec       $unwind$?try_make_writable@hb_blob_t@@QEAA_NXZ 00000001800bd0ec     hb-blob.obj
 0002:000320ec       $unwind$hb_face_get_user_data 00000001800bd0ec     hb-face.obj
 0002:000320f8       $chain$1$?try_make_writable@hb_blob_t@@QEAA_NXZ 00000001800bd0f8     hb-blob.obj
 0002:00032110       $chain$3$?try_make_writable@hb_blob_t@@QEAA_NXZ 00000001800bd110     hb-blob.obj
 0002:00032128       $chain$4$?try_make_writable@hb_blob_t@@QEAA_NXZ 00000001800bd128     hb-blob.obj
 0002:00032138       $chain$0$?_hb_blob_destroy@@YAXPEAX@Z 00000001800bd138     hb-blob.obj
 0002:0003214c       $chain$1$?_hb_blob_destroy@@YAXPEAX@Z 00000001800bd14c     hb-blob.obj
 0002:0003215c       $unwind$hb_buffer_serialize_unicode 00000001800bd15c     hb-buffer-serialize.obj
 0002:00032180       $unwind$snprintf           00000001800bd180     hb-buffer-serialize.obj
 0002:00032190       $unwind$fprintf            00000001800bd190     hb-buffer-verify.obj
 0002:0003219c       $unwind$?verify@hb_buffer_t@@QEAA_NPEAU1@PEAUhb_font_t@@PEBUhb_feature_t@@IPEBQEBD@Z 00000001800bd19c     hb-buffer-verify.obj
 0002:000321b4       $unwind$?buffer_verify_error@@YAXPEAUhb_buffer_t@@PEAUhb_font_t@@PEBDZZ 00000001800bd1b4     hb-buffer-verify.obj
 0002:000321c4       $unwind$?buffer_verify_unsafe_to_break@@YA_NPEAUhb_buffer_t@@0PEAUhb_font_t@@PEBUhb_feature_t@@IPEBQEBD@Z 00000001800bd1c4     hb-buffer-verify.obj
 0002:000321d0       $chain$5$?buffer_verify_unsafe_to_break@@YA_NPEAUhb_buffer_t@@0PEAUhb_font_t@@PEBUhb_feature_t@@IPEBQEBD@Z 00000001800bd1d0     hb-buffer-verify.obj
 0002:000321f8       $chain$7$?buffer_verify_unsafe_to_break@@YA_NPEAUhb_buffer_t@@0PEAUhb_font_t@@PEBUhb_feature_t@@IPEBQEBD@Z 00000001800bd1f8     hb-buffer-verify.obj
 0002:00032220       $unwind$?buffer_verify_unsafe_to_concat@@YA_NPEAUhb_buffer_t@@0PEAUhb_font_t@@PEBUhb_feature_t@@IPEBQEBD@Z 00000001800bd220     hb-buffer-verify.obj
 0002:00032230       $chain$4$?buffer_verify_unsafe_to_concat@@YA_NPEAUhb_buffer_t@@0PEAUhb_font_t@@PEBUhb_feature_t@@IPEBQEBD@Z 00000001800bd230     hb-buffer-verify.obj
 0002:00032254       $chain$6$?buffer_verify_unsafe_to_concat@@YA_NPEAUhb_buffer_t@@0PEAUhb_font_t@@PEBUhb_feature_t@@IPEBQEBD@Z 00000001800bd254     hb-buffer-verify.obj
 0002:00032278       $unwind$hb_buffer_destroy  00000001800bd278     hb-buffer.obj
 0002:00032278       $unwind$hb_draw_funcs_destroy 00000001800bd278     hb-draw.obj
 0002:00032278       $unwind$hb_font_destroy    00000001800bd278     hb-font.obj
 0002:00032278       $unwind$hb_font_funcs_destroy 00000001800bd278     hb-font.obj
 0002:00032278       $unwind$hb_paint_funcs_destroy 00000001800bd278     hb-paint.obj
 0002:00032278       $unwind$hb_unicode_funcs_destroy 00000001800bd278     hb-unicode.obj
 0002:00032280       $chain$0$hb_buffer_destroy 00000001800bd280     hb-buffer.obj
 0002:00032294       $chain$1$hb_buffer_destroy 00000001800bd294     hb-buffer.obj
 0002:000322a4       $unwind$hb_buffer_append   00000001800bd2a4     hb-buffer.obj
 0002:000322b0       $chain$0$hb_buffer_append  00000001800bd2b0     hb-buffer.obj
 0002:000322c4       $chain$6$hb_buffer_append  00000001800bd2c4     hb-buffer.obj
 0002:000322e8       $chain$7$hb_buffer_append  00000001800bd2e8     hb-buffer.obj
 0002:000322f8       $unwind$hb_buffer_diff     00000001800bd2f8     hb-buffer.obj
 0002:00032308       $chain$0$hb_buffer_diff    00000001800bd308     hb-buffer.obj
 0002:0003231c       $chain$2$hb_buffer_diff    00000001800bd31c     hb-buffer.obj
 0002:00032330       $chain$3$hb_buffer_diff    00000001800bd330     hb-buffer.obj
 0002:00032344       $chain$4$hb_buffer_diff    00000001800bd344     hb-buffer.obj
 0002:00032354       $unwind$?sync@hb_buffer_t@@QEAA_NXZ 00000001800bd354     hb-buffer.obj
 0002:00032354       $unwind$??4?$machine_index_t@U?$hb_zip_iter_t@U?$hb_iota_iter_t@II@@U?$hb_filter_iter_t@U?$hb_filter_iter_t@U?$hb_zip_iter_t@U?$hb_iota_iter_t@II@@U?$hb_array_t@Uhb_glyph_info_t@@@@@@V<lambda_e52748becc06432fe81365edeb8c4003>@@AEBU<unnamed-type-hb_second>@@$0A@@@V<lambda_a2885d5959499a7c5bcf896c0de144bb>@@AEBU<unnamed-type-hb_identity>@@$0A@@@@@@@QEAAXAEBU0@@Z 00000001800bd354     hb-ot-shaper-use.obj
 0002:00032360       $chain$1$?sync@hb_buffer_t@@QEAA_NXZ 00000001800bd360     hb-buffer.obj
 0002:00032378       $chain$2$?sync@hb_buffer_t@@QEAA_NXZ 00000001800bd378     hb-buffer.obj
 0002:00032388       $unwind$?sync_so_far@hb_buffer_t@@QEAAHXZ 00000001800bd388     hb-buffer.obj
 0002:00032394       $chain$1$?sync_so_far@hb_buffer_t@@QEAAHXZ 00000001800bd394     hb-buffer.obj
 0002:000323ac       $chain$4$?sync_so_far@hb_buffer_t@@QEAAHXZ 00000001800bd3ac     hb-buffer.obj
 0002:000323c8       $chain$5$?sync_so_far@hb_buffer_t@@QEAAHXZ 00000001800bd3c8     hb-buffer.obj
 0002:000323d8       $chain$6$?sync_so_far@hb_buffer_t@@QEAAHXZ 00000001800bd3d8     hb-buffer.obj
 0002:000323e8       $unwind$?set_masks@hb_buffer_t@@QEAAXIIII@Z 00000001800bd3e8     hb-buffer.obj
 0002:000323f4       $unwind$?merge_clusters_impl@hb_buffer_t@@QEAAXII@Z 00000001800bd3f4     hb-buffer.obj
 0002:000323f4       $unwind$??$sanitize@I@?$OffsetTo@UIndexSubtable@OT@@U?$IntType@I$03@2@$00@OT@@QEBA_NPEAUhb_sanitize_context_t@@PEBX$$QEAI@Z 00000001800bd3f4     hb-ot-color.obj
 0002:000323f4       $unwind$?get_advance_delta_unscaled@HVARVVAR@OT@@QEBAMIPEBHIPEAM@Z 00000001800bd3f4     hb-ot-font.obj
 0002:000323f4       $unwind$?get_extents@ClipList@OT@@QEBA_NIPEAUhb_glyph_extents_t@@AEBUVarStoreInstancer@2@@Z 00000001800bd3f4     hb-ot-font.obj
 0002:000323f4       $unwind$?hb_ot_get_glyph_extents@@YAHPEAUhb_font_t@@PEAXIPEAUhb_glyph_extents_t@@1@Z 00000001800bd3f4     hb-ot-font.obj
 0002:000323f4       $unwind$?process_op@cff2_top_dict_opset_t@CFF@@SAXIAEAU?$interp_env_t@Unumber_t@CFF@@@2@AEAUcff2_top_dict_values_t@2@@Z 00000001800bd3f4     hb-ot-font.obj
 0002:000323f4       $unwind$?compose_indic@@YA_NPEBUhb_ot_shape_normalize_context_t@@IIPEAI@Z 00000001800bd3f4     hb-ot-shaper-indic.obj
 0002:00032408       $chain$1$?merge_out_clusters@hb_buffer_t@@QEAAXII@Z 00000001800bd408     hb-buffer.obj
 0002:00032420       $chain$2$?merge_out_clusters@hb_buffer_t@@QEAAXII@Z 00000001800bd420     hb-buffer.obj
 0002:00032434       $chain$3$?merge_out_clusters@hb_buffer_t@@QEAAXII@Z 00000001800bd434     hb-buffer.obj
 0002:00032444       $unwind$?delete_glyphs_inplace@hb_buffer_t@@QEAAXP6A_NPEBUhb_glyph_info_t@@@Z@Z 00000001800bd444     hb-buffer.obj
 0002:00032454       $chain$2$?delete_glyphs_inplace@hb_buffer_t@@QEAAXP6A_NPEBUhb_glyph_info_t@@@Z@Z 00000001800bd454     hb-buffer.obj
 0002:00032470       $chain$3$?delete_glyphs_inplace@hb_buffer_t@@QEAAXP6A_NPEBUhb_glyph_info_t@@@Z@Z 00000001800bd470     hb-buffer.obj
 0002:00032480       $chain$0$?move_to@hb_buffer_t@@QEAA_NI@Z 00000001800bd480     hb-buffer.obj
 0002:00032494       $chain$2$?move_to@hb_buffer_t@@QEAA_NI@Z 00000001800bd494     hb-buffer.obj
 0002:00032494       $chain$4$?move_to@hb_buffer_t@@QEAA_NI@Z 00000001800bd494     hb-buffer.obj
 0002:000324a8       $unwind$?enlarge@hb_buffer_t@@QEAA_NI@Z 00000001800bd4a8     hb-buffer.obj
 0002:000324b0       $chain$4$?enlarge@hb_buffer_t@@QEAA_NI@Z 00000001800bd4b0     hb-buffer.obj
 0002:000324d4       $chain$5$?enlarge@hb_buffer_t@@QEAA_NI@Z 00000001800bd4d4     hb-buffer.obj
 0002:000324e8       $chain$6$?enlarge@hb_buffer_t@@QEAA_NI@Z 00000001800bd4e8     hb-buffer.obj
 0002:000324f8       $chain$7$?enlarge@hb_buffer_t@@QEAA_NI@Z 00000001800bd4f8     hb-buffer.obj
 0002:00032518       $chain$8$?enlarge@hb_buffer_t@@QEAA_NI@Z 00000001800bd518     hb-buffer.obj
 0002:00032530       $chain$9$?enlarge@hb_buffer_t@@QEAA_NI@Z 00000001800bd530     hb-buffer.obj
 0002:00032544       $unwind$?ensure@hb_buffer_t@@QEAA_NI@Z 00000001800bd544     hb-buffer.obj
 0002:00032550       $chain$3$?ensure@hb_buffer_t@@QEAA_NI@Z 00000001800bd550     hb-buffer.obj
 0002:00032570       $chain$4$?ensure@hb_buffer_t@@QEAA_NI@Z 00000001800bd570     hb-buffer.obj
 0002:00032584       $chain$5$?ensure@hb_buffer_t@@QEAA_NI@Z 00000001800bd584     hb-buffer.obj
 0002:00032594       $chain$6$?ensure@hb_buffer_t@@QEAA_NI@Z 00000001800bd594     hb-buffer.obj
 0002:000325b0       $chain$7$?ensure@hb_buffer_t@@QEAA_NI@Z 00000001800bd5b0     hb-buffer.obj
 0002:000325c4       $chain$8$?ensure@hb_buffer_t@@QEAA_NI@Z 00000001800bd5c4     hb-buffer.obj
 0002:000325d4       $unwind$?sort@hb_buffer_t@@QEAAXIIP6AHPEBUhb_glyph_info_t@@0@Z@Z 00000001800bd5d4     hb-buffer.obj
 0002:000325e0       $chain$4$?sort@hb_buffer_t@@QEAAXIIP6AHPEBUhb_glyph_info_t@@0@Z@Z 00000001800bd5e0     hb-buffer.obj
 0002:00032604       $chain$5$?sort@hb_buffer_t@@QEAAXIIP6AHPEBUhb_glyph_info_t@@0@Z@Z 00000001800bd604     hb-buffer.obj
 0002:00032614       $unwind$?message_impl@hb_buffer_t@@QEAA_NPEAUhb_font_t@@PEBDPEAD@Z 00000001800bd614     hb-buffer.obj
 0002:0003262c       $unwind$??$reverse_groups@$$A6A_NAEBUhb_glyph_info_t@@0@Z@hb_buffer_t@@QEAAXA6A_NAEBUhb_glyph_info_t@@0@Z_N@Z 00000001800bd62c     hb-buffer.obj
 0002:0003262c       $unwind$?final_reordering_indic@@YA_NPEBUhb_ot_shape_plan_t@@PEAUhb_font_t@@PEAUhb_buffer_t@@@Z 00000001800bd62c     hb-ot-shaper-indic.obj
 0002:0003263c       $chain$1$??$reverse_groups@$$A6A_NAEBUhb_glyph_info_t@@0@Z@hb_buffer_t@@QEAAXA6A_NAEBUhb_glyph_info_t@@0@Z_N@Z 00000001800bd63c     hb-buffer.obj
 0002:00032654       $chain$2$??$reverse_groups@$$A6A_NAEBUhb_glyph_info_t@@0@Z@hb_buffer_t@@QEAAXA6A_NAEBUhb_glyph_info_t@@0@Z_N@Z 00000001800bd654     hb-buffer.obj
 0002:00032664       $unwind$??$hb_buffer_add_utf@U?$hb_utf16_xe_t@G@@@@YAXPEAUhb_buffer_t@@PEBGHIH@Z 00000001800bd664     hb-buffer.obj
 0002:00032674       $chain$0$??$hb_buffer_add_utf@U?$hb_utf16_xe_t@G@@@@YAXPEAUhb_buffer_t@@PEBGHIH@Z 00000001800bd674     hb-buffer.obj
 0002:00032688       $chain$1$??$hb_buffer_add_utf@U?$hb_utf16_xe_t@G@@@@YAXPEAUhb_buffer_t@@PEBGHIH@Z 00000001800bd688     hb-buffer.obj
 0002:0003269c       $chain$2$??$hb_buffer_add_utf@U?$hb_utf16_xe_t@G@@@@YAXPEAUhb_buffer_t@@PEBGHIH@Z 00000001800bd69c     hb-buffer.obj
 0002:000326b0       $chain$3$??$hb_buffer_add_utf@U?$hb_utf16_xe_t@G@@@@YAXPEAUhb_buffer_t@@PEBGHIH@Z 00000001800bd6b0     hb-buffer.obj
 0002:000326c0       $chain$4$??$hb_buffer_add_utf@U?$hb_utf16_xe_t@G@@@@YAXPEAUhb_buffer_t@@PEBGHIH@Z 00000001800bd6c0     hb-buffer.obj
 0002:000326d0       $chain$5$??$hb_buffer_add_utf@U?$hb_utf16_xe_t@G@@@@YAXPEAUhb_buffer_t@@PEBGHIH@Z 00000001800bd6d0     hb-buffer.obj
 0002:000326e0       $unwind$hb_language_from_string 00000001800bd6e0     hb-common.obj
 0002:000326f0       $chain$0$hb_language_from_string 00000001800bd6f0     hb-common.obj
 0002:00032704       $chain$2$hb_language_from_string 00000001800bd704     hb-common.obj
 0002:00032704       $chain$4$hb_language_from_string 00000001800bd704     hb-common.obj
 0002:00032718       $chain$3$hb_language_from_string 00000001800bd718     hb-common.obj
 0002:00032728       $chain$0$hb_language_matches 00000001800bd728     hb-common.obj
 0002:0003273c       $chain$2$hb_language_matches 00000001800bd73c     hb-common.obj
 0002:00032750       $chain$3$hb_language_matches 00000001800bd750     hb-common.obj
 0002:00032760       $unwind$hb_feature_from_string 00000001800bd760     hb-common.obj
 0002:00032768       $chain$1$?_hb_options_init@@YAXXZ 00000001800bd768     hb-common.obj
 0002:00032780       $chain$2$?_hb_options_init@@YAXXZ 00000001800bd780     hb-common.obj
 0002:00032790       $unwind$?lang_find_or_insert@@YAPEAUhb_language_item_t@@PEBD@Z 00000001800bd790     hb-common.obj
 0002:000327a4       $unwind$?get@?$hb_lazy_loader_t@Uhmtx_accelerator_t@OT@@U?$hb_face_lazy_loader_t@Uhmtx_accelerator_t@OT@@$04@@Uhb_face_t@@$04U12@@@QEBAPEBUhmtx_accelerator_t@OT@@XZ 00000001800bd7a4     hb-common.obj
 0002:000327a4       $unwind$?get@?$hb_lazy_loader_t@Uvmtx_accelerator_t@OT@@U?$hb_face_lazy_loader_t@Uvmtx_accelerator_t@OT@@$0M@@@Uhb_face_t@@$0M@U12@@@QEBAPEBUvmtx_accelerator_t@OT@@XZ 00000001800bd7a4     hb-common.obj
 0002:000327a4       $unwind$?parse_tag@@YA_NPEAPEBDPEBDPEAI@Z 00000001800bd7a4     hb-common.obj
 0002:000327a4       $unwind$??C?$hb_lazy_loader_t@Ucmap_accelerator_t@OT@@U?$hb_face_lazy_loader_t@Ucmap_accelerator_t@OT@@$02@@Uhb_face_t@@$02U12@@@QEBAPEBUcmap_accelerator_t@OT@@XZ 00000001800bd7a4     hb-face.obj
 0002:000327a4       $unwind$??C?$hb_lazy_loader_t@Upost_accelerator_t@OT@@U?$hb_face_lazy_loader_t@Upost_accelerator_t@OT@@$06@@Uhb_face_t@@$06U12@@@QEBAPEBUpost_accelerator_t@OT@@XZ 00000001800bd7a4     hb-ot-font.obj
 0002:000327a4       $unwind$?get_stored@?$hb_lazy_loader_t@Ucff1_accelerator_t@OT@@U?$hb_face_lazy_loader_t@Ucff1_accelerator_t@OT@@$0BA@@@Uhb_face_t@@$0BA@U12@@@QEBAPEAUcff1_accelerator_t@OT@@XZ 00000001800bd7a4     hb-ot-font.obj
 0002:000327a4       $unwind$??$apply_string@UGSUBProxy@@@@YA_NPEAUhb_ot_apply_context_t@OT@@AEBUSubstLookup@GSUB_impl@Layout@1@AEBUhb_ot_layout_lookup_accelerator_t@1@@Z 00000001800bd7a4     hb-ot-layout.obj
 0002:000327b8       $unwind$?parse_one_feature@@YA_NPEAPEBDPEBDPEAUhb_feature_t@@@Z 00000001800bd7b8     hb-common.obj
 0002:000327b8       $unwind$hb_draw_funcs_set_close_path_func 00000001800bd7b8     hb-draw.obj
 0002:000327b8       $unwind$hb_draw_funcs_set_cubic_to_func 00000001800bd7b8     hb-draw.obj
 0002:000327b8       $unwind$hb_draw_funcs_set_line_to_func 00000001800bd7b8     hb-draw.obj
 0002:000327b8       $unwind$hb_draw_funcs_set_move_to_func 00000001800bd7b8     hb-draw.obj
 0002:000327b8       $unwind$hb_draw_funcs_set_quadratic_to_func 00000001800bd7b8     hb-draw.obj
 0002:000327b8       $unwind$hb_font_funcs_set_draw_glyph_func 00000001800bd7b8     hb-font.obj
 0002:000327b8       $unwind$hb_font_funcs_set_font_h_extents_func 00000001800bd7b8     hb-font.obj
 0002:000327b8       $unwind$hb_font_funcs_set_font_v_extents_func 00000001800bd7b8     hb-font.obj
 0002:000327b8       $unwind$hb_font_funcs_set_glyph_contour_point_func 00000001800bd7b8     hb-font.obj
 0002:000327b8       $unwind$hb_font_funcs_set_glyph_extents_func 00000001800bd7b8     hb-font.obj
 0002:000327b8       $unwind$hb_font_funcs_set_glyph_from_name_func 00000001800bd7b8     hb-font.obj
 0002:000327b8       $unwind$hb_font_funcs_set_glyph_h_advance_func 00000001800bd7b8     hb-font.obj
 0002:000327b8       $unwind$hb_font_funcs_set_glyph_h_advances_func 00000001800bd7b8     hb-font.obj
 0002:000327b8       $unwind$hb_font_funcs_set_glyph_h_kerning_func 00000001800bd7b8     hb-font.obj
 0002:000327b8       $unwind$hb_font_funcs_set_glyph_h_origin_func 00000001800bd7b8     hb-font.obj
 0002:000327b8       $unwind$hb_font_funcs_set_glyph_name_func 00000001800bd7b8     hb-font.obj
 0002:000327b8       $unwind$hb_font_funcs_set_glyph_v_advance_func 00000001800bd7b8     hb-font.obj
 0002:000327b8       $unwind$hb_font_funcs_set_glyph_v_advances_func 00000001800bd7b8     hb-font.obj
 0002:000327b8       $unwind$hb_font_funcs_set_glyph_v_kerning_func 00000001800bd7b8     hb-font.obj
 0002:000327b8       $unwind$hb_font_funcs_set_glyph_v_origin_func 00000001800bd7b8     hb-font.obj
 0002:000327b8       $unwind$hb_font_funcs_set_nominal_glyph_func 00000001800bd7b8     hb-font.obj
 0002:000327b8       $unwind$hb_font_funcs_set_nominal_glyphs_func 00000001800bd7b8     hb-font.obj
 0002:000327b8       $unwind$hb_font_funcs_set_paint_glyph_func 00000001800bd7b8     hb-font.obj
 0002:000327b8       $unwind$hb_font_funcs_set_variation_glyph_func 00000001800bd7b8     hb-font.obj
 0002:000327b8       $unwind$??A?$CFFIndex@U?$IntType@I$03@OT@@@CFF@@QEBA?AU?$hb_array_t@$$CBE@@I@Z 00000001800bd7b8     hb-ot-cff2-table.obj
 0002:000327b8       $unwind$hb_paint_funcs_set_color_func 00000001800bd7b8     hb-paint.obj
 0002:000327b8       $unwind$hb_paint_funcs_set_image_func 00000001800bd7b8     hb-paint.obj
 0002:000327b8       $unwind$hb_paint_funcs_set_linear_gradient_func 00000001800bd7b8     hb-paint.obj
 0002:000327b8       $unwind$hb_paint_funcs_set_pop_clip_func 00000001800bd7b8     hb-paint.obj
 0002:000327b8       $unwind$hb_paint_funcs_set_pop_group_func 00000001800bd7b8     hb-paint.obj
 0002:000327b8       $unwind$hb_paint_funcs_set_pop_transform_func 00000001800bd7b8     hb-paint.obj
 0002:000327b8       $unwind$hb_paint_funcs_set_push_clip_glyph_func 00000001800bd7b8     hb-paint.obj
 0002:000327b8       $unwind$hb_paint_funcs_set_push_clip_rectangle_func 00000001800bd7b8     hb-paint.obj
 0002:000327b8       $unwind$hb_paint_funcs_set_push_group_func 00000001800bd7b8     hb-paint.obj
 0002:000327b8       $unwind$hb_paint_funcs_set_push_transform_func 00000001800bd7b8     hb-paint.obj
 0002:000327b8       $unwind$hb_paint_funcs_set_radial_gradient_func 00000001800bd7b8     hb-paint.obj
 0002:000327b8       $unwind$hb_paint_funcs_set_sweep_gradient_func 00000001800bd7b8     hb-paint.obj
 0002:000327cc       $chain$0$?get@?$hb_lazy_loader_t@Uhead@OT@@U?$hb_table_lazy_loader_t@Uhead@OT@@$00$00@@Uhb_face_t@@$00Uhb_blob_t@@@@QEBAPEBUhead@OT@@XZ 00000001800bd7cc     hb-common.obj
 0002:000327e0       $chain$1$?get@?$hb_lazy_loader_t@Uhead@OT@@U?$hb_table_lazy_loader_t@Uhead@OT@@$00$00@@Uhb_face_t@@$00Uhb_blob_t@@@@QEBAPEBUhead@OT@@XZ 00000001800bd7e0     hb-common.obj
 0002:000327f0       $chain$0$??C?$hb_lazy_loader_t@Umaxp@OT@@U?$hb_table_lazy_loader_t@Umaxp@OT@@$01$00@@Uhb_face_t@@$01Uhb_blob_t@@@@QEBAPEBUmaxp@OT@@XZ 00000001800bd7f0     hb-common.obj
 0002:00032804       $chain$1$??C?$hb_lazy_loader_t@Umaxp@OT@@U?$hb_table_lazy_loader_t@Umaxp@OT@@$01$00@@Uhb_face_t@@$01Uhb_blob_t@@@@QEBAPEBUmaxp@OT@@XZ 00000001800bd804     hb-common.obj
 0002:00032814       $chain$0$??C?$hb_lazy_loader_t@Uhhea@OT@@U?$hb_table_lazy_loader_t@Uhhea@OT@@$03$00@@Uhb_face_t@@$03Uhb_blob_t@@@@QEBAPEBUhhea@OT@@XZ 00000001800bd814     hb-common.obj
 0002:00032828       $chain$1$??C?$hb_lazy_loader_t@Uhhea@OT@@U?$hb_table_lazy_loader_t@Uhhea@OT@@$03$00@@Uhb_face_t@@$03Uhb_blob_t@@@@QEBAPEBUhhea@OT@@XZ 00000001800bd828     hb-common.obj
 0002:00032838       $chain$0$??C?$hb_lazy_loader_t@Uvhea@OT@@U?$hb_table_lazy_loader_t@Uvhea@OT@@$0L@$00@@Uhb_face_t@@$0L@Uhb_blob_t@@@@QEBAPEBUvhea@OT@@XZ 00000001800bd838     hb-common.obj
 0002:0003284c       $chain$1$??C?$hb_lazy_loader_t@Uvhea@OT@@U?$hb_table_lazy_loader_t@Uvhea@OT@@$0L@$00@@Uhb_face_t@@$0L@Uhb_blob_t@@@@QEBAPEBUvhea@OT@@XZ 00000001800bd84c     hb-common.obj
 0002:0003285c       $unwind$??C?$hb_lazy_loader_t@Uglyf_accelerator_t@OT@@U?$hb_face_lazy_loader_t@Uglyf_accelerator_t@OT@@$0P@@@Uhb_face_t@@$0P@U12@@@QEBAPEBUglyf_accelerator_t@OT@@XZ 00000001800bd85c     hb-common.obj
 0002:0003285c       $unwind$?hb_parse_double@@YA_NPEAPEBDPEBDPEAN_N@Z 00000001800bd85c     hb-number.obj
 0002:0003285c       $unwind$??A?$CFFIndex@U?$IntType@G$01@OT@@@CFF@@QEBA?AU?$hb_array_t@$$CBE@@I@Z 00000001800bd85c     hb-ot-cff1-table.obj
 0002:0003285c       $unwind$??C?$hb_lazy_loader_t@Ucff2_accelerator_t@OT@@U?$hb_face_lazy_loader_t@Ucff2_accelerator_t@OT@@$0BB@@@Uhb_face_t@@$0BB@U12@@@QEBAPEBUcff2_accelerator_t@OT@@XZ 00000001800bd85c     hb-ot-font.obj
 0002:0003285c       $unwind$?sanitize@MVAR@OT@@QEBA_NPEAUhb_sanitize_context_t@@@Z 00000001800bd85c     hb-ot-metrics.obj
 0002:00032870       $unwind$?scale_glyph_extents@hb_font_t@@QEAAXPEAUhb_glyph_extents_t@@@Z 00000001800bd870     hb-common.obj
 0002:00032894       $unwind$?calculate_scalar@TupleVariationHeader@OT@@QEBAMU?$hb_array_t@H@@IU?$hb_array_t@$$CBU?$HBFixed@U?$IntType@F$01@OT@@$0O@@OT@@@@PEBU?$hb_vector_t@H$0A@@@@Z 00000001800bd894     hb-common.obj
 0002:00032894       $unwind$?read_points@SimpleGlyph@glyf_impl@OT@@SA_NAEAPEBU?$IntType@E$00@3@AEAUcontour_point_vector_t@3@PEBU43@PEQcontour_point_t@3@MW4simple_glyph_flag_t@123@4@Z 00000001800bd894     hb-common.obj
 0002:00032894       $unwind$?find_syllables_indic@@YAXPEAUhb_buffer_t@@@Z 00000001800bd894     hb-ot-shaper-indic.obj
 0002:00032894       $unwind$?find_syllables_khmer@@YAXPEAUhb_buffer_t@@@Z 00000001800bd894     hb-ot-shaper-khmer.obj
 0002:00032894       $unwind$?find_syllables_myanmar@@YAXPEAUhb_buffer_t@@@Z 00000001800bd894     hb-ot-shaper-myanmar.obj
 0002:00032894       $unwind$?__next__@?$hb_filter_iter_t@U?$hb_filter_iter_t@U?$hb_zip_iter_t@U?$hb_iota_iter_t@II@@U?$hb_array_t@Uhb_glyph_info_t@@@@@@V<lambda_e52748becc06432fe81365edeb8c4003>@@AEBU<unnamed-type-hb_second>@@$0A@@@V<lambda_a2885d5959499a7c5bcf896c0de144bb>@@AEBU<unnamed-type-hb_identity>@@$0A@@@QEAAXXZ 00000001800bd894     hb-ot-shaper-use.obj
 0002:00032894       $unwind$?__prev__@?$hb_filter_iter_t@U?$hb_filter_iter_t@U?$hb_zip_iter_t@U?$hb_iota_iter_t@II@@U?$hb_array_t@Uhb_glyph_info_t@@@@@@V<lambda_e52748becc06432fe81365edeb8c4003>@@AEBU<unnamed-type-hb_second>@@$0A@@@V<lambda_a2885d5959499a7c5bcf896c0de144bb>@@AEBU<unnamed-type-hb_identity>@@$0A@@@QEAAXXZ 00000001800bd894     hb-ot-shaper-use.obj
 0002:000328b0       $unwind$?_glyf_get_leading_bearing_with_var_unscaled@@YA_NPEAUhb_font_t@@I_NPEAH@Z 00000001800bd8b0     hb-common.obj
 0002:000328cc       $unwind$?_glyf_get_advance_with_var_unscaled@@YAIPEAUhb_font_t@@I_N@Z 00000001800bd8cc     hb-common.obj
 0002:000328ec       $chain$0$?_glyf_get_advance_with_var_unscaled@@YAIPEAUhb_font_t@@I_N@Z 00000001800bd8ec     hb-common.obj
 0002:00032900       $chain$1$?_glyf_get_advance_with_var_unscaled@@YAIPEAUhb_font_t@@I_N@Z 00000001800bd900     hb-common.obj
 0002:00032910       $unwind$??0accelerator_t@?$hmtxvmtx@Uhmtx@OT@@Uhhea@2@UHVAR@2@@OT@@QEAA@PEAUhb_face_t@@@Z 00000001800bd910     hb-common.obj
 0002:00032910       $unwind$??0accelerator_t@?$hmtxvmtx@Uvmtx@OT@@Uvhea@2@UVVAR@2@@OT@@QEAA@PEAUhb_face_t@@@Z 00000001800bd910     hb-common.obj
 0002:00032928       $unwind$?get_advance_without_var_unscaled@accelerator_t@?$hmtxvmtx@Uhmtx@OT@@Uhhea@2@UHVAR@2@@OT@@QEBAII@Z 00000001800bd928     hb-common.obj
 0002:00032928       $unwind$?get_advance_without_var_unscaled@accelerator_t@?$hmtxvmtx@Uvmtx@OT@@Uvhea@2@UVVAR@2@@OT@@QEBAII@Z 00000001800bd928     hb-common.obj
 0002:00032930       $chain$0$?alloc@?$hb_vector_t@Ucontour_point_t@OT@@$0A@@@QEAA_NI_N@Z 00000001800bd930     hb-common.obj
 0002:00032930       $chain$0$?alloc@?$hb_vector_t@Ulookup_map_t@hb_ot_map_t@@$0A@@@QEAA_NI_N@Z 00000001800bd930     hb-ot-map.obj
 0002:00032944       $chain$2$?alloc@?$hb_vector_t@Ucontour_point_t@OT@@$0A@@@QEAA_NI_N@Z 00000001800bd944     hb-common.obj
 0002:00032944       $chain$4$?alloc@?$hb_vector_t@Ucontour_point_t@OT@@$0A@@@QEAA_NI_N@Z 00000001800bd944     hb-common.obj
 0002:00032944       $chain$2$?alloc@?$hb_vector_t@Ulookup_map_t@hb_ot_map_t@@$0A@@@QEAA_NI_N@Z 00000001800bd944     hb-ot-map.obj
 0002:00032944       $chain$4$?alloc@?$hb_vector_t@Ulookup_map_t@hb_ot_map_t@@$0A@@@QEAA_NI_N@Z 00000001800bd944     hb-ot-map.obj
 0002:00032958       $unwind$?extend@contour_point_vector_t@OT@@QEAAXAEBU?$hb_array_t@Ucontour_point_t@OT@@@@@Z 00000001800bd958     hb-common.obj
 0002:00032970       $chain$0$?extend@contour_point_vector_t@OT@@QEAAXAEBU?$hb_array_t@Ucontour_point_t@OT@@@@@Z 00000001800bd970     hb-common.obj
 0002:00032984       $chain$1$?extend@contour_point_vector_t@OT@@QEAAXAEBU?$hb_array_t@Ucontour_point_t@OT@@@@@Z 00000001800bd984     hb-common.obj
 0002:00032994       $chain$0$?translate@contour_point_vector_t@OT@@QEAAXAEBUcontour_point_t@2@@Z 00000001800bd994     hb-common.obj
 0002:000329a8       $chain$1$?translate@contour_point_vector_t@OT@@QEAAXAEBUcontour_point_t@2@@Z 00000001800bd9a8     hb-common.obj
 0002:000329b8       $unwind$?get_glyph_var_data_bytes@gvar@OT@@IEBA?BU?$hb_array_t@$$CBD@@PEAUhb_blob_t@@II@Z 00000001800bd9b8     hb-common.obj
 0002:000329c4       $chain$0$?get_glyph_var_data_bytes@gvar@OT@@IEBA?BU?$hb_array_t@$$CBD@@PEAUhb_blob_t@@II@Z 00000001800bd9c4     hb-common.obj
 0002:000329d8       $chain$1$?get_glyph_var_data_bytes@gvar@OT@@IEBA?BU?$hb_array_t@$$CBD@@PEAUhb_blob_t@@II@Z 00000001800bd9d8     hb-common.obj
 0002:000329e8       $unwind$??0accelerator_t@gvar@OT@@QEAA@PEAUhb_face_t@@@Z 00000001800bd9e8     hb-common.obj
 0002:000329fc       $chain$1$??0accelerator_t@gvar@OT@@QEAA@PEAUhb_face_t@@@Z 00000001800bd9fc     hb-common.obj
 0002:00032a14       $chain$2$??0accelerator_t@gvar@OT@@QEAA@PEAUhb_face_t@@@Z 00000001800bda14     hb-common.obj
 0002:00032a14       $chain$4$??0accelerator_t@gvar@OT@@QEAA@PEAUhb_face_t@@@Z 00000001800bda14     hb-common.obj
 0002:00032a24       $chain$3$??0accelerator_t@gvar@OT@@QEAA@PEAUhb_face_t@@@Z 00000001800bda24     hb-common.obj
 0002:00032a3c       $unwind$?apply_deltas_to_points@accelerator_t@gvar@OT@@QEBA_NIU?$hb_array_t@H@@U?$hb_array_t@Ucontour_point_t@OT@@@@@Z 00000001800bda3c     hb-common.obj
 0002:00032a50       $chain$1$?apply_deltas_to_points@accelerator_t@gvar@OT@@QEBA_NIU?$hb_array_t@H@@U?$hb_array_t@Ucontour_point_t@OT@@@@@Z 00000001800bda50     hb-common.obj
 0002:00032a68       $chain$6$?apply_deltas_to_points@accelerator_t@gvar@OT@@QEBA_NIU?$hb_array_t@H@@U?$hb_array_t@Ucontour_point_t@OT@@@@@Z 00000001800bda68     hb-common.obj
 0002:00032a8c       $chain$8$?apply_deltas_to_points@accelerator_t@gvar@OT@@QEBA_NIU?$hb_array_t@H@@U?$hb_array_t@Ucontour_point_t@OT@@@@@Z 00000001800bda8c     hb-common.obj
 0002:00032ab0       $chain$9$?apply_deltas_to_points@accelerator_t@gvar@OT@@QEBA_NIU?$hb_array_t@H@@U?$hb_array_t@Ucontour_point_t@OT@@@@@Z 00000001800bdab0     hb-common.obj
 0002:00032ac0       $chain$10$?apply_deltas_to_points@accelerator_t@gvar@OT@@QEBA_NIU?$hb_array_t@H@@U?$hb_array_t@Ucontour_point_t@OT@@@@@Z 00000001800bdac0     hb-common.obj
 0002:00032ad0       $unwind$?trim_padding@SimpleGlyph@glyf_impl@OT@@QEBA?BU?$hb_array_t@$$CBD@@XZ 00000001800bdad0     hb-common.obj
 0002:00032ad0       $unwind$??0?$hb_filter_iter_t@U?$hb_filter_iter_t@U?$hb_zip_iter_t@U?$hb_iota_iter_t@II@@U?$hb_array_t@Uhb_glyph_info_t@@@@@@V<lambda_e52748becc06432fe81365edeb8c4003>@@AEBU<unnamed-type-hb_second>@@$0A@@@V<lambda_a2885d5959499a7c5bcf896c0de144bb>@@AEBU<unnamed-type-hb_identity>@@$0A@@@QEAA@AEBU?$hb_filter_iter_t@U?$hb_zip_iter_t@U?$hb_iota_iter_t@II@@U?$hb_array_t@Uhb_glyph_info_t@@@@@@V<lambda_e52748becc06432fe81365edeb8c4003>@@AEBU<unnamed-type-hb_second>@@$0A@@@V<lambda_a2885d5959499a7c5bcf896c0de144bb>@@AEBU<unnamed-type-hb_identity>@@@Z 00000001800bdad0     hb-ot-shaper-use.obj
 0002:00032ae8       $unwind$?get_contour_points@SimpleGlyph@glyf_impl@OT@@QEBA_NAEAUcontour_point_vector_t@3@_N@Z 00000001800bdae8     hb-common.obj
 0002:00032b00       $unwind$?get_transformation@CompositeGlyphRecord@glyf_impl@OT@@QEBA_NAEAY03MAEAUcontour_point_t@3@@Z 00000001800bdb00     hb-common.obj
 0002:00032b00       $unwind$?find_table@IndexSubtableArray@OT@@QEBAPEBUIndexSubtableRecord@2@II@Z 00000001800bdb00     hb-ot-color.obj
 0002:00032b14       $unwind$??$get_points@Uglyf_accelerator_t@OT@@@Glyph@glyf_impl@OT@@QEBA_NPEAUhb_font_t@@AEBUglyf_accelerator_t@2@AEAUcontour_point_vector_t@2@PEAU52@PEAUhead_maxp_info_t@@PEAI_N66U?$hb_array_t@H@@I5@Z 00000001800bdb14     hb-common.obj
 0002:00032b24       $chain$4$??$get_points@Uglyf_accelerator_t@OT@@@Glyph@glyf_impl@OT@@QEBA_NPEAUhb_font_t@@AEBUglyf_accelerator_t@2@AEAUcontour_point_vector_t@2@PEAU52@PEAUhead_maxp_info_t@@PEAI_N66U?$hb_array_t@H@@I5@Z 00000001800bdb24     hb-common.obj
 0002:00032b48       $chain$6$??$get_points@Uglyf_accelerator_t@OT@@@Glyph@glyf_impl@OT@@QEBA_NPEAUhb_font_t@@AEBUglyf_accelerator_t@2@AEAUcontour_point_vector_t@2@PEAU52@PEAUhead_maxp_info_t@@PEAI_N66U?$hb_array_t@H@@I5@Z 00000001800bdb48     hb-common.obj
 0002:00032b6c       $chain$7$??$get_points@Uglyf_accelerator_t@OT@@@Glyph@glyf_impl@OT@@QEBA_NPEAUhb_font_t@@AEBUglyf_accelerator_t@2@AEAUcontour_point_vector_t@2@PEAU52@PEAUhead_maxp_info_t@@PEAI_N66U?$hb_array_t@H@@I5@Z 00000001800bdb6c     hb-common.obj
 0002:00032b7c       $unwind$??0glyf_accelerator_t@OT@@QEAA@PEAUhb_face_t@@@Z 00000001800bdb7c     hb-common.obj
 0002:00032b8c       $chain$1$??0glyf_accelerator_t@OT@@QEAA@PEAUhb_face_t@@@Z 00000001800bdb8c     hb-common.obj
 0002:00032ba4       $chain$2$??0glyf_accelerator_t@OT@@QEAA@PEAUhb_face_t@@@Z 00000001800bdba4     hb-common.obj
 0002:00032bb4       $unwind$?glyph_for_gid@glyf_accelerator_t@OT@@QEBA?BUGlyph@glyf_impl@2@I_N@Z 00000001800bdbb4     hb-common.obj
 0002:00032bcc       $chain$0$?glyph_for_gid@glyf_accelerator_t@OT@@QEBA?BUGlyph@glyf_impl@2@I_N@Z 00000001800bdbcc     hb-common.obj
 0002:00032be0       $chain$1$?glyph_for_gid@glyf_accelerator_t@OT@@QEBA?BUGlyph@glyf_impl@2@I_N@Z 00000001800bdbe0     hb-common.obj
 0002:00032bf0       $unwind$??$get_points@Upoints_aggregator_t@glyf_accelerator_t@OT@@@glyf_accelerator_t@OT@@IEBA_NPEAUhb_font_t@@IUpoints_aggregator_t@01@@Z 00000001800bdbf0     hb-common.obj
 0002:00032c0c       $chain$6$??$get_points@Upoints_aggregator_t@glyf_accelerator_t@OT@@@glyf_accelerator_t@OT@@IEBA_NPEAUhb_font_t@@IUpoints_aggregator_t@01@@Z 00000001800bdc0c     hb-common.obj
 0002:00032c2c       $chain$7$??$get_points@Upoints_aggregator_t@glyf_accelerator_t@OT@@@glyf_accelerator_t@OT@@IEBA_NPEAUhb_font_t@@IUpoints_aggregator_t@01@@Z 00000001800bdc2c     hb-common.obj
 0002:00032c48       $chain$8$??$get_points@Upoints_aggregator_t@glyf_accelerator_t@OT@@@glyf_accelerator_t@OT@@IEBA_NPEAUhb_font_t@@IUpoints_aggregator_t@01@@Z 00000001800bdc48     hb-common.obj
 0002:00032c58       $unwind$??$sanitize_blob@Ugvar@OT@@@hb_sanitize_context_t@@QEAAPEAUhb_blob_t@@PEAU1@@Z 00000001800bdc58     hb-common.obj
 0002:00032c74       $unwind$??$sanitize_blob@Uhead@OT@@@hb_sanitize_context_t@@QEAAPEAUhb_blob_t@@PEAU1@@Z 00000001800bdc74     hb-common.obj
 0002:00032c74       $unwind$??$sanitize_blob@Uhhea@OT@@@hb_sanitize_context_t@@QEAAPEAUhb_blob_t@@PEAU1@@Z 00000001800bdc74     hb-common.obj
 0002:00032c74       $unwind$??$sanitize_blob@Uvhea@OT@@@hb_sanitize_context_t@@QEAAPEAUhb_blob_t@@PEAU1@@Z 00000001800bdc74     hb-common.obj
 0002:00032c74       $unwind$??$sanitize_blob@UCBDT@OT@@@hb_sanitize_context_t@@QEAAPEAUhb_blob_t@@PEAU1@@Z 00000001800bdc74     hb-ot-color.obj
 0002:00032c90       $unwind$??$sanitize_blob@UVVAR@OT@@@hb_sanitize_context_t@@QEAAPEAUhb_blob_t@@PEAU1@@Z 00000001800bdc90     hb-common.obj
 0002:00032cac       $unwind$??$sanitize_blob@UHVAR@OT@@@hb_sanitize_context_t@@QEAAPEAUhb_blob_t@@PEAU1@@Z 00000001800bdcac     hb-common.obj
 0002:00032cac       $unwind$??$sanitize_blob@USVG@OT@@@hb_sanitize_context_t@@QEAAPEAUhb_blob_t@@PEAU1@@Z 00000001800bdcac     hb-ot-color.obj
 0002:00032cac       $unwind$??$sanitize_blob@Upost@OT@@@hb_sanitize_context_t@@QEAAPEAUhb_blob_t@@PEAU1@@Z 00000001800bdcac     hb-ot-font.obj
 0002:00032cac       $unwind$??$sanitize_blob@UGPOS@Layout@OT@@@hb_sanitize_context_t@@QEAAPEAUhb_blob_t@@PEAU1@@Z 00000001800bdcac     hb-ot-layout.obj
 0002:00032cac       $unwind$??$sanitize_blob@UGSUB@Layout@OT@@@hb_sanitize_context_t@@QEAAPEAUhb_blob_t@@PEAU1@@Z 00000001800bdcac     hb-ot-layout.obj
 0002:00032cac       $unwind$??$sanitize_blob@Ukern@OT@@@hb_sanitize_context_t@@QEAAPEAUhb_blob_t@@PEAU1@@Z 00000001800bdcac     hb-ot-layout.obj
 0002:00032cc8       $unwind$??$sanitize_blob@Umaxp@OT@@@hb_sanitize_context_t@@QEAAPEAUhb_blob_t@@PEAU1@@Z 00000001800bdcc8     hb-common.obj
 0002:00032cc8       $unwind$??$sanitize_blob@UOS2@OT@@@hb_sanitize_context_t@@QEAAPEAUhb_blob_t@@PEAU1@@Z 00000001800bdcc8     hb-face.obj
 0002:00032ce4       $chain$0$hb_draw_funcs_set_move_to_func 00000001800bdce4     hb-draw.obj
 0002:00032cf8       $chain$1$hb_draw_funcs_set_move_to_func 00000001800bdcf8     hb-draw.obj
 0002:00032d08       $chain$0$hb_draw_funcs_set_line_to_func 00000001800bdd08     hb-draw.obj
 0002:00032d1c       $chain$1$hb_draw_funcs_set_line_to_func 00000001800bdd1c     hb-draw.obj
 0002:00032d2c       $chain$0$hb_draw_funcs_set_quadratic_to_func 00000001800bdd2c     hb-draw.obj
 0002:00032d40       $chain$1$hb_draw_funcs_set_quadratic_to_func 00000001800bdd40     hb-draw.obj
 0002:00032d50       $chain$0$hb_draw_funcs_set_cubic_to_func 00000001800bdd50     hb-draw.obj
 0002:00032d64       $chain$1$hb_draw_funcs_set_cubic_to_func 00000001800bdd64     hb-draw.obj
 0002:00032d74       $chain$0$hb_draw_funcs_set_close_path_func 00000001800bdd74     hb-draw.obj
 0002:00032d88       $chain$1$hb_draw_funcs_set_close_path_func 00000001800bdd88     hb-draw.obj
 0002:00032d98       $chain$1$hb_draw_funcs_destroy 00000001800bdd98     hb-draw.obj
 0002:00032db0       $chain$2$hb_draw_funcs_destroy 00000001800bddb0     hb-draw.obj
 0002:00032dc4       $chain$3$hb_draw_funcs_destroy 00000001800bddc4     hb-draw.obj
 0002:00032dd4       $unwind$?line_to@hb_draw_funcs_t@@QEAAXPEAXAEAUhb_draw_state_t@@MM@Z 00000001800bddd4     hb-draw.obj
 0002:00032df0       $unwind$?quadratic_to@hb_draw_funcs_t@@QEAAXPEAXAEAUhb_draw_state_t@@MMMM@Z 00000001800bddf0     hb-draw.obj
 0002:00032e10       $unwind$?cubic_to@hb_draw_funcs_t@@QEAAXPEAXAEAUhb_draw_state_t@@MMMMMM@Z 00000001800bde10     hb-draw.obj
 0002:00032e30       $unwind$?hb_draw_quadratic_to_nil@@YAXPEAUhb_draw_funcs_t@@PEAXPEAUhb_draw_state_t@@MMMM1@Z 00000001800bde30     hb-draw.obj
 0002:00032e3c       $unwind$?end_serialize@hb_serialize_context_t@@QEAAXXZ 00000001800bde3c     hb-face-builder.obj
 0002:00032e44       $unwind$?pop_pack@hb_serialize_context_t@@QEAAI_N@Z 00000001800bde44     hb-face-builder.obj
 0002:00032e58       $chain$1$?pop_pack@hb_serialize_context_t@@QEAAI_N@Z 00000001800bde58     hb-face-builder.obj
 0002:00032e70       $chain$3$?pop_pack@hb_serialize_context_t@@QEAAI_N@Z 00000001800bde70     hb-face-builder.obj
 0002:00032e88       $chain$4$?pop_pack@hb_serialize_context_t@@QEAAI_N@Z 00000001800bde88     hb-face-builder.obj
 0002:00032e98       $chain$1$?resolve_links@hb_serialize_context_t@@QEAAXXZ 00000001800bde98     hb-face-builder.obj
 0002:00032eb0       $chain$5$?resolve_links@hb_serialize_context_t@@QEAAXXZ 00000001800bdeb0     hb-face-builder.obj
 0002:00032ed0       $chain$6$?resolve_links@hb_serialize_context_t@@QEAAXXZ 00000001800bded0     hb-face-builder.obj
 0002:00032ee0       $chain$7$?resolve_links@hb_serialize_context_t@@QEAAXXZ 00000001800bdee0     hb-face-builder.obj
 0002:00032ef0       $unwind$??1?$hb_pool_t@Uobject_t@hb_serialize_context_t@@$0CA@@@QEAA@XZ 00000001800bdef0     hb-face-builder.obj
 0002:00032f0c       $chain$0$?alloc@?$hb_pool_t@Uobject_t@hb_serialize_context_t@@$0CA@@@QEAAPEAUobject_t@hb_serialize_context_t@@XZ 00000001800bdf0c     hb-face-builder.obj
 0002:00032f20       $chain$1$?alloc@?$hb_pool_t@Uobject_t@hb_serialize_context_t@@$0CA@@@QEAAPEAUobject_t@hb_serialize_context_t@@XZ 00000001800bdf20     hb-face-builder.obj
 0002:00032f20       $chain$3$?alloc@?$hb_pool_t@Uobject_t@hb_serialize_context_t@@$0CA@@@QEAAPEAUobject_t@hb_serialize_context_t@@XZ 00000001800bdf20     hb-face-builder.obj
 0002:00032f30       $chain$2$?alloc@?$hb_pool_t@Uobject_t@hb_serialize_context_t@@$0CA@@@QEAAPEAUobject_t@hb_serialize_context_t@@XZ 00000001800bdf30     hb-face-builder.obj
 0002:00032f44       $unwind$?resize@?$hb_hashmap_t@PEBUobject_t@hb_serialize_context_t@@I$0A@@@QEAA_NI@Z 00000001800bdf44     hb-face-builder.obj
 0002:00032f58       $chain$0$?resize@?$hb_hashmap_t@PEBUobject_t@hb_serialize_context_t@@I$0A@@@QEAA_NI@Z 00000001800bdf58     hb-face-builder.obj
 0002:00032f6c       $chain$4$?resize@?$hb_hashmap_t@PEBUobject_t@hb_serialize_context_t@@I$0A@@@QEAA_NI@Z 00000001800bdf6c     hb-face-builder.obj
 0002:00032f8c       $chain$5$?resize@?$hb_hashmap_t@PEBUobject_t@hb_serialize_context_t@@I$0A@@@QEAA_NI@Z 00000001800bdf8c     hb-face-builder.obj
 0002:00032fa0       $chain$6$?resize@?$hb_hashmap_t@PEBUobject_t@hb_serialize_context_t@@I$0A@@@QEAA_NI@Z 00000001800bdfa0     hb-face-builder.obj
 0002:00032fb0       $chain$7$?resize@?$hb_hashmap_t@PEBUobject_t@hb_serialize_context_t@@I$0A@@@QEAA_NI@Z 00000001800bdfb0     hb-face-builder.obj
 0002:00032fc0       $chain$8$?resize@?$hb_hashmap_t@PEBUobject_t@hb_serialize_context_t@@I$0A@@@QEAA_NI@Z 00000001800bdfc0     hb-face-builder.obj
 0002:00032fd0       $unwind$??8item_t@?$hb_hashmap_t@PEBUobject_t@hb_serialize_context_t@@I$0A@@@QEBA_NAEBQEBUobject_t@hb_serialize_context_t@@@Z 00000001800bdfd0     hb-face-builder.obj
 0002:00032fe4       $unwind$?item_for_hash@?$hb_hashmap_t@PEBUobject_t@hb_serialize_context_t@@I$0A@@@QEBAAEAUitem_t@1@AEBQEBUobject_t@hb_serialize_context_t@@I@Z 00000001800bdfe4     hb-face-builder.obj
 0002:00032ffc       $unwind$hb_face_destroy    00000001800bdffc     hb-face.obj
 0002:00032ffc       $unwind$hb_shape_plan_destroy 00000001800bdffc     hb-shape-plan.obj
 0002:00033004       $chain$1$hb_face_destroy   00000001800be004     hb-face.obj
 0002:0003301c       $chain$2$hb_face_destroy   00000001800be01c     hb-face.obj
 0002:0003302c       $chain$0$hb_face_get_user_data 00000001800be02c     hb-face.obj
 0002:00033040       $chain$3$hb_face_get_user_data 00000001800be040     hb-face.obj
 0002:00033058       $chain$5$hb_face_get_user_data 00000001800be058     hb-face.obj
 0002:00033070       $chain$6$hb_face_get_user_data 00000001800be070     hb-face.obj
 0002:00033080       $chain$0$??C?$hb_lazy_loader_t@UOS2@OT@@U?$hb_table_lazy_loader_t@UOS2@OT@@$05$00@@Uhb_face_t@@$05Uhb_blob_t@@@@QEBAPEBUOS2@OT@@XZ 00000001800be080     hb-face.obj
 0002:00033094       $chain$1$??C?$hb_lazy_loader_t@UOS2@OT@@U?$hb_table_lazy_loader_t@UOS2@OT@@$05$00@@Uhb_face_t@@$05Uhb_blob_t@@@@QEBAPEBUOS2@OT@@XZ 00000001800be094     hb-face.obj
 0002:000330a4       $unwind$?get_glyph@accelerator_t@CmapSubtableFormat4@OT@@QEBA_NIPEAI@Z 00000001800be0a4     hb-face.obj
 0002:000330bc       $unwind$?get_glyph@?$CmapSubtableLongSegmented@UCmapSubtableFormat12@OT@@@OT@@QEBA_NIPEAI@Z 00000001800be0bc     hb-face.obj
 0002:000330c4       $unwind$?sanitize@CmapSubtable@OT@@QEBA_NPEAUhb_sanitize_context_t@@@Z 00000001800be0c4     hb-face.obj
 0002:000330d0       $chain$1$?sanitize@CmapSubtable@OT@@QEBA_NPEAUhb_sanitize_context_t@@@Z 00000001800be0d0     hb-face.obj
 0002:000330e8       $chain$3$?sanitize@CmapSubtable@OT@@QEBA_NPEAUhb_sanitize_context_t@@@Z 00000001800be0e8     hb-face.obj
 0002:000330e8       $chain$5$?sanitize@CmapSubtable@OT@@QEBA_NPEAUhb_sanitize_context_t@@@Z 00000001800be0e8     hb-face.obj
 0002:000330e8       $chain$7$?sanitize@CmapSubtable@OT@@QEBA_NPEAUhb_sanitize_context_t@@@Z 00000001800be0e8     hb-face.obj
 0002:00033100       $chain$10$?sanitize@CmapSubtable@OT@@QEBA_NPEAUhb_sanitize_context_t@@@Z 00000001800be100     hb-face.obj
 0002:0003311c       $chain$12$?sanitize@CmapSubtable@OT@@QEBA_NPEAUhb_sanitize_context_t@@@Z 00000001800be11c     hb-face.obj
 0002:00033138       $chain$13$?sanitize@CmapSubtable@OT@@QEBA_NPEAUhb_sanitize_context_t@@@Z 00000001800be138     hb-face.obj
 0002:00033148       $unwind$??0accelerator_t@cmap@OT@@QEAA@PEAUhb_face_t@@@Z 00000001800be148     hb-face.obj
 0002:00033164       $unwind$?find_subtable@cmap@OT@@IEBAPEBUCmapSubtable@2@II@Z 00000001800be164     hb-face.obj
 0002:00033164       $unwind$__scrt_is_nonwritable_in_current_image$filt$0 00000001800be164     MSVCRT:utility.obj
 0002:0003316c       $chain$3$?find_subtable@cmap@OT@@IEBAPEBUCmapSubtable@2@II@Z 00000001800be16c     hb-face.obj
 0002:0003318c       $chain$4$?find_subtable@cmap@OT@@IEBAPEBUCmapSubtable@2@II@Z 00000001800be18c     hb-face.obj
 0002:0003319c       $unwind$?sanitize@cmap@OT@@QEBA_NPEAUhb_sanitize_context_t@@@Z 00000001800be19c     hb-face.obj
 0002:000331b4       $unwind$??$hb_object_set_user_data@Uhb_face_t@@@@YA_NPEAUhb_face_t@@PEAUhb_user_data_key_t@@PEAXP6AX2@ZH@Z 00000001800be1b4     hb-face.obj
 0002:000331b4       $unwind$?get_extents@accelerator_t@CBDT@OT@@QEBA_NPEAUhb_font_t@@IPEAUhb_glyph_extents_t@@_N@Z 00000001800be1b4     hb-ot-font.obj
 0002:000331cc       $unwind$??$sanitize_blob@Ucmap@OT@@@hb_sanitize_context_t@@QEAAPEAUhb_blob_t@@PEAU1@@Z 00000001800be1cc     hb-face.obj
 0002:000331cc       $unwind$??$sanitize_blob@Uavar@OT@@@hb_sanitize_context_t@@QEAAPEAUhb_blob_t@@PEAU1@@Z 00000001800be1cc     hb-font.obj
 0002:000331e8       $unwind$_hb_fallback_shape 00000001800be1e8     hb-fallback-shape.obj
 0002:000331f4       $chain$1$_hb_fallback_shape 00000001800be1f4     hb-fallback-shape.obj
 0002:0003320c       $chain$5$_hb_fallback_shape 00000001800be20c     hb-fallback-shape.obj
 0002:0003322c       $chain$6$_hb_fallback_shape 00000001800be22c     hb-fallback-shape.obj
 0002:0003323c       $chain$7$_hb_fallback_shape 00000001800be23c     hb-fallback-shape.obj
 0002:0003324c       $chain$1$hb_font_funcs_destroy 00000001800be24c     hb-font.obj
 0002:00033264       $chain$2$hb_font_funcs_destroy 00000001800be264     hb-font.obj
 0002:00033278       $chain$3$hb_font_funcs_destroy 00000001800be278     hb-font.obj
 0002:00033288       $chain$0$hb_font_funcs_set_font_h_extents_func 00000001800be288     hb-font.obj
 0002:0003329c       $chain$1$hb_font_funcs_set_font_h_extents_func 00000001800be29c     hb-font.obj
 0002:000332ac       $chain$0$hb_font_funcs_set_font_v_extents_func 00000001800be2ac     hb-font.obj
 0002:000332c0       $chain$1$hb_font_funcs_set_font_v_extents_func 00000001800be2c0     hb-font.obj
 0002:000332d0       $chain$0$hb_font_funcs_set_nominal_glyph_func 00000001800be2d0     hb-font.obj
 0002:000332e4       $chain$1$hb_font_funcs_set_nominal_glyph_func 00000001800be2e4     hb-font.obj
 0002:000332f4       $chain$0$hb_font_funcs_set_nominal_glyphs_func 00000001800be2f4     hb-font.obj
 0002:00033308       $chain$1$hb_font_funcs_set_nominal_glyphs_func 00000001800be308     hb-font.obj
 0002:00033318       $chain$0$hb_font_funcs_set_variation_glyph_func 00000001800be318     hb-font.obj
 0002:0003332c       $chain$1$hb_font_funcs_set_variation_glyph_func 00000001800be32c     hb-font.obj
 0002:0003333c       $chain$0$hb_font_funcs_set_glyph_h_advance_func 00000001800be33c     hb-font.obj
 0002:00033350       $chain$1$hb_font_funcs_set_glyph_h_advance_func 00000001800be350     hb-font.obj
 0002:00033360       $chain$0$hb_font_funcs_set_glyph_v_advance_func 00000001800be360     hb-font.obj
 0002:00033374       $chain$1$hb_font_funcs_set_glyph_v_advance_func 00000001800be374     hb-font.obj
 0002:00033384       $chain$0$hb_font_funcs_set_glyph_h_advances_func 00000001800be384     hb-font.obj
 0002:00033398       $chain$1$hb_font_funcs_set_glyph_h_advances_func 00000001800be398     hb-font.obj
 0002:000333a8       $chain$0$hb_font_funcs_set_glyph_v_advances_func 00000001800be3a8     hb-font.obj
 0002:000333bc       $chain$1$hb_font_funcs_set_glyph_v_advances_func 00000001800be3bc     hb-font.obj
 0002:000333cc       $chain$0$hb_font_funcs_set_glyph_h_origin_func 00000001800be3cc     hb-font.obj
 0002:000333e0       $chain$1$hb_font_funcs_set_glyph_h_origin_func 00000001800be3e0     hb-font.obj
 0002:000333f0       $chain$0$hb_font_funcs_set_glyph_v_origin_func 00000001800be3f0     hb-font.obj
 0002:00033404       $chain$1$hb_font_funcs_set_glyph_v_origin_func 00000001800be404     hb-font.obj
 0002:00033414       $chain$0$hb_font_funcs_set_glyph_h_kerning_func 00000001800be414     hb-font.obj
 0002:00033428       $chain$1$hb_font_funcs_set_glyph_h_kerning_func 00000001800be428     hb-font.obj
 0002:00033438       $chain$0$hb_font_funcs_set_glyph_extents_func 00000001800be438     hb-font.obj
 0002:0003344c       $chain$1$hb_font_funcs_set_glyph_extents_func 00000001800be44c     hb-font.obj
 0002:0003345c       $chain$0$hb_font_funcs_set_glyph_contour_point_func 00000001800be45c     hb-font.obj
 0002:00033470       $chain$1$hb_font_funcs_set_glyph_contour_point_func 00000001800be470     hb-font.obj
 0002:00033480       $chain$0$hb_font_funcs_set_glyph_name_func 00000001800be480     hb-font.obj
 0002:00033494       $chain$1$hb_font_funcs_set_glyph_name_func 00000001800be494     hb-font.obj
 0002:000334a4       $chain$0$hb_font_funcs_set_glyph_from_name_func 00000001800be4a4     hb-font.obj
 0002:000334b8       $chain$1$hb_font_funcs_set_glyph_from_name_func 00000001800be4b8     hb-font.obj
 0002:000334c8       $chain$0$hb_font_funcs_set_draw_glyph_func 00000001800be4c8     hb-font.obj
 0002:000334dc       $chain$1$hb_font_funcs_set_draw_glyph_func 00000001800be4dc     hb-font.obj
 0002:000334ec       $chain$0$hb_font_funcs_set_paint_glyph_func 00000001800be4ec     hb-font.obj
 0002:00033500       $chain$1$hb_font_funcs_set_paint_glyph_func 00000001800be500     hb-font.obj
 0002:00033510       $chain$0$hb_font_destroy   00000001800be510     hb-font.obj
 0002:00033524       $chain$1$hb_font_destroy   00000001800be524     hb-font.obj
 0002:00033534       $unwind$hb_font_set_funcs  00000001800be534     hb-font.obj
 0002:00033544       $chain$1$hb_font_set_funcs 00000001800be544     hb-font.obj
 0002:0003355c       $chain$2$hb_font_set_funcs 00000001800be55c     hb-font.obj
 0002:0003356c       $unwind$hb_font_set_variations 00000001800be56c     hb-font.obj
 0002:00033578       $chain$4$hb_font_set_variations 00000001800be578     hb-font.obj
 0002:0003359c       $chain$5$hb_font_set_variations 00000001800be59c     hb-font.obj
 0002:000335ac       $unwind$hb_font_set_var_coords_normalized 00000001800be5ac     hb-font.obj
 0002:000335b8       $chain$3$hb_font_set_var_coords_normalized 00000001800be5b8     hb-font.obj
 0002:000335d8       $chain$4$hb_font_set_var_coords_normalized 00000001800be5d8     hb-font.obj
 0002:000335ec       $chain$7$hb_font_set_var_coords_normalized 00000001800be5ec     hb-font.obj
 0002:00033608       $chain$8$hb_font_set_var_coords_normalized 00000001800be608     hb-font.obj
 0002:00033618       $chain$9$hb_font_set_var_coords_normalized 00000001800be618     hb-font.obj
 0002:00033628       $chain$10$hb_font_set_var_coords_normalized 00000001800be628     hb-font.obj
 0002:00033638       $chain$0$hb_font_funcs_set_glyph_v_kerning_func 00000001800be638     hb-font.obj
 0002:0003364c       $chain$1$hb_font_funcs_set_glyph_v_kerning_func 00000001800be64c     hb-font.obj
 0002:0003365c       $chain$0$?get@?$hb_lazy_loader_t@Ufvar@OT@@U?$hb_table_lazy_loader_t@Ufvar@OT@@$0BC@$00@@Uhb_face_t@@$0BC@Uhb_blob_t@@@@QEBAPEBUfvar@OT@@XZ 00000001800be65c     hb-font.obj
 0002:00033670       $chain$1$?get@?$hb_lazy_loader_t@Ufvar@OT@@U?$hb_table_lazy_loader_t@Ufvar@OT@@$0BC@$00@@Uhb_face_t@@$0BC@Uhb_blob_t@@@@QEBAPEBUfvar@OT@@XZ 00000001800be670     hb-font.obj
 0002:00033680       $chain$0$??C?$hb_lazy_loader_t@Uavar@OT@@U?$hb_table_lazy_loader_t@Uavar@OT@@$0BD@$00@@Uhb_face_t@@$0BD@Uhb_blob_t@@@@QEBAPEBUavar@OT@@XZ 00000001800be680     hb-font.obj
 0002:00033694       $chain$1$??C?$hb_lazy_loader_t@Uavar@OT@@U?$hb_table_lazy_loader_t@Uavar@OT@@$0BD@$00@@Uhb_face_t@@$0BD@Uhb_blob_t@@@@QEBAPEBUavar@OT@@XZ 00000001800be694     hb-font.obj
 0002:000336a4       $unwind$?mults_changed@hb_font_t@@QEAAXXZ 00000001800be6a4     hb-font.obj
 0002:000336b8       $unwind$?get_delta@VarData@OT@@QEBAMIPEBHIAEBUVarRegionList@2@PEAM@Z 00000001800be6b8     hb-font.obj
 0002:000336c0       $chain$7$?get_delta@VarData@OT@@QEBAMIPEBHIAEBUVarRegionList@2@PEAM@Z 00000001800be6c0     hb-font.obj
 0002:000336f0       $chain$9$?get_delta@VarData@OT@@QEBAMIPEBHIAEBUVarRegionList@2@PEAM@Z 00000001800be6f0     hb-font.obj
 0002:00033720       $unwind$?get_delta@VariationStore@OT@@QEBAMIPEBHIPEAM@Z 00000001800be720     hb-font.obj
 0002:00033720       $unwind$?hb_font_get_glyph_h_origin_default@@YAHPEAUhb_font_t@@PEAXIPEAH21@Z 00000001800be720     hb-font.obj
 0002:00033720       $unwind$?hb_font_get_glyph_v_origin_default@@YAHPEAUhb_font_t@@PEAXIPEAH21@Z 00000001800be720     hb-font.obj
 0002:00033720       $unwind$?hb_jdk_get_glyph_h_advance@@YAHPEAUhb_font_t@@PEAXI1@Z 00000001800be720     hb-jdk-font.obj
 0002:00033720       $unwind$?reference_table@@YAPEAUhb_blob_t@@PEAUhb_face_t@@IPEAX@Z 00000001800be720     hb-jdk-font.obj
 0002:00033720       $unwind$Java_sun_font_SunLayoutEngine_createFace 00000001800be720     hb-jdk-font.obj
 0002:00033720       $unwind$hb_ot_color_palette_get_colors 00000001800be720     hb-ot-color.obj
 0002:00033720       $unwind$?apply@?$SingleSubstFormat1_3@USmallTypes@Layout@OT@@@GSUB_impl@Layout@OT@@QEBA_NPEAUhb_ot_apply_context_t@4@@Z 00000001800be720     hb-ot-layout.obj
 0002:00033720       $unwind$?apply@SinglePosFormat1@GPOS_impl@Layout@OT@@QEBA_NPEAUhb_ot_apply_context_t@4@@Z 00000001800be720     hb-ot-layout.obj
 0002:00033730       $unwind$?map@SegmentMaps@OT@@QEBAHHII@Z 00000001800be730     hb-font.obj
 0002:0003373c       $chain$0$?map@SegmentMaps@OT@@QEBAHHII@Z 00000001800be73c     hb-font.obj
 0002:00033750       $chain$5$?map@SegmentMaps@OT@@QEBAHHII@Z 00000001800be750     hb-font.obj
 0002:00033770       $unwind$?sanitize@avar@OT@@QEBA_NPEAUhb_sanitize_context_t@@@Z 00000001800be770     hb-font.obj
 0002:00033770       $unwind$?sanitize@FeatureTableSubstitution@OT@@QEBA_NPEAUhb_sanitize_context_t@@@Z 00000001800be770     hb-ot-layout.obj
 0002:00033788       $unwind$?map_coords@avar@OT@@QEBAXPEAHI@Z 00000001800be788     hb-font.obj
 0002:00033798       $chain$1$?map_coords@avar@OT@@QEBAXPEAHI@Z 00000001800be798     hb-font.obj
 0002:000337b0       $chain$3$?map_coords@avar@OT@@QEBAXPEAHI@Z 00000001800be7b0     hb-font.obj
 0002:000337c8       $chain$4$?map_coords@avar@OT@@QEBAXPEAHI@Z 00000001800be7c8     hb-font.obj
 0002:000337c8       $chain$6$?map_coords@avar@OT@@QEBAXPEAHI@Z 00000001800be7c8     hb-font.obj
 0002:000337d8       $chain$5$?map_coords@avar@OT@@QEBAXPEAHI@Z 00000001800be7d8     hb-font.obj
 0002:000337f0       $chain$7$?map_coords@avar@OT@@QEBAXPEAHI@Z 00000001800be7f0     hb-font.obj
 0002:00033800       $unwind$?hb_font_get_nominal_glyph_default@@YAHPEAUhb_font_t@@PEAXIPEAI1@Z 00000001800be800     hb-font.obj
 0002:00033808       $unwind$?hb_font_get_nominal_glyphs_default@@YAIPEAUhb_font_t@@PEAXIPEBIIPEAII1@Z 00000001800be808     hb-font.obj
 0002:00033818       $chain$3$?hb_font_get_nominal_glyphs_default@@YAIPEAUhb_font_t@@PEAXIPEBIIPEAII1@Z 00000001800be818     hb-font.obj
 0002:00033838       $chain$5$?hb_font_get_nominal_glyphs_default@@YAIPEAUhb_font_t@@PEAXIPEBIIPEAII1@Z 00000001800be838     hb-font.obj
 0002:00033858       $chain$6$?hb_font_get_nominal_glyphs_default@@YAIPEAUhb_font_t@@PEAXIPEBIIPEAII1@Z 00000001800be858     hb-font.obj
 0002:00033868       $unwind$?hb_font_get_glyph_h_advance_default@@YAHPEAUhb_font_t@@PEAXI1@Z 00000001800be868     hb-font.obj
 0002:00033868       $unwind$?hb_font_get_glyph_v_advance_default@@YAHPEAUhb_font_t@@PEAXI1@Z 00000001800be868     hb-font.obj
 0002:00033870       $unwind$?hb_font_get_glyph_h_advances_default@@YAXPEAUhb_font_t@@PEAXIPEBIIPEAHI1@Z 00000001800be870     hb-font.obj
 0002:00033870       $unwind$?hb_font_get_glyph_v_advances_default@@YAXPEAUhb_font_t@@PEAXIPEBIIPEAHI1@Z 00000001800be870     hb-font.obj
 0002:00033884       $chain$1$?hb_font_get_glyph_h_advances_default@@YAXPEAUhb_font_t@@PEAXIPEBIIPEAHI1@Z 00000001800be884     hb-font.obj
 0002:0003389c       $chain$2$?hb_font_get_glyph_h_advances_default@@YAXPEAUhb_font_t@@PEAXIPEBIIPEAHI1@Z 00000001800be89c     hb-font.obj
 0002:000338ac       $chain$1$?hb_font_get_glyph_v_advances_default@@YAXPEAUhb_font_t@@PEAXIPEBIIPEAHI1@Z 00000001800be8ac     hb-font.obj
 0002:000338c4       $chain$2$?hb_font_get_glyph_v_advances_default@@YAXPEAUhb_font_t@@PEAXIPEBIIPEAHI1@Z 00000001800be8c4     hb-font.obj
 0002:000338d4       $unwind$?hb_font_get_glyph_contour_point_default@@YAHPEAUhb_font_t@@PEAXIIPEAH21@Z 00000001800be8d4     hb-font.obj
 0002:000338e4       $unwind$?hb_draw_line_to_default@@YAXPEAUhb_draw_funcs_t@@PEAXPEAUhb_draw_state_t@@MM1@Z 00000001800be8e4     hb-font.obj
 0002:000338f0       $unwind$?hb_draw_quadratic_to_default@@YAXPEAUhb_draw_funcs_t@@PEAXPEAUhb_draw_state_t@@MMMM1@Z 00000001800be8f0     hb-font.obj
 0002:00033900       $unwind$?hb_draw_cubic_to_default@@YAXPEAUhb_draw_funcs_t@@PEAXPEAUhb_draw_state_t@@MMMMMM1@Z 00000001800be900     hb-font.obj
 0002:00033918       $unwind$?hb_font_paint_glyph_default@@YAXPEAUhb_font_t@@PEAXIPEAUhb_paint_funcs_t@@1II1@Z 00000001800be918     hb-font.obj
 0002:00033918       $unwind$?paint_glyph@PaintGlyph@OT@@QEBAXPEAUhb_paint_context_t@2@@Z 00000001800be918     hb-ot-font.obj
 0002:00033918       $unwind$?apply@?$ChainContextFormat1_4@USmallTypes@Layout@OT@@@OT@@QEBA_NPEAUhb_ot_apply_context_t@2@@Z 00000001800be918     hb-ot-layout.obj
 0002:00033930       $unwind$??$sanitize_blob@Ufvar@OT@@@hb_sanitize_context_t@@QEAAPEAUhb_blob_t@@PEAU1@@Z 00000001800be930     hb-font.obj
 0002:0003394c       $chain$0$?hb_jdk_get_glyph_h_advance@@YAHPEAUhb_font_t@@PEAXI1@Z 00000001800be94c     hb-jdk-font.obj
 0002:00033960       $chain$1$?hb_jdk_get_glyph_h_advance@@YAHPEAUhb_font_t@@PEAXI1@Z 00000001800be960     hb-jdk-font.obj
 0002:00033970       $chain$0$?hb_jdk_get_glyph_v_advance@@YAHPEAUhb_font_t@@PEAXI1@Z 00000001800be970     hb-jdk-font.obj
 0002:00033984       $chain$1$?hb_jdk_get_glyph_v_advance@@YAHPEAUhb_font_t@@PEAXI1@Z 00000001800be984     hb-jdk-font.obj
 0002:00033994       $unwind$?hb_parse_int@@YA_NPEAPEBDPEBDPEAH_N@Z 00000001800be994     hb-number.obj
 0002:000339ac       $unwind$?strtod_rl@@YANPEBDPEAPEBD@Z 00000001800be9ac     hb-number.obj
 0002:000339bc       $chain$6$?strtod_rl@@YANPEBDPEAPEBD@Z 00000001800be9bc     hb-number.obj
 0002:000339e8       $chain$7$?strtod_rl@@YANPEBDPEAPEBD@Z 00000001800be9e8     hb-number.obj
 0002:000339fc       $chain$8$?strtod_rl@@YANPEBDPEAPEBD@Z 00000001800be9fc     hb-number.obj
 0002:00033a0c       $unwind$?move_to@hb_draw_session_t@@QEAAXMM@Z 00000001800bea0c     hb-ot-cff1-table.obj
 0002:00033a1c       $unwind$?cubic_to@hb_draw_session_t@@QEAAXMMMMMM@Z 00000001800bea1c     hb-ot-cff1-table.obj
 0002:00033a2c       $unwind$?get_fd@FDSelect@CFF@@QEBAII@Z 00000001800bea2c     hb-ot-cff1-table.obj
 0002:00033a34       $chain$4$?get_fd@FDSelect@CFF@@QEBAII@Z 00000001800bea34     hb-ot-cff1-table.obj
 0002:00033a58       $chain$5$?get_fd@FDSelect@CFF@@QEBAII@Z 00000001800bea58     hb-ot-cff1-table.obj
 0002:00033a68       $chain$0$?get_glyph@Charset@CFF@@QEBAIII@Z 00000001800bea68     hb-ot-cff1-table.obj
 0002:00033a7c       $chain$1$?get_glyph@Charset@CFF@@QEBAIII@Z 00000001800bea7c     hb-ot-cff1-table.obj
 0002:00033a7c       $chain$11$?get_glyph@Charset@CFF@@QEBAIII@Z 00000001800bea7c     hb-ot-cff1-table.obj
 0002:00033a8c       $chain$4$?get_glyph@Charset@CFF@@QEBAIII@Z 00000001800bea8c     hb-ot-cff1-table.obj
 0002:00033aa8       $chain$6$?get_glyph@Charset@CFF@@QEBAIII@Z 00000001800beaa8     hb-ot-cff1-table.obj
 0002:00033ac4       $chain$10$?get_glyph@Charset@CFF@@QEBAIII@Z 00000001800beac4     hb-ot-cff1-table.obj
 0002:00033ac4       $chain$8$?get_glyph@Charset@CFF@@QEBAIII@Z 00000001800beac4     hb-ot-cff1-table.obj
 0002:00033ad8       $chain$0$??A?$CFFIndex@U?$IntType@G$01@OT@@@CFF@@QEBA?AU?$hb_array_t@$$CBE@@I@Z 00000001800bead8     hb-ot-cff1-table.obj
 0002:00033aec       $chain$1$??A?$CFFIndex@U?$IntType@G$01@OT@@@CFF@@QEBA?AU?$hb_array_t@$$CBE@@I@Z 00000001800beaec     hb-ot-cff1-table.obj
 0002:00033afc       $unwind$?get_extents@accelerator_t@cff1@OT@@QEBA_NPEAUhb_font_t@@IPEAUhb_glyph_extents_t@@@Z 00000001800beafc     hb-ot-cff1-table.obj
 0002:00033b14       $chain$6$?get_extents@accelerator_t@cff1@OT@@QEBA_NPEAUhb_font_t@@IPEAUhb_glyph_extents_t@@@Z 00000001800beb14     hb-ot-cff1-table.obj
 0002:00033b34       $chain$7$?get_extents@accelerator_t@cff1@OT@@QEBA_NPEAUhb_font_t@@IPEAUhb_glyph_extents_t@@@Z 00000001800beb34     hb-ot-cff1-table.obj
 0002:00033b50       $chain$8$?get_extents@accelerator_t@cff1@OT@@QEBA_NPEAUhb_font_t@@IPEAUhb_glyph_extents_t@@@Z 00000001800beb50     hb-ot-cff1-table.obj
 0002:00033b60       $unwind$?call_subr@?$cs_interp_env_t@Unumber_t@CFF@@U?$Subrs@U?$IntType@G$01@OT@@@2@@CFF@@QEAAXAEBU?$biased_subrs_t@U?$Subrs@U?$IntType@G$01@OT@@@CFF@@@2@W4cs_type_t@2@@Z 00000001800beb60     hb-ot-cff1-table.obj
 0002:00033b60       $unwind$?call_subr@?$cs_interp_env_t@Unumber_t@CFF@@U?$Subrs@U?$IntType@I$03@OT@@@2@@CFF@@QEAAXAEBU?$biased_subrs_t@U?$Subrs@U?$IntType@I$03@OT@@@CFF@@@2@W4cs_type_t@2@@Z 00000001800beb60     hb-ot-cff2-table.obj
 0002:00033b70       $chain$0$?call_subr@?$cs_interp_env_t@Unumber_t@CFF@@U?$Subrs@U?$IntType@G$01@OT@@@2@@CFF@@QEAAXAEBU?$biased_subrs_t@U?$Subrs@U?$IntType@G$01@OT@@@CFF@@@2@W4cs_type_t@2@@Z 00000001800beb70     hb-ot-cff1-table.obj
 0002:00033b84       $chain$1$?call_subr@?$cs_interp_env_t@Unumber_t@CFF@@U?$Subrs@U?$IntType@G$01@OT@@@2@@CFF@@QEAAXAEBU?$biased_subrs_t@U?$Subrs@U?$IntType@G$01@OT@@@CFF@@@2@W4cs_type_t@2@@Z 00000001800beb84     hb-ot-cff1-table.obj
 0002:00033b94       $chain$1$?rrcurveto@?$path_procs_t@Ucff1_path_procs_extents_t@@Ucff1_cs_interp_env_t@CFF@@Ucff1_extents_param_t@@@CFF@@SAXAEAUcff1_cs_interp_env_t@2@AEAUcff1_extents_param_t@@@Z 00000001800beb94     hb-ot-cff1-table.obj
 0002:00033bac       $chain$2$?rrcurveto@?$path_procs_t@Ucff1_path_procs_extents_t@@Ucff1_cs_interp_env_t@CFF@@Ucff1_extents_param_t@@@CFF@@SAXAEAUcff1_cs_interp_env_t@2@AEAUcff1_extents_param_t@@@Z 00000001800bebac     hb-ot-cff1-table.obj
 0002:00033bbc       $chain$0$?rcurveline@?$path_procs_t@Ucff1_path_procs_extents_t@@Ucff1_cs_interp_env_t@CFF@@Ucff1_extents_param_t@@@CFF@@SAXAEAUcff1_cs_interp_env_t@2@AEAUcff1_extents_param_t@@@Z 00000001800bebbc     hb-ot-cff1-table.obj
 0002:00033bd0       $chain$2$?rcurveline@?$path_procs_t@Ucff1_path_procs_extents_t@@Ucff1_cs_interp_env_t@CFF@@Ucff1_extents_param_t@@@CFF@@SAXAEAUcff1_cs_interp_env_t@2@AEAUcff1_extents_param_t@@@Z 00000001800bebd0     hb-ot-cff1-table.obj
 0002:00033be8       $chain$3$?rcurveline@?$path_procs_t@Ucff1_path_procs_extents_t@@Ucff1_cs_interp_env_t@CFF@@Ucff1_extents_param_t@@@CFF@@SAXAEAUcff1_cs_interp_env_t@2@AEAUcff1_extents_param_t@@@Z 00000001800bebe8     hb-ot-cff1-table.obj
 0002:00033bf8       $chain$4$?rcurveline@?$path_procs_t@Ucff1_path_procs_extents_t@@Ucff1_cs_interp_env_t@CFF@@Ucff1_extents_param_t@@@CFF@@SAXAEAUcff1_cs_interp_env_t@2@AEAUcff1_extents_param_t@@@Z 00000001800bebf8     hb-ot-cff1-table.obj
 0002:00033c08       $chain$2$?rlinecurve@?$path_procs_t@Ucff1_path_procs_extents_t@@Ucff1_cs_interp_env_t@CFF@@Ucff1_extents_param_t@@@CFF@@SAXAEAUcff1_cs_interp_env_t@2@AEAUcff1_extents_param_t@@@Z 00000001800bec08     hb-ot-cff1-table.obj
 0002:00033c24       $chain$3$?rlinecurve@?$path_procs_t@Ucff1_path_procs_extents_t@@Ucff1_cs_interp_env_t@CFF@@Ucff1_extents_param_t@@@CFF@@SAXAEAUcff1_cs_interp_env_t@2@AEAUcff1_extents_param_t@@@Z 00000001800bec24     hb-ot-cff1-table.obj
 0002:00033c3c       $chain$4$?rlinecurve@?$path_procs_t@Ucff1_path_procs_extents_t@@Ucff1_cs_interp_env_t@CFF@@Ucff1_extents_param_t@@@CFF@@SAXAEAUcff1_cs_interp_env_t@2@AEAUcff1_extents_param_t@@@Z 00000001800bec3c     hb-ot-cff1-table.obj
 0002:00033c50       $chain$5$?rlinecurve@?$path_procs_t@Ucff1_path_procs_extents_t@@Ucff1_cs_interp_env_t@CFF@@Ucff1_extents_param_t@@@CFF@@SAXAEAUcff1_cs_interp_env_t@2@AEAUcff1_extents_param_t@@@Z 00000001800bec50     hb-ot-cff1-table.obj
 0002:00033c60       $chain$0$?vvcurveto@?$path_procs_t@Ucff1_path_procs_extents_t@@Ucff1_cs_interp_env_t@CFF@@Ucff1_extents_param_t@@@CFF@@SAXAEAUcff1_cs_interp_env_t@2@AEAUcff1_extents_param_t@@@Z 00000001800bec60     hb-ot-cff1-table.obj
 0002:00033c74       $chain$1$?vvcurveto@?$path_procs_t@Ucff1_path_procs_extents_t@@Ucff1_cs_interp_env_t@CFF@@Ucff1_extents_param_t@@@CFF@@SAXAEAUcff1_cs_interp_env_t@2@AEAUcff1_extents_param_t@@@Z 00000001800bec74     hb-ot-cff1-table.obj
 0002:00033c84       $chain$0$?hhcurveto@?$path_procs_t@Ucff1_path_procs_extents_t@@Ucff1_cs_interp_env_t@CFF@@Ucff1_extents_param_t@@@CFF@@SAXAEAUcff1_cs_interp_env_t@2@AEAUcff1_extents_param_t@@@Z 00000001800bec84     hb-ot-cff1-table.obj
 0002:00033c98       $chain$1$?hhcurveto@?$path_procs_t@Ucff1_path_procs_extents_t@@Ucff1_cs_interp_env_t@CFF@@Ucff1_extents_param_t@@@CFF@@SAXAEAUcff1_cs_interp_env_t@2@AEAUcff1_extents_param_t@@@Z 00000001800bec98     hb-ot-cff1-table.obj
 0002:00033ca8       $unwind$?hvcurveto@?$path_procs_t@Ucff1_path_procs_extents_t@@Ucff1_cs_interp_env_t@CFF@@Ucff1_extents_param_t@@@CFF@@SAXAEAUcff1_cs_interp_env_t@2@AEAUcff1_extents_param_t@@@Z 00000001800beca8     hb-ot-cff1-table.obj
 0002:00033ca8       $unwind$?vhcurveto@?$path_procs_t@Ucff1_path_procs_extents_t@@Ucff1_cs_interp_env_t@CFF@@Ucff1_extents_param_t@@@CFF@@SAXAEAUcff1_cs_interp_env_t@2@AEAUcff1_extents_param_t@@@Z 00000001800beca8     hb-ot-cff1-table.obj
 0002:00033cbc       $chain$0$?vhcurveto@?$path_procs_t@Ucff1_path_procs_extents_t@@Ucff1_cs_interp_env_t@CFF@@Ucff1_extents_param_t@@@CFF@@SAXAEAUcff1_cs_interp_env_t@2@AEAUcff1_extents_param_t@@@Z 00000001800becbc     hb-ot-cff1-table.obj
 0002:00033cd0       $chain$1$?vhcurveto@?$path_procs_t@Ucff1_path_procs_extents_t@@Ucff1_cs_interp_env_t@CFF@@Ucff1_extents_param_t@@@CFF@@SAXAEAUcff1_cs_interp_env_t@2@AEAUcff1_extents_param_t@@@Z 00000001800becd0     hb-ot-cff1-table.obj
 0002:00033ce0       $chain$2$?vhcurveto@?$path_procs_t@Ucff1_path_procs_extents_t@@Ucff1_cs_interp_env_t@CFF@@Ucff1_extents_param_t@@@CFF@@SAXAEAUcff1_cs_interp_env_t@2@AEAUcff1_extents_param_t@@@Z 00000001800bece0     hb-ot-cff1-table.obj
 0002:00033cf4       $chain$3$?vhcurveto@?$path_procs_t@Ucff1_path_procs_extents_t@@Ucff1_cs_interp_env_t@CFF@@Ucff1_extents_param_t@@@CFF@@SAXAEAUcff1_cs_interp_env_t@2@AEAUcff1_extents_param_t@@@Z 00000001800becf4     hb-ot-cff1-table.obj
 0002:00033d04       $chain$0$?hvcurveto@?$path_procs_t@Ucff1_path_procs_extents_t@@Ucff1_cs_interp_env_t@CFF@@Ucff1_extents_param_t@@@CFF@@SAXAEAUcff1_cs_interp_env_t@2@AEAUcff1_extents_param_t@@@Z 00000001800bed04     hb-ot-cff1-table.obj
 0002:00033d18       $chain$1$?hvcurveto@?$path_procs_t@Ucff1_path_procs_extents_t@@Ucff1_cs_interp_env_t@CFF@@Ucff1_extents_param_t@@@CFF@@SAXAEAUcff1_cs_interp_env_t@2@AEAUcff1_extents_param_t@@@Z 00000001800bed18     hb-ot-cff1-table.obj
 0002:00033d28       $chain$2$?hvcurveto@?$path_procs_t@Ucff1_path_procs_extents_t@@Ucff1_cs_interp_env_t@CFF@@Ucff1_extents_param_t@@@CFF@@SAXAEAUcff1_cs_interp_env_t@2@AEAUcff1_extents_param_t@@@Z 00000001800bed28     hb-ot-cff1-table.obj
 0002:00033d3c       $chain$3$?hvcurveto@?$path_procs_t@Ucff1_path_procs_extents_t@@Ucff1_cs_interp_env_t@CFF@@Ucff1_extents_param_t@@@CFF@@SAXAEAUcff1_cs_interp_env_t@2@AEAUcff1_extents_param_t@@@Z 00000001800bed3c     hb-ot-cff1-table.obj
 0002:00033d4c       $unwind$?flex1@?$path_procs_t@Ucff1_path_procs_extents_t@@Ucff1_cs_interp_env_t@CFF@@Ucff1_extents_param_t@@@CFF@@SAXAEAUcff1_cs_interp_env_t@2@AEAUcff1_extents_param_t@@@Z 00000001800bed4c     hb-ot-cff1-table.obj
 0002:00033d4c       $unwind$?flex1@?$path_procs_t@Ucff1_path_procs_path_t@@Ucff1_cs_interp_env_t@CFF@@Ucff1_path_param_t@@@CFF@@SAXAEAUcff1_cs_interp_env_t@2@AEAUcff1_path_param_t@@@Z 00000001800bed4c     hb-ot-cff1-table.obj
 0002:00033d4c       $unwind$?flex@?$path_procs_t@Ucff1_path_procs_extents_t@@Ucff1_cs_interp_env_t@CFF@@Ucff1_extents_param_t@@@CFF@@SAXAEAUcff1_cs_interp_env_t@2@AEAUcff1_extents_param_t@@@Z 00000001800bed4c     hb-ot-cff1-table.obj
 0002:00033d4c       $unwind$?flex@?$path_procs_t@Ucff1_path_procs_path_t@@Ucff1_cs_interp_env_t@CFF@@Ucff1_path_param_t@@@CFF@@SAXAEAUcff1_cs_interp_env_t@2@AEAUcff1_path_param_t@@@Z 00000001800bed4c     hb-ot-cff1-table.obj
 0002:00033d4c       $unwind$?hflex1@?$path_procs_t@Ucff1_path_procs_extents_t@@Ucff1_cs_interp_env_t@CFF@@Ucff1_extents_param_t@@@CFF@@SAXAEAUcff1_cs_interp_env_t@2@AEAUcff1_extents_param_t@@@Z 00000001800bed4c     hb-ot-cff1-table.obj
 0002:00033d4c       $unwind$?hflex1@?$path_procs_t@Ucff1_path_procs_path_t@@Ucff1_cs_interp_env_t@CFF@@Ucff1_path_param_t@@@CFF@@SAXAEAUcff1_cs_interp_env_t@2@AEAUcff1_path_param_t@@@Z 00000001800bed4c     hb-ot-cff1-table.obj
 0002:00033d4c       $unwind$?hflex@?$path_procs_t@Ucff1_path_procs_extents_t@@Ucff1_cs_interp_env_t@CFF@@Ucff1_extents_param_t@@@CFF@@SAXAEAUcff1_cs_interp_env_t@2@AEAUcff1_extents_param_t@@@Z 00000001800bed4c     hb-ot-cff1-table.obj
 0002:00033d4c       $unwind$?hflex@?$path_procs_t@Ucff1_path_procs_path_t@@Ucff1_cs_interp_env_t@CFF@@Ucff1_path_param_t@@@CFF@@SAXAEAUcff1_cs_interp_env_t@2@AEAUcff1_path_param_t@@@Z 00000001800bed4c     hb-ot-cff1-table.obj
 0002:00033d4c       $unwind$?flex1@?$path_procs_t@Ucff2_path_procs_extents_t@@U?$cff2_cs_interp_env_t@Unumber_t@CFF@@@CFF@@Ucff2_extents_param_t@@@CFF@@SAXAEAU?$cff2_cs_interp_env_t@Unumber_t@CFF@@@2@AEAUcff2_extents_param_t@@@Z 00000001800bed4c     hb-ot-cff2-table.obj
 0002:00033d4c       $unwind$?flex@?$path_procs_t@Ucff2_path_procs_extents_t@@U?$cff2_cs_interp_env_t@Unumber_t@CFF@@@CFF@@Ucff2_extents_param_t@@@CFF@@SAXAEAU?$cff2_cs_interp_env_t@Unumber_t@CFF@@@2@AEAUcff2_extents_param_t@@@Z 00000001800bed4c     hb-ot-cff2-table.obj
 0002:00033d4c       $unwind$?hflex1@?$path_procs_t@Ucff2_path_procs_extents_t@@U?$cff2_cs_interp_env_t@Unumber_t@CFF@@@CFF@@Ucff2_extents_param_t@@@CFF@@SAXAEAU?$cff2_cs_interp_env_t@Unumber_t@CFF@@@2@AEAUcff2_extents_param_t@@@Z 00000001800bed4c     hb-ot-cff2-table.obj
 0002:00033d4c       $unwind$?hflex@?$path_procs_t@Ucff2_path_procs_extents_t@@U?$cff2_cs_interp_env_t@Unumber_t@CFF@@@CFF@@Ucff2_extents_param_t@@@CFF@@SAXAEAU?$cff2_cs_interp_env_t@Unumber_t@CFF@@@2@AEAUcff2_extents_param_t@@@Z 00000001800bed4c     hb-ot-cff2-table.obj
 0002:00033d5c       $unwind$?_get_bounds@@YA_NPEBUaccelerator_t@cff1@OT@@IAEAUbounds_t@@_N@Z 00000001800bed5c     hb-ot-cff1-table.obj
 0002:00033d74       $chain$0$?_get_bounds@@YA_NPEBUaccelerator_t@cff1@OT@@IAEAUbounds_t@@_N@Z 00000001800bed74     hb-ot-cff1-table.obj
 0002:00033d88       $chain$1$?_get_bounds@@YA_NPEBUaccelerator_t@cff1@OT@@IAEAUbounds_t@@_N@Z 00000001800bed88     hb-ot-cff1-table.obj
 0002:00033d98       $unwind$?process_seac@cff1_cs_opset_extents_t@@SAXAEAUcff1_cs_interp_env_t@CFF@@AEAUcff1_extents_param_t@@@Z 00000001800bed98     hb-ot-cff1-table.obj
 0002:00033da8       $chain$2$?process_seac@cff1_cs_opset_extents_t@@SAXAEAUcff1_cs_interp_env_t@CFF@@AEAUcff1_extents_param_t@@@Z 00000001800beda8     hb-ot-cff1-table.obj
 0002:00033dc4       $chain$3$?process_seac@cff1_cs_opset_extents_t@@SAXAEAUcff1_cs_interp_env_t@CFF@@AEAUcff1_extents_param_t@@@Z 00000001800bedc4     hb-ot-cff1-table.obj
 0002:00033ddc       $unwind$??$?0$$CBUaccelerator_t@cff1@OT@@@cff1_cs_interp_env_t@CFF@@QEAA@AEBU?$hb_array_t@$$CBE@@AEBUaccelerator_t@cff1@OT@@IPEBHI@Z 00000001800beddc     hb-ot-cff1-table.obj
 0002:00033df4       $unwind$?interpret@?$cs_interpreter_t@Ucff1_cs_interp_env_t@CFF@@Ucff1_cs_opset_extents_t@@Ucff1_extents_param_t@@@CFF@@QEAA_NAEAUcff1_extents_param_t@@@Z 00000001800bedf4     hb-ot-cff1-table.obj
 0002:00033df4       $unwind$?interpret@?$cs_interpreter_t@Ucff1_cs_interp_env_t@CFF@@Ucff1_cs_opset_path_t@@Ucff1_path_param_t@@@CFF@@QEAA_NAEAUcff1_path_param_t@@@Z 00000001800bedf4     hb-ot-cff1-table.obj
 0002:00033e0c       $unwind$?hlineto@?$path_procs_t@Ucff1_path_procs_path_t@@Ucff1_cs_interp_env_t@CFF@@Ucff1_path_param_t@@@CFF@@SAXAEAUcff1_cs_interp_env_t@2@AEAUcff1_path_param_t@@@Z 00000001800bee0c     hb-ot-cff1-table.obj
 0002:00033e0c       $unwind$?vlineto@?$path_procs_t@Ucff1_path_procs_path_t@@Ucff1_cs_interp_env_t@CFF@@Ucff1_path_param_t@@@CFF@@SAXAEAUcff1_cs_interp_env_t@2@AEAUcff1_path_param_t@@@Z 00000001800bee0c     hb-ot-cff1-table.obj
 0002:00033e2c       $chain$0$?hlineto@?$path_procs_t@Ucff1_path_procs_path_t@@Ucff1_cs_interp_env_t@CFF@@Ucff1_path_param_t@@@CFF@@SAXAEAUcff1_cs_interp_env_t@2@AEAUcff1_path_param_t@@@Z 00000001800bee2c     hb-ot-cff1-table.obj
 0002:00033e40       $chain$1$?hlineto@?$path_procs_t@Ucff1_path_procs_path_t@@Ucff1_cs_interp_env_t@CFF@@Ucff1_path_param_t@@@CFF@@SAXAEAUcff1_cs_interp_env_t@2@AEAUcff1_path_param_t@@@Z 00000001800bee40     hb-ot-cff1-table.obj
 0002:00033e50       $chain$0$?vlineto@?$path_procs_t@Ucff1_path_procs_path_t@@Ucff1_cs_interp_env_t@CFF@@Ucff1_path_param_t@@@CFF@@SAXAEAUcff1_cs_interp_env_t@2@AEAUcff1_path_param_t@@@Z 00000001800bee50     hb-ot-cff1-table.obj
 0002:00033e64       $chain$1$?vlineto@?$path_procs_t@Ucff1_path_procs_path_t@@Ucff1_cs_interp_env_t@CFF@@Ucff1_path_param_t@@@CFF@@SAXAEAUcff1_cs_interp_env_t@2@AEAUcff1_path_param_t@@@Z 00000001800bee64     hb-ot-cff1-table.obj
 0002:00033e74       $unwind$?rrcurveto@?$path_procs_t@Ucff1_path_procs_path_t@@Ucff1_cs_interp_env_t@CFF@@Ucff1_path_param_t@@@CFF@@SAXAEAUcff1_cs_interp_env_t@2@AEAUcff1_path_param_t@@@Z 00000001800bee74     hb-ot-cff1-table.obj
 0002:00033e84       $chain$7$?rrcurveto@?$path_procs_t@Ucff1_path_procs_path_t@@Ucff1_cs_interp_env_t@CFF@@Ucff1_path_param_t@@@CFF@@SAXAEAUcff1_cs_interp_env_t@2@AEAUcff1_path_param_t@@@Z 00000001800bee84     hb-ot-cff1-table.obj
 0002:00033eb4       $chain$8$?rrcurveto@?$path_procs_t@Ucff1_path_procs_path_t@@Ucff1_cs_interp_env_t@CFF@@Ucff1_path_param_t@@@CFF@@SAXAEAUcff1_cs_interp_env_t@2@AEAUcff1_path_param_t@@@Z 00000001800beeb4     hb-ot-cff1-table.obj
 0002:00033ec4       $unwind$?rcurveline@?$path_procs_t@Ucff1_path_procs_path_t@@Ucff1_cs_interp_env_t@CFF@@Ucff1_path_param_t@@@CFF@@SAXAEAUcff1_cs_interp_env_t@2@AEAUcff1_path_param_t@@@Z 00000001800beec4     hb-ot-cff1-table.obj
 0002:00033ed0       $chain$1$?rcurveline@?$path_procs_t@Ucff1_path_procs_path_t@@Ucff1_cs_interp_env_t@CFF@@Ucff1_path_param_t@@@CFF@@SAXAEAUcff1_cs_interp_env_t@2@AEAUcff1_path_param_t@@@Z 00000001800beed0     hb-ot-cff1-table.obj
 0002:00033ee8       $chain$4$?rcurveline@?$path_procs_t@Ucff1_path_procs_path_t@@Ucff1_cs_interp_env_t@CFF@@Ucff1_path_param_t@@@CFF@@SAXAEAUcff1_cs_interp_env_t@2@AEAUcff1_path_param_t@@@Z 00000001800beee8     hb-ot-cff1-table.obj
 0002:00033f04       $chain$9$?rcurveline@?$path_procs_t@Ucff1_path_procs_path_t@@Ucff1_cs_interp_env_t@CFF@@Ucff1_path_param_t@@@CFF@@SAXAEAUcff1_cs_interp_env_t@2@AEAUcff1_path_param_t@@@Z 00000001800bef04     hb-ot-cff1-table.obj
 0002:00033f28       $chain$10$?rcurveline@?$path_procs_t@Ucff1_path_procs_path_t@@Ucff1_cs_interp_env_t@CFF@@Ucff1_path_param_t@@@CFF@@SAXAEAUcff1_cs_interp_env_t@2@AEAUcff1_path_param_t@@@Z 00000001800bef28     hb-ot-cff1-table.obj
 0002:00033f38       $chain$11$?rcurveline@?$path_procs_t@Ucff1_path_procs_path_t@@Ucff1_cs_interp_env_t@CFF@@Ucff1_path_param_t@@@CFF@@SAXAEAUcff1_cs_interp_env_t@2@AEAUcff1_path_param_t@@@Z 00000001800bef38     hb-ot-cff1-table.obj
 0002:00033f50       $chain$12$?rcurveline@?$path_procs_t@Ucff1_path_procs_path_t@@Ucff1_cs_interp_env_t@CFF@@Ucff1_path_param_t@@@CFF@@SAXAEAUcff1_cs_interp_env_t@2@AEAUcff1_path_param_t@@@Z 00000001800bef50     hb-ot-cff1-table.obj
 0002:00033f68       $chain$13$?rcurveline@?$path_procs_t@Ucff1_path_procs_path_t@@Ucff1_cs_interp_env_t@CFF@@Ucff1_path_param_t@@@CFF@@SAXAEAUcff1_cs_interp_env_t@2@AEAUcff1_path_param_t@@@Z 00000001800bef68     hb-ot-cff1-table.obj
 0002:00033f78       $unwind$?rlinecurve@?$path_procs_t@Ucff1_path_procs_path_t@@Ucff1_cs_interp_env_t@CFF@@Ucff1_path_param_t@@@CFF@@SAXAEAUcff1_cs_interp_env_t@2@AEAUcff1_path_param_t@@@Z 00000001800bef78     hb-ot-cff1-table.obj
 0002:00033f84       $chain$1$?rlinecurve@?$path_procs_t@Ucff1_path_procs_path_t@@Ucff1_cs_interp_env_t@CFF@@Ucff1_path_param_t@@@CFF@@SAXAEAUcff1_cs_interp_env_t@2@AEAUcff1_path_param_t@@@Z 00000001800bef84     hb-ot-cff1-table.obj
 0002:00033f9c       $chain$2$?rlinecurve@?$path_procs_t@Ucff1_path_procs_path_t@@Ucff1_cs_interp_env_t@CFF@@Ucff1_path_param_t@@@CFF@@SAXAEAUcff1_cs_interp_env_t@2@AEAUcff1_path_param_t@@@Z 00000001800bef9c     hb-ot-cff1-table.obj
 0002:00033fb0       $chain$5$?rlinecurve@?$path_procs_t@Ucff1_path_procs_path_t@@Ucff1_cs_interp_env_t@CFF@@Ucff1_path_param_t@@@CFF@@SAXAEAUcff1_cs_interp_env_t@2@AEAUcff1_path_param_t@@@Z 00000001800befb0     hb-ot-cff1-table.obj
 0002:00033fcc       $chain$6$?rlinecurve@?$path_procs_t@Ucff1_path_procs_path_t@@Ucff1_cs_interp_env_t@CFF@@Ucff1_path_param_t@@@CFF@@SAXAEAUcff1_cs_interp_env_t@2@AEAUcff1_path_param_t@@@Z 00000001800befcc     hb-ot-cff1-table.obj
 0002:00033fdc       $chain$7$?rlinecurve@?$path_procs_t@Ucff1_path_procs_path_t@@Ucff1_cs_interp_env_t@CFF@@Ucff1_path_param_t@@@CFF@@SAXAEAUcff1_cs_interp_env_t@2@AEAUcff1_path_param_t@@@Z 00000001800befdc     hb-ot-cff1-table.obj
 0002:00033fec       $chain$8$?rlinecurve@?$path_procs_t@Ucff1_path_procs_path_t@@Ucff1_cs_interp_env_t@CFF@@Ucff1_path_param_t@@@CFF@@SAXAEAUcff1_cs_interp_env_t@2@AEAUcff1_path_param_t@@@Z 00000001800befec     hb-ot-cff1-table.obj
 0002:00033ffc       $unwind$?vvcurveto@?$path_procs_t@Ucff1_path_procs_path_t@@Ucff1_cs_interp_env_t@CFF@@Ucff1_path_param_t@@@CFF@@SAXAEAUcff1_cs_interp_env_t@2@AEAUcff1_path_param_t@@@Z 00000001800beffc     hb-ot-cff1-table.obj
 0002:00034018       $chain$3$?vvcurveto@?$path_procs_t@Ucff1_path_procs_path_t@@Ucff1_cs_interp_env_t@CFF@@Ucff1_path_param_t@@@CFF@@SAXAEAUcff1_cs_interp_env_t@2@AEAUcff1_path_param_t@@@Z 00000001800bf018     hb-ot-cff1-table.obj
 0002:00034038       $chain$4$?vvcurveto@?$path_procs_t@Ucff1_path_procs_path_t@@Ucff1_cs_interp_env_t@CFF@@Ucff1_path_param_t@@@CFF@@SAXAEAUcff1_cs_interp_env_t@2@AEAUcff1_path_param_t@@@Z 00000001800bf038     hb-ot-cff1-table.obj
 0002:00034048       $unwind$?hhcurveto@?$path_procs_t@Ucff1_path_procs_path_t@@Ucff1_cs_interp_env_t@CFF@@Ucff1_path_param_t@@@CFF@@SAXAEAUcff1_cs_interp_env_t@2@AEAUcff1_path_param_t@@@Z 00000001800bf048     hb-ot-cff1-table.obj
 0002:00034064       $chain$2$?hhcurveto@?$path_procs_t@Ucff1_path_procs_path_t@@Ucff1_cs_interp_env_t@CFF@@Ucff1_path_param_t@@@CFF@@SAXAEAUcff1_cs_interp_env_t@2@AEAUcff1_path_param_t@@@Z 00000001800bf064     hb-ot-cff1-table.obj
 0002:00034080       $chain$3$?hhcurveto@?$path_procs_t@Ucff1_path_procs_path_t@@Ucff1_cs_interp_env_t@CFF@@Ucff1_path_param_t@@@CFF@@SAXAEAUcff1_cs_interp_env_t@2@AEAUcff1_path_param_t@@@Z 00000001800bf080     hb-ot-cff1-table.obj
 0002:00034090       $unwind$?vhcurveto@?$path_procs_t@Ucff1_path_procs_path_t@@Ucff1_cs_interp_env_t@CFF@@Ucff1_path_param_t@@@CFF@@SAXAEAUcff1_cs_interp_env_t@2@AEAUcff1_path_param_t@@@Z 00000001800bf090     hb-ot-cff1-table.obj
 0002:000340c4       $unwind$?hvcurveto@?$path_procs_t@Ucff1_path_procs_path_t@@Ucff1_cs_interp_env_t@CFF@@Ucff1_path_param_t@@@CFF@@SAXAEAUcff1_cs_interp_env_t@2@AEAUcff1_path_param_t@@@Z 00000001800bf0c4     hb-ot-cff1-table.obj
 0002:000340f8       $chain$0$?hvcurveto@?$path_procs_t@Ucff1_path_procs_path_t@@Ucff1_cs_interp_env_t@CFF@@Ucff1_path_param_t@@@CFF@@SAXAEAUcff1_cs_interp_env_t@2@AEAUcff1_path_param_t@@@Z 00000001800bf0f8     hb-ot-cff1-table.obj
 0002:0003410c       $chain$1$?hvcurveto@?$path_procs_t@Ucff1_path_procs_path_t@@Ucff1_cs_interp_env_t@CFF@@Ucff1_path_param_t@@@CFF@@SAXAEAUcff1_cs_interp_env_t@2@AEAUcff1_path_param_t@@@Z 00000001800bf10c     hb-ot-cff1-table.obj
 0002:0003411c       $unwind$?moveto@cff1_path_procs_path_t@@SAXAEAUcff1_cs_interp_env_t@CFF@@AEAUcff1_path_param_t@@AEBUpoint_t@3@@Z 00000001800bf11c     hb-ot-cff1-table.obj
 0002:00034134       $unwind$?curve@cff1_path_procs_path_t@@SAXAEAUcff1_cs_interp_env_t@CFF@@AEAUcff1_path_param_t@@AEBUpoint_t@3@22@Z 00000001800bf134     hb-ot-cff1-table.obj
 0002:00034150       $unwind$?_get_path@@YA_NPEBUaccelerator_t@cff1@OT@@PEAUhb_font_t@@IAEAUhb_draw_session_t@@_NPEAUpoint_t@CFF@@@Z 00000001800bf150     hb-ot-cff1-table.obj
 0002:0003416c       $chain$0$?_get_path@@YA_NPEBUaccelerator_t@cff1@OT@@PEAUhb_font_t@@IAEAUhb_draw_session_t@@_NPEAUpoint_t@CFF@@@Z 00000001800bf16c     hb-ot-cff1-table.obj
 0002:00034180       $chain$1$?_get_path@@YA_NPEBUaccelerator_t@cff1@OT@@PEAUhb_font_t@@IAEAUhb_draw_session_t@@_NPEAUpoint_t@CFF@@@Z 00000001800bf180     hb-ot-cff1-table.obj
 0002:00034190       $unwind$?process_op@?$cs_opset_t@Unumber_t@CFF@@Ucff1_cs_opset_path_t@@Ucff1_cs_interp_env_t@2@Ucff1_path_param_t@@Ucff1_path_procs_path_t@@@CFF@@SAXIAEAUcff1_cs_interp_env_t@2@AEAUcff1_path_param_t@@@Z 00000001800bf190     hb-ot-cff1-table.obj
 0002:000341a4       $chain$1$?process_op@?$cs_opset_t@Unumber_t@CFF@@Ucff1_cs_opset_path_t@@Ucff1_cs_interp_env_t@2@Ucff1_path_param_t@@Ucff1_path_procs_path_t@@@CFF@@SAXIAEAUcff1_cs_interp_env_t@2@AEAUcff1_path_param_t@@@Z 00000001800bf1a4     hb-ot-cff1-table.obj
 0002:000341bc       $chain$2$?process_op@?$cs_opset_t@Unumber_t@CFF@@Ucff1_cs_opset_path_t@@Ucff1_cs_interp_env_t@2@Ucff1_path_param_t@@Ucff1_path_procs_path_t@@@CFF@@SAXIAEAUcff1_cs_interp_env_t@2@AEAUcff1_path_param_t@@@Z 00000001800bf1bc     hb-ot-cff1-table.obj
 0002:000341cc       $unwind$?process_seac@cff1_cs_opset_path_t@@SAXAEAUcff1_cs_interp_env_t@CFF@@AEAUcff1_path_param_t@@@Z 00000001800bf1cc     hb-ot-cff1-table.obj
 0002:000341dc       $chain$1$?process_seac@cff1_cs_opset_path_t@@SAXAEAUcff1_cs_interp_env_t@CFF@@AEAUcff1_path_param_t@@@Z 00000001800bf1dc     hb-ot-cff1-table.obj
 0002:000341f4       $chain$3$?process_seac@cff1_cs_opset_path_t@@SAXAEAUcff1_cs_interp_env_t@CFF@@AEAUcff1_path_param_t@@@Z 00000001800bf1f4     hb-ot-cff1-table.obj
 0002:0003420c       $chain$4$?process_seac@cff1_cs_opset_path_t@@SAXAEAUcff1_cs_interp_env_t@CFF@@AEAUcff1_path_param_t@@@Z 00000001800bf20c     hb-ot-cff1-table.obj
 0002:00034220       $chain$5$?process_seac@cff1_cs_opset_path_t@@SAXAEAUcff1_cs_interp_env_t@CFF@@AEAUcff1_path_param_t@@@Z 00000001800bf220     hb-ot-cff1-table.obj
 0002:00034234       $unwind$?get_region_scalars@VarData@OT@@QEBAXPEBHIAEBUVarRegionList@2@PEAMI@Z 00000001800bf234     hb-ot-cff2-table.obj
 0002:0003423c       $chain$1$?get_region_scalars@VarData@OT@@QEBAXPEBHIAEBUVarRegionList@2@PEAMI@Z 00000001800bf23c     hb-ot-cff2-table.obj
 0002:00034254       $chain$6$?get_region_scalars@VarData@OT@@QEBAXPEBHIAEBUVarRegionList@2@PEAMI@Z 00000001800bf254     hb-ot-cff2-table.obj
 0002:00034278       $chain$7$?get_region_scalars@VarData@OT@@QEBAXPEBHIAEBUVarRegionList@2@PEAMI@Z 00000001800bf278     hb-ot-cff2-table.obj
 0002:00034288       $chain$8$?get_region_scalars@VarData@OT@@QEBAXPEBHIAEBUVarRegionList@2@PEAMI@Z 00000001800bf288     hb-ot-cff2-table.obj
 0002:00034298       $unwind$?get_fd@CFF2FDSelect@CFF@@QEBAII@Z 00000001800bf298     hb-ot-cff2-table.obj
 0002:000342a0       $chain$3$?get_fd@CFF2FDSelect@CFF@@QEBAII@Z 00000001800bf2a0     hb-ot-cff2-table.obj
 0002:000342c0       $chain$5$?get_fd@CFF2FDSelect@CFF@@QEBAII@Z 00000001800bf2c0     hb-ot-cff2-table.obj
 0002:000342e0       $chain$6$?get_fd@CFF2FDSelect@CFF@@QEBAII@Z 00000001800bf2e0     hb-ot-cff2-table.obj
 0002:000342f4       $chain$8$?get_fd@CFF2FDSelect@CFF@@QEBAII@Z 00000001800bf2f4     hb-ot-cff2-table.obj
 0002:00034308       $chain$10$?get_fd@CFF2FDSelect@CFF@@QEBAII@Z 00000001800bf308     hb-ot-cff2-table.obj
 0002:00034318       $chain$0$??A?$CFFIndex@U?$IntType@I$03@OT@@@CFF@@QEBA?AU?$hb_array_t@$$CBE@@I@Z 00000001800bf318     hb-ot-cff2-table.obj
 0002:0003432c       $chain$1$??A?$CFFIndex@U?$IntType@I$03@OT@@@CFF@@QEBA?AU?$hb_array_t@$$CBE@@I@Z 00000001800bf32c     hb-ot-cff2-table.obj
 0002:0003433c       $unwind$?get_extents@accelerator_t@cff2@OT@@QEBA_NPEAUhb_font_t@@IPEAUhb_glyph_extents_t@@@Z 00000001800bf33c     hb-ot-cff2-table.obj
 0002:00034358       $chain$0$?get_extents@accelerator_t@cff2@OT@@QEBA_NPEAUhb_font_t@@IPEAUhb_glyph_extents_t@@@Z 00000001800bf358     hb-ot-cff2-table.obj
 0002:0003436c       $chain$2$?get_extents@accelerator_t@cff2@OT@@QEBA_NPEAUhb_font_t@@IPEAUhb_glyph_extents_t@@@Z 00000001800bf36c     hb-ot-cff2-table.obj
 0002:00034384       $chain$5$?get_extents@accelerator_t@cff2@OT@@QEBA_NPEAUhb_font_t@@IPEAUhb_glyph_extents_t@@@Z 00000001800bf384     hb-ot-cff2-table.obj
 0002:000343a0       $chain$6$?get_extents@accelerator_t@cff2@OT@@QEBA_NPEAUhb_font_t@@IPEAUhb_glyph_extents_t@@@Z 00000001800bf3a0     hb-ot-cff2-table.obj
 0002:000343b0       $chain$7$?get_extents@accelerator_t@cff2@OT@@QEBA_NPEAUhb_font_t@@IPEAUhb_glyph_extents_t@@@Z 00000001800bf3b0     hb-ot-cff2-table.obj
 0002:000343c0       $chain$8$?get_extents@accelerator_t@cff2@OT@@QEBA_NPEAUhb_font_t@@IPEAUhb_glyph_extents_t@@@Z 00000001800bf3c0     hb-ot-cff2-table.obj
 0002:000343d0       $unwind$?get_path@accelerator_t@cff2@OT@@QEBA_NPEAUhb_font_t@@IAEAUhb_draw_session_t@@@Z 00000001800bf3d0     hb-ot-cff2-table.obj
 0002:000343ec       $chain$0$?get_path@accelerator_t@cff2@OT@@QEBA_NPEAUhb_font_t@@IAEAUhb_draw_session_t@@@Z 00000001800bf3ec     hb-ot-cff2-table.obj
 0002:00034400       $chain$2$?get_path@accelerator_t@cff2@OT@@QEBA_NPEAUhb_font_t@@IAEAUhb_draw_session_t@@@Z 00000001800bf400     hb-ot-cff2-table.obj
 0002:00034418       $chain$3$?get_path@accelerator_t@cff2@OT@@QEBA_NPEAUhb_font_t@@IAEAUhb_draw_session_t@@@Z 00000001800bf418     hb-ot-cff2-table.obj
 0002:00034428       $chain$4$?get_path@accelerator_t@cff2@OT@@QEBA_NPEAUhb_font_t@@IAEAUhb_draw_session_t@@@Z 00000001800bf428     hb-ot-cff2-table.obj
 0002:00034438       $unwind$?hlineto@?$path_procs_t@Ucff2_path_procs_extents_t@@U?$cff2_cs_interp_env_t@Unumber_t@CFF@@@CFF@@Ucff2_extents_param_t@@@CFF@@SAXAEAU?$cff2_cs_interp_env_t@Unumber_t@CFF@@@2@AEAUcff2_extents_param_t@@@Z 00000001800bf438     hb-ot-cff2-table.obj
 0002:00034438       $unwind$?vlineto@?$path_procs_t@Ucff2_path_procs_extents_t@@U?$cff2_cs_interp_env_t@Unumber_t@CFF@@@CFF@@Ucff2_extents_param_t@@@CFF@@SAXAEAU?$cff2_cs_interp_env_t@Unumber_t@CFF@@@2@AEAUcff2_extents_param_t@@@Z 00000001800bf438     hb-ot-cff2-table.obj
 0002:00034444       $chain$0$?hlineto@?$path_procs_t@Ucff2_path_procs_extents_t@@U?$cff2_cs_interp_env_t@Unumber_t@CFF@@@CFF@@Ucff2_extents_param_t@@@CFF@@SAXAEAU?$cff2_cs_interp_env_t@Unumber_t@CFF@@@2@AEAUcff2_extents_param_t@@@Z 00000001800bf444     hb-ot-cff2-table.obj
 0002:00034458       $chain$1$?hlineto@?$path_procs_t@Ucff2_path_procs_extents_t@@U?$cff2_cs_interp_env_t@Unumber_t@CFF@@@CFF@@Ucff2_extents_param_t@@@CFF@@SAXAEAU?$cff2_cs_interp_env_t@Unumber_t@CFF@@@2@AEAUcff2_extents_param_t@@@Z 00000001800bf458     hb-ot-cff2-table.obj
 0002:0003446c       $chain$2$?hlineto@?$path_procs_t@Ucff2_path_procs_extents_t@@U?$cff2_cs_interp_env_t@Unumber_t@CFF@@@CFF@@Ucff2_extents_param_t@@@CFF@@SAXAEAU?$cff2_cs_interp_env_t@Unumber_t@CFF@@@2@AEAUcff2_extents_param_t@@@Z 00000001800bf46c     hb-ot-cff2-table.obj
 0002:0003447c       $chain$3$?hlineto@?$path_procs_t@Ucff2_path_procs_extents_t@@U?$cff2_cs_interp_env_t@Unumber_t@CFF@@@CFF@@Ucff2_extents_param_t@@@CFF@@SAXAEAU?$cff2_cs_interp_env_t@Unumber_t@CFF@@@2@AEAUcff2_extents_param_t@@@Z 00000001800bf47c     hb-ot-cff2-table.obj
 0002:0003448c       $chain$0$?vlineto@?$path_procs_t@Ucff2_path_procs_extents_t@@U?$cff2_cs_interp_env_t@Unumber_t@CFF@@@CFF@@Ucff2_extents_param_t@@@CFF@@SAXAEAU?$cff2_cs_interp_env_t@Unumber_t@CFF@@@2@AEAUcff2_extents_param_t@@@Z 00000001800bf48c     hb-ot-cff2-table.obj
 0002:000344a0       $chain$1$?vlineto@?$path_procs_t@Ucff2_path_procs_extents_t@@U?$cff2_cs_interp_env_t@Unumber_t@CFF@@@CFF@@Ucff2_extents_param_t@@@CFF@@SAXAEAU?$cff2_cs_interp_env_t@Unumber_t@CFF@@@2@AEAUcff2_extents_param_t@@@Z 00000001800bf4a0     hb-ot-cff2-table.obj
 0002:000344b4       $chain$2$?vlineto@?$path_procs_t@Ucff2_path_procs_extents_t@@U?$cff2_cs_interp_env_t@Unumber_t@CFF@@@CFF@@Ucff2_extents_param_t@@@CFF@@SAXAEAU?$cff2_cs_interp_env_t@Unumber_t@CFF@@@2@AEAUcff2_extents_param_t@@@Z 00000001800bf4b4     hb-ot-cff2-table.obj
 0002:000344c4       $chain$3$?vlineto@?$path_procs_t@Ucff2_path_procs_extents_t@@U?$cff2_cs_interp_env_t@Unumber_t@CFF@@@CFF@@Ucff2_extents_param_t@@@CFF@@SAXAEAU?$cff2_cs_interp_env_t@Unumber_t@CFF@@@2@AEAUcff2_extents_param_t@@@Z 00000001800bf4c4     hb-ot-cff2-table.obj
 0002:000344d4       $chain$3$?rrcurveto@?$path_procs_t@Ucff2_path_procs_extents_t@@U?$cff2_cs_interp_env_t@Unumber_t@CFF@@@CFF@@Ucff2_extents_param_t@@@CFF@@SAXAEAU?$cff2_cs_interp_env_t@Unumber_t@CFF@@@2@AEAUcff2_extents_param_t@@@Z 00000001800bf4d4     hb-ot-cff2-table.obj
 0002:000344f4       $chain$4$?rrcurveto@?$path_procs_t@Ucff2_path_procs_extents_t@@U?$cff2_cs_interp_env_t@Unumber_t@CFF@@@CFF@@Ucff2_extents_param_t@@@CFF@@SAXAEAU?$cff2_cs_interp_env_t@Unumber_t@CFF@@@2@AEAUcff2_extents_param_t@@@Z 00000001800bf4f4     hb-ot-cff2-table.obj
 0002:00034504       $chain$0$?rcurveline@?$path_procs_t@Ucff2_path_procs_extents_t@@U?$cff2_cs_interp_env_t@Unumber_t@CFF@@@CFF@@Ucff2_extents_param_t@@@CFF@@SAXAEAU?$cff2_cs_interp_env_t@Unumber_t@CFF@@@2@AEAUcff2_extents_param_t@@@Z 00000001800bf504     hb-ot-cff2-table.obj
 0002:00034518       $chain$4$?rcurveline@?$path_procs_t@Ucff2_path_procs_extents_t@@U?$cff2_cs_interp_env_t@Unumber_t@CFF@@@CFF@@Ucff2_extents_param_t@@@CFF@@SAXAEAU?$cff2_cs_interp_env_t@Unumber_t@CFF@@@2@AEAUcff2_extents_param_t@@@Z 00000001800bf518     hb-ot-cff2-table.obj
 0002:00034538       $chain$5$?rcurveline@?$path_procs_t@Ucff2_path_procs_extents_t@@U?$cff2_cs_interp_env_t@Unumber_t@CFF@@@CFF@@Ucff2_extents_param_t@@@CFF@@SAXAEAU?$cff2_cs_interp_env_t@Unumber_t@CFF@@@2@AEAUcff2_extents_param_t@@@Z 00000001800bf538     hb-ot-cff2-table.obj
 0002:00034548       $chain$6$?rcurveline@?$path_procs_t@Ucff2_path_procs_extents_t@@U?$cff2_cs_interp_env_t@Unumber_t@CFF@@@CFF@@Ucff2_extents_param_t@@@CFF@@SAXAEAU?$cff2_cs_interp_env_t@Unumber_t@CFF@@@2@AEAUcff2_extents_param_t@@@Z 00000001800bf548     hb-ot-cff2-table.obj
 0002:00034558       $chain$4$?rlinecurve@?$path_procs_t@Ucff2_path_procs_extents_t@@U?$cff2_cs_interp_env_t@Unumber_t@CFF@@@CFF@@Ucff2_extents_param_t@@@CFF@@SAXAEAU?$cff2_cs_interp_env_t@Unumber_t@CFF@@@2@AEAUcff2_extents_param_t@@@Z 00000001800bf558     hb-ot-cff2-table.obj
 0002:0003457c       $chain$5$?rlinecurve@?$path_procs_t@Ucff2_path_procs_extents_t@@U?$cff2_cs_interp_env_t@Unumber_t@CFF@@@CFF@@Ucff2_extents_param_t@@@CFF@@SAXAEAU?$cff2_cs_interp_env_t@Unumber_t@CFF@@@2@AEAUcff2_extents_param_t@@@Z 00000001800bf57c     hb-ot-cff2-table.obj
 0002:0003459c       $chain$6$?rlinecurve@?$path_procs_t@Ucff2_path_procs_extents_t@@U?$cff2_cs_interp_env_t@Unumber_t@CFF@@@CFF@@Ucff2_extents_param_t@@@CFF@@SAXAEAU?$cff2_cs_interp_env_t@Unumber_t@CFF@@@2@AEAUcff2_extents_param_t@@@Z 00000001800bf59c     hb-ot-cff2-table.obj
 0002:000345b8       $chain$7$?rlinecurve@?$path_procs_t@Ucff2_path_procs_extents_t@@U?$cff2_cs_interp_env_t@Unumber_t@CFF@@@CFF@@Ucff2_extents_param_t@@@CFF@@SAXAEAU?$cff2_cs_interp_env_t@Unumber_t@CFF@@@2@AEAUcff2_extents_param_t@@@Z 00000001800bf5b8     hb-ot-cff2-table.obj
 0002:000345d0       $chain$8$?rlinecurve@?$path_procs_t@Ucff2_path_procs_extents_t@@U?$cff2_cs_interp_env_t@Unumber_t@CFF@@@CFF@@Ucff2_extents_param_t@@@CFF@@SAXAEAU?$cff2_cs_interp_env_t@Unumber_t@CFF@@@2@AEAUcff2_extents_param_t@@@Z 00000001800bf5d0     hb-ot-cff2-table.obj
 0002:000345e4       $chain$9$?rlinecurve@?$path_procs_t@Ucff2_path_procs_extents_t@@U?$cff2_cs_interp_env_t@Unumber_t@CFF@@@CFF@@Ucff2_extents_param_t@@@CFF@@SAXAEAU?$cff2_cs_interp_env_t@Unumber_t@CFF@@@2@AEAUcff2_extents_param_t@@@Z 00000001800bf5e4     hb-ot-cff2-table.obj
 0002:000345f4       $chain$2$?vvcurveto@?$path_procs_t@Ucff2_path_procs_extents_t@@U?$cff2_cs_interp_env_t@Unumber_t@CFF@@@CFF@@Ucff2_extents_param_t@@@CFF@@SAXAEAU?$cff2_cs_interp_env_t@Unumber_t@CFF@@@2@AEAUcff2_extents_param_t@@@Z 00000001800bf5f4     hb-ot-cff2-table.obj
 0002:00034610       $chain$3$?vvcurveto@?$path_procs_t@Ucff2_path_procs_extents_t@@U?$cff2_cs_interp_env_t@Unumber_t@CFF@@@CFF@@Ucff2_extents_param_t@@@CFF@@SAXAEAU?$cff2_cs_interp_env_t@Unumber_t@CFF@@@2@AEAUcff2_extents_param_t@@@Z 00000001800bf610     hb-ot-cff2-table.obj
 0002:00034620       $chain$2$?hhcurveto@?$path_procs_t@Ucff2_path_procs_extents_t@@U?$cff2_cs_interp_env_t@Unumber_t@CFF@@@CFF@@Ucff2_extents_param_t@@@CFF@@SAXAEAU?$cff2_cs_interp_env_t@Unumber_t@CFF@@@2@AEAUcff2_extents_param_t@@@Z 00000001800bf620     hb-ot-cff2-table.obj
 0002:0003463c       $chain$3$?hhcurveto@?$path_procs_t@Ucff2_path_procs_extents_t@@U?$cff2_cs_interp_env_t@Unumber_t@CFF@@@CFF@@Ucff2_extents_param_t@@@CFF@@SAXAEAU?$cff2_cs_interp_env_t@Unumber_t@CFF@@@2@AEAUcff2_extents_param_t@@@Z 00000001800bf63c     hb-ot-cff2-table.obj
 0002:0003464c       $unwind$?hvcurveto@?$path_procs_t@Ucff2_path_procs_extents_t@@U?$cff2_cs_interp_env_t@Unumber_t@CFF@@@CFF@@Ucff2_extents_param_t@@@CFF@@SAXAEAU?$cff2_cs_interp_env_t@Unumber_t@CFF@@@2@AEAUcff2_extents_param_t@@@Z 00000001800bf64c     hb-ot-cff2-table.obj
 0002:0003464c       $unwind$?vhcurveto@?$path_procs_t@Ucff2_path_procs_extents_t@@U?$cff2_cs_interp_env_t@Unumber_t@CFF@@@CFF@@Ucff2_extents_param_t@@@CFF@@SAXAEAU?$cff2_cs_interp_env_t@Unumber_t@CFF@@@2@AEAUcff2_extents_param_t@@@Z 00000001800bf64c     hb-ot-cff2-table.obj
 0002:00034668       $chain$0$?call_subr@?$cs_interp_env_t@Unumber_t@CFF@@U?$Subrs@U?$IntType@I$03@OT@@@2@@CFF@@QEAAXAEBU?$biased_subrs_t@U?$Subrs@U?$IntType@I$03@OT@@@CFF@@@2@W4cs_type_t@2@@Z 00000001800bf668     hb-ot-cff2-table.obj
 0002:0003467c       $chain$1$?call_subr@?$cs_interp_env_t@Unumber_t@CFF@@U?$Subrs@U?$IntType@I$03@OT@@@2@@CFF@@QEAAXAEBU?$biased_subrs_t@U?$Subrs@U?$IntType@I$03@OT@@@CFF@@@2@W4cs_type_t@2@@Z 00000001800bf67c     hb-ot-cff2-table.obj
 0002:0003468c       $chain$4$?process_blend@?$cff2_cs_interp_env_t@Unumber_t@CFF@@@CFF@@QEAAXXZ 00000001800bf68c     hb-ot-cff2-table.obj
 0002:000346b0       $chain$6$?process_blend@?$cff2_cs_interp_env_t@Unumber_t@CFF@@@CFF@@QEAAXXZ 00000001800bf6b0     hb-ot-cff2-table.obj
 0002:000346c8       $chain$7$?process_blend@?$cff2_cs_interp_env_t@Unumber_t@CFF@@@CFF@@QEAAXXZ 00000001800bf6c8     hb-ot-cff2-table.obj
 0002:000346d8       $chain$8$?process_blend@?$cff2_cs_interp_env_t@Unumber_t@CFF@@@CFF@@QEAAXXZ 00000001800bf6d8     hb-ot-cff2-table.obj
 0002:000346e8       $chain$9$?process_blend@?$cff2_cs_interp_env_t@Unumber_t@CFF@@@CFF@@QEAAXXZ 00000001800bf6e8     hb-ot-cff2-table.obj
 0002:00034714       $chain$1$?blend_deltas@?$cff2_cs_interp_env_t@Unumber_t@CFF@@@CFF@@QEBANU?$hb_array_t@$$CBUnumber_t@CFF@@@@@Z 00000001800bf714     hb-ot-cff2-table.obj
 0002:0003472c       $chain$3$?blend_deltas@?$cff2_cs_interp_env_t@Unumber_t@CFF@@@CFF@@QEBANU?$hb_array_t@$$CBUnumber_t@CFF@@@@@Z 00000001800bf72c     hb-ot-cff2-table.obj
 0002:0003472c       $chain$5$?blend_deltas@?$cff2_cs_interp_env_t@Unumber_t@CFF@@@CFF@@QEBANU?$hb_array_t@$$CBUnumber_t@CFF@@@@@Z 00000001800bf72c     hb-ot-cff2-table.obj
 0002:00034744       $chain$6$?blend_deltas@?$cff2_cs_interp_env_t@Unumber_t@CFF@@@CFF@@QEBANU?$hb_array_t@$$CBUnumber_t@CFF@@@@@Z 00000001800bf744     hb-ot-cff2-table.obj
 0002:00034754       $unwind$??$?0$$CBUaccelerator_t@cff2@OT@@@?$cff2_cs_interp_env_t@Unumber_t@CFF@@@CFF@@QEAA@AEBU?$hb_array_t@$$CBE@@AEBUaccelerator_t@cff2@OT@@IPEBHI@Z 00000001800bf754     hb-ot-cff2-table.obj
 0002:00034770       $unwind$?hlineto@?$path_procs_t@Ucff2_path_procs_path_t@@U?$cff2_cs_interp_env_t@Unumber_t@CFF@@@CFF@@Ucff2_path_param_t@@@CFF@@SAXAEAU?$cff2_cs_interp_env_t@Unumber_t@CFF@@@2@AEAUcff2_path_param_t@@@Z 00000001800bf770     hb-ot-cff2-table.obj
 0002:00034770       $unwind$?vlineto@?$path_procs_t@Ucff2_path_procs_path_t@@U?$cff2_cs_interp_env_t@Unumber_t@CFF@@@CFF@@Ucff2_path_param_t@@@CFF@@SAXAEAU?$cff2_cs_interp_env_t@Unumber_t@CFF@@@2@AEAUcff2_path_param_t@@@Z 00000001800bf770     hb-ot-cff2-table.obj
 0002:0003478c       $chain$0$?hlineto@?$path_procs_t@Ucff2_path_procs_path_t@@U?$cff2_cs_interp_env_t@Unumber_t@CFF@@@CFF@@Ucff2_path_param_t@@@CFF@@SAXAEAU?$cff2_cs_interp_env_t@Unumber_t@CFF@@@2@AEAUcff2_path_param_t@@@Z 00000001800bf78c     hb-ot-cff2-table.obj
 0002:000347a0       $chain$2$?hlineto@?$path_procs_t@Ucff2_path_procs_path_t@@U?$cff2_cs_interp_env_t@Unumber_t@CFF@@@CFF@@Ucff2_path_param_t@@@CFF@@SAXAEAU?$cff2_cs_interp_env_t@Unumber_t@CFF@@@2@AEAUcff2_path_param_t@@@Z 00000001800bf7a0     hb-ot-cff2-table.obj
 0002:000347b8       $chain$3$?hlineto@?$path_procs_t@Ucff2_path_procs_path_t@@U?$cff2_cs_interp_env_t@Unumber_t@CFF@@@CFF@@Ucff2_path_param_t@@@CFF@@SAXAEAU?$cff2_cs_interp_env_t@Unumber_t@CFF@@@2@AEAUcff2_path_param_t@@@Z 00000001800bf7b8     hb-ot-cff2-table.obj
 0002:000347c8       $chain$4$?hlineto@?$path_procs_t@Ucff2_path_procs_path_t@@U?$cff2_cs_interp_env_t@Unumber_t@CFF@@@CFF@@Ucff2_path_param_t@@@CFF@@SAXAEAU?$cff2_cs_interp_env_t@Unumber_t@CFF@@@2@AEAUcff2_path_param_t@@@Z 00000001800bf7c8     hb-ot-cff2-table.obj
 0002:000347d8       $chain$0$?vlineto@?$path_procs_t@Ucff2_path_procs_path_t@@U?$cff2_cs_interp_env_t@Unumber_t@CFF@@@CFF@@Ucff2_path_param_t@@@CFF@@SAXAEAU?$cff2_cs_interp_env_t@Unumber_t@CFF@@@2@AEAUcff2_path_param_t@@@Z 00000001800bf7d8     hb-ot-cff2-table.obj
 0002:000347ec       $chain$2$?vlineto@?$path_procs_t@Ucff2_path_procs_path_t@@U?$cff2_cs_interp_env_t@Unumber_t@CFF@@@CFF@@Ucff2_path_param_t@@@CFF@@SAXAEAU?$cff2_cs_interp_env_t@Unumber_t@CFF@@@2@AEAUcff2_path_param_t@@@Z 00000001800bf7ec     hb-ot-cff2-table.obj
 0002:00034804       $chain$3$?vlineto@?$path_procs_t@Ucff2_path_procs_path_t@@U?$cff2_cs_interp_env_t@Unumber_t@CFF@@@CFF@@Ucff2_path_param_t@@@CFF@@SAXAEAU?$cff2_cs_interp_env_t@Unumber_t@CFF@@@2@AEAUcff2_path_param_t@@@Z 00000001800bf804     hb-ot-cff2-table.obj
 0002:00034814       $chain$4$?vlineto@?$path_procs_t@Ucff2_path_procs_path_t@@U?$cff2_cs_interp_env_t@Unumber_t@CFF@@@CFF@@Ucff2_path_param_t@@@CFF@@SAXAEAU?$cff2_cs_interp_env_t@Unumber_t@CFF@@@2@AEAUcff2_path_param_t@@@Z 00000001800bf814     hb-ot-cff2-table.obj
 0002:00034824       $unwind$?rrcurveto@?$path_procs_t@Ucff2_path_procs_path_t@@U?$cff2_cs_interp_env_t@Unumber_t@CFF@@@CFF@@Ucff2_path_param_t@@@CFF@@SAXAEAU?$cff2_cs_interp_env_t@Unumber_t@CFF@@@2@AEAUcff2_path_param_t@@@Z 00000001800bf824     hb-ot-cff2-table.obj
 0002:00034834       $chain$6$?rrcurveto@?$path_procs_t@Ucff2_path_procs_path_t@@U?$cff2_cs_interp_env_t@Unumber_t@CFF@@@CFF@@Ucff2_path_param_t@@@CFF@@SAXAEAU?$cff2_cs_interp_env_t@Unumber_t@CFF@@@2@AEAUcff2_path_param_t@@@Z 00000001800bf834     hb-ot-cff2-table.obj
 0002:00034860       $chain$7$?rrcurveto@?$path_procs_t@Ucff2_path_procs_path_t@@U?$cff2_cs_interp_env_t@Unumber_t@CFF@@@CFF@@Ucff2_path_param_t@@@CFF@@SAXAEAU?$cff2_cs_interp_env_t@Unumber_t@CFF@@@2@AEAUcff2_path_param_t@@@Z 00000001800bf860     hb-ot-cff2-table.obj
 0002:00034870       $unwind$?rcurveline@?$path_procs_t@Ucff2_path_procs_path_t@@U?$cff2_cs_interp_env_t@Unumber_t@CFF@@@CFF@@Ucff2_path_param_t@@@CFF@@SAXAEAU?$cff2_cs_interp_env_t@Unumber_t@CFF@@@2@AEAUcff2_path_param_t@@@Z 00000001800bf870     hb-ot-cff2-table.obj
 0002:00034870       $unwind$?rlinecurve@?$path_procs_t@Ucff2_path_procs_path_t@@U?$cff2_cs_interp_env_t@Unumber_t@CFF@@@CFF@@Ucff2_path_param_t@@@CFF@@SAXAEAU?$cff2_cs_interp_env_t@Unumber_t@CFF@@@2@AEAUcff2_path_param_t@@@Z 00000001800bf870     hb-ot-cff2-table.obj
 0002:0003487c       $chain$1$?rcurveline@?$path_procs_t@Ucff2_path_procs_path_t@@U?$cff2_cs_interp_env_t@Unumber_t@CFF@@@CFF@@Ucff2_path_param_t@@@CFF@@SAXAEAU?$cff2_cs_interp_env_t@Unumber_t@CFF@@@2@AEAUcff2_path_param_t@@@Z 00000001800bf87c     hb-ot-cff2-table.obj
 0002:00034894       $chain$4$?rcurveline@?$path_procs_t@Ucff2_path_procs_path_t@@U?$cff2_cs_interp_env_t@Unumber_t@CFF@@@CFF@@Ucff2_path_param_t@@@CFF@@SAXAEAU?$cff2_cs_interp_env_t@Unumber_t@CFF@@@2@AEAUcff2_path_param_t@@@Z 00000001800bf894     hb-ot-cff2-table.obj
 0002:000348b0       $chain$8$?rcurveline@?$path_procs_t@Ucff2_path_procs_path_t@@U?$cff2_cs_interp_env_t@Unumber_t@CFF@@@CFF@@Ucff2_path_param_t@@@CFF@@SAXAEAU?$cff2_cs_interp_env_t@Unumber_t@CFF@@@2@AEAUcff2_path_param_t@@@Z 00000001800bf8b0     hb-ot-cff2-table.obj
 0002:000348d0       $chain$9$?rcurveline@?$path_procs_t@Ucff2_path_procs_path_t@@U?$cff2_cs_interp_env_t@Unumber_t@CFF@@@CFF@@Ucff2_path_param_t@@@CFF@@SAXAEAU?$cff2_cs_interp_env_t@Unumber_t@CFF@@@2@AEAUcff2_path_param_t@@@Z 00000001800bf8d0     hb-ot-cff2-table.obj
 0002:000348e0       $chain$10$?rcurveline@?$path_procs_t@Ucff2_path_procs_path_t@@U?$cff2_cs_interp_env_t@Unumber_t@CFF@@@CFF@@Ucff2_path_param_t@@@CFF@@SAXAEAU?$cff2_cs_interp_env_t@Unumber_t@CFF@@@2@AEAUcff2_path_param_t@@@Z 00000001800bf8e0     hb-ot-cff2-table.obj
 0002:000348f8       $chain$11$?rcurveline@?$path_procs_t@Ucff2_path_procs_path_t@@U?$cff2_cs_interp_env_t@Unumber_t@CFF@@@CFF@@Ucff2_path_param_t@@@CFF@@SAXAEAU?$cff2_cs_interp_env_t@Unumber_t@CFF@@@2@AEAUcff2_path_param_t@@@Z 00000001800bf8f8     hb-ot-cff2-table.obj
 0002:00034910       $chain$12$?rcurveline@?$path_procs_t@Ucff2_path_procs_path_t@@U?$cff2_cs_interp_env_t@Unumber_t@CFF@@@CFF@@Ucff2_path_param_t@@@CFF@@SAXAEAU?$cff2_cs_interp_env_t@Unumber_t@CFF@@@2@AEAUcff2_path_param_t@@@Z 00000001800bf910     hb-ot-cff2-table.obj
 0002:00034920       $chain$1$?rlinecurve@?$path_procs_t@Ucff2_path_procs_path_t@@U?$cff2_cs_interp_env_t@Unumber_t@CFF@@@CFF@@Ucff2_path_param_t@@@CFF@@SAXAEAU?$cff2_cs_interp_env_t@Unumber_t@CFF@@@2@AEAUcff2_path_param_t@@@Z 00000001800bf920     hb-ot-cff2-table.obj
 0002:00034938       $chain$7$?rlinecurve@?$path_procs_t@Ucff2_path_procs_path_t@@U?$cff2_cs_interp_env_t@Unumber_t@CFF@@@CFF@@Ucff2_path_param_t@@@CFF@@SAXAEAU?$cff2_cs_interp_env_t@Unumber_t@CFF@@@2@AEAUcff2_path_param_t@@@Z 00000001800bf938     hb-ot-cff2-table.obj
 0002:00034960       $chain$8$?rlinecurve@?$path_procs_t@Ucff2_path_procs_path_t@@U?$cff2_cs_interp_env_t@Unumber_t@CFF@@@CFF@@Ucff2_path_param_t@@@CFF@@SAXAEAU?$cff2_cs_interp_env_t@Unumber_t@CFF@@@2@AEAUcff2_path_param_t@@@Z 00000001800bf960     hb-ot-cff2-table.obj
 0002:00034974       $chain$9$?rlinecurve@?$path_procs_t@Ucff2_path_procs_path_t@@U?$cff2_cs_interp_env_t@Unumber_t@CFF@@@CFF@@Ucff2_path_param_t@@@CFF@@SAXAEAU?$cff2_cs_interp_env_t@Unumber_t@CFF@@@2@AEAUcff2_path_param_t@@@Z 00000001800bf974     hb-ot-cff2-table.obj
 0002:00034984       $chain$10$?rlinecurve@?$path_procs_t@Ucff2_path_procs_path_t@@U?$cff2_cs_interp_env_t@Unumber_t@CFF@@@CFF@@Ucff2_path_param_t@@@CFF@@SAXAEAU?$cff2_cs_interp_env_t@Unumber_t@CFF@@@2@AEAUcff2_path_param_t@@@Z 00000001800bf984     hb-ot-cff2-table.obj
 0002:000349a8       $chain$11$?rlinecurve@?$path_procs_t@Ucff2_path_procs_path_t@@U?$cff2_cs_interp_env_t@Unumber_t@CFF@@@CFF@@Ucff2_path_param_t@@@CFF@@SAXAEAU?$cff2_cs_interp_env_t@Unumber_t@CFF@@@2@AEAUcff2_path_param_t@@@Z 00000001800bf9a8     hb-ot-cff2-table.obj
 0002:000349cc       $chain$12$?rlinecurve@?$path_procs_t@Ucff2_path_procs_path_t@@U?$cff2_cs_interp_env_t@Unumber_t@CFF@@@CFF@@Ucff2_path_param_t@@@CFF@@SAXAEAU?$cff2_cs_interp_env_t@Unumber_t@CFF@@@2@AEAUcff2_path_param_t@@@Z 00000001800bf9cc     hb-ot-cff2-table.obj
 0002:000349dc       $unwind$?hhcurveto@?$path_procs_t@Ucff2_path_procs_path_t@@U?$cff2_cs_interp_env_t@Unumber_t@CFF@@@CFF@@Ucff2_path_param_t@@@CFF@@SAXAEAU?$cff2_cs_interp_env_t@Unumber_t@CFF@@@2@AEAUcff2_path_param_t@@@Z 00000001800bf9dc     hb-ot-cff2-table.obj
 0002:000349dc       $unwind$?vvcurveto@?$path_procs_t@Ucff2_path_procs_path_t@@U?$cff2_cs_interp_env_t@Unumber_t@CFF@@@CFF@@Ucff2_path_param_t@@@CFF@@SAXAEAU?$cff2_cs_interp_env_t@Unumber_t@CFF@@@2@AEAUcff2_path_param_t@@@Z 00000001800bf9dc     hb-ot-cff2-table.obj
 0002:000349f8       $chain$2$?vvcurveto@?$path_procs_t@Ucff2_path_procs_path_t@@U?$cff2_cs_interp_env_t@Unumber_t@CFF@@@CFF@@Ucff2_path_param_t@@@CFF@@SAXAEAU?$cff2_cs_interp_env_t@Unumber_t@CFF@@@2@AEAUcff2_path_param_t@@@Z 00000001800bf9f8     hb-ot-cff2-table.obj
 0002:00034a14       $chain$3$?vvcurveto@?$path_procs_t@Ucff2_path_procs_path_t@@U?$cff2_cs_interp_env_t@Unumber_t@CFF@@@CFF@@Ucff2_path_param_t@@@CFF@@SAXAEAU?$cff2_cs_interp_env_t@Unumber_t@CFF@@@2@AEAUcff2_path_param_t@@@Z 00000001800bfa14     hb-ot-cff2-table.obj
 0002:00034a24       $chain$2$?hhcurveto@?$path_procs_t@Ucff2_path_procs_path_t@@U?$cff2_cs_interp_env_t@Unumber_t@CFF@@@CFF@@Ucff2_path_param_t@@@CFF@@SAXAEAU?$cff2_cs_interp_env_t@Unumber_t@CFF@@@2@AEAUcff2_path_param_t@@@Z 00000001800bfa24     hb-ot-cff2-table.obj
 0002:00034a40       $chain$3$?hhcurveto@?$path_procs_t@Ucff2_path_procs_path_t@@U?$cff2_cs_interp_env_t@Unumber_t@CFF@@@CFF@@Ucff2_path_param_t@@@CFF@@SAXAEAU?$cff2_cs_interp_env_t@Unumber_t@CFF@@@2@AEAUcff2_path_param_t@@@Z 00000001800bfa40     hb-ot-cff2-table.obj
 0002:00034a50       $unwind$?hvcurveto@?$path_procs_t@Ucff2_path_procs_path_t@@U?$cff2_cs_interp_env_t@Unumber_t@CFF@@@CFF@@Ucff2_path_param_t@@@CFF@@SAXAEAU?$cff2_cs_interp_env_t@Unumber_t@CFF@@@2@AEAUcff2_path_param_t@@@Z 00000001800bfa50     hb-ot-cff2-table.obj
 0002:00034a50       $unwind$?vhcurveto@?$path_procs_t@Ucff2_path_procs_path_t@@U?$cff2_cs_interp_env_t@Unumber_t@CFF@@@CFF@@Ucff2_path_param_t@@@CFF@@SAXAEAU?$cff2_cs_interp_env_t@Unumber_t@CFF@@@2@AEAUcff2_path_param_t@@@Z 00000001800bfa50     hb-ot-cff2-table.obj
 0002:00034a84       $chain$0$?vhcurveto@?$path_procs_t@Ucff2_path_procs_path_t@@U?$cff2_cs_interp_env_t@Unumber_t@CFF@@@CFF@@Ucff2_path_param_t@@@CFF@@SAXAEAU?$cff2_cs_interp_env_t@Unumber_t@CFF@@@2@AEAUcff2_path_param_t@@@Z 00000001800bfa84     hb-ot-cff2-table.obj
 0002:00034a98       $chain$1$?vhcurveto@?$path_procs_t@Ucff2_path_procs_path_t@@U?$cff2_cs_interp_env_t@Unumber_t@CFF@@@CFF@@Ucff2_path_param_t@@@CFF@@SAXAEAU?$cff2_cs_interp_env_t@Unumber_t@CFF@@@2@AEAUcff2_path_param_t@@@Z 00000001800bfa98     hb-ot-cff2-table.obj
 0002:00034aa8       $chain$0$?hvcurveto@?$path_procs_t@Ucff2_path_procs_path_t@@U?$cff2_cs_interp_env_t@Unumber_t@CFF@@@CFF@@Ucff2_path_param_t@@@CFF@@SAXAEAU?$cff2_cs_interp_env_t@Unumber_t@CFF@@@2@AEAUcff2_path_param_t@@@Z 00000001800bfaa8     hb-ot-cff2-table.obj
 0002:00034abc       $chain$1$?hvcurveto@?$path_procs_t@Ucff2_path_procs_path_t@@U?$cff2_cs_interp_env_t@Unumber_t@CFF@@@CFF@@Ucff2_path_param_t@@@CFF@@SAXAEAU?$cff2_cs_interp_env_t@Unumber_t@CFF@@@2@AEAUcff2_path_param_t@@@Z 00000001800bfabc     hb-ot-cff2-table.obj
 0002:00034acc       $unwind$?hflex1@?$path_procs_t@Ucff2_path_procs_path_t@@U?$cff2_cs_interp_env_t@Unumber_t@CFF@@@CFF@@Ucff2_path_param_t@@@CFF@@SAXAEAU?$cff2_cs_interp_env_t@Unumber_t@CFF@@@2@AEAUcff2_path_param_t@@@Z 00000001800bfacc     hb-ot-cff2-table.obj
 0002:00034acc       $unwind$?hflex@?$path_procs_t@Ucff2_path_procs_path_t@@U?$cff2_cs_interp_env_t@Unumber_t@CFF@@@CFF@@Ucff2_path_param_t@@@CFF@@SAXAEAU?$cff2_cs_interp_env_t@Unumber_t@CFF@@@2@AEAUcff2_path_param_t@@@Z 00000001800bfacc     hb-ot-cff2-table.obj
 0002:00034adc       $chain$9$?hflex@?$path_procs_t@Ucff2_path_procs_path_t@@U?$cff2_cs_interp_env_t@Unumber_t@CFF@@@CFF@@Ucff2_path_param_t@@@CFF@@SAXAEAU?$cff2_cs_interp_env_t@Unumber_t@CFF@@@2@AEAUcff2_path_param_t@@@Z 00000001800bfadc     hb-ot-cff2-table.obj
 0002:00034b14       $chain$10$?hflex@?$path_procs_t@Ucff2_path_procs_path_t@@U?$cff2_cs_interp_env_t@Unumber_t@CFF@@@CFF@@Ucff2_path_param_t@@@CFF@@SAXAEAU?$cff2_cs_interp_env_t@Unumber_t@CFF@@@2@AEAUcff2_path_param_t@@@Z 00000001800bfb14     hb-ot-cff2-table.obj
 0002:00034b34       $chain$11$?hflex@?$path_procs_t@Ucff2_path_procs_path_t@@U?$cff2_cs_interp_env_t@Unumber_t@CFF@@@CFF@@Ucff2_path_param_t@@@CFF@@SAXAEAU?$cff2_cs_interp_env_t@Unumber_t@CFF@@@2@AEAUcff2_path_param_t@@@Z 00000001800bfb34     hb-ot-cff2-table.obj
 0002:00034b44       $unwind$?flex@?$path_procs_t@Ucff2_path_procs_path_t@@U?$cff2_cs_interp_env_t@Unumber_t@CFF@@@CFF@@Ucff2_path_param_t@@@CFF@@SAXAEAU?$cff2_cs_interp_env_t@Unumber_t@CFF@@@2@AEAUcff2_path_param_t@@@Z 00000001800bfb44     hb-ot-cff2-table.obj
 0002:00034b54       $chain$1$?flex@?$path_procs_t@Ucff2_path_procs_path_t@@U?$cff2_cs_interp_env_t@Unumber_t@CFF@@@CFF@@Ucff2_path_param_t@@@CFF@@SAXAEAU?$cff2_cs_interp_env_t@Unumber_t@CFF@@@2@AEAUcff2_path_param_t@@@Z 00000001800bfb54     hb-ot-cff2-table.obj
 0002:00034b6c       $chain$9$?flex@?$path_procs_t@Ucff2_path_procs_path_t@@U?$cff2_cs_interp_env_t@Unumber_t@CFF@@@CFF@@Ucff2_path_param_t@@@CFF@@SAXAEAU?$cff2_cs_interp_env_t@Unumber_t@CFF@@@2@AEAUcff2_path_param_t@@@Z 00000001800bfb6c     hb-ot-cff2-table.obj
 0002:00034b9c       $chain$10$?flex@?$path_procs_t@Ucff2_path_procs_path_t@@U?$cff2_cs_interp_env_t@Unumber_t@CFF@@@CFF@@Ucff2_path_param_t@@@CFF@@SAXAEAU?$cff2_cs_interp_env_t@Unumber_t@CFF@@@2@AEAUcff2_path_param_t@@@Z 00000001800bfb9c     hb-ot-cff2-table.obj
 0002:00034bb8       $chain$11$?flex@?$path_procs_t@Ucff2_path_procs_path_t@@U?$cff2_cs_interp_env_t@Unumber_t@CFF@@@CFF@@Ucff2_path_param_t@@@CFF@@SAXAEAU?$cff2_cs_interp_env_t@Unumber_t@CFF@@@2@AEAUcff2_path_param_t@@@Z 00000001800bfbb8     hb-ot-cff2-table.obj
 0002:00034bc8       $chain$1$?hflex1@?$path_procs_t@Ucff2_path_procs_path_t@@U?$cff2_cs_interp_env_t@Unumber_t@CFF@@@CFF@@Ucff2_path_param_t@@@CFF@@SAXAEAU?$cff2_cs_interp_env_t@Unumber_t@CFF@@@2@AEAUcff2_path_param_t@@@Z 00000001800bfbc8     hb-ot-cff2-table.obj
 0002:00034be0       $chain$8$?hflex1@?$path_procs_t@Ucff2_path_procs_path_t@@U?$cff2_cs_interp_env_t@Unumber_t@CFF@@@CFF@@Ucff2_path_param_t@@@CFF@@SAXAEAU?$cff2_cs_interp_env_t@Unumber_t@CFF@@@2@AEAUcff2_path_param_t@@@Z 00000001800bfbe0     hb-ot-cff2-table.obj
 0002:00034c0c       $chain$9$?hflex1@?$path_procs_t@Ucff2_path_procs_path_t@@U?$cff2_cs_interp_env_t@Unumber_t@CFF@@@CFF@@Ucff2_path_param_t@@@CFF@@SAXAEAU?$cff2_cs_interp_env_t@Unumber_t@CFF@@@2@AEAUcff2_path_param_t@@@Z 00000001800bfc0c     hb-ot-cff2-table.obj
 0002:00034c28       $chain$10$?hflex1@?$path_procs_t@Ucff2_path_procs_path_t@@U?$cff2_cs_interp_env_t@Unumber_t@CFF@@@CFF@@Ucff2_path_param_t@@@CFF@@SAXAEAU?$cff2_cs_interp_env_t@Unumber_t@CFF@@@2@AEAUcff2_path_param_t@@@Z 00000001800bfc28     hb-ot-cff2-table.obj
 0002:00034c38       $unwind$?flex1@?$path_procs_t@Ucff2_path_procs_path_t@@U?$cff2_cs_interp_env_t@Unumber_t@CFF@@@CFF@@Ucff2_path_param_t@@@CFF@@SAXAEAU?$cff2_cs_interp_env_t@Unumber_t@CFF@@@2@AEAUcff2_path_param_t@@@Z 00000001800bfc38     hb-ot-cff2-table.obj
 0002:00034c48       $chain$4$?flex1@?$path_procs_t@Ucff2_path_procs_path_t@@U?$cff2_cs_interp_env_t@Unumber_t@CFF@@@CFF@@Ucff2_path_param_t@@@CFF@@SAXAEAU?$cff2_cs_interp_env_t@Unumber_t@CFF@@@2@AEAUcff2_path_param_t@@@Z 00000001800bfc48     hb-ot-cff2-table.obj
 0002:00034c6c       $chain$9$?flex1@?$path_procs_t@Ucff2_path_procs_path_t@@U?$cff2_cs_interp_env_t@Unumber_t@CFF@@@CFF@@Ucff2_path_param_t@@@CFF@@SAXAEAU?$cff2_cs_interp_env_t@Unumber_t@CFF@@@2@AEAUcff2_path_param_t@@@Z 00000001800bfc6c     hb-ot-cff2-table.obj
 0002:00034c90       $chain$10$?flex1@?$path_procs_t@Ucff2_path_procs_path_t@@U?$cff2_cs_interp_env_t@Unumber_t@CFF@@@CFF@@Ucff2_path_param_t@@@CFF@@SAXAEAU?$cff2_cs_interp_env_t@Unumber_t@CFF@@@2@AEAUcff2_path_param_t@@@Z 00000001800bfc90     hb-ot-cff2-table.obj
 0002:00034ca0       $chain$11$?flex1@?$path_procs_t@Ucff2_path_procs_path_t@@U?$cff2_cs_interp_env_t@Unumber_t@CFF@@@CFF@@Ucff2_path_param_t@@@CFF@@SAXAEAU?$cff2_cs_interp_env_t@Unumber_t@CFF@@@2@AEAUcff2_path_param_t@@@Z 00000001800bfca0     hb-ot-cff2-table.obj
 0002:00034cb0       $unwind$?process_op@?$cs_opset_t@Unumber_t@CFF@@Ucff2_cs_opset_path_t@@U?$cff2_cs_interp_env_t@Unumber_t@CFF@@@2@Ucff2_path_param_t@@Ucff2_path_procs_path_t@@@CFF@@SAXIAEAU?$cff2_cs_interp_env_t@Unumber_t@CFF@@@2@AEAUcff2_path_param_t@@@Z 00000001800bfcb0     hb-ot-cff2-table.obj
 0002:00034cd4       $chain$0$??C?$hb_lazy_loader_t@UCOLR@OT@@U?$hb_table_lazy_loader_t@UCOLR@OT@@$0CD@$00@@Uhb_face_t@@$0CD@Uhb_blob_t@@@@QEBAPEBUCOLR@OT@@XZ 00000001800bfcd4     hb-ot-color.obj
 0002:00034ce8       $chain$1$??C?$hb_lazy_loader_t@UCOLR@OT@@U?$hb_table_lazy_loader_t@UCOLR@OT@@$0CD@$00@@Uhb_face_t@@$0CD@Uhb_blob_t@@@@QEBAPEBUCOLR@OT@@XZ 00000001800bfce8     hb-ot-color.obj
 0002:00034cf8       $chain$0$??C?$hb_lazy_loader_t@UCPAL@OT@@U?$hb_table_lazy_loader_t@UCPAL@OT@@$0CE@$00@@Uhb_face_t@@$0CE@Uhb_blob_t@@@@QEBAPEBUCPAL@OT@@XZ 00000001800bfcf8     hb-ot-color.obj
 0002:00034d0c       $chain$1$??C?$hb_lazy_loader_t@UCPAL@OT@@U?$hb_table_lazy_loader_t@UCPAL@OT@@$0CE@$00@@Uhb_face_t@@$0CE@Uhb_blob_t@@@@QEBAPEBUCPAL@OT@@XZ 00000001800bfd0c     hb-ot-color.obj
 0002:00034d1c       $unwind$?get_stored@?$hb_lazy_loader_t@UCBDT_accelerator_t@OT@@U?$hb_face_lazy_loader_t@UCBDT_accelerator_t@OT@@$0CF@@@Uhb_face_t@@$0CF@U12@@@QEBAPEAUCBDT_accelerator_t@OT@@XZ 00000001800bfd1c     hb-ot-color.obj
 0002:00034d34       $unwind$?get_image_data@IndexSubtable@OT@@QEBA_NIPEAI00@Z 00000001800bfd34     hb-ot-color.obj
 0002:00034d48       $chain$0$?get_image_data@IndexSubtable@OT@@QEBA_NIPEAI00@Z 00000001800bfd48     hb-ot-color.obj
 0002:00034d5c       $chain$2$?get_image_data@IndexSubtable@OT@@QEBA_NIPEAI00@Z 00000001800bfd5c     hb-ot-color.obj
 0002:00034d70       $chain$3$?get_image_data@IndexSubtable@OT@@QEBA_NIPEAI00@Z 00000001800bfd70     hb-ot-color.obj
 0002:00034d80       $unwind$?choose_strike@CBLC@OT@@IEBAAEBUBitmapSizeTable@2@PEAUhb_font_t@@@Z 00000001800bfd80     hb-ot-color.obj
 0002:00034d8c       $chain$1$?choose_strike@CBLC@OT@@IEBAAEBUBitmapSizeTable@2@PEAUhb_font_t@@@Z 00000001800bfd8c     hb-ot-color.obj
 0002:00034da4       $chain$3$?choose_strike@CBLC@OT@@IEBAAEBUBitmapSizeTable@2@PEAUhb_font_t@@@Z 00000001800bfda4     hb-ot-color.obj
 0002:00034dbc       $unwind$?reference_png@accelerator_t@CBDT@OT@@QEBAPEAUhb_blob_t@@PEAUhb_font_t@@I@Z 00000001800bfdbc     hb-ot-color.obj
 0002:00034dd0       $unwind$?get_base_glyph_paint@COLR@OT@@QEBAPEBUPaint@2@I@Z 00000001800bfdd0     hb-ot-color.obj
 0002:00034de4       $unwind$?get_palette_colors@CPAL@OT@@QEBAIIIPEAI0@Z 00000001800bfde4     hb-ot-color.obj
 0002:00034df8       $chain$2$?get_palette_colors@CPAL@OT@@QEBAIIIPEAI0@Z 00000001800bfdf8     hb-ot-color.obj
 0002:00034e0c       $chain$3$?get_palette_colors@CPAL@OT@@QEBAIIIPEAI0@Z 00000001800bfe0c     hb-ot-color.obj
 0002:00034e1c       $unwind$?get_glyph_blob@SBIXStrike@OT@@QEBAPEAUhb_blob_t@@IPEAU3@IPEAH1IPEAI@Z 00000001800bfe1c     hb-ot-color.obj
 0002:00034e28       $chain$4$?get_glyph_blob@SBIXStrike@OT@@QEBAPEAUhb_blob_t@@IPEAU3@IPEAH1IPEAI@Z 00000001800bfe28     hb-ot-color.obj
 0002:00034e4c       $chain$6$?get_glyph_blob@SBIXStrike@OT@@QEBAPEAUhb_blob_t@@IPEAU3@IPEAH1IPEAI@Z 00000001800bfe4c     hb-ot-color.obj
 0002:00034e70       $unwind$?choose_strike@accelerator_t@sbix@OT@@AEBAAEBUSBIXStrike@3@PEAUhb_font_t@@@Z 00000001800bfe70     hb-ot-color.obj
 0002:00034e84       $chain$4$?choose_strike@accelerator_t@sbix@OT@@AEBAAEBUSBIXStrike@3@PEAUhb_font_t@@@Z 00000001800bfe84     hb-ot-color.obj
 0002:00034ea0       $chain$5$?choose_strike@accelerator_t@sbix@OT@@AEBAAEBUSBIXStrike@3@PEAUhb_font_t@@@Z 00000001800bfea0     hb-ot-color.obj
 0002:00034eb0       $unwind$??$sanitize@PEBUsbix@OT@@@?$ArrayOf@U?$OffsetTo@USBIXStrike@OT@@U?$IntType@I$03@2@$00@OT@@U?$IntType@I$03@2@@OT@@QEBA_NPEAUhb_sanitize_context_t@@$$QEAPEBUsbix@1@@Z 00000001800bfeb0     hb-ot-color.obj
 0002:00034eb0       $unwind$??$sanitize@PEBUFeatureVariations@OT@@@?$ArrayOf@UFeatureVariationRecord@OT@@U?$IntType@I$03@2@@OT@@QEBA_NPEAUhb_sanitize_context_t@@$$QEAPEBUFeatureVariations@1@@Z 00000001800bfeb0     hb-ot-layout.obj
 0002:00034ec8       $unwind$?reference_blob_for_glyph@accelerator_t@SVG@OT@@QEBAPEAUhb_blob_t@@I@Z 00000001800bfec8     hb-ot-color.obj
 0002:00034edc       $chain$0$??$dispatch@Uhb_sanitize_context_t@@$$V@Paint@OT@@QEBA_NPEAUhb_sanitize_context_t@@@Z 00000001800bfedc     hb-ot-color.obj
 0002:00034ef0       $chain$2$??$dispatch@Uhb_sanitize_context_t@@$$V@Paint@OT@@QEBA_NPEAUhb_sanitize_context_t@@@Z 00000001800bfef0     hb-ot-color.obj
 0002:00034ef0       $chain$4$??$dispatch@Uhb_sanitize_context_t@@$$V@Paint@OT@@QEBA_NPEAUhb_sanitize_context_t@@@Z 00000001800bfef0     hb-ot-color.obj
 0002:00034ef0       $chain$6$??$dispatch@Uhb_sanitize_context_t@@$$V@Paint@OT@@QEBA_NPEAUhb_sanitize_context_t@@@Z 00000001800bfef0     hb-ot-color.obj
 0002:00034ef0       $chain$8$??$dispatch@Uhb_sanitize_context_t@@$$V@Paint@OT@@QEBA_NPEAUhb_sanitize_context_t@@@Z 00000001800bfef0     hb-ot-color.obj
 0002:00034f04       $chain$9$??$dispatch@Uhb_sanitize_context_t@@$$V@Paint@OT@@QEBA_NPEAUhb_sanitize_context_t@@@Z 00000001800bff04     hb-ot-color.obj
 0002:00034f14       $unwind$??$sanitize_blob@Usbix@OT@@@hb_sanitize_context_t@@QEAAPEAUhb_blob_t@@PEAU1@@Z 00000001800bff14     hb-ot-color.obj
 0002:00034f30       $unwind$??$sanitize_blob@UCPAL@OT@@@hb_sanitize_context_t@@QEAAPEAUhb_blob_t@@PEAU1@@Z 00000001800bff30     hb-ot-color.obj
 0002:00034f4c       $chain$1$?shrink_vector@?$hb_vector_t@U?$cff1_private_dict_values_base_t@Udict_val_t@CFF@@@CFF@@$0A@@@QEAAXI@Z 00000001800bff4c     hb-ot-face.obj
 0002:00034f4c       $chain$1$?shrink_vector@?$hb_vector_t@Ucff1_font_dict_values_t@CFF@@$0A@@@QEAAXI@Z 00000001800bff4c     hb-ot-face.obj
 0002:00034f4c       $chain$1$?shrink_vector@?$hb_vector_t@Ucff2_font_dict_values_t@CFF@@$0A@@@QEAAXI@Z 00000001800bff4c     hb-ot-face.obj
 0002:00034f64       $chain$2$?shrink_vector@?$hb_vector_t@U?$cff1_private_dict_values_base_t@Udict_val_t@CFF@@@CFF@@$0A@@@QEAAXI@Z 00000001800bff64     hb-ot-face.obj
 0002:00034f64       $chain$2$?shrink_vector@?$hb_vector_t@Ucff1_font_dict_values_t@CFF@@$0A@@@QEAAXI@Z 00000001800bff64     hb-ot-face.obj
 0002:00034f64       $chain$2$?shrink_vector@?$hb_vector_t@Ucff2_font_dict_values_t@CFF@@$0A@@@QEAAXI@Z 00000001800bff64     hb-ot-face.obj
 0002:00034f74       $chain$1$?shrink_vector@?$hb_vector_t@U?$cff2_private_dict_values_base_t@Udict_val_t@CFF@@@CFF@@$0A@@@QEAAXI@Z 00000001800bff74     hb-ot-face.obj
 0002:00034f8c       $chain$2$?shrink_vector@?$hb_vector_t@U?$cff2_private_dict_values_base_t@Udict_val_t@CFF@@@CFF@@$0A@@@QEAAXI@Z 00000001800bff8c     hb-ot-face.obj
 0002:00034f9c       $unwind$hb_ot_font_set_funcs 00000001800bff9c     hb-ot-font.obj
 0002:00034fa8       $chain$0$hb_ot_font_set_funcs 00000001800bffa8     hb-ot-font.obj
 0002:00034fbc       $chain$1$hb_ot_font_set_funcs 00000001800bffbc     hb-ot-font.obj
 0002:00034fcc       $unwind$??$sort_r_simple@PEAX@@YAXPEAX_K1P6AHPEBX20@Z0@Z 00000001800bffcc     hb-ot-font.obj
 0002:00034fe4       $unwind$?get_glyph@VariationSelectorRecord@OT@@QEBA?AW4glyph_variant_t@2@IPEAIPEBX@Z 00000001800bffe4     hb-ot-font.obj
 0002:00034ff8       $unwind$?get_nominal_glyph@accelerator_t@cmap@OT@@QEBA_NIPEAIPEAU?$hb_cache_t@$0BF@$0BA@$07$00@@@Z 00000001800bfff8     hb-ot-font.obj
 0002:0003500c       $unwind$?cmp_gids@accelerator_t@post@OT@@KAHPEBX0PEAX@Z 00000001800c000c     hb-ot-font.obj
 0002:0003500c       $unwind$?push_root_transform@hb_paint_funcs_t@@QEAAXPEAXPEBUhb_font_t@@@Z 00000001800c000c     hb-ot-font.obj
 0002:0003501c       $unwind$?push_rotate@hb_paint_funcs_t@@QEAA_NPEAXM@Z 00000001800c001c     hb-ot-font.obj
 0002:00035030       $chain$0$?push_rotate@hb_paint_funcs_t@@QEAA_NPEAXM@Z 00000001800c0030     hb-ot-font.obj
 0002:00035044       $chain$1$?push_rotate@hb_paint_funcs_t@@QEAA_NPEAXM@Z 00000001800c0044     hb-ot-font.obj
 0002:00035054       $unwind$?push_skew@hb_paint_funcs_t@@QEAA_NPEAXMM@Z 00000001800c0054     hb-ot-font.obj
 0002:00035068       $chain$0$?push_skew@hb_paint_funcs_t@@QEAA_NPEAXMM@Z 00000001800c0068     hb-ot-font.obj
 0002:0003507c       $chain$1$?push_skew@hb_paint_funcs_t@@QEAA_NPEAXMM@Z 00000001800c007c     hb-ot-font.obj
 0002:0003508c       $unwind$?consume_point@path_builder_t@glyf_impl@OT@@QEAAXAEBUcontour_point_t@3@@Z 00000001800c008c     hb-ot-font.obj
 0002:000350a8       $chain$0$?consume_point@path_builder_t@glyf_impl@OT@@QEAAXAEBUcontour_point_t@3@@Z 00000001800c00a8     hb-ot-font.obj
 0002:000350bc       $chain$1$?consume_point@path_builder_t@glyf_impl@OT@@QEAAXAEBUcontour_point_t@3@@Z 00000001800c00bc     hb-ot-font.obj
 0002:000350bc       $chain$3$?consume_point@path_builder_t@glyf_impl@OT@@QEAAXAEBUcontour_point_t@3@@Z 00000001800c00bc     hb-ot-font.obj
 0002:000350cc       $chain$2$?consume_point@path_builder_t@glyf_impl@OT@@QEAAXAEBUcontour_point_t@3@@Z 00000001800c00cc     hb-ot-font.obj
 0002:000350e0       $unwind$?get_extents@glyf_accelerator_t@OT@@QEBA_NPEAUhb_font_t@@IPEAUhb_glyph_extents_t@@@Z 00000001800c00e0     hb-ot-font.obj
 0002:000350f4       $chain$1$?parse_bcd@dict_opset_t@CFF@@SANAEAUbyte_str_ref_t@2@@Z 00000001800c00f4     hb-ot-font.obj
 0002:0003510c       $chain$3$?parse_bcd@dict_opset_t@CFF@@SANAEAUbyte_str_ref_t@2@@Z 00000001800c010c     hb-ot-font.obj
 0002:00035124       $unwind$?sanitize@FDSelect0@CFF@@QEBA_NPEAUhb_sanitize_context_t@@I@Z 00000001800c0124     hb-ot-font.obj
 0002:0003512c       $unwind$?sanitize@Charset@CFF@@QEBA_NPEAUhb_sanitize_context_t@@@Z 00000001800c012c     hb-ot-font.obj
 0002:00035138       $chain$2$?sanitize@Charset@CFF@@QEBA_NPEAUhb_sanitize_context_t@@@Z 00000001800c0138     hb-ot-font.obj
 0002:00035154       $chain$4$?sanitize@Charset@CFF@@QEBA_NPEAUhb_sanitize_context_t@@@Z 00000001800c0154     hb-ot-font.obj
 0002:00035170       $chain$5$?sanitize@Charset@CFF@@QEBA_NPEAUhb_sanitize_context_t@@@Z 00000001800c0170     hb-ot-font.obj
 0002:00035180       $unwind$?process_op@cff1_top_dict_opset_t@CFF@@SAXIAEAUcff1_top_dict_interp_env_t@2@AEAUcff1_top_dict_values_t@2@@Z 00000001800c0180     hb-ot-font.obj
 0002:00035198       $chain$0$?process_op@cff1_top_dict_opset_t@CFF@@SAXIAEAUcff1_top_dict_interp_env_t@2@AEAUcff1_top_dict_values_t@2@@Z 00000001800c0198     hb-ot-font.obj
 0002:000351ac       $chain$1$?process_op@cff1_top_dict_opset_t@CFF@@SAXIAEAUcff1_top_dict_interp_env_t@2@AEAUcff1_top_dict_values_t@2@@Z 00000001800c01ac     hb-ot-font.obj
 0002:000351bc       $chain$2$?alloc@?$hb_vector_t@Ucff1_font_dict_values_t@CFF@@$0A@@@QEAA_NI_N@Z 00000001800c01bc     hb-ot-font.obj
 0002:000351d8       $chain$4$?alloc@?$hb_vector_t@Ucff1_font_dict_values_t@CFF@@$0A@@@QEAA_NI_N@Z 00000001800c01d8     hb-ot-font.obj
 0002:000351f4       $chain$5$?alloc@?$hb_vector_t@Ucff1_font_dict_values_t@CFF@@$0A@@@QEAA_NI_N@Z 00000001800c01f4     hb-ot-font.obj
 0002:00035208       $chain$6$?alloc@?$hb_vector_t@Ucff1_font_dict_values_t@CFF@@$0A@@@QEAA_NI_N@Z 00000001800c0208     hb-ot-font.obj
 0002:0003521c       $chain$7$?alloc@?$hb_vector_t@Ucff1_font_dict_values_t@CFF@@$0A@@@QEAA_NI_N@Z 00000001800c021c     hb-ot-font.obj
 0002:0003522c       $chain$8$?alloc@?$hb_vector_t@Ucff1_font_dict_values_t@CFF@@$0A@@@QEAA_NI_N@Z 00000001800c022c     hb-ot-font.obj
 0002:0003523c       $unwind$?init@?$accelerator_templ_t@Ucff1_private_dict_opset_t@CFF@@U?$cff1_private_dict_values_base_t@Udict_val_t@CFF@@@2@@cff1@OT@@QEAAXPEAUhb_face_t@@@Z 00000001800c023c     hb-ot-font.obj
 0002:00035260       $chain$2$?alloc@?$hb_vector_t@U?$cff1_private_dict_values_base_t@Udict_val_t@CFF@@@CFF@@$0A@@@QEAA_NI_N@Z 00000001800c0260     hb-ot-font.obj
 0002:0003527c       $chain$4$?alloc@?$hb_vector_t@U?$cff1_private_dict_values_base_t@Udict_val_t@CFF@@@CFF@@$0A@@@QEAA_NI_N@Z 00000001800c027c     hb-ot-font.obj
 0002:00035298       $chain$5$?alloc@?$hb_vector_t@U?$cff1_private_dict_values_base_t@Udict_val_t@CFF@@@CFF@@$0A@@@QEAA_NI_N@Z 00000001800c0298     hb-ot-font.obj
 0002:000352ac       $chain$6$?alloc@?$hb_vector_t@U?$cff1_private_dict_values_base_t@Udict_val_t@CFF@@@CFF@@$0A@@@QEAA_NI_N@Z 00000001800c02ac     hb-ot-font.obj
 0002:000352c0       $chain$7$?alloc@?$hb_vector_t@U?$cff1_private_dict_values_base_t@Udict_val_t@CFF@@@CFF@@$0A@@@QEAA_NI_N@Z 00000001800c02c0     hb-ot-font.obj
 0002:000352d0       $chain$8$?alloc@?$hb_vector_t@U?$cff1_private_dict_values_base_t@Udict_val_t@CFF@@@CFF@@$0A@@@QEAA_NI_N@Z 00000001800c02d0     hb-ot-font.obj
 0002:000352e0       $unwind$?get_glyph_from_name@accelerator_t@cff1@OT@@QEBA_NPEBDHPEAI@Z 00000001800c02e0     hb-ot-font.obj
 0002:000352fc       $chain$2$?alloc@?$hb_vector_t@Ucff2_font_dict_values_t@CFF@@$0A@@@QEAA_NI_N@Z 00000001800c02fc     hb-ot-font.obj
 0002:00035318       $chain$4$?alloc@?$hb_vector_t@Ucff2_font_dict_values_t@CFF@@$0A@@@QEAA_NI_N@Z 00000001800c0318     hb-ot-font.obj
 0002:00035334       $chain$5$?alloc@?$hb_vector_t@Ucff2_font_dict_values_t@CFF@@$0A@@@QEAA_NI_N@Z 00000001800c0334     hb-ot-font.obj
 0002:00035348       $chain$6$?alloc@?$hb_vector_t@Ucff2_font_dict_values_t@CFF@@$0A@@@QEAA_NI_N@Z 00000001800c0348     hb-ot-font.obj
 0002:0003535c       $chain$7$?alloc@?$hb_vector_t@Ucff2_font_dict_values_t@CFF@@$0A@@@QEAA_NI_N@Z 00000001800c035c     hb-ot-font.obj
 0002:0003536c       $chain$8$?alloc@?$hb_vector_t@Ucff2_font_dict_values_t@CFF@@$0A@@@QEAA_NI_N@Z 00000001800c036c     hb-ot-font.obj
 0002:0003537c       $unwind$??0?$accelerator_templ_t@Ucff2_private_dict_opset_t@CFF@@U?$cff2_private_dict_values_base_t@Udict_val_t@CFF@@@2@@cff2@OT@@QEAA@PEAUhb_face_t@@@Z 00000001800c037c     hb-ot-font.obj
 0002:000353a0       $unwind$??0accelerator_t@post@OT@@QEAA@PEAUhb_face_t@@@Z 00000001800c03a0     hb-ot-font.obj
 0002:000353b0       $chain$0$??0accelerator_t@post@OT@@QEAA@PEAUhb_face_t@@@Z 00000001800c03b0     hb-ot-font.obj
 0002:000353c4       $chain$1$??0accelerator_t@post@OT@@QEAA@PEAUhb_face_t@@@Z 00000001800c03c4     hb-ot-font.obj
 0002:000353d8       $chain$2$??0accelerator_t@post@OT@@QEAA@PEAUhb_face_t@@@Z 00000001800c03d8     hb-ot-font.obj
 0002:000353e8       $chain$4$??0accelerator_t@post@OT@@QEAA@PEAUhb_face_t@@@Z 00000001800c03e8     hb-ot-font.obj
 0002:000353fc       $chain$5$??0accelerator_t@post@OT@@QEAA@PEAUhb_face_t@@@Z 00000001800c03fc     hb-ot-font.obj
 0002:0003540c       $unwind$?get_glyph_from_name@accelerator_t@post@OT@@QEBA_NPEBDHPEAI@Z 00000001800c040c     hb-ot-font.obj
 0002:00035424       $chain$2$?get_extents@accelerator_t@CBDT@OT@@QEBA_NPEAUhb_font_t@@IPEAUhb_glyph_extents_t@@_N@Z 00000001800c0424     hb-ot-font.obj
 0002:00035440       $chain$3$?get_extents@accelerator_t@CBDT@OT@@QEBA_NPEAUhb_font_t@@IPEAUhb_glyph_extents_t@@_N@Z 00000001800c0440     hb-ot-font.obj
 0002:00035450       $unwind$??0hb_paint_extents_context_t@@QEAA@XZ 00000001800c0450     hb-ot-font.obj
 0002:00035468       $unwind$?get_color@hb_paint_context_t@OT@@QEAAIIMPEAH@Z 00000001800c0468     hb-ot-font.obj
 0002:0003547c       $unwind$?get_color_stop@ColorStop@OT@@QEBAXPEAUhb_paint_context_t@2@PEAUhb_color_stop_t@@IAEBUVarStoreInstancer@2@@Z 00000001800c047c     hb-ot-font.obj
 0002:00035494       $unwind$?paint_glyph@Affine2x3@OT@@QEBAXPEAUhb_paint_context_t@2@I@Z 00000001800c0494     hb-ot-font.obj
 0002:000354c8       $unwind$?paint_glyph@PaintColrLayers@OT@@QEBAXPEAUhb_paint_context_t@2@@Z 00000001800c04c8     hb-ot-font.obj
 0002:000354d8       $chain$2$?paint_glyph@PaintColrLayers@OT@@QEBAXPEAUhb_paint_context_t@2@@Z 00000001800c04d8     hb-ot-font.obj
 0002:000354f4       $chain$3$?paint_glyph@PaintColrLayers@OT@@QEBAXPEAUhb_paint_context_t@2@@Z 00000001800c04f4     hb-ot-font.obj
 0002:00035504       $unwind$?paint_glyph@PaintSolid@OT@@QEBAXPEAUhb_paint_context_t@2@I@Z 00000001800c0504     hb-ot-font.obj
 0002:00035518       $unwind$?paint_glyph@PaintColrGlyph@OT@@QEBAXPEAUhb_paint_context_t@2@@Z 00000001800c0518     hb-ot-font.obj
 0002:0003552c       $unwind$?paint_glyph@PaintTranslate@OT@@QEBAXPEAUhb_paint_context_t@2@I@Z 00000001800c052c     hb-ot-font.obj
 0002:0003554c       $unwind$?paint_glyph@PaintScale@OT@@QEBAXPEAUhb_paint_context_t@2@I@Z 00000001800c054c     hb-ot-font.obj
 0002:00035568       $unwind$?paint_glyph@PaintScaleAroundCenter@OT@@QEBAXPEAUhb_paint_context_t@2@I@Z 00000001800c0568     hb-ot-font.obj
 0002:00035568       $unwind$?paint_glyph@PaintSkewAroundCenter@OT@@QEBAXPEAUhb_paint_context_t@2@I@Z 00000001800c0568     hb-ot-font.obj
 0002:000355a0       $unwind$?paint_glyph@PaintScaleUniform@OT@@QEBAXPEAUhb_paint_context_t@2@I@Z 00000001800c05a0     hb-ot-font.obj
 0002:000355b8       $unwind$?paint_glyph@PaintRotateAroundCenter@OT@@QEBAXPEAUhb_paint_context_t@2@I@Z 00000001800c05b8     hb-ot-font.obj
 0002:000355b8       $unwind$?paint_glyph@PaintScaleUniformAroundCenter@OT@@QEBAXPEAUhb_paint_context_t@2@I@Z 00000001800c05b8     hb-ot-font.obj
 0002:000355ec       $unwind$?paint_glyph@PaintRotate@OT@@QEBAXPEAUhb_paint_context_t@2@I@Z 00000001800c05ec     hb-ot-font.obj
 0002:00035600       $unwind$?paint_glyph@PaintSkew@OT@@QEBAXPEAUhb_paint_context_t@2@I@Z 00000001800c0600     hb-ot-font.obj
 0002:0003561c       $chain$1$?get_clip_box@ClipBoxFormat2@OT@@QEBAXAEAUClipBoxData@2@AEBUVarStoreInstancer@2@@Z 00000001800c061c     hb-ot-font.obj
 0002:00035634       $chain$2$?get_clip_box@ClipBoxFormat2@OT@@QEBAXAEAUClipBoxData@2@AEBUVarStoreInstancer@2@@Z 00000001800c0634     hb-ot-font.obj
 0002:00035644       $unwind$?paint_glyph@?$PaintLinearGradient@UNoVariable@OT@@@OT@@QEBAXPEAUhb_paint_context_t@2@I@Z 00000001800c0644     hb-ot-font.obj
 0002:00035644       $unwind$?paint_glyph@?$PaintLinearGradient@UVariable@OT@@@OT@@QEBAXPEAUhb_paint_context_t@2@I@Z 00000001800c0644     hb-ot-font.obj
 0002:00035644       $unwind$?paint_glyph@?$PaintRadialGradient@UNoVariable@OT@@@OT@@QEBAXPEAUhb_paint_context_t@2@I@Z 00000001800c0644     hb-ot-font.obj
 0002:00035644       $unwind$?paint_glyph@?$PaintRadialGradient@UVariable@OT@@@OT@@QEBAXPEAUhb_paint_context_t@2@I@Z 00000001800c0644     hb-ot-font.obj
 0002:00035678       $unwind$?static_get_color_stops@?$ColorLine@UNoVariable@OT@@@OT@@SAIPEAUhb_color_line_t@@PEAXIPEAIPEAUhb_color_stop_t@@1@Z 00000001800c0678     hb-ot-font.obj
 0002:00035678       $unwind$?static_get_color_stops@?$ColorLine@UVariable@OT@@@OT@@SAIPEAUhb_color_line_t@@PEAXIPEAIPEAUhb_color_stop_t@@1@Z 00000001800c0678     hb-ot-font.obj
 0002:0003568c       $chain$0$?static_get_color_stops@?$ColorLine@UNoVariable@OT@@@OT@@SAIPEAUhb_color_line_t@@PEAXIPEAIPEAUhb_color_stop_t@@1@Z 00000001800c068c     hb-ot-font.obj
 0002:000356a0       $chain$1$?static_get_color_stops@?$ColorLine@UNoVariable@OT@@@OT@@SAIPEAUhb_color_line_t@@PEAXIPEAIPEAUhb_color_stop_t@@1@Z 00000001800c06a0     hb-ot-font.obj
 0002:000356b4       $chain$2$?static_get_color_stops@?$ColorLine@UNoVariable@OT@@@OT@@SAIPEAUhb_color_line_t@@PEAXIPEAIPEAUhb_color_stop_t@@1@Z 00000001800c06b4     hb-ot-font.obj
 0002:000356c4       $chain$4$?static_get_color_stops@?$ColorLine@UNoVariable@OT@@@OT@@SAIPEAUhb_color_line_t@@PEAXIPEAIPEAUhb_color_stop_t@@1@Z 00000001800c06c4     hb-ot-font.obj
 0002:000356d8       $chain$5$?static_get_color_stops@?$ColorLine@UNoVariable@OT@@@OT@@SAIPEAUhb_color_line_t@@PEAXIPEAIPEAUhb_color_stop_t@@1@Z 00000001800c06d8     hb-ot-font.obj
 0002:000356e8       $chain$0$?static_get_color_stops@?$ColorLine@UVariable@OT@@@OT@@SAIPEAUhb_color_line_t@@PEAXIPEAIPEAUhb_color_stop_t@@1@Z 00000001800c06e8     hb-ot-font.obj
 0002:000356fc       $chain$1$?static_get_color_stops@?$ColorLine@UVariable@OT@@@OT@@SAIPEAUhb_color_line_t@@PEAXIPEAIPEAUhb_color_stop_t@@1@Z 00000001800c06fc     hb-ot-font.obj
 0002:00035710       $chain$2$?static_get_color_stops@?$ColorLine@UVariable@OT@@@OT@@SAIPEAUhb_color_line_t@@PEAXIPEAIPEAUhb_color_stop_t@@1@Z 00000001800c0710     hb-ot-font.obj
 0002:00035720       $chain$4$?static_get_color_stops@?$ColorLine@UVariable@OT@@@OT@@SAIPEAUhb_color_line_t@@PEAXIPEAIPEAUhb_color_stop_t@@1@Z 00000001800c0720     hb-ot-font.obj
 0002:00035734       $chain$5$?static_get_color_stops@?$ColorLine@UVariable@OT@@@OT@@SAIPEAUhb_color_line_t@@PEAXIPEAIPEAUhb_color_stop_t@@1@Z 00000001800c0734     hb-ot-font.obj
 0002:00035744       $unwind$?paint_glyph@?$PaintSweepGradient@UNoVariable@OT@@@OT@@QEBAXPEAUhb_paint_context_t@2@I@Z 00000001800c0744     hb-ot-font.obj
 0002:00035744       $unwind$?paint_glyph@?$PaintSweepGradient@UVariable@OT@@@OT@@QEBAXPEAUhb_paint_context_t@2@I@Z 00000001800c0744     hb-ot-font.obj
 0002:00035770       $unwind$?get_extents@COLR@OT@@QEBA_NPEAUhb_font_t@@IPEAUhb_glyph_extents_t@@@Z 00000001800c0770     hb-ot-font.obj
 0002:00035788       $chain$0$?get_extents@COLR@OT@@QEBA_NPEAUhb_font_t@@IPEAUhb_glyph_extents_t@@@Z 00000001800c0788     hb-ot-font.obj
 0002:0003579c       $chain$1$?get_extents@COLR@OT@@QEBA_NPEAUhb_font_t@@IPEAUhb_glyph_extents_t@@@Z 00000001800c079c     hb-ot-font.obj
 0002:000357b0       $chain$2$?get_extents@COLR@OT@@QEBA_NPEAUhb_font_t@@IPEAUhb_glyph_extents_t@@@Z 00000001800c07b0     hb-ot-font.obj
 0002:000357c0       $chain$3$?get_extents@COLR@OT@@QEBA_NPEAUhb_font_t@@IPEAUhb_glyph_extents_t@@@Z 00000001800c07c0     hb-ot-font.obj
 0002:000357d0       $unwind$?paint_glyph@COLR@OT@@QEBA_NPEAUhb_font_t@@IPEAUhb_paint_funcs_t@@PEAXII_N@Z 00000001800c07d0     hb-ot-font.obj
 0002:000357ec       $chain$0$?paint_glyph@COLR@OT@@QEBA_NPEAUhb_font_t@@IPEAUhb_paint_funcs_t@@PEAXII_N@Z 00000001800c07ec     hb-ot-font.obj
 0002:00035800       $chain$1$?paint_glyph@COLR@OT@@QEBA_NPEAUhb_font_t@@IPEAUhb_paint_funcs_t@@PEAXII_N@Z 00000001800c0800     hb-ot-font.obj
 0002:00035810       $unwind$?get_png_extents@accelerator_t@sbix@OT@@AEBA_NPEAUhb_font_t@@IPEAUhb_glyph_extents_t@@_N@Z 00000001800c0810     hb-ot-font.obj
 0002:00035828       $unwind$?hb_ot_get_nominal_glyph@@YAHPEAUhb_font_t@@PEAXIPEAI1@Z 00000001800c0828     hb-ot-font.obj
 0002:0003583c       $unwind$?hb_ot_get_nominal_glyphs@@YAIPEAUhb_font_t@@PEAXIPEBIIPEAII1@Z 00000001800c083c     hb-ot-font.obj
 0002:00035850       $chain$1$?hb_ot_get_nominal_glyphs@@YAIPEAUhb_font_t@@PEAXIPEBIIPEAII1@Z 00000001800c0850     hb-ot-font.obj
 0002:00035868       $chain$2$?hb_ot_get_nominal_glyphs@@YAIPEAUhb_font_t@@PEAXIPEBIIPEAII1@Z 00000001800c0868     hb-ot-font.obj
 0002:00035878       $unwind$?hb_ot_get_glyph_h_advances@@YAXPEAUhb_font_t@@PEAXIPEBIIPEAHI1@Z 00000001800c0878     hb-ot-font.obj
 0002:00035884       $chain$5$?hb_ot_get_glyph_h_advances@@YAXPEAUhb_font_t@@PEAXIPEBIIPEAHI1@Z 00000001800c0884     hb-ot-font.obj
 0002:000358ac       $chain$6$?hb_ot_get_glyph_h_advances@@YAXPEAUhb_font_t@@PEAXIPEBIIPEAHI1@Z 00000001800c08ac     hb-ot-font.obj
 0002:000358bc       $unwind$?hb_ot_get_glyph_v_advances@@YAXPEAUhb_font_t@@PEAXIPEBIIPEAHI1@Z 00000001800c08bc     hb-ot-font.obj
 0002:000358d4       $chain$2$?hb_ot_get_glyph_v_advances@@YAXPEAUhb_font_t@@PEAXIPEBIIPEAHI1@Z 00000001800c08d4     hb-ot-font.obj
 0002:000358f0       $chain$4$?hb_ot_get_glyph_v_advances@@YAXPEAUhb_font_t@@PEAXIPEBIIPEAHI1@Z 00000001800c08f0     hb-ot-font.obj
 0002:00035908       $chain$5$?hb_ot_get_glyph_v_advances@@YAXPEAUhb_font_t@@PEAXIPEBIIPEAHI1@Z 00000001800c0908     hb-ot-font.obj
 0002:00035918       $chain$6$?hb_ot_get_glyph_v_advances@@YAXPEAUhb_font_t@@PEAXIPEBIIPEAHI1@Z 00000001800c0918     hb-ot-font.obj
 0002:00035928       $unwind$?hb_ot_get_glyph_v_origin@@YAHPEAUhb_font_t@@PEAXIPEAH21@Z 00000001800c0928     hb-ot-font.obj
 0002:00035948       $chain$0$?hb_ot_get_glyph_v_origin@@YAHPEAUhb_font_t@@PEAXIPEAH21@Z 00000001800c0948     hb-ot-font.obj
 0002:0003595c       $unwind$?hb_ot_get_glyph_name@@YAHPEAUhb_font_t@@PEAXIPEADI1@Z 00000001800c095c     hb-ot-font.obj
 0002:00035970       $unwind$?hb_ot_draw_glyph@@YAXPEAUhb_font_t@@PEAXIPEAUhb_draw_funcs_t@@11@Z 00000001800c0970     hb-ot-font.obj
 0002:00035998       $unwind$?hb_ot_paint_glyph@@YAXPEAUhb_font_t@@PEAXIPEAUhb_paint_funcs_t@@1II1@Z 00000001800c0998     hb-ot-font.obj
 0002:000359b4       $chain$2$?hb_ot_paint_glyph@@YAXPEAUhb_font_t@@PEAXIPEAUhb_paint_funcs_t@@1II1@Z 00000001800c09b4     hb-ot-font.obj
 0002:000359d0       $chain$3$?hb_ot_paint_glyph@@YAXPEAUhb_font_t@@PEAXIPEAUhb_paint_funcs_t@@1II1@Z 00000001800c09d0     hb-ot-font.obj
 0002:000359e0       $unwind$?interpret@?$dict_interpreter_t@Ucff1_font_dict_opset_t@CFF@@Ucff1_font_dict_values_t@2@U?$interp_env_t@Unumber_t@CFF@@@2@@CFF@@QEAA_NAEAUcff1_font_dict_values_t@2@@Z 00000001800c09e0     hb-ot-font.obj
 0002:000359e0       $unwind$?interpret@?$dict_interpreter_t@Ucff2_font_dict_opset_t@CFF@@Ucff2_font_dict_values_t@2@U?$interp_env_t@Unumber_t@CFF@@@2@@CFF@@QEAA_NAEAUcff2_font_dict_values_t@2@@Z 00000001800c09e0     hb-ot-font.obj
 0002:000359e0       $unwind$?apply@?$ContextFormat2_5@USmallTypes@Layout@OT@@@OT@@QEBA_NPEAUhb_ot_apply_context_t@2@_N@Z 00000001800c09e0     hb-ot-layout.obj
 0002:000359e0       $unwind$?has_feature@hb_ot_map_builder_t@@QEAA_NI@Z 00000001800c09e0     hb-ot-map.obj
 0002:000359e0       $unwind$?get_var@MVAR@OT@@QEBAMIPEBHI@Z 00000001800c09e0     hb-ot-metrics.obj
 0002:000359e0       $unwind$?would_substitute@hb_indic_would_substitute_feature_t@@QEBA_NPEBIIPEAUhb_face_t@@@Z 00000001800c09e0     hb-ot-shaper-indic.obj
 0002:000359f8       $unwind$?interpret@?$dict_interpreter_t@Ucff1_private_dict_opset_t@CFF@@U?$cff1_private_dict_values_base_t@Udict_val_t@CFF@@@2@U?$interp_env_t@Unumber_t@CFF@@@2@@CFF@@QEAA_NAEAU?$cff1_private_dict_values_base_t@Udict_val_t@CFF@@@2@@Z 00000001800c09f8     hb-ot-font.obj
 0002:000359f8       $unwind$?interpret@?$dict_interpreter_t@Ucff2_private_dict_opset_t@CFF@@U?$cff2_private_dict_values_base_t@Udict_val_t@CFF@@@2@Ucff2_priv_dict_interp_env_t@2@@CFF@@QEAA_NAEAU?$cff2_private_dict_values_base_t@Udict_val_t@CFF@@@2@@Z 00000001800c09f8     hb-ot-font.obj
 0002:00035a10       $unwind$??$realloc_vector@U?$cff2_private_dict_values_base_t@Udict_val_t@CFF@@@CFF@@$0A@@?$hb_vector_t@U?$cff2_private_dict_values_base_t@Udict_val_t@CFF@@@CFF@@$0A@@@QEAAPEAU?$cff2_private_dict_values_base_t@Udict_val_t@CFF@@@CFF@@I@Z 00000001800c0a10     hb-ot-font.obj
 0002:00035a1c       $chain$2$??$realloc_vector@U?$cff2_private_dict_values_base_t@Udict_val_t@CFF@@@CFF@@$0A@@?$hb_vector_t@U?$cff2_private_dict_values_base_t@Udict_val_t@CFF@@@CFF@@$0A@@@QEAAPEAU?$cff2_private_dict_values_base_t@Udict_val_t@CFF@@@CFF@@I@Z 00000001800c0a1c     hb-ot-font.obj
 0002:00035a34       $chain$3$??$realloc_vector@U?$cff2_private_dict_values_base_t@Udict_val_t@CFF@@@CFF@@$0A@@?$hb_vector_t@U?$cff2_private_dict_values_base_t@Udict_val_t@CFF@@@CFF@@$0A@@@QEAAPEAU?$cff2_private_dict_values_base_t@Udict_val_t@CFF@@@CFF@@I@Z 00000001800c0a34     hb-ot-font.obj
 0002:00035a48       $chain$4$??$realloc_vector@U?$cff2_private_dict_values_base_t@Udict_val_t@CFF@@@CFF@@$0A@@?$hb_vector_t@U?$cff2_private_dict_values_base_t@Udict_val_t@CFF@@@CFF@@$0A@@@QEAAPEAU?$cff2_private_dict_values_base_t@Udict_val_t@CFF@@@CFF@@I@Z 00000001800c0a48     hb-ot-font.obj
 0002:00035a58       $chain$5$??$realloc_vector@U?$cff2_private_dict_values_base_t@Udict_val_t@CFF@@@CFF@@$0A@@?$hb_vector_t@U?$cff2_private_dict_values_base_t@Udict_val_t@CFF@@@CFF@@$0A@@@QEAAPEAU?$cff2_private_dict_values_base_t@Udict_val_t@CFF@@@CFF@@I@Z 00000001800c0a58     hb-ot-font.obj
 0002:00035a68       $unwind$??$sanitize_blob@Ucff1@OT@@@hb_sanitize_context_t@@QEAAPEAUhb_blob_t@@PEAU1@@Z 00000001800c0a68     hb-ot-font.obj
 0002:00035a68       $unwind$??$sanitize_blob@Ucff2@OT@@@hb_sanitize_context_t@@QEAAPEAUhb_blob_t@@PEAU1@@Z 00000001800c0a68     hb-ot-font.obj
 0002:00035a84       $unwind$??$sanitize_blob@UVORG@OT@@@hb_sanitize_context_t@@QEAAPEAUhb_blob_t@@PEAU1@@Z 00000001800c0a84     hb-ot-font.obj
 0002:00035aa0       $unwind$hb_ot_layout_lookup_would_substitute 00000001800c0aa0     hb-ot-layout.obj
 0002:00035ab4       $chain$2$hb_ot_layout_lookup_would_substitute 00000001800c0ab4     hb-ot-layout.obj
 0002:00035acc       $chain$3$hb_ot_layout_lookup_would_substitute 00000001800c0acc     hb-ot-layout.obj
 0002:00035adc       $unwind$?position@hb_ot_map_t@@QEBAXPEBUhb_ot_shape_plan_t@@PEAUhb_font_t@@PEAUhb_buffer_t@@@Z 00000001800c0adc     hb-ot-layout.obj
 0002:00035adc       $unwind$?substitute@hb_ot_map_t@@QEBAXPEBUhb_ot_shape_plan_t@@PEAUhb_font_t@@PEAUhb_buffer_t@@@Z 00000001800c0adc     hb-ot-layout.obj
 0002:00035af0       $unwind$?get_stored@?$hb_lazy_loader_t@UGPOS_accelerator_t@OT@@U?$hb_face_lazy_loader_t@UGPOS_accelerator_t@OT@@$0BK@@@Uhb_face_t@@$0BK@U12@@@QEBAPEAUGPOS_accelerator_t@OT@@XZ 00000001800c0af0     hb-ot-layout.obj
 0002:00035af0       $unwind$?get_stored@?$hb_lazy_loader_t@UGSUB_accelerator_t@OT@@U?$hb_face_lazy_loader_t@UGSUB_accelerator_t@OT@@$0BJ@@@Uhb_face_t@@$0BJ@U12@@@QEBAPEAUGSUB_accelerator_t@OT@@XZ 00000001800c0af0     hb-ot-layout.obj
 0002:00035b08       $unwind$?hb_ot_layout_substitute_start@@YAXPEAUhb_font_t@@PEAUhb_buffer_t@@@Z 00000001800c0b08     hb-ot-layout.obj
 0002:00035b14       $chain$4$?hb_ot_layout_substitute_start@@YAXPEAUhb_font_t@@PEAUhb_buffer_t@@@Z 00000001800c0b14     hb-ot-layout.obj
 0002:00035b38       $chain$5$?hb_ot_layout_substitute_start@@YAXPEAUhb_font_t@@PEAUhb_buffer_t@@@Z 00000001800c0b38     hb-ot-layout.obj
 0002:00035b48       $chain$0$?get_population@Coverage@Common@Layout@OT@@QEBAIXZ 00000001800c0b48     hb-ot-layout.obj
 0002:00035b5c       $chain$1$?get_population@Coverage@Common@Layout@OT@@QEBAIXZ 00000001800c0b5c     hb-ot-layout.obj
 0002:00035b6c       $unwind$?get_indexes@IndexArray@OT@@QEBAIIPEAI0@Z 00000001800c0b6c     hb-ot-layout.obj
 0002:00035b88       $unwind$?sanitize@Feature@OT@@QEBA_NPEAUhb_sanitize_context_t@@PEBURecord_sanitize_closure_t@2@@Z 00000001800c0b88     hb-ot-layout.obj
 0002:00035ba0       $unwind$??$sanitize@I@?$OffsetTo@UFeatureParams@OT@@U?$IntType@G$01@2@$00@OT@@QEBA_NPEAUhb_sanitize_context_t@@PEBX$$QEAI@Z 00000001800c0ba0     hb-ot-layout.obj
 0002:00035ba0       $unwind$?compose_hebrew@@YA_NPEBUhb_ot_shape_normalize_context_t@@IIPEAI@Z 00000001800c0ba0     hb-ot-shaper-hebrew.obj
 0002:00035ba0       $unwind$?compose_khmer@@YA_NPEBUhb_ot_shape_normalize_context_t@@IIPEAI@Z 00000001800c0ba0     hb-ot-shaper-khmer.obj
 0002:00035ba0       $unwind$?compose_use@@YA_NPEBUhb_ot_shape_normalize_context_t@@IIPEAI@Z 00000001800c0ba0     hb-ot-shaper-use.obj
 0002:00035bb4       $unwind$?sanitize@?$RecordListOf@UFeature@OT@@@OT@@QEBA_NPEAUhb_sanitize_context_t@@@Z 00000001800c0bb4     hb-ot-layout.obj
 0002:00035bc0       $chain$4$?sanitize@?$RecordListOf@UFeature@OT@@@OT@@QEBA_NPEAUhb_sanitize_context_t@@@Z 00000001800c0bc0     hb-ot-layout.obj
 0002:00035be4       $chain$6$?sanitize@?$RecordListOf@UFeature@OT@@@OT@@QEBA_NPEAUhb_sanitize_context_t@@@Z 00000001800c0be4     hb-ot-layout.obj
 0002:00035c08       $chain$7$?sanitize@?$RecordListOf@UFeature@OT@@@OT@@QEBA_NPEAUhb_sanitize_context_t@@@Z 00000001800c0c08     hb-ot-layout.obj
 0002:00035c18       $unwind$?find_index@FeatureVariations@OT@@QEBA_NPEBHIPEAI@Z 00000001800c0c18     hb-ot-layout.obj
 0002:00035c30       $unwind$?get_delta@HintingDevice@OT@@AEBAHIH@Z 00000001800c0c30     hb-ot-layout.obj
 0002:00035c40       $chain$0$?get_delta@HintingDevice@OT@@AEBAHIH@Z 00000001800c0c40     hb-ot-layout.obj
 0002:00035c54       $chain$1$?get_delta@HintingDevice@OT@@AEBAHIH@Z 00000001800c0c54     hb-ot-layout.obj
 0002:00035c64       $unwind$?ligate_input@OT@@YA_NPEAUhb_ot_apply_context_t@1@IQEBIIII@Z 00000001800c0c64     hb-ot-layout.obj
 0002:00035c7c       $unwind$?apply_lookup@OT@@YAXPEAUhb_ot_apply_context_t@1@IQEAIIQEBULookupRecord@1@I@Z 00000001800c0c7c     hb-ot-layout.obj
 0002:00035c90       $chain$1$?apply_lookup@OT@@YAXPEAUhb_ot_apply_context_t@1@IQEAIIQEBULookupRecord@1@I@Z 00000001800c0c90     hb-ot-layout.obj
 0002:00035ca8       $chain$2$?apply_lookup@OT@@YAXPEAUhb_ot_apply_context_t@1@IQEAIIQEBULookupRecord@1@I@Z 00000001800c0ca8     hb-ot-layout.obj
 0002:00035cb8       $chain$3$?apply_lookup@OT@@YAXPEAUhb_ot_apply_context_t@1@IQEAIIQEBULookupRecord@1@I@Z 00000001800c0cb8     hb-ot-layout.obj
 0002:00035cd0       $unwind$?apply@ContextFormat3@OT@@QEBA_NPEAUhb_ot_apply_context_t@2@@Z 00000001800c0cd0     hb-ot-layout.obj
 0002:00035cdc       $unwind$??$context_apply_lookup@U?$IntType@G$01@OT@@@OT@@YA_NPEAUhb_ot_apply_context_t@0@IQEBU?$IntType@G$01@0@IQEBULookupRecord@0@AEBUContextApplyLookupContext@0@@Z 00000001800c0cdc     hb-ot-layout.obj
 0002:00035cf8       $chain$0$??$context_apply_lookup@U?$IntType@G$01@OT@@@OT@@YA_NPEAUhb_ot_apply_context_t@0@IQEBU?$IntType@G$01@0@IQEBULookupRecord@0@AEBUContextApplyLookupContext@0@@Z 00000001800c0cf8     hb-ot-layout.obj
 0002:00035d0c       $chain$1$??$context_apply_lookup@U?$IntType@G$01@OT@@@OT@@YA_NPEAUhb_ot_apply_context_t@0@IQEBU?$IntType@G$01@0@IQEBULookupRecord@0@AEBUContextApplyLookupContext@0@@Z 00000001800c0d0c     hb-ot-layout.obj
 0002:00035d1c       $unwind$?apply@?$RuleSet@USmallTypes@Layout@OT@@@OT@@QEBA_NPEAUhb_ot_apply_context_t@2@AEBUContextApplyLookupContext@2@@Z 00000001800c0d1c     hb-ot-layout.obj
 0002:00035d1c       $unwind$?would_apply@?$RuleSet@USmallTypes@Layout@OT@@@OT@@QEBA_NPEAUhb_would_apply_context_t@2@AEBUContextApplyLookupContext@2@@Z 00000001800c0d1c     hb-ot-layout.obj
 0002:00035d3c       $unwind$?apply@ChainContextFormat3@OT@@QEBA_NPEAUhb_ot_apply_context_t@2@@Z 00000001800c0d3c     hb-ot-layout.obj
 0002:00035d4c       $chain$1$?apply@ChainContextFormat3@OT@@QEBA_NPEAUhb_ot_apply_context_t@2@@Z 00000001800c0d4c     hb-ot-layout.obj
 0002:00035d64       $chain$2$?apply@ChainContextFormat3@OT@@QEBA_NPEAUhb_ot_apply_context_t@2@@Z 00000001800c0d64     hb-ot-layout.obj
 0002:00035d74       $unwind$??$chain_context_apply_lookup@U?$IntType@G$01@OT@@@OT@@YA_NPEAUhb_ot_apply_context_t@0@IQEBU?$IntType@G$01@0@I1I1IQEBULookupRecord@0@AEBUChainContextApplyLookupContext@0@@Z 00000001800c0d74     hb-ot-layout.obj
 0002:00035d94       $unwind$?would_apply@?$ChainRuleSet@USmallTypes@Layout@OT@@@OT@@QEBA_NPEAUhb_would_apply_context_t@2@AEBUChainContextApplyLookupContext@2@@Z 00000001800c0d94     hb-ot-layout.obj
 0002:00035db4       $unwind$?apply@?$ChainRuleSet@USmallTypes@Layout@OT@@@OT@@QEBA_NPEAUhb_ot_apply_context_t@2@AEBUChainContextApplyLookupContext@2@@Z 00000001800c0db4     hb-ot-layout.obj
 0002:00035dd4       $unwind$?apply@hb_ot_layout_lookup_accelerator_t@OT@@QEBA_NPEAUhb_ot_apply_context_t@2@I_N@Z 00000001800c0dd4     hb-ot-layout.obj
 0002:00035de8       $unwind$?get_lookup@GSUBGPOS@OT@@QEBAAEBULookup@2@I@Z 00000001800c0de8     hb-ot-layout.obj
 0002:00035df8       $unwind$?get_feature_variation@GSUBGPOS@OT@@QEBAAEBUFeature@2@II@Z 00000001800c0df8     hb-ot-layout.obj
 0002:00035e04       $unwind$?apply_value@ValueFormat@GPOS_impl@Layout@OT@@QEBA_NPEAUhb_ot_apply_context_t@4@PEBXPEBU?$IntType@G$01@4@AEAUhb_glyph_position_t@@@Z 00000001800c0e04     hb-ot-layout.obj
 0002:00035e20       $chain$3$?apply_value@ValueFormat@GPOS_impl@Layout@OT@@QEBA_NPEAUhb_ot_apply_context_t@4@PEBXPEBU?$IntType@G$01@4@AEAUhb_glyph_position_t@@@Z 00000001800c0e20     hb-ot-layout.obj
 0002:00035e34       $unwind$?sanitize_values@ValueFormat@GPOS_impl@Layout@OT@@QEBA_NPEAUhb_sanitize_context_t@@PEBXPEBU?$IntType@G$01@4@I@Z 00000001800c0e34     hb-ot-layout.obj
 0002:00035e34       $unwind$?sanitize_values_stride_unsafe@ValueFormat@GPOS_impl@Layout@OT@@QEBA_NPEAUhb_sanitize_context_t@@PEBXPEBU?$IntType@G$01@4@II@Z 00000001800c0e34     hb-ot-layout.obj
 0002:00035e50       $unwind$?apply@SinglePosFormat2@GPOS_impl@Layout@OT@@QEBA_NPEAUhb_ot_apply_context_t@4@@Z 00000001800c0e50     hb-ot-layout.obj
 0002:00035e64       $chain$1$?apply@SinglePosFormat2@GPOS_impl@Layout@OT@@QEBA_NPEAUhb_ot_apply_context_t@4@@Z 00000001800c0e64     hb-ot-layout.obj
 0002:00035e78       $chain$2$?apply@SinglePosFormat2@GPOS_impl@Layout@OT@@QEBA_NPEAUhb_ot_apply_context_t@4@@Z 00000001800c0e78     hb-ot-layout.obj
 0002:00035e88       $unwind$?apply@?$PairSet@USmallTypes@Layout@OT@@@GPOS_impl@Layout@OT@@QEBA_NPEAUhb_ot_apply_context_t@4@PEBUValueFormat@234@I@Z 00000001800c0e88     hb-ot-layout.obj
 0002:00035ea0       $unwind$?sanitize@?$PairPosFormat1_3@USmallTypes@Layout@OT@@@GPOS_impl@Layout@OT@@QEBA_NPEAUhb_sanitize_context_t@@@Z 00000001800c0ea0     hb-ot-layout.obj
 0002:00035eb8       $unwind$?apply@?$PairPosFormat1_3@USmallTypes@Layout@OT@@@GPOS_impl@Layout@OT@@QEBA_NPEAUhb_ot_apply_context_t@4@@Z 00000001800c0eb8     hb-ot-layout.obj
 0002:00035ed0       $chain$1$?apply@?$PairPosFormat1_3@USmallTypes@Layout@OT@@@GPOS_impl@Layout@OT@@QEBA_NPEAUhb_ot_apply_context_t@4@@Z 00000001800c0ed0     hb-ot-layout.obj
 0002:00035ee4       $chain$2$?apply@?$PairPosFormat1_3@USmallTypes@Layout@OT@@@GPOS_impl@Layout@OT@@QEBA_NPEAUhb_ot_apply_context_t@4@@Z 00000001800c0ee4     hb-ot-layout.obj
 0002:00035ef4       $unwind$?sanitize@?$PairPosFormat2_4@USmallTypes@Layout@OT@@@GPOS_impl@Layout@OT@@QEBA_NPEAUhb_sanitize_context_t@@@Z 00000001800c0ef4     hb-ot-layout.obj
 0002:00035f00       $chain$5$?sanitize@?$PairPosFormat2_4@USmallTypes@Layout@OT@@@GPOS_impl@Layout@OT@@QEBA_NPEAUhb_sanitize_context_t@@@Z 00000001800c0f00     hb-ot-layout.obj
 0002:00035f28       $chain$6$?sanitize@?$PairPosFormat2_4@USmallTypes@Layout@OT@@@GPOS_impl@Layout@OT@@QEBA_NPEAUhb_sanitize_context_t@@@Z 00000001800c0f28     hb-ot-layout.obj
 0002:00035f38       $unwind$?apply@?$PairPosFormat2_4@USmallTypes@Layout@OT@@@GPOS_impl@Layout@OT@@QEBA_NPEAUhb_ot_apply_context_t@4@@Z 00000001800c0f38     hb-ot-layout.obj
 0002:00035f4c       $chain$2$?apply@?$PairPosFormat2_4@USmallTypes@Layout@OT@@@GPOS_impl@Layout@OT@@QEBA_NPEAUhb_ot_apply_context_t@4@@Z 00000001800c0f4c     hb-ot-layout.obj
 0002:00035f64       $chain$3$?apply@?$PairPosFormat2_4@USmallTypes@Layout@OT@@@GPOS_impl@Layout@OT@@QEBA_NPEAUhb_ot_apply_context_t@4@@Z 00000001800c0f64     hb-ot-layout.obj
 0002:00035f74       $unwind$?get_anchor@AnchorFormat3@GPOS_impl@Layout@OT@@QEBAXPEAUhb_ot_apply_context_t@4@IPEAM1@Z 00000001800c0f74     hb-ot-layout.obj
 0002:00035f8c       $chain$0$?get_anchor@AnchorFormat3@GPOS_impl@Layout@OT@@QEBAXPEAUhb_ot_apply_context_t@4@IPEAM1@Z 00000001800c0f8c     hb-ot-layout.obj
 0002:00035fa0       $chain$1$?get_anchor@AnchorFormat3@GPOS_impl@Layout@OT@@QEBAXPEAUhb_ot_apply_context_t@4@IPEAM1@Z 00000001800c0fa0     hb-ot-layout.obj
 0002:00035fb0       $unwind$?get_anchor@Anchor@GPOS_impl@Layout@OT@@QEBAXPEAUhb_ot_apply_context_t@4@IPEAM1@Z 00000001800c0fb0     hb-ot-layout.obj
 0002:00035fc0       $chain$2$?get_anchor@Anchor@GPOS_impl@Layout@OT@@QEBAXPEAUhb_ot_apply_context_t@4@IPEAM1@Z 00000001800c0fc0     hb-ot-layout.obj
 0002:00035fdc       $chain$3$?get_anchor@Anchor@GPOS_impl@Layout@OT@@QEBAXPEAUhb_ot_apply_context_t@4@IPEAM1@Z 00000001800c0fdc     hb-ot-layout.obj
 0002:00035fec       $unwind$?reverse_cursive_minor_offset@GPOS_impl@Layout@OT@@YAXPEAUhb_glyph_position_t@@IW4hb_direction_t@@I@Z 00000001800c0fec     hb-ot-layout.obj
 0002:00036000       $chain$0$?reverse_cursive_minor_offset@GPOS_impl@Layout@OT@@YAXPEAUhb_glyph_position_t@@IW4hb_direction_t@@I@Z 00000001800c1000     hb-ot-layout.obj
 0002:00036014       $chain$1$?reverse_cursive_minor_offset@GPOS_impl@Layout@OT@@YAXPEAUhb_glyph_position_t@@IW4hb_direction_t@@I@Z 00000001800c1014     hb-ot-layout.obj
 0002:00036024       $unwind$?apply@CursivePosFormat1@GPOS_impl@Layout@OT@@QEBA_NPEAUhb_ot_apply_context_t@4@@Z 00000001800c1024     hb-ot-layout.obj
 0002:00036038       $chain$0$?apply@CursivePosFormat1@GPOS_impl@Layout@OT@@QEBA_NPEAUhb_ot_apply_context_t@4@@Z 00000001800c1038     hb-ot-layout.obj
 0002:0003604c       $chain$3$?apply@CursivePosFormat1@GPOS_impl@Layout@OT@@QEBA_NPEAUhb_ot_apply_context_t@4@@Z 00000001800c104c     hb-ot-layout.obj
 0002:00036068       $chain$4$?apply@CursivePosFormat1@GPOS_impl@Layout@OT@@QEBA_NPEAUhb_ot_apply_context_t@4@@Z 00000001800c1068     hb-ot-layout.obj
 0002:00036078       $chain$5$?apply@CursivePosFormat1@GPOS_impl@Layout@OT@@QEBA_NPEAUhb_ot_apply_context_t@4@@Z 00000001800c1078     hb-ot-layout.obj
 0002:00036088       $unwind$?apply@MarkArray@GPOS_impl@Layout@OT@@QEBA_NPEAUhb_ot_apply_context_t@4@IIAEBUAnchorMatrix@234@II@Z 00000001800c1088     hb-ot-layout.obj
 0002:0003609c       $unwind$?apply@?$MarkBasePosFormat1_2@USmallTypes@Layout@OT@@@GPOS_impl@Layout@OT@@QEBA_NPEAUhb_ot_apply_context_t@4@@Z 00000001800c109c     hb-ot-layout.obj
 0002:000360b8       $unwind$?apply@?$MarkLigPosFormat1_2@USmallTypes@Layout@OT@@@GPOS_impl@Layout@OT@@QEBA_NPEAUhb_ot_apply_context_t@4@@Z 00000001800c10b8     hb-ot-layout.obj
 0002:000360d4       $unwind$?apply@?$MarkMarkPosFormat1_2@USmallTypes@Layout@OT@@@GPOS_impl@Layout@OT@@QEBA_NPEAUhb_ot_apply_context_t@4@@Z 00000001800c10d4     hb-ot-layout.obj
 0002:000360e8       $chain$1$?apply@?$MarkMarkPosFormat1_2@USmallTypes@Layout@OT@@@GPOS_impl@Layout@OT@@QEBA_NPEAUhb_ot_apply_context_t@4@@Z 00000001800c10e8     hb-ot-layout.obj
 0002:000360fc       $chain$2$?apply@?$MarkMarkPosFormat1_2@USmallTypes@Layout@OT@@@GPOS_impl@Layout@OT@@QEBA_NPEAUhb_ot_apply_context_t@4@@Z 00000001800c10fc     hb-ot-layout.obj
 0002:00036110       $chain$3$?apply@?$MarkMarkPosFormat1_2@USmallTypes@Layout@OT@@@GPOS_impl@Layout@OT@@QEBA_NPEAUhb_ot_apply_context_t@4@@Z 00000001800c1110     hb-ot-layout.obj
 0002:00036120       $chain$4$?apply@?$MarkMarkPosFormat1_2@USmallTypes@Layout@OT@@@GPOS_impl@Layout@OT@@QEBA_NPEAUhb_ot_apply_context_t@4@@Z 00000001800c1120     hb-ot-layout.obj
 0002:00036130       $chain$5$?apply@?$MarkMarkPosFormat1_2@USmallTypes@Layout@OT@@@GPOS_impl@Layout@OT@@QEBA_NPEAUhb_ot_apply_context_t@4@@Z 00000001800c1130     hb-ot-layout.obj
 0002:00036148       $unwind$??$sanitize@UPosLookupSubTable@GPOS_impl@Layout@OT@@@Lookup@OT@@QEBA_NPEAUhb_sanitize_context_t@@@Z 00000001800c1148     hb-ot-layout.obj
 0002:00036148       $unwind$??$sanitize@USubstLookupSubTable@GSUB_impl@Layout@OT@@@Lookup@OT@@QEBA_NPEAUhb_sanitize_context_t@@@Z 00000001800c1148     hb-ot-layout.obj
 0002:00036164       $unwind$?propagate_attachment_offsets@Layout@OT@@YAXPEAUhb_glyph_position_t@@IIW4hb_direction_t@@I@Z 00000001800c1164     hb-ot-layout.obj
 0002:00036178       $chain$0$?propagate_attachment_offsets@Layout@OT@@YAXPEAUhb_glyph_position_t@@IIW4hb_direction_t@@I@Z 00000001800c1178     hb-ot-layout.obj
 0002:0003618c       $chain$1$?propagate_attachment_offsets@Layout@OT@@YAXPEAUhb_glyph_position_t@@IIW4hb_direction_t@@I@Z 00000001800c118c     hb-ot-layout.obj
 0002:0003619c       $unwind$?position_finish_offsets@GPOS@Layout@OT@@SAXPEAUhb_font_t@@PEAUhb_buffer_t@@@Z 00000001800c119c     hb-ot-layout.obj
 0002:000361ac       $chain$0$?position_finish_offsets@GPOS@Layout@OT@@SAXPEAUhb_font_t@@PEAUhb_buffer_t@@@Z 00000001800c11ac     hb-ot-layout.obj
 0002:000361c0       $chain$1$?position_finish_offsets@GPOS@Layout@OT@@SAXPEAUhb_font_t@@PEAUhb_buffer_t@@@Z 00000001800c11c0     hb-ot-layout.obj
 0002:000361d4       $chain$3$?position_finish_offsets@GPOS@Layout@OT@@SAXPEAUhb_font_t@@PEAUhb_buffer_t@@@Z 00000001800c11d4     hb-ot-layout.obj
 0002:000361ec       $chain$4$?position_finish_offsets@GPOS@Layout@OT@@SAXPEAUhb_font_t@@PEAUhb_buffer_t@@@Z 00000001800c11ec     hb-ot-layout.obj
 0002:000361fc       $chain$5$?position_finish_offsets@GPOS@Layout@OT@@SAXPEAUhb_font_t@@PEAUhb_buffer_t@@@Z 00000001800c11fc     hb-ot-layout.obj
 0002:0003620c       $chain$6$?position_finish_offsets@GPOS@Layout@OT@@SAXPEAUhb_font_t@@PEAUhb_buffer_t@@@Z 00000001800c120c     hb-ot-layout.obj
 0002:0003621c       $chain$7$?position_finish_offsets@GPOS@Layout@OT@@SAXPEAUhb_font_t@@PEAUhb_buffer_t@@@Z 00000001800c121c     hb-ot-layout.obj
 0002:00036230       $chain$8$?position_finish_offsets@GPOS@Layout@OT@@SAXPEAUhb_font_t@@PEAUhb_buffer_t@@@Z 00000001800c1230     hb-ot-layout.obj
 0002:00036240       $unwind$?get_accel@?$accelerator_t@UGPOS@Layout@OT@@@GSUBGPOS@OT@@QEBAPEAUhb_ot_layout_lookup_accelerator_t@3@I@Z 00000001800c1240     hb-ot-layout.obj
 0002:00036240       $unwind$?get_accel@?$accelerator_t@UGSUB@Layout@OT@@@GSUBGPOS@OT@@QEBAPEAUhb_ot_layout_lookup_accelerator_t@3@I@Z 00000001800c1240     hb-ot-layout.obj
 0002:00036258       $unwind$?apply@?$KerxTable@UKernOT@OT@@@AAT@@QEBA_NPEAUhb_aat_apply_context_t@2@@Z 00000001800c1258     hb-ot-layout.obj
 0002:00036274       $unwind$?apply@?$KerxTable@UKernAAT@OT@@@AAT@@QEBA_NPEAUhb_aat_apply_context_t@2@@Z 00000001800c1274     hb-ot-layout.obj
 0002:0003629c       $unwind$?apply@?$SingleSubstFormat2_4@USmallTypes@Layout@OT@@@GSUB_impl@Layout@OT@@QEBA_NPEAUhb_ot_apply_context_t@4@@Z 00000001800c129c     hb-ot-layout.obj
 0002:000362b0       $unwind$?apply@?$Sequence@USmallTypes@Layout@OT@@@GSUB_impl@Layout@OT@@QEBA_NPEAUhb_ot_apply_context_t@4@@Z 00000001800c12b0     hb-ot-layout.obj
 0002:000362cc       $chain$1$?apply@?$Sequence@USmallTypes@Layout@OT@@@GSUB_impl@Layout@OT@@QEBA_NPEAUhb_ot_apply_context_t@4@@Z 00000001800c12cc     hb-ot-layout.obj
 0002:000362e4       $chain$2$?apply@?$Sequence@USmallTypes@Layout@OT@@@GSUB_impl@Layout@OT@@QEBA_NPEAUhb_ot_apply_context_t@4@@Z 00000001800c12e4     hb-ot-layout.obj
 0002:000362f8       $chain$3$?apply@?$Sequence@USmallTypes@Layout@OT@@@GSUB_impl@Layout@OT@@QEBA_NPEAUhb_ot_apply_context_t@4@@Z 00000001800c12f8     hb-ot-layout.obj
 0002:00036308       $chain$4$?apply@?$Sequence@USmallTypes@Layout@OT@@@GSUB_impl@Layout@OT@@QEBA_NPEAUhb_ot_apply_context_t@4@@Z 00000001800c1308     hb-ot-layout.obj
 0002:00036318       $unwind$?apply@?$AlternateSet@USmallTypes@Layout@OT@@@GSUB_impl@Layout@OT@@QEBA_NPEAUhb_ot_apply_context_t@4@@Z 00000001800c1318     hb-ot-layout.obj
 0002:00036328       $unwind$?apply@?$Ligature@USmallTypes@Layout@OT@@@GSUB_impl@Layout@OT@@QEBA_NPEAUhb_ot_apply_context_t@4@@Z 00000001800c1328     hb-ot-layout.obj
 0002:00036340       $chain$1$?apply@?$Ligature@USmallTypes@Layout@OT@@@GSUB_impl@Layout@OT@@QEBA_NPEAUhb_ot_apply_context_t@4@@Z 00000001800c1340     hb-ot-layout.obj
 0002:00036358       $chain$3$?apply@?$Ligature@USmallTypes@Layout@OT@@@GSUB_impl@Layout@OT@@QEBA_NPEAUhb_ot_apply_context_t@4@@Z 00000001800c1358     hb-ot-layout.obj
 0002:00036370       $chain$4$?apply@?$Ligature@USmallTypes@Layout@OT@@@GSUB_impl@Layout@OT@@QEBA_NPEAUhb_ot_apply_context_t@4@@Z 00000001800c1370     hb-ot-layout.obj
 0002:00036384       $chain$5$?apply@?$Ligature@USmallTypes@Layout@OT@@@GSUB_impl@Layout@OT@@QEBA_NPEAUhb_ot_apply_context_t@4@@Z 00000001800c1384     hb-ot-layout.obj
 0002:00036394       $chain$6$?apply@?$Ligature@USmallTypes@Layout@OT@@@GSUB_impl@Layout@OT@@QEBA_NPEAUhb_ot_apply_context_t@4@@Z 00000001800c1394     hb-ot-layout.obj
 0002:000363a8       $chain$7$?apply@?$Ligature@USmallTypes@Layout@OT@@@GSUB_impl@Layout@OT@@QEBA_NPEAUhb_ot_apply_context_t@4@@Z 00000001800c13a8     hb-ot-layout.obj
 0002:000363b8       $chain$8$?apply@?$Ligature@USmallTypes@Layout@OT@@@GSUB_impl@Layout@OT@@QEBA_NPEAUhb_ot_apply_context_t@4@@Z 00000001800c13b8     hb-ot-layout.obj
 0002:000363c8       $unwind$?would_apply@?$LigatureSubstFormat1_2@USmallTypes@Layout@OT@@@GSUB_impl@Layout@OT@@QEBA_NPEAUhb_would_apply_context_t@4@@Z 00000001800c13c8     hb-ot-layout.obj
 0002:000363dc       $chain$1$?would_apply@?$LigatureSubstFormat1_2@USmallTypes@Layout@OT@@@GSUB_impl@Layout@OT@@QEBA_NPEAUhb_would_apply_context_t@4@@Z 00000001800c13dc     hb-ot-layout.obj
 0002:000363f4       $chain$2$?would_apply@?$LigatureSubstFormat1_2@USmallTypes@Layout@OT@@@GSUB_impl@Layout@OT@@QEBA_NPEAUhb_would_apply_context_t@4@@Z 00000001800c13f4     hb-ot-layout.obj
 0002:00036404       $unwind$?apply@?$LigatureSubstFormat1_2@USmallTypes@Layout@OT@@@GSUB_impl@Layout@OT@@QEBA_NPEAUhb_ot_apply_context_t@4@@Z 00000001800c1404     hb-ot-layout.obj
 0002:00036414       $chain$2$?apply@?$LigatureSubstFormat1_2@USmallTypes@Layout@OT@@@GSUB_impl@Layout@OT@@QEBA_NPEAUhb_ot_apply_context_t@4@@Z 00000001800c1414     hb-ot-layout.obj
 0002:00036430       $chain$4$?apply@?$LigatureSubstFormat1_2@USmallTypes@Layout@OT@@@GSUB_impl@Layout@OT@@QEBA_NPEAUhb_ot_apply_context_t@4@@Z 00000001800c1430     hb-ot-layout.obj
 0002:0003644c       $unwind$?apply@ReverseChainSingleSubstFormat1@GSUB_impl@Layout@OT@@QEBA_NPEAUhb_ot_apply_context_t@4@@Z 00000001800c144c     hb-ot-layout.obj
 0002:00036464       $unwind$??$match_backtrack@U?$IntType@G$01@OT@@@OT@@YA_NPEAUhb_ot_apply_context_t@0@IQEBU?$IntType@G$01@0@P6A_NAEAUhb_glyph_info_t@@IPEBX@Z3PEAI@Z 00000001800c1464     hb-ot-layout.obj
 0002:00036480       $unwind$??$match_lookahead@U?$IntType@G$01@OT@@@OT@@YA_NPEAUhb_ot_apply_context_t@0@IQEBU?$IntType@G$01@0@P6A_NAEAUhb_glyph_info_t@@IPEBX@Z3IPEAI@Z 00000001800c1480     hb-ot-layout.obj
 0002:0003649c       $unwind$?apply_forward@@YA_NPEAUhb_ot_apply_context_t@OT@@AEBUhb_ot_layout_lookup_accelerator_t@2@I@Z 00000001800c149c     hb-ot-layout.obj
 0002:000364ac       $chain$2$?apply_forward@@YA_NPEAUhb_ot_apply_context_t@OT@@AEBUhb_ot_layout_lookup_accelerator_t@2@I@Z 00000001800c14ac     hb-ot-layout.obj
 0002:000364c8       $chain$3$?apply_forward@@YA_NPEAUhb_ot_apply_context_t@OT@@AEBUhb_ot_layout_lookup_accelerator_t@2@I@Z 00000001800c14c8     hb-ot-layout.obj
 0002:000364dc       $chain$4$?apply_forward@@YA_NPEAUhb_ot_apply_context_t@OT@@AEBUhb_ot_layout_lookup_accelerator_t@2@I@Z 00000001800c14dc     hb-ot-layout.obj
 0002:000364ec       $chain$5$?apply_forward@@YA_NPEAUhb_ot_apply_context_t@OT@@AEBUhb_ot_layout_lookup_accelerator_t@2@I@Z 00000001800c14ec     hb-ot-layout.obj
 0002:000364fc       $unwind$?apply_backward@@YA_NPEAUhb_ot_apply_context_t@OT@@AEBUhb_ot_layout_lookup_accelerator_t@2@I@Z 00000001800c14fc     hb-ot-layout.obj
 0002:00036518       $unwind$??$apply@UGPOSProxy@@@hb_ot_map_t@@QEBAXAEBUGPOSProxy@@PEBUhb_ot_shape_plan_t@@PEAUhb_font_t@@PEAUhb_buffer_t@@@Z 00000001800c1518     hb-ot-layout.obj
 0002:00036518       $unwind$??$apply@UGSUBProxy@@@hb_ot_map_t@@QEBAXAEBUGSUBProxy@@PEBUhb_ot_shape_plan_t@@PEAUhb_font_t@@PEAUhb_buffer_t@@@Z 00000001800c1518     hb-ot-layout.obj
 0002:00036530       $chain$0$??$apply_string@UGSUBProxy@@@@YA_NPEAUhb_ot_apply_context_t@OT@@AEBUSubstLookup@GSUB_impl@Layout@1@AEBUhb_ot_layout_lookup_accelerator_t@1@@Z 00000001800c1530     hb-ot-layout.obj
 0002:00036544       $chain$2$??$apply_string@UGSUBProxy@@@@YA_NPEAUhb_ot_apply_context_t@OT@@AEBUSubstLookup@GSUB_impl@Layout@1@AEBUhb_ot_layout_lookup_accelerator_t@1@@Z 00000001800c1544     hb-ot-layout.obj
 0002:00036558       $chain$3$??$apply_string@UGSUBProxy@@@@YA_NPEAUhb_ot_apply_context_t@OT@@AEBUSubstLookup@GSUB_impl@Layout@1@AEBUhb_ot_layout_lookup_accelerator_t@1@@Z 00000001800c1558     hb-ot-layout.obj
 0002:00036568       $unwind$??$create@USubstLookup@GSUB_impl@Layout@OT@@@hb_ot_layout_lookup_accelerator_t@OT@@SAPEAU01@AEBUSubstLookup@GSUB_impl@Layout@1@@Z 00000001800c1568     hb-ot-layout.obj
 0002:00036574       $chain$4$??$create@USubstLookup@GSUB_impl@Layout@OT@@@hb_ot_layout_lookup_accelerator_t@OT@@SAPEAU01@AEBUSubstLookup@GSUB_impl@Layout@1@@Z 00000001800c1574     hb-ot-layout.obj
 0002:00036598       $chain$5$??$create@USubstLookup@GSUB_impl@Layout@OT@@@hb_ot_layout_lookup_accelerator_t@OT@@SAPEAU01@AEBUSubstLookup@GSUB_impl@Layout@1@@Z 00000001800c1598     hb-ot-layout.obj
 0002:000365b0       $chain$6$??$create@USubstLookup@GSUB_impl@Layout@OT@@@hb_ot_layout_lookup_accelerator_t@OT@@SAPEAU01@AEBUSubstLookup@GSUB_impl@Layout@1@@Z 00000001800c15b0     hb-ot-layout.obj
 0002:000365c4       $unwind$??$would_match_input@U?$IntType@G$01@OT@@@OT@@YA_NPEAUhb_would_apply_context_t@0@IQEBU?$IntType@G$01@0@P6A_NAEAUhb_glyph_info_t@@IPEBX@Z3@Z 00000001800c15c4     hb-ot-layout.obj
 0002:000365e0       $unwind$??$match_input@U?$IntType@G$01@OT@@@OT@@YA_NPEAUhb_ot_apply_context_t@0@IQEBU?$IntType@G$01@0@P6A_NAEAUhb_glyph_info_t@@IPEBX@Z3PEAIQEAI5@Z 00000001800c15e0     hb-ot-layout.obj
 0002:000365e0       $unwind$??$match_input@UHBGlyphID16@OT@@@OT@@YA_NPEAUhb_ot_apply_context_t@0@IQEBUHBGlyphID16@0@P6A_NAEAUhb_glyph_info_t@@IPEBX@Z3PEAIQEAI5@Z 00000001800c15e0     hb-ot-layout.obj
 0002:000365fc       $unwind$??$dispatch@Uhb_would_apply_context_t@OT@@$$V@Context@OT@@QEBA_NPEAUhb_would_apply_context_t@1@@Z 00000001800c15fc     hb-ot-layout.obj
 0002:00036610       $chain$0$??$dispatch@Uhb_would_apply_context_t@OT@@$$V@Context@OT@@QEBA_NPEAUhb_would_apply_context_t@1@@Z 00000001800c1610     hb-ot-layout.obj
 0002:00036624       $chain$1$??$dispatch@Uhb_would_apply_context_t@OT@@$$V@Context@OT@@QEBA_NPEAUhb_would_apply_context_t@1@@Z 00000001800c1624     hb-ot-layout.obj
 0002:00036634       $unwind$??$dispatch@Uhb_would_apply_context_t@OT@@$$V@ChainContext@OT@@QEBA_NPEAUhb_would_apply_context_t@1@@Z 00000001800c1634     hb-ot-layout.obj
 0002:00036644       $chain$2$??$dispatch@Uhb_would_apply_context_t@OT@@$$V@ChainContext@OT@@QEBA_NPEAUhb_would_apply_context_t@1@@Z 00000001800c1644     hb-ot-layout.obj
 0002:00036660       $chain$3$??$dispatch@Uhb_would_apply_context_t@OT@@$$V@ChainContext@OT@@QEBA_NPEAUhb_would_apply_context_t@1@@Z 00000001800c1660     hb-ot-layout.obj
 0002:00036670       $chain$0$??$dispatch@Uhb_accelerate_subtables_context_t@OT@@$$V@ChainContext@OT@@QEBA?AUhb_empty_t@@PEAUhb_accelerate_subtables_context_t@1@@Z 00000001800c1670     hb-ot-layout.obj
 0002:00036684       $chain$1$??$dispatch@Uhb_accelerate_subtables_context_t@OT@@$$V@ChainContext@OT@@QEBA?AUhb_empty_t@@PEAUhb_accelerate_subtables_context_t@1@@Z 00000001800c1684     hb-ot-layout.obj
 0002:00036694       $unwind$?kern@?$hb_kern_machine_t@U?$KernSubTableFormat3@UKernAATSubTableHeader@OT@@@OT@@@OT@@QEBAXPEAUhb_font_t@@PEAUhb_buffer_t@@I_N@Z 00000001800c1694     hb-ot-layout.obj
 0002:000366a8       $chain$0$?kern@?$hb_kern_machine_t@U?$KernSubTableFormat3@UKernAATSubTableHeader@OT@@@OT@@@OT@@QEBAXPEAUhb_font_t@@PEAUhb_buffer_t@@I_N@Z 00000001800c16a8     hb-ot-layout.obj
 0002:000366bc       $chain$2$?kern@?$hb_kern_machine_t@U?$KernSubTableFormat3@UKernAATSubTableHeader@OT@@@OT@@@OT@@QEBAXPEAUhb_font_t@@PEAUhb_buffer_t@@I_N@Z 00000001800c16bc     hb-ot-layout.obj
 0002:000366d4       $chain$3$?kern@?$hb_kern_machine_t@U?$KernSubTableFormat3@UKernAATSubTableHeader@OT@@@OT@@@OT@@QEBAXPEAUhb_font_t@@PEAUhb_buffer_t@@I_N@Z 00000001800c16d4     hb-ot-layout.obj
 0002:000366e4       $chain$4$?kern@?$hb_kern_machine_t@U?$KernSubTableFormat3@UKernAATSubTableHeader@OT@@@OT@@@OT@@QEBAXPEAUhb_font_t@@PEAUhb_buffer_t@@I_N@Z 00000001800c16e4     hb-ot-layout.obj
 0002:000366f4       $chain$1$?kern@?$hb_kern_machine_t@Uaccelerator_t@?$KerxSubTableFormat2@UKernAATSubTableHeader@OT@@@AAT@@@OT@@QEBAXPEAUhb_font_t@@PEAUhb_buffer_t@@I_N@Z 00000001800c16f4     hb-ot-layout.obj
 0002:0003670c       $chain$3$?kern@?$hb_kern_machine_t@Uaccelerator_t@?$KerxSubTableFormat2@UKernAATSubTableHeader@OT@@@AAT@@@OT@@QEBAXPEAUhb_font_t@@PEAUhb_buffer_t@@I_N@Z 00000001800c170c     hb-ot-layout.obj
 0002:00036724       $chain$4$?kern@?$hb_kern_machine_t@Uaccelerator_t@?$KerxSubTableFormat2@UKernAATSubTableHeader@OT@@@AAT@@@OT@@QEBAXPEAUhb_font_t@@PEAUhb_buffer_t@@I_N@Z 00000001800c1724     hb-ot-layout.obj
 0002:00036734       $chain$5$?kern@?$hb_kern_machine_t@Uaccelerator_t@?$KerxSubTableFormat2@UKernAATSubTableHeader@OT@@@AAT@@@OT@@QEBAXPEAUhb_font_t@@PEAUhb_buffer_t@@I_N@Z 00000001800c1734     hb-ot-layout.obj
 0002:00036744       $unwind$?transition@driver_context_t@?$KerxSubTableFormat1@UKernAATSubTableHeader@OT@@@AAT@@QEAAXPEAU?$StateTableDriver@UObsoleteTypes@AAT@@X@3@AEBU?$Entry@X@3@@Z 00000001800c1744     hb-ot-layout.obj
 0002:00036750       $chain$2$?transition@driver_context_t@?$KerxSubTableFormat1@UKernAATSubTableHeader@OT@@@AAT@@QEAAXPEAU?$StateTableDriver@UObsoleteTypes@AAT@@X@3@AEBU?$Entry@X@3@@Z 00000001800c1750     hb-ot-layout.obj
 0002:0003676c       $chain$3$?transition@driver_context_t@?$KerxSubTableFormat1@UKernAATSubTableHeader@OT@@@AAT@@QEAAXPEAU?$StateTableDriver@UObsoleteTypes@AAT@@X@3@AEBU?$Entry@X@3@@Z 00000001800c176c     hb-ot-layout.obj
 0002:0003677c       $chain$3$??$drive@Udriver_context_t@?$KerxSubTableFormat1@UKernAATSubTableHeader@OT@@@AAT@@@?$StateTableDriver@UObsoleteTypes@AAT@@X@AAT@@QEAAXPEAUdriver_context_t@?$KerxSubTableFormat1@UKernAATSubTableHeader@OT@@@1@PEAUhb_aat_apply_context_t@1@@Z 00000001800c177c     hb-ot-layout.obj
 0002:0003679c       $chain$4$??$drive@Udriver_context_t@?$KerxSubTableFormat1@UKernAATSubTableHeader@OT@@@AAT@@@?$StateTableDriver@UObsoleteTypes@AAT@@X@AAT@@QEAAXPEAUdriver_context_t@?$KerxSubTableFormat1@UKernAATSubTableHeader@OT@@@1@PEAUhb_aat_apply_context_t@1@@Z 00000001800c179c     hb-ot-layout.obj
 0002:000367ac       $chain$1$?kern@?$hb_kern_machine_t@Uaccelerator_t@?$KerxSubTableFormat0@UKernAATSubTableHeader@OT@@@AAT@@@OT@@QEBAXPEAUhb_font_t@@PEAUhb_buffer_t@@I_N@Z 00000001800c17ac     hb-ot-layout.obj
 0002:000367c4       $chain$3$?kern@?$hb_kern_machine_t@Uaccelerator_t@?$KerxSubTableFormat0@UKernAATSubTableHeader@OT@@@AAT@@@OT@@QEBAXPEAUhb_font_t@@PEAUhb_buffer_t@@I_N@Z 00000001800c17c4     hb-ot-layout.obj
 0002:000367dc       $chain$4$?kern@?$hb_kern_machine_t@Uaccelerator_t@?$KerxSubTableFormat0@UKernAATSubTableHeader@OT@@@AAT@@@OT@@QEBAXPEAUhb_font_t@@PEAUhb_buffer_t@@I_N@Z 00000001800c17dc     hb-ot-layout.obj
 0002:000367ec       $chain$5$?kern@?$hb_kern_machine_t@Uaccelerator_t@?$KerxSubTableFormat0@UKernAATSubTableHeader@OT@@@AAT@@@OT@@QEBAXPEAUhb_font_t@@PEAUhb_buffer_t@@I_N@Z 00000001800c17ec     hb-ot-layout.obj
 0002:000367fc       $chain$1$?kern@?$hb_kern_machine_t@Uaccelerator_t@?$KerxSubTableFormat2@UKernOTSubTableHeader@OT@@@AAT@@@OT@@QEBAXPEAUhb_font_t@@PEAUhb_buffer_t@@I_N@Z 00000001800c17fc     hb-ot-layout.obj
 0002:00036814       $chain$3$?kern@?$hb_kern_machine_t@Uaccelerator_t@?$KerxSubTableFormat2@UKernOTSubTableHeader@OT@@@AAT@@@OT@@QEBAXPEAUhb_font_t@@PEAUhb_buffer_t@@I_N@Z 00000001800c1814     hb-ot-layout.obj
 0002:0003682c       $chain$4$?kern@?$hb_kern_machine_t@Uaccelerator_t@?$KerxSubTableFormat2@UKernOTSubTableHeader@OT@@@AAT@@@OT@@QEBAXPEAUhb_font_t@@PEAUhb_buffer_t@@I_N@Z 00000001800c182c     hb-ot-layout.obj
 0002:0003683c       $chain$5$?kern@?$hb_kern_machine_t@Uaccelerator_t@?$KerxSubTableFormat2@UKernOTSubTableHeader@OT@@@AAT@@@OT@@QEBAXPEAUhb_font_t@@PEAUhb_buffer_t@@I_N@Z 00000001800c183c     hb-ot-layout.obj
 0002:0003684c       $chain$1$?kern@?$hb_kern_machine_t@Uaccelerator_t@?$KerxSubTableFormat0@UKernOTSubTableHeader@OT@@@AAT@@@OT@@QEBAXPEAUhb_font_t@@PEAUhb_buffer_t@@I_N@Z 00000001800c184c     hb-ot-layout.obj
 0002:00036864       $chain$3$?kern@?$hb_kern_machine_t@Uaccelerator_t@?$KerxSubTableFormat0@UKernOTSubTableHeader@OT@@@AAT@@@OT@@QEBAXPEAUhb_font_t@@PEAUhb_buffer_t@@I_N@Z 00000001800c1864     hb-ot-layout.obj
 0002:0003687c       $chain$4$?kern@?$hb_kern_machine_t@Uaccelerator_t@?$KerxSubTableFormat0@UKernOTSubTableHeader@OT@@@AAT@@@OT@@QEBAXPEAUhb_font_t@@PEAUhb_buffer_t@@I_N@Z 00000001800c187c     hb-ot-layout.obj
 0002:0003688c       $chain$5$?kern@?$hb_kern_machine_t@Uaccelerator_t@?$KerxSubTableFormat0@UKernOTSubTableHeader@OT@@@AAT@@@OT@@QEBAXPEAUhb_font_t@@PEAUhb_buffer_t@@I_N@Z 00000001800c188c     hb-ot-layout.obj
 0002:0003689c       $unwind$??$dispatch@Uhb_sanitize_context_t@@$$V@PosLookupSubTable@GPOS_impl@Layout@OT@@QEBA_NPEAUhb_sanitize_context_t@@I@Z 00000001800c189c     hb-ot-layout.obj
 0002:000368a8       $chain$3$??$dispatch@Uhb_sanitize_context_t@@$$V@PosLookupSubTable@GPOS_impl@Layout@OT@@QEBA_NPEAUhb_sanitize_context_t@@I@Z 00000001800c18a8     hb-ot-layout.obj
 0002:000368c8       $chain$4$??$dispatch@Uhb_sanitize_context_t@@$$V@PosLookupSubTable@GPOS_impl@Layout@OT@@QEBA_NPEAUhb_sanitize_context_t@@I@Z 00000001800c18c8     hb-ot-layout.obj
 0002:000368d8       $unwind$??$dispatch@Uhb_sanitize_context_t@@$$V@SubstLookupSubTable@GSUB_impl@Layout@OT@@QEBA_NPEAUhb_sanitize_context_t@@I@Z 00000001800c18d8     hb-ot-layout.obj
 0002:000368ec       $chain$0$??$dispatch@Uhb_sanitize_context_t@@$$V@SubstLookupSubTable@GSUB_impl@Layout@OT@@QEBA_NPEAUhb_sanitize_context_t@@I@Z 00000001800c18ec     hb-ot-layout.obj
 0002:00036900       $chain$2$??$dispatch@Uhb_sanitize_context_t@@$$V@SubstLookupSubTable@GSUB_impl@Layout@OT@@QEBA_NPEAUhb_sanitize_context_t@@I@Z 00000001800c1900     hb-ot-layout.obj
 0002:00036900       $chain$4$??$dispatch@Uhb_sanitize_context_t@@$$V@SubstLookupSubTable@GSUB_impl@Layout@OT@@QEBA_NPEAUhb_sanitize_context_t@@I@Z 00000001800c1900     hb-ot-layout.obj
 0002:00036914       $chain$5$??$dispatch@Uhb_sanitize_context_t@@$$V@SubstLookupSubTable@GSUB_impl@Layout@OT@@QEBA_NPEAUhb_sanitize_context_t@@I@Z 00000001800c1914     hb-ot-layout.obj
 0002:00036924       $unwind$??$dispatch@U?$ChainContextFormat2_5@USmallTypes@Layout@OT@@@OT@@@hb_accelerate_subtables_context_t@OT@@QEAA?AUhb_empty_t@@AEBU?$ChainContextFormat2_5@USmallTypes@Layout@OT@@@1@@Z 00000001800c1924     hb-ot-layout.obj
 0002:00036924       $unwind$??$dispatch@U?$ContextFormat2_5@USmallTypes@Layout@OT@@@OT@@@hb_accelerate_subtables_context_t@OT@@QEAA?AUhb_empty_t@@AEBU?$ContextFormat2_5@USmallTypes@Layout@OT@@@1@@Z 00000001800c1924     hb-ot-layout.obj
 0002:00036940       $chain$1$??$collect_coverage@U?$hb_set_digest_combiner_t@U?$hb_set_digest_bits_pattern_t@K$03@@U?$hb_set_digest_combiner_t@U?$hb_set_digest_bits_pattern_t@K$0A@@@U?$hb_set_digest_bits_pattern_t@K$08@@@@@@@Coverage@Common@Layout@OT@@QEBA_NPEAU?$hb_set_digest_combiner_t@U?$hb_set_digest_bits_pattern_t@K$03@@U?$hb_set_digest_combiner_t@U?$hb_set_digest_bits_pattern_t@K$0A@@@U?$hb_set_digest_bits_pattern_t@K$08@@@@@@@Z 00000001800c1940     hb-ot-layout.obj
 0002:00036958       $chain$2$??$collect_coverage@U?$hb_set_digest_combiner_t@U?$hb_set_digest_bits_pattern_t@K$03@@U?$hb_set_digest_combiner_t@U?$hb_set_digest_bits_pattern_t@K$0A@@@U?$hb_set_digest_bits_pattern_t@K$08@@@@@@@Coverage@Common@Layout@OT@@QEBA_NPEAU?$hb_set_digest_combiner_t@U?$hb_set_digest_bits_pattern_t@K$03@@U?$hb_set_digest_combiner_t@U?$hb_set_digest_bits_pattern_t@K$0A@@@U?$hb_set_digest_bits_pattern_t@K$08@@@@@@@Z 00000001800c1958     hb-ot-layout.obj
 0002:0003696c       $chain$3$??$collect_coverage@U?$hb_set_digest_combiner_t@U?$hb_set_digest_bits_pattern_t@K$03@@U?$hb_set_digest_combiner_t@U?$hb_set_digest_bits_pattern_t@K$0A@@@U?$hb_set_digest_bits_pattern_t@K$08@@@@@@@Coverage@Common@Layout@OT@@QEBA_NPEAU?$hb_set_digest_combiner_t@U?$hb_set_digest_bits_pattern_t@K$03@@U?$hb_set_digest_combiner_t@U?$hb_set_digest_bits_pattern_t@K$0A@@@U?$hb_set_digest_bits_pattern_t@K$08@@@@@@@Z 00000001800c196c     hb-ot-layout.obj
 0002:0003697c       $chain$4$??$collect_coverage@U?$hb_set_digest_combiner_t@U?$hb_set_digest_bits_pattern_t@K$03@@U?$hb_set_digest_combiner_t@U?$hb_set_digest_bits_pattern_t@K$0A@@@U?$hb_set_digest_bits_pattern_t@K$08@@@@@@@Coverage@Common@Layout@OT@@QEBA_NPEAU?$hb_set_digest_combiner_t@U?$hb_set_digest_bits_pattern_t@K$03@@U?$hb_set_digest_combiner_t@U?$hb_set_digest_bits_pattern_t@K$0A@@@U?$hb_set_digest_bits_pattern_t@K$08@@@@@@@Z 00000001800c197c     hb-ot-layout.obj
 0002:0003698c       $unwind$??$dispatch@Uhb_sanitize_context_t@@$$V@Context@OT@@QEBA_NPEAUhb_sanitize_context_t@@@Z 00000001800c198c     hb-ot-layout.obj
 0002:000369a4       $chain$3$??$dispatch@Uhb_sanitize_context_t@@$$V@Context@OT@@QEBA_NPEAUhb_sanitize_context_t@@@Z 00000001800c19a4     hb-ot-layout.obj
 0002:000369b8       $chain$5$??$dispatch@Uhb_sanitize_context_t@@$$V@Context@OT@@QEBA_NPEAUhb_sanitize_context_t@@@Z 00000001800c19b8     hb-ot-layout.obj
 0002:000369cc       $chain$6$??$dispatch@Uhb_sanitize_context_t@@$$V@Context@OT@@QEBA_NPEAUhb_sanitize_context_t@@@Z 00000001800c19cc     hb-ot-layout.obj
 0002:000369dc       $unwind$??$dispatch@Uhb_sanitize_context_t@@$$V@ChainContext@OT@@QEBA_NPEAUhb_sanitize_context_t@@@Z 00000001800c19dc     hb-ot-layout.obj
 0002:000369f4       $unwind$??$dispatch@Uhb_sanitize_context_t@@$$V@AlternateSubst@GSUB_impl@Layout@OT@@QEBA_NPEAUhb_sanitize_context_t@@@Z 00000001800c19f4     hb-ot-layout.obj
 0002:000369f4       $unwind$??$dispatch@Uhb_sanitize_context_t@@$$V@MultipleSubst@GSUB_impl@Layout@OT@@QEBA_NPEAUhb_sanitize_context_t@@@Z 00000001800c19f4     hb-ot-layout.obj
 0002:00036a18       $unwind$??$sanitize@I@?$OffsetTo@UAnchorMatrix@GPOS_impl@Layout@OT@@U?$IntType@G$01@4@$00@OT@@QEBA_NPEAUhb_sanitize_context_t@@PEBX$$QEAI@Z 00000001800c1a18     hb-ot-layout.obj
 0002:00036a34       $unwind$??$sanitize@PEAUsanitize_closure_t@?$PairSet@USmallTypes@Layout@OT@@@GPOS_impl@Layout@OT@@@?$OffsetTo@U?$PairSet@USmallTypes@Layout@OT@@@GPOS_impl@Layout@OT@@U?$IntType@G$01@4@$00@OT@@QEBA_NPEAUhb_sanitize_context_t@@PEBX$$QEAPEAUsanitize_closure_t@?$PairSet@USmallTypes@Layout@OT@@@GPOS_impl@Layout@1@@Z 00000001800c1a34     hb-ot-layout.obj
 0002:00036a48       $chain$0$??$sanitize@PEAUsanitize_closure_t@?$PairSet@USmallTypes@Layout@OT@@@GPOS_impl@Layout@OT@@@?$OffsetTo@U?$PairSet@USmallTypes@Layout@OT@@@GPOS_impl@Layout@OT@@U?$IntType@G$01@4@$00@OT@@QEBA_NPEAUhb_sanitize_context_t@@PEBX$$QEAPEAUsanitize_closure_t@?$PairSet@USmallTypes@Layout@OT@@@GPOS_impl@Layout@1@@Z 00000001800c1a48     hb-ot-layout.obj
 0002:00036a5c       $chain$1$??$sanitize@PEAUsanitize_closure_t@?$PairSet@USmallTypes@Layout@OT@@@GPOS_impl@Layout@OT@@@?$OffsetTo@U?$PairSet@USmallTypes@Layout@OT@@@GPOS_impl@Layout@OT@@U?$IntType@G$01@4@$00@OT@@QEBA_NPEAUhb_sanitize_context_t@@PEBX$$QEAPEAUsanitize_closure_t@?$PairSet@USmallTypes@Layout@OT@@@GPOS_impl@Layout@1@@Z 00000001800c1a5c     hb-ot-layout.obj
 0002:00036a6c       $chain$0$??$_dispatch@U?$ChainRule@USmallTypes@Layout@OT@@@OT@@$$V@hb_sanitize_context_t@@AEAA_NAEBU?$ChainRule@USmallTypes@Layout@OT@@@OT@@U?$hb_priority@$00@@@Z 00000001800c1a6c     hb-ot-layout.obj
 0002:00036a80       $chain$2$??$_dispatch@U?$ChainRule@USmallTypes@Layout@OT@@@OT@@$$V@hb_sanitize_context_t@@AEAA_NAEBU?$ChainRule@USmallTypes@Layout@OT@@@OT@@U?$hb_priority@$00@@@Z 00000001800c1a80     hb-ot-layout.obj
 0002:00036a94       $chain$3$??$_dispatch@U?$ChainRule@USmallTypes@Layout@OT@@@OT@@$$V@hb_sanitize_context_t@@AEAA_NAEBU?$ChainRule@USmallTypes@Layout@OT@@@OT@@U?$hb_priority@$00@@@Z 00000001800c1a94     hb-ot-layout.obj
 0002:00036aa4       $unwind$??0hb_ot_map_builder_t@@QEAA@PEAUhb_face_t@@AEBUhb_segment_properties_t@@@Z 00000001800c1aa4     hb-ot-map.obj
 0002:00036ab8       $unwind$?add_feature@hb_ot_map_builder_t@@QEAAXIW4hb_ot_map_feature_flags_t@@I@Z 00000001800c1ab8     hb-ot-map.obj
 0002:00036ac8       $chain$3$?add_feature@hb_ot_map_builder_t@@QEAAXIW4hb_ot_map_feature_flags_t@@I@Z 00000001800c1ac8     hb-ot-map.obj
 0002:00036ae8       $chain$4$?add_feature@hb_ot_map_builder_t@@QEAAXIW4hb_ot_map_feature_flags_t@@I@Z 00000001800c1ae8     hb-ot-map.obj
 0002:00036af8       $unwind$?compile@hb_ot_map_builder_t@@QEAAXAEAUhb_ot_map_t@@AEBUhb_ot_shape_plan_key_t@@@Z 00000001800c1af8     hb-ot-map.obj
 0002:00036b14       $unwind$?add_lookups@hb_ot_map_builder_t@@AEAAXAEAUhb_ot_map_t@@IIII_N111I@Z 00000001800c1b14     hb-ot-map.obj
 0002:00036b34       $chain$0$?alloc@?$hb_vector_t@Ufeature_info_t@hb_ot_map_builder_t@@$0A@@@QEAA_NI_N@Z 00000001800c1b34     hb-ot-map.obj
 0002:00036b48       $chain$2$?alloc@?$hb_vector_t@Ufeature_info_t@hb_ot_map_builder_t@@$0A@@@QEAA_NI_N@Z 00000001800c1b48     hb-ot-map.obj
 0002:00036b48       $chain$4$?alloc@?$hb_vector_t@Ufeature_info_t@hb_ot_map_builder_t@@$0A@@@QEAA_NI_N@Z 00000001800c1b48     hb-ot-map.obj
 0002:00036b5c       $chain$0$?get@?$hb_lazy_loader_t@UMVAR@OT@@U?$hb_table_lazy_loader_t@UMVAR@OT@@$0BG@$00@@Uhb_face_t@@$0BG@Uhb_blob_t@@@@QEBAPEBUMVAR@OT@@XZ 00000001800c1b5c     hb-ot-metrics.obj
 0002:00036b70       $chain$1$?get@?$hb_lazy_loader_t@UMVAR@OT@@U?$hb_table_lazy_loader_t@UMVAR@OT@@$0BG@$00@@Uhb_face_t@@$0BG@Uhb_blob_t@@@@QEBAPEBUMVAR@OT@@XZ 00000001800c1b70     hb-ot-metrics.obj
 0002:00036b80       $unwind$??$sanitize_blob@UMVAR@OT@@@hb_sanitize_context_t@@QEAAPEAUhb_blob_t@@PEAU1@@Z 00000001800c1b80     hb-ot-metrics.obj
 0002:00036b9c       $unwind$?_hb_ot_shape_fallback_mark_position@@YAXPEBUhb_ot_shape_plan_t@@PEAUhb_font_t@@PEAUhb_buffer_t@@_N@Z 00000001800c1b9c     hb-ot-shape-fallback.obj
 0002:00036bac       $chain$0$?_hb_ot_shape_fallback_mark_position@@YAXPEBUhb_ot_shape_plan_t@@PEAUhb_font_t@@PEAUhb_buffer_t@@_N@Z 00000001800c1bac     hb-ot-shape-fallback.obj
 0002:00036bc0       $chain$3$?_hb_ot_shape_fallback_mark_position@@YAXPEBUhb_ot_shape_plan_t@@PEAUhb_font_t@@PEAUhb_buffer_t@@_N@Z 00000001800c1bc0     hb-ot-shape-fallback.obj
 0002:00036bdc       $chain$4$?_hb_ot_shape_fallback_mark_position@@YAXPEBUhb_ot_shape_plan_t@@PEAUhb_font_t@@PEAUhb_buffer_t@@_N@Z 00000001800c1bdc     hb-ot-shape-fallback.obj
 0002:00036bec       $chain$5$?_hb_ot_shape_fallback_mark_position@@YAXPEBUhb_ot_shape_plan_t@@PEAUhb_font_t@@PEAUhb_buffer_t@@_N@Z 00000001800c1bec     hb-ot-shape-fallback.obj
 0002:00036bfc       $chain$2$?_hb_ot_shape_fallback_mark_position_recategorize_marks@@YAXPEBUhb_ot_shape_plan_t@@PEAUhb_font_t@@PEAUhb_buffer_t@@@Z 00000001800c1bfc     hb-ot-shape-fallback.obj
 0002:00036c18       $chain$3$?_hb_ot_shape_fallback_mark_position_recategorize_marks@@YAXPEBUhb_ot_shape_plan_t@@PEAUhb_font_t@@PEAUhb_buffer_t@@@Z 00000001800c1c18     hb-ot-shape-fallback.obj
 0002:00036c28       $unwind$?_hb_ot_shape_fallback_kern@@YAXPEBUhb_ot_shape_plan_t@@PEAUhb_font_t@@PEAUhb_buffer_t@@@Z 00000001800c1c28     hb-ot-shape-fallback.obj
 0002:00036c38       $chain$0$?_hb_ot_shape_fallback_kern@@YAXPEBUhb_ot_shape_plan_t@@PEAUhb_font_t@@PEAUhb_buffer_t@@@Z 00000001800c1c38     hb-ot-shape-fallback.obj
 0002:00036c4c       $chain$1$?_hb_ot_shape_fallback_kern@@YAXPEBUhb_ot_shape_plan_t@@PEAUhb_font_t@@PEAUhb_buffer_t@@@Z 00000001800c1c4c     hb-ot-shape-fallback.obj
 0002:00036c5c       $unwind$?_hb_ot_shape_fallback_spaces@@YAXPEBUhb_ot_shape_plan_t@@PEAUhb_font_t@@PEAUhb_buffer_t@@@Z 00000001800c1c5c     hb-ot-shape-fallback.obj
 0002:00036c68       $chain$4$?_hb_ot_shape_fallback_spaces@@YAXPEBUhb_ot_shape_plan_t@@PEAUhb_font_t@@PEAUhb_buffer_t@@@Z 00000001800c1c68     hb-ot-shape-fallback.obj
 0002:00036c8c       $chain$5$?_hb_ot_shape_fallback_spaces@@YAXPEBUhb_ot_shape_plan_t@@PEAUhb_font_t@@PEAUhb_buffer_t@@@Z 00000001800c1c8c     hb-ot-shape-fallback.obj
 0002:00036c9c       $chain$6$?_hb_ot_shape_fallback_spaces@@YAXPEBUhb_ot_shape_plan_t@@PEAUhb_font_t@@PEAUhb_buffer_t@@@Z 00000001800c1c9c     hb-ot-shape-fallback.obj
 0002:00036cc0       $unwind$?position_mark@@YAXPEBUhb_ot_shape_plan_t@@PEAUhb_font_t@@PEAUhb_buffer_t@@AEAUhb_glyph_extents_t@@II@Z 00000001800c1cc0     hb-ot-shape-fallback.obj
 0002:00036cc0       $unwind$?consonant_position_from_face@@YA?AW4ot_position_t@@PEBUindic_shape_plan_t@@IIPEAUhb_face_t@@@Z 00000001800c1cc0     hb-ot-shaper-indic.obj
 0002:00036cd8       $unwind$?position_around_base@@YAXPEBUhb_ot_shape_plan_t@@PEAUhb_font_t@@PEAUhb_buffer_t@@II_N@Z 00000001800c1cd8     hb-ot-shape-fallback.obj
 0002:00036cf8       $chain$2$?position_around_base@@YAXPEBUhb_ot_shape_plan_t@@PEAUhb_font_t@@PEAUhb_buffer_t@@II_N@Z 00000001800c1cf8     hb-ot-shape-fallback.obj
 0002:00036d14       $chain$3$?position_around_base@@YAXPEBUhb_ot_shape_plan_t@@PEAUhb_font_t@@PEAUhb_buffer_t@@II_N@Z 00000001800c1d14     hb-ot-shape-fallback.obj
 0002:00036d24       $unwind$?position_cluster@@YAXPEBUhb_ot_shape_plan_t@@PEAUhb_font_t@@PEAUhb_buffer_t@@II_N@Z 00000001800c1d24     hb-ot-shape-fallback.obj
 0002:00036d34       $chain$0$?position_cluster@@YAXPEBUhb_ot_shape_plan_t@@PEAUhb_font_t@@PEAUhb_buffer_t@@II_N@Z 00000001800c1d34     hb-ot-shape-fallback.obj
 0002:00036d48       $chain$2$?position_cluster@@YAXPEBUhb_ot_shape_plan_t@@PEAUhb_font_t@@PEAUhb_buffer_t@@II_N@Z 00000001800c1d48     hb-ot-shape-fallback.obj
 0002:00036d60       $chain$3$?position_cluster@@YAXPEBUhb_ot_shape_plan_t@@PEAUhb_font_t@@PEAUhb_buffer_t@@II_N@Z 00000001800c1d60     hb-ot-shape-fallback.obj
 0002:00036d70       $chain$4$?position_cluster@@YAXPEBUhb_ot_shape_plan_t@@PEAUhb_font_t@@PEAUhb_buffer_t@@II_N@Z 00000001800c1d70     hb-ot-shape-fallback.obj
 0002:00036d80       $unwind$?kern@?$hb_kern_machine_t@Uhb_ot_shape_fallback_kern_driver_t@@@OT@@QEBAXPEAUhb_font_t@@PEAUhb_buffer_t@@I_N@Z 00000001800c1d80     hb-ot-shape-fallback.obj
 0002:00036d90       $chain$1$?kern@?$hb_kern_machine_t@Uhb_ot_shape_fallback_kern_driver_t@@@OT@@QEBAXPEAUhb_font_t@@PEAUhb_buffer_t@@I_N@Z 00000001800c1d90     hb-ot-shape-fallback.obj
 0002:00036da8       $chain$3$?kern@?$hb_kern_machine_t@Uhb_ot_shape_fallback_kern_driver_t@@@OT@@QEBAXPEAUhb_font_t@@PEAUhb_buffer_t@@I_N@Z 00000001800c1da8     hb-ot-shape-fallback.obj
 0002:00036dc0       $chain$4$?kern@?$hb_kern_machine_t@Uhb_ot_shape_fallback_kern_driver_t@@@OT@@QEBAXPEAUhb_font_t@@PEAUhb_buffer_t@@I_N@Z 00000001800c1dc0     hb-ot-shape-fallback.obj
 0002:00036dd0       $chain$5$?kern@?$hb_kern_machine_t@Uhb_ot_shape_fallback_kern_driver_t@@@OT@@QEBAXPEAUhb_font_t@@PEAUhb_buffer_t@@I_N@Z 00000001800c1dd0     hb-ot-shape-fallback.obj
 0002:00036de0       $unwind$?_hb_ot_shape_normalize@@YAXPEBUhb_ot_shape_plan_t@@PEAUhb_buffer_t@@PEAUhb_font_t@@@Z 00000001800c1de0     hb-ot-shape-normalize.obj
 0002:00036df0       $chain$4$?_hb_ot_shape_normalize@@YAXPEBUhb_ot_shape_plan_t@@PEAUhb_buffer_t@@PEAUhb_font_t@@@Z 00000001800c1df0     hb-ot-shape-normalize.obj
 0002:00036e14       $chain$5$?_hb_ot_shape_normalize@@YAXPEBUhb_ot_shape_plan_t@@PEAUhb_buffer_t@@PEAUhb_font_t@@@Z 00000001800c1e14     hb-ot-shape-normalize.obj
 0002:00036e24       $unwind$?decompose@@YAIPEBUhb_ot_shape_normalize_context_t@@_NI@Z 00000001800c1e24     hb-ot-shape-normalize.obj
 0002:00036e38       $unwind$?decompose_current_character@@YAXPEBUhb_ot_shape_normalize_context_t@@_N@Z 00000001800c1e38     hb-ot-shape-normalize.obj
 0002:00036e50       $unwind$?handle_variation_selector_cluster@@YAXPEBUhb_ot_shape_normalize_context_t@@I_N@Z 00000001800c1e50     hb-ot-shape-normalize.obj
 0002:00036e5c       $chain$1$?handle_variation_selector_cluster@@YAXPEBUhb_ot_shape_normalize_context_t@@I_N@Z 00000001800c1e5c     hb-ot-shape-normalize.obj
 0002:00036e74       $chain$3$?handle_variation_selector_cluster@@YAXPEBUhb_ot_shape_normalize_context_t@@I_N@Z 00000001800c1e74     hb-ot-shape-normalize.obj
 0002:00036e8c       $chain$4$?handle_variation_selector_cluster@@YAXPEBUhb_ot_shape_normalize_context_t@@I_N@Z 00000001800c1e8c     hb-ot-shape-normalize.obj
 0002:00036e9c       $chain$5$?handle_variation_selector_cluster@@YAXPEBUhb_ot_shape_normalize_context_t@@I_N@Z 00000001800c1e9c     hb-ot-shape-normalize.obj
 0002:00036eac       $unwind$?init0@hb_ot_shape_plan_t@@QEAA_NPEAUhb_face_t@@PEBUhb_shape_plan_key_t@@@Z 00000001800c1eac     hb-ot-shape.obj
 0002:00036ec8       $unwind$?compile@hb_ot_shape_planner_t@@QEAAXAEAUhb_ot_shape_plan_t@@AEBUhb_ot_shape_plan_key_t@@@Z 00000001800c1ec8     hb-ot-shape.obj
 0002:00036ed4       $chain$0$?compile@hb_ot_shape_planner_t@@QEAAXAEAUhb_ot_shape_plan_t@@AEBUhb_ot_shape_plan_key_t@@@Z 00000001800c1ed4     hb-ot-shape.obj
 0002:00036ee8       $chain$3$?compile@hb_ot_shape_planner_t@@QEAAXAEAUhb_ot_shape_plan_t@@AEBUhb_ot_shape_plan_key_t@@@Z 00000001800c1ee8     hb-ot-shape.obj
 0002:00036f04       $chain$4$?compile@hb_ot_shape_planner_t@@QEAAXAEAUhb_ot_shape_plan_t@@AEBUhb_ot_shape_plan_key_t@@@Z 00000001800c1f04     hb-ot-shape.obj
 0002:00036f18       $chain$5$?compile@hb_ot_shape_planner_t@@QEAAXAEAUhb_ot_shape_plan_t@@AEBUhb_ot_shape_plan_key_t@@@Z 00000001800c1f18     hb-ot-shape.obj
 0002:00036f28       $chain$6$?compile@hb_ot_shape_planner_t@@QEAAXAEAUhb_ot_shape_plan_t@@AEBUhb_ot_shape_plan_key_t@@@Z 00000001800c1f28     hb-ot-shape.obj
 0002:00036f3c       $chain$7$?compile@hb_ot_shape_planner_t@@QEAAXAEAUhb_ot_shape_plan_t@@AEBUhb_ot_shape_plan_key_t@@@Z 00000001800c1f3c     hb-ot-shape.obj
 0002:00036f58       $chain$8$?compile@hb_ot_shape_planner_t@@QEAAXAEAUhb_ot_shape_plan_t@@AEBUhb_ot_shape_plan_key_t@@@Z 00000001800c1f58     hb-ot-shape.obj
 0002:00036f74       $chain$9$?compile@hb_ot_shape_planner_t@@QEAAXAEAUhb_ot_shape_plan_t@@AEBUhb_ot_shape_plan_key_t@@@Z 00000001800c1f74     hb-ot-shape.obj
 0002:00036f88       $chain$10$?compile@hb_ot_shape_planner_t@@QEAAXAEAUhb_ot_shape_plan_t@@AEBUhb_ot_shape_plan_key_t@@@Z 00000001800c1f88     hb-ot-shape.obj
 0002:00036f98       $unwind$?hb_ot_shape_collect_features@@YAXPEAUhb_ot_shape_planner_t@@PEBUhb_feature_t@@I@Z 00000001800c1f98     hb-ot-shape.obj
 0002:00036fb4       $unwind$?hb_set_unicode_props@@YAXPEAUhb_buffer_t@@@Z 00000001800c1fb4     hb-ot-shape.obj
 0002:00036fc4       $chain$3$?hb_set_unicode_props@@YAXPEAUhb_buffer_t@@@Z 00000001800c1fc4     hb-ot-shape.obj
 0002:00036fe4       $chain$4$?hb_set_unicode_props@@YAXPEAUhb_buffer_t@@@Z 00000001800c1fe4     hb-ot-shape.obj
 0002:00036ff4       $unwind$?hb_form_clusters@@YAXPEAUhb_buffer_t@@@Z 00000001800c1ff4     hb-ot-shape.obj
 0002:00036ff4       $unwind$?hb_ot_substitute_default@@YAXPEBUhb_ot_shape_context_t@@@Z 00000001800c1ff4     hb-ot-shape.obj
 0002:00036ffc       $chain$2$?hb_form_clusters@@YAXPEAUhb_buffer_t@@@Z 00000001800c1ffc     hb-ot-shape.obj
 0002:00037018       $chain$3$?hb_form_clusters@@YAXPEAUhb_buffer_t@@@Z 00000001800c2018     hb-ot-shape.obj
 0002:0003702c       $chain$4$?hb_form_clusters@@YAXPEAUhb_buffer_t@@@Z 00000001800c202c     hb-ot-shape.obj
 0002:00037040       $chain$5$?hb_form_clusters@@YAXPEAUhb_buffer_t@@@Z 00000001800c2040     hb-ot-shape.obj
 0002:00037050       $chain$6$?hb_form_clusters@@YAXPEAUhb_buffer_t@@@Z 00000001800c2050     hb-ot-shape.obj
 0002:00037060       $chain$7$?hb_form_clusters@@YAXPEAUhb_buffer_t@@@Z 00000001800c2060     hb-ot-shape.obj
 0002:00037070       $unwind$?hb_ot_rotate_chars@@YAXPEBUhb_ot_shape_context_t@@@Z 00000001800c2070     hb-ot-shape.obj
 0002:00037084       $chain$0$?hb_ot_rotate_chars@@YAXPEBUhb_ot_shape_context_t@@@Z 00000001800c2084     hb-ot-shape.obj
 0002:00037098       $chain$1$?hb_ot_rotate_chars@@YAXPEBUhb_ot_shape_context_t@@@Z 00000001800c2098     hb-ot-shape.obj
 0002:000370ac       $chain$2$?hb_ot_rotate_chars@@YAXPEBUhb_ot_shape_context_t@@@Z 00000001800c20ac     hb-ot-shape.obj
 0002:000370bc       $chain$3$?hb_ot_rotate_chars@@YAXPEBUhb_ot_shape_context_t@@@Z 00000001800c20bc     hb-ot-shape.obj
 0002:000370cc       $unwind$?hb_ot_shape_setup_masks_fraction@@YAXPEBUhb_ot_shape_context_t@@@Z 00000001800c20cc     hb-ot-shape.obj
 0002:000370d4       $chain$4$?hb_ot_shape_setup_masks_fraction@@YAXPEBUhb_ot_shape_context_t@@@Z 00000001800c20d4     hb-ot-shape.obj
 0002:000370f8       $chain$7$?hb_ot_shape_setup_masks_fraction@@YAXPEBUhb_ot_shape_context_t@@@Z 00000001800c20f8     hb-ot-shape.obj
 0002:00037114       $chain$8$?hb_ot_shape_setup_masks_fraction@@YAXPEBUhb_ot_shape_context_t@@@Z 00000001800c2114     hb-ot-shape.obj
 0002:00037124       $chain$9$?hb_ot_shape_setup_masks_fraction@@YAXPEBUhb_ot_shape_context_t@@@Z 00000001800c2124     hb-ot-shape.obj
 0002:00037134       $chain$0$?hb_ot_substitute_default@@YAXPEBUhb_ot_shape_context_t@@@Z 00000001800c2134     hb-ot-shape.obj
 0002:00037148       $chain$3$?hb_ot_substitute_default@@YAXPEBUhb_ot_shape_context_t@@@Z 00000001800c2148     hb-ot-shape.obj
 0002:00037164       $chain$5$?hb_ot_substitute_default@@YAXPEBUhb_ot_shape_context_t@@@Z 00000001800c2164     hb-ot-shape.obj
 0002:0003717c       $chain$6$?hb_ot_substitute_default@@YAXPEBUhb_ot_shape_context_t@@@Z 00000001800c217c     hb-ot-shape.obj
 0002:0003718c       $chain$7$?hb_ot_substitute_default@@YAXPEBUhb_ot_shape_context_t@@@Z 00000001800c218c     hb-ot-shape.obj
 0002:0003719c       $chain$8$?hb_ot_substitute_default@@YAXPEBUhb_ot_shape_context_t@@@Z 00000001800c219c     hb-ot-shape.obj
 0002:000371ac       $chain$9$?hb_ot_substitute_default@@YAXPEBUhb_ot_shape_context_t@@@Z 00000001800c21ac     hb-ot-shape.obj
 0002:000371d4       $chain$0$?hb_ot_substitute_post@@YAXPEBUhb_ot_shape_context_t@@@Z 00000001800c21d4     hb-ot-shape.obj
 0002:000371e8       $chain$2$?hb_ot_substitute_post@@YAXPEBUhb_ot_shape_context_t@@@Z 00000001800c21e8     hb-ot-shape.obj
 0002:00037200       $chain$3$?hb_ot_substitute_post@@YAXPEBUhb_ot_shape_context_t@@@Z 00000001800c2200     hb-ot-shape.obj
 0002:00037210       $chain$4$?hb_ot_substitute_post@@YAXPEBUhb_ot_shape_context_t@@@Z 00000001800c2210     hb-ot-shape.obj
 0002:00037220       $unwind$?hb_ot_position_default@@YAXPEBUhb_ot_shape_context_t@@@Z 00000001800c2220     hb-ot-shape.obj
 0002:00037228       $chain$3$?hb_ot_position_default@@YAXPEBUhb_ot_shape_context_t@@@Z 00000001800c2228     hb-ot-shape.obj
 0002:00037248       $chain$4$?hb_ot_position_default@@YAXPEBUhb_ot_shape_context_t@@@Z 00000001800c2248     hb-ot-shape.obj
 0002:0003725c       $chain$5$?hb_ot_position_default@@YAXPEBUhb_ot_shape_context_t@@@Z 00000001800c225c     hb-ot-shape.obj
 0002:0003726c       $chain$6$?hb_ot_position_default@@YAXPEBUhb_ot_shape_context_t@@@Z 00000001800c226c     hb-ot-shape.obj
 0002:0003727c       $unwind$?hb_ot_position_plan@@YAXPEBUhb_ot_shape_context_t@@@Z 00000001800c227c     hb-ot-shape.obj
 0002:00037288       $chain$0$?hb_ot_position_plan@@YAXPEBUhb_ot_shape_context_t@@@Z 00000001800c2288     hb-ot-shape.obj
 0002:0003729c       $chain$5$?hb_ot_position_plan@@YAXPEBUhb_ot_shape_context_t@@@Z 00000001800c229c     hb-ot-shape.obj
 0002:000372c0       $chain$6$?hb_ot_position_plan@@YAXPEBUhb_ot_shape_context_t@@@Z 00000001800c22c0     hb-ot-shape.obj
 0002:000372e0       $chain$7$?hb_ot_position_plan@@YAXPEBUhb_ot_shape_context_t@@@Z 00000001800c22e0     hb-ot-shape.obj
 0002:000372f0       $unwind$?hb_propagate_flags@@YAXPEAUhb_buffer_t@@@Z 00000001800c22f0     hb-ot-shape.obj
 0002:000372f8       $chain$2$?hb_propagate_flags@@YAXPEAUhb_buffer_t@@@Z 00000001800c22f8     hb-ot-shape.obj
 0002:00037314       $chain$7$?hb_propagate_flags@@YAXPEAUhb_buffer_t@@@Z 00000001800c2314     hb-ot-shape.obj
 0002:00037338       $chain$8$?hb_propagate_flags@@YAXPEAUhb_buffer_t@@@Z 00000001800c2338     hb-ot-shape.obj
 0002:00037348       $chain$9$?hb_propagate_flags@@YAXPEAUhb_buffer_t@@@Z 00000001800c2348     hb-ot-shape.obj
 0002:00037358       $unwind$?hb_ot_shape_internal@@YAXPEAUhb_ot_shape_context_t@@@Z 00000001800c2358     hb-ot-shape.obj
 0002:00037370       $unwind$?safe_to_insert_tatweel@hb_buffer_t@@QEAAXII@Z 00000001800c2370     hb-ot-shaper-arabic.obj
 0002:00037380       $unwind$?discard_stale_objects@hb_serialize_context_t@@QEAAXXZ 00000001800c2380     hb-ot-shaper-arabic.obj
 0002:00037388       $chain$6$?discard_stale_objects@hb_serialize_context_t@@QEAAXXZ 00000001800c2388     hb-ot-shaper-arabic.obj
 0002:000373b4       $chain$7$?discard_stale_objects@hb_serialize_context_t@@QEAAXXZ 00000001800c23b4     hb-ot-shaper-arabic.obj
 0002:000373c4       $unwind$?data_create_arabic@@YAPEAXPEBUhb_ot_shape_plan_t@@@Z 00000001800c23c4     hb-ot-shaper-arabic.obj
 0002:000373e0       $unwind$?data_destroy_arabic@@YAXPEAX@Z 00000001800c23e0     hb-ot-shaper-arabic.obj
 0002:000373ec       $chain$0$?data_destroy_arabic@@YAXPEAX@Z 00000001800c23ec     hb-ot-shaper-arabic.obj
 0002:00037400       $chain$1$?data_destroy_arabic@@YAXPEAX@Z 00000001800c2400     hb-ot-shaper-arabic.obj
 0002:00037414       $chain$2$?data_destroy_arabic@@YAXPEAX@Z 00000001800c2414     hb-ot-shaper-arabic.obj
 0002:00037424       $chain$3$?data_destroy_arabic@@YAXPEAX@Z 00000001800c2424     hb-ot-shaper-arabic.obj
 0002:00037434       $unwind$?arabic_fallback_shape@@YA_NPEBUhb_ot_shape_plan_t@@PEAUhb_font_t@@PEAUhb_buffer_t@@@Z 00000001800c2434     hb-ot-shaper-arabic.obj
 0002:00037454       $unwind$?serialize@?$ArrayOf@UHBGlyphID16@OT@@U?$IntType@G$01@2@@OT@@QEAA_NPEAUhb_serialize_context_t@@I_N@Z 00000001800c2454     hb-ot-shaper-arabic.obj
 0002:00037454       $unwind$?serialize@?$HeadlessArrayOf@UHBGlyphID16@OT@@U?$IntType@G$01@2@@OT@@QEAA_NPEAUhb_serialize_context_t@@I_N@Z 00000001800c2454     hb-ot-shaper-arabic.obj
 0002:00037468       $unwind$??$extend_min@U?$CoverageFormat2_4@USmallTypes@Layout@OT@@@Common@Layout@OT@@@hb_serialize_context_t@@QEAAPEAU?$CoverageFormat2_4@USmallTypes@Layout@OT@@@Common@Layout@OT@@PEAU1234@@Z 00000001800c2468     hb-ot-shaper-arabic.obj
 0002:00037468       $unwind$??$extend_min@U?$IntType@G$01@OT@@@hb_serialize_context_t@@QEAAPEAU?$IntType@G$01@OT@@AEAU12@@Z 00000001800c2468     hb-ot-shaper-arabic.obj
 0002:00037468       $unwind$??$extend_min@U?$Ligature@USmallTypes@Layout@OT@@@GSUB_impl@Layout@OT@@@hb_serialize_context_t@@QEAAPEAU?$Ligature@USmallTypes@Layout@OT@@@GSUB_impl@Layout@OT@@PEAU1234@@Z 00000001800c2468     hb-ot-shaper-arabic.obj
 0002:00037468       $unwind$??$extend_min@U?$LigatureSet@USmallTypes@Layout@OT@@@GSUB_impl@Layout@OT@@@hb_serialize_context_t@@QEAAPEAU?$LigatureSet@USmallTypes@Layout@OT@@@GSUB_impl@Layout@OT@@PEAU1234@@Z 00000001800c2468     hb-ot-shaper-arabic.obj
 0002:00037468       $unwind$??$extend_min@U?$LigatureSubstFormat1_2@USmallTypes@Layout@OT@@@GSUB_impl@Layout@OT@@@hb_serialize_context_t@@QEAAPEAU?$LigatureSubstFormat1_2@USmallTypes@Layout@OT@@@GSUB_impl@Layout@OT@@PEAU1234@@Z 00000001800c2468     hb-ot-shaper-arabic.obj
 0002:00037468       $unwind$??$extend_min@U?$SingleSubstFormat1_3@USmallTypes@Layout@OT@@@GSUB_impl@Layout@OT@@@hb_serialize_context_t@@QEAAPEAU?$SingleSubstFormat1_3@USmallTypes@Layout@OT@@@GSUB_impl@Layout@OT@@PEAU1234@@Z 00000001800c2468     hb-ot-shaper-arabic.obj
 0002:00037468       $unwind$??$extend_min@U?$SingleSubstFormat2_4@USmallTypes@Layout@OT@@@GSUB_impl@Layout@OT@@@hb_serialize_context_t@@QEAAPEAU?$SingleSubstFormat2_4@USmallTypes@Layout@OT@@@GSUB_impl@Layout@OT@@PEAU1234@@Z 00000001800c2468     hb-ot-shaper-arabic.obj
 0002:00037468       $unwind$??$extend_min@UCoverage@Common@Layout@OT@@@hb_serialize_context_t@@QEAAPEAUCoverage@Common@Layout@OT@@PEAU1234@@Z 00000001800c2468     hb-ot-shaper-arabic.obj
 0002:00037468       $unwind$??$extend_min@ULookup@OT@@@hb_serialize_context_t@@QEAAPEAULookup@OT@@PEAU12@@Z 00000001800c2468     hb-ot-shaper-arabic.obj
 0002:00037468       $unwind$Java_sun_font_StrikeCache_getGlyphCacheDescription 00000001800c2468     sunFont.obj
 0002:00037474       $chain$0$??$extend_min@U?$LigatureSubstFormat1_2@USmallTypes@Layout@OT@@@GSUB_impl@Layout@OT@@@hb_serialize_context_t@@QEAAPEAU?$LigatureSubstFormat1_2@USmallTypes@Layout@OT@@@GSUB_impl@Layout@OT@@PEAU1234@@Z 00000001800c2474     hb-ot-shaper-arabic.obj
 0002:00037474       $chain$0$??$extend_min@U?$SingleSubstFormat1_3@USmallTypes@Layout@OT@@@GSUB_impl@Layout@OT@@@hb_serialize_context_t@@QEAAPEAU?$SingleSubstFormat1_3@USmallTypes@Layout@OT@@@GSUB_impl@Layout@OT@@PEAU1234@@Z 00000001800c2474     hb-ot-shaper-arabic.obj
 0002:00037474       $chain$0$??$extend_min@U?$SingleSubstFormat2_4@USmallTypes@Layout@OT@@@GSUB_impl@Layout@OT@@@hb_serialize_context_t@@QEAAPEAU?$SingleSubstFormat2_4@USmallTypes@Layout@OT@@@GSUB_impl@Layout@OT@@PEAU1234@@Z 00000001800c2474     hb-ot-shaper-arabic.obj
 0002:00037474       $chain$0$??$extend_min@ULookup@OT@@@hb_serialize_context_t@@QEAAPEAULookup@OT@@PEAU12@@Z 00000001800c2474     hb-ot-shaper-arabic.obj
 0002:00037488       $chain$2$??$extend_min@U?$LigatureSubstFormat1_2@USmallTypes@Layout@OT@@@GSUB_impl@Layout@OT@@@hb_serialize_context_t@@QEAAPEAU?$LigatureSubstFormat1_2@USmallTypes@Layout@OT@@@GSUB_impl@Layout@OT@@PEAU1234@@Z 00000001800c2488     hb-ot-shaper-arabic.obj
 0002:00037488       $chain$2$??$extend_min@U?$SingleSubstFormat1_3@USmallTypes@Layout@OT@@@GSUB_impl@Layout@OT@@@hb_serialize_context_t@@QEAAPEAU?$SingleSubstFormat1_3@USmallTypes@Layout@OT@@@GSUB_impl@Layout@OT@@PEAU1234@@Z 00000001800c2488     hb-ot-shaper-arabic.obj
 0002:00037488       $chain$2$??$extend_min@U?$SingleSubstFormat2_4@USmallTypes@Layout@OT@@@GSUB_impl@Layout@OT@@@hb_serialize_context_t@@QEAAPEAU?$SingleSubstFormat2_4@USmallTypes@Layout@OT@@@GSUB_impl@Layout@OT@@PEAU1234@@Z 00000001800c2488     hb-ot-shaper-arabic.obj
 0002:00037488       $chain$2$??$extend_min@ULookup@OT@@@hb_serialize_context_t@@QEAAPEAULookup@OT@@PEAU12@@Z 00000001800c2488     hb-ot-shaper-arabic.obj
 0002:0003749c       $chain$0$??$extend_min@U?$IntType@G$01@OT@@@hb_serialize_context_t@@QEAAPEAU?$IntType@G$01@OT@@AEAU12@@Z 00000001800c249c     hb-ot-shaper-arabic.obj
 0002:0003749c       $chain$0$??$extend_min@U?$LigatureSet@USmallTypes@Layout@OT@@@GSUB_impl@Layout@OT@@@hb_serialize_context_t@@QEAAPEAU?$LigatureSet@USmallTypes@Layout@OT@@@GSUB_impl@Layout@OT@@PEAU1234@@Z 00000001800c249c     hb-ot-shaper-arabic.obj
 0002:0003749c       $chain$0$??$extend_min@UCoverage@Common@Layout@OT@@@hb_serialize_context_t@@QEAAPEAUCoverage@Common@Layout@OT@@PEAU1234@@Z 00000001800c249c     hb-ot-shaper-arabic.obj
 0002:000374b0       $chain$2$??$extend_min@U?$IntType@G$01@OT@@@hb_serialize_context_t@@QEAAPEAU?$IntType@G$01@OT@@AEAU12@@Z 00000001800c24b0     hb-ot-shaper-arabic.obj
 0002:000374b0       $chain$2$??$extend_min@U?$LigatureSet@USmallTypes@Layout@OT@@@GSUB_impl@Layout@OT@@@hb_serialize_context_t@@QEAAPEAU?$LigatureSet@USmallTypes@Layout@OT@@@GSUB_impl@Layout@OT@@PEAU1234@@Z 00000001800c24b0     hb-ot-shaper-arabic.obj
 0002:000374b0       $chain$2$??$extend_min@UCoverage@Common@Layout@OT@@@hb_serialize_context_t@@QEAAPEAUCoverage@Common@Layout@OT@@PEAU1234@@Z 00000001800c24b0     hb-ot-shaper-arabic.obj
 0002:000374c4       $unwind$?serialize@?$LigatureSet@USmallTypes@Layout@OT@@@GSUB_impl@Layout@OT@@QEAA_NPEAUhb_serialize_context_t@@U?$hb_array_t@$$CBUHBGlyphID16@OT@@@@U?$hb_array_t@$$CBI@@AEAU6@@Z 00000001800c24c4     hb-ot-shaper-arabic.obj
 0002:000374dc       $unwind$?serialize@?$LigatureSubstFormat1_2@USmallTypes@Layout@OT@@@GSUB_impl@Layout@OT@@QEAA_NPEAUhb_serialize_context_t@@U?$hb_sorted_array_t@$$CBUHBGlyphID16@OT@@@@U?$hb_array_t@$$CBI@@U?$hb_array_t@$$CBUHBGlyphID16@OT@@@@23@Z 00000001800c24dc     hb-ot-shaper-arabic.obj
 0002:000374f8       $unwind$?arabic_fallback_synthesize_lookup_single@@YAPEAUSubstLookup@GSUB_impl@Layout@OT@@PEBUhb_ot_shape_plan_t@@PEAUhb_font_t@@I@Z 00000001800c24f8     hb-ot-shaper-arabic.obj
 0002:00037518       $chain$0$?arabic_fallback_synthesize_lookup_single@@YAPEAUSubstLookup@GSUB_impl@Layout@OT@@PEBUhb_ot_shape_plan_t@@PEAUhb_font_t@@I@Z 00000001800c2518     hb-ot-shaper-arabic.obj
 0002:0003752c       $chain$1$?arabic_fallback_synthesize_lookup_single@@YAPEAUSubstLookup@GSUB_impl@Layout@OT@@PEBUhb_ot_shape_plan_t@@PEAUhb_font_t@@I@Z 00000001800c252c     hb-ot-shaper-arabic.obj
 0002:0003753c       $unwind$??$arabic_fallback_synthesize_lookup_ligature@$$BY00Uligature_3_set_t@@@@YAPEAUSubstLookup@GSUB_impl@Layout@OT@@PEBUhb_ot_shape_plan_t@@PEAUhb_font_t@@AEAY00$$CBUligature_3_set_t@@I@Z 00000001800c253c     hb-ot-shaper-arabic.obj
 0002:0003755c       $chain$2$??$arabic_fallback_synthesize_lookup_ligature@$$BY00Uligature_3_set_t@@@@YAPEAUSubstLookup@GSUB_impl@Layout@OT@@PEBUhb_ot_shape_plan_t@@PEAUhb_font_t@@AEAY00$$CBUligature_3_set_t@@I@Z 00000001800c255c     hb-ot-shaper-arabic.obj
 0002:00037574       $chain$3$??$arabic_fallback_synthesize_lookup_ligature@$$BY00Uligature_3_set_t@@@@YAPEAUSubstLookup@GSUB_impl@Layout@OT@@PEBUhb_ot_shape_plan_t@@PEAUhb_font_t@@AEAY00$$CBUligature_3_set_t@@I@Z 00000001800c2574     hb-ot-shaper-arabic.obj
 0002:00037584       $unwind$??$arabic_fallback_synthesize_lookup_ligature@$$BY0BC@Uligature_set_t@@@@YAPEAUSubstLookup@GSUB_impl@Layout@OT@@PEBUhb_ot_shape_plan_t@@PEAUhb_font_t@@AEAY0BC@$$CBUligature_set_t@@I@Z 00000001800c2584     hb-ot-shaper-arabic.obj
 0002:000375a8       $unwind$??$arabic_fallback_synthesize_lookup_ligature@$$BY00Uligature_mark_set_t@@@@YAPEAUSubstLookup@GSUB_impl@Layout@OT@@PEBUhb_ot_shape_plan_t@@PEAUhb_font_t@@AEAY00$$CBUligature_mark_set_t@@I@Z 00000001800c25a8     hb-ot-shaper-arabic.obj
 0002:000375c8       $chain$2$??$arabic_fallback_synthesize_lookup_ligature@$$BY00Uligature_mark_set_t@@@@YAPEAUSubstLookup@GSUB_impl@Layout@OT@@PEBUhb_ot_shape_plan_t@@PEAUhb_font_t@@AEAY00$$CBUligature_mark_set_t@@I@Z 00000001800c25c8     hb-ot-shaper-arabic.obj
 0002:000375e0       $chain$3$??$arabic_fallback_synthesize_lookup_ligature@$$BY00Uligature_mark_set_t@@@@YAPEAUSubstLookup@GSUB_impl@Layout@OT@@PEBUhb_ot_shape_plan_t@@PEAUhb_font_t@@AEAY00$$CBUligature_mark_set_t@@I@Z 00000001800c25e0     hb-ot-shaper-arabic.obj
 0002:000375f0       $unwind$?arabic_fallback_plan_init_win1256@@YA_NPEAUarabic_fallback_plan_t@@PEBUhb_ot_shape_plan_t@@PEAUhb_font_t@@@Z 00000001800c25f0     hb-ot-shaper-arabic.obj
 0002:000375fc       $chain$4$?arabic_fallback_plan_init_win1256@@YA_NPEAUarabic_fallback_plan_t@@PEBUhb_ot_shape_plan_t@@PEAUhb_font_t@@@Z 00000001800c25fc     hb-ot-shaper-arabic.obj
 0002:00037620       $chain$6$?arabic_fallback_plan_init_win1256@@YA_NPEAUarabic_fallback_plan_t@@PEBUhb_ot_shape_plan_t@@PEAUhb_font_t@@@Z 00000001800c2620     hb-ot-shaper-arabic.obj
 0002:00037644       $chain$7$?arabic_fallback_plan_init_win1256@@YA_NPEAUarabic_fallback_plan_t@@PEBUhb_ot_shape_plan_t@@PEAUhb_font_t@@@Z 00000001800c2644     hb-ot-shaper-arabic.obj
 0002:00037654       $unwind$?arabic_fallback_plan_init_unicode@@YA_NPEAUarabic_fallback_plan_t@@PEBUhb_ot_shape_plan_t@@PEAUhb_font_t@@@Z 00000001800c2654     hb-ot-shaper-arabic.obj
 0002:0003766c       $unwind$?arabic_joining@@YAXPEAUhb_buffer_t@@@Z 00000001800c266c     hb-ot-shaper-arabic.obj
 0002:00037680       $chain$0$?arabic_joining@@YAXPEAUhb_buffer_t@@@Z 00000001800c2680     hb-ot-shaper-arabic.obj
 0002:00037694       $chain$1$?arabic_joining@@YAXPEAUhb_buffer_t@@@Z 00000001800c2694     hb-ot-shaper-arabic.obj
 0002:000376a8       $chain$2$?arabic_joining@@YAXPEAUhb_buffer_t@@@Z 00000001800c26a8     hb-ot-shaper-arabic.obj
 0002:000376a8       $chain$4$?arabic_joining@@YAXPEAUhb_buffer_t@@@Z 00000001800c26a8     hb-ot-shaper-arabic.obj
 0002:000376b8       $chain$3$?arabic_joining@@YAXPEAUhb_buffer_t@@@Z 00000001800c26b8     hb-ot-shaper-arabic.obj
 0002:000376cc       $chain$5$?arabic_joining@@YAXPEAUhb_buffer_t@@@Z 00000001800c26cc     hb-ot-shaper-arabic.obj
 0002:000376dc       $unwind$?apply_stch@@YAXPEBUhb_ot_shape_plan_t@@PEAUhb_buffer_t@@PEAUhb_font_t@@@Z 00000001800c26dc     hb-ot-shaper-arabic.obj
 0002:000376e8       $chain$6$?apply_stch@@YAXPEBUhb_ot_shape_plan_t@@PEAUhb_buffer_t@@PEAUhb_font_t@@@Z 00000001800c26e8     hb-ot-shaper-arabic.obj
 0002:00037714       $chain$7$?apply_stch@@YAXPEBUhb_ot_shape_plan_t@@PEAUhb_buffer_t@@PEAUhb_font_t@@@Z 00000001800c2714     hb-ot-shaper-arabic.obj
 0002:00037724       $unwind$?reorder_marks_arabic@@YAXPEBUhb_ot_shape_plan_t@@PEAUhb_buffer_t@@II@Z 00000001800c2724     hb-ot-shaper-arabic.obj
 0002:00037748       $unwind$??$serialize_serialize@AEAU?$hb_sorted_array_t@$$CBUHBGlyphID16@OT@@@@@?$OffsetTo@UCoverage@Common@Layout@OT@@U?$IntType@G$01@4@$00@OT@@QEAA_NPEAUhb_serialize_context_t@@AEAU?$hb_sorted_array_t@$$CBUHBGlyphID16@OT@@@@@Z 00000001800c2748     hb-ot-shaper-arabic.obj
 0002:00037758       $chain$2$??$serialize_serialize@AEAU?$hb_sorted_array_t@$$CBUHBGlyphID16@OT@@@@@?$OffsetTo@UCoverage@Common@Layout@OT@@U?$IntType@G$01@4@$00@OT@@QEAA_NPEAUhb_serialize_context_t@@AEAU?$hb_sorted_array_t@$$CBUHBGlyphID16@OT@@@@@Z 00000001800c2758     hb-ot-shaper-arabic.obj
 0002:00037774       $chain$3$??$serialize_serialize@AEAU?$hb_sorted_array_t@$$CBUHBGlyphID16@OT@@@@@?$OffsetTo@UCoverage@Common@Layout@OT@@U?$IntType@G$01@4@$00@OT@@QEAA_NPEAUhb_serialize_context_t@@AEAU?$hb_sorted_array_t@$$CBUHBGlyphID16@OT@@@@@Z 00000001800c2774     hb-ot-shaper-arabic.obj
 0002:00037784       $unwind$??$serialize@U?$hb_zip_iter_t@U?$hb_sorted_array_t@UHBGlyphID16@OT@@@@U?$hb_array_t@UHBGlyphID16@OT@@@@@@$0A@@SingleSubst@GSUB_impl@Layout@OT@@QEAA_NPEAUhb_serialize_context_t@@U?$hb_zip_iter_t@U?$hb_sorted_array_t@UHBGlyphID16@OT@@@@U?$hb_array_t@UHBGlyphID16@OT@@@@@@@Z 00000001800c2784     hb-ot-shaper-arabic.obj
 0002:0003779c       $chain$3$??$serialize@U?$hb_zip_iter_t@U?$hb_sorted_array_t@UHBGlyphID16@OT@@@@U?$hb_array_t@UHBGlyphID16@OT@@@@@@$0A@@SingleSubst@GSUB_impl@Layout@OT@@QEAA_NPEAUhb_serialize_context_t@@U?$hb_zip_iter_t@U?$hb_sorted_array_t@UHBGlyphID16@OT@@@@U?$hb_array_t@UHBGlyphID16@OT@@@@@@@Z 00000001800c279c     hb-ot-shaper-arabic.obj
 0002:000377b4       $chain$4$??$serialize@U?$hb_zip_iter_t@U?$hb_sorted_array_t@UHBGlyphID16@OT@@@@U?$hb_array_t@UHBGlyphID16@OT@@@@@@$0A@@SingleSubst@GSUB_impl@Layout@OT@@QEAA_NPEAUhb_serialize_context_t@@U?$hb_zip_iter_t@U?$hb_sorted_array_t@UHBGlyphID16@OT@@@@U?$hb_array_t@UHBGlyphID16@OT@@@@@@@Z 00000001800c27b4     hb-ot-shaper-arabic.obj
 0002:000377c4       $unwind$??$hb_stable_sort@UHBGlyphID16@OT@@U?$IntType@G$01@2@I@@YAXPEAUHBGlyphID16@OT@@IP6AHPEBU?$IntType@G$01@1@1@ZPEAI@Z 00000001800c27c4     hb-ot-shaper-arabic.obj
 0002:000377d0       $chain$5$??$hb_stable_sort@UHBGlyphID16@OT@@U?$IntType@G$01@2@I@@YAXPEAUHBGlyphID16@OT@@IP6AHPEBU?$IntType@G$01@1@1@ZPEAI@Z 00000001800c27d0     hb-ot-shaper-arabic.obj
 0002:000377f8       $chain$6$??$hb_stable_sort@UHBGlyphID16@OT@@U?$IntType@G$01@2@I@@YAXPEAUHBGlyphID16@OT@@IP6AHPEBU?$IntType@G$01@1@1@ZPEAI@Z 00000001800c27f8     hb-ot-shaper-arabic.obj
 0002:00037808       $chain$0$??$extend_min@U?$CoverageFormat2_4@USmallTypes@Layout@OT@@@Common@Layout@OT@@@hb_serialize_context_t@@QEAAPEAU?$CoverageFormat2_4@USmallTypes@Layout@OT@@@Common@Layout@OT@@PEAU1234@@Z 00000001800c2808     hb-ot-shaper-arabic.obj
 0002:00037808       $chain$0$??$extend_min@U?$Ligature@USmallTypes@Layout@OT@@@GSUB_impl@Layout@OT@@@hb_serialize_context_t@@QEAAPEAU?$Ligature@USmallTypes@Layout@OT@@@GSUB_impl@Layout@OT@@PEAU1234@@Z 00000001800c2808     hb-ot-shaper-arabic.obj
 0002:0003781c       $chain$2$??$extend_min@U?$CoverageFormat2_4@USmallTypes@Layout@OT@@@Common@Layout@OT@@@hb_serialize_context_t@@QEAAPEAU?$CoverageFormat2_4@USmallTypes@Layout@OT@@@Common@Layout@OT@@PEAU1234@@Z 00000001800c281c     hb-ot-shaper-arabic.obj
 0002:0003781c       $chain$2$??$extend_min@U?$Ligature@USmallTypes@Layout@OT@@@GSUB_impl@Layout@OT@@@hb_serialize_context_t@@QEAAPEAU?$Ligature@USmallTypes@Layout@OT@@@GSUB_impl@Layout@OT@@PEAU1234@@Z 00000001800c281c     hb-ot-shaper-arabic.obj
 0002:00037830       $unwind$??$serialize_serialize@AEAU?$hb_map_iter_t@U?$hb_zip_iter_t@U?$hb_sorted_array_t@UHBGlyphID16@OT@@@@U?$hb_array_t@UHBGlyphID16@OT@@@@@@AEBU<unnamed-type-hb_first>@@$00$0A@@@@?$OffsetTo@UCoverage@Common@Layout@OT@@U?$IntType@G$01@4@$00@OT@@QEAA_NPEAUhb_serialize_context_t@@AEAU?$hb_map_iter_t@U?$hb_zip_iter_t@U?$hb_sorted_array_t@UHBGlyphID16@OT@@@@U?$hb_array_t@UHBGlyphID16@OT@@@@@@AEBU<unnamed-type-hb_first>@@$00$0A@@@@Z 00000001800c2830     hb-ot-shaper-arabic.obj
 0002:00037840       $unwind$??$serialize@U?$hb_map_iter_t@U?$hb_zip_iter_t@U?$hb_sorted_array_t@UHBGlyphID16@OT@@@@U?$hb_array_t@UHBGlyphID16@OT@@@@@@AEBU<unnamed-type-hb_first>@@$00$0A@@@$0A@@Coverage@Common@Layout@OT@@QEAA_NPEAUhb_serialize_context_t@@U?$hb_map_iter_t@U?$hb_zip_iter_t@U?$hb_sorted_array_t@UHBGlyphID16@OT@@@@U?$hb_array_t@UHBGlyphID16@OT@@@@@@AEBU<unnamed-type-hb_first>@@$00$0A@@@@Z 00000001800c2840     hb-ot-shaper-arabic.obj
 0002:00037858       $chain$6$??$serialize@U?$hb_map_iter_t@U?$hb_zip_iter_t@U?$hb_sorted_array_t@UHBGlyphID16@OT@@@@U?$hb_array_t@UHBGlyphID16@OT@@@@@@AEBU<unnamed-type-hb_first>@@$00$0A@@@$0A@@Coverage@Common@Layout@OT@@QEAA_NPEAUhb_serialize_context_t@@U?$hb_map_iter_t@U?$hb_zip_iter_t@U?$hb_sorted_array_t@UHBGlyphID16@OT@@@@U?$hb_array_t@UHBGlyphID16@OT@@@@@@AEBU<unnamed-type-hb_first>@@$00$0A@@@@Z 00000001800c2858     hb-ot-shaper-arabic.obj
 0002:00037878       $chain$7$??$serialize@U?$hb_map_iter_t@U?$hb_zip_iter_t@U?$hb_sorted_array_t@UHBGlyphID16@OT@@@@U?$hb_array_t@UHBGlyphID16@OT@@@@@@AEBU<unnamed-type-hb_first>@@$00$0A@@@$0A@@Coverage@Common@Layout@OT@@QEAA_NPEAUhb_serialize_context_t@@U?$hb_map_iter_t@U?$hb_zip_iter_t@U?$hb_sorted_array_t@UHBGlyphID16@OT@@@@U?$hb_array_t@UHBGlyphID16@OT@@@@@@AEBU<unnamed-type-hb_first>@@$00$0A@@@@Z 00000001800c2878     hb-ot-shaper-arabic.obj
 0002:00037888       $unwind$??$serialize@U?$hb_map_iter_t@U?$hb_zip_iter_t@U?$hb_sorted_array_t@UHBGlyphID16@OT@@@@U?$hb_array_t@UHBGlyphID16@OT@@@@@@AEBU<unnamed-type-hb_first>@@$00$0A@@@$0A@@?$CoverageFormat2_4@USmallTypes@Layout@OT@@@Common@Layout@OT@@AEAA_NPEAUhb_serialize_context_t@@U?$hb_map_iter_t@U?$hb_zip_iter_t@U?$hb_sorted_array_t@UHBGlyphID16@OT@@@@U?$hb_array_t@UHBGlyphID16@OT@@@@@@AEBU<unnamed-type-hb_first>@@$00$0A@@@@Z 00000001800c2888     hb-ot-shaper-arabic.obj
 0002:000378a0       $unwind$?data_create_hangul@@YAPEAXPEBUhb_ot_shape_plan_t@@@Z 00000001800c28a0     hb-ot-shaper-hangul.obj
 0002:000378b0       $unwind$?preprocess_text_hangul@@YAXPEBUhb_ot_shape_plan_t@@PEAUhb_buffer_t@@PEAUhb_font_t@@@Z 00000001800c28b0     hb-ot-shaper-hangul.obj
 0002:000378cc       $chain$2$?preprocess_text_hangul@@YAXPEBUhb_ot_shape_plan_t@@PEAUhb_buffer_t@@PEAUhb_font_t@@@Z 00000001800c28cc     hb-ot-shaper-hangul.obj
 0002:000378e8       $chain$3$?preprocess_text_hangul@@YAXPEBUhb_ot_shape_plan_t@@PEAUhb_buffer_t@@PEAUhb_font_t@@@Z 00000001800c28e8     hb-ot-shaper-hangul.obj
 0002:000378f8       $unwind$?reorder_marks_hebrew@@YAXPEBUhb_ot_shape_plan_t@@PEAUhb_buffer_t@@II@Z 00000001800c28f8     hb-ot-shaper-hebrew.obj
 0002:00037904       $chain$2$?reorder_marks_hebrew@@YAXPEBUhb_ot_shape_plan_t@@PEAUhb_buffer_t@@II@Z 00000001800c2904     hb-ot-shaper-hebrew.obj
 0002:00037920       $chain$3$?reorder_marks_hebrew@@YAXPEBUhb_ot_shape_plan_t@@PEAUhb_buffer_t@@II@Z 00000001800c2920     hb-ot-shaper-hebrew.obj
 0002:00037930       $unwind$?setup_syllables_indic@@YA_NPEBUhb_ot_shape_plan_t@@PEAUhb_font_t@@PEAUhb_buffer_t@@@Z 00000001800c2930     hb-ot-shaper-indic.obj
 0002:00037930       $unwind$?setup_syllables_khmer@@YA_NPEBUhb_ot_shape_plan_t@@PEAUhb_font_t@@PEAUhb_buffer_t@@@Z 00000001800c2930     hb-ot-shaper-khmer.obj
 0002:00037930       $unwind$?setup_syllables_myanmar@@YA_NPEBUhb_ot_shape_plan_t@@PEAUhb_font_t@@PEAUhb_buffer_t@@@Z 00000001800c2930     hb-ot-shaper-myanmar.obj
 0002:0003793c       $chain$0$?setup_syllables_indic@@YA_NPEBUhb_ot_shape_plan_t@@PEAUhb_font_t@@PEAUhb_buffer_t@@@Z 00000001800c293c     hb-ot-shaper-indic.obj
 0002:00037950       $chain$2$?setup_syllables_indic@@YA_NPEBUhb_ot_shape_plan_t@@PEAUhb_font_t@@PEAUhb_buffer_t@@@Z 00000001800c2950     hb-ot-shaper-indic.obj
 0002:00037968       $chain$3$?setup_syllables_indic@@YA_NPEBUhb_ot_shape_plan_t@@PEAUhb_font_t@@PEAUhb_buffer_t@@@Z 00000001800c2968     hb-ot-shaper-indic.obj
 0002:00037978       $chain$4$?setup_syllables_indic@@YA_NPEBUhb_ot_shape_plan_t@@PEAUhb_font_t@@PEAUhb_buffer_t@@@Z 00000001800c2978     hb-ot-shaper-indic.obj
 0002:00037988       $unwind$?initial_reordering_indic@@YA_NPEBUhb_ot_shape_plan_t@@PEAUhb_font_t@@PEAUhb_buffer_t@@@Z 00000001800c2988     hb-ot-shaper-indic.obj
 0002:000379a4       $chain$4$?initial_reordering_indic@@YA_NPEBUhb_ot_shape_plan_t@@PEAUhb_font_t@@PEAUhb_buffer_t@@@Z 00000001800c29a4     hb-ot-shaper-indic.obj
 0002:000379b8       $chain$5$?initial_reordering_indic@@YA_NPEBUhb_ot_shape_plan_t@@PEAUhb_font_t@@PEAUhb_buffer_t@@@Z 00000001800c29b8     hb-ot-shaper-indic.obj
 0002:000379c8       $chain$0$?final_reordering_indic@@YA_NPEBUhb_ot_shape_plan_t@@PEAUhb_font_t@@PEAUhb_buffer_t@@@Z 00000001800c29c8     hb-ot-shaper-indic.obj
 0002:000379dc       $chain$1$?final_reordering_indic@@YA_NPEBUhb_ot_shape_plan_t@@PEAUhb_font_t@@PEAUhb_buffer_t@@@Z 00000001800c29dc     hb-ot-shaper-indic.obj
 0002:000379f0       $chain$2$?final_reordering_indic@@YA_NPEBUhb_ot_shape_plan_t@@PEAUhb_font_t@@PEAUhb_buffer_t@@@Z 00000001800c29f0     hb-ot-shaper-indic.obj
 0002:00037a00       $chain$3$?final_reordering_indic@@YA_NPEBUhb_ot_shape_plan_t@@PEAUhb_font_t@@PEAUhb_buffer_t@@@Z 00000001800c2a00     hb-ot-shaper-indic.obj
 0002:00037a10       $unwind$?data_create_indic@@YAPEAXPEBUhb_ot_shape_plan_t@@@Z 00000001800c2a10     hb-ot-shaper-indic.obj
 0002:00037a20       $chain$1$?data_create_indic@@YAPEAXPEBUhb_ot_shape_plan_t@@@Z 00000001800c2a20     hb-ot-shaper-indic.obj
 0002:00037a38       $chain$3$?data_create_indic@@YAPEAXPEBUhb_ot_shape_plan_t@@@Z 00000001800c2a38     hb-ot-shaper-indic.obj
 0002:00037a50       $chain$0$?setup_masks_indic@@YAXPEBUhb_ot_shape_plan_t@@PEAUhb_buffer_t@@PEAUhb_font_t@@@Z 00000001800c2a50     hb-ot-shaper-indic.obj
 0002:00037a64       $chain$1$?setup_masks_indic@@YAXPEBUhb_ot_shape_plan_t@@PEAUhb_buffer_t@@PEAUhb_font_t@@@Z 00000001800c2a64     hb-ot-shaper-indic.obj
 0002:00037a74       $unwind$?initial_reordering_consonant_syllable@@YAXPEBUhb_ot_shape_plan_t@@PEAUhb_face_t@@PEAUhb_buffer_t@@II@Z 00000001800c2a74     hb-ot-shaper-indic.obj
 0002:00037a94       $unwind$?final_reordering_syllable_indic@@YAXPEBUhb_ot_shape_plan_t@@PEAUhb_buffer_t@@II@Z 00000001800c2a94     hb-ot-shaper-indic.obj
 0002:00037aa0       $chain$4$?final_reordering_syllable_indic@@YAXPEBUhb_ot_shape_plan_t@@PEAUhb_buffer_t@@II@Z 00000001800c2aa0     hb-ot-shaper-indic.obj
 0002:00037ac4       $chain$5$?final_reordering_syllable_indic@@YAXPEBUhb_ot_shape_plan_t@@PEAUhb_buffer_t@@II@Z 00000001800c2ac4     hb-ot-shaper-indic.obj
 0002:00037ad8       $chain$6$?final_reordering_syllable_indic@@YAXPEBUhb_ot_shape_plan_t@@PEAUhb_buffer_t@@II@Z 00000001800c2ad8     hb-ot-shaper-indic.obj
 0002:00037ae8       $chain$0$?setup_syllables_khmer@@YA_NPEBUhb_ot_shape_plan_t@@PEAUhb_font_t@@PEAUhb_buffer_t@@@Z 00000001800c2ae8     hb-ot-shaper-khmer.obj
 0002:00037afc       $chain$2$?setup_syllables_khmer@@YA_NPEBUhb_ot_shape_plan_t@@PEAUhb_font_t@@PEAUhb_buffer_t@@@Z 00000001800c2afc     hb-ot-shaper-khmer.obj
 0002:00037b14       $chain$3$?setup_syllables_khmer@@YA_NPEBUhb_ot_shape_plan_t@@PEAUhb_font_t@@PEAUhb_buffer_t@@@Z 00000001800c2b14     hb-ot-shaper-khmer.obj
 0002:00037b24       $chain$4$?setup_syllables_khmer@@YA_NPEBUhb_ot_shape_plan_t@@PEAUhb_font_t@@PEAUhb_buffer_t@@@Z 00000001800c2b24     hb-ot-shaper-khmer.obj
 0002:00037b34       $unwind$?reorder_khmer@@YA_NPEBUhb_ot_shape_plan_t@@PEAUhb_font_t@@PEAUhb_buffer_t@@@Z 00000001800c2b34     hb-ot-shaper-khmer.obj
 0002:00037b44       $chain$0$?reorder_khmer@@YA_NPEBUhb_ot_shape_plan_t@@PEAUhb_font_t@@PEAUhb_buffer_t@@@Z 00000001800c2b44     hb-ot-shaper-khmer.obj
 0002:00037b58       $chain$1$?reorder_khmer@@YA_NPEBUhb_ot_shape_plan_t@@PEAUhb_font_t@@PEAUhb_buffer_t@@@Z 00000001800c2b58     hb-ot-shaper-khmer.obj
 0002:00037b6c       $chain$2$?reorder_khmer@@YA_NPEBUhb_ot_shape_plan_t@@PEAUhb_font_t@@PEAUhb_buffer_t@@@Z 00000001800c2b6c     hb-ot-shaper-khmer.obj
 0002:00037b7c       $chain$3$?reorder_khmer@@YA_NPEBUhb_ot_shape_plan_t@@PEAUhb_font_t@@PEAUhb_buffer_t@@@Z 00000001800c2b7c     hb-ot-shaper-khmer.obj
 0002:00037b8c       $unwind$?data_create_khmer@@YAPEAXPEBUhb_ot_shape_plan_t@@@Z 00000001800c2b8c     hb-ot-shaper-khmer.obj
 0002:00037b98       $chain$2$?data_create_khmer@@YAPEAXPEBUhb_ot_shape_plan_t@@@Z 00000001800c2b98     hb-ot-shaper-khmer.obj
 0002:00037bb4       $chain$4$?data_create_khmer@@YAPEAXPEBUhb_ot_shape_plan_t@@@Z 00000001800c2bb4     hb-ot-shaper-khmer.obj
 0002:00037bd0       $chain$0$?setup_masks_khmer@@YAXPEBUhb_ot_shape_plan_t@@PEAUhb_buffer_t@@PEAUhb_font_t@@@Z 00000001800c2bd0     hb-ot-shaper-khmer.obj
 0002:00037be4       $chain$1$?setup_masks_khmer@@YAXPEBUhb_ot_shape_plan_t@@PEAUhb_buffer_t@@PEAUhb_font_t@@@Z 00000001800c2be4     hb-ot-shaper-khmer.obj
 0002:00037bf4       $unwind$?reorder_consonant_syllable@@YAXPEBUhb_ot_shape_plan_t@@PEAUhb_face_t@@PEAUhb_buffer_t@@II@Z 00000001800c2bf4     hb-ot-shaper-khmer.obj
 0002:00037c00       $chain$4$?reorder_consonant_syllable@@YAXPEBUhb_ot_shape_plan_t@@PEAUhb_face_t@@PEAUhb_buffer_t@@II@Z 00000001800c2c00     hb-ot-shaper-khmer.obj
 0002:00037c24       $chain$5$?reorder_consonant_syllable@@YAXPEBUhb_ot_shape_plan_t@@PEAUhb_face_t@@PEAUhb_buffer_t@@II@Z 00000001800c2c24     hb-ot-shaper-khmer.obj
 0002:00037c34       $chain$0$?setup_syllables_myanmar@@YA_NPEBUhb_ot_shape_plan_t@@PEAUhb_font_t@@PEAUhb_buffer_t@@@Z 00000001800c2c34     hb-ot-shaper-myanmar.obj
 0002:00037c48       $chain$2$?setup_syllables_myanmar@@YA_NPEBUhb_ot_shape_plan_t@@PEAUhb_font_t@@PEAUhb_buffer_t@@@Z 00000001800c2c48     hb-ot-shaper-myanmar.obj
 0002:00037c60       $chain$3$?setup_syllables_myanmar@@YA_NPEBUhb_ot_shape_plan_t@@PEAUhb_font_t@@PEAUhb_buffer_t@@@Z 00000001800c2c60     hb-ot-shaper-myanmar.obj
 0002:00037c70       $chain$4$?setup_syllables_myanmar@@YA_NPEBUhb_ot_shape_plan_t@@PEAUhb_font_t@@PEAUhb_buffer_t@@@Z 00000001800c2c70     hb-ot-shaper-myanmar.obj
 0002:00037c80       $unwind$?reorder_myanmar@@YA_NPEBUhb_ot_shape_plan_t@@PEAUhb_font_t@@PEAUhb_buffer_t@@@Z 00000001800c2c80     hb-ot-shaper-myanmar.obj
 0002:00037c80       $unwind$?reorder_use@@YA_NPEBUhb_ot_shape_plan_t@@PEAUhb_font_t@@PEAUhb_buffer_t@@@Z 00000001800c2c80     hb-ot-shaper-use.obj
 0002:00037c90       $chain$0$?reorder_myanmar@@YA_NPEBUhb_ot_shape_plan_t@@PEAUhb_font_t@@PEAUhb_buffer_t@@@Z 00000001800c2c90     hb-ot-shaper-myanmar.obj
 0002:00037ca4       $chain$1$?reorder_myanmar@@YA_NPEBUhb_ot_shape_plan_t@@PEAUhb_font_t@@PEAUhb_buffer_t@@@Z 00000001800c2ca4     hb-ot-shaper-myanmar.obj
 0002:00037cb8       $chain$2$?reorder_myanmar@@YA_NPEBUhb_ot_shape_plan_t@@PEAUhb_font_t@@PEAUhb_buffer_t@@@Z 00000001800c2cb8     hb-ot-shaper-myanmar.obj
 0002:00037cc8       $chain$3$?reorder_myanmar@@YA_NPEBUhb_ot_shape_plan_t@@PEAUhb_font_t@@PEAUhb_buffer_t@@@Z 00000001800c2cc8     hb-ot-shaper-myanmar.obj
 0002:00037cd8       $chain$0$?setup_masks_myanmar@@YAXPEBUhb_ot_shape_plan_t@@PEAUhb_buffer_t@@PEAUhb_font_t@@@Z 00000001800c2cd8     hb-ot-shaper-myanmar.obj
 0002:00037cec       $chain$1$?setup_masks_myanmar@@YAXPEBUhb_ot_shape_plan_t@@PEAUhb_buffer_t@@PEAUhb_font_t@@@Z 00000001800c2cec     hb-ot-shaper-myanmar.obj
 0002:00037cfc       $unwind$?hb_syllabic_insert_dotted_circles@@YA_NPEAUhb_font_t@@PEAUhb_buffer_t@@IIHH@Z 00000001800c2cfc     hb-ot-shaper-syllabic.obj
 0002:00037d0c       $chain$2$?hb_syllabic_insert_dotted_circles@@YA_NPEAUhb_font_t@@PEAUhb_buffer_t@@IIHH@Z 00000001800c2d0c     hb-ot-shaper-syllabic.obj
 0002:00037d28       $chain$3$?hb_syllabic_insert_dotted_circles@@YA_NPEAUhb_font_t@@PEAUhb_buffer_t@@IIHH@Z 00000001800c2d28     hb-ot-shaper-syllabic.obj
 0002:00037d38       $unwind$?thai_pua_shape@@YAIIW4thai_action_t@@PEAUhb_font_t@@@Z 00000001800c2d38     hb-ot-shaper-thai.obj
 0002:00037d48       $unwind$?do_thai_pua_shaping@@YAXPEBUhb_ot_shape_plan_t@@PEAUhb_buffer_t@@PEAUhb_font_t@@@Z 00000001800c2d48     hb-ot-shaper-thai.obj
 0002:00037d58       $chain$3$?do_thai_pua_shaping@@YAXPEBUhb_ot_shape_plan_t@@PEAUhb_buffer_t@@PEAUhb_font_t@@@Z 00000001800c2d58     hb-ot-shaper-thai.obj
 0002:00037d78       $chain$4$?do_thai_pua_shaping@@YAXPEBUhb_ot_shape_plan_t@@PEAUhb_buffer_t@@PEAUhb_font_t@@@Z 00000001800c2d78     hb-ot-shaper-thai.obj
 0002:00037d88       $unwind$?preprocess_text_thai@@YAXPEBUhb_ot_shape_plan_t@@PEAUhb_buffer_t@@PEAUhb_font_t@@@Z 00000001800c2d88     hb-ot-shaper-thai.obj
 0002:00037d94       $chain$1$?preprocess_text_thai@@YAXPEBUhb_ot_shape_plan_t@@PEAUhb_buffer_t@@PEAUhb_font_t@@@Z 00000001800c2d94     hb-ot-shaper-thai.obj
 0002:00037dac       $chain$4$?preprocess_text_thai@@YAXPEBUhb_ot_shape_plan_t@@PEAUhb_buffer_t@@PEAUhb_font_t@@@Z 00000001800c2dac     hb-ot-shaper-thai.obj
 0002:00037dc8       $chain$5$?preprocess_text_thai@@YAXPEBUhb_ot_shape_plan_t@@PEAUhb_buffer_t@@PEAUhb_font_t@@@Z 00000001800c2dc8     hb-ot-shaper-thai.obj
 0002:00037dd8       $chain$6$?preprocess_text_thai@@YAXPEBUhb_ot_shape_plan_t@@PEAUhb_buffer_t@@PEAUhb_font_t@@@Z 00000001800c2dd8     hb-ot-shaper-thai.obj
 0002:00037de8       $unwind$?find_syllables_use@@YAXPEAUhb_buffer_t@@@Z 00000001800c2de8     hb-ot-shaper-use.obj
 0002:00037e1c       $chain$0$?find_syllables_use@@YAXPEAUhb_buffer_t@@@Z 00000001800c2e1c     hb-ot-shaper-use.obj
 0002:00037e30       $unwind$?__item__@?$hb_zip_iter_t@U?$hb_iota_iter_t@II@@U?$hb_filter_iter_t@U?$hb_filter_iter_t@U?$hb_zip_iter_t@U?$hb_iota_iter_t@II@@U?$hb_array_t@Uhb_glyph_info_t@@@@@@V<lambda_e52748becc06432fe81365edeb8c4003>@@AEBU<unnamed-type-hb_second>@@$0A@@@V<lambda_a2885d5959499a7c5bcf896c0de144bb>@@AEBU<unnamed-type-hb_identity>@@$0A@@@@@QEBA?AU?$hb_pair_t@IU?$hb_pair_t@IAEAUhb_glyph_info_t@@@@@@XZ 00000001800c2e30     hb-ot-shaper-use.obj
 0002:00037e38       $chain$1$??4?$machine_index_t@U?$hb_zip_iter_t@U?$hb_iota_iter_t@II@@U?$hb_filter_iter_t@U?$hb_filter_iter_t@U?$hb_zip_iter_t@U?$hb_iota_iter_t@II@@U?$hb_array_t@Uhb_glyph_info_t@@@@@@V<lambda_e52748becc06432fe81365edeb8c4003>@@AEBU<unnamed-type-hb_second>@@$0A@@@V<lambda_a2885d5959499a7c5bcf896c0de144bb>@@AEBU<unnamed-type-hb_identity>@@$0A@@@@@@@QEAAXAEBU0@@Z 00000001800c2e38     hb-ot-shaper-use.obj
 0002:00037e50       $chain$2$??4?$machine_index_t@U?$hb_zip_iter_t@U?$hb_iota_iter_t@II@@U?$hb_filter_iter_t@U?$hb_filter_iter_t@U?$hb_zip_iter_t@U?$hb_iota_iter_t@II@@U?$hb_array_t@Uhb_glyph_info_t@@@@@@V<lambda_e52748becc06432fe81365edeb8c4003>@@AEBU<unnamed-type-hb_second>@@$0A@@@V<lambda_a2885d5959499a7c5bcf896c0de144bb>@@AEBU<unnamed-type-hb_identity>@@$0A@@@@@@@QEAAXAEBU0@@Z 00000001800c2e50     hb-ot-shaper-use.obj
 0002:00037e60       $unwind$?setup_syllables_use@@YA_NPEBUhb_ot_shape_plan_t@@PEAUhb_font_t@@PEAUhb_buffer_t@@@Z 00000001800c2e60     hb-ot-shaper-use.obj
 0002:00037e74       $chain$1$?setup_syllables_use@@YA_NPEBUhb_ot_shape_plan_t@@PEAUhb_font_t@@PEAUhb_buffer_t@@@Z 00000001800c2e74     hb-ot-shaper-use.obj
 0002:00037e8c       $chain$2$?setup_syllables_use@@YA_NPEBUhb_ot_shape_plan_t@@PEAUhb_font_t@@PEAUhb_buffer_t@@@Z 00000001800c2e8c     hb-ot-shaper-use.obj
 0002:00037e9c       $unwind$?record_rphf_use@@YA_NPEBUhb_ot_shape_plan_t@@PEAUhb_font_t@@PEAUhb_buffer_t@@@Z 00000001800c2e9c     hb-ot-shaper-use.obj
 0002:00037ea8       $chain$1$?record_rphf_use@@YA_NPEBUhb_ot_shape_plan_t@@PEAUhb_font_t@@PEAUhb_buffer_t@@@Z 00000001800c2ea8     hb-ot-shaper-use.obj
 0002:00037ec0       $chain$2$?record_rphf_use@@YA_NPEBUhb_ot_shape_plan_t@@PEAUhb_font_t@@PEAUhb_buffer_t@@@Z 00000001800c2ec0     hb-ot-shaper-use.obj
 0002:00037ed0       $chain$0$?reorder_use@@YA_NPEBUhb_ot_shape_plan_t@@PEAUhb_font_t@@PEAUhb_buffer_t@@@Z 00000001800c2ed0     hb-ot-shaper-use.obj
 0002:00037ee4       $chain$1$?reorder_use@@YA_NPEBUhb_ot_shape_plan_t@@PEAUhb_font_t@@PEAUhb_buffer_t@@@Z 00000001800c2ee4     hb-ot-shaper-use.obj
 0002:00037ef8       $chain$2$?reorder_use@@YA_NPEBUhb_ot_shape_plan_t@@PEAUhb_font_t@@PEAUhb_buffer_t@@@Z 00000001800c2ef8     hb-ot-shaper-use.obj
 0002:00037f08       $chain$3$?reorder_use@@YA_NPEBUhb_ot_shape_plan_t@@PEAUhb_font_t@@PEAUhb_buffer_t@@@Z 00000001800c2f08     hb-ot-shaper-use.obj
 0002:00037f18       $unwind$?setup_topographical_masks@@YAXPEBUhb_ot_shape_plan_t@@PEAUhb_buffer_t@@@Z 00000001800c2f18     hb-ot-shaper-use.obj
 0002:00037f28       $chain$3$?setup_topographical_masks@@YAXPEBUhb_ot_shape_plan_t@@PEAUhb_buffer_t@@@Z 00000001800c2f28     hb-ot-shaper-use.obj
 0002:00037f48       $chain$6$?setup_topographical_masks@@YAXPEBUhb_ot_shape_plan_t@@PEAUhb_buffer_t@@@Z 00000001800c2f48     hb-ot-shaper-use.obj
 0002:00037f64       $chain$10$?setup_topographical_masks@@YAXPEBUhb_ot_shape_plan_t@@PEAUhb_buffer_t@@@Z 00000001800c2f64     hb-ot-shaper-use.obj
 0002:00037f64       $chain$7$?setup_topographical_masks@@YAXPEBUhb_ot_shape_plan_t@@PEAUhb_buffer_t@@@Z 00000001800c2f64     hb-ot-shaper-use.obj
 0002:00037f74       $chain$8$?setup_topographical_masks@@YAXPEBUhb_ot_shape_plan_t@@PEAUhb_buffer_t@@@Z 00000001800c2f74     hb-ot-shaper-use.obj
 0002:00037f90       $chain$9$?setup_topographical_masks@@YAXPEBUhb_ot_shape_plan_t@@PEAUhb_buffer_t@@@Z 00000001800c2f90     hb-ot-shaper-use.obj
 0002:00037fa8       $chain$11$?setup_topographical_masks@@YAXPEBUhb_ot_shape_plan_t@@PEAUhb_buffer_t@@@Z 00000001800c2fa8     hb-ot-shaper-use.obj
 0002:00037fb8       $unwind$?reorder_syllable_use@@YAXPEAUhb_buffer_t@@II@Z 00000001800c2fb8     hb-ot-shaper-use.obj
 0002:00037fc8       $chain$1$?reorder_syllable_use@@YAXPEAUhb_buffer_t@@II@Z 00000001800c2fc8     hb-ot-shaper-use.obj
 0002:00037fe0       $chain$2$?reorder_syllable_use@@YAXPEAUhb_buffer_t@@II@Z 00000001800c2fe0     hb-ot-shaper-use.obj
 0002:00037ff4       $chain$3$?reorder_syllable_use@@YAXPEAUhb_buffer_t@@II@Z 00000001800c2ff4     hb-ot-shaper-use.obj
 0002:00037ff4       $chain$5$?reorder_syllable_use@@YAXPEAUhb_buffer_t@@II@Z 00000001800c2ff4     hb-ot-shaper-use.obj
 0002:00038004       $chain$4$?reorder_syllable_use@@YAXPEAUhb_buffer_t@@II@Z 00000001800c3004     hb-ot-shaper-use.obj
 0002:00038018       $chain$6$?reorder_syllable_use@@YAXPEAUhb_buffer_t@@II@Z 00000001800c3018     hb-ot-shaper-use.obj
 0002:00038028       $chain$2$?_hb_preprocess_text_vowel_constraints@@YAXPEBUhb_ot_shape_plan_t@@PEAUhb_buffer_t@@PEAUhb_font_t@@@Z 00000001800c3028     hb-ot-shaper-vowel-constraints.obj
 0002:00038044       $chain$3$?_hb_preprocess_text_vowel_constraints@@YAXPEBUhb_ot_shape_plan_t@@PEAUhb_buffer_t@@PEAUhb_font_t@@@Z 00000001800c3044     hb-ot-shaper-vowel-constraints.obj
 0002:00038054       $unwind$hb_ot_tags_from_script_and_language 00000001800c3054     hb-ot-tag.obj
 0002:00038064       $chain$3$hb_ot_tags_from_script_and_language 00000001800c3064     hb-ot-tag.obj
 0002:00038084       $chain$4$hb_ot_tags_from_script_and_language 00000001800c3084     hb-ot-tag.obj
 0002:00038084       $chain$6$hb_ot_tags_from_script_and_language 00000001800c3084     hb-ot-tag.obj
 0002:00038094       $chain$5$hb_ot_tags_from_script_and_language 00000001800c3094     hb-ot-tag.obj
 0002:000380b4       $unwind$hb_ot_tag_to_language 00000001800c30b4     hb-ot-tag.obj
 0002:000380c4       $unwind$?hb_ot_tags_from_complex_language@@YA_NPEBD0PEAI1@Z 00000001800c30c4     hb-ot-tag.obj
 0002:000380d8       $chain$0$?hb_ot_tags_from_complex_language@@YA_NPEBD0PEAI1@Z 00000001800c30d8     hb-ot-tag.obj
 0002:000380ec       $chain$2$?hb_ot_tags_from_complex_language@@YA_NPEBD0PEAI1@Z 00000001800c30ec     hb-ot-tag.obj
 0002:00038100       $unwind$?hb_ot_tags_from_language@@YAXPEBD0PEAI1@Z 00000001800c3100     hb-ot-tag.obj
 0002:00038110       $chain$3$?hb_ot_tags_from_language@@YAXPEBD0PEAI1@Z 00000001800c3110     hb-ot-tag.obj
 0002:00038130       $chain$4$?hb_ot_tags_from_language@@YAXPEBD0PEAI1@Z 00000001800c3130     hb-ot-tag.obj
 0002:00038140       $unwind$hb_ot_var_normalize_coords 00000001800c3140     hb-ot-var.obj
 0002:00038158       $chain$4$hb_ot_var_normalize_coords 00000001800c3158     hb-ot-var.obj
 0002:0003817c       $chain$5$hb_ot_var_normalize_coords 00000001800c317c     hb-ot-var.obj
 0002:0003818c       $unwind$?replay@hb_outline_t@@QEBAXPEAUhb_draw_funcs_t@@PEAX@Z 00000001800c318c     hb-outline.obj
 0002:000381a4       $chain$5$?replay@hb_outline_t@@QEBAXPEAUhb_draw_funcs_t@@PEAX@Z 00000001800c31a4     hb-outline.obj
 0002:000381cc       $chain$6$?replay@hb_outline_t@@QEBAXPEAUhb_draw_funcs_t@@PEAX@Z 00000001800c31cc     hb-outline.obj
 0002:000381dc       $unwind$?control_area@hb_outline_t@@QEBAMXZ 00000001800c31dc     hb-outline.obj
 0002:000381e8       $chain$4$?control_area@hb_outline_t@@QEBAMXZ 00000001800c31e8     hb-outline.obj
 0002:0003820c       $chain$5$?control_area@hb_outline_t@@QEBAMXZ 00000001800c320c     hb-outline.obj
 0002:0003821c       $unwind$?embolden@hb_outline_t@@QEAAXMMMM@Z 00000001800c321c     hb-outline.obj
 0002:00038230       $chain$1$?embolden@hb_outline_t@@QEAAXMMMM@Z 00000001800c3230     hb-outline.obj
 0002:00038248       $chain$14$?embolden@hb_outline_t@@QEAAXMMMM@Z 00000001800c3248     hb-outline.obj
 0002:0003828c       $chain$15$?embolden@hb_outline_t@@QEAAXMMMM@Z 00000001800c328c     hb-outline.obj
 0002:0003829c       $chain$16$?embolden@hb_outline_t@@QEAAXMMMM@Z 00000001800c329c     hb-outline.obj
 0002:000382ac       $chain$0$?hb_outline_recording_pen_get_funcs@@YAPEAUhb_draw_funcs_t@@XZ 00000001800c32ac     hb-outline.obj
 0002:000382c0       $chain$2$?hb_outline_recording_pen_get_funcs@@YAPEAUhb_draw_funcs_t@@XZ 00000001800c32c0     hb-outline.obj
 0002:000382d4       $chain$3$?hb_outline_recording_pen_get_funcs@@YAPEAUhb_draw_funcs_t@@XZ 00000001800c32d4     hb-outline.obj
 0002:000382e4       $unwind$?transform_extents@hb_transform_t@@QEBAXAEAUhb_extents_t@@@Z 00000001800c32e4     hb-paint-extents.obj
 0002:000382fc       $unwind$?push_transform@hb_paint_extents_context_t@@QEAAXAEBUhb_transform_t@@@Z 00000001800c32fc     hb-paint-extents.obj
 0002:00038338       $chain$0$?hb_paint_extents_get_funcs@@YAPEAUhb_paint_funcs_t@@XZ 00000001800c3338     hb-paint-extents.obj
 0002:0003834c       $chain$2$?hb_paint_extents_get_funcs@@YAPEAUhb_paint_funcs_t@@XZ 00000001800c334c     hb-paint-extents.obj
 0002:00038360       $chain$3$?hb_paint_extents_get_funcs@@YAPEAUhb_paint_funcs_t@@XZ 00000001800c3360     hb-paint-extents.obj
 0002:00038370       $unwind$?hb_paint_extents_push_transform@@YAXPEAUhb_paint_funcs_t@@PEAXMMMMMM1@Z 00000001800c3370     hb-paint-extents.obj
 0002:00038378       $unwind$?hb_paint_extents_push_clip_glyph@@YAXPEAUhb_paint_funcs_t@@PEAXIPEAUhb_font_t@@1@Z 00000001800c3378     hb-paint-extents.obj
 0002:0003838c       $chain$1$hb_paint_funcs_destroy 00000001800c338c     hb-paint.obj
 0002:000383a4       $chain$2$hb_paint_funcs_destroy 00000001800c33a4     hb-paint.obj
 0002:000383b8       $chain$3$hb_paint_funcs_destroy 00000001800c33b8     hb-paint.obj
 0002:000383c8       $chain$0$hb_paint_funcs_set_push_transform_func 00000001800c33c8     hb-paint.obj
 0002:000383dc       $chain$1$hb_paint_funcs_set_push_transform_func 00000001800c33dc     hb-paint.obj
 0002:000383ec       $chain$0$hb_paint_funcs_set_pop_transform_func 00000001800c33ec     hb-paint.obj
 0002:00038400       $chain$1$hb_paint_funcs_set_pop_transform_func 00000001800c3400     hb-paint.obj
 0002:00038410       $chain$0$hb_paint_funcs_set_push_clip_glyph_func 00000001800c3410     hb-paint.obj
 0002:00038424       $chain$1$hb_paint_funcs_set_push_clip_glyph_func 00000001800c3424     hb-paint.obj
 0002:00038434       $chain$0$hb_paint_funcs_set_push_clip_rectangle_func 00000001800c3434     hb-paint.obj
 0002:00038448       $chain$1$hb_paint_funcs_set_push_clip_rectangle_func 00000001800c3448     hb-paint.obj
 0002:00038458       $chain$0$hb_paint_funcs_set_pop_clip_func 00000001800c3458     hb-paint.obj
 0002:0003846c       $chain$1$hb_paint_funcs_set_pop_clip_func 00000001800c346c     hb-paint.obj
 0002:0003847c       $chain$0$hb_paint_funcs_set_color_func 00000001800c347c     hb-paint.obj
 0002:00038490       $chain$1$hb_paint_funcs_set_color_func 00000001800c3490     hb-paint.obj
 0002:000384a0       $chain$0$hb_paint_funcs_set_image_func 00000001800c34a0     hb-paint.obj
 0002:000384b4       $chain$1$hb_paint_funcs_set_image_func 00000001800c34b4     hb-paint.obj
 0002:000384c4       $chain$0$hb_paint_funcs_set_linear_gradient_func 00000001800c34c4     hb-paint.obj
 0002:000384d8       $chain$1$hb_paint_funcs_set_linear_gradient_func 00000001800c34d8     hb-paint.obj
 0002:000384e8       $chain$0$hb_paint_funcs_set_radial_gradient_func 00000001800c34e8     hb-paint.obj
 0002:000384fc       $chain$1$hb_paint_funcs_set_radial_gradient_func 00000001800c34fc     hb-paint.obj
 0002:0003850c       $chain$0$hb_paint_funcs_set_sweep_gradient_func 00000001800c350c     hb-paint.obj
 0002:00038520       $chain$1$hb_paint_funcs_set_sweep_gradient_func 00000001800c3520     hb-paint.obj
 0002:00038530       $chain$0$hb_paint_funcs_set_push_group_func 00000001800c3530     hb-paint.obj
 0002:00038544       $chain$1$hb_paint_funcs_set_push_group_func 00000001800c3544     hb-paint.obj
 0002:00038554       $chain$0$hb_paint_funcs_set_pop_group_func 00000001800c3554     hb-paint.obj
 0002:00038568       $chain$1$hb_paint_funcs_set_pop_group_func 00000001800c3568     hb-paint.obj
 0002:00038578       $unwind$hb_shape_plan_create2 00000001800c3578     hb-shape-plan.obj
 0002:00038590       $chain$0$hb_shape_plan_create2 00000001800c3590     hb-shape-plan.obj
 0002:000385a4       $chain$1$hb_shape_plan_create2 00000001800c35a4     hb-shape-plan.obj
 0002:000385b4       $chain$2$hb_shape_plan_create2 00000001800c35b4     hb-shape-plan.obj
 0002:000385c8       $unwind$hb_shape_plan_create_cached2 00000001800c35c8     hb-shape-plan.obj
 0002:000385e8       $chain$0$hb_shape_plan_destroy 00000001800c35e8     hb-shape-plan.obj
 0002:000385fc       $chain$1$hb_shape_plan_destroy 00000001800c35fc     hb-shape-plan.obj
 0002:0003860c       $unwind$?init@hb_shape_plan_key_t@@QEAA_N_NPEAUhb_face_t@@PEBUhb_segment_properties_t@@PEBUhb_feature_t@@IPEBHIPEBQEBD@Z 00000001800c360c     hb-shape-plan.obj
 0002:00038624       $chain$0$?init@hb_shape_plan_key_t@@QEAA_N_NPEAUhb_face_t@@PEBUhb_segment_properties_t@@PEBUhb_feature_t@@IPEBHIPEBQEBD@Z 00000001800c3624     hb-shape-plan.obj
 0002:00038638       $chain$1$?init@hb_shape_plan_key_t@@QEAA_N_NPEAUhb_face_t@@PEBUhb_segment_properties_t@@PEBUhb_feature_t@@IPEBHIPEBQEBD@Z 00000001800c3638     hb-shape-plan.obj
 0002:00038648       $unwind$?_hb_shape_plan_execute_internal@@YA_NPEAUhb_shape_plan_t@@PEAUhb_font_t@@PEAUhb_buffer_t@@PEBUhb_feature_t@@I@Z 00000001800c3648     hb-shape-plan.obj
 0002:0003865c       $unwind$hb_shape_full      00000001800c365c     hb-shape.obj
 0002:00038674       $chain$3$hb_shape_full     00000001800c3674     hb-shape.obj
 0002:0003868c       $chain$4$hb_shape_full     00000001800c368c     hb-shape.obj
 0002:000386a0       $unwind$?get_stored@?$hb_lazy_loader_t@Uhb_shaper_entry_t@@Uhb_shapers_lazy_loader_t@@X$0A@U1@@@QEBAPEAUhb_shaper_entry_t@@XZ 00000001800c36a0     hb-shaper.obj
 0002:000386a8       $chain$6$?get_stored@?$hb_lazy_loader_t@Uhb_shaper_entry_t@@Uhb_shapers_lazy_loader_t@@X$0A@U1@@@QEBAPEAUhb_shaper_entry_t@@XZ 00000001800c36a8     hb-shaper.obj
 0002:000386d4       $chain$7$?get_stored@?$hb_lazy_loader_t@Uhb_shaper_entry_t@@Uhb_shapers_lazy_loader_t@@X$0A@U1@@@QEBAPEAUhb_shaper_entry_t@@XZ 00000001800c36d4     hb-shaper.obj
 0002:000386e4       $chain$0$hb_ucd_get_unicode_funcs 00000001800c36e4     hb-ucd.obj
 0002:000386f8       $chain$2$hb_ucd_get_unicode_funcs 00000001800c36f8     hb-ucd.obj
 0002:0003870c       $chain$3$hb_ucd_get_unicode_funcs 00000001800c370c     hb-ucd.obj
 0002:0003871c       $chain$1$?hb_ucd_compose@@YAHPEAUhb_unicode_funcs_t@@IIPEAIPEAX@Z 00000001800c371c     hb-ucd.obj
 0002:00038734       $chain$3$?hb_ucd_compose@@YAHPEAUhb_unicode_funcs_t@@IIPEAIPEAX@Z 00000001800c3734     hb-ucd.obj
 0002:00038734       $chain$5$?hb_ucd_compose@@YAHPEAUhb_unicode_funcs_t@@IIPEAIPEAX@Z 00000001800c3734     hb-ucd.obj
 0002:0003874c       $chain$0$hb_unicode_funcs_destroy 00000001800c374c     hb-unicode.obj
 0002:00038760       $chain$1$hb_unicode_funcs_destroy 00000001800c3760     hb-unicode.obj
 0002:00038770       $unwind$Java_sun_font_FileFontStrike__1getGlyphImageFromWindows 00000001800c3770     lcdglyph.obj
 0002:0003879c       $chain$0$Java_sun_font_StrikeCache_getGlyphCacheDescription 00000001800c379c     sunFont.obj
 0002:000387b0       $chain$2$Java_sun_font_StrikeCache_getGlyphCacheDescription 00000001800c37b0     sunFont.obj
 0002:000387c4       $chain$3$Java_sun_font_StrikeCache_getGlyphCacheDescription 00000001800c37c4     sunFont.obj
 0002:000387d4       $unwind$Java_sun_font_StrikeCache_freeIntMemory 00000001800c37d4     sunFont.obj
 0002:000387d4       $unwind$Java_sun_font_StrikeCache_freeLongMemory 00000001800c37d4     sunFont.obj
 0002:000387d4       $unwind$?filt$0@?0??dllmain_dispatch@@YAHQEAUHINSTANCE__@@KQEAX@Z@4HA 00000001800c37d4     MSVCRT:dll_dllmain.obj
 0002:000387dc       $chain$3$Java_sun_font_StrikeCache_freeIntMemory 00000001800c37dc     sunFont.obj
 0002:000387fc       $chain$4$Java_sun_font_StrikeCache_freeIntMemory 00000001800c37fc     sunFont.obj
 0002:00038810       $chain$5$Java_sun_font_StrikeCache_freeIntMemory 00000001800c3810     sunFont.obj
 0002:00038824       $chain$6$Java_sun_font_StrikeCache_freeIntMemory 00000001800c3824     sunFont.obj
 0002:00038834       $chain$7$Java_sun_font_StrikeCache_freeIntMemory 00000001800c3834     sunFont.obj
 0002:00038844       $chain$8$Java_sun_font_StrikeCache_freeIntMemory 00000001800c3844     sunFont.obj
 0002:00038854       $chain$3$Java_sun_font_StrikeCache_freeLongMemory 00000001800c3854     sunFont.obj
 0002:00038874       $chain$4$Java_sun_font_StrikeCache_freeLongMemory 00000001800c3874     sunFont.obj
 0002:00038888       $chain$5$Java_sun_font_StrikeCache_freeLongMemory 00000001800c3888     sunFont.obj
 0002:0003889c       $chain$6$Java_sun_font_StrikeCache_freeLongMemory 00000001800c389c     sunFont.obj
 0002:000388ac       $chain$7$Java_sun_font_StrikeCache_freeLongMemory 00000001800c38ac     sunFont.obj
 0002:000388bc       $chain$8$Java_sun_font_StrikeCache_freeLongMemory 00000001800c38bc     sunFont.obj
 0002:000388cc       $chain$0$initFontIDs       00000001800c38cc     sunFont.obj
 0002:000388e0       $chain$1$initFontIDs       00000001800c38e0     sunFont.obj
 0002:000388f0       $xdatasym                  00000001800c38f0     MSVCRT:amdsecgs.obj
 0002:000388f4       $unwind$__report_securityfailure 00000001800c38f4     MSVCRT:gs_report.obj
 0002:000388fc       $unwind$__report_gsfailure 00000001800c38fc     MSVCRT:gs_report.obj
 0002:00038904       $unwind$capture_current_context 00000001800c3904     MSVCRT:gs_report.obj
 0002:00038910       $xdatasym                  00000001800c3910     MSVCRT:chkstk.obj
 0002:00038918       $unwind$?dllmain_crt_process_attach@@YAHQEAUHINSTANCE__@@QEAX@Z 00000001800c3918     MSVCRT:dll_dllmain.obj
 0002:00038954       $unwind$?fin$0@?0??dllmain_crt_process_attach@@YAHQEAUHINSTANCE__@@QEAX@Z@4HA 00000001800c3954     MSVCRT:dll_dllmain.obj
 0002:00038954       $unwind$?fin$0@?0??dllmain_crt_process_detach@@YAH_N@Z@4HA 00000001800c3954     MSVCRT:dll_dllmain.obj
 0002:00038954       $unwind$?fin$1@?0??dllmain_crt_process_detach@@YAH_N@Z@4HA 00000001800c3954     MSVCRT:dll_dllmain.obj
 0002:0003895c       $unwind$?dllmain_crt_process_detach@@YAH_N@Z 00000001800c395c     MSVCRT:dll_dllmain.obj
 0002:000389b0       $unwind$?dllmain_dispatch@@YAHQEAUHINSTANCE__@@KQEAX@Z 00000001800c39b0     MSVCRT:dll_dllmain.obj
 0002:000389d8       $unwind$__isa_available_init 00000001800c39d8     MSVCRT:cpu_disp.obj
 0002:000389e8       $unwind$__security_init_cookie 00000001800c39e8     MSVCRT:gs_support.obj
 0002:000389f4       $unwind$__scrt_is_nonwritable_in_current_image 00000001800c39f4     MSVCRT:utility.obj
 0002:00038a14       $unwind$__scrt_fastfail    00000001800c3a14     MSVCRT:utility_desktop.obj
 0002:00038a28       $xdatasym                  00000001800c3a28     MSVCRT:guard_dispatch.obj
 0002:00038a30       $xdatasym                  00000001800c3a30     MSVCRT:guard_xfg_dispatch.obj
 0002:00038a40       .edata                     00000001800c3a40     fontmanager.exp
 0002:00038a68       rgpv                       00000001800c3a68     fontmanager.exp
 0002:00038b00       rgszName                   00000001800c3b00     fontmanager.exp
 0002:00038b98       rgwOrd                     00000001800c3b98     fontmanager.exp
 0002:00038be4       szName                     00000001800c3be4     fontmanager.exp
 0002:00038bf4       $N00001                    00000001800c3bf4     fontmanager.exp
 0002:00038c1e       $N00002                    00000001800c3c1e     fontmanager.exp
 0002:00038c55       $N00003                    00000001800c3c55     fontmanager.exp
 0002:00038c81       $N00004                    00000001800c3c81     fontmanager.exp
 0002:00038cb5       $N00005                    00000001800c3cb5     fontmanager.exp
 0002:00038ced       $N00006                    00000001800c3ced     fontmanager.exp
 0002:00038d15       $N00007                    00000001800c3d15     fontmanager.exp
 0002:00038d50       $N00008                    00000001800c3d50     fontmanager.exp
 0002:00038d85       $N00009                    00000001800c3d85     fontmanager.exp
 0002:00038dbb       $N00010                    00000001800c3dbb     fontmanager.exp
 0002:00038df2       $N00011                    00000001800c3df2     fontmanager.exp
 0002:00038e26       $N00012                    00000001800c3e26     fontmanager.exp
 0002:00038e5b       $N00013                    00000001800c3e5b     fontmanager.exp
 0002:00038e92       $N00014                    00000001800c3e92     fontmanager.exp
 0002:00038ecf       $N00015                    00000001800c3ecf     fontmanager.exp
 0002:00038f06       $N00016                    00000001800c3f06     fontmanager.exp
 0002:00038f3b       $N00017                    00000001800c3f3b     fontmanager.exp
 0002:00038f78       $N00018                    00000001800c3f78     fontmanager.exp
 0002:00038fb3       $N00019                    00000001800c3fb3     fontmanager.exp
 0002:00038fe7       $N00020                    00000001800c3fe7     fontmanager.exp
 0002:0003901c       $N00021                    00000001800c401c     fontmanager.exp
 0002:00039045       $N00022                    00000001800c4045     fontmanager.exp
 0002:00039077       $N00023                    00000001800c4077     fontmanager.exp
 0002:000390a2       $N00024                    00000001800c40a2     fontmanager.exp
 0002:000390d4       $N00025                    00000001800c40d4     fontmanager.exp
 0002:000390fc       $N00026                    00000001800c40fc     fontmanager.exp
 0002:00039125       $N00027                    00000001800c4125     fontmanager.exp
 0002:0003914e       $N00028                    00000001800c414e     fontmanager.exp
 0002:00039178       $N00029                    00000001800c4178     fontmanager.exp
 0002:000391ab       $N00030                    00000001800c41ab     fontmanager.exp
 0002:000391d0       $N00031                    00000001800c41d0     fontmanager.exp
 0002:000391f9       $N00032                    00000001800c41f9     fontmanager.exp
 0002:00039223       $N00033                    00000001800c4223     fontmanager.exp
 0002:00039247       $N00034                    00000001800c4247     fontmanager.exp
 0002:0003927d       $N00035                    00000001800c427d     fontmanager.exp
 0002:000392b5       $N00036                    00000001800c42b5     fontmanager.exp
 0002:000392e7       $N00037                    00000001800c42e7     fontmanager.exp
 0002:000392f5       $N00038                    00000001800c42f5     fontmanager.exp
 0002:00039a40       .idata$6                   00000001800c4a40     freetype:freetype.dll
 0002:00039ae4       .idata$6                   00000001800c4ae4     java:java.dll
 0002:00039b30       .idata$6                   00000001800c4b30     advapi32:ADVAPI32.dll
 0002:00039b98       .idata$6                   00000001800c4b98     user32:USER32.dll
 0002:00039cbc       .idata$6                   00000001800c4cbc     gdi32:GDI32.dll
 0002:00039dc2       .idata$6                   00000001800c4dc2     awt:awt.dll
 0002:00039fc2       .idata$6                   00000001800c4fc2     kernel32:KERNEL32.dll
 0002:0003a062       .idata$6                   00000001800c5062     vcruntime:VCRUNTIME140.dll
 0002:0003a224       .idata$6                   00000001800c5224     ucrt:api-ms-win-crt-heap-l1-1-0.dll
 0002:0003a244       .idata$6                   00000001800c5244     ucrt:api-ms-win-crt-math-l1-1-0.dll
 0002:0003a264       .idata$6                   00000001800c5264     ucrt:api-ms-win-crt-environment-l1-1-0.dll
 0002:0003a28a       .idata$6                   00000001800c528a     ucrt:api-ms-win-crt-convert-l1-1-0.dll
 0002:0003a2ac       .idata$6                   00000001800c52ac     ucrt:api-ms-win-crt-stdio-l1-1-0.dll
 0002:0003a2cc       .idata$6                   00000001800c52cc     ucrt:api-ms-win-crt-string-l1-1-0.dll
 0002:0003a2ee       .idata$6                   00000001800c52ee     ucrt:api-ms-win-crt-runtime-l1-1-0.dll
 0003:00000200       gvdClassName               00000001800c6200     HBShaper.obj
 0003:00000208       ?PADBYTES@?1??getGlyphImageNativeInternal@@9@9 00000001800c6208     freetypeScaler.obj
 0003:00000210       ?_hb_buffer_serialize_formats@@3PAPEBDA 00000001800c6210     hb-buffer-serialize.obj
 0003:00000680       ?_hb_draw_funcs_default@@3Uhb_draw_funcs_t@@B 00000001800c6680     hb-font.obj
 0003:000006d0       ?_hb_font_funcs_default@@3Uhb_font_funcs_t@@B 00000001800c66d0     hb-font.obj
 0003:00000788       ?modifier_combining_marks@@3PAIA 00000001800c6788     hb-ot-shaper-arabic.obj
 0003:000007c0       ?thai_above_start_state@@3PAW4thai_above_state_t@@A 00000001800c67c0     hb-ot-shaper-thai.obj
 0003:000007d8       ?thai_below_start_state@@3PAW4thai_below_state_t@@A 00000001800c67d8     hb-ot-shaper-thai.obj
 0003:00000880       ?known_tables@@3PAIA       00000001800c6880     hb-subset.obj
 0003:00000b60       gvdClass                   00000001800c6b60     HBShaper.obj
 0003:00000b68       gvdCountFID                00000001800c6b68     HBShaper.obj
 0003:00000b70       gvdFlagsFID                00000001800c6b70     HBShaper.obj
 0003:00000b78       gvdGlyphsFID               00000001800c6b78     HBShaper.obj
 0003:00000b80       gvdPositionsFID            00000001800c6b80     HBShaper.obj
 0003:00000b88       gvdIndicesFID              00000001800c6b88     HBShaper.obj
 0003:00000b90       gvdGrowMID                 00000001800c6b90     HBShaper.obj
 0003:00000b98       jniInited                  00000001800c6b98     HBShaper.obj
 0003:00000ba0       screenDC                   00000001800c6ba0     fontpath.obj
 0003:00000ba8       invalidateScalerMID        00000001800c6ba8     freetypeScaler.obj
 0003:00000bb0       debugFonts                 00000001800c6bb0     freetypeScaler.obj
 0003:00000d88       ?langs@@3U?$hb_atomic_ptr_t@Uhb_language_item_t@@@@A 00000001800c6d88     hb-common.obj
 0003:00000d90       ?jdk_ffuncs@?1??_hb_jdk_get_font_funcs@@YAPEAUhb_font_funcs_t@@XZ@4PEAU2@EA 00000001800c6d90     hb-jdk-font.obj
 0003:00000d98       ?hb_ot_font_cmap_cache_user_data_key@@3Uhb_user_data_key_t@@A 00000001800c6d98     hb-ot-font.obj
 0003:00000da0       ?static_ot_funcs@@3Uhb_ot_font_funcs_lazy_loader_t@@A 00000001800c6da0     hb-ot-font.obj
 0003:00000da8       ?last_tag_idx@?4??hb_ot_tags_from_language@@YAXPEBD0PEAI1@Z@4Uhb_atomic_int_t@@A 00000001800c6da8     hb-ot-tag.obj
 0003:00000db0       ?static_outline_recording_pen_funcs@@3Uhb_outline_recording_pen_funcs_lazy_loader_t@@A 00000001800c6db0     hb-outline.obj
 0003:00000db8       ?static_draw_extents_funcs@@3Uhb_draw_extents_funcs_lazy_loader_t@@A 00000001800c6db8     hb-paint-extents.obj
 0003:00000dc0       ?static_paint_extents_funcs@@3Uhb_paint_extents_funcs_lazy_loader_t@@A 00000001800c6dc0     hb-paint-extents.obj
 0003:00000dc8       ?static_shaper_list@@3Uhb_shaper_list_lazy_loader_t@@A 00000001800c6dc8     hb-shape.obj
 0003:00000dd0       ?static_shapers@@3Uhb_shapers_lazy_loader_t@@A 00000001800c6dd0     hb-shaper.obj
 0003:00000de0       ?static_ucd_funcs@@3Uhb_ucd_unicode_funcs_lazy_loader_t@@A 00000001800c6de0     hb-ucd.obj
 0003:00000df0       igLUTable                  00000001800c6df0     lcdglyph.obj
 0003:000011b8       theNullScalerContext       00000001800c71b8     sunFont.obj
 0003:000011c0       initialisedFontIDs         00000001800c71c0     sunFont.obj
 0003:000011d0       GS_ExceptionRecord         00000001800c71d0     MSVCRT:gs_report.obj
 0003:00001270       GS_ContextRecord           00000001800c7270     MSVCRT:gs_report.obj
 0003:00001740       ?__proc_attached@@3HA      00000001800c7740     MSVCRT:dll_dllmain.obj
 0003:00001778       ?is_initialized_as_dll@@3_NA 00000001800c7778     MSVCRT:utility.obj
 0003:00001779       ?module_local_atexit_table_initialized@@3_NA 00000001800c7779     MSVCRT:utility.obj
 0003:00001780       ?module_local_atexit_table@@3U_onexit_table_t@@A 00000001800c7780     MSVCRT:utility.obj
 0003:00001798       ?module_local_at_quick_exit_table@@3U_onexit_table_t@@A 00000001800c7798     MSVCRT:utility.obj
 0005:00000000       _2il0floatpacket$0         00000001800d0000     MSVCRT:svml_sfloorf4_sse2.obj
 0005:00000010       _2il0floatpacket$1         00000001800d0010     MSVCRT:svml_sfloorf4_sse2.obj
 0005:00000020       _2il0floatpacket$2         00000001800d0020     MSVCRT:svml_sfloorf4_sse2.obj
 0006:00000060       $R000000                   00000001800d1060     fontmanager.dll.res
